 quake3

 Timestamp is 4839b8eb (Sun May 25 23:07:23 2008)

 Preferred load address is 00400000

 Start         Length     Name                   Class
 0001:00000000 000baac8H .text                   CODE
 0002:00000000 000002e0H .idata$5                DATA
 0002:000002e0 0001a940H .rdata                  DATA
 0002:0001ac20 00000050H .rdata$debug            DATA
 0002:0001ac70 00000008H .rdata$sxdata           DATA
 0002:0001ac78 00000004H .rtc$IAA                DATA
 0002:0001ac7c 00000004H .rtc$IZZ                DATA
 0002:0001ac80 00000004H .rtc$TAA                DATA
 0002:0001ac84 00000004H .rtc$TZZ                DATA
 0002:0001ac88 0000008cH .idata$2                DATA
 0002:0001ad14 00000014H .idata$3                DATA
 0002:0001ad28 000002e0H .idata$4                DATA
 0002:0001b008 00000b20H .idata$6                DATA
 0002:0001bb28 00000000H .edata                  DATA
 0003:00000000 00000004H .CRT$XCA                DATA
 0003:00000004 00000004H .CRT$XCAA               DATA
 0003:00000008 00000004H .CRT$XCZ                DATA
 0003:0000000c 00000004H .CRT$XIA                DATA
 0003:00000010 00000014H .CRT$XIC                DATA
 0003:00000024 00000004H .CRT$XIZ                DATA
 0003:00000028 00000004H .CRT$XPA                DATA
 0003:0000002c 00000004H .CRT$XPX                DATA
 0003:00000030 00000004H .CRT$XPZ                DATA
 0003:00000034 00000004H .CRT$XTA                DATA
 0003:00000038 00000004H .CRT$XTZ                DATA
 0003:00000040 000050fcH .data                   DATA
 0003:00005140 00790b24H .bss                    DATA
 0004:00000000 000000e8H .rsrc$01                DATA
 0004:000000f0 00000330H .rsrc$02                DATA

  Address         Publics by Value              Rva+Base     Lib:Object

 0000:00000000       __except_list              00000000     <absolute>
 0000:00000002       ___safe_se_handler_count   00000002     <absolute>
 0001:00000000       _CL_GetGameState           00401000 f   cl_cgame.obj
 0001:00000020       _CL_GetGlconfig            00401020 f   cl_cgame.obj
 0001:00000040       _CL_GetUserCmd             00401040 f   cl_cgame.obj
 0001:000000b0       _CL_GetCurrentCmdNumber    004010b0 f   cl_cgame.obj
 0001:000000c0       _CL_GetParseEntityState    004010c0 f   cl_cgame.obj
 0001:00000120       _CL_GetCurrentSnapshotNumber 00401120 f   cl_cgame.obj
 0001:00000140       _CL_GetSnapshot            00401140 f   cl_cgame.obj
 0001:00000250       _CL_SetUserCmdValue        00401250 f   cl_cgame.obj
 0001:00000270       _CL_AddCgameCommand        00401270 f   cl_cgame.obj
 0001:00000280       _CL_CgameError             00401280 f   cl_cgame.obj
 0001:000002a0       _CL_ConfigstringModified   004012a0 f   cl_cgame.obj
 0001:00000400       _CL_GetServerCommand       00401400 f   cl_cgame.obj
 0001:00000700       _CL_CM_LoadMap             00401700 f   cl_cgame.obj
 0001:00000720       _CL_ShutdownCGame          00401720 f   cl_cgame.obj
 0001:00000780       _CL_CgameSystemCalls       00401780 f   cl_cgame.obj
 0001:00001540       _CL_InitCGame              00402540 f   cl_cgame.obj
 0001:00001650       _CL_GameCommand            00402650 f   cl_cgame.obj
 0001:00001670       _CL_CGameRendering         00402670 f   cl_cgame.obj
 0001:000016a0       _CL_AdjustTimeDelta        004026a0 f   cl_cgame.obj
 0001:000017b0       _CL_FirstSnapshot          004027b0 f   cl_cgame.obj
 0001:00001810       _CL_SetCGameTime           00402810 f   cl_cgame.obj
 0001:00001a80       _RllDecodeMonoToMono       00402a80 f   cl_cin.obj
 0001:00001ad0       _RllDecodeMonoToStereo     00402ad0 f   cl_cin.obj
 0001:00001b30       _RllDecodeStereoToStereo   00402b30 f   cl_cin.obj
 0001:00001bd0       _RllDecodeStereoToMono     00402bd0 f   cl_cin.obj
 0001:000037e0       _CIN_StopCinematic         004047e0 f   cl_cin.obj
 0001:00003860       _CIN_SetExtents            00404860 f   cl_cin.obj
 0001:000038b0       _CIN_SetLooping            004048b0 f   cl_cin.obj
 0001:000038e0       _CIN_DrawCinematic         004048e0 f   cl_cin.obj
 0001:00003bf0       _SCR_DrawCinematic         00404bf0 f   cl_cin.obj
 0001:00003c10       _SCR_StopCinematic         00404c10 f   cl_cin.obj
 0001:00003c40       _CIN_UploadCinematic       00404c40 f   cl_cin.obj
 0001:00003d00       _CIN_CloseAllVideos        00404d00 f   cl_cin.obj
 0001:00004290       _CIN_RunCinematic          00405290 f   cl_cin.obj
 0001:000044c0       _CIN_PlayCinematic         004054c0 f   cl_cin.obj
 0001:00004880       _SCR_RunCinematic          00405880 f   cl_cin.obj
 0001:000048a0       _CL_PlayCinematic_f        004058a0 f   cl_cin.obj
 0001:000049a0       _Con_MessageMode_f         004059a0 f   cl_console.obj
 0001:000049e0       _Con_MessageMode2_f        004059e0 f   cl_console.obj
 0001:00004a20       _Con_MessageMode3_f        00405a20 f   cl_console.obj
 0001:00004a80       _Con_MessageMode4_f        00405a80 f   cl_console.obj
 0001:00004ae0       _Con_Dump_f                00405ae0 f   cl_console.obj
 0001:00004c40       _Con_ClearNotify           00405c40 f   cl_console.obj
 0001:00004c60       _Con_CheckResize           00405c60 f   cl_console.obj
 0001:00004d60       _Con_Linefeed              00405d60 f   cl_console.obj
 0001:00004e00       _CL_ConsolePrint           00405e00 f   cl_console.obj
 0001:00004fc0       _Con_DrawInput             00405fc0 f   cl_console.obj
 0001:00005030       _Con_DrawNotify            00406030 f   cl_console.obj
 0001:000051f0       _Con_DrawSolidConsole      004061f0 f   cl_console.obj
 0001:00005510       _Con_DrawConsole           00406510 f   cl_console.obj
 0001:00005570       _Con_RunConsole            00406570 f   cl_console.obj
 0001:00005640       _Con_PageUp                00406640 f   cl_console.obj
 0001:00005670       _Con_PageDown              00406670 f   cl_console.obj
 0001:00005690       _Con_Top                   00406690 f   cl_console.obj
 0001:000056b0       _Con_Bottom                004066b0 f   cl_console.obj
 0001:000056c0       _Con_Close                 004066c0 f   cl_console.obj
 0001:00005710       _Con_ToggleConsole_f       00406710 f   cl_console.obj
 0001:00005770       _Con_Clear_f               00406770 f   cl_console.obj
 0001:00005790       _Con_Init                  00406790 f   cl_console.obj
 0001:00005870       _IN_MLookDown              00406870 f   cl_input.obj
 0001:00005880       _IN_KeyDown                00406880 f   cl_input.obj
 0001:00005900       _IN_KeyUp                  00406900 f   cl_input.obj
 0001:00005990       _CL_KeyState               00406990 f   cl_input.obj
 0001:00005a20       _IN_UpDown                 00406a20 f   cl_input.obj
 0001:00005a30       _IN_UpUp                   00406a30 f   cl_input.obj
 0001:00005a40       _IN_DownDown               00406a40 f   cl_input.obj
 0001:00005a50       _IN_DownUp                 00406a50 f   cl_input.obj
 0001:00005a60       _IN_LeftDown               00406a60 f   cl_input.obj
 0001:00005a70       _IN_LeftUp                 00406a70 f   cl_input.obj
 0001:00005a80       _IN_RightDown              00406a80 f   cl_input.obj
 0001:00005a90       _IN_RightUp                00406a90 f   cl_input.obj
 0001:00005aa0       _IN_ForwardDown            00406aa0 f   cl_input.obj
 0001:00005ab0       _IN_ForwardUp              00406ab0 f   cl_input.obj
 0001:00005ac0       _IN_BackDown               00406ac0 f   cl_input.obj
 0001:00005ad0       _IN_BackUp                 00406ad0 f   cl_input.obj
 0001:00005ae0       _IN_LookupDown             00406ae0 f   cl_input.obj
 0001:00005af0       _IN_LookupUp               00406af0 f   cl_input.obj
 0001:00005b00       _IN_LookdownDown           00406b00 f   cl_input.obj
 0001:00005b10       _IN_LookdownUp             00406b10 f   cl_input.obj
 0001:00005b20       _IN_MoveleftDown           00406b20 f   cl_input.obj
 0001:00005b30       _IN_MoveleftUp             00406b30 f   cl_input.obj
 0001:00005b40       _IN_MoverightDown          00406b40 f   cl_input.obj
 0001:00005b50       _IN_MoverightUp            00406b50 f   cl_input.obj
 0001:00005b60       _IN_SpeedDown              00406b60 f   cl_input.obj
 0001:00005b70       _IN_SpeedUp                00406b70 f   cl_input.obj
 0001:00005b80       _IN_StrafeDown             00406b80 f   cl_input.obj
 0001:00005b90       _IN_StrafeUp               00406b90 f   cl_input.obj
 0001:00005ba0       _IN_Button0Down            00406ba0 f   cl_input.obj
 0001:00005bb0       _IN_Button0Up              00406bb0 f   cl_input.obj
 0001:00005bc0       _IN_Button1Down            00406bc0 f   cl_input.obj
 0001:00005bd0       _IN_Button1Up              00406bd0 f   cl_input.obj
 0001:00005be0       _IN_Button2Down            00406be0 f   cl_input.obj
 0001:00005bf0       _IN_Button2Up              00406bf0 f   cl_input.obj
 0001:00005c00       _IN_Button3Down            00406c00 f   cl_input.obj
 0001:00005c10       _IN_Button3Up              00406c10 f   cl_input.obj
 0001:00005c20       _IN_Button4Down            00406c20 f   cl_input.obj
 0001:00005c30       _IN_Button4Up              00406c30 f   cl_input.obj
 0001:00005c40       _IN_Button5Down            00406c40 f   cl_input.obj
 0001:00005c50       _IN_Button5Up              00406c50 f   cl_input.obj
 0001:00005c60       _IN_Button6Down            00406c60 f   cl_input.obj
 0001:00005c70       _IN_Button6Up              00406c70 f   cl_input.obj
 0001:00005c80       _IN_Button7Down            00406c80 f   cl_input.obj
 0001:00005c90       _IN_Button7Up              00406c90 f   cl_input.obj
 0001:00005ca0       _IN_Button8Down            00406ca0 f   cl_input.obj
 0001:00005cb0       _IN_Button8Up              00406cb0 f   cl_input.obj
 0001:00005cc0       _IN_Button9Down            00406cc0 f   cl_input.obj
 0001:00005cd0       _IN_Button9Up              00406cd0 f   cl_input.obj
 0001:00005ce0       _IN_Button10Down           00406ce0 f   cl_input.obj
 0001:00005cf0       _IN_Button10Up             00406cf0 f   cl_input.obj
 0001:00005d00       _IN_Button11Down           00406d00 f   cl_input.obj
 0001:00005d10       _IN_Button11Up             00406d10 f   cl_input.obj
 0001:00005d20       _IN_Button12Down           00406d20 f   cl_input.obj
 0001:00005d30       _IN_Button12Up             00406d30 f   cl_input.obj
 0001:00005d40       _IN_Button13Down           00406d40 f   cl_input.obj
 0001:00005d50       _IN_Button13Up             00406d50 f   cl_input.obj
 0001:00005d60       _IN_Button14Down           00406d60 f   cl_input.obj
 0001:00005d70       _IN_Button14Up             00406d70 f   cl_input.obj
 0001:00005d80       _IN_Button15Down           00406d80 f   cl_input.obj
 0001:00005d90       _IN_Button15Up             00406d90 f   cl_input.obj
 0001:00005da0       _IN_ButtonDown             00406da0 f   cl_input.obj
 0001:00005db0       _IN_ButtonUp               00406db0 f   cl_input.obj
 0001:00005dc0       _IN_CenterView             00406dc0 f   cl_input.obj
 0001:00005de0       _CL_AdjustAngles           00406de0 f   cl_input.obj
 0001:00005ea0       _CL_KeyMove                00406ea0 f   cl_input.obj
 0001:00006010       _CL_MouseEvent             00407010 f   cl_input.obj
 0001:00006080       _CL_JoystickEvent          00407080 f   cl_input.obj
 0001:000060c0       _CL_JoystickMove           004070c0 f   cl_input.obj
 0001:000061a0       _CL_MouseMove              004071a0 f   cl_input.obj
 0001:000063b0       _CL_CmdButtons             004073b0 f   cl_input.obj
 0001:00006420       _CL_FinishMove             00407420 f   cl_input.obj
 0001:00006470       _CL_CreateCmd              00407470 f   cl_input.obj
 0001:000065c0       _CL_CreateNewCommands      004075c0 f   cl_input.obj
 0001:00006650       _CL_ReadyToSendPacket      00407650 f   cl_input.obj
 0001:00006760       _CL_WritePacket            00407760 f   cl_input.obj
 0001:00006a30       _CL_SendCmd                00407a30 f   cl_input.obj
 0001:00006a90       _IN_MLookUp                00407a90 f   cl_input.obj
 0001:00006ac0       _CL_InitInput              00407ac0 f   cl_input.obj
 0001:00006e80       _Field_VariableSizeDraw    00407e80 f   cl_keys.obj
 0001:00007030       _Field_Draw                00408030 f   cl_keys.obj
 0001:00007060       _Field_BigDraw             00408060 f   cl_keys.obj
 0001:00007090       _Field_CharEvent           00408090 f   cl_keys.obj
 0001:000071b0       _Key_GetOverstrikeMode     004081b0 f   cl_keys.obj
 0001:000071c0       _Key_SetOverstrikeMode     004081c0 f   cl_keys.obj
 0001:000071d0       _Key_IsDown                004081d0 f   cl_keys.obj
 0001:000071f0       _Key_StringToKeynum        004081f0 f   cl_keys.obj
 0001:000072d0       _Key_KeynumToString        004082d0 f   cl_keys.obj
 0001:00007390       _Key_SetBinding            00408390 f   cl_keys.obj
 0001:000073e0       _Key_GetBinding            004083e0 f   cl_keys.obj
 0001:00007400       _Key_GetKey                00408400 f   cl_keys.obj
 0001:00007440       _Key_Unbind_f              00408440 f   cl_keys.obj
 0001:000074a0       _Key_Unbindall_f           004084a0 f   cl_keys.obj
 0001:000074f0       _Key_Bind_f                004084f0 f   cl_keys.obj
 0001:00007660       _Key_WriteBindings         00408660 f   cl_keys.obj
 0001:000076c0       _Key_Bindlist_f            004086c0 f   cl_keys.obj
 0001:00007710       _CL_InitKeyCommands        00408710 f   cl_keys.obj
 0001:00007750       _CL_AddKeyUpCommands       00408750 f   cl_keys.obj
 0001:00007820       _CL_CharEvent              00408820 f   cl_keys.obj
 0001:00007890       _Field_Paste               00408890 f   cl_keys.obj
 0001:000078e0       _Field_KeyDownEvent        004088e0 f   cl_keys.obj
 0001:00007a10       _Console_Key               00408a10 f   cl_keys.obj
 0001:00007d20       _Message_Key               00408d20 f   cl_keys.obj
 0001:00007df0       _CL_KeyEvent               00408df0 f   cl_keys.obj
 0001:00008160       _Key_ClearStates           00409160 f   cl_keys.obj
 0001:00008200       _CL_CDDialog               00409200 f   cl_main.obj
 0001:00008210       _CL_AddReliableCommand     00409210 f   cl_main.obj
 0001:00008260       _CL_ChangeReliableCommand  00409260 f   cl_main.obj
 0001:000082b0       _CL_WriteDemoMessage       004092b0 f   cl_main.obj
 0001:00008320       _CL_StopRecord_f           00409320 f   cl_main.obj
 0001:000083a0       _CL_DemoFilename           004093a0 f   cl_main.obj
 0001:00008440       _CL_Record_f               00409440 f   cl_main.obj
 0001:00008800       _CL_StartDemoLoop          00409800 f   cl_main.obj
 0001:00008820       _CL_NextDemo               00409820 f   cl_main.obj
 0001:000088a0       _CL_ShutdownAll            004098a0 f   cl_main.obj
 0001:000088e0       _CL_ClearState             004098e0 f   cl_main.obj
 0001:00008900       _CL_Disconnect             00409900 f   cl_main.obj
 0001:00008a20       _CL_ForwardCommandToServer 00409a20 f   cl_main.obj
 0001:00008a80       _CL_RequestMotd            00409a80 f   cl_main.obj
 0001:00008be0       _CL_RequestAuthorization   00409be0 f   cl_main.obj
 0001:00008d80       _CL_ForwardToServer_f      00409d80 f   cl_main.obj
 0001:00008dc0       _CL_Setenv_f               00409dc0 f   cl_main.obj
 0001:00008ee0       _CL_Disconnect_f           00409ee0 f   cl_main.obj
 0001:00008f20       _CL_Reconnect_f            00409f20 f   cl_main.obj
 0001:00008f90       _CL_Connect_f              00409f90 f   cl_main.obj
 0001:00009130       _CL_Rcon_f                 0040a130 f   cl_main.obj
 0001:000092f0       _CL_SendPureChecksums      0040a2f0 f   cl_main.obj
 0001:000093b0       _CL_ResetPureClientAtServer 0040a3b0 f   cl_main.obj
 0001:000093d0       _CL_OpenedPK3List_f        0040a3d0 f   cl_main.obj
 0001:000093f0       _CL_ReferencedPK3List_f    0040a3f0 f   cl_main.obj
 0001:00009410       _CL_Configstrings_f        0040a410 f   cl_main.obj
 0001:00009460       _CL_Clientinfo_f           0040a460 f   cl_main.obj
 0001:000094b0       _CL_BeginDownload          0040a4b0 f   cl_main.obj
 0001:00009550       _CL_CheckForResend         0040a550 f   cl_main.obj
 0001:000097b0       _CL_DisconnectPacket       0040a7b0 f   cl_main.obj
 0001:00009860       _CL_MotdPacket             0040a860 f   cl_main.obj
 0001:00009950       _CL_InitServerInfo         0040a950 f   cl_main.obj
 0001:000099b0       _CL_ServersResponsePacket  0040a9b0 f   cl_main.obj
 0001:00009c50       _CL_CheckTimeout           0040ac50 f   cl_main.obj
 0001:00009ce0       _CL_CheckUserinfo          0040ace0 f   cl_main.obj
 0001:00009d30       _CL_Frame                  0040ad30 f   cl_main.obj
 0001:00009e80       _CL_RefPrintf              0040ae80 f   cl_main.obj
 0001:00009f10       _CL_ShutdownRef            0040af10 f   cl_main.obj
 0001:00009f30       _CL_InitRenderer           0040af30 f   cl_main.obj
 0001:00009f90       _CL_StartHunkUsers         0040af90 f   cl_main.obj
 0001:0000a000       _CL_RefMalloc              0040b000 f   cl_main.obj
 0001:0000a010       _CL_ScaledMilliseconds     0040b010 f   cl_main.obj
 0001:0000a030       _CL_InitRef                0040b030 f   cl_main.obj
 0001:0000a160       _CL_SetModel_f             0040b160 f   cl_main.obj
 0001:0000a1d0       _CL_Shutdown               0040b1d0 f   cl_main.obj
 0001:0000a610       _CL_ServerInfoPacket       0040b610 f   cl_main.obj
 0001:0000a9e0       _CL_GetServerStatus        0040b9e0 f   cl_main.obj
 0001:0000ab30       _CL_ServerStatus           0040bb30 f   cl_main.obj
 0001:0000ad80       _CL_ServerStatusResponse   0040bd80 f   cl_main.obj
 0001:0000b070       _CL_LocalServers_f         0040c070 f   cl_main.obj
 0001:0000b1b0       _CL_GlobalServers_f        0040c1b0 f   cl_main.obj
 0001:0000b330       _CL_GetPing                0040c330 f   cl_main.obj
 0001:0000b420       _CL_UpdateServerInfo       0040c420 f   cl_main.obj
 0001:0000b480       _CL_GetPingInfo            0040c480 f   cl_main.obj
 0001:0000b4c0       _CL_ClearPing              0040c4c0 f   cl_main.obj
 0001:0000b4e0       _CL_GetPingQueueCount      0040c4e0 f   cl_main.obj
 0001:0000b530       _CL_GetFreePing            0040c530 f   cl_main.obj
 0001:0000b600       _CL_Ping_f                 0040c600 f   cl_main.obj
 0001:0000b6f0       _CL_UpdateVisiblePings_f   0040c6f0 f   cl_main.obj
 0001:0000ba10       _CL_ServerStatus_f         0040ca10 f   cl_main.obj
 0001:0000bb30       _CL_ShowIP_f               0040cb30 f   cl_main.obj
 0001:0000bb40       _CL_CDKeyValidate          0040cb40 f   cl_main.obj
 0001:0000bc30       _CL_DemoCompleted          0040cc30 f   cl_main.obj
 0001:0000bca0       _CL_ReadDemoMessage        0040cca0 f   cl_main.obj
 0001:0000bd90       _CL_PlayDemo_f             0040cd90 f   cl_main.obj
 0001:0000bfa0       _CL_FlushMemory            0040cfa0 f   cl_main.obj
 0001:0000c000       _CL_MapLoading             0040d000 f   cl_main.obj
 0001:0000c100       _CL_Vid_Restart_f          0040d100 f   cl_main.obj
 0001:0000c1d0       _CL_Snd_Restart_f          0040d1d0 f   cl_main.obj
 0001:0000c1e0       _CL_DownloadsComplete      0040d1e0 f   cl_main.obj
 0001:0000c260       _CL_NextDownload           0040d260 f   cl_main.obj
 0001:0000c300       _CL_InitDownloads          0040d300 f   cl_main.obj
 0001:0000c390       _CL_ConnectionlessPacket   0040d390 f   cl_main.obj
 0001:0000c800       _CL_PacketEvent            0040d800 f   cl_main.obj
 0001:0000c9a0       _CL_Init                   0040d9a0 f   cl_main.obj
 0001:0000d120       _CL_Netchan_TransmitNextFragment 0040e120 f   cl_net_chan.obj
 0001:0000d130       _CL_Netchan_Transmit       0040e130 f   cl_net_chan.obj
 0001:0000d160       _CL_Netchan_Process        0040e160 f   cl_net_chan.obj
 0001:0000d190       _SHOWNET                   0040e190 f   cl_parse.obj
 0001:0000d1c0       _CL_DeltaEntity            0040e1c0 f   cl_parse.obj
 0001:0000d230       _CL_ParsePacketEntities    0040e230 f   cl_parse.obj
 0001:0000d570       _CL_ParseSnapshot          0040e570 f   cl_parse.obj
 0001:0000d7f0       _CL_SystemInfoChanged      0040e7f0 f   cl_parse.obj
 0001:0000d960       _CL_ParseGamestate         0040e960 f   cl_parse.obj
 0001:0000db20       _CL_ParseDownload          0040eb20 f   cl_parse.obj
 0001:0000dd00       _CL_ParseCommandString     0040ed00 f   cl_parse.obj
 0001:0000dd50       _CL_ParseServerMessage     0040ed50 f   cl_parse.obj
 0001:0000def0       _SCR_AdjustFrom640         0040eef0 f   cl_scrn.obj
 0001:0000df50       _SCR_FillRect              0040ef50 f   cl_scrn.obj
 0001:0000dfc0       _SCR_DrawPic               0040efc0 f   cl_scrn.obj
 0001:0000e110       _SCR_DrawSmallChar         0040f110 f   cl_scrn.obj
 0001:0000e1b0       _SCR_DrawStringExt         0040f1b0 f   cl_scrn.obj
 0001:0000e300       _SCR_DrawBigString         0040f300 f   cl_scrn.obj
 0001:0000e350       _SCR_DrawBigStringColor    0040f350 f   cl_scrn.obj
 0001:0000e380       _SCR_DrawSmallStringExt    0040f380 f   cl_scrn.obj
 0001:0000e450       _SCR_GetBigStringWidth     0040f450 f   cl_scrn.obj
 0001:0000e490       _SCR_DrawDemoRecording     0040f490 f   cl_scrn.obj
 0001:0000e520       _SCR_DebugGraph            0040f520 f   cl_scrn.obj
 0001:0000e550       _SCR_DrawDebugGraph        0040f550 f   cl_scrn.obj
 0001:0000e6b0       _SCR_Init                  0040f6b0 f   cl_scrn.obj
 0001:0000e740       _SCR_DrawScreenField       0040f740 f   cl_scrn.obj
 0001:0000e920       _SCR_UpdateScreen          0040f920 f   cl_scrn.obj
 0001:0000e9c0       _SCR_DrawNamedPic          0040f9c0 f   cl_scrn.obj
 0001:0000ea90       _LAN_LoadCachedServers     0040fa90 f   cl_ui.obj
 0001:0000eba0       _LAN_SaveServersToCache    0040fba0 f   cl_ui.obj
 0001:0000f600       _LAN_UpdateVisiblePings    00410600 f   cl_ui.obj
 0001:0000f610       _LAN_GetServerStatus       00410610 f   cl_ui.obj
 0001:0000f6c0       _Key_GetCatcher            004106c0 f   cl_ui.obj
 0001:0000f6d0       _Key_SetCatcher            004106d0 f   cl_ui.obj
 0001:0000f730       _CL_ShutdownUI             00410730 f   cl_ui.obj
 0001:0000f780       _UI_usesUniqueCDKey        00410780 f   cl_ui.obj
 0001:0000f7a0       _UI_GameCommand            004107a0 f   cl_ui.obj
 0001:0000f8c0       _CL_UISystemCalls          004108c0 f   cl_ui.obj
 0001:00010560       _CL_InitUI                 00411560 f   cl_ui.obj
 0001:00010660       _CMod_LoadShaders          00411660 f   cm_load.obj
 0001:000106f0       _CMod_LoadSubmodels        004116f0 f   cm_load.obj
 0001:00010870       _CMod_LoadNodes            00411870 f   cm_load.obj
 0001:00010910       _CM_BoundBrush             00411910 f   cm_load.obj
 0001:00010960       _CMod_LoadBrushes          00411960 f   cm_load.obj
 0001:00010a60       _CMod_LoadLeafs            00411a60 f   cm_load.obj
 0001:00010b60       _CMod_LoadPlanes           00411b60 f   cm_load.obj
 0001:00010c80       _CMod_LoadLeafBrushes      00411c80 f   cm_load.obj
 0001:00010ce0       _CMod_LoadLeafSurfaces     00411ce0 f   cm_load.obj
 0001:00010d40       _CMod_LoadBrushSides       00411d40 f   cm_load.obj
 0001:00010df0       _CMod_LoadEntityString     00411df0 f   cm_load.obj
 0001:00010e30       _CMod_LoadVisibility       00411e30 f   cm_load.obj
 0001:00010ec0       _CMod_LoadPatches          00411ec0 f   cm_load.obj
 0001:000110d0       _CM_LumpChecksum           004120d0 f   cm_load.obj
 0001:000110f0       _CM_Checksum               004120f0 f   cm_load.obj
 0001:00011220       _CM_ClearMap               00412220 f   cm_load.obj
 0001:00011240       _CM_ClipHandleToModel      00412240 f   cm_load.obj
 0001:000112c0       _CM_InlineModel            004122c0 f   cm_load.obj
 0001:000112f0       _CM_NumClusters            004122f0 f   cm_load.obj
 0001:00011300       _CM_NumInlineModels        00412300 f   cm_load.obj
 0001:00011310       _CM_EntityString           00412310 f   cm_load.obj
 0001:00011320       _CM_LeafCluster            00412320 f   cm_load.obj
 0001:00011350       _CM_LeafArea               00412350 f   cm_load.obj
 0001:00011380       _CM_InitBoxHull            00412380 f   cm_load.obj
 0001:000114b0       _CM_TempBoxModel           004124b0 f   cm_load.obj
 0001:00011600       _CM_ModelBounds            00412600 f   cm_load.obj
 0001:00011640       _CM_LoadMap                00412640 f   cm_load.obj
 0001:000118d0       _CM_ClearLevelPatches      004128d0 f   cm_patch.obj
 0001:000121b0       _CM_PlaneEqual             004131b0 f   cm_patch.obj
 0001:000122b0       _CM_SnapVector             004132b0 f   cm_patch.obj
 0001:00012320       _CM_FindPlane2             00413320 f   cm_patch.obj
 0001:00012a90       _CM_AddFacetBevels         00413a90 f   cm_patch.obj
 0001:000131e0       _CM_TracePointThroughPatchCollide 004141e0 f   cm_patch.obj
 0001:000135a0       _CM_CheckFacetPlane        004145a0 f   cm_patch.obj
 0001:000136e0       _CM_TraceThroughPatchCollide 004146e0 f   cm_patch.obj
 0001:00013c00       _CM_PositionTestInPatchCollide 00414c00 f   cm_patch.obj
 0001:00013e90       _CM_DrawDebugSurface       00414e90 f   cm_patch.obj
 0001:000150b0       _CM_GeneratePatchCollide   004160b0 f   cm_patch.obj
 0001:00015420       _pw                        00416420 f   cm_polylib.obj
 0001:00015470       _AllocWinding              00416470 f   cm_polylib.obj
 0001:000154d0       _FreeWinding               004164d0 f   cm_polylib.obj
 0001:00015540       _RemoveColinearPoints      00416540 f   cm_polylib.obj
 0001:000156c0       _WindingArea               004166c0 f   cm_polylib.obj
 0001:00015770       _WindingBounds             00416770 f   cm_polylib.obj
 0001:00015810       _WindingCenter             00416810 f   cm_polylib.obj
 0001:00015890       _BaseWindingForPlane       00416890 f   cm_polylib.obj
 0001:00015b60       _CopyWinding               00416b60 f   cm_polylib.obj
 0001:00015b90       _ReverseWinding            00416b90 f   cm_polylib.obj
 0001:00015bf0       _ClipWindingEpsilon        00416bf0 f   cm_polylib.obj
 0001:00015ff0       _ChopWindingInPlace        00416ff0 f   cm_polylib.obj
 0001:00016310       _ChopWinding               00417310 f   cm_polylib.obj
 0001:000163b0       _WindingOnPlaneSide        004173b0 f   cm_polylib.obj
 0001:00016450       _AddWindingToConvexHull    00417450 f   cm_polylib.obj
 0001:000169a0       _WindingPlane              004179a0 f   cm_polylib.obj
 0001:00016a40       _CheckWinding              00417a40 f   cm_polylib.obj
 0001:00016cb0       _CM_PointLeafnum_r         00417cb0 f   cm_test.obj
 0001:00016d30       _CM_PointLeafnum           00417d30 f   cm_test.obj
 0001:00016d50       _CM_StoreLeafs             00417d50 f   cm_test.obj
 0001:00016d90       _CM_StoreBrushes           00417d90 f   cm_test.obj
 0001:00016e50       _CM_BoxLeafnums_r          00417e50 f   cm_test.obj
 0001:00016ec0       _CM_BoxLeafnums            00417ec0 f   cm_test.obj
 0001:00016f40       _CM_BoxBrushes             00417f40 f   cm_test.obj
 0001:00016fc0       _CM_PointContents          00417fc0 f   cm_test.obj
 0001:00017170       _CM_TransformedPointContents 00418170 f   cm_test.obj
 0001:00017280       _CM_ClusterPVS             00418280 f   cm_test.obj
 0001:000172b0       _CM_FloodArea_r            004182b0 f   cm_test.obj
 0001:00017330       _CM_FloodAreaConnections   00418330 f   cm_test.obj
 0001:00017380       _CM_AdjustAreaPortalState  00418380 f   cm_test.obj
 0001:00017450       _CM_AreasConnected         00418450 f   cm_test.obj
 0001:000174b0       _CM_WriteAreaBits          004184b0 f   cm_test.obj
 0001:00017540       _RotatePoint               00418540 f   cm_trace.obj
 0001:00017590       _TransposeMatrix           00418590 f   cm_trace.obj
 0001:000175c0       _CM_ProjectPointOntoVector 004185c0 f   cm_trace.obj
 0001:00017650       _CM_VectorDistanceSquared  00418650 f   cm_trace.obj
 0001:00017680       _SquareRootFloat           00418680 f   cm_trace.obj
 0001:000176f0       _CM_TestBoxInBrush         004186f0 f   cm_trace.obj
 0001:000178d0       _CM_TestInLeaf             004188d0 f   cm_trace.obj
 0001:000179e0       _CM_TestCapsuleInCapsule   004189e0 f   cm_trace.obj
 0001:00017c80       _CM_TestBoundingBoxInCapsule 00418c80 f   cm_trace.obj
 0001:00017d90       _CM_PositionTest           00418d90 f   cm_trace.obj
 0001:00017ec0       _CM_TraceThroughPatch      00418ec0 f   cm_trace.obj
 0001:00017f20       _CM_TraceThroughBrush      00418f20 f   cm_trace.obj
 0001:000183f0       _CM_TraceThroughLeaf       004193f0 f   cm_trace.obj
 0001:00018530       _CM_TraceBoundingBoxThroughCapsule 00419530 f   cm_trace.obj
 0001:00018640       _CM_TraceThroughTree       00419640 f   cm_trace.obj
 0001:00018950       _CreateRotationMatrix      00419950 f   cm_trace.obj
 0001:00018990       _CM_DistanceFromLineSquared 00419990 f   cm_trace.obj
 0001:00018a90       _CM_TraceThroughSphere     00419a90 f   cm_trace.obj
 0001:00018d80       _CM_TraceThroughVerticalCylinder 00419d80 f   cm_trace.obj
 0001:000190f0       _CM_TraceCapsuleThroughCapsule 0041a0f0 f   cm_trace.obj
 0001:00019390       _CM_Trace                  0041a390 f   cm_trace.obj
 0001:00019a60       _CM_BoxTrace               0041aa60 f   cm_trace.obj
 0001:00019aa0       _CM_TransformedBoxTrace    0041aaa0 f   cm_trace.obj
 0001:00019f10       _Cbuf_Init                 0041af10 f   cmd.obj
 0001:00019f30       _Cbuf_AddText              0041af30 f   cmd.obj
 0001:00019f90       _Cbuf_InsertText           0041af90 f   cmd.obj
 0001:0001a020       _Cmd_Argc                  0041b020 f   cmd.obj
 0001:0001a030       _Cmd_Argv                  0041b030 f   cmd.obj
 0001:0001a050       _Cmd_ArgvBuffer            0041b050 f   cmd.obj
 0001:0001a090       _Cmd_Args                  0041b090 f   cmd.obj
 0001:0001a120       _Cmd_ArgsFrom              0041b120 f   cmd.obj
 0001:0001a1b0       _Cmd_ArgsBuffer            0041b1b0 f   cmd.obj
 0001:0001a1d0       _Cmd_Cmd                   0041b1d0 f   cmd.obj
 0001:0001a1e0       _Cmd_TokenizeString        0041b1e0 f   cmd.obj
 0001:0001a310       _Cmd_AddCommand            0041b310 f   cmd.obj
 0001:0001a3b0       _Cmd_RemoveCommand         0041b3b0 f   cmd.obj
 0001:0001a430       _Cmd_CommandCompletion     0041b430 f   cmd.obj
 0001:0001a460       _Cmd_ExecuteString         0041b460 f   cmd.obj
 0001:0001a540       _Cmd_List_f                0041b540 f   cmd.obj
 0001:0001a5c0       _Cmd_Wait_f                0041b5c0 f   cmd.obj
 0001:0001a5f0       _Cbuf_Execute              0041b5f0 f   cmd.obj
 0001:0001a6d0       _Cmd_Exec_f                0041b6d0 f   cmd.obj
 0001:0001a790       _Cmd_Vstr_f                0041b790 f   cmd.obj
 0001:0001a7d0       _Cmd_Echo_f                0041b7d0 f   cmd.obj
 0001:0001a820       _Cmd_Init                  0041b820 f   cmd.obj
 0001:0001a870       _Cbuf_ExecuteText          0041b870 f   cmd.obj
 0001:0001a8e0       _Com_BeginRedirect         0041b8e0 f   common.obj
 0001:0001a910       _Com_EndRedirect           0041b910 f   common.obj
 0001:0001a950       _Com_Printf                0041b950 f   common.obj
 0001:0001ab00       _Com_DPrintf               0041bb00 f   common.obj
 0001:0001ab60       _Com_ParseCommandLine      0041bb60 f   common.obj
 0001:0001abd0       _Com_SafeMode              0041bbd0 f   common.obj
 0001:0001ac50       _Com_StartupVariable       0041bc50 f   common.obj
 0001:0001ad20       _Com_AddStartupCommands    0041bd20 f   common.obj
 0001:0001ad90       _Com_StringContains        0041bd90 f   common.obj
 0001:0001ae50       _Com_Filter                0041be50 f   common.obj
 0001:0001b050       _Com_FilterPath            0041c050 f   common.obj
 0001:0001b0e0       _Com_HashKey               0041c0e0 f   common.obj
 0001:0001b130       _Com_RealTime              0041c130 f   common.obj
 0001:0001b1a0       _Z_ClearZone               0041c1a0 f   common.obj
 0001:0001b1f0       _Z_AvailableZoneMemory     0041c1f0 f   common.obj
 0001:0001b200       _Z_AvailableMemory         0041c200 f   common.obj
 0001:0001b210       _Z_LogZoneHeap             0041c210 f   common.obj
 0001:0001b340       _Z_LogHeap                 0041c340 f   common.obj
 0001:0001b370       _Com_Meminfo_f             0041c370 f   common.obj
 0001:0001b5d0       _Hunk_Log                  0041c5d0 f   common.obj
 0001:0001b6e0       _Hunk_SmallLog             0041c6e0 f   common.obj
 0001:0001b850       _Hunk_MemoryRemaining      0041c850 f   common.obj
 0001:0001b880       _Hunk_SetMark              0041c880 f   common.obj
 0001:0001b8a0       _Hunk_ClearToMark          0041c8a0 f   common.obj
 0001:0001b8c0       _Hunk_CheckMark            0041c8c0 f   common.obj
 0001:0001b8e0       _Hunk_Clear                0041c8e0 f   common.obj
 0001:0001b990       _Hunk_ClearTempMemory      0041c990 f   common.obj
 0001:0001b9b0       _Hunk_Trash                0041c9b0 f   common.obj
 0001:0001b9c0       _Com_InitJournaling        0041c9c0 f   common.obj
 0001:0001baa0       _Com_InitPushEvent         0041caa0 f   common.obj
 0001:0001bac0       _Com_RunAndTimeServerPacket 0041cac0 f   common.obj
 0001:0001bc00       _Com_WriteConfigToFile     0041cc00 f   common.obj
 0001:0001bc50       _Com_WriteConfiguration    0041cc50 f   common.obj
 0001:0001bcd0       _Com_WriteConfig_f         0041ccd0 f   common.obj
 0001:0001bd40       _Com_ModifyMsec            0041cd40 f   common.obj
 0001:0001be00       _Com_Shutdown              0041ce00 f   common.obj
 0001:0001be40       __copyDWord                0041ce40 f   common.obj
 0001:0001bed0       _Com_Memset                0041ced0 f   common.obj
 0001:0001bf80       _Com_Memcmp                0041cf80 f   common.obj
 0001:0001c020       _Com_Prefetch              0041d020 f   common.obj
 0001:0001c060       _Q_acos                    0041d060 f   common.obj
 0001:0001c090       _Field_Clear               0041d090 f   common.obj
 0001:0001c2a0       _Com_Error                 0041d2a0 f   common.obj
 0001:0001c450       _Com_Quit_f                0041d450 f   common.obj
 0001:0001c4c0       _Info_Print                0041d4c0 f   common.obj
 0001:0001c5a0       _Z_Free                    0041d5a0 f   common.obj
 0001:0001c690       _Z_FreeTags                0041d690 f   common.obj
 0001:0001c6e0       _Z_TagMalloc               0041d6e0 f   common.obj
 0001:0001c7c0       _Z_Malloc                  0041d7c0 f   common.obj
 0001:0001c7f0       _S_Malloc                  0041d7f0 f   common.obj
 0001:0001c800       _Z_CheckHeap               0041d800 f   common.obj
 0001:0001c880       _CopyString                0041d880 f   common.obj
 0001:0001c8f0       _Com_TouchMemory           0041d8f0 f   common.obj
 0001:0001c930       _Com_InitSmallZoneMemory   0041d930 f   common.obj
 0001:0001c9d0       _Com_InitZoneMemory        0041d9d0 f   common.obj
 0001:0001ca90       _Com_InitHunkMemory        0041da90 f   common.obj
 0001:0001cb80       _Hunk_Alloc                0041db80 f   common.obj
 0001:0001ccc0       _Hunk_AllocateTempMemory   0041dcc0 f   common.obj
 0001:0001cda0       _Hunk_FreeTempMemory       0041dda0 f   common.obj
 0001:0001ce20       _Com_GetRealEvent          0041de20 f   common.obj
 0001:0001cf90       _Com_PushEvent             0041df90 f   common.obj
 0001:0001d030       _Com_GetEvent              0041e030 f   common.obj
 0001:0001d0d0       _Com_Milliseconds          0041e0d0 f   common.obj
 0001:0001d1d0       _Com_ReadCDKey             0041e1d0 f   common.obj
 0001:0001d280       _Com_AppendCDKey           0041e280 f   common.obj
 0001:0001d350       _Com_Init                  0041e350 f   common.obj
 0001:0001d7b0       _Com_Memcpy                0041e7b0 f   common.obj
 0001:0001d8e0       _Field_CompleteCommand     0041e8e0 f   common.obj
 0001:0001da60       _Com_EventLoop             0041ea60 f   common.obj
 0001:0001dd10       _Com_Frame                 0041ed10 f   common.obj
 0001:0001e060       _Cvar_VariableValue        0041f060 f   cvar.obj
 0001:0001e0a0       _Cvar_VariableIntegerValue 0041f0a0 f   cvar.obj
 0001:0001e0e0       _Cvar_VariableString       0041f0e0 f   cvar.obj
 0001:0001e120       _Cvar_VariableStringBuffer 0041f120 f   cvar.obj
 0001:0001e180       _Cvar_CommandCompletion    0041f180 f   cvar.obj
 0001:0001e1b0       _Cvar_Get                  0041f1b0 f   cvar.obj
 0001:0001e3c0       _Cvar_Set2                 0041f3c0 f   cvar.obj
 0001:0001e680       _Cvar_Set                  0041f680 f   cvar.obj
 0001:0001e6a0       _Cvar_SetLatched           0041f6a0 f   cvar.obj
 0001:0001e6c0       _Cvar_SetValue             0041f6c0 f   cvar.obj
 0001:0001e740       _Cvar_Reset                0041f740 f   cvar.obj
 0001:0001e760       _Cvar_SetCheatState        0041f760 f   cvar.obj
 0001:0001e7e0       _Cvar_Command              0041f7e0 f   cvar.obj
 0001:0001e880       _Cvar_Toggle_f             0041f880 f   cvar.obj
 0001:0001e8e0       _Cvar_Set_f                0041f8e0 f   cvar.obj
 0001:0001e9d0       _Cvar_SetU_f               0041f9d0 f   cvar.obj
 0001:0001ea10       _Cvar_SetS_f               0041fa10 f   cvar.obj
 0001:0001ea50       _Cvar_SetA_f               0041fa50 f   cvar.obj
 0001:0001ea90       _Cvar_Reset_f              0041fa90 f   cvar.obj
 0001:0001eac0       _Cvar_WriteVariables       0041fac0 f   cvar.obj
 0001:0001eb50       _Cvar_List_f               0041fb50 f   cvar.obj
 0001:0001eca0       _Cvar_Restart_f            0041fca0 f   cvar.obj
 0001:0001ed30       _Cvar_InfoString           0041fd30 f   cvar.obj
 0001:0001ed70       _Cvar_InfoString_Big       0041fd70 f   cvar.obj
 0001:0001edb0       _Cvar_InfoStringBuffer     0041fdb0 f   cvar.obj
 0001:0001ede0       _Cvar_Update               0041fde0 f   cvar.obj
 0001:0001ee90       _Cvar_Init                 0041fe90 f   cvar.obj
 0001:0001ef30       _Cvar_Register             0041ff30 f   cvar.obj
 0001:0001ef80       _FS_Initialized            0041ff80 f   files.obj
 0001:0001ef90       _FS_PakIsPure              0041ff90 f   files.obj
 0001:0001efd0       _FS_LoadStack              0041ffd0 f   files.obj
 0001:0001f0e0       _FS_ForceFlush             004200e0 f   files.obj
 0001:0001f100       _FS_filelength             00420100 f   files.obj
 0001:0001f160       _FS_BuildOSPath            00420160 f   files.obj
 0001:0001f3a0       _FS_FileExists             004203a0 f   files.obj
 0001:0001f3e0       _FS_SV_FileExists          004203e0 f   files.obj
 0001:0001f440       _FS_SV_FOpenFileWrite      00420440 f   files.obj
 0001:0001f520       _FS_SV_FOpenFileRead       00420520 f   files.obj
 0001:0001f720       _FS_SV_Rename              00420720 f   files.obj
 0001:0001f7e0       _FS_Rename                 004207e0 f   files.obj
 0001:0001f880       _FS_FCloseFile             00420880 f   files.obj
 0001:0001f930       _FS_FOpenFileWrite         00420930 f   files.obj
 0001:0001f9f0       _FS_FOpenFileAppend        004209f0 f   files.obj
 0001:0001fab0       _FS_FilenameCompare        00420ab0 f   files.obj
 0001:0001fb10       _FS_ShiftedStrStr          00420b10 f   files.obj
 0001:0001fb70       _FS_FOpenFileRead          00420b70 f   files.obj
 0001:00020260       _FS_Read                   00421260 f   files.obj
 0001:00020330       _FS_Write                  00421330 f   files.obj
 0001:000203f0       _FS_Printf                 004213f0 f   files.obj
 0001:00020450       _FS_Seek                   00421450 f   files.obj
 0001:000205c0       _FS_FileIsInPAK            004215c0 f   files.obj
 0001:000206e0       _FS_FreeFile               004216e0 f   files.obj
 0001:00020740       _FS_WriteFile              00421740 f   files.obj
 0001:00020b90       _FS_ListFilteredFiles      00421b90 f   files.obj
 0001:00020ed0       _FS_ListFiles              00421ed0 f   files.obj
 0001:00020ef0       _FS_FreeFileList           00421ef0 f   files.obj
 0001:00021060       _FS_GetModList             00422060 f   files.obj
 0001:000213d0       _FS_Dir_f                  004223d0 f   files.obj
 0001:00021490       _FS_ConvertPath            00422490 f   files.obj
 0001:000214c0       _FS_PathCmp                004224c0 f   files.obj
 0001:00021530       _FS_SortFileList           00422530 f   files.obj
 0001:000215d0       _FS_NewDir_f               004225d0 f   files.obj
 0001:00021690       _FS_Path_f                 00422690 f   files.obj
 0001:00021770       _FS_TouchFile_f            00422770 f   files.obj
 0001:000219a0       _FS_idPak                  004229a0 f   files.obj
 0001:000219f0       _FS_ComparePaks            004229f0 f   files.obj
 0001:00021be0       _FS_Shutdown               00422be0 f   files.obj
 0001:00022080       _FS_GamePureChecksum       00423080 f   files.obj
 0001:000220d0       _FS_LoadedPakChecksums     004230d0 f   files.obj
 0001:00022120       _FS_LoadedPakNames         00423120 f   files.obj
 0001:00022190       _FS_LoadedPakPureChecksums 00423190 f   files.obj
 0001:000221e0       _FS_ReferencedPakChecksums 004231e0 f   files.obj
 0001:00022250       _FS_ReferencedPakPureChecksums 00423250 f   files.obj
 0001:000223a0       _FS_ReferencedPakNames     004233a0 f   files.obj
 0001:00022470       _FS_ClearPakReferences     00423470 f   files.obj
 0001:000224b0       _FS_PureServerSetLoadedPaks 004234b0 f   files.obj
 0001:000225c0       _FS_PureServerSetReferencedPaks 004235c0 f   files.obj
 0001:00022690       _FS_FOpenFileByMode        00423690 f   files.obj
 0001:000227c0       _FS_FTell                  004237c0 f   files.obj
 0001:00022800       _FS_Flush                  00423800 f   files.obj
 0001:00022820       _FS_Read2                  00423820 f   files.obj
 0001:00022890       _FS_ReadFile               00423890 f   files.obj
 0001:00022b40       _FS_GetFileList            00423b40 f   files.obj
 0001:00022df0       _FS_InitFilesystem         00423df0 f   files.obj
 0001:00022ea0       _FS_Restart                00423ea0 f   files.obj
 0001:00022fe0       _FS_ConditionalRestart     00423fe0 f   files.obj
 0001:00023010       _Huff_putBit               00424010 f   huffman.obj
 0001:00023060       _Huff_getBit               00424060 f   huffman.obj
 0001:000232d0       _Huff_addRef               004242d0 f   huffman.obj
 0001:00023470       _Huff_Receive              00424470 f   huffman.obj
 0001:000234d0       _Huff_offsetReceive        004244d0 f   huffman.obj
 0001:000235e0       _Huff_transmit             004245e0 f   huffman.obj
 0001:00023780       _Huff_offsetTransmit       00424780 f   huffman.obj
 0001:000237c0       _Huff_Decompress           004247c0 f   huffman.obj
 0001:00023a10       _Huff_Compress             00424a10 f   huffman.obj
 0001:00023b40       _Huff_Init                 00424b40 f   huffman.obj
 0001:00023c20       _MD4Init                   00424c20 f   md4.obj
 0001:00024330       _MD4Update                 00425330 f   md4.obj
 0001:000243e0       _MD4Final                  004253e0 f   md4.obj
 0001:000244a0       _Com_BlockChecksum         004254a0 f   md4.obj
 0001:00024510       _Com_BlockChecksumKey      00425510 f   md4.obj
 0001:00024590       _MSG_Clear                 00425590 f   msg.obj
 0001:000245a0       _MSG_Bitstream             004255a0 f   msg.obj
 0001:000245b0       _MSG_BeginReading          004255b0 f   msg.obj
 0001:000245c0       _MSG_BeginReadingOOB       004255c0 f   msg.obj
 0001:000245e0       _MSG_Copy                  004255e0 f   msg.obj
 0001:00024630       _MSG_WriteBits             00425630 f   msg.obj
 0001:000247d0       _MSG_ReadBits              004257d0 f   msg.obj
 0001:00024910       _MSG_WriteChar             00425910 f   msg.obj
 0001:00024930       _MSG_WriteByte             00425930 f   msg.obj
 0001:00024950       _MSG_WriteData             00425950 f   msg.obj
 0001:00024980       _MSG_WriteShort            00425980 f   msg.obj
 0001:000249a0       _MSG_WriteLong             004259a0 f   msg.obj
 0001:000249c0       _MSG_WriteFloat            004259c0 f   msg.obj
 0001:000249e0       _MSG_WriteString           004259e0 f   msg.obj
 0001:00024ab0       _MSG_WriteBigString        00425ab0 f   msg.obj
 0001:00024b80       _MSG_WriteAngle            00425b80 f   msg.obj
 0001:00024bb0       _MSG_WriteAngle16          00425bb0 f   msg.obj
 0001:00024be0       _MSG_ReadChar              00425be0 f   msg.obj
 0001:00024c10       _MSG_ReadByte              00425c10 f   msg.obj
 0001:00024c40       _MSG_ReadShort             00425c40 f   msg.obj
 0001:00024c70       _MSG_ReadLong              00425c70 f   msg.obj
 0001:00024c90       _MSG_ReadFloat             00425c90 f   msg.obj
 0001:00024cc0       _MSG_ReadString            00425cc0 f   msg.obj
 0001:00024d30       _MSG_ReadBigString         00425d30 f   msg.obj
 0001:00024d90       _MSG_ReadStringLine        00425d90 f   msg.obj
 0001:00024e00       _MSG_ReadAngle16           00425e00 f   msg.obj
 0001:00024e40       _MSG_ReadData              00425e40 f   msg.obj
 0001:00024e80       _MSG_WriteDelta            00425e80 f   msg.obj
 0001:00024ed0       _MSG_ReadDelta             00425ed0 f   msg.obj
 0001:00024f00       _MSG_WriteDeltaFloat       00425f00 f   msg.obj
 0001:00024f50       _MSG_ReadDeltaFloat        00425f50 f   msg.obj
 0001:00024f90       _MSG_WriteDeltaKey         00425f90 f   msg.obj
 0001:00024fe0       _MSG_ReadDeltaKey          00425fe0 f   msg.obj
 0001:00025020       _MSG_WriteDeltaKeyFloat    00426020 f   msg.obj
 0001:00025070       _MSG_ReadDeltaKeyFloat     00426070 f   msg.obj
 0001:000250b0       _MSG_WriteDeltaUsercmd     004260b0 f   msg.obj
 0001:00025270       _MSG_ReadDeltaUsercmd      00426270 f   msg.obj
 0001:000253e0       _MSG_WriteDeltaUsercmdKey  004263e0 f   msg.obj
 0001:00025640       _MSG_ReadDeltaUsercmdKey   00426640 f   msg.obj
 0001:00025880       _MSG_ReportChangeVectors_f 00426880 f   msg.obj
 0001:000258b0       _MSG_WriteDeltaEntity      004268b0 f   msg.obj
 0001:00025b20       _MSG_ReadDeltaEntity       00426b20 f   msg.obj
 0001:00025dc0       _MSG_WriteDeltaPlayerstate 00426dc0 f   msg.obj
 0001:00026390       _MSG_ReadDeltaPlayerstate  00427390 f   msg.obj
 0001:00026810       _MSG_initHuffman           00427810 f   msg.obj
 0001:00026870       _MSG_Init                  00427870 f   msg.obj
 0001:000268a0       _MSG_InitOOB               004278a0 f   msg.obj
 0001:000268e0       _Netchan_Init              004278e0 f   net_chan.obj
 0001:00026950       _Netchan_Setup             00427950 f   net_chan.obj
 0001:000269c0       _NET_CompareBaseAdr        004279c0 f   net_chan.obj
 0001:00026a40       _NET_AdrToString           00427a40 f   net_chan.obj
 0001:00026b30       _NET_CompareAdr            00427b30 f   net_chan.obj
 0001:00026bd0       _NET_IsLocalAddress        00427bd0 f   net_chan.obj
 0001:00026be0       _NET_GetLoopPacket         00427be0 f   net_chan.obj
 0001:00026c70       _NET_SendLoopPacket        00427c70 f   net_chan.obj
 0001:00026cc0       _NET_SendPacket            00427cc0 f   net_chan.obj
 0001:00026d60       _NET_OutOfBandPrint        00427d60 f   net_chan.obj
 0001:00026e00       _NET_OutOfBandData         00427e00 f   net_chan.obj
 0001:00026ea0       _NET_StringToAdr           00427ea0 f   net_chan.obj
 0001:00026fa0       _Netchan_TransmitNextFragment 00427fa0 f   net_chan.obj
 0001:00027100       _Netchan_Transmit          00428100 f   net_chan.obj
 0001:00027250       _Netchan_Process           00428250 f   net_chan.obj
 0001:00027590       _Q_rand                    00428590 f   q_math.obj
 0001:000275a0       _Q_random                  004285a0 f   q_math.obj
 0001:000275d0       _Q_crandom                 004285d0 f   q_math.obj
 0001:00027600       _ClampChar                 00428600 f   q_math.obj
 0001:00027620       _ClampShort                00428620 f   q_math.obj
 0001:00027670       _DirToByte                 00428670 f   q_math.obj
 0001:00027830       _ByteToDir                 00428830 f   q_math.obj
 0001:00027890       _ColorBytes3               00428890 f   q_math.obj
 0001:000278d0       _ColorBytes4               004288d0 f   q_math.obj
 0001:00027960       _NormalizeColor            00428960 f   q_math.obj
 0001:000279d0       _vectoangles               004289d0 f   q_math.obj
 0001:00027ae0       _AxisClear                 00428ae0 f   q_math.obj
 0001:00027b10       _AxisCopy                  00428b10 f   q_math.obj
 0001:00027b50       _ProjectPointOnPlane       00428b50 f   q_math.obj
 0001:00027bd0       _VectorRotate              00428bd0 f   q_math.obj
 0001:00027c30       _Q_rsqrt                   00428c30 f   q_math.obj
 0001:00027c70       _Q_fabs                    00428c70 f   q_math.obj
 0001:00027c90       _LerpAngle                 00428c90 f   q_math.obj
 0001:00027ce0       _AngleSubtract             00428ce0 f   q_math.obj
 0001:00027d40       _AnglesSubtract            00428d40 f   q_math.obj
 0001:00027d80       _AngleMod                  00428d80 f   q_math.obj
 0001:00027db0       _AngleNormalize360         00428db0 f   q_math.obj
 0001:00027de0       _AngleNormalize180         00428de0 f   q_math.obj
 0001:00027e20       _AngleDelta                00428e20 f   q_math.obj
 0001:00027e60       _SetPlaneSignbits          00428e60 f   q_math.obj
 0001:00027eb0       _BoxOnPlaneSide            00428eb0 f   q_math.obj
 0001:000280f0       _RadiusFromBounds          004290f0 f   q_math.obj
 0001:00028170       _ClearBounds               00429170 f   q_math.obj
 0001:000281a0       _AddPointToBounds          004291a0 f   q_math.obj
 0001:00028220       _VectorNormalize           00429220 f   q_math.obj
 0001:00028280       _VectorNormalize2          00429280 f   q_math.obj
 0001:000282f0       __VectorMA                 004292f0 f   q_math.obj
 0001:00028330       __DotProduct               00429330 f   q_math.obj
 0001:00028350       __VectorSubtract           00429350 f   q_math.obj
 0001:00028380       __VectorAdd                00429380 f   q_math.obj
 0001:000283b0       __VectorCopy               004293b0 f   q_math.obj
 0001:000283d0       __VectorScale              004293d0 f   q_math.obj
 0001:00028400       _Vector4Scale              00429400 f   q_math.obj
 0001:00028430       _Q_log2                    00429430 f   q_math.obj
 0001:00028450       _MatrixMultiply            00429450 f   q_math.obj
 0001:00028540       _AngleVectors              00429540 f   q_math.obj
 0001:00028680       _PerpendicularVector       00429680 f   q_math.obj
 0001:00028770       _PlaneFromPoints           00429770 f   q_math.obj
 0001:00028820       _RotatePointAroundVector   00429820 f   q_math.obj
 0001:00028a20       _RotateAroundDirection     00429a20 f   q_math.obj
 0001:00028ab0       _AnglesToAxis              00429ab0 f   q_math.obj
 0001:00028b00       _MakeNormalVectors         00429b00 f   q_math.obj
 0001:00028b90       _Com_Clamp                 00429b90 f   q_shared.obj
 0001:00028bc0       _COM_SkipPath              00429bc0 f   q_shared.obj
 0001:00028bf0       _COM_StripExtension        00429bf0 f   q_shared.obj
 0001:00028c20       _ShortSwap                 00429c20 f   q_shared.obj
 0001:00028c40       _ShortNoSwap               00429c40 f   q_shared.obj
 0001:00028c50       _LongSwap                  00429c50 f   q_shared.obj
 0001:00028c80       _LongNoSwap                00429c80 f   q_shared.obj
 0001:00028c90       _Long64Swap                00429c90 f   q_shared.obj
 0001:00028cf0       _Long64NoSwap              00429cf0 f   q_shared.obj
 0001:00028d00       _FloatSwap                 00429d00 f   q_shared.obj
 0001:00028d40       _FloatNoSwap               00429d40 f   q_shared.obj
 0001:00028d50       _COM_GetCurrentParseLine   00429d50 f   q_shared.obj
 0001:00028d60       _COM_ParseError            00429d60 f   q_shared.obj
 0001:00028da0       _COM_ParseWarning          00429da0 f   q_shared.obj
 0001:00028e20       _COM_Compress              00429e20 f   q_shared.obj
 0001:00028f20       _COM_ParseExt              00429f20 f   q_shared.obj
 0001:00029090       _SkipBracedSection         0042a090 f   q_shared.obj
 0001:000290d0       _SkipRestOfLine            0042a0d0 f   q_shared.obj
 0001:00029100       _Q_isprint                 0042a100 f   q_shared.obj
 0001:00029120       _Q_islower                 0042a120 f   q_shared.obj
 0001:00029140       _Q_isupper                 0042a140 f   q_shared.obj
 0001:00029160       _Q_isalpha                 0042a160 f   q_shared.obj
 0001:00029190       _Q_strrchr                 0042a190 f   q_shared.obj
 0001:000291c0       _Q_strncpyz                0042a1c0 f   q_shared.obj
 0001:00029220       _Q_stricmpn                0042a220 f   q_shared.obj
 0001:000292a0       _Q_strncmp                 0042a2a0 f   q_shared.obj
 0001:000292e0       _Q_stricmp                 0042a2e0 f   q_shared.obj
 0001:00029310       _Q_strlwr                  0042a310 f   q_shared.obj
 0001:00029340       _Q_strupr                  0042a340 f   q_shared.obj
 0001:00029370       _Q_strcat                  0042a370 f   q_shared.obj
 0001:000293c0       _Q_PrintStrlen             0042a3c0 f   q_shared.obj
 0001:00029400       _Q_CleanStr                0042a400 f   q_shared.obj
 0001:00029450       _Com_sprintf               0042a450 f   q_shared.obj
 0001:000294d0       _va                        0042a4d0 f   q_shared.obj
 0001:00029510       _Info_ValueForKey          0042a510 f   q_shared.obj
 0001:00029610       _Info_NextPair             0042a610 f   q_shared.obj
 0001:00029670       _Info_RemoveKey            0042a670 f   q_shared.obj
 0001:00029770       _Info_RemoveKey_Big        0042a770 f   q_shared.obj
 0001:00029880       _Info_Validate             0042a880 f   q_shared.obj
 0001:000298b0       _Info_SetValueForKey       0042a8b0 f   q_shared.obj
 0001:00029a80       _Info_SetValueForKey_Big   0042aa80 f   q_shared.obj
 0001:00029c50       _COM_DefaultExtension      0042ac50 f   q_shared.obj
 0001:00029cd0       _COM_BeginParseSession     0042acd0 f   q_shared.obj
 0001:00029d00       _COM_Parse                 0042ad00 f   q_shared.obj
 0001:00029d10       _COM_MatchToken            0042ad10 f   q_shared.obj
 0001:00029d80       _Parse1DMatrix             0042ad80 f   q_shared.obj
 0001:00029e00       _Parse2DMatrix             0042ae00 f   q_shared.obj
 0001:00029e90       _Parse3DMatrix             0042ae90 f   q_shared.obj
 0001:00029f20       _S_AdpcmEncode             0042af20 f   snd_adpcm.obj
 0001:0002a080       _S_AdpcmDecode             0042b080 f   snd_adpcm.obj
 0001:0002a1a0       _S_AdpcmMemoryNeeded       0042b1a0 f   snd_adpcm.obj
 0001:0002a1f0       _S_AdpcmGetSamples         0042b1f0 f   snd_adpcm.obj
 0001:0002a230       _S_AdpcmEncodeSound        0042b230 f   snd_adpcm.obj
 0001:0002a2c0       _S_SoundInfo_f             0042b2c0 f   snd_dma.obj
 0001:0002a400       _S_ChannelFree             0042b400 f   snd_dma.obj
 0001:0002a420       _S_ChannelMalloc           0042b420 f   snd_dma.obj
 0001:0002a450       _S_ChannelSetup            0042b450 f   snd_dma.obj
 0001:0002a4a0       _S_Shutdown                0042b4a0 f   snd_dma.obj
 0001:0002a650       _S_DefaultSound            0042b650 f   snd_dma.obj
 0001:0002a690       _S_memoryLoad              0042b690 f   snd_dma.obj
 0001:0002a6c0       _S_SpatializeOrigin        0042b6c0 f   snd_dma.obj
 0001:0002a800       _S_StartSound              0042b800 f   snd_dma.obj
 0001:0002abe0       _S_StartLocalSound         0042bbe0 f   snd_dma.obj
 0001:0002ac30       _S_ClearSoundBuffer        0042bc30 f   snd_dma.obj
 0001:0002acd0       _S_StopLoopingSound        0042bcd0 f   snd_dma.obj
 0001:0002acf0       _S_ClearLoopingSounds      0042bcf0 f   snd_dma.obj
 0001:0002ad30       _S_AddLoopingSound         0042bd30 f   snd_dma.obj
 0001:0002af20       _S_AddRealLoopingSound     0042bf20 f   snd_dma.obj
 0001:0002b010       _S_AddLoopSounds           0042c010 f   snd_dma.obj
 0001:0002b1b0       _S_ByteSwapRawSamples      0042c1b0 f   snd_dma.obj
 0001:0002b1c0       _S_GetRawSamplePointer     0042c1c0 f   snd_dma.obj
 0001:0002b1d0       _S_RawSamples              0042c1d0 f   snd_dma.obj
 0001:0002b4b0       _S_UpdateEntityPosition    0042c4b0 f   snd_dma.obj
 0001:0002b500       _S_Respatialize            0042c500 f   snd_dma.obj
 0001:0002b620       _S_ScanChannelStarts       0042c620 f   snd_dma.obj
 0001:0002b690       _S_SoundList_f             0042c690 f   snd_dma.obj
 0001:0002b7a0       _FGetLittleLong            0042c7a0 f   snd_dma.obj
 0001:0002b7c0       _FGetLittleShort           0042c7c0 f   snd_dma.obj
 0001:0002b7e0       _S_FindWavChunk            0042c7e0 f   snd_dma.obj
 0001:0002b880       _S_StopBackgroundTrack     0042c880 f   snd_dma.obj
 0001:0002b8c0       _S_StartBackgroundTrack    0042c8c0 f   snd_dma.obj
 0001:0002bb60       _S_UpdateBackgroundTrack   0042cb60 f   snd_dma.obj
 0001:0002bd10       _S_FreeOldestSound         0042cd10 f   snd_dma.obj
 0001:0002bda0       _S_RegisterSound           0042cda0 f   snd_dma.obj
 0001:0002be30       _S_StopAllSounds           0042ce30 f   snd_dma.obj
 0001:0002be70       _S_GetSoundtime            0042ce70 f   snd_dma.obj
 0001:0002bf20       _S_Update_                 0042cf20 f   snd_dma.obj
 0001:0002c030       _S_Play_f                  0042d030 f   snd_dma.obj
 0001:0002c120       _S_Music_f                 0042d120 f   snd_dma.obj
 0001:0002c180       _S_Init                    0042d180 f   snd_dma.obj
 0001:0002c340       _S_DisableSounds           0042d340 f   snd_dma.obj
 0001:0002c390       _S_BeginRegistration       0042d390 f   snd_dma.obj
 0001:0002c3f0       _S_Update                  0042d3f0 f   snd_dma.obj
 0001:0002c480       _SND_free                  0042d480 f   snd_mem.obj
 0001:0002c4a0       _SND_malloc                0042d4a0 f   snd_mem.obj
 0001:0002c500       _SND_setup                 0042d500 f   snd_mem.obj
 0001:0002c9d0       _S_LoadSound               0042d9d0 f   snd_mem.obj
 0001:0002cb30       _S_DisplayFreeMemory       0042db30 f   snd_mem.obj
 0001:0002cb50       _S_WriteLinearBlastStereo16 0042db50 f   snd_mix.obj
 0001:0002cbd0       _S_TransferStereo16        0042dbd0 f   snd_mix.obj
 0001:0002cc40       _S_TransferPaintBuffer     0042dc40 f   snd_mix.obj
 0001:0002d0a0       _S_PaintChannelFromWavelet 0042e0a0 f   snd_mix.obj
 0001:0002d1d0       _S_PaintChannelFromADPCM   0042e1d0 f   snd_mix.obj
 0001:0002d310       _S_PaintChannelFromMuLaw   0042e310 f   snd_mix.obj
 0001:0002d490       _S_PaintChannels           0042e490 f   snd_mix.obj
 0001:0002d7a0       _daub4                     0042e7a0 f   snd_wavelet.obj
 0001:0002dbb0       _wt1                       0042ebb0 f   snd_wavelet.obj
 0001:0002dc10       _MuLawEncode               0042ec10 f   snd_wavelet.obj
 0001:0002dc70       _MuLawDecode               0042ec70 f   snd_wavelet.obj
 0001:0002dca0       _NXPutc                    0042eca0 f   snd_wavelet.obj
 0001:0002dcc0       _encodeWavelet             0042ecc0 f   snd_wavelet.obj
 0001:0002df10       _decodeWavelet             0042ef10 f   snd_wavelet.obj
 0001:0002e020       _encodeMuLaw               0042f020 f   snd_wavelet.obj
 0001:0002e1b0       _decodeMuLaw               0042f1b0 f   snd_wavelet.obj
 0001:0002e1f0       _SV_BotAllocateClient      0042f1f0 f   sv_bot.obj
 0001:0002e260       _SV_BotFreeClient          0042f260 f   sv_bot.obj
 0001:0002e2c0       _BotDrawDebugPolygons      0042f2c0 f   sv_bot.obj
 0001:0002e440       _BotImport_Print           0042f440 f   sv_bot.obj
 0001:0002e550       _BotImport_Trace           0042f550 f   sv_bot.obj
 0001:0002e600       _BotImport_EntityTrace     0042f600 f   sv_bot.obj
 0001:0002e6b0       _BotImport_PointContents   0042f6b0 f   sv_bot.obj
 0001:0002e6c0       _BotImport_inPVS           0042f6c0 f   sv_bot.obj
 0001:0002e6d0       _BotImport_BSPEntityData   0042f6d0 f   sv_bot.obj
 0001:0002e6e0       _BotImport_BSPModelMinsMaxsOrigin 0042f6e0 f   sv_bot.obj
 0001:0002e7c0       _BotImport_GetMemory       0042f7c0 f   sv_bot.obj
 0001:0002e7d0       _BotImport_FreeMemory      0042f7d0 f   sv_bot.obj
 0001:0002e7e0       _BotImport_HunkAlloc       0042f7e0 f   sv_bot.obj
 0001:0002e810       _BotImport_DebugPolygonCreate 0042f810 f   sv_bot.obj
 0001:0002e890       _BotImport_DebugPolygonShow 0042f890 f   sv_bot.obj
 0001:0002e8e0       _BotImport_DebugPolygonDelete 0042f8e0 f   sv_bot.obj
 0001:0002e900       _BotImport_DebugLineCreate 0042f900 f   sv_bot.obj
 0001:0002e920       _BotImport_DebugLineDelete 0042f920 f   sv_bot.obj
 0001:0002e940       _BotImport_DebugLineShow   0042f940 f   sv_bot.obj
 0001:0002eb30       _BotClientCommand          0042fb30 f   sv_bot.obj
 0001:0002eb60       _SV_BotFrame               0042fb60 f   sv_bot.obj
 0001:0002eb90       _SV_BotLibSetup            0042fb90 f   sv_bot.obj
 0001:0002ebc0       _SV_BotLibShutdown         0042fbc0 f   sv_bot.obj
 0001:0002ebe0       _SV_BotInitCvars           0042fbe0 f   sv_bot.obj
 0001:0002ee20       _SV_BotInitBotLib          0042fe20 f   sv_bot.obj
 0001:0002ef50       _SV_BotGetConsoleMessage   0042ff50 f   sv_bot.obj
 0001:0002efc0       _SV_BotGetSnapshotEntity   0042ffc0 f   sv_bot.obj
 0001:0002fd40       _SV_Heartbeat_f            00430d40 f   sv_ccmds.obj
 0001:0002fe00       _SV_AddOperatorCommands    00430e00 f   sv_ccmds.obj
 0001:0002ff30       _SV_RemoveOperatorCommands 00430f30 f   sv_ccmds.obj
 0001:0002ff50       _SV_AuthorizeIpPacket      00430f50 f   sv_client.obj
 0001:00030220       _SV_SendClientGameState    00431220 f   sv_client.obj
 0001:000303c0       _SV_ClientEnterWorld       004313c0 f   sv_client.obj
 0001:000304e0       _SV_StopDownload_f         004314e0 f   sv_client.obj
 0001:00030530       _SV_DoneDownload_f         00431530 f   sv_client.obj
 0001:00030560       _SV_BeginDownload_f        00431560 f   sv_client.obj
 0001:00030590       _SV_WriteDownloadToClient  00431590 f   sv_client.obj
 0001:00030a80       _SV_UserinfoChanged        00431a80 f   sv_client.obj
 0001:00030d20       _SV_ExecuteClientCommand   00431d20 f   sv_client.obj
 0001:00030e10       _SV_ClientThink            00431e10 f   sv_client.obj
 0001:00030e80       _SV_GetChallenge           00431e80 f   sv_client.obj
 0001:00031290       _SV_DropClient             00432290 f   sv_client.obj
 0001:00031440       _SV_NextDownload_f         00432440 f   sv_client.obj
 0001:00031a90       _SV_ExecuteClientMessage   00432a90 f   sv_client.obj
 0001:00031c00       _SV_DirectConnect          00432c00 f   sv_client.obj
 0001:00032570       _SV_GameError              00433570 f   sv_game.obj
 0001:00032590       _SV_GamePrint              00433590 f   sv_game.obj
 0001:000325b0       _SV_NumForGentity          004335b0 f   sv_game.obj
 0001:000325d0       _SV_GentityNum             004335d0 f   sv_game.obj
 0001:000325f0       _SV_GameClientNum          004335f0 f   sv_game.obj
 0001:00032610       _SV_SvEntityForGentity     00433610 f   sv_game.obj
 0001:00032650       _SV_GEntityForSvEntity     00433650 f   sv_game.obj
 0001:00032680       _SV_GameSendServerCommand  00433680 f   sv_game.obj
 0001:000326d0       _SV_GameDropClient         004336d0 f   sv_game.obj
 0001:00032700       _SV_SetBrushModel          00433700 f   sv_game.obj
 0001:000327c0       _SV_inPVS                  004337c0 f   sv_game.obj
 0001:00032840       _SV_inPVSIgnorePortals     00433840 f   sv_game.obj
 0001:000328b0       _SV_AdjustAreaPortalState  004338b0 f   sv_game.obj
 0001:00032910       _SV_EntityContact          00433910 f   sv_game.obj
 0001:00032960       _SV_GetServerinfo          00433960 f   sv_game.obj
 0001:000329a0       _SV_LocateGameData         004339a0 f   sv_game.obj
 0001:000329e0       _SV_GetUsercmd             004339e0 f   sv_game.obj
 0001:00032a50       _SV_GameSystemCalls        00433a50 f   sv_game.obj
 0001:00034960       _SV_ShutdownGameProgs      00435960 f   sv_game.obj
 0001:00034a00       _SV_RestartGameProgs       00435a00 f   sv_game.obj
 0001:00034a50       _SV_InitGameProgs          00435a50 f   sv_game.obj
 0001:00034ac0       _SV_GameCommand            00435ac0 f   sv_game.obj
 0001:00034ae0       _SV_SetConfigstring        00435ae0 f   sv_init.obj
 0001:00034cc0       _SV_GetConfigstring        00435cc0 f   sv_init.obj
 0001:00034d30       _SV_SetUserinfo            00435d30 f   sv_init.obj
 0001:00034db0       _SV_GetUserinfo            00435db0 f   sv_init.obj
 0001:00034e10       _SV_CreateBaseline         00435e10 f   sv_init.obj
 0001:00034e60       _SV_BoundMaxClients        00435e60 f   sv_init.obj
 0001:00034ec0       _SV_Startup                00435ec0 f   sv_init.obj
 0001:00034f50       _SV_ChangeMaxClients       00435f50 f   sv_init.obj
 0001:00035100       _SV_ClearServer            00436100 f   sv_init.obj
 0001:00035140       _SV_TouchCGame             00436140 f   sv_init.obj
 0001:00035190       _SV_SpawnServer            00436190 f   sv_init.obj
 0001:00035620       _SV_Init                   00436620 f   sv_init.obj
 0001:000359a0       _SV_FinalMessage           004369a0 f   sv_init.obj
 0001:00035a30       _SV_Shutdown               00436a30 f   sv_init.obj
 0001:00035af0       _SV_ExpandNewlines         00436af0 f   sv_main.obj
 0001:00035b40       _SV_ReplacePendingServerCommands 00436b40 f   sv_main.obj
 0001:00035c00       _SV_AddServerCommand       00436c00 f   sv_main.obj
 0001:00035cc0       _SV_SendServerCommand      00436cc0 f   sv_main.obj
 0001:00035d90       _SV_MasterHeartbeat        00436d90 f   sv_main.obj
 0001:00035f00       _SV_MasterShutdown         00436f00 f   sv_main.obj
 0001:00035f20       _SVC_Status                00436f20 f   sv_main.obj
 0001:00036100       _SVC_Info                  00437100 f   sv_main.obj
 0001:00036350       _SV_FlushRedirect          00437350 f   sv_main.obj
 0001:000363a0       _SVC_RemoteCommand         004373a0 f   sv_main.obj
 0001:000365f0       _SV_ConnectionlessPacket   004375f0 f   sv_main.obj
 0001:00036850       _SV_PacketEvent            00437850 f   sv_main.obj
 0001:000369e0       _SV_CalcPings              004379e0 f   sv_main.obj
 0001:00036b10       _SV_CheckTimeouts          00437b10 f   sv_main.obj
 0001:00036bf0       _SV_CheckPaused            00437bf0 f   sv_main.obj
 0001:00036c80       _SV_Frame                  00437c80 f   sv_main.obj
 0001:00037020       _SV_Netchan_TransmitNextFragment 00438020 f   sv_net_chan.obj
 0001:000370e0       _SV_Netchan_Transmit       004380e0 f   sv_net_chan.obj
 0001:00037180       _SV_Netchan_Process        00438180 f   sv_net_chan.obj
 0001:00037440       _SV_UpdateServerCommandsToClient 00438440 f   sv_snapshot.obj
 0001:00037a40       _SV_SendMessageToClient    00438a40 f   sv_snapshot.obj
 0001:00037b70       _SV_SendClientSnapshot     00438b70 f   sv_snapshot.obj
 0001:00037c30       _SV_SendClientMessages     00438c30 f   sv_snapshot.obj
 0001:00037cb0       _SV_ClipHandleForEntity    00438cb0 f   sv_world.obj
 0001:00037d10       _SV_SectorList_f           00438d10 f   sv_world.obj
 0001:00037d50       _SV_CreateworldSector      00438d50 f   sv_world.obj
 0001:00037e60       _SV_ClearWorld             00438e60 f   sv_world.obj
 0001:00037eb0       _SV_UnlinkEntity           00438eb0 f   sv_world.obj
 0001:00037f10       _SV_LinkEntity             00438f10 f   sv_world.obj
 0001:00038340       _SV_AreaEntities_r         00439340 f   sv_world.obj
 0001:00038460       _SV_AreaEntities           00439460 f   sv_world.obj
 0001:000384a0       _SV_ClipToEntity           004394a0 f   sv_world.obj
 0001:00038540       _SV_ClipMoveToEntities     00439540 f   sv_world.obj
 0001:000386f0       _SV_Trace                  004396f0 f   sv_world.obj
 0001:000388d0       _SV_PointContents          004398d0 f   sv_world.obj
 0001:00038a60       _unzStringFileNameCompare  00439a60 f   unzip.obj
 0001:00038ac0       _unzlocal_SearchCentralDir 00439ac0 f   unzip.obj
 0001:00038bf0       _unzReOpen                 00439bf0 f   unzip.obj
 0001:00038c40       _unzOpen                   00439c40 f   unzip.obj
 0001:00038dd0       _unzGetGlobalInfo          00439dd0 f   unzip.obj
 0001:00039200       _unzGetCurrentFileInfo     0043a200 f   unzip.obj
 0001:00039240       _unzGoToFirstFile          0043a240 f   unzip.obj
 0001:00039290       _unzGoToNextFile           0043a290 f   unzip.obj
 0001:00039300       _unzGetCurrentFileInfoPosition 0043a300 f   unzip.obj
 0001:00039320       _unzSetCurrentFileInfoPosition 0043a320 f   unzip.obj
 0001:00039370       _unzLocateFile             0043a370 f   unzip.obj
 0001:00039650       _unztell                   0043a650 f   unzip.obj
 0001:00039670       _unzeof                    0043a670 f   unzip.obj
 0001:000396a0       _unzGetLocalExtrafield     0043a6a0 f   unzip.obj
 0001:00039730       _unzGetGlobalComment       0043a730 f   unzip.obj
 0001:0003be60       _unzReadCurrentFile        0043ce60 f   unzip.obj
 0001:0003c010       _unzCloseCurrentFile       0043d010 f   unzip.obj
 0001:0003c070       _unzClose                  0043d070 f   unzip.obj
 0001:0003c0b0       _unzOpenCurrentFile        0043d0b0 f   unzip.obj
 0001:0003c1e0       _VM_VM2C                   0043d1e0 f   vm.obj
 0001:0003c1f0       _VM_Debug                  0043d1f0 f   vm.obj
 0001:0003c200       _VM_ValueToSymbol          0043d200 f   vm.obj
 0001:0003c260       _VM_ValueToFunctionSymbol  0043d260 f   vm.obj
 0001:0003c290       _VM_SymbolToValue          0043d290 f   vm.obj
 0001:0003c2f0       _VM_SymbolForCompiledPointer 0043d2f0 f   vm.obj
 0001:0003c340       _ParseHex                  0043d340 f   vm.obj
 0001:0003c3a0       _VM_LoadSymbols            0043d3a0 f   vm.obj
 0001:0003c570       _VM_DllSyscall             0043d570 f   vm.obj
 0001:0003c590       _VM_Free                   0043d590 f   vm.obj
 0001:0003c5e0       _VM_Clear                  0043d5e0 f   vm.obj
 0001:0003c630       _VM_ArgPtr                 0043d630 f   vm.obj
 0001:0003c660       _VM_ExplicitArgPtr         0043d660 f   vm.obj
 0001:0003c690       _VM_Call                   0043d690 f   vm.obj
 0001:0003c7c0       _VM_VmProfile_f            0043d7c0 f   vm.obj
 0001:0003c8d0       _VM_VmInfo_f               0043d8d0 f   vm.obj
 0001:0003c970       _VM_LogSyscalls            0043d970 f   vm.obj
 0001:0003c9e0       _VM_Init                   0043d9e0 f   vm.obj
 0001:0003ca50       _VM_Create                 0043da50 f   vm.obj
 0001:0003cd60       _VM_Restart                0043dd60 f   vm.obj
 0001:0003cf00       _VM_Indent                 0043df00 f   vm_interpreted.obj
 0001:0003cf30       _VM_StackTrace             0043df30 f   vm_interpreted.obj
 0001:0003cf70       _VM_PrepareInterpreter     0043df70 f   vm_interpreted.obj
 0001:0003d0c0       _VM_CallInterpreted        0043e0c0 f   vm_interpreted.obj
 0001:0003d700       _AsmCall                   0043e700 f   vm_x86.obj
 0001:0003dab0       _EmitMovEBXEDI             0043eab0 f   vm_x86.obj
 0001:0003db80       _VM_Compile                0043eb80 f   vm_x86.obj
 0001:0003f080       _VM_CallCompiled           00440080 f   vm_x86.obj
 0001:0003f190       _IN_InitWin32Mouse         00440190 f   win_input.obj
 0001:0003f1a0       _IN_ShutdownWin32Mouse     004401a0 f   win_input.obj
 0001:0003f1b0       _IN_ActivateWin32Mouse     004401b0 f   win_input.obj
 0001:0003f270       _IN_DeactivateWin32Mouse   00440270 f   win_input.obj
 0001:0003f290       _IN_Win32Mouse             00440290 f   win_input.obj
 0001:0003f2e0       _IN_ShutdownDIMouse        004402e0 f   win_input.obj
 0001:0003f320       _IN_DeactivateDIMouse      00440320 f   win_input.obj
 0001:0003f330       _IN_DIMouse                00440330 f   win_input.obj
 0001:0003f5b0       _IN_DeactivateMouse        004405b0 f   win_input.obj
 0001:0003f600       _IN_MouseEvent             00440600 f   win_input.obj
 0001:0003f690       _IN_MouseMove              00440690 f   win_input.obj
 0001:0003f710       _IN_Activate               00440710 f   win_input.obj
 0001:0003f730       _IN_ClearStates            00440730 f   win_input.obj
 0001:0003f740       _IN_StartupJoystick        00440740 f   win_input.obj
 0001:0003f8e0       _JoyToF                    004408e0 f   win_input.obj
 0001:0003f930       _JoyToI                    00440930 f   win_input.obj
 0001:0003f940       _IN_JoyMove                00440940 f   win_input.obj
 0001:0003ff80       _IN_InitDIMouse            00440f80 f   win_input.obj
 0001:00040130       _IN_ActivateDIMouse        00441130 f   win_input.obj
 0001:00040170       _IN_ActivateMouse          00441170 f   win_input.obj
 0001:000401b0       _IN_StartupMouse           004411b0 f   win_input.obj
 0001:00040280       _IN_Startup                00441280 f   win_input.obj
 0001:000402c0       _IN_Shutdown               004412c0 f   win_input.obj
 0001:00040330       _IN_Init                   00441330 f   win_input.obj
 0001:00040460       _IN_Frame                  00441460 f   win_input.obj
 0001:00040500       _Spk_Open                  00441500 f   win_main.obj
 0001:00040520       _Spk_Close                 00441520 f   win_main.obj
 0001:00040540       _Spk_Printf                00441540 f   win_main.obj
 0001:000405b0       _Sys_LowPhysicalMemory     004415b0 f   win_main.obj
 0001:000405d0       _Sys_BeginProfiling        004415d0 f   win_main.obj
 0001:000405e0       _Sys_Error                 004415e0 f   win_main.obj
 0001:00040680       _Sys_Quit                  00441680 f   win_main.obj
 0001:000406a0       _Sys_Print                 004416a0 f   win_main.obj
 0001:000406b0       _Sys_Mkdir                 004416b0 f   win_main.obj
 0001:000406c0       _Sys_Cwd                   004416c0 f   win_main.obj
 0001:000406e0       _Sys_DefaultCDPath         004416e0 f   win_main.obj
 0001:000406f0       _Sys_DefaultBasePath       004416f0 f   win_main.obj
 0001:00040710       _Sys_ListFilteredFiles     00441710 f   win_main.obj
 0001:00040960       _Sys_ListFiles             00441960 f   win_main.obj
 0001:00040bc0       _Sys_FreeFileList          00441bc0 f   win_main.obj
 0001:00040c00       _Sys_ScanForCD             00441c00 f   win_main.obj
 0001:00040d00       _Sys_CheckCD               00441d00 f   win_main.obj
 0001:00040d10       _Sys_GetClipboardData      00441d10 f   win_main.obj
 0001:00040d90       _Sys_UnloadDll             00441d90 f   win_main.obj
 0001:00040dc0       _Sys_LoadDll               00441dc0 f   win_main.obj
 0001:00040f20       _Sys_InitStreamThread      00441f20 f   win_main.obj
 0001:00040f30       _Sys_ShutdownStreamThread  00441f30 f   win_main.obj
 0001:00040f40       _Sys_BeginStreamedFile     00441f40 f   win_main.obj
 0001:00040f50       _Sys_EndStreamedFile       00441f50 f   win_main.obj
 0001:00040f60       _Sys_StreamedRead          00441f60 f   win_main.obj
 0001:00040f80       _Sys_StreamSeek            00441f80 f   win_main.obj
 0001:00040f90       _Sys_QueEvent              00441f90 f   win_main.obj
 0001:00041020       _Sys_GetEvent              00442020 f   win_main.obj
 0001:00041240       _Sys_In_Restart_f          00442240 f   win_main.obj
 0001:00041250       _Sys_Net_Restart_f         00442250 f   win_main.obj
 0001:00041260       _Sys_Init                  00442260 f   win_main.obj
 0001:00041640       _WinMain@16                00442640 f   win_main.obj
 0001:00041740       _NET_ErrorString           00442740 f   win_net.obj
 0001:00041990       _NetadrToSockadr           00442990 f   win_net.obj
 0001:00041a30       _SockadrToNetadr           00442a30 f   win_net.obj
 0001:00041a90       _Sys_StringToSockaddr      00442a90 f   win_net.obj
 0001:00041cf0       _Sys_StringToAdr           00442cf0 f   win_net.obj
 0001:00041d30       _Sys_GetPacket             00442d30 f   win_net.obj
 0001:00041f00       _Sys_SendPacket            00442f00 f   win_net.obj
 0001:00042040       _Sys_IsLANAddress          00443040 f   win_net.obj
 0001:00042170       _Sys_ShowIP                00443170 f   win_net.obj
 0001:000421c0       _NET_IPSocket              004431c0 f   win_net.obj
 0001:00042330       _NET_OpenSocks             00443330 f   win_net.obj
 0001:00042700       _NET_GetLocalAddress       00443700 f   win_net.obj
 0001:00042820       _NET_OpenIP                00443820 f   win_net.obj
 0001:000428d0       _NET_IPXSocket             004438d0 f   win_net.obj
 0001:000429f0       _NET_OpenIPX               004439f0 f   win_net.obj
 0001:00042b80       _NET_Config                00443b80 f   win_net.obj
 0001:00042c70       _NET_Init                  00443c70 f   win_net.obj
 0001:00042cc0       _NET_Shutdown              00443cc0 f   win_net.obj
 0001:00042cf0       _NET_Sleep                 00443cf0 f   win_net.obj
 0001:00042d00       _NET_Restart               00443d00 f   win_net.obj
 0001:00042d10       _Sys_Milliseconds          00443d10 f   win_shared.obj
 0001:00042d40       _fastftol                  00443d40 f   win_shared.obj
 0001:00042d50       _Sys_SnapVector            00443d50 f   win_shared.obj
 0001:00042f30       _Sys_GetProcessorId        00443f30 f   win_shared.obj
 0001:00042f80       _Sys_GetCurrentUser        00443f80 f   win_shared.obj
 0001:00042ff0       _Sys_DefaultHomePath       00443ff0 f   win_shared.obj
 0001:00043000       _Sys_DefaultInstallPath    00444000 f   win_shared.obj
 0001:00043050       _SNDDMA_Shutdown           00444050 f   win_snd.obj
 0001:00043190       _SNDDMA_GetDMAPos          00444190 f   win_snd.obj
 0001:000431e0       _SNDDMA_BeginPainting      004441e0 f   win_snd.obj
 0001:000432e0       _SNDDMA_Submit             004442e0 f   win_snd.obj
 0001:00043310       _SNDDMA_Activate           00444310 f   win_snd.obj
 0001:00043340       _SNDDMA_InitDS             00444340 f   win_snd.obj
 0001:00043630       _SNDDMA_Init               00444630 f   win_snd.obj
 0001:00043690       _InputLineWndProc@16       00444690 f   win_syscon.obj
 0001:000437b0       _Sys_DestroyConsole        004447b0 f   win_syscon.obj
 0001:000437f0       _Sys_ShowConsole           004447f0 f   win_syscon.obj
 0001:00043870       _Sys_ConsoleInput          00444870 f   win_syscon.obj
 0001:000438a0       _Conbuf_AppendText         004448a0 f   win_syscon.obj
 0001:000439f0       _Sys_SetErrorText          004449f0 f   win_syscon.obj
 0001:00043e60       _Sys_CreateConsole         00444e60 f   win_syscon.obj
 0001:00044460       _MainWndProc@16            00445460 f   win_wndproc.obj
 0001:0004497c       _joyGetDevCapsA@12         0044597c f   winmm:WINMM.dll
 0001:00044982       _joyGetPosEx@8             00445982 f   winmm:WINMM.dll
 0001:00044988       _joyGetNumDevs@0           00445988 f   winmm:WINMM.dll
 0001:0004498e       _midiInStart@4             0044598e f   winmm:WINMM.dll
 0001:00044994       _midiInOpen@20             00445994 f   winmm:WINMM.dll
 0001:0004499a       _midiInGetDevCapsA@12      0044599a f   winmm:WINMM.dll
 0001:000449a0       _midiInGetNumDevs@0        004459a0 f   winmm:WINMM.dll
 0001:000449a6       _midiInClose@4             004459a6 f   winmm:WINMM.dll
 0001:000449ac       _timeEndPeriod@4           004459ac f   winmm:WINMM.dll
 0001:000449b2       _timeGetTime@0             004459b2 f   winmm:WINMM.dll
 0001:000449b8       _timeBeginPeriod@4         004459b8 f   winmm:WINMM.dll
 0001:000449be       _WSAGetLastError@0         004459be f   wsock32:WSOCK32.dll
 0001:000449c4       _gethostbyname@4           004459c4 f   wsock32:WSOCK32.dll
 0001:000449ca       _inet_addr@4               004459ca f   wsock32:WSOCK32.dll
 0001:000449d0       _recvfrom@24               004459d0 f   wsock32:WSOCK32.dll
 0001:000449d6       _sendto@24                 004459d6 f   wsock32:WSOCK32.dll
 0001:000449dc       _closesocket@4             004459dc f   wsock32:WSOCK32.dll
 0001:000449e2       _bind@12                   004459e2 f   wsock32:WSOCK32.dll
 0001:000449e8       _htons@4                   004459e8 f   wsock32:WSOCK32.dll
 0001:000449ee       _setsockopt@20             004459ee f   wsock32:WSOCK32.dll
 0001:000449f4       _ioctlsocket@12            004459f4 f   wsock32:WSOCK32.dll
 0001:000449fa       _socket@12                 004459fa f   wsock32:WSOCK32.dll
 0001:00044a00       _recv@16                   00445a00 f   wsock32:WSOCK32.dll
 0001:00044a06       _send@16                   00445a06 f   wsock32:WSOCK32.dll
 0001:00044a0c       _connect@12                00445a0c f   wsock32:WSOCK32.dll
 0001:00044a12       _ntohl@4                   00445a12 f   wsock32:WSOCK32.dll
 0001:00044a18       _gethostname@8             00445a18 f   wsock32:WSOCK32.dll
 0001:00044a1e       _WSAStartup@8              00445a1e f   wsock32:WSOCK32.dll
 0001:00044a24       _WSACleanup@0              00445a24 f   wsock32:WSOCK32.dll
 0001:00044a2a       _GetProcAddress@8          00445a2a f   kernel32:KERNEL32.dll
 0001:00044a30       _LoadLibraryA@4            00445a30 f   kernel32:KERNEL32.dll
 0001:00044a36       _GlobalMemoryStatus@4      00445a36 f   kernel32:KERNEL32.dll
 0001:00044a3c       _GetDriveTypeA@4           00445a3c f   kernel32:KERNEL32.dll
 0001:00044a42       _GlobalUnlock@4            00445a42 f   kernel32:KERNEL32.dll
 0001:00044a48       _GlobalSize@4              00445a48 f   kernel32:KERNEL32.dll
 0001:00044a4e       _GlobalLock@4              00445a4e f   kernel32:KERNEL32.dll
 0001:00044a54       _FreeLibrary@4             00445a54 f   kernel32:KERNEL32.dll
 0001:00044a5a       _GetVersionExA@4           00445a5a f   kernel32:KERNEL32.dll
 0001:00044a60       _Sleep@4                   00445a60 f   kernel32:KERNEL32.dll
 0001:00044a66       _SetErrorMode@4            00445a66 f   kernel32:KERNEL32.dll
 0001:00044a6c       _MulDiv@12                 00445a6c f   kernel32:KERNEL32.dll
 0001:00044a72       _ShowCursor@4              00445a72 f   user32:USER32.dll
 0001:00044a78       _ClipCursor@4              00445a78 f   user32:USER32.dll
 0001:00044a7e       _SetCapture@4              00445a7e f   user32:USER32.dll
 0001:00044a84       _SetCursorPos@8            00445a84 f   user32:USER32.dll
 0001:00044a8a       _GetWindowRect@8           00445a8a f   user32:USER32.dll
 0001:00044a90       _GetSystemMetrics@4        00445a90 f   user32:USER32.dll
 0001:00044a96       _ReleaseCapture@0          00445a96 f   user32:USER32.dll
 0001:00044a9c       _GetCursorPos@4            00445a9c f   user32:USER32.dll
 0001:00044aa2       _DispatchMessageA@4        00445aa2 f   user32:USER32.dll
 0001:00044aa8       _TranslateMessage@4        00445aa8 f   user32:USER32.dll
 0001:00044aae       _GetMessageA@16            00445aae f   user32:USER32.dll
 0001:00044ab4       _CloseClipboard@0          00445ab4 f   user32:USER32.dll
 0001:00044aba       _GetClipboardData@4        00445aba f   user32:USER32.dll
 0001:00044ac0       _OpenClipboard@4           00445ac0 f   user32:USER32.dll
 0001:00044ac6       _MessageBoxExA@20          00445ac6 f   user32:USER32.dll
 0001:00044acc       _PeekMessageA@20           00445acc f   user32:USER32.dll
 0001:00044ad2       _SetFocus@4                00445ad2 f   user32:USER32.dll
 0001:00044ad8       _CallWindowProcA@20        00445ad8 f   user32:USER32.dll
 0001:00044ade       _SetWindowTextA@8          00445ade f   user32:USER32.dll
 0001:00044ae4       _GetWindowTextA@12         00445ae4 f   user32:USER32.dll
 0001:00044aea       _DestroyWindow@4           00445aea f   user32:USER32.dll
 0001:00044af0       _CloseWindow@4             00445af0 f   user32:USER32.dll
 0001:00044af6       _ShowWindow@8              00445af6 f   user32:USER32.dll
 0001:00044afc       _SendMessageA@16           00445afc f   user32:USER32.dll
 0001:00044b02       _CreateWindowExA@48        00445b02 f   user32:USER32.dll
 0001:00044b08       _UpdateWindow@4            00445b08 f   user32:USER32.dll
 0001:00044b0e       _InvalidateRect@12         00445b0e f   user32:USER32.dll
 0001:00044b14       _SetTimer@16               00445b14 f   user32:USER32.dll
 0001:00044b1a       _DefWindowProcA@16         00445b1a f   user32:USER32.dll
 0001:00044b20       _PostQuitMessage@4         00445b20 f   user32:USER32.dll
 0001:00044b26       _SetForegroundWindow@4     00445b26 f   user32:USER32.dll
 0001:00044b2c       _SetWindowLongA@12         00445b2c f   user32:USER32.dll
 0001:00044b32       _ReleaseDC@8               00445b32 f   user32:USER32.dll
 0001:00044b38       _GetDC@4                   00445b38 f   user32:USER32.dll
 0001:00044b3e       _GetDesktopWindow@0        00445b3e f   user32:USER32.dll
 0001:00044b44       _AdjustWindowRect@12       00445b44 f   user32:USER32.dll
 0001:00044b4a       _RegisterClassA@4          00445b4a f   user32:USER32.dll
 0001:00044b50       _LoadCursorA@8             00445b50 f   user32:USER32.dll
 0001:00044b56       _LoadIconA@8               00445b56 f   user32:USER32.dll
 0001:00044b5c       _SystemParametersInfoA@16  00445b5c f   user32:USER32.dll
 0001:00044b62       _RegisterHotKey@16         00445b62 f   user32:USER32.dll
 0001:00044b68       _UnregisterHotKey@8        00445b68 f   user32:USER32.dll
 0001:00044b6e       _RegisterWindowMessageA@4  00445b6e f   user32:USER32.dll
 0001:00044b74       _GetWindowLongA@8          00445b74 f   user32:USER32.dll
 0001:00044b7a       _SetTextColor@8            00445b7a f   gdi32:GDI32.dll
 0001:00044b80       _SetBkColor@8              00445b80 f   gdi32:GDI32.dll
 0001:00044b86       _CreateSolidBrush@4        00445b86 f   gdi32:GDI32.dll
 0001:00044b8c       _CreateFontA@56            00445b8c f   gdi32:GDI32.dll
 0001:00044b92       _GetDeviceCaps@8           00445b92 f   gdi32:GDI32.dll
 0001:00044b98       _GetUserNameA@8            00445b98 f   advapi32:ADVAPI32.dll
 0001:00044b9e       _CoUninitialize@0          00445b9e f   ole32:ole32.dll
 0001:00044ba4       _CoCreateInstance@20       00445ba4 f   ole32:ole32.dll
 0001:00044baa       _CoInitialize@4            00445baa f   ole32:ole32.dll
 0001:00044cb0       _GL_CheckErrors            00445cb0 f   renderer:tr_init.obj
 0001:00044e70       _R_GetModeInfo             00445e70 f   renderer:tr_init.obj
 0001:00044f50       _RB_TakeScreenshot         00445f50 f   renderer:tr_init.obj
 0001:00045040       _RB_TakeScreenshotJPEG     00446040 f   renderer:tr_init.obj
 0001:000450e0       _RB_TakeScreenshotCmd      004460e0 f   renderer:tr_init.obj
 0001:00045130       _R_TakeScreenshot          00446130 f   renderer:tr_init.obj
 0001:00045190       _R_ScreenshotFilename      00446190 f   renderer:tr_init.obj
 0001:00045230       _R_ScreenshotFilenameJPEG  00446230 f   renderer:tr_init.obj
 0001:000452d0       _R_LevelShot               004462d0 f   renderer:tr_init.obj
 0001:00045520       _R_ScreenShot_f            00446520 f   renderer:tr_init.obj
 0001:000456a0       _R_ScreenShotJPEG_f        004466a0 f   renderer:tr_init.obj
 0001:00045820       _GL_SetDefaultState        00446820 f   renderer:tr_init.obj
 0001:00045c60       _R_Register                00446c60 f   renderer:tr_init.obj
 0001:00046650       _RE_Shutdown               00447650 f   renderer:tr_init.obj
 0001:00046700       _RE_EndRegistration        00447700 f   renderer:tr_init.obj
 0001:00046720       _GetRefAPI                 00447720 f   renderer:tr_init.obj
 0001:00046910       _R_Init                    00447910 f   renderer:tr_init.obj
 0001:00046b90       _R_CullLocalBox            00447b90 f   renderer:tr_main.obj
 0001:00047230       _R_CullPointAndRadius      00448230 f   renderer:tr_main.obj
 0001:000472c0       _R_LocalNormalToWorld      004482c0 f   renderer:tr_main.obj
 0001:00047330       _R_LocalPointToWorld       00448330 f   renderer:tr_main.obj
 0001:000473b0       _R_WorldToLocal            004483b0 f   renderer:tr_main.obj
 0001:00047420       _R_TransformModelToClip    00448420 f   renderer:tr_main.obj
 0001:00047520       _R_TransformClipToWindow   00448520 f   renderer:tr_main.obj
 0001:000475c0       _myGlMultMatrix            004485c0 f   renderer:tr_main.obj
 0001:00047670       _R_RotateForEntity         00448670 f   renderer:tr_main.obj
 0001:00047830       _R_RotateForViewer         00448830 f   renderer:tr_main.obj
 0001:00047cb0       _R_SetupProjection         00448cb0 f   renderer:tr_main.obj
 0001:00047e00       _R_SetupFrustum            00448e00 f   renderer:tr_main.obj
 0001:00047fe0       _R_MirrorPoint             00448fe0 f   renderer:tr_main.obj
 0001:000480c0       _R_MirrorVector            004490c0 f   renderer:tr_main.obj
 0001:00048170       _R_PlaneForSurface         00449170 f   renderer:tr_main.obj
 0001:00048270       _R_GetPortalOrientations   00449270 f   renderer:tr_main.obj
 0001:00048880       _R_SpriteFogNum            00449880 f   renderer:tr_main.obj
 0001:00048960       _qsortFast                 00449960 f   renderer:tr_main.obj
 0001:00048ab0       _R_AddDrawSurf             00449ab0 f   renderer:tr_main.obj
 0001:00048b00       _R_DecomposeSort           00449b00 f   renderer:tr_main.obj
 0001:00048b50       _R_AddEntitySurfaces       00449b50 f   renderer:tr_main.obj
 0001:00048d10       _R_GenerateDrawSurfs       00449d10 f   renderer:tr_main.obj
 0001:00048d30       _R_DebugPolygon            00449d30 f   renderer:tr_main.obj
 0001:00048e30       _R_DebugGraphics           00449e30 f   renderer:tr_main.obj
 0001:00048e70       _R_CullLocalPointAndRadius 00449e70 f   renderer:tr_main.obj
 0001:000490e0       _R_MirrorViewBySurface     0044a0e0 f   renderer:tr_main.obj
 0001:000492a0       _R_SortDrawSurfs           0044a2a0 f   renderer:tr_main.obj
 0001:00049380       _R_RenderView              0044a380 f   renderer:tr_main.obj
 0001:0004cac0       _QGL_Shutdown              0044dac0 f   renderer:win_qgl.obj
 0001:0004d380       _QGL_EnableLogging         0044e380 f   renderer:win_qgl.obj
 0001:0004f0c0       _QGL_Init                  004500c0 f   renderer:win_qgl.obj
 0001:00051280       _R_GammaCorrect            00452280 f   renderer:tr_image.obj
 0001:00051300       _GL_TextureMode            00452300 f   renderer:tr_image.obj
 0001:00051400       _R_SumOfUsedImages         00452400 f   renderer:tr_image.obj
 0001:00051440       _R_ImageList_f             00452440 f   renderer:tr_image.obj
 0001:000517d0       _R_LightScaleTexture       004527d0 f   renderer:tr_image.obj
 0001:00052220       _R_CreateImage             00453220 f   renderer:tr_image.obj
 0001:00052f20       _init_destination          00453f20 f   renderer:tr_image.obj
 0001:00052f40       _empty_output_buffer       00453f40 f   renderer:tr_image.obj
 0001:00052f50       _jpeg_start_compress       00453f50 f   renderer:tr_image.obj
 0001:00052fd0       _jpeg_write_scanlines      00453fd0 f   renderer:tr_image.obj
 0001:000530a0       _term_destination          004540a0 f   renderer:tr_image.obj
 0001:000530c0       _jpegDest                  004540c0 f   renderer:tr_image.obj
 0001:00053110       _SaveJPG                   00454110 f   renderer:tr_image.obj
 0001:000532e0       _R_LoadImage               004542e0 f   renderer:tr_image.obj
 0001:00053430       _R_FindImageFile           00454430 f   renderer:tr_image.obj
 0001:000536c0       _R_InitFogTable            004546c0 f   renderer:tr_image.obj
 0001:00053700       _R_FogFactor               00454700 f   renderer:tr_image.obj
 0001:00053950       _R_CreateBuiltinImages     00454950 f   renderer:tr_image.obj
 0001:00053a30       _R_SetColorMappings        00454a30 f   renderer:tr_image.obj
 0001:00053c30       _R_InitImages              00454c30 f   renderer:tr_image.obj
 0001:00053c50       _R_DeleteTextures          00454c50 f   renderer:tr_image.obj
 0001:00053e10       _RE_RegisterSkin           00454e10 f   renderer:tr_image.obj
 0001:00054060       _R_InitSkins               00455060 f   renderer:tr_image.obj
 0001:000540b0       _R_GetSkinByHandle         004550b0 f   renderer:tr_image.obj
 0001:000540d0       _R_SkinList_f              004550d0 f   renderer:tr_image.obj
 0001:00054160       _R_PerformanceCounters     00455160 f   renderer:tr_cmds.obj
 0001:00054380       _R_InitCommandBuffers      00455380 f   renderer:tr_cmds.obj
 0001:000543e0       _R_ShutdownCommandBuffers  004553e0 f   renderer:tr_cmds.obj
 0001:00054400       _R_IssueRenderCommands     00455400 f   renderer:tr_cmds.obj
 0001:000544d0       _R_SyncRenderThread        004554d0 f   renderer:tr_cmds.obj
 0001:00054500       _R_GetCommandBuffer        00455500 f   renderer:tr_cmds.obj
 0001:00054560       _R_AddDrawSurfCmd          00455560 f   renderer:tr_cmds.obj
 0001:000545e0       _RE_SetColor               004555e0 f   renderer:tr_cmds.obj
 0001:00054650       _RE_StretchPic             00455650 f   renderer:tr_cmds.obj
 0001:000546f0       _RE_BeginFrame             004556f0 f   renderer:tr_cmds.obj
 0001:00054980       _RE_EndFrame               00455980 f   renderer:tr_cmds.obj
 0001:00054a10       _GL_Bind                   00455a10 f   renderer:tr_backend.obj
 0001:00054a90       _GL_SelectTexture          00455a90 f   renderer:tr_backend.obj
 0001:00054b40       _GL_BindMultitexture       00455b40 f   renderer:tr_backend.obj
 0001:00054c40       _GL_Cull                   00455c40 f   renderer:tr_backend.obj
 0001:00054ca0       _GL_TexEnv                 00455ca0 f   renderer:tr_backend.obj
 0001:00054d50       _GL_State                  00455d50 f   renderer:tr_backend.obj
 0001:00055120       _RB_BeginDrawingView       00456120 f   renderer:tr_backend.obj
 0001:000552f0       _RB_RenderDrawSurfList     004562f0 f   renderer:tr_backend.obj
 0001:000555b0       _RB_SetGL2D                004565b0 f   renderer:tr_backend.obj
 0001:00055690       _RE_StretchRaw             00456690 f   renderer:tr_backend.obj
 0001:00055970       _RE_UploadCinematic        00456970 f   renderer:tr_backend.obj
 0001:00055a80       _RB_SetColor               00456a80 f   renderer:tr_backend.obj
 0001:00055ae0       _RB_StretchPic             00456ae0 f   renderer:tr_backend.obj
 0001:00055c90       _RB_DrawSurfs              00456c90 f   renderer:tr_backend.obj
 0001:00055cf0       _RB_DrawBuffer             00456cf0 f   renderer:tr_backend.obj
 0001:00055d40       _RB_ShowImages             00456d40 f   renderer:tr_backend.obj
 0001:00055f00       _RB_SwapBuffers            00456f00 f   renderer:tr_backend.obj
 0001:00055fe0       _RB_ExecuteRenderCommands  00456fe0 f   renderer:tr_backend.obj
 0001:00056170       _RB_RenderThread           00457170 f   renderer:tr_backend.obj
 0001:000561b0       _R_GetModelByHandle        004571b0 f   renderer:tr_model.obj
 0001:000561d0       _R_AllocModel              004571d0 f   renderer:tr_model.obj
 0001:00056690       _RE_BeginRegistration      00457690 f   renderer:tr_model.obj
 0001:000566f0       _R_ModelInit               004576f0 f   renderer:tr_model.obj
 0001:00056740       _R_Modellist_f             00457740 f   renderer:tr_model.obj
 0001:00056840       _R_LerpTag                 00457840 f   renderer:tr_model.obj
 0001:000569e0       _R_ModelBounds             004579e0 f   renderer:tr_model.obj
 0001:00056aa0       _RE_RegisterModel          00457aa0 f   renderer:tr_model.obj
 0001:00058700       _ParseSort                 00459700 f   renderer:tr_shader.obj
 0001:000599e0       _R_FindShaderByName        0045a9e0 f   renderer:tr_shader.obj
 0001:00059a50       _R_FindShader              0045aa50 f   renderer:tr_shader.obj
 0001:00059d50       _RE_RegisterShaderFromImage 0045ad50 f   renderer:tr_shader.obj
 0001:00059f50       _RE_RegisterShaderLightMap 0045af50 f   renderer:tr_shader.obj
 0001:00059fa0       _RE_RegisterShader         0045afa0 f   renderer:tr_shader.obj
 0001:00059ff0       _RE_RegisterShaderNoMip    0045aff0 f   renderer:tr_shader.obj
 0001:0005a040       _R_GetShaderByHandle       0045b040 f   renderer:tr_shader.obj
 0001:0005a070       _R_ShaderList_f            0045b070 f   renderer:tr_shader.obj
 0001:0005a5e0       _R_InitShaders             0045b5e0 f   renderer:tr_shader.obj
 0001:0005a650       _R_RemapShader             0045b650 f   renderer:tr_shader.obj
 0001:0005ba30       _GLimp_EndFrame            0045ca30 f   renderer:win_glimp.obj
 0001:0005bae0       _GLimp_Shutdown            0045cae0 f   renderer:win_glimp.obj
 0001:0005bc70       _GLimp_LogComment          0045cc70 f   renderer:win_glimp.obj
 0001:0005bc90       _GLimp_RenderThreadWrapper 0045cc90 f   renderer:win_glimp.obj
 0001:0005bcb0       _GLimp_SpawnRenderThread   0045ccb0 f   renderer:win_glimp.obj
 0001:0005bd20       _GLimp_RendererSleep       0045cd20 f   renderer:win_glimp.obj
 0001:0005bdb0       _GLimp_FrontEndSleep       0045cdb0 f   renderer:win_glimp.obj
 0001:0005bde0       _GLimp_WakeRenderer        0045cde0 f   renderer:win_glimp.obj
 0001:0005c0c0       _GLimp_Init                0045d0c0 f   renderer:win_glimp.obj
 0001:0005c460       _readInt                   0045d460 f   renderer:tr_font.obj
 0001:0005c4a0       _readFloat                 0045d4a0 f   renderer:tr_font.obj
 0001:0005c4e0       _RE_RegisterFont           0045d4e0 f   renderer:tr_font.obj
 0001:0005c8c0       _R_InitFreeType            0045d8c0 f   renderer:tr_font.obj
 0001:0005c8d0       _R_DoneFreeType            0045d8d0 f   renderer:tr_font.obj
 0001:0005d000       _R_AddBrushModelSurfaces   0045e000 f   renderer:tr_world.obj
 0001:0005d470       _R_inPVS                   0045e470 f   renderer:tr_world.obj
 0001:0005d640       _R_AddWorldSurfaces        0045e640 f   renderer:tr_world.obj
 0001:0005dac0       _RE_SetWorldVisData        0045eac0 f   renderer:tr_bsp.obj
 0001:0005e350       _R_MergedWidthPoints       0045f350 f   renderer:tr_bsp.obj
 0001:0005e3e0       _R_MergedHeightPoints      0045f3e0 f   renderer:tr_bsp.obj
 0001:0005e500       _R_FixSharedVertexLodError_r 0045f500 f   renderer:tr_bsp.obj
 0001:0005e9f0       _R_FixSharedVertexLodError 0045f9f0 f   renderer:tr_bsp.obj
 0001:0005ea40       _R_StitchPatches           0045fa40 f   renderer:tr_bsp.obj
 0001:0005faf0       _R_TryStitchingPatch       00460af0 f   renderer:tr_bsp.obj
 0001:0005fbb0       _R_StitchAllPatches        00460bb0 f   renderer:tr_bsp.obj
 0001:0005fc20       _R_MovePatchSurfacesToHunk 00460c20 f   renderer:tr_bsp.obj
 0001:000606a0       _R_LoadLightGrid           004616a0 f   renderer:tr_bsp.obj
 0001:00060800       _R_LoadEntities            00461800 f   renderer:tr_bsp.obj
 0001:00060a40       _R_GetEntityToken          00461a40 f   renderer:tr_bsp.obj
 0001:00060a90       _RE_LoadWorldMap           00461a90 f   renderer:tr_bsp.obj
 0001:00060c50       _R_ToggleSmpFrame          00461c50 f   renderer:tr_scene.obj
 0001:00060cb0       _RE_ClearScene             00461cb0 f   renderer:tr_scene.obj
 0001:00060ce0       _R_AddPolygonSurfaces      00461ce0 f   renderer:tr_scene.obj
 0001:00060d30       _RE_AddPolyToScene         00461d30 f   renderer:tr_scene.obj
 0001:00061160       _RE_AddRefEntityToScene    00462160 f   renderer:tr_scene.obj
 0001:000611f0       _RE_AddDynamicLightToScene 004621f0 f   renderer:tr_scene.obj
 0001:00061280       _RE_AddLightToScene        00462280 f   renderer:tr_scene.obj
 0001:000612b0       _RE_AddAdditiveLightToScene 004622b0 f   renderer:tr_scene.obj
 0001:000612e0       _RE_RenderScene            004622e0 f   renderer:tr_scene.obj
 0001:000616e0       _R_TransformDlights        004626e0 f   renderer:tr_light.obj
 0001:000618f0       _R_DlightBmodel            004628f0 f   renderer:tr_light.obj
 0001:00061e80       _R_SetupEntityLighting     00462e80 f   renderer:tr_light.obj
 0001:00062200       _R_LightForPoint           00463200 f   renderer:tr_light.obj
 0001:00062550       _R_BoxSurfaces_r           00463550 f   renderer:tr_marks.obj
 0001:000626c0       _R_AddMarkFragments        004636c0 f   renderer:tr_marks.obj
 0001:000627b0       _R_MarkFragments           004637b0 f   renderer:tr_marks.obj
 0001:00063280       _R_NoiseInit               00464280 f   renderer:tr_noise.obj
 0001:000632f0       _R_NoiseGet4f              004642f0 f   renderer:tr_noise.obj
 0001:00063a50       _RB_BeginSurface           00464a50 f   renderer:tr_shade.obj
 0001:00064a60       _RB_StageIteratorGeneric   00465a60 f   renderer:tr_shade.obj
 0001:00064c40       _RB_StageIteratorVertexLitTexture 00465c40 f   renderer:tr_shade.obj
 0001:00064d90       _RB_StageIteratorLightmappedMultitexture 00465d90 f   renderer:tr_shade.obj
 0001:00064f50       _RB_EndSurface             00465f50 f   renderer:tr_shade.obj
 0001:00065070       _R_AddAnimSurfaces         00466070 f   renderer:tr_animation.obj
 0001:000650c0       _RB_SurfaceAnim            004660c0 f   renderer:tr_animation.obj
 0001:00065700       _R_ComputeLOD              00466700 f   renderer:tr_mesh.obj
 0001:000657e0       _R_ComputeFogNum           004667e0 f   renderer:tr_mesh.obj
 0001:000658a0       _R_AddMD3Surfaces          004668a0 f   renderer:tr_mesh.obj
 0001:00065b80       _RB_CheckOverflow          00466b80 f   renderer:tr_surface.obj
 0001:00065c10       _RB_AddQuadStampExt        00466c10 f   renderer:tr_surface.obj
 0001:00065f40       _RB_AddQuadStamp           00466f40 f   renderer:tr_surface.obj
 0001:00066100       _RB_SurfacePolychain       00467100 f   renderer:tr_surface.obj
 0001:00066220       _RB_SurfaceTriangles       00467220 f   renderer:tr_surface.obj
 0001:00066400       _RB_SurfaceBeam            00467400 f   renderer:tr_surface.obj
 0001:00066de0       _RB_SurfaceRailRings       00467de0 f   renderer:tr_surface.obj
 0001:00066eb0       _RB_SurfaceRailCore        00467eb0 f   renderer:tr_surface.obj
 0001:00067010       _RB_SurfaceLightningBolt   00468010 f   renderer:tr_surface.obj
 0001:000677a0       _RB_SurfaceMesh            004687a0 f   renderer:tr_surface.obj
 0001:00067910       _RB_SurfaceFace            00468910 f   renderer:tr_surface.obj
 0001:00067c00       _RB_SurfaceGrid            00468c00 f   renderer:tr_surface.obj
 0001:000682c0       _RB_SurfaceAxis            004692c0 f   renderer:tr_surface.obj
 0001:00068380       _RB_SurfaceEntity          00469380 f   renderer:tr_surface.obj
 0001:000683d0       _RB_SurfaceBad             004693d0 f   renderer:tr_surface.obj
 0001:000683f0       _RB_SurfaceFlare           004693f0 f   renderer:tr_surface.obj
 0001:00068400       _RB_SurfaceDisplayList     00469400 f   renderer:tr_surface.obj
 0001:00068410       _RB_SurfaceSkip            00469410 f   renderer:tr_surface.obj
 0001:00068420       _jpeg_create_decompress    00469420 f   renderer:jdapimin.obj
 0001:000684b0       _jpeg_destroy_decompress   004694b0 f   renderer:jdapimin.obj
 0001:000684c0       _jpeg_abort_decompress     004694c0 f   renderer:jdapimin.obj
 0001:000684d0       _jpeg_set_marker_processor 004694d0 f   renderer:jdapimin.obj
 0001:000686c0       _jpeg_consume_input        004696c0 f   renderer:jdapimin.obj
 0001:00068780       _jpeg_input_complete       00469780 f   renderer:jdapimin.obj
 0001:000687d0       _jpeg_has_multiple_scans   004697d0 f   renderer:jdapimin.obj
 0001:00068820       _jpeg_finish_decompress    00469820 f   renderer:jdapimin.obj
 0001:000688e0       _jpeg_read_header          004698e0 f   renderer:jdapimin.obj
 0001:000689c0       _jpeg_read_scanlines       004699c0 f   renderer:jdapistd.obj
 0001:00068a60       _jpeg_read_raw_data        00469a60 f   renderer:jdapistd.obj
 0001:00068b10       _jpeg_start_decompress     00469b10 f   renderer:jdapistd.obj
 0001:00068c70       _jpeg_stdio_src            00469c70 f   renderer:jdatasrc.obj
 0001:00068e60       _jpeg_std_error            00469e60 f   renderer:jerror.obj
 0001:00068eb0       _jinit_compress_master     00469eb0 f   renderer:jcinit.obj
 0001:00068f70       _jpeg_create_compress      00469f70 f   renderer:jcapimin.obj
 0001:00068fe0       _jpeg_destroy_compress     00469fe0 f   renderer:jcapimin.obj
 0001:00068ff0       _jpeg_abort_compress       00469ff0 f   renderer:jcapimin.obj
 0001:00069000       _jpeg_suppress_tables      0046a000 f   renderer:jcapimin.obj
 0001:00069070       _jpeg_finish_compress      0046a070 f   renderer:jcapimin.obj
 0001:00069180       _jpeg_write_marker         0046a180 f   renderer:jcapimin.obj
 0001:000691e0       _jpeg_write_tables         0046a1e0 f   renderer:jcapimin.obj
 0001:00069240       _jpeg_add_quant_table      0046a240 f   renderer:jcparam.obj
 0001:000693f0       _jpeg_set_linear_quality   0046a3f0 f   renderer:jcparam.obj
 0001:00069430       _jpeg_quality_scaling      0046a430 f   renderer:jcparam.obj
 0001:00069470       _jpeg_set_quality          0046a470 f   renderer:jcparam.obj
 0001:000696c0       _jpeg_set_colorspace       0046a6c0 f   renderer:jcparam.obj
 0001:00069a80       _jpeg_simple_progression   0046aa80 f   renderer:jcparam.obj
 0001:00069cc0       _jpeg_default_colorspace   0046acc0 f   renderer:jcparam.obj
 0001:00069f70       _jpeg_set_defaults         0046af70 f   renderer:jcparam.obj
 0001:0006a070       _WG_CheckHardwareGamma     0046b070 f   renderer:win_gamma.obj
 0001:0006a1a0       _GLimp_SetGamma            0046b1a0 f   renderer:win_gamma.obj
 0001:0006a470       _WG_RestoreGamma           0046b470 f   renderer:win_gamma.obj
 0001:0006a4c0       _R_ClearFlares             0046b4c0 f   renderer:tr_flares.obj
 0001:0006a540       _RB_TestFlare              0046b540 f   renderer:tr_flares.obj
 0001:0006a660       _RB_RenderFlare            0046b660 f   renderer:tr_flares.obj
 0001:0006a9c0       _RB_RenderFlares           0046b9c0 f   renderer:tr_flares.obj
 0001:0006ab80       _RB_AddFlare               0046bb80 f   renderer:tr_flares.obj
 0001:0006add0       _RB_AddDlightFlares        0046bdd0 f   renderer:tr_flares.obj
 0001:0006ae90       _R_AddEdgeDef              0046be90 f   renderer:tr_shadows.obj
 0001:0006aed0       _R_RenderShadowEdges       0046bed0 f   renderer:tr_shadows.obj
 0001:0006b020       _RB_ShadowFinish           0046c020 f   renderer:tr_shadows.obj
 0001:0006b130       _RB_ProjectionShadowDeform 0046c130 f   renderer:tr_shadows.obj
 0001:0006b280       _RB_ShadowTessEnd          0046c280 f   renderer:tr_shadows.obj
 0001:0006bd00       _RB_ClipSkyPolygons        0046cd00 f   renderer:tr_sky.obj
 0001:0006c840       _R_BuildCloudData          0046d840 f   renderer:tr_sky.obj
 0001:0006c8b0       _R_InitSkyTexCoords        0046d8b0 f   renderer:tr_sky.obj
 0001:0006ca40       _RB_DrawSun                0046da40 f   renderer:tr_sky.obj
 0001:0006cef0       _RB_StageIteratorSky       0046def0 f   renderer:tr_sky.obj
 0001:0006dba0       _R_CreateSurfaceGridMesh   0046eba0 f   renderer:tr_curve.obj
 0001:0006dd50       _R_FreeSurfaceGridMesh     0046ed50 f   renderer:tr_curve.obj
 0001:0006dd80       _R_SubdividePatchToGrid    0046ed80 f   renderer:tr_curve.obj
 0001:0006e400       _R_GridInsertColumn        0046f400 f   renderer:tr_curve.obj
 0001:0006e680       _R_GridInsertRow           0046f680 f   renderer:tr_curve.obj
 0001:0006e9d0       _RB_CalcDeformNormals      0046f9d0 f   renderer:tr_shade_calc.obj
 0001:0006eb50       _RB_CalcBulgeVertexes      0046fb50 f   renderer:tr_shade_calc.obj
 0001:0006ebf0       _DeformText                0046fbf0 f   renderer:tr_shade_calc.obj
 0001:0006f830       _RB_CalcColorFromEntity    00470830 f   renderer:tr_shade_calc.obj
 0001:0006f870       _RB_CalcColorFromOneMinusEntity 00470870 f   renderer:tr_shade_calc.obj
 0001:0006f8e0       _RB_CalcAlphaFromEntity    004708e0 f   renderer:tr_shade_calc.obj
 0001:0006f920       _RB_CalcAlphaFromOneMinusEntity 00470920 f   renderer:tr_shade_calc.obj
 0001:0006f970       _RB_CalcFogTexCoords       00470970 f   renderer:tr_shade_calc.obj
 0001:0006fbd0       _RB_CalcEnvironmentTexCoords 00470bd0 f   renderer:tr_shade_calc.obj
 0001:0006fcd0       _RB_CalcTurbulentTexCoords 00470cd0 f   renderer:tr_shade_calc.obj
 0001:0006fd70       _RB_CalcScaleTexCoords     00470d70 f   renderer:tr_shade_calc.obj
 0001:0006fdb0       _RB_CalcScrollTexCoords    00470db0 f   renderer:tr_shade_calc.obj
 0001:0006fe40       _RB_CalcTransformTexCoords 00470e40 f   renderer:tr_shade_calc.obj
 0001:0006fe90       _RB_CalcRotateTexCoords    00470e90 f   renderer:tr_shade_calc.obj
 0001:0006ff30       _myftol                    00470f30 f   renderer:tr_shade_calc.obj
 0001:0006ff40       _RB_CalcSpecularAlpha      00470f40 f   renderer:tr_shade_calc.obj
 0001:000700d0       _RB_CalcDiffuseColor       004710d0 f   renderer:tr_shade_calc.obj
 0001:000702e0       _RB_CalcStretchTexCoords   004712e0 f   renderer:tr_shade_calc.obj
 0001:00070380       _RB_CalcDeformVertexes     00471380 f   renderer:tr_shade_calc.obj
 0001:00070500       _RB_CalcMoveVertexes       00471500 f   renderer:tr_shade_calc.obj
 0001:000705a0       _RB_DeformTessGeometry     004715a0 f   renderer:tr_shade_calc.obj
 0001:00070680       _RB_CalcWaveColor          00471680 f   renderer:tr_shade_calc.obj
 0001:00070780       _RB_CalcWaveAlpha          00471780 f   renderer:tr_shade_calc.obj
 0001:000707d0       _RB_CalcModulateColorsByFog 004717d0 f   renderer:tr_shade_calc.obj
 0001:00070870       _RB_CalcModulateAlphasByFog 00471870 f   renderer:tr_shade_calc.obj
 0001:000708f0       _RB_CalcModulateRGBAsByFog 004718f0 f   renderer:tr_shade_calc.obj
 0001:00070f50       _jinit_input_controller    00471f50 f   renderer:jdinput.obj
 0001:00072820       _jpeg_resync_to_restart    00473820 f   renderer:jdmarker.obj
 0001:00072960       _jinit_marker_reader       00473960 f   renderer:jdmarker.obj
 0001:00073540       _jinit_memory_mgr          00474540 f   renderer:jmemmgr.obj
 0001:00073660       _jpeg_abort                00474660 f   renderer:jcomapi.obj
 0001:00073690       _jpeg_destroy              00474690 f   renderer:jcomapi.obj
 0001:000736b0       _jpeg_alloc_quant_table    004746b0 f   renderer:jcomapi.obj
 0001:000736d0       _jpeg_alloc_huff_table     004746d0 f   renderer:jcomapi.obj
 0001:00073700       _jpeg_calc_output_dimensions 00474700 f   renderer:jdmaster.obj
 0001:00073b00       _jinit_master_decompress   00474b00 f   renderer:jdmaster.obj
 0001:000749b0       _jinit_marker_writer       004759b0 f   renderer:jcmarker.obj
 0001:00074b20       _jinit_c_main_controller   00475b20 f   renderer:jcmainct.obj
 0001:000753d0       _jinit_c_coef_controller   004763d0 f   renderer:jccoefct.obj
 0001:000754d0       _jpeg_make_c_derived_tbl   004764d0 f   renderer:jchuff.obj
 0001:00075d40       _jpeg_gen_optimal_table    00476d40 f   renderer:jchuff.obj
 0001:00076230       _jinit_huff_encoder        00477230 f   renderer:jchuff.obj
 0001:00076fc0       _jinit_phuff_encoder       00477fc0 f   renderer:jcphuff.obj
 0001:00077910       _jinit_forward_dct         00478910 f   renderer:jcdctmgr.obj
 0001:00078030       _jinit_c_prep_controller   00479030 f   renderer:jcprepct.obj
 0001:00078900       _jinit_downsampler         00479900 f   renderer:jcsample.obj
 0001:00078fa0       _jinit_color_converter     00479fa0 f   renderer:jccolor.obj
 0001:00079c80       _jinit_c_master_control    0047ac80 f   renderer:jcmaster.obj
 0001:00079d30       _jdiv_round_up             0047ad30 f   renderer:jutils.obj
 0001:00079d40       _jround_up                 0047ad40 f   renderer:jutils.obj
 0001:00079d60       _jcopy_sample_rows         0047ad60 f   renderer:jutils.obj
 0001:00079db0       _jcopy_block_row           0047adb0 f   renderer:jutils.obj
 0001:00079de0       _jzero_far                 0047ade0 f   renderer:jutils.obj
 0001:00079e00       _jpeg_get_small            0047ae00 f   renderer:jmemnobs.obj
 0001:00079e10       _jpeg_free_small           0047ae10 f   renderer:jmemnobs.obj
 0001:00079e20       _jpeg_get_large            0047ae20 f   renderer:jmemnobs.obj
 0001:00079e30       _jpeg_free_large           0047ae30 f   renderer:jmemnobs.obj
 0001:00079e40       _jpeg_mem_available        0047ae40 f   renderer:jmemnobs.obj
 0001:00079e50       _jpeg_open_backing_store   0047ae50 f   renderer:jmemnobs.obj
 0001:00079e70       _jpeg_mem_init             0047ae70 f   renderer:jmemnobs.obj
 0001:00079e80       _jpeg_mem_term             0047ae80 f   renderer:jmemnobs.obj
 0001:0007a430       _jinit_d_main_controller   0047b430 f   renderer:jdmainct.obj
 0001:0007a830       _jinit_d_coef_controller   0047b830 f   renderer:jdcoefct.obj
 0001:0007a8f0       _jpeg_make_d_derived_tbl   0047b8f0 f   renderer:jdhuff.obj
 0001:0007aad0       _jpeg_fill_bit_buffer      0047bad0 f   renderer:jdhuff.obj
 0001:0007abd0       _jpeg_huff_decode          0047bbd0 f   renderer:jdhuff.obj
 0001:0007b2e0       _jinit_huff_decoder        0047c2e0 f   renderer:jdhuff.obj
 0001:0007b550       _jinit_inverse_dct         0047c550 f   renderer:jddctmgr.obj
 0001:0007b6d0       _jinit_d_post_controller   0047c6d0 f   renderer:jdpostct.obj
 0001:0007bc30       _jinit_upsampler           0047cc30 f   renderer:jdsample.obj
 0001:0007c220       _jinit_color_deconverter   0047d220 f   renderer:jdcolor.obj
 0001:0007c3d0       _jpeg_fdct_float           0047d3d0 f   renderer:jfdctflt.obj
 0001:0007d510       _jpeg_idct_float           0047e510 f   renderer:jidctflt.obj
 0001:0007d960       _Sys_MilliSeconds          0047e960 f   botlib:be_interface.obj
 0001:0007d980       _ValidClientNumber         0047e980 f   botlib:be_interface.obj
 0001:0007d9c0       _ValidEntityNumber         0047e9c0 f   botlib:be_interface.obj
 0001:0007da00       _BotLibSetup               0047ea00 f   botlib:be_interface.obj
 0001:0007da30       _Export_BotLibSetup        0047ea30 f   botlib:be_interface.obj
 0001:0007db00       _Export_BotLibShutdown     0047eb00 f   botlib:be_interface.obj
 0001:0007db80       _Export_BotLibVarSet       0047eb80 f   botlib:be_interface.obj
 0001:0007dba0       _Export_BotLibVarGet       0047eba0 f   botlib:be_interface.obj
 0001:0007dbd0       _Export_BotLibStartFrame   0047ebd0 f   botlib:be_interface.obj
 0001:0007dc00       _Export_BotLibLoadMap      0047ec00 f   botlib:be_interface.obj
 0001:0007dc60       _Export_BotLibUpdateEntity 0047ec60 f   botlib:be_interface.obj
 0001:0007dcc0       _BotExportTest             0047ecc0 f   botlib:be_interface.obj
 0001:0007e0b0       _GetBotLibAPI              0047f0b0 f   botlib:be_interface.obj
 0001:0007e1a0       _BotAllocMoveState         0047f1a0 f   botlib:be_ai_move.obj
 0001:0007e1e0       _BotFreeMoveState          0047f1e0 f   botlib:be_ai_move.obj
 0001:0007e240       _BotMoveStateFromHandle    0047f240 f   botlib:be_ai_move.obj
 0001:0007e280       _BotInitMoveState          0047f280 f   botlib:be_ai_move.obj
 0001:0007e3f0       _AngleDiff                 0047f3f0 f   botlib:be_ai_move.obj
 0001:0007e430       _BotFuzzyPointReachabilityArea 0047f430 f   botlib:be_ai_move.obj
 0001:0007e630       _BotReachabilityArea       0047f630 f   botlib:be_ai_move.obj
 0001:0007e810       _BotOnMover                0047f810 f   botlib:be_ai_move.obj
 0001:0007e9e0       _MoverDown                 0047f9e0 f   botlib:be_ai_move.obj
 0001:0007ea70       _BotSetBrushModelTypes     0047fa70 f   botlib:be_ai_move.obj
 0001:0007ebe0       _BotOnTopOfEntity          0047fbe0 f   botlib:be_ai_move.obj
 0001:0007ec80       _BotValidTravel            0047fc80 f   botlib:be_ai_move.obj
 0001:0007ecc0       _BotAddToAvoidReach        0047fcc0 f   botlib:be_ai_move.obj
 0001:0007ed60       _DistanceFromLineSquared   0047fd60 f   botlib:be_ai_move.obj
 0001:0007ee60       _VectorDistanceSquared     0047fe60 f   botlib:be_ai_move.obj
 0001:0007ee90       _BotAvoidSpots             0047fe90 f   botlib:be_ai_move.obj
 0001:0007f080       _BotAddAvoidSpot           00480080 f   botlib:be_ai_move.obj
 0001:0007f140       _BotGetReachabilityToGoal  00480140 f   botlib:be_ai_move.obj
 0001:0007f2e0       _BotAddToTarget            004802e0 f   botlib:be_ai_move.obj
 0001:0007f390       _BotMovementViewTarget     00480390 f   botlib:be_ai_move.obj
 0001:0007f560       _BotVisible                00480560 f   botlib:be_ai_move.obj
 0001:0007f5d0       _BotPredictVisiblePosition 004805d0 f   botlib:be_ai_move.obj
 0001:0007f730       _MoverBottomCenter         00480730 f   botlib:be_ai_move.obj
 0001:0007f7f0       _BotGapDistance            004807f0 f   botlib:be_ai_move.obj
 0001:0007f9b0       _BotCheckBarrierJump       004809b0 f   botlib:be_ai_move.obj
 0001:0007fba0       _BotSwimInDirection        00480ba0 f   botlib:be_ai_move.obj
 0001:0007fbf0       _BotWalkInDirection        00480bf0 f   botlib:be_ai_move.obj
 0001:0007fee0       _BotMoveInDirection        00480ee0 f   botlib:be_ai_move.obj
 0001:0007ff60       _Intersection              00480f60 f   botlib:be_ai_move.obj
 0001:00080030       _BotCheckBlocked           00481030 f   botlib:be_ai_move.obj
 0001:000801f0       _BotClearMoveResult        004811f0 f   botlib:be_ai_move.obj
 0001:00080210       _BotTravel_Walk            00481210 f   botlib:be_ai_move.obj
 0001:000803b0       _BotFinishTravel_Walk      004813b0 f   botlib:be_ai_move.obj
 0001:00080470       _BotTravel_Crouch          00481470 f   botlib:be_ai_move.obj
 0001:00080520       _BotTravel_BarrierJump     00481520 f   botlib:be_ai_move.obj
 0001:00080620       _BotFinishTravel_BarrierJump 00481620 f   botlib:be_ai_move.obj
 0001:000806e0       _BotTravel_Swim            004816e0 f   botlib:be_ai_move.obj
 0001:000807b0       _BotTravel_WaterJump       004817b0 f   botlib:be_ai_move.obj
 0001:000808d0       _BotFinishTravel_WaterJump 004818d0 f   botlib:be_ai_move.obj
 0001:00080a50       _BotTravel_WalkOffLedge    00481a50 f   botlib:be_ai_move.obj
 0001:00080c20       _BotAirControl             00481c20 f   botlib:be_ai_move.obj
 0001:00080da0       _BotFinishTravel_WalkOffLedge 00481da0 f   botlib:be_ai_move.obj
 0001:00080f10       _BotTravel_Jump            00481f10 f   botlib:be_ai_move.obj
 0001:00081240       _BotFinishTravel_Jump      00482240 f   botlib:be_ai_move.obj
 0001:00081340       _BotTravel_Ladder          00482340 f   botlib:be_ai_move.obj
 0001:00081430       _BotTravel_Teleport        00482430 f   botlib:be_ai_move.obj
 0001:00081530       _BotTravel_Elevator        00482530 f   botlib:be_ai_move.obj
 0001:00081a50       _BotFinishTravel_Elevator  00482a50 f   botlib:be_ai_move.obj
 0001:00081b20       _BotFuncBobStartEnd        00482b20 f   botlib:be_ai_move.obj
 0001:00081cd0       _BotTravel_FuncBobbing     00482cd0 f   botlib:be_ai_move.obj
 0001:00082280       _BotFinishTravel_FuncBobbing 00483280 f   botlib:be_ai_move.obj
 0001:000824a0       _GrappleState              004834a0 f   botlib:be_ai_move.obj
 0001:00082540       _BotResetGrapple           00483540 f   botlib:be_ai_move.obj
 0001:000825d0       _BotTravel_Grapple         004835d0 f   botlib:be_ai_move.obj
 0001:00082a70       _BotTravel_RocketJump      00483a70 f   botlib:be_ai_move.obj
 0001:00082c90       _BotTravel_BFGJump         00483c90 f   botlib:be_ai_move.obj
 0001:00082e90       _BotFinishTravel_WeaponJump 00483e90 f   botlib:be_ai_move.obj
 0001:00082f60       _BotTravel_JumpPad         00483f60 f   botlib:be_ai_move.obj
 0001:00083010       _BotFinishTravel_JumpPad   00484010 f   botlib:be_ai_move.obj
 0001:000830e0       _BotReachabilityTime       004840e0 f   botlib:be_ai_move.obj
 0001:00083170       _BotMoveInGoalArea         00484170 f   botlib:be_ai_move.obj
 0001:000832c0       _BotMoveToGoal             004842c0 f   botlib:be_ai_move.obj
 0001:00083e10       _BotResetAvoidReach        00484e10 f   botlib:be_ai_move.obj
 0001:00083e80       _BotResetLastAvoidReach    00484e80 f   botlib:be_ai_move.obj
 0001:00083f00       _BotResetMoveState         00484f00 f   botlib:be_ai_move.obj
 0001:00083f50       _BotSetupMoveAI            00484f50 f   botlib:be_ai_move.obj
 0001:00084030       _BotShutdownMoveAI         00485030 f   botlib:be_ai_move.obj
 0001:00084060       _BotChatStateFromHandle    00485060 f   botlib:be_ai_chat.obj
 0001:000840a0       _InitConsoleMessageHeap    004850a0 f   botlib:be_ai_chat.obj
 0001:00084170       _AllocConsoleMessage       00485170 f   botlib:be_ai_chat.obj
 0001:000841a0       _FreeConsoleMessage        004851a0 f   botlib:be_ai_chat.obj
 0001:000841d0       _BotRemoveConsoleMessage   004851d0 f   botlib:be_ai_chat.obj
 0001:000842b0       _BotQueueConsoleMessage    004852b0 f   botlib:be_ai_chat.obj
 0001:000843f0       _BotNextConsoleMessage     004853f0 f   botlib:be_ai_chat.obj
 0001:00084470       _BotNumConsoleMessages     00485470 f   botlib:be_ai_chat.obj
 0001:000844c0       _IsWhiteSpace              004854c0 f   botlib:be_ai_chat.obj
 0001:00084520       _BotRemoveTildes           00485520 f   botlib:be_ai_chat.obj
 0001:00084570       _UnifyWhiteSpaces          00485570 f   botlib:be_ai_chat.obj
 0001:00084690       _StringContains            00485690 f   botlib:be_ai_chat.obj
 0001:00084770       _StringContainsWord        00485770 f   botlib:be_ai_chat.obj
 0001:00084890       _StringReplaceWords        00485890 f   botlib:be_ai_chat.obj
 0001:000849b0       _BotDumpSynonymList        004859b0 f   botlib:be_ai_chat.obj
 0001:00084a30       _BotLoadSynonyms           00485a30 f   botlib:be_ai_chat.obj
 0001:00084ed0       _BotReplaceSynonyms        00485ed0 f   botlib:be_ai_chat.obj
 0001:00084f20       _BotReplaceWeightedSynonyms 00485f20 f   botlib:be_ai_chat.obj
 0001:00084fd0       _BotReplaceReplySynonyms   00485fd0 f   botlib:be_ai_chat.obj
 0001:00085110       _BotLoadChatMessage        00486110 f   botlib:be_ai_chat.obj
 0001:000852f0       _BotDumpRandomStringList   004862f0 f   botlib:be_ai_chat.obj
 0001:00085360       _BotLoadRandomStrings      00486360 f   botlib:be_ai_chat.obj
 0001:000855e0       _RandomString              004865e0 f   botlib:be_ai_chat.obj
 0001:00085680       _BotDumpMatchTemplates     00486680 f   botlib:be_ai_chat.obj
 0001:00085750       _BotFreeMatchPieces        00486750 f   botlib:be_ai_chat.obj
 0001:000857a0       _BotLoadMatchPieces        004867a0 f   botlib:be_ai_chat.obj
 0001:00085a70       _BotFreeMatchTemplates     00486a70 f   botlib:be_ai_chat.obj
 0001:00085aa0       _BotLoadMatchTemplates     00486aa0 f   botlib:be_ai_chat.obj
 0001:00085d50       _StringsMatch              00486d50 f   botlib:be_ai_chat.obj
 0001:00085e80       _BotFindMatch              00486e80 f   botlib:be_ai_chat.obj
 0001:00085f60       _BotMatchVariable          00486f60 f   botlib:be_ai_chat.obj
 0001:00085fd0       _BotFindStringInList       00486fd0 f   botlib:be_ai_chat.obj
 0001:00086030       _BotCheckChatMessageIntegrety 00487030 f   botlib:be_ai_chat.obj
 0001:00086180       _BotCheckInitialChatIntegrety 00487180 f   botlib:be_ai_chat.obj
 0001:000861d0       _BotCheckReplyChatIntegrety 004871d0 f   botlib:be_ai_chat.obj
 0001:00086220       _BotDumpReplyChat          00487220 f   botlib:be_ai_chat.obj
 0001:00086410       _BotFreeReplyChat          00487410 f   botlib:be_ai_chat.obj
 0001:000864a0       _BotCheckValidReplyChatKeySet 004874a0 f   botlib:be_ai_chat.obj
 0001:000866c0       _BotLoadReplyChat          004876c0 f   botlib:be_ai_chat.obj
 0001:00086bd0       _BotDumpInitialChat        00487bd0 f   botlib:be_ai_chat.obj
 0001:00086c60       _BotLoadInitialChat        00487c60 f   botlib:be_ai_chat.obj
 0001:000870c0       _BotFreeChatFile           004880c0 f   botlib:be_ai_chat.obj
 0001:00087120       _BotLoadChatFile           00488120 f   botlib:be_ai_chat.obj
 0001:00087300       _BotExpandChatMessage      00488300 f   botlib:be_ai_chat.obj
 0001:000875f0       _BotConstructChatMessage   004885f0 f   botlib:be_ai_chat.obj
 0001:000876b0       _BotChooseInitialChatMessage 004886b0 f   botlib:be_ai_chat.obj
 0001:000877c0       _BotNumInitialChats        004887c0 f   botlib:be_ai_chat.obj
 0001:00087870       _BotInitialChat            00488870 f   botlib:be_ai_chat.obj
 0001:00087c30       _BotPrintReplyChatKeys     00488c30 f   botlib:be_ai_chat.obj
 0001:00087dc0       _BotReplyChat              00488dc0 f   botlib:be_ai_chat.obj
 0001:00088410       _BotChatLength             00489410 f   botlib:be_ai_chat.obj
 0001:00088460       _BotEnterChat              00489460 f   botlib:be_ai_chat.obj
 0001:00088560       _BotGetChatMessage         00489560 f   botlib:be_ai_chat.obj
 0001:000885e0       _BotSetChatGender          004895e0 f   botlib:be_ai_chat.obj
 0001:00088640       _BotSetChatName            00489640 f   botlib:be_ai_chat.obj
 0001:000886c0       _BotResetChatAI            004896c0 f   botlib:be_ai_chat.obj
 0001:000886f0       _BotAllocChatState         004896f0 f   botlib:be_ai_chat.obj
 0001:00088730       _BotFreeChatState          00489730 f   botlib:be_ai_chat.obj
 0001:00088810       _BotSetupChatAI            00489810 f   botlib:be_ai_chat.obj
 0001:000888b0       _BotShutdownChatAI         004898b0 f   botlib:be_ai_chat.obj
 0001:00088990       _BotGoalStateFromHandle    00489990 f   botlib:be_ai_goal.obj
 0001:000889d0       _BotInterbreedGoalFuzzyLogic 004899d0 f   botlib:be_ai_goal.obj
 0001:00088aa0       _BotSaveGoalFuzzyLogic     00489aa0 f   botlib:be_ai_goal.obj
 0001:00088ae0       _BotMutateGoalFuzzyLogic   00489ae0 f   botlib:be_ai_goal.obj
 0001:00088b30       _LoadItemConfig            00489b30 f   botlib:be_ai_goal.obj
 0001:00088da0       _ItemWeightIndex           00489da0 f   botlib:be_ai_goal.obj
 0001:00088e10       _InitLevelItemHeap         00489e10 f   botlib:be_ai_goal.obj
 0001:00088eb0       _AllocLevelItem            00489eb0 f   botlib:be_ai_goal.obj
 0001:00088ef0       _FreeLevelItem             00489ef0 f   botlib:be_ai_goal.obj
 0001:00088f10       _AddLevelItemToList        00489f10 f   botlib:be_ai_goal.obj
 0001:00088f40       _RemoveLevelItemFromList   00489f40 f   botlib:be_ai_goal.obj
 0001:00088f70       _BotFreeInfoEntities       00489f70 f   botlib:be_ai_goal.obj
 0001:00088fe0       _BotInitInfoEntities       00489fe0 f   botlib:be_ai_goal.obj
 0001:000891d0       _BotInitLevelItems         0048a1d0 f   botlib:be_ai_goal.obj
 0001:000896a0       _BotGoalName               0048a6a0 f   botlib:be_ai_goal.obj
 0001:00089700       _BotResetAvoidGoals        0048a700 f   botlib:be_ai_goal.obj
 0001:00089770       _BotDumpAvoidGoals         0048a770 f   botlib:be_ai_goal.obj
 0001:00089830       _BotAddToAvoidGoals        0048a830 f   botlib:be_ai_goal.obj
 0001:000898c0       _BotRemoveFromAvoidGoals   0048a8c0 f   botlib:be_ai_goal.obj
 0001:00089950       _BotAvoidGoalTime          0048a950 f   botlib:be_ai_goal.obj
 0001:000899e0       _BotSetAvoidGoalTime       0048a9e0 f   botlib:be_ai_goal.obj
 0001:00089ae0       _BotGetLevelItemGoal       0048aae0 f   botlib:be_ai_goal.obj
 0001:00089c70       _BotGetMapLocationGoal     0048ac70 f   botlib:be_ai_goal.obj
 0001:00089cf0       _BotGetNextCampSpotGoal    0048acf0 f   botlib:be_ai_goal.obj
 0001:00089d60       _BotFindEntityForLevelItem 0048ad60 f   botlib:be_ai_goal.obj
 0001:00089e60       _BotUpdateEntityItems      0048ae60 f   botlib:be_ai_goal.obj
 0001:0008a2a0       _BotDumpGoalStack          0048b2a0 f   botlib:be_ai_goal.obj
 0001:0008a340       _BotPushGoal               0048b340 f   botlib:be_ai_goal.obj
 0001:0008a3d0       _BotPopGoal                0048b3d0 f   botlib:be_ai_goal.obj
 0001:0008a420       _BotEmptyGoalStack         0048b420 f   botlib:be_ai_goal.obj
 0001:0008a470       _BotGetTopGoal             0048b470 f   botlib:be_ai_goal.obj
 0001:0008a4e0       _BotGetSecondGoal          0048b4e0 f   botlib:be_ai_goal.obj
 0001:0008a550       _BotChooseLTGItem          0048b550 f   botlib:be_ai_goal.obj
 0001:0008a880       _BotChooseNBGItem          0048b880 f   botlib:be_ai_goal.obj
 0001:0008ac40       _BotTouchingGoal           0048bc40 f   botlib:be_ai_goal.obj
 0001:0008ad40       _BotItemGoalInVisButNotVisible 0048bd40 f   botlib:be_ai_goal.obj
 0001:0008ae40       _BotResetGoalState         0048be40 f   botlib:be_ai_goal.obj
 0001:0008aeb0       _BotLoadItemWeights        0048beb0 f   botlib:be_ai_goal.obj
 0001:0008af30       _BotFreeItemWeights        0048bf30 f   botlib:be_ai_goal.obj
 0001:0008af90       _BotAllocGoalState         0048bf90 f   botlib:be_ai_goal.obj
 0001:0008afe0       _BotFreeGoalState          0048bfe0 f   botlib:be_ai_goal.obj
 0001:0008b050       _BotSetupGoalAI            0048c050 f   botlib:be_ai_goal.obj
 0001:0008b0c0       _BotShutdownGoalAI         0048c0c0 f   botlib:be_ai_goal.obj
 0001:0008b130       _BotValidWeaponNumber      0048c130 f   botlib:be_ai_weap.obj
 0001:0008b160       _BotWeaponStateFromHandle  0048c160 f   botlib:be_ai_weap.obj
 0001:0008b1a0       _LoadWeaponConfig          0048c1a0 f   botlib:be_ai_weap.obj
 0001:0008b630       _WeaponWeightIndex         0048c630 f   botlib:be_ai_weap.obj
 0001:0008b680       _BotFreeWeaponWeights      0048c680 f   botlib:be_ai_weap.obj
 0001:0008b6e0       _BotLoadWeaponWeights      0048c6e0 f   botlib:be_ai_weap.obj
 0001:0008b770       _BotGetWeaponInfo          0048c770 f   botlib:be_ai_weap.obj
 0001:0008b810       _BotChooseBestFightWeapon  0048c810 f   botlib:be_ai_weap.obj
 0001:0008b8f0       _BotResetWeaponState       0048c8f0 f   botlib:be_ai_weap.obj
 0001:0008b930       _BotAllocWeaponState       0048c930 f   botlib:be_ai_weap.obj
 0001:0008b970       _BotFreeWeaponState        0048c970 f   botlib:be_ai_weap.obj
 0001:0008b9e0       _BotSetupWeaponAI          0048c9e0 f   botlib:be_ai_weap.obj
 0001:0008ba20       _BotShutdownWeaponAI       0048ca20 f   botlib:be_ai_weap.obj
 0001:0008ba60       _EA_Say                    0048ca60 f   botlib:be_ea.obj
 0001:0008ba80       _EA_SayTeam                0048ca80 f   botlib:be_ea.obj
 0001:0008baa0       _EA_Tell                   0048caa0 f   botlib:be_ea.obj
 0001:0008bad0       _EA_UseItem                0048cad0 f   botlib:be_ea.obj
 0001:0008baf0       _EA_DropItem               0048caf0 f   botlib:be_ea.obj
 0001:0008bb10       _EA_UseInv                 0048cb10 f   botlib:be_ea.obj
 0001:0008bb30       _EA_DropInv                0048cb30 f   botlib:be_ea.obj
 0001:0008bb50       _EA_Gesture                0048cb50 f   botlib:be_ea.obj
 0001:0008bb70       _EA_Command                0048cb70 f   botlib:be_ea.obj
 0001:0008bb80       _EA_SelectWeapon           0048cb80 f   botlib:be_ea.obj
 0001:0008bba0       _EA_Attack                 0048cba0 f   botlib:be_ea.obj
 0001:0008bbc0       _EA_Talk                   0048cbc0 f   botlib:be_ea.obj
 0001:0008bbe0       _EA_Use                    0048cbe0 f   botlib:be_ea.obj
 0001:0008bc00       _EA_Respawn                0048cc00 f   botlib:be_ea.obj
 0001:0008bc20       _EA_Jump                   0048cc20 f   botlib:be_ea.obj
 0001:0008bc50       _EA_DelayedJump            0048cc50 f   botlib:be_ea.obj
 0001:0008bc80       _EA_Crouch                 0048cc80 f   botlib:be_ea.obj
 0001:0008bca0       _EA_Walk                   0048cca0 f   botlib:be_ea.obj
 0001:0008bcc0       _EA_Action                 0048ccc0 f   botlib:be_ea.obj
 0001:0008bce0       _EA_MoveUp                 0048cce0 f   botlib:be_ea.obj
 0001:0008bd00       _EA_MoveDown               0048cd00 f   botlib:be_ea.obj
 0001:0008bd20       _EA_MoveForward            0048cd20 f   botlib:be_ea.obj
 0001:0008bd40       _EA_MoveBack               0048cd40 f   botlib:be_ea.obj
 0001:0008bd60       _EA_MoveLeft               0048cd60 f   botlib:be_ea.obj
 0001:0008bd80       _EA_MoveRight              0048cd80 f   botlib:be_ea.obj
 0001:0008bda0       _EA_Move                   0048cda0 f   botlib:be_ea.obj
 0001:0008be00       _EA_View                   0048ce00 f   botlib:be_ea.obj
 0001:0008be30       _EA_EndRegular             0048ce30 f   botlib:be_ea.obj
 0001:0008be40       _EA_GetInput               0048ce40 f   botlib:be_ea.obj
 0001:0008be70       _EA_ResetInput             0048ce70 f   botlib:be_ea.obj
 0001:0008beb0       _EA_Setup                  0048ceb0 f   botlib:be_ea.obj
 0001:0008bed0       _EA_Shutdown               0048ced0 f   botlib:be_ea.obj
 0001:0008bef0       _AAS_Error                 0048cef0 f   botlib:be_aas_main.obj
 0001:0008bf30       _AAS_StringFromIndex       0048cf30 f   botlib:be_aas_main.obj
 0001:0008bfb0       _AAS_IndexFromString       0048cfb0 f   botlib:be_aas_main.obj
 0001:0008c020       _AAS_ModelFromIndex        0048d020 f   botlib:be_aas_main.obj
 0001:0008c040       _AAS_IndexFromModel        0048d040 f   botlib:be_aas_main.obj
 0001:0008c060       _AAS_UpdateStringIndexes   0048d060 f   botlib:be_aas_main.obj
 0001:0008c0c0       _AAS_Loaded                0048d0c0 f   botlib:be_aas_main.obj
 0001:0008c0d0       _AAS_Initialized           0048d0d0 f   botlib:be_aas_main.obj
 0001:0008c0e0       _AAS_SetInitialized        0048d0e0 f   botlib:be_aas_main.obj
 0001:0008c100       _AAS_ContinueInit          0048d100 f   botlib:be_aas_main.obj
 0001:0008c1d0       _AAS_StartFrame            0048d1d0 f   botlib:be_aas_main.obj
 0001:0008c2e0       _AAS_Time                  0048d2e0 f   botlib:be_aas_main.obj
 0001:0008c2f0       _AAS_ProjectPointOntoVector 0048d2f0 f   botlib:be_aas_main.obj
 0001:0008c390       _AAS_LoadFiles             0048d390 f   botlib:be_aas_main.obj
 0001:0008c410       _AAS_LoadMap               0048d410 f   botlib:be_aas_main.obj
 0001:0008c460       _AAS_Setup                 0048d460 f   botlib:be_aas_main.obj
 0001:0008c4f0       _AAS_Shutdown              0048d4f0 f   botlib:be_aas_main.obj
 0001:0008c550       _LibVarStringValue         0048d550 f   botlib:l_libvar.obj
 0001:0008c5d0       _LibVarAlloc               0048d5d0 f   botlib:l_libvar.obj
 0001:0008c630       _LibVarDeAlloc             0048d630 f   botlib:l_libvar.obj
 0001:0008c650       _LibVarDeAllocAll          0048d650 f   botlib:l_libvar.obj
 0001:0008c6a0       _LibVarGet                 0048d6a0 f   botlib:l_libvar.obj
 0001:0008c6e0       _LibVarGetString           0048d6e0 f   botlib:l_libvar.obj
 0001:0008c700       _LibVarGetValue            0048d700 f   botlib:l_libvar.obj
 0001:0008c720       _LibVar                    0048d720 f   botlib:l_libvar.obj
 0001:0008c790       _LibVarString              0048d790 f   botlib:l_libvar.obj
 0001:0008c7b0       _LibVarValue               0048d7b0 f   botlib:l_libvar.obj
 0001:0008c7d0       _LibVarSet                 0048d7d0 f   botlib:l_libvar.obj
 0001:0008c850       _LibVarChanged             0048d850 f   botlib:l_libvar.obj
 0001:0008c870       _LibVarSetNotModified      0048d870 f   botlib:l_libvar.obj
 0001:0008c890       _Log_Open                  0048d890 f   botlib:l_log.obj
 0001:0008c960       _Log_Close                 0048d960 f   botlib:l_log.obj
 0001:0008c9b0       _Log_Shutdown              0048d9b0 f   botlib:l_log.obj
 0001:0008c9c0       _Log_Write                 0048d9c0 f   botlib:l_log.obj
 0001:0008c9f0       _Log_WriteTimeStamped      0048d9f0 f   botlib:l_log.obj
 0001:0008cab0       _Log_FilePointer           0048dab0 f   botlib:l_log.obj
 0001:0008cac0       _Log_Flush                 0048dac0 f   botlib:l_log.obj
 0001:0008cae0       _SourceError               0048dae0 f   botlib:l_precomp.obj
 0001:0008cb30       _SourceWarning             0048db30 f   botlib:l_precomp.obj
 0001:0008cb80       _PC_PushIndent             0048db80 f   botlib:l_precomp.obj
 0001:0008cbd0       _PC_PopIndent              0048dbd0 f   botlib:l_precomp.obj
 0001:0008cc40       _PC_PushScript             0048dc40 f   botlib:l_precomp.obj
 0001:0008cca0       _PC_InitTokenHeap          0048dca0 f   botlib:l_precomp.obj
 0001:0008ccb0       _PC_CopyToken              0048dcb0 f   botlib:l_precomp.obj
 0001:0008cd10       _PC_FreeToken              0048dd10 f   botlib:l_precomp.obj
 0001:0008cd30       _PC_ReadSourceToken        0048dd30 f   botlib:l_precomp.obj
 0001:0008ce60       _PC_UnreadSourceToken      0048de60 f   botlib:l_precomp.obj
 0001:0008ce90       _PC_ReadDefineParms        0048de90 f   botlib:l_precomp.obj
 0001:0008d1c0       _PC_StringizeTokens        0048e1c0 f   botlib:l_precomp.obj
 0001:0008d270       _PC_MergeTokens            0048e270 f   botlib:l_precomp.obj
 0001:0008d310       _PC_PrintDefineHashTable   0048e310 f   botlib:l_precomp.obj
 0001:0008d370       _PC_NameHash               0048e370 f   botlib:l_precomp.obj
 0001:0008d3b0       _PC_AddDefineToHash        0048e3b0 f   botlib:l_precomp.obj
 0001:0008d3d0       _PC_FindHashedDefine       0048e3d0 f   botlib:l_precomp.obj
 0001:0008d440       _PC_FindDefine             0048e440 f   botlib:l_precomp.obj
 0001:0008d4a0       _PC_FindDefineParm         0048e4a0 f   botlib:l_precomp.obj
 0001:0008d510       _PC_FreeDefine             0048e510 f   botlib:l_precomp.obj
 0001:0008d580       _PC_AddBuiltinDefines      0048e580 f   botlib:l_precomp.obj
 0001:0008d6a0       _PC_ExpandBuiltinDefine    0048e6a0 f   botlib:l_precomp.obj
 0001:0008d8b0       _PC_ExpandDefine           0048e8b0 f   botlib:l_precomp.obj
 0001:0008dbf0       _PC_ExpandDefineIntoSource 0048ebf0 f   botlib:l_precomp.obj
 0001:0008dc50       _PC_ConvertPath            0048ec50 f   botlib:l_precomp.obj
 0001:0008dcc0       _PC_Directive_include      0048ecc0 f   botlib:l_precomp.obj
 0001:0008df00       _PC_ReadLine               0048ef00 f   botlib:l_precomp.obj
 0001:0008df70       _PC_WhiteSpaceBeforeToken  0048ef70 f   botlib:l_precomp.obj
 0001:0008df90       _PC_ClearTokenWhiteSpace   0048ef90 f   botlib:l_precomp.obj
 0001:0008dfb0       _PC_Directive_undef        0048efb0 f   botlib:l_precomp.obj
 0001:0008e110       _PC_RemoveGlobalDefine     0048f110 f   botlib:l_precomp.obj
 0001:0008e140       _PC_RemoveAllGlobalDefines 0048f140 f   botlib:l_precomp.obj
 0001:0008e170       _PC_CopyDefine             0048f170 f   botlib:l_precomp.obj
 0001:0008e2d0       _PC_AddGlobalDefinesToSource 0048f2d0 f   botlib:l_precomp.obj
 0001:0008e350       _PC_Directive_if_def       0048f350 f   botlib:l_precomp.obj
 0001:0008e410       _PC_Directive_ifdef        0048f410 f   botlib:l_precomp.obj
 0001:0008e420       _PC_Directive_ifndef       0048f420 f   botlib:l_precomp.obj
 0001:0008e430       _PC_Directive_else         0048f430 f   botlib:l_precomp.obj
 0001:0008e4b0       _PC_Directive_endif        0048f4b0 f   botlib:l_precomp.obj
 0001:0008e500       _PC_OperatorPriority       0048f500 f   botlib:l_precomp.obj
 0001:0008e5d0       _PC_EvaluateTokens         0048f5d0 f   botlib:l_precomp.obj
 0001:0008eff0       _PC_Evaluate               0048fff0 f   botlib:l_precomp.obj
 0001:0008f260       _PC_DollarEvaluate         00490260 f   botlib:l_precomp.obj
 0001:0008f530       _PC_Directive_elif         00490530 f   botlib:l_precomp.obj
 0001:0008f5b0       _PC_Directive_if           004905b0 f   botlib:l_precomp.obj
 0001:0008f5f0       _PC_Directive_line         004905f0 f   botlib:l_precomp.obj
 0001:0008f610       _PC_Directive_error        00490610 f   botlib:l_precomp.obj
 0001:0008f650       _PC_Directive_pragma       00490650 f   botlib:l_precomp.obj
 0001:0008f690       _UnreadSignToken           00490690 f   botlib:l_precomp.obj
 0001:0008f720       _PC_Directive_eval         00490720 f   botlib:l_precomp.obj
 0001:0008f7f0       _PC_Directive_evalfloat    004907f0 f   botlib:l_precomp.obj
 0001:0008f8d0       _PC_ReadDirective          004908d0 f   botlib:l_precomp.obj
 0001:0008f9e0       _PC_DollarDirective_evalint 004909e0 f   botlib:l_precomp.obj
 0001:0008fad0       _PC_DollarDirective_evalfloat 00490ad0 f   botlib:l_precomp.obj
 0001:0008fbd0       _PC_ReadDollarDirective    00490bd0 f   botlib:l_precomp.obj
 0001:0008fd00       _PC_UnreadLastToken        00490d00 f   botlib:l_precomp.obj
 0001:0008fd30       _PC_UnreadToken            00490d30 f   botlib:l_precomp.obj
 0001:0008fd60       _PC_SetIncludePath         00490d60 f   botlib:l_precomp.obj
 0001:0008fdd0       _PC_SetPunctuations        00490dd0 f   botlib:l_precomp.obj
 0001:0008fde0       _LoadSourceFile            00490de0 f   botlib:l_precomp.obj
 0001:0008fe70       _LoadSourceMemory          00490e70 f   botlib:l_precomp.obj
 0001:0008ff00       _FreeSource                00490f00 f   botlib:l_precomp.obj
 0001:00090010       _PC_LoadSourceHandle       00491010 f   botlib:l_precomp.obj
 0001:00090090       _PC_FreeSourceHandle       00491090 f   botlib:l_precomp.obj
 0001:000900d0       _PC_SourceFileAndLine      004910d0 f   botlib:l_precomp.obj
 0001:00090140       _PC_SetBaseFolder          00491140 f   botlib:l_precomp.obj
 0001:00090150       _PC_CheckOpenSourceHandles 00491150 f   botlib:l_precomp.obj
 0001:00090180       _PC_ReadToken              00491180 f   botlib:l_precomp.obj
 0001:00090340       _PC_ExpectTokenString      00491340 f   botlib:l_precomp.obj
 0001:00090400       _PC_ExpectTokenType        00491400 f   botlib:l_precomp.obj
 0001:000906b0       _PC_ExpectAnyToken         004916b0 f   botlib:l_precomp.obj
 0001:000906e0       _PC_CheckTokenString       004916e0 f   botlib:l_precomp.obj
 0001:00090780       _PC_CheckTokenType         00491780 f   botlib:l_precomp.obj
 0001:00090820       _PC_SkipUntilString        00491820 f   botlib:l_precomp.obj
 0001:000908c0       _PC_ReadTokenHandle        004918c0 f   botlib:l_precomp.obj
 0001:00090970       _PC_Directive_define       00491970 f   botlib:l_precomp.obj
 0001:00090de0       _PC_DefineFromString       00491de0 f   botlib:l_precomp.obj
 0001:00090f00       _PC_AddDefine              00491f00 f   botlib:l_precomp.obj
 0001:00090f40       _PC_AddGlobalDefine        00491f40 f   botlib:l_precomp.obj
 0001:00090f70       _BotCharacterFromHandle    00491f70 f   botlib:be_ai_char.obj
 0001:00090fb0       _BotDumpCharacter          00491fb0 f   botlib:be_ai_char.obj
 0001:00091040       _BotFreeCharacterStrings   00492040 f   botlib:be_ai_char.obj
 0001:00091070       _BotFreeCharacter2         00492070 f   botlib:be_ai_char.obj
 0001:000910e0       _BotFreeCharacter          004920e0 f   botlib:be_ai_char.obj
 0001:00091110       _BotDefaultCharacteristics 00492110 f   botlib:be_ai_char.obj
 0001:000911a0       _BotLoadCharacterFromFile  004921a0 f   botlib:be_ai_char.obj
 0001:00091550       _BotFindCachedCharacter    00492550 f   botlib:be_ai_char.obj
 0001:000915e0       _BotLoadCachedCharacter    004925e0 f   botlib:be_ai_char.obj
 0001:00091850       _BotLoadCharacterSkill     00492850 f   botlib:be_ai_char.obj
 0001:000918b0       _BotInterpolateCharacters  004928b0 f   botlib:be_ai_char.obj
 0001:00091a70       _BotLoadCharacter          00492a70 f   botlib:be_ai_char.obj
 0001:00091bb0       _CheckCharacteristicIndex  00492bb0 f   botlib:be_ai_char.obj
 0001:00091c40       _Characteristic_Float      00492c40 f   botlib:be_ai_char.obj
 0001:00091cd0       _Characteristic_BFloat     00492cd0 f   botlib:be_ai_char.obj
 0001:00091d80       _Characteristic_Integer    00492d80 f   botlib:be_ai_char.obj
 0001:00091e10       _Characteristic_BInteger   00492e10 f   botlib:be_ai_char.obj
 0001:00091ea0       _Characteristic_String     00492ea0 f   botlib:be_ai_char.obj
 0001:00091f30       _BotShutdownCharacters     00492f30 f   botlib:be_ai_char.obj
 0001:00091f60       _ReadValue                 00492f60 f   botlib:be_ai_weight.obj
 0001:00092000       _ReadFuzzyWeight           00493000 f   botlib:be_ai_weight.obj
 0001:000920f0       _FreeFuzzySeperators_r     004930f0 f   botlib:be_ai_weight.obj
 0001:00092130       _FreeWeightConfig2         00493130 f   botlib:be_ai_weight.obj
 0001:000921a0       _FreeWeightConfig          004931a0 f   botlib:be_ai_weight.obj
 0001:000921d0       _ReadFuzzySeperators_r     004931d0 f   botlib:be_ai_weight.obj
 0001:00092510       _ReadWeightConfig          00493510 f   botlib:be_ai_weight.obj
 0001:000928e0       _FindFuzzyWeight           004938e0 f   botlib:be_ai_weight.obj
 0001:00092950       _FuzzyWeight_r             00493950 f   botlib:be_ai_weight.obj
 0001:00092a00       _FuzzyWeightUndecided_r    00493a00 f   botlib:be_ai_weight.obj
 0001:00092b10       _FuzzyWeight               00493b10 f   botlib:be_ai_weight.obj
 0001:00092b30       _FuzzyWeightUndecided      00493b30 f   botlib:be_ai_weight.obj
 0001:00092b50       _EvolveFuzzySeperator_r    00493b50 f   botlib:be_ai_weight.obj
 0001:00092c30       _EvolveWeightConfig        00493c30 f   botlib:be_ai_weight.obj
 0001:00092c60       _ScaleFuzzySeperator_r     00493c60 f   botlib:be_ai_weight.obj
 0001:00092cd0       _ScaleWeight               00493cd0 f   botlib:be_ai_weight.obj
 0001:00092d80       _ScaleFuzzySeperatorBalanceRange_r 00493d80 f   botlib:be_ai_weight.obj
 0001:00092e10       _ScaleFuzzyBalanceRange    00493e10 f   botlib:be_ai_weight.obj
 0001:00092e80       _InterbreedFuzzySeperator_r 00493e80 f   botlib:be_ai_weight.obj
 0001:00092f70       _InterbreedWeightConfigs   00493f70 f   botlib:be_ai_weight.obj
 0001:00092fe0       _BotShutdownWeights        00493fe0 f   botlib:be_ai_weight.obj
 0001:00093080       _AAS_EntityInfo            00494080 f   botlib:be_aas_entity.obj
 0001:00093100       _AAS_EntityOrigin          00494100 f   botlib:be_aas_entity.obj
 0001:00093170       _AAS_EntityModelindex      00494170 f   botlib:be_aas_entity.obj
 0001:000931b0       _AAS_EntityType            004941b0 f   botlib:be_aas_entity.obj
 0001:000931f0       _AAS_EntityModelNum        004941f0 f   botlib:be_aas_entity.obj
 0001:00093230       _AAS_OriginOfMoverWithModelNum 00494230 f   botlib:be_aas_entity.obj
 0001:00093290       _AAS_EntitySize            00494290 f   botlib:be_aas_entity.obj
 0001:00093300       _AAS_EntityBSPData         00494300 f   botlib:be_aas_entity.obj
 0001:00093380       _AAS_ResetEntityLinks      00494380 f   botlib:be_aas_entity.obj
 0001:000933c0       _AAS_InvalidateEntities    004943c0 f   botlib:be_aas_entity.obj
 0001:00093400       _AAS_UnlinkInvalidEntities 00494400 f   botlib:be_aas_entity.obj
 0001:00093460       _AAS_NearestEntity         00494460 f   botlib:be_aas_entity.obj
 0001:00093530       _AAS_BestReachableEntityArea 00494530 f   botlib:be_aas_entity.obj
 0001:00093560       _AAS_NextEntity            00494560 f   botlib:be_aas_entity.obj
 0001:000935b0       _AAS_UpdateEntity          004945b0 f   botlib:be_aas_entity.obj
 0001:00093870       _AAS_DropToFloor           00494870 f   botlib:be_aas_move.obj
 0001:00093910       _AAS_InitSettings          00494910 f   botlib:be_aas_move.obj
 0001:00093cb0       _AAS_AgainstLadder         00494cb0 f   botlib:be_aas_move.obj
 0001:00093e40       _AAS_OnGround              00494e40 f   botlib:be_aas_move.obj
 0001:00093f00       _AAS_Swimming              00494f00 f   botlib:be_aas_move.obj
 0001:00093f40       _AAS_SetMovedir            00494f40 f   botlib:be_aas_move.obj
 0001:00094000       _AAS_WeaponJumpZVelocity   00495000 f   botlib:be_aas_move.obj
 0001:000941e0       _AAS_RocketJumpZVelocity   004951e0 f   botlib:be_aas_move.obj
 0001:00094200       _AAS_BFGJumpZVelocity      00495200 f   botlib:be_aas_move.obj
 0001:00094220       _AAS_Accelerate            00495220 f   botlib:be_aas_move.obj
 0001:00094290       _AAS_AirControl            00495290 f   botlib:be_aas_move.obj
 0001:000942a0       _AAS_ApplyFriction         004952a0 f   botlib:be_aas_move.obj
 0001:00094310       _AAS_ClipToBBox            00495310 f   botlib:be_aas_move.obj
 0001:00094530       _AAS_ClientMovementPrediction 00495530 f   botlib:be_aas_move.obj
 0001:000954d0       _AAS_PredictClientMovement 004964d0 f   botlib:be_aas_move.obj
 0001:00095530       _AAS_ClientMovementHitBBox 00496530 f   botlib:be_aas_move.obj
 0001:00095590       _AAS_TestMovementPrediction 00496590 f   botlib:be_aas_move.obj
 0001:00095680       _AAS_HorizontalVelocityForJump 00496680 f   botlib:be_aas_move.obj
 0001:00095750       _AAS_JumpReachRunStart     00496750 f   botlib:be_aas_move.obj
 0001:00095850       _AAS_AltRoutingFloodCluster_r 00496850 f   botlib:be_aas_routealt.obj
 0001:00095930       _AAS_InitAlternativeRouting 00496930 f   botlib:be_aas_routealt.obj
 0001:00095990       _AAS_ShutdownAlternativeRouting 00496990 f   botlib:be_aas_routealt.obj
 0001:000959d0       _AAS_AlternativeRouteGoals 004969d0 f   botlib:be_aas_routealt.obj
 0001:00095de0       _AAS_RoutingInfo           00496de0 f   botlib:be_aas_route.obj
 0001:00095e20       _AAS_ClusterAreaNum        00496e20 f i botlib:be_aas_route.obj
 0001:00095e70       _AAS_InitTravelFlagFromType 00496e70 f   botlib:be_aas_route.obj
 0001:00095fd0       _AAS_TravelFlagForType_inline 00496fd0 f i botlib:be_aas_route.obj
 0001:00096020       _AAS_TravelFlagForType     00497020 f   botlib:be_aas_route.obj
 0001:00096040       _AAS_UnlinkCache           00497040 f   botlib:be_aas_route.obj
 0001:00096090       _AAS_LinkCache             00497090 f   botlib:be_aas_route.obj
 0001:000960d0       _AAS_FreeRoutingCache      004970d0 f   botlib:be_aas_route.obj
 0001:00096120       _AAS_RemoveRoutingCacheInCluster 00497120 f   botlib:be_aas_route.obj
 0001:000961e0       _AAS_RemoveRoutingCacheUsingArea 004971e0 f   botlib:be_aas_route.obj
 0001:000962c0       _AAS_EnableRoutingArea     004972c0 f   botlib:be_aas_route.obj
 0001:00096340       _AAS_RoutingTime           00497340 f i botlib:be_aas_route.obj
 0001:00096350       _AAS_GetAreaContentsTravelFlags 00497350 f   botlib:be_aas_route.obj
 0001:000963c0       _AAS_AreaContentsTravelFlags_inline 004973c0 f i botlib:be_aas_route.obj
 0001:000963d0       _AAS_AreaContentsTravelFlags 004973d0 f   botlib:be_aas_route.obj
 0001:000963e0       _AAS_InitAreaContentsTravelFlags 004973e0 f   botlib:be_aas_route.obj
 0001:000964a0       _AAS_CreateReversedReachability 004974a0 f   botlib:be_aas_route.obj
 0001:000965c0       _AAS_AreaTravelTime        004975c0 f   botlib:be_aas_route.obj
 0001:00096640       _AAS_CalculateAreaTravelTimes 00497640 f   botlib:be_aas_route.obj
 0001:000967c0       _AAS_PortalMaxTravelTime   004977c0 f   botlib:be_aas_route.obj
 0001:00096840       _AAS_InitPortalMaxTravelTimes 00497840 f   botlib:be_aas_route.obj
 0001:000968a0       _AAS_FreeOldestCache       004978a0 f   botlib:be_aas_route.obj
 0001:000969c0       _AAS_AllocRoutingCache     004979c0 f   botlib:be_aas_route.obj
 0001:000969f0       _AAS_FreeAllClusterAreaCache 004979f0 f   botlib:be_aas_route.obj
 0001:00096b00       _AAS_InitClusterAreaCache  00497b00 f   botlib:be_aas_route.obj
 0001:00096b70       _AAS_FreeAllPortalCache    00497b70 f   botlib:be_aas_route.obj
 0001:00096c30       _AAS_InitPortalCache       00497c30 f   botlib:be_aas_route.obj
 0001:00096c50       _AAS_InitRoutingUpdate     00497c50 f   botlib:be_aas_route.obj
 0001:00096cd0       _AAS_WriteRouteCache       00497cd0 f   botlib:be_aas_route.obj
 0001:00096f10       _AAS_ReadCache             00497f10 f   botlib:be_aas_route.obj
 0001:00096f70       _AAS_ReadRouteCache        00497f70 f   botlib:be_aas_route.obj
 0001:00097130       _AAS_InitReachabilityAreas 00498130 f   botlib:be_aas_route.obj
 0001:000972c0       _AAS_InitRouting           004982c0 f   botlib:be_aas_route.obj
 0001:00097340       _AAS_FreeRoutingCaches     00498340 f   botlib:be_aas_route.obj
 0001:00097410       _AAS_UpdateAreaRoutingCache 00498410 f   botlib:be_aas_route.obj
 0001:00097700       _AAS_GetAreaRoutingCache   00498700 f   botlib:be_aas_route.obj
 0001:000978b0       _AAS_UpdatePortalRoutingCache 004988b0 f   botlib:be_aas_route.obj
 0001:00097ad0       _AAS_GetPortalRoutingCache 00498ad0 f   botlib:be_aas_route.obj
 0001:00097c30       _AAS_AreaRouteToGoalArea   00498c30 f   botlib:be_aas_route.obj
 0001:00098020       _AAS_AreaTravelTimeToGoalArea 00499020 f   botlib:be_aas_route.obj
 0001:00098060       _AAS_AreaReachabilityToGoalArea 00499060 f   botlib:be_aas_route.obj
 0001:000980a0       _AAS_PredictRoute          004990a0 f   botlib:be_aas_route.obj
 0001:00098460       _AAS_BridgeWalkable        00499460 f   botlib:be_aas_route.obj
 0001:00098470       _AAS_ReachabilityFromNum   00499470 f   botlib:be_aas_route.obj
 0001:000984d0       _AAS_NextAreaReachability  004994d0 f   botlib:be_aas_route.obj
 0001:00098550       _AAS_NextModelReachability 00499550 f   botlib:be_aas_route.obj
 0001:000985c0       _AAS_RandomGoalArea        004995c0 f   botlib:be_aas_route.obj
 0001:00098800       _AAS_AreaVisible           00499800 f   botlib:be_aas_route.obj
 0001:00098810       _DistancePointToLine       00499810 f   botlib:be_aas_route.obj
 0001:00098870       _AAS_NearestHideArea       00499870 f   botlib:be_aas_route.obj
 0001:00098bc0       _AAS_CreateAllRoutingCache 00499bc0 f   botlib:be_aas_route.obj
 0001:00098ca0       _AAS_GetJumpPadInfo        00499ca0 f   botlib:be_aas_reach.obj
 0001:00099030       _AAS_SetupReachabilityHeap 0049a030 f   botlib:be_aas_reach.obj
 0001:00099090       _AAS_ShutDownReachabilityHeap 0049a090 f   botlib:be_aas_reach.obj
 0001:000990b0       _AAS_AllocReachability     0049a0b0 f   botlib:be_aas_reach.obj
 0001:000990f0       _AAS_FreeReachability      0049a0f0 f   botlib:be_aas_reach.obj
 0001:00099120       _AAS_AreaReachability      0049a120 f   botlib:be_aas_reach.obj
 0001:00099150       _AAS_FaceCenter            0049a150 f   botlib:be_aas_reach.obj
 0001:00099250       _AAS_FallDamageDistance    0049a250 f   botlib:be_aas_reach.obj
 0001:00099280       _AAS_FallDelta             0049a280 f   botlib:be_aas_reach.obj
 0001:000992b0       _AAS_MaxJumpHeight         0049a2b0 f   botlib:be_aas_reach.obj
 0001:000992d0       _AAS_MaxJumpDistance       0049a2d0 f   botlib:be_aas_reach.obj
 0001:00099300       _AAS_AreaCrouch            0049a300 f   botlib:be_aas_reach.obj
 0001:00099320       _AAS_AreaSwim              0049a320 f   botlib:be_aas_reach.obj
 0001:00099340       _AAS_AreaLiquid            0049a340 f   botlib:be_aas_reach.obj
 0001:00099360       _AAS_AreaLava              0049a360 f   botlib:be_aas_reach.obj
 0001:00099380       _AAS_AreaSlime             0049a380 f   botlib:be_aas_reach.obj
 0001:000993a0       _AAS_AreaGrounded          0049a3a0 f   botlib:be_aas_reach.obj
 0001:000993c0       _AAS_AreaLadder            0049a3c0 f   botlib:be_aas_reach.obj
 0001:000993e0       _AAS_AreaJumpPad           0049a3e0 f   botlib:be_aas_reach.obj
 0001:00099400       _AAS_AreaTeleporter        0049a400 f   botlib:be_aas_reach.obj
 0001:00099420       _AAS_AreaClusterPortal     0049a420 f   botlib:be_aas_reach.obj
 0001:00099440       _AAS_AreaDoNotEnter        0049a440 f   botlib:be_aas_reach.obj
 0001:00099460       _AAS_BarrierJumpTravelTime 0049a460 f   botlib:be_aas_reach.obj
 0001:00099480       _AAS_ReachabilityExists    0049a480 f   botlib:be_aas_reach.obj
 0001:000994b0       _AAS_NearbySolidOrGap      0049a4b0 f   botlib:be_aas_reach.obj
 0001:000995b0       _AAS_Reachability_EqualFloorHeight 0049a5b0 f   botlib:be_aas_reach.obj
 0001:00099b20       _AAS_Reachability_Step_Barrier_WaterJump_WalkOffLedge 0049ab20 f   botlib:be_aas_reach.obj
 0001:0009b1f0       _VectorDistance            0049c1f0 f   botlib:be_aas_reach.obj
 0001:0009b230       _VectorBetweenVectors      0049c230 f   botlib:be_aas_reach.obj
 0001:0009b290       _VectorMiddle              0049c290 f   botlib:be_aas_reach.obj
 0001:0009b2e0       _AAS_ClosestEdgePoints     0049c2e0 f   botlib:be_aas_reach.obj
 0001:0009c0f0       _AAS_Reachability_Jump     0049d0f0 f   botlib:be_aas_reach.obj
 0001:0009cc00       _AAS_TravelFlagsForTeam    0049dc00 f   botlib:be_aas_reach.obj
 0001:0009cc40       _AAS_Reachability_Teleport 0049dc40 f   botlib:be_aas_reach.obj
 0001:0009d440       _AAS_Reachability_Elevator 0049e440 f   botlib:be_aas_reach.obj
 0001:0009dda0       _AAS_FindFaceReachabilities 0049eda0 f   botlib:be_aas_reach.obj
 0001:0009e290       _AAS_Reachability_FuncBobbing 0049f290 f   botlib:be_aas_reach.obj
 0001:0009ec00       _AAS_Reachability_JumpPad  0049fc00 f   botlib:be_aas_reach.obj
 0001:0009f3d0       _AAS_Reachability_Grapple  004a03d0 f   botlib:be_aas_reach.obj
 0001:0009fa50       _AAS_Reachability_WeaponJump 004a0a50 f   botlib:be_aas_reach.obj
 0001:0009fe00       _AAS_Reachability_WalkOffLedge 004a0e00 f   botlib:be_aas_reach.obj
 0001:000a0440       _AAS_StoreReachability     004a1440 f   botlib:be_aas_reach.obj
 0001:000a0540       _AAS_FaceArea              004a1540 f   botlib:be_aas_reach.obj
 0001:000a0670       _AAS_AreaVolume            004a1670 f   botlib:be_aas_reach.obj
 0001:000a0770       _AAS_BestReachableLinkArea 004a1770 f   botlib:be_aas_reach.obj
 0001:000a07f0       _AAS_BestReachableFromJumpPadArea 004a17f0 f   botlib:be_aas_reach.obj
 0001:000a0a30       _AAS_BestReachableArea     004a1a30 f   botlib:be_aas_reach.obj
 0001:000a0cc0       _AAS_AreaGroundFaceArea    004a1cc0 f   botlib:be_aas_reach.obj
 0001:000a0d40       _AAS_Reachability_Swim     004a1d40 f   botlib:be_aas_reach.obj
 0001:000a0f80       _AAS_Reachability_Ladder   004a1f80 f   botlib:be_aas_reach.obj
 0001:000a1df0       _AAS_SetWeaponJumpAreaFlags 004a2df0 f   botlib:be_aas_reach.obj
 0001:000a20a0       _AAS_ContinueInitReachability 004a30a0 f   botlib:be_aas_reach.obj
 0001:000a23b0       _AAS_InitReachability      004a33b0 f   botlib:be_aas_reach.obj
 0001:000a2430       _AAS_Trace                 004a3430 f   botlib:be_aas_bspq3.obj
 0001:000a2480       _AAS_PointContents         004a3480 f   botlib:be_aas_bspq3.obj
 0001:000a2490       _AAS_EntityCollision       004a3490 f   botlib:be_aas_bspq3.obj
 0001:000a2500       _AAS_inPVS                 004a3500 f   botlib:be_aas_bspq3.obj
 0001:000a2510       _AAS_inPHS                 004a3510 f   botlib:be_aas_bspq3.obj
 0001:000a2520       _AAS_BSPModelMinsMaxsOrigin 004a3520 f   botlib:be_aas_bspq3.obj
 0001:000a2530       _AAS_UnlinkFromBSPLeaves   004a3530 f   botlib:be_aas_bspq3.obj
 0001:000a2540       _AAS_BSPLinkEntity         004a3540 f   botlib:be_aas_bspq3.obj
 0001:000a2550       _AAS_BoxEntities           004a3550 f   botlib:be_aas_bspq3.obj
 0001:000a2560       _AAS_NextBSPEntity         004a3560 f   botlib:be_aas_bspq3.obj
 0001:000a2580       _AAS_BSPEntityInRange      004a3580 f   botlib:be_aas_bspq3.obj
 0001:000a25b0       _AAS_ValueForBSPEpairKey   004a35b0 f   botlib:be_aas_bspq3.obj
 0001:000a2660       _AAS_VectorForBSPEpairKey  004a3660 f   botlib:be_aas_bspq3.obj
 0001:000a2700       _AAS_FloatForBSPEpairKey   004a3700 f   botlib:be_aas_bspq3.obj
 0001:000a2760       _AAS_IntForBSPEpairKey     004a3760 f   botlib:be_aas_bspq3.obj
 0001:000a27c0       _AAS_FreeBSPEntities       004a37c0 f   botlib:be_aas_bspq3.obj
 0001:000a2830       _AAS_ParseBSPEntities      004a3830 f   botlib:be_aas_bspq3.obj
 0001:000a2a90       _AAS_BSPTraceLight         004a3a90 f   botlib:be_aas_bspq3.obj
 0001:000a2aa0       _AAS_DumpBSPData           004a3aa0 f   botlib:be_aas_bspq3.obj
 0001:000a2af0       _AAS_LoadBSPFile           004a3af0 f   botlib:be_aas_bspq3.obj
 0001:000a2b90       _AAS_PresenceTypeBoundingBox 004a3b90 f   botlib:be_aas_sample.obj
 0001:000a2c90       _AAS_InitAASLinkHeap       004a3c90 f   botlib:be_aas_sample.obj
 0001:000a2d60       _AAS_FreeAASLinkHeap       004a3d60 f   botlib:be_aas_sample.obj
 0001:000a2dc0       _AAS_AllocAASLink          004a3dc0 f   botlib:be_aas_sample.obj
 0001:000a2e00       _AAS_DeAllocAASLink        004a3e00 f   botlib:be_aas_sample.obj
 0001:000a2e40       _AAS_InitAASLinkedEntities 004a3e40 f   botlib:be_aas_sample.obj
 0001:000a2e80       _AAS_FreeAASLinkedEntities 004a3e80 f   botlib:be_aas_sample.obj
 0001:000a2ea0       _AAS_PointAreaNum          004a3ea0 f   botlib:be_aas_sample.obj
 0001:000a2f70       _AAS_PointReachabilityAreaIndex 004a3f70 f   botlib:be_aas_sample.obj
 0001:000a3030       _AAS_AreaCluster           004a4030 f   botlib:be_aas_sample.obj
 0001:000a3070       _AAS_AreaPresenceType      004a4070 f   botlib:be_aas_sample.obj
 0001:000a30b0       _AAS_PointPresenceType     004a40b0 f   botlib:be_aas_sample.obj
 0001:000a30f0       _AAS_BoxOriginDistanceFromPlane 004a40f0 f   botlib:be_aas_sample.obj
 0001:000a31e0       _AAS_AreaEntityCollision   004a41e0 f   botlib:be_aas_sample.obj
 0001:000a32e0       _AAS_TraceClientBBox       004a42e0 f   botlib:be_aas_sample.obj
 0001:000a3940       _AAS_TraceAreas            004a4940 f   botlib:be_aas_sample.obj
 0001:000a3c40       _AAS_InsideFace            004a4c40 f   botlib:be_aas_sample.obj
 0001:000a3d90       _AAS_PointInsideFace       004a4d90 f   botlib:be_aas_sample.obj
 0001:000a3ef0       _AAS_AreaGroundFace        004a4ef0 f   botlib:be_aas_sample.obj
 0001:000a3fc0       _AAS_FacePlane             004a4fc0 f   botlib:be_aas_sample.obj
 0001:000a4000       _AAS_TraceEndFace          004a5000 f   botlib:be_aas_sample.obj
 0001:000a40d0       _AAS_BoxOnPlaneSide2       004a50d0 f   botlib:be_aas_sample.obj
 0001:000a41b0       _AAS_UnlinkFromAreas       004a51b0 f   botlib:be_aas_sample.obj
 0001:000a4230       _AAS_AASLinkEntity         004a5230 f   botlib:be_aas_sample.obj
 0001:000a43d0       _AAS_LinkEntityClientBBox  004a53d0 f   botlib:be_aas_sample.obj
 0001:000a4450       _AAS_BBoxAreas             004a5450 f   botlib:be_aas_sample.obj
 0001:000a44a0       _AAS_AreaInfo              004a54a0 f   botlib:be_aas_sample.obj
 0001:000a4580       _AAS_PlaneFromNum          004a5580 f   botlib:be_aas_sample.obj
 0001:000a45a0       _GeneticSelection          004a55a0 f   botlib:be_ai_gen.obj
 0001:000a4700       _GeneticParentsAndChildSelection 004a5700 f   botlib:be_ai_gen.obj
 0001:000a4a50       _GetMemory                 004a5a50 f   botlib:l_memory.obj
 0001:000a4a70       _GetClearedMemory          004a5a70 f   botlib:l_memory.obj
 0001:000a4ac0       _GetHunkMemory             004a5ac0 f   botlib:l_memory.obj
 0001:000a4ae0       _GetClearedHunkMemory      004a5ae0 f   botlib:l_memory.obj
 0001:000a4b30       _FreeMemory                004a5b30 f   botlib:l_memory.obj
 0001:000a4b50       _AvailableMemory           004a5b50 f   botlib:l_memory.obj
 0001:000a4b60       _PrintUsedMemorySize       004a5b60 f   botlib:l_memory.obj
 0001:000a4b70       _PrintMemoryLabels         004a5b70 f   botlib:l_memory.obj
 0001:000a4b80       _PS_CreatePunctuationTable 004a5b80 f   botlib:l_script.obj
 0001:000a4c80       _PunctuationFromNum        004a5c80 f   botlib:l_script.obj
 0001:000a4cd0       _ScriptError               004a5cd0 f   botlib:l_script.obj
 0001:000a4d30       _ScriptWarning             004a5d30 f   botlib:l_script.obj
 0001:000a4d90       _SetScriptPunctuations     004a5d90 f   botlib:l_script.obj
 0001:000a4dd0       _PS_ReadWhiteSpace         004a5dd0 f   botlib:l_script.obj
 0001:000a4ea0       _PS_ReadEscapeCharacter    004a5ea0 f   botlib:l_script.obj
 0001:000a50c0       _PS_ReadString             004a60c0 f   botlib:l_script.obj
 0001:000a5230       _PS_ReadName               004a6230 f   botlib:l_script.obj
 0001:000a52b0       _NumberValue               004a62b0 f   botlib:l_script.obj
 0001:000a5440       _PS_ReadNumber             004a6440 f   botlib:l_script.obj
 0001:000a5720       _PS_ReadLiteral            004a6720 f   botlib:l_script.obj
 0001:000a5810       _PS_ReadPunctuation        004a6810 f   botlib:l_script.obj
 0001:000a58b0       _PS_ReadPrimitive          004a68b0 f   botlib:l_script.obj
 0001:000a5940       _PS_ReadToken              004a6940 f   botlib:l_script.obj
 0001:000a5ae0       _PS_ExpectTokenString      004a6ae0 f   botlib:l_script.obj
 0001:000a5ba0       _PS_ExpectTokenType        004a6ba0 f   botlib:l_script.obj
 0001:000a5e80       _PS_ExpectAnyToken         004a6e80 f   botlib:l_script.obj
 0001:000a5eb0       _PS_CheckTokenString       004a6eb0 f   botlib:l_script.obj
 0001:000a5f40       _PS_CheckTokenType         004a6f40 f   botlib:l_script.obj
 0001:000a5fd0       _PS_SkipUntilString        004a6fd0 f   botlib:l_script.obj
 0001:000a6070       _PS_UnreadLastToken        004a7070 f   botlib:l_script.obj
 0001:000a6080       _PS_UnreadToken            004a7080 f   botlib:l_script.obj
 0001:000a60b0       _PS_NextWhiteSpaceChar     004a70b0 f   botlib:l_script.obj
 0001:000a60d0       _StripDoubleQuotes         004a70d0 f   botlib:l_script.obj
 0001:000a6120       _StripSingleQuotes         004a7120 f   botlib:l_script.obj
 0001:000a6170       _ReadSignedFloat           004a7170 f   botlib:l_script.obj
 0001:000a6220       _ReadSignedInt             004a7220 f   botlib:l_script.obj
 0001:000a62e0       _SetScriptFlags            004a72e0 f   botlib:l_script.obj
 0001:000a62f0       _GetScriptFlags            004a72f0 f   botlib:l_script.obj
 0001:000a6300       _ResetScript               004a7300 f   botlib:l_script.obj
 0001:000a6350       _EndOfScript               004a7350 f   botlib:l_script.obj
 0001:000a6370       _NumLinesCrossed           004a7370 f   botlib:l_script.obj
 0001:000a6390       _ScriptSkipTo              004a7390 f   botlib:l_script.obj
 0001:000a6410       _LoadScriptFile            004a7410 f   botlib:l_script.obj
 0001:000a6560       _LoadScriptMemory          004a7560 f   botlib:l_script.obj
 0001:000a6620       _FreeScript                004a7620 f   botlib:l_script.obj
 0001:000a6650       _PS_SetBaseFolder          004a7650 f   botlib:l_script.obj
 0001:000a6670       _FindField                 004a7670 f   botlib:l_struct.obj
 0001:000a66e0       _ReadNumber                004a76e0 f   botlib:l_struct.obj
 0001:000a6a30       _ReadChar                  004a7a30 f   botlib:l_struct.obj
 0001:000a6ab0       _ReadString                004a7ab0 f   botlib:l_struct.obj
 0001:000a6b10       _ReadStructure             004a7b10 f   botlib:l_struct.obj
 0001:000a6db0       _WriteIndent               004a7db0 f   botlib:l_struct.obj
 0001:000a6df0       _WriteFloat                004a7df0 f   botlib:l_struct.obj
 0001:000a6e80       _WriteStructWithIndent     004a7e80 f   botlib:l_struct.obj
 0001:000a70d0       _WriteStructure            004a80d0 f   botlib:l_struct.obj
 0001:000a70f0       _AAS_SwapAASData           004a80f0 f   botlib:be_aas_file.obj
 0001:000a7250       _AAS_DumpAASData           004a8250 f   botlib:be_aas_file.obj
 0001:000a7420       _AAS_LoadAASLump           004a8420 f   botlib:be_aas_file.obj
 0001:000a74b0       _AAS_DData                 004a84b0 f   botlib:be_aas_file.obj
 0001:000a74e0       _AAS_LoadAASFile           004a84e0 f   botlib:be_aas_file.obj
 0001:000a79b0       _AAS_WriteAASLump          004a89b0 f   botlib:be_aas_file.obj
 0001:000a79f0       _AAS_WriteAASFile          004a89f0 f   botlib:be_aas_file.obj
 0001:000a7d80       _AAS_KeepEdge              004a8d80 f   botlib:be_aas_optimize.obj
 0001:000a7d90       _AAS_OptimizeEdge          004a8d90 f   botlib:be_aas_optimize.obj
 0001:000a7ee0       _AAS_KeepFace              004a8ee0 f   botlib:be_aas_optimize.obj
 0001:000a7ef0       _AAS_OptimizeFace          004a8ef0 f   botlib:be_aas_optimize.obj
 0001:000a7fc0       _AAS_OptimizeArea          004a8fc0 f   botlib:be_aas_optimize.obj
 0001:000a8040       _AAS_OptimizeAlloc         004a9040 f   botlib:be_aas_optimize.obj
 0001:000a8140       _AAS_OptimizeStore         004a9140 f   botlib:be_aas_optimize.obj
 0001:000a8240       _AAS_Optimize              004a9240 f   botlib:be_aas_optimize.obj
 0001:000a8340       _AAS_RemoveClusterAreas    004a9340 f   botlib:be_aas_cluster.obj
 0001:000a8380       _AAS_ClearCluster          004a9380 f   botlib:be_aas_cluster.obj
 0001:000a83d0       _AAS_RemovePortalsClusterReference 004a93d0 f   botlib:be_aas_cluster.obj
 0001:000a8430       _AAS_UpdatePortal          004a9430 f   botlib:be_aas_cluster.obj
 0001:000a8530       _AAS_FloodClusterAreas_r   004a9530 f   botlib:be_aas_cluster.obj
 0001:000a86b0       _AAS_FloodClusterAreasUsingReachabilities 004a96b0 f   botlib:be_aas_cluster.obj
 0001:000a8750       _AAS_NumberClusterPortals  004a9750 f   botlib:be_aas_cluster.obj
 0001:000a87b0       _AAS_NumberClusterAreas    004a97b0 f   botlib:be_aas_cluster.obj
 0001:000a8970       _AAS_FindClusters          004a9970 f   botlib:be_aas_cluster.obj
 0001:000a8a60       _AAS_CreatePortals         004a9a60 f   botlib:be_aas_cluster.obj
 0001:000a8ae0       _AAS_ConnectedAreas_r      004a9ae0 f   botlib:be_aas_cluster.obj
 0001:000a8b90       _AAS_ConnectedAreas        004a9b90 f   botlib:be_aas_cluster.obj
 0001:000a8c10       _AAS_GetAdjacentAreasWithLessPresenceTypes_r 004a9c10 f   botlib:be_aas_cluster.obj
 0001:000a8d10       _AAS_CheckAreaForPossiblePortals 004a9d10 f   botlib:be_aas_cluster.obj
 0001:000a90f0       _AAS_FindPossiblePortals   004aa0f0 f   botlib:be_aas_cluster.obj
 0001:000a9130       _AAS_RemoveAllPortals      004aa130 f   botlib:be_aas_cluster.obj
 0001:000a9170       _AAS_TestPortals           004aa170 f   botlib:be_aas_cluster.obj
 0001:000a9200       _AAS_CountForcedClusterPortals 004aa200 f   botlib:be_aas_cluster.obj
 0001:000a9260       _AAS_CreateViewPortals     004aa260 f   botlib:be_aas_cluster.obj
 0001:000a92b0       _AAS_SetViewPortalsAsClusterPortals 004aa2b0 f   botlib:be_aas_cluster.obj
 0001:000a9300       _AAS_InitClustering        004aa300 f   botlib:be_aas_cluster.obj
 0001:000a9520       _AAS_ClearShownPolygons    004aa520 f   botlib:be_aas_debug.obj
 0001:000a9550       _AAS_ShowPolygon           004aa550 f   botlib:be_aas_debug.obj
 0001:000a9590       _AAS_ClearShownDebugLines  004aa590 f   botlib:be_aas_debug.obj
 0001:000a95d0       _AAS_DebugLine             004aa5d0 f   botlib:be_aas_debug.obj
 0001:000a9650       _AAS_PermanentLine         004aa650 f   botlib:be_aas_debug.obj
 0001:000a9670       _AAS_DrawPermanentCross    004aa670 f   botlib:be_aas_debug.obj
 0001:000a9700       _AAS_DrawPlaneCross        004aa700 f   botlib:be_aas_debug.obj
 0001:000a9940       _AAS_ShowBoundingBox       004aa940 f   botlib:be_aas_debug.obj
 0001:000a9ad0       _AAS_ShowFace              004aaad0 f   botlib:be_aas_debug.obj
 0001:000a9c40       _AAS_ShowFacePolygon       004aac40 f   botlib:be_aas_debug.obj
 0001:000a9f60       _AAS_ShowArea              004aaf60 f   botlib:be_aas_debug.obj
 0001:000aa190       _AAS_ShowAreaPolygons      004ab190 f   botlib:be_aas_debug.obj
 0001:000aa260       _AAS_DrawCross             004ab260 f   botlib:be_aas_debug.obj
 0001:000aa2d0       _AAS_PrintTravelType       004ab2d0 f   botlib:be_aas_debug.obj
 0001:000aa2e0       _AAS_DrawArrow             004ab2e0 f   botlib:be_aas_debug.obj
 0001:000aa470       _AAS_ShowReachability      004ab470 f   botlib:be_aas_debug.obj
 0001:000aa700       _AAS_ShowReachableAreas    004ab700 f   botlib:be_aas_debug.obj
 0001:000aa7b0       _AAS_FloodAreas_r          004ab7b0 f   botlib:be_aas_debug.obj
 0001:000aa8f0       _AAS_FloodAreas            004ab8f0 f   botlib:be_aas_debug.obj
 0001:000aa930       _CRC_Init                  004ab930 f   botlib:l_crc.obj
 0001:000aa940       _CRC_ProcessByte           004ab940 f   botlib:l_crc.obj
 0001:000aa970       _CRC_Value                 004ab970 f   botlib:l_crc.obj
 0001:000aa980       _CRC_ProcessString         004ab980 f   botlib:l_crc.obj
 0001:000aa9d0       _CRC_ContinueProcessString 004ab9d0 f   botlib:l_crc.obj
 0001:000aaa0e       __fpclear                  004aba0e f   LIBC:fpinit.obj
 0001:000aaa0f       __cfltcvt_init             004aba0f f   LIBC:fpinit.obj
 0001:000aaa47       ___setfflag                004aba47 f   LIBC:fpinit.obj
 0001:000aaa57       __fpmath                   004aba57 f   LIBC:fpinit.obj
 0001:000aaa75       _atol                      004aba75 f   LIBC:atox.obj
 0001:000aaacd       _atoi                      004abacd f   LIBC:atox.obj
 0001:000aaad2       __atoi64                   004abad2 f   LIBC:atox.obj
 0001:000aab50       __alloca_probe             004abb50     LIBC:chkstk.obj
 0001:000aab50       __chkstk                   004abb50 f   LIBC:chkstk.obj
 0001:000aab90       _ceil                      004abb90 f   LIBC:ceil_pentium4.obj
 0001:000aabd0       __ceil_pentium4            004abbd0 f   LIBC:ceil_pentium4.obj
 0001:000aacb0       _floor                     004abcb0 f   LIBC:floor_pentium4.obj
 0001:000aacf0       __floor_pentium4           004abcf0 f   LIBC:floor_pentium4.obj
 0001:000aade0       _strncpy                   004abde0 f   LIBC:strncpy.obj
 0001:000aaf04       __ftol2                    004abf04 f   LIBC:ftol2.obj
 0001:000aaf80       _strstr                    004abf80 f   LIBC:strstr.obj
 0001:000ab010       _memmove                   004ac010 f   LIBC:memmove.obj
 0001:000ab34d       _time                      004ac34d f   LIBC:time.obj
 0001:000ab386       __tolower                  004ac386 f   LIBC:tolower.obj
 0001:000ab38e       _tolower                   004ac38e f   LIBC:tolower.obj
 0001:000ab463       _srand                     004ac463 f   LIBC:rand.obj
 0001:000ab46d       _rand                      004ac46d f   LIBC:rand.obj
 0001:000ab490       _getenv                    004ac490 f   LIBC:getenv.obj
 0001:000ab511       __vsnprintf                004ac511 f   LIBC:vsnprint.obj
 0001:000ab567       _printf                    004ac567 f   LIBC:printf.obj
 0001:000ab5a0       _strncat                   004ac5a0 f   LIBC:strncat.obj
 0001:000ab6f0       _strchr                    004ac6f0 f   LIBC:strchr.obj
 0001:000ab6f6       ___from_strstr_to_strchr   004ac6f6     LIBC:strchr.obj
 0001:000ab7ae       _sscanf                    004ac7ae f   LIBC:sscanf.obj
 0001:000ab7e2       _sprintf                   004ac7e2 f   LIBC:sprintf.obj
 0001:000ab83a       __scprintf                 004ac83a f   LIBC:sprintf.obj
 0001:000ab881       _asctime                   004ac881 f   LIBC:asctime.obj
 0001:000ab96b       _localtime                 004ac96b f   LIBC:localtim.obj
 0001:000abaeb       __toupper                  004acaeb f   LIBC:toupper.obj
 0001:000abaf3       _toupper                   004acaf3 f   LIBC:toupper.obj
 0001:000abbd0       __CIacos                   004acbd0 f   LIBC:acos.obj
 0001:000abbe4       _acos                      004acbe4     LIBC:acos.obj
 0001:000abc9c       _longjmp                   004acc9c f   LIBC:longjmp.obj
 0001:000abd15       _vsprintf                  004acd15 f   LIBC:vsprintf.obj
 0001:000abd6c       __vscprintf                004acd6c f   LIBC:vsprintf.obj
 0001:000abd9c       _calloc                    004acd9c f   LIBC:calloc.obj
 0001:000abe17       _atof                      004ace17 f   LIBC:atof.obj
 0001:000abe64       __setjmp3                  004ace64 f   LIBC:setjmp3.obj
 0001:000abedf       _setvbuf                   004acedf f   LIBC:setvbuf.obj
 0001:000abf80       _fseek                     004acf80 f   LIBC:fseek.obj
 0001:000ac00e       _ftell                     004ad00e f   LIBC:ftell.obj
 0001:000ac167       _free                      004ad167 f   LIBC:free.obj
 0001:000ac19f       _fwrite                    004ad19f f   LIBC:fwrite.obj
 0001:000ac2a6       _fclose                    004ad2a6 f   LIBC:fclose.obj
 0001:000ac2fc       _fread                     004ad2fc f   LIBC:fread.obj
 0001:000ac3e5       __heap_alloc               004ad3e5 f   LIBC:malloc.obj
 0001:000ac42b       __nh_malloc                004ad42b f   LIBC:malloc.obj
 0001:000ac457       _malloc                    004ad457 f   LIBC:malloc.obj
 0001:000ac469       __fsopen                   004ad469 f   LIBC:fopen.obj
 0001:000ac493       _fopen                     004ad493 f   LIBC:fopen.obj
 0001:000ac4a6       _remove                    004ad4a6 f   LIBC:unlink.obj
 0001:000ac4d0       __unlink                   004ad4d0 f   LIBC:unlink.obj
 0001:000ac4d5       _rename                    004ad4d5 f   LIBC:rename.obj
 0001:000ac503       __flush                    004ad503 f   LIBC:fflush.obj
 0001:000ac560       _fflush                    004ad560 f   LIBC:fflush.obj
 0001:000ac608       __flushall                 004ad608 f   LIBC:fflush.obj
 0001:000ac6b0       _qsort                     004ad6b0 f   LIBC:qsort.obj
 0001:000ac940       _strncmp                   004ad940 f   LIBC:strncmp.obj
 0001:000ac979       _fprintf                   004ad979 f   LIBC:fprintf.obj
 0001:000ac9ac       __ftol                     004ad9ac f   LIBC:ftol.obj
 0001:000ac9d3       __commit                   004ad9d3 f   LIBC:commit.obj
 0001:000aca2a       ___crtExitProcess          004ada2a f   LIBC:crt0dat.obj
 0001:000aca90       __cinit                    004ada90 f   LIBC:crt0dat.obj
 0001:000acbbb       _exit                      004adbbb f   LIBC:crt0dat.obj
 0001:000acbcc       __exit                     004adbcc f   LIBC:crt0dat.obj
 0001:000acbdd       __cexit                    004adbdd f   LIBC:crt0dat.obj
 0001:000acbec       __c_exit                   004adbec f   LIBC:crt0dat.obj
 0001:000acbfb       __mkdir                    004adbfb f   LIBC:mkdir.obj
 0001:000acc27       __validdrive               004adc27 f   LIBC:getcwd.obj
 0001:000acc5e       __getdcwd                  004adc5e f   LIBC:getcwd.obj
 0001:000acd45       __getcwd                   004add45 f   LIBC:getcwd.obj
 0001:000acd58       __findclose                004add58 f   LIBC:findfile.obj
 0001:000acd77       ___timet_from_ft           004add77 f   LIBC:findfile.obj
 0001:000acddb       __findfirst                004adddb f   LIBC:findfile.obj
 0001:000aceb5       __findnext                 004adeb5 f   LIBC:findfile.obj
 0001:000acf8a       _strtok                    004adf8a f   LIBC:strtok.obj
 0001:000ad037       __amsg_exit                004ae037 f   LIBC:wincrt0.obj
 0001:000ad0d6       _WinMainCRTStartup         004ae0d6 f   LIBC:wincrt0.obj
 0001:000ad2c0       _pow                       004ae2c0 f   LIBC:pow.obj
 0001:000ad300       __CIpow                    004ae300 f   LIBC:pow.obj
 0001:000ad33b       __CIpow_default            004ae33b f   LIBC:pow.obj
 0001:000ad354       __pow_default              004ae354     LIBC:pow.obj
 0001:000ad550       _strrchr                   004ae550 f   LIBC:strrchr.obj
 0001:000ad57d       _putenv                    004ae57d f   LIBC:putenv.obj
 0001:000ad57d       __putenv                   004ae57d f   LIBC:putenv.obj
 0001:000ad644       _clock                     004ae644 f   LIBC:clock.obj
 0001:000ad687       ___inittime                004ae687 f   LIBC:clock.obj
 0001:000ad6be       _vfprintf                  004ae6be f   LIBC:vfprintf.obj
 0001:000ad6ef       _ctime                     004ae6ef f   LIBC:ctime.obj
 0001:000ad708       __forcdecpt                004ae708 f   LIBC:cvt.obj
 0001:000ad760       __cropzeros                004ae760 f   LIBC:cvt.obj
 0001:000ad7ab       __positive                 004ae7ab f   LIBC:cvt.obj
 0001:000ad7c5       __fassign                  004ae7c5 f   LIBC:cvt.obj
 0001:000ad820       __cftoe                    004ae820 f   LIBC:cvt.obj
 0001:000ad938       __cftof                    004ae938 f   LIBC:cvt.obj
 0001:000ada38       __cftog                    004aea38 f   LIBC:cvt.obj
 0001:000adae2       __cfltcvt                  004aeae2 f   LIBC:cvt.obj
 0001:000adb33       __setdefaultprecision      004aeb33 f   LIBC:fp8.obj
 0001:000adb45       __ms_p5_test_fdiv          004aeb45 f   LIBC:testfdiv.obj
 0001:000adb85       __ms_p5_mp_test_fdiv       004aeb85 f   LIBC:testfdiv.obj
 0001:000adbae       __ismbcspace               004aebae f   LIBC:ismbspc.obj
 0001:000adc40       __allmul                   004aec40 f   LIBC:llmul.obj
 0001:000adc74       ___libm_error_support      004aec74 f   LIBC:libm_error.obj
 0001:000adf35       ___sse2_available_init     004aef35 f   LIBC:cpu_disp.obj
 0001:000ae003       __set_SSE2_enable          004af003 f   LIBC:cpu_disp.obj
 0001:000ae017       __ceil_default             004af017 f   LIBC:ceil.obj
 0001:000ae0ea       __floor_default            004af0ea f   LIBC:floor.obj
 0001:000ae1c0       __aulldiv                  004af1c0 f   LIBC:ulldiv.obj
 0001:000ae244       ___crtLCMapStringA         004af244 f   LIBC:a_map.obj
 0001:000ae600       ___pwctype_func            004af600 f   LIBC:ctype.obj
 0001:000ae606       ___pctype_func             004af606 f   LIBC:ctype.obj
 0001:000ae60c       __chvalidator              004af60c f   LIBC:isctype.obj
 0001:000ae61f       __isctype                  004af61f f   LIBC:isctype.obj
 0001:000ae69d       __mbsnbicoll               004af69d f   LIBC:mbsnbico.obj
 0001:000ae6e0       _strlen                    004af6e0 f   LIBC:strlen.obj
 0001:000ae76b       ___wtomb_environ           004af76b f   LIBC:wtombenv.obj
 0001:000ae7fb       __flsbuf                   004af7fb f   LIBC:_flsbuf.obj
 0001:000ae9be       __output                   004af9be f   LIBC:output.obj
 0001:000af1b8       __stbuf                    004b01b8 f   LIBC:_sftbuf.obj
 0001:000af240       __ftbuf                    004b0240 f   LIBC:_sftbuf.obj
 0001:000af27c       ___iob_func                004b027c f   LIBC:_file.obj
 0001:000af282       ___initstdio               004b0282 f   LIBC:_file.obj
 0001:000af328       ___endstdio                004b0328 f   LIBC:_file.obj
 0001:000af3ae       __input                    004b03ae f   LIBC:input.obj
 0001:000b0215       __tzset                    004b1215 f   LIBC:tzset.obj
 0001:000b0620       __isindst                  004b1620 f   LIBC:tzset.obj
 0001:000b07ad       ___tzset                   004b17ad f   LIBC:tzset.obj
 0001:000b07c2       _gmtime                    004b17c2 f   LIBC:gmtime.obj
 0001:000b08c0       __trandisp1                004b18c0 f   LIBC:87disp.obj
 0001:000b0927       __trandisp2                004b1927 f   LIBC:87disp.obj
 0001:000b09b3       __rttospopde               004b19b3     LIBC:87disp.obj
 0001:000b09b8       __rttospop                 004b19b8     LIBC:87disp.obj
 0001:000b09ba       __rtnospop                 004b19ba     LIBC:87disp.obj
 0001:000b09bc       __rttosnpop                004b19bc     LIBC:87disp.obj
 0001:000b09bd       __rtnospopde               004b19bd     LIBC:87disp.obj
 0001:000b09c4       __rtzeropop                004b19c4     LIBC:87disp.obj
 0001:000b09c6       __rtzeronpop               004b19c6     LIBC:87disp.obj
 0001:000b09cb       __rtonepop                 004b19cb     LIBC:87disp.obj
 0001:000b09cd       __rtonenpop                004b19cd     LIBC:87disp.obj
 0001:000b09d2       __tosnan1                  004b19d2     LIBC:87disp.obj
 0001:000b09fd       __nosnan2                  004b19fd     LIBC:87disp.obj
 0001:000b09ff       __tosnan2                  004b19ff     LIBC:87disp.obj
 0001:000b0a27       __nan2                     004b1a27     LIBC:87disp.obj
 0001:000b0a66       __rtindfpop                004b1a66     LIBC:87disp.obj
 0001:000b0a68       __rtindfnpop               004b1a68     LIBC:87disp.obj
 0001:000b0a79       __rttosnpopde              004b1a79     LIBC:87disp.obj
 0001:000b0a83       __rtchsifneg               004b1a83     LIBC:87disp.obj
 0001:000b0a90       __startTwoArgErrorHandling 004b1a90 f   LIBC:genexcep.obj
 0001:000b0aa7       __startOneArgErrorHandling 004b1aa7 f   LIBC:genexcep.obj
 0001:000b0af0       __twoToTOS                 004b1af0 f   LIBC:common.obj
 0001:000b0b05       __load_CW                  004b1b05 f   LIBC:common.obj
 0001:000b0b1c       __convertTOStoQNaN         004b1b1c f   LIBC:common.obj
 0001:000b0b35       __fload_withFB             004b1b35 f   LIBC:common.obj
 0001:000b0b78       __checkTOS_withFB          004b1b78 f   LIBC:common.obj
 0001:000b0b8e       __fast_exit                004b1b8e f   LIBC:common.obj
 0001:000b0b9b       __math_exit                004b1b9b f   LIBC:common.obj
 0001:000b0bc5       __check_overflow_exit      004b1bc5 f   LIBC:common.obj
 0001:000b0bd9       __check_range_exit         004b1bd9 f   LIBC:common.obj
 0001:000b0c7c       __global_unwind2           004b1c7c f   LIBC:exsup.obj
 0001:000b0cbe       __local_unwind2            004b1cbe f   LIBC:exsup.obj
 0001:000b0d16       __NLG_Return2              004b1d16     LIBC:exsup.obj
 0001:000b0d26       __abnormal_termination     004b1d26 f   LIBC:exsup.obj
 0001:000b0d49       __NLG_Notify1              004b1d49 f   LIBC:exsup.obj
 0001:000b0d52       __NLG_Notify               004b1d52 f   LIBC:exsup.obj
 0001:000b0d65       __NLG_Dispatch             004b1d65     LIBC:exsup.obj
 0001:000b0d6a       __rt_probe_read4@4         004b1d6a f   LIBC:sehsupp.obj
 0001:000b0db0       _memset                    004b1db0 f   LIBC:memset.obj
 0001:000b0e10       ?_set_new_handler@@YAP6AHI@ZP6AHI@Z@Z 004b1e10 f   LIBC:handler.obj
 0001:000b0e20       ?_query_new_handler@@YAP6AHI@ZXZ 004b1e20 f   LIBC:handler.obj
 0001:000b0e26       __callnewh                 004b1e26 f   LIBC:handler.obj
 0001:000b0e41       ___heap_select             004b1e41 f   LIBC:heapinit.obj
 0001:000b0e5b       __heap_init                004b1e5b f   LIBC:heapinit.obj
 0001:000b0eac       __heap_term                004b1eac f   LIBC:heapinit.obj
 0001:000b0f2b       __get_heap_handle          004b1f2b f   LIBC:heapinit.obj
 0001:000b0f31       __get_sbh_threshold        004b1f31 f   LIBC:sbheap.obj
 0001:000b0f46       ___sbh_heap_init           004b1f46 f   LIBC:sbheap.obj
 0001:000b0f8e       ___sbh_find_block          004b1f8e f   LIBC:sbheap.obj
 0001:000b0fb9       ___sbh_free_block          004b1fb9 f   LIBC:sbheap.obj
 0001:000b12d1       ___sbh_alloc_new_region    004b22d1 f   LIBC:sbheap.obj
 0001:000b1388       ___sbh_alloc_new_group     004b2388 f   LIBC:sbheap.obj
 0001:000b148e       ___sbh_resize_block        004b248e f   LIBC:sbheap.obj
 0001:000b176d       ___sbh_heapmin             004b276d f   LIBC:sbheap.obj
 0001:000b183e       ___sbh_heap_check          004b283e f   LIBC:sbheap.obj
 0001:000b1b57       __set_sbh_threshold        004b2b57 f   LIBC:sbheap.obj
 0001:000b1bb2       ___sbh_alloc_block         004b2bb2 f   LIBC:sbheap.obj
 0001:000b1eae       __fltin                    004b2eae f   LIBC:cfin.obj
 0001:000b1f45       __freebuf                  004b2f45 f   LIBC:_freebuf.obj
 0001:000b1f70       __lseek                    004b2f70 f   LIBC:lseek.obj
 0001:000b1ffc       __ioinit                   004b2ffc f   LIBC:ioinit.obj
 0001:000b21a7       __ioterm                   004b31a7 f   LIBC:ioinit.obj
 0001:000b21ca       _write                     004b31ca f   LIBC:write.obj
 0001:000b21ca       __write                    004b31ca f   LIBC:write.obj
 0001:000b23c0       _memcpy                    004b33c0 f   LIBC:memcpy.obj
 0001:000b26fd       _close                     004b36fd f   LIBC:close.obj
 0001:000b26fd       __close                    004b36fd f   LIBC:close.obj
 0001:000b27b0       __filbuf                   004b37b0 f   LIBC:_filbuf.obj
 0001:000b288e       __read                     004b388e f   LIBC:read.obj
 0001:000b2a7c       __openfile                 004b3a7c f   LIBC:_open.obj
 0001:000b2be4       __getstream                004b3be4 f   LIBC:stream.obj
 0001:000b2c56       __dosmaperr                004b3c56 f   LIBC:dosmap.obj
 0001:000b2cb5       __alloc_osfhnd             004b3cb5 f   LIBC:osfinfo.obj
 0001:000b2d52       __set_osfhnd               004b3d52 f   LIBC:osfinfo.obj
 0001:000b2dc9       __free_osfhnd              004b3dc9 f   LIBC:osfinfo.obj
 0001:000b2e43       __get_osfhandle            004b3e43 f   LIBC:osfinfo.obj
 0001:000b2e7f       __open_osfhandle           004b3e7f f   LIBC:osfinfo.obj
 0001:000b2f1c       __onexit                   004b3f1c f   LIBC:onexit.obj
 0001:000b2f9e       _atexit                    004b3f9e f   LIBC:onexit.obj
 0001:000b2fb0       ___onexitinit              004b3fb0 f   LIBC:onexit.obj
 0001:000b2fd8       __RTC_Initialize           004b3fd8 f   LIBC:initsect.obj
 0001:000b301c       __RTC_Terminate            004b401c f   LIBC:initsect.obj
 0001:000b3060       _strcpy                    004b4060 f   LIBC:strcat.obj
 0001:000b3070       _strcat                    004b4070 f   LIBC:strcat.obj
 0001:000b3189       @__security_check_cookie@4 004b4189 f   LIBC:secchk.obj
 0001:000b3197       ___loctotime_t             004b4197 f   LIBC:dtoxtime.obj
 0001:000b32a5       __NMSG_WRITE               004b42a5 f   LIBC:crt0msg.obj
 0001:000b341c       __GET_RTERRMSG             004b441c f   LIBC:crt0msg.obj
 0001:000b3446       __FF_MSGBANNER             004b4446 f   LIBC:crt0msg.obj
 0001:000b34b6       __XcptFilter               004b44b6 f   LIBC:winxfltr.obj
 0001:000b3627       ___CppXcptFilter           004b4627 f   LIBC:winxfltr.obj
 0001:000b3642       __wincmdln                 004b4642 f   LIBC:wincmdln.obj
 0001:000b369f       __setenvp                  004b469f f   LIBC:stdenvp.obj
 0001:000b38d2       __setargv                  004b48d2 f   LIBC:stdargv.obj
 0001:000b3974       ___crtGetEnvironmentStringsA 004b4974 f   LIBC:a_env.obj
 0001:000b3a98       __SEH_prolog               004b4a98 f   LIBC:sehprolg.obj
 0001:000b3ad3       __SEH_epilog               004b4ad3 f   LIBC:sehprolg.obj
 0001:000b3aec       __except_handler3          004b4aec f   LIBC:exsup3.obj
 0001:000b3bd2       __seh_longjmp_unwind@4     004b4bd2 f   LIBC:exsup3.obj
 0001:000b3bf0       __CIpow_pentium4           004b4bf0 f   LIBC:pow_pentium4.obj
 0001:000b3c09       __pow_pentium4             004b4c09     LIBC:pow_pentium4.obj
 0001:000b4751       __fFEXP                    004b5751     LIBC:87tran.obj
 0001:000b47b8       __rtinfpopse               004b57b8     LIBC:87tran.obj
 0001:000b47ba       __rtinfnpopse              004b57ba     LIBC:87tran.obj
 0001:000b47ca       __fFLN                     004b57ca     LIBC:87tran.obj
 0001:000b487f       __rtinfpop                 004b587f     LIBC:87tran.obj
 0001:000b4881       __rtinfnpop                004b5881     LIBC:87tran.obj
 0001:000b489e       __ffexpm1                  004b589e     LIBC:87tran.obj
 0001:000b4947       __d_inttype                004b5947 f   LIBC:powhlp.obj
 0001:000b49b5       __powhlp                   004b59b5 f   LIBC:powhlp.obj
 0001:000b4bc9       ___crtwsetenv              004b5bc9 f   LIBC:wsetenv.obj
 0001:000b4f43       ___crtsetenv               004b5f43 f   LIBC:setenv.obj
 0001:000b5118       __ZeroTail                 004b6118 f   LIBC:intrncvt.obj
 0001:000b514a       __IncMan                   004b614a f   LIBC:intrncvt.obj
 0001:000b5197       __RoundMan                 004b6197 f   LIBC:intrncvt.obj
 0001:000b5209       __CopyMan                  004b6209 f   LIBC:intrncvt.obj
 0001:000b5224       __FillZeroMan              004b6224 f   LIBC:intrncvt.obj
 0001:000b5230       __IsZeroMan                004b6230 f   LIBC:intrncvt.obj
 0001:000b5249       __ShrMan                   004b6249 f   LIBC:intrncvt.obj
 0001:000b52c4       __ld12cvt                  004b62c4 f   LIBC:intrncvt.obj
 0001:000b541c       __ld12tod                  004b641c f   LIBC:intrncvt.obj
 0001:000b5432       __ld12tof                  004b6432 f   LIBC:intrncvt.obj
 0001:000b5448       __ld12told                 004b6448 f   LIBC:intrncvt.obj
 0001:000b54c4       __atodbl                   004b64c4 f   LIBC:intrncvt.obj
 0001:000b5501       __atoldbl                  004b6501 f   LIBC:intrncvt.obj
 0001:000b553f       __atoflt                   004b653f f   LIBC:intrncvt.obj
 0001:000b557c       __fptostr                  004b657c f   LIBC:_fptostr.obj
 0001:000b55f3       ___dtold                   004b65f3 f   LIBC:cfout.obj
 0001:000b56ad       __fltout                   004b66ad f   LIBC:cfout.obj
 0001:000b5721       __fptrap                   004b6721 f   LIBC:crt0fp.obj
 0001:000b572a       __fpreset                  004b672a f   LIBC:ieee87.obj
 0001:000b58ad       __statusfp                 004b68ad f   LIBC:ieee87.obj
 0001:000b58bd       __clearfp                  004b68bd f   LIBC:ieee87.obj
 0001:000b58ce       __control87                004b68ce f   LIBC:ieee87.obj
 0001:000b5900       __controlfp                004b6900 f   LIBC:ieee87.obj
 0001:000b5916       ___crtGetStringTypeA       004b6916 f   LIBC:a_str.obj
 0001:000b5cfa       __setmbcp                  004b6cfa f   LIBC:mbctype.obj
 0001:000b5ee0       __getmbcp                  004b6ee0 f   LIBC:mbctype.obj
 0001:000b5ef0       ___initmbctable            004b6ef0 f   LIBC:mbctype.obj
 0001:000b5f0e       __matherr                  004b6f0e f   LIBC:matherr.obj
 0001:000b5f11       __raise_exc                004b6f11 f   LIBC:fpexcept.obj
 0001:000b61b6       __handle_exc               004b71b6 f   LIBC:fpexcept.obj
 0001:000b63da       __set_errno                004b73da f   LIBC:fpexcept.obj
 0001:000b6420       __errcode                  004b7420 f   LIBC:fpexcept.obj
 0001:000b644d       __umatherr                 004b744d f   LIBC:fpexcept.obj
 0001:000b64ed       __handle_qnan1             004b74ed f   LIBC:fpexcept.obj
 0001:000b653f       __handle_qnan2             004b753f f   LIBC:fpexcept.obj
 0001:000b659d       __except1                  004b759d f   LIBC:fpexcept.obj
 0001:000b6655       __except2                  004b7655 f   LIBC:fpexcept.obj
 0001:000b671e       __frnd                     004b771e f   LIBC:frnd.obj
 0001:000b672f       __set_exp                  004b772f f   LIBC:util.obj
 0001:000b6759       __get_exp                  004b7759 f   LIBC:util.obj
 0001:000b676e       __add_exp                  004b776e f   LIBC:util.obj
 0001:000b6798       __set_bexp                 004b7798 f   LIBC:util.obj
 0001:000b67bd       __sptype                   004b77bd f   LIBC:util.obj
 0001:000b6818       __decomp                   004b7818 f   LIBC:util.obj
 0001:000b68d4       __statfp                   004b78d4 f   LIBC:fpctrl.obj
 0001:000b68df       __clrfp                    004b78df f   LIBC:fpctrl.obj
 0001:000b68eb       __ctrlfp                   004b78eb f   LIBC:fpctrl.obj
 0001:000b690f       __set_statfp               004b790f f   LIBC:fpctrl.obj
 0001:000b6965       ___ansicp                  004b7965 f   LIBC:convrtcp.obj
 0001:000b69a8       ___convertcp               004b79a8 f   LIBC:convrtcp.obj
 0001:000b6b71       __resetstkoflw             004b7b71 f   LIBC:resetstk.obj
 0001:000b6c70       ___crtCompareStringA       004b7c70 f   LIBC:a_cmp.obj
 0001:000b6ff4       __getbuf                   004b7ff4 f   LIBC:_getbuf.obj
 0001:000b7038       __isatty                   004b8038 f   LIBC:isatty.obj
 0001:000b705f       _wctomb                    004b805f f   LIBC:wctomb.obj
 0001:000b70d0       __aulldvrm                 004b80d0 f   LIBC:ulldvrm.obj
 0001:000b7165       __fcloseall                004b8165 f   LIBC:closeall.obj
 0001:000b71bd       _ungetc                    004b81bd f   LIBC:ungetc.obj
 0001:000b7229       _isalpha                   004b8229 f   LIBC:_ctype.obj
 0001:000b7257       _isupper                   004b8257 f   LIBC:_ctype.obj
 0001:000b7280       _islower                   004b8280 f   LIBC:_ctype.obj
 0001:000b72a9       _isdigit                   004b82a9 f   LIBC:_ctype.obj
 0001:000b72d2       _isxdigit                  004b82d2 f   LIBC:_ctype.obj
 0001:000b7300       _isspace                   004b8300 f   LIBC:_ctype.obj
 0001:000b7329       _ispunct                   004b8329 f   LIBC:_ctype.obj
 0001:000b7352       _isalnum                   004b8352 f   LIBC:_ctype.obj
 0001:000b7380       _isprint                   004b8380 f   LIBC:_ctype.obj
 0001:000b73ae       _isgraph                   004b83ae f   LIBC:_ctype.obj
 0001:000b73dc       _iscntrl                   004b83dc f   LIBC:_ctype.obj
 0001:000b7405       ___isascii                 004b8405 f   LIBC:_ctype.obj
 0001:000b7412       ___toascii                 004b8412 f   LIBC:_ctype.obj
 0001:000b741a       ___iscsymf                 004b841a f   LIBC:_ctype.obj
 0001:000b7457       ___iscsym                  004b8457 f   LIBC:_ctype.obj
 0001:000b7494       _mbtowc                    004b8494 f   LIBC:mbtowc.obj
 0001:000b7560       _strcmp                    004b8560 f   LIBC:strcmp.obj
 0001:000b75e8       __87except                 004b85e8 f   LIBC:87except.obj
 0001:000b76e0       ___strgtold12              004b86e0 f   LIBC:strgtold.obj
 0001:000b7b67       ___STRINGTOLD              004b8b67 f   LIBC:strgtold.obj
 0001:000b7bb3       __lseeki64                 004b8bb3 f   LIBC:lseeki64.obj
 0001:000b7c52       __sopen                    004b8c52 f   LIBC:open.obj
 0001:000b7f22       _open                      004b8f22 f   LIBC:open.obj
 0001:000b7f22       __open                     004b8f22 f   LIBC:open.obj
 0001:000b7f39       _realloc                   004b8f39 f   LIBC:realloc.obj
 0001:000b809b       __msize                    004b909b f   LIBC:msize.obj
 0001:000b80d3       ___security_init_cookie    004b90d3 f   LIBC:seccinit.obj
 0001:000b8139       ___security_error_handler  004b9139 f   LIBC:secfail.obj
 0001:000b8281       __set_security_error_handler 004b9281 f   LIBC:secfail.obj
 0001:000b8291       ___buffer_overrun          004b9291 f   LIBC:secfail.obj
 0001:000b829d       ___set_buffer_overrun_handler 004b929d f   LIBC:secfail.obj
 0001:000b82ad       ___crtMessageBoxA          004b92ad f   LIBC:crtmbox.obj
 0001:000b83d9       __ismbbkalnum              004b93d9 f   LIBC:ismbbyte.obj
 0001:000b83ea       __ismbbkprint              004b93ea f   LIBC:ismbbyte.obj
 0001:000b83fb       __ismbbkpunct              004b93fb f   LIBC:ismbbyte.obj
 0001:000b840c       __ismbbalnum               004b940c f   LIBC:ismbbyte.obj
 0001:000b8420       __ismbbalpha               004b9420 f   LIBC:ismbbyte.obj
 0001:000b8434       __ismbbgraph               004b9434 f   LIBC:ismbbyte.obj
 0001:000b8448       __ismbbprint               004b9448 f   LIBC:ismbbyte.obj
 0001:000b845c       __ismbbpunct               004b945c f   LIBC:ismbbyte.obj
 0001:000b846d       __ismbblead                004b946d f   LIBC:ismbbyte.obj
 0001:000b847e       __ismbbtrail               004b947e f   LIBC:ismbbyte.obj
 0001:000b848f       __ismbbkana                004b948f f   LIBC:ismbbyte.obj
 0001:000b84b6       __ValidateEH3RN            004b94b6 f   LIBC:eh3valid.obj
 0001:000b86e0       _fdiv_main_routine         004b96e0 f   LIBC:adj_fdiv.obj
 0001:000b87f7       __adj_fdiv_r               004b97f7 f   LIBC:adj_fdiv.obj
 0001:000b8c96       __fdivp_sti_st             004b9c96 f   LIBC:adj_fdiv.obj
 0001:000b8ca9       __fdivrp_sti_st            004b9ca9 f   LIBC:adj_fdiv.obj
 0001:000b8cbc       __adj_fdiv_m32             004b9cbc f   LIBC:adj_fdiv.obj
 0001:000b8d08       __adj_fdiv_m64             004b9d08 f   LIBC:adj_fdiv.obj
 0001:000b8d54       __adj_fdiv_m16i            004b9d54 f   LIBC:adj_fdiv.obj
 0001:000b8d88       __adj_fdiv_m32i            004b9d88 f   LIBC:adj_fdiv.obj
 0001:000b8dbc       __adj_fdivr_m32            004b9dbc f   LIBC:adj_fdiv.obj
 0001:000b8e08       __adj_fdivr_m64            004b9e08 f   LIBC:adj_fdiv.obj
 0001:000b8e54       __adj_fdivr_m16i           004b9e54 f   LIBC:adj_fdiv.obj
 0001:000b8e88       __adj_fdivr_m32i           004b9e88 f   LIBC:adj_fdiv.obj
 0001:000b8ebc       __safe_fdiv                004b9ebc f   LIBC:adj_fdiv.obj
 0001:000b8ed1       __safe_fdivr               004b9ed1 f   LIBC:adj_fdiv.obj
 0001:000b8ee6       __fprem_common             004b9ee6 f   LIBC:adj_fdiv.obj
 0001:000b90ec       __adj_fprem                004ba0ec f   LIBC:adj_fdiv.obj
 0001:000b919e       __fprem1_common            004ba19e f   LIBC:adj_fdiv.obj
 0001:000b93a4       __adj_fprem1               004ba3a4 f   LIBC:adj_fdiv.obj
 0001:000b9459       __safe_fprem               004ba459 f   LIBC:adj_fdiv.obj
 0001:000b945f       __safe_fprem1              004ba45f f   LIBC:adj_fdiv.obj
 0001:000b9465       __adj_fpatan               004ba465 f   LIBC:adj_fdiv.obj
 0001:000b9468       __adj_fptan                004ba468 f   LIBC:adj_fdiv.obj
 0001:000b946b       __copysign                 004ba46b f   LIBC:ieeemisc.obj
 0001:000b948c       __chgsign                  004ba48c f   LIBC:ieeemisc.obj
 0001:000b94b2       __scalb                    004ba4b2 f   LIBC:ieeemisc.obj
 0001:000b94c8       __logb                     004ba4c8 f   LIBC:ieeemisc.obj
 0001:000b95b3       __nextafter                004ba5b3 f   LIBC:ieeemisc.obj
 0001:000b9856       __finite                   004ba856 f   LIBC:ieeemisc.obj
 0001:000b986b       __isnan                    004ba86b f   LIBC:ieeemisc.obj
 0001:000b9899       __fpclass                  004ba899 f   LIBC:ieeemisc.obj
 0001:000b9935       __wcsnicoll                004ba935 f   LIBC:wcsnicol.obj
 0001:000b99de       __wcsdup                   004ba9de f   LIBC:wcsdup.obj
 0001:000b9a0c       _wcscat                    004baa0c f   LIBC:wcscat.obj
 0001:000b9a36       _wcscpy                    004baa36 f   LIBC:wcscat.obj
 0001:000b9a52       _wcslen                    004baa52 f   LIBC:wcslen.obj
 0001:000b9a68       ___mbtow_environ           004baa68 f   LIBC:mbtowenv.obj
 0001:000b9aea       _wcschr                    004baaea f   LIBC:wcschr.obj
 0001:000b9b0c       __strdup                   004bab0c f   LIBC:strdup.obj
 0001:000b9b37       __mbschr                   004bab37 f   LIBC:mbschr.obj
 0001:000b9b9e       ___addl                    004bab9e f   LIBC:mantold.obj
 0001:000b9bbf       ___add_12                  004babbf f   LIBC:mantold.obj
 0001:000b9c1d       ___shl_12                  004bac1d f   LIBC:mantold.obj
 0001:000b9c4b       ___shr_12                  004bac4b f   LIBC:mantold.obj
 0001:000b9c78       ___mtold12                 004bac78 f   LIBC:mantold.obj
 0001:000b9d56       _$I10_OUTPUT               004bad56 f   LIBC:x10fout.obj
 0001:000b9fe4       ___ld12mul                 004bafe4 f   LIBC:tenpow.obj
 0001:000ba216       ___multtenpow12            004bb216 f   LIBC:tenpow.obj
 0001:000ba29c       __chsize                   004bb29c f   LIBC:chsize.obj
 0001:000ba3f8       _ldexp                     004bb3f8 f   LIBC:ldexp.obj
 0001:000ba601       ___crtCompareStringW       004bb601 f   LIBC:w_cmp.obj
 0001:000ba853       __setmode                  004bb853 f   LIBC:setmode.obj
 0001:000ba8d6       _GetSystemDirectoryA@8     004bb8d6 f   kernel32:KERNEL32.dll
 0001:000ba8dc       _CreateThread@24           004bb8dc f   kernel32:KERNEL32.dll
 0001:000ba8e2       _CreateEventA@16           004bb8e2 f   kernel32:KERNEL32.dll
 0001:000ba8e8       _WaitForSingleObject@8     004bb8e8 f   kernel32:KERNEL32.dll
 0001:000ba8ee       _SetEvent@4                004bb8ee f   kernel32:KERNEL32.dll
 0001:000ba8f4       _ResetEvent@4              004bb8f4 f   kernel32:KERNEL32.dll
 0001:000ba8fa       _GetSystemTimeAsFileTime@4 004bb8fa f   kernel32:KERNEL32.dll
 0001:000ba900       _HeapAlloc@12              004bb900 f   kernel32:KERNEL32.dll
 0001:000ba906       _HeapFree@12               004bb906 f   kernel32:KERNEL32.dll
 0001:000ba90c       _GetLastError@0            004bb90c f   kernel32:KERNEL32.dll
 0001:000ba912       _DeleteFileA@4             004bb912 f   kernel32:KERNEL32.dll
 0001:000ba918       _MoveFileA@8               004bb918 f   kernel32:KERNEL32.dll
 0001:000ba91e       _FlushFileBuffers@4        004bb91e f   kernel32:KERNEL32.dll
 0001:000ba924       _ExitProcess@4             004bb924 f   kernel32:KERNEL32.dll
 0001:000ba92a       _GetModuleHandleA@4        004bb92a f   kernel32:KERNEL32.dll
 0001:000ba930       _TerminateProcess@8        004bb930 f   kernel32:KERNEL32.dll
 0001:000ba936       _GetCurrentProcess@0       004bb936 f   kernel32:KERNEL32.dll
 0001:000ba93c       _CreateDirectoryA@8        004bb93c f   kernel32:KERNEL32.dll
 0001:000ba942       _GetCurrentDirectoryA@8    004bb942 f   kernel32:KERNEL32.dll
 0001:000ba948       _GetFullPathNameA@16       004bb948 f   kernel32:KERNEL32.dll
 0001:000ba94e       _FindClose@4               004bb94e f   kernel32:KERNEL32.dll
 0001:000ba954       _FileTimeToSystemTime@8    004bb954 f   kernel32:KERNEL32.dll
 0001:000ba95a       _FileTimeToLocalFileTime@8 004bb95a f   kernel32:KERNEL32.dll
 0001:000ba960       _FindFirstFileA@8          004bb960 f   kernel32:KERNEL32.dll
 0001:000ba966       _FindNextFileA@8           004bb966 f   kernel32:KERNEL32.dll
 0001:000ba96c       _GetStartupInfoA@4         004bb96c f   kernel32:KERNEL32.dll
 0001:000ba972       _GetCommandLineA@0         004bb972 f   kernel32:KERNEL32.dll
 0001:000ba978       _MultiByteToWideChar@24    004bb978 f   kernel32:KERNEL32.dll
 0001:000ba97e       _LCMapStringA@24           004bb97e f   kernel32:KERNEL32.dll
 0001:000ba984       _WideCharToMultiByte@32    004bb984 f   kernel32:KERNEL32.dll
 0001:000ba98a       _LCMapStringW@24           004bb98a f   kernel32:KERNEL32.dll
 0001:000ba990       _GetTimeZoneInformation@4  004bb990 f   kernel32:KERNEL32.dll
 0001:000ba996       _RtlUnwind@16              004bb996 f   kernel32:KERNEL32.dll
 0001:000ba99c       _HeapDestroy@4             004bb99c f   kernel32:KERNEL32.dll
 0001:000ba9a2       _HeapCreate@12             004bb9a2 f   kernel32:KERNEL32.dll
 0001:000ba9a8       _VirtualFree@12            004bb9a8 f   kernel32:KERNEL32.dll
 0001:000ba9ae       _VirtualAlloc@16           004bb9ae f   kernel32:KERNEL32.dll
 0001:000ba9b4       _HeapReAlloc@16            004bb9b4 f   kernel32:KERNEL32.dll
 0001:000ba9ba       _IsBadWritePtr@8           004bb9ba f   kernel32:KERNEL32.dll
 0001:000ba9c0       _SetFilePointer@16         004bb9c0 f   kernel32:KERNEL32.dll
 0001:000ba9c6       _SetHandleCount@4          004bb9c6 f   kernel32:KERNEL32.dll
 0001:000ba9cc       _GetStdHandle@4            004bb9cc f   kernel32:KERNEL32.dll
 0001:000ba9d2       _GetFileType@4             004bb9d2 f   kernel32:KERNEL32.dll
 0001:000ba9d8       _WriteFile@20              004bb9d8 f   kernel32:KERNEL32.dll
 0001:000ba9de       _CloseHandle@4             004bb9de f   kernel32:KERNEL32.dll
 0001:000ba9e4       _ReadFile@20               004bb9e4 f   kernel32:KERNEL32.dll
 0001:000ba9ea       _SetStdHandle@8            004bb9ea f   kernel32:KERNEL32.dll
 0001:000ba9f0       _GetModuleFileNameA@12     004bb9f0 f   kernel32:KERNEL32.dll
 0001:000ba9f6       _UnhandledExceptionFilter@4 004bb9f6 f   kernel32:KERNEL32.dll
 0001:000ba9fc       _FreeEnvironmentStringsA@4 004bb9fc f   kernel32:KERNEL32.dll
 0001:000baa02       _GetEnvironmentStrings@0   004bba02 f   kernel32:KERNEL32.dll
 0001:000baa08       _FreeEnvironmentStringsW@4 004bba08 f   kernel32:KERNEL32.dll
 0001:000baa0e       _GetEnvironmentStringsW@0  004bba0e f   kernel32:KERNEL32.dll
 0001:000baa14       _SetEnvironmentVariableA@8 004bba14 f   kernel32:KERNEL32.dll
 0001:000baa1a       _SetEnvironmentVariableW@8 004bba1a f   kernel32:KERNEL32.dll
 0001:000baa20       _GetStringTypeA@20         004bba20 f   kernel32:KERNEL32.dll
 0001:000baa26       _GetStringTypeW@16         004bba26 f   kernel32:KERNEL32.dll
 0001:000baa2c       _GetACP@0                  004bba2c f   kernel32:KERNEL32.dll
 0001:000baa32       _GetOEMCP@0                004bba32 f   kernel32:KERNEL32.dll
 0001:000baa38       _GetCPInfo@8               004bba38 f   kernel32:KERNEL32.dll
 0001:000baa3e       _RaiseException@16         004bba3e f   kernel32:KERNEL32.dll
 0001:000baa44       _GetLocaleInfoA@16         004bba44 f   kernel32:KERNEL32.dll
 0001:000baa4a       _VirtualProtect@16         004bba4a f   kernel32:KERNEL32.dll
 0001:000baa50       _GetSystemInfo@4           004bba50 f   kernel32:KERNEL32.dll
 0001:000baa56       _VirtualQuery@12           004bba56 f   kernel32:KERNEL32.dll
 0001:000baa5c       _CompareStringA@24         004bba5c f   kernel32:KERNEL32.dll
 0001:000baa62       _CompareStringW@24         004bba62 f   kernel32:KERNEL32.dll
 0001:000baa68       _CreateFileA@28            004bba68 f   kernel32:KERNEL32.dll
 0001:000baa6e       _HeapSize@12               004bba6e f   kernel32:KERNEL32.dll
 0001:000baa74       _QueryPerformanceCounter@4 004bba74 f   kernel32:KERNEL32.dll
 0001:000baa7a       _GetTickCount@0            004bba7a f   kernel32:KERNEL32.dll
 0001:000baa80       _GetCurrentThreadId@0      004bba80 f   kernel32:KERNEL32.dll
 0001:000baa86       _GetCurrentProcessId@0     004bba86 f   kernel32:KERNEL32.dll
 0001:000baa8c       _InterlockedExchange@8     004bba8c f   kernel32:KERNEL32.dll
 0001:000baa92       _SetEndOfFile@4            004bba92 f   kernel32:KERNEL32.dll
 0001:000baa98       _EnumDisplaySettingsA@12   004bba98 f   user32:USER32.dll
 0001:000baa9e       _ChangeDisplaySettingsA@8  004bba9e f   user32:USER32.dll
 0001:000baaa4       _MessageBoxA@16            004bbaa4 f   user32:USER32.dll
 0001:000baaaa       _DescribePixelFormat@16    004bbaaa f   gdi32:GDI32.dll
 0001:000baab0       _SetPixelFormat@12         004bbab0 f   gdi32:GDI32.dll
 0001:000baab6       _SwapBuffers@4             004bbab6 f   gdi32:GDI32.dll
 0001:000baabc       _GetDeviceGammaRamp@8      004bbabc f   gdi32:GDI32.dll
 0001:000baac2       _SetDeviceGammaRamp@8      004bbac2 f   gdi32:GDI32.dll
 0002:00000000       __imp__GetUserNameA@8      004bc000     advapi32:ADVAPI32.dll
 0002:00000004       \177ADVAPI32_NULL_THUNK_DATA 004bc004     advapi32:ADVAPI32.dll
 0002:00000008       __imp__SetPixelFormat@12   004bc008     gdi32:GDI32.dll
 0002:0000000c       __imp__DescribePixelFormat@16 004bc00c     gdi32:GDI32.dll
 0002:00000010       __imp__SwapBuffers@4       004bc010     gdi32:GDI32.dll
 0002:00000014       __imp__GetDeviceGammaRamp@8 004bc014     gdi32:GDI32.dll
 0002:00000018       __imp__CreateFontA@56      004bc018     gdi32:GDI32.dll
 0002:0000001c       __imp__GetDeviceCaps@8     004bc01c     gdi32:GDI32.dll
 0002:00000020       __imp__SetDeviceGammaRamp@8 004bc020     gdi32:GDI32.dll
 0002:00000024       __imp__CreateSolidBrush@4  004bc024     gdi32:GDI32.dll
 0002:00000028       __imp__SetBkColor@8        004bc028     gdi32:GDI32.dll
 0002:0000002c       __imp__SetTextColor@8      004bc02c     gdi32:GDI32.dll
 0002:00000030       \177GDI32_NULL_THUNK_DATA  004bc030     gdi32:GDI32.dll
 0002:00000034       __imp__GetOEMCP@0          004bc034     kernel32:KERNEL32.dll
 0002:00000038       __imp__SetStdHandle@8      004bc038     kernel32:KERNEL32.dll
 0002:0000003c       __imp__ReadFile@20         004bc03c     kernel32:KERNEL32.dll
 0002:00000040       __imp__CloseHandle@4       004bc040     kernel32:KERNEL32.dll
 0002:00000044       __imp__SetEndOfFile@4      004bc044     kernel32:KERNEL32.dll
 0002:00000048       __imp__InterlockedExchange@8 004bc048     kernel32:KERNEL32.dll
 0002:0000004c       __imp__GetCurrentProcessId@0 004bc04c     kernel32:KERNEL32.dll
 0002:00000050       __imp__GetCurrentThreadId@0 004bc050     kernel32:KERNEL32.dll
 0002:00000054       __imp__GetTickCount@0      004bc054     kernel32:KERNEL32.dll
 0002:00000058       __imp__QueryPerformanceCounter@4 004bc058     kernel32:KERNEL32.dll
 0002:0000005c       __imp__HeapSize@12         004bc05c     kernel32:KERNEL32.dll
 0002:00000060       __imp__CreateFileA@28      004bc060     kernel32:KERNEL32.dll
 0002:00000064       __imp__CompareStringW@24   004bc064     kernel32:KERNEL32.dll
 0002:00000068       __imp__CompareStringA@24   004bc068     kernel32:KERNEL32.dll
 0002:0000006c       __imp__VirtualQuery@12     004bc06c     kernel32:KERNEL32.dll
 0002:00000070       __imp__GetSystemInfo@4     004bc070     kernel32:KERNEL32.dll
 0002:00000074       __imp__VirtualProtect@16   004bc074     kernel32:KERNEL32.dll
 0002:00000078       __imp__GetLocaleInfoA@16   004bc078     kernel32:KERNEL32.dll
 0002:0000007c       __imp__GetProcAddress@8    004bc07c     kernel32:KERNEL32.dll
 0002:00000080       __imp__LoadLibraryA@4      004bc080     kernel32:KERNEL32.dll
 0002:00000084       __imp__GlobalMemoryStatus@4 004bc084     kernel32:KERNEL32.dll
 0002:00000088       __imp__GetDriveTypeA@4     004bc088     kernel32:KERNEL32.dll
 0002:0000008c       __imp__GlobalUnlock@4      004bc08c     kernel32:KERNEL32.dll
 0002:00000090       __imp__GlobalSize@4        004bc090     kernel32:KERNEL32.dll
 0002:00000094       __imp__GlobalLock@4        004bc094     kernel32:KERNEL32.dll
 0002:00000098       __imp__FreeLibrary@4       004bc098     kernel32:KERNEL32.dll
 0002:0000009c       __imp__GetVersionExA@4     004bc09c     kernel32:KERNEL32.dll
 0002:000000a0       __imp__Sleep@4             004bc0a0     kernel32:KERNEL32.dll
 0002:000000a4       __imp__SetErrorMode@4      004bc0a4     kernel32:KERNEL32.dll
 0002:000000a8       __imp__MulDiv@12           004bc0a8     kernel32:KERNEL32.dll
 0002:000000ac       __imp__WriteFile@20        004bc0ac     kernel32:KERNEL32.dll
 0002:000000b0       __imp__GetFileType@4       004bc0b0     kernel32:KERNEL32.dll
 0002:000000b4       __imp__GetStdHandle@4      004bc0b4     kernel32:KERNEL32.dll
 0002:000000b8       __imp__SetHandleCount@4    004bc0b8     kernel32:KERNEL32.dll
 0002:000000bc       __imp__SetFilePointer@16   004bc0bc     kernel32:KERNEL32.dll
 0002:000000c0       __imp__IsBadWritePtr@8     004bc0c0     kernel32:KERNEL32.dll
 0002:000000c4       __imp__HeapReAlloc@16      004bc0c4     kernel32:KERNEL32.dll
 0002:000000c8       __imp__VirtualAlloc@16     004bc0c8     kernel32:KERNEL32.dll
 0002:000000cc       __imp__VirtualFree@12      004bc0cc     kernel32:KERNEL32.dll
 0002:000000d0       __imp__HeapCreate@12       004bc0d0     kernel32:KERNEL32.dll
 0002:000000d4       __imp__HeapDestroy@4       004bc0d4     kernel32:KERNEL32.dll
 0002:000000d8       __imp__RtlUnwind@16        004bc0d8     kernel32:KERNEL32.dll
 0002:000000dc       __imp__GetTimeZoneInformation@4 004bc0dc     kernel32:KERNEL32.dll
 0002:000000e0       __imp__LCMapStringW@24     004bc0e0     kernel32:KERNEL32.dll
 0002:000000e4       __imp__WideCharToMultiByte@32 004bc0e4     kernel32:KERNEL32.dll
 0002:000000e8       __imp__LCMapStringA@24     004bc0e8     kernel32:KERNEL32.dll
 0002:000000ec       __imp__MultiByteToWideChar@24 004bc0ec     kernel32:KERNEL32.dll
 0002:000000f0       __imp__GetCommandLineA@0   004bc0f0     kernel32:KERNEL32.dll
 0002:000000f4       __imp__GetStartupInfoA@4   004bc0f4     kernel32:KERNEL32.dll
 0002:000000f8       __imp__FindNextFileA@8     004bc0f8     kernel32:KERNEL32.dll
 0002:000000fc       __imp__FindFirstFileA@8    004bc0fc     kernel32:KERNEL32.dll
 0002:00000100       __imp__FileTimeToLocalFileTime@8 004bc100     kernel32:KERNEL32.dll
 0002:00000104       __imp__FileTimeToSystemTime@8 004bc104     kernel32:KERNEL32.dll
 0002:00000108       __imp__FindClose@4         004bc108     kernel32:KERNEL32.dll
 0002:0000010c       __imp__GetFullPathNameA@16 004bc10c     kernel32:KERNEL32.dll
 0002:00000110       __imp__GetCurrentDirectoryA@8 004bc110     kernel32:KERNEL32.dll
 0002:00000114       __imp__CreateDirectoryA@8  004bc114     kernel32:KERNEL32.dll
 0002:00000118       __imp__GetCurrentProcess@0 004bc118     kernel32:KERNEL32.dll
 0002:0000011c       __imp__TerminateProcess@8  004bc11c     kernel32:KERNEL32.dll
 0002:00000120       __imp__GetModuleHandleA@4  004bc120     kernel32:KERNEL32.dll
 0002:00000124       __imp__ExitProcess@4       004bc124     kernel32:KERNEL32.dll
 0002:00000128       __imp__FlushFileBuffers@4  004bc128     kernel32:KERNEL32.dll
 0002:0000012c       __imp__MoveFileA@8         004bc12c     kernel32:KERNEL32.dll
 0002:00000130       __imp__DeleteFileA@4       004bc130     kernel32:KERNEL32.dll
 0002:00000134       __imp__GetLastError@0      004bc134     kernel32:KERNEL32.dll
 0002:00000138       __imp__HeapFree@12         004bc138     kernel32:KERNEL32.dll
 0002:0000013c       __imp__HeapAlloc@12        004bc13c     kernel32:KERNEL32.dll
 0002:00000140       __imp__GetModuleFileNameA@12 004bc140     kernel32:KERNEL32.dll
 0002:00000144       __imp__GetSystemTimeAsFileTime@4 004bc144     kernel32:KERNEL32.dll
 0002:00000148       __imp__ResetEvent@4        004bc148     kernel32:KERNEL32.dll
 0002:0000014c       __imp__SetEvent@4          004bc14c     kernel32:KERNEL32.dll
 0002:00000150       __imp__WaitForSingleObject@8 004bc150     kernel32:KERNEL32.dll
 0002:00000154       __imp__CreateEventA@16     004bc154     kernel32:KERNEL32.dll
 0002:00000158       __imp__CreateThread@24     004bc158     kernel32:KERNEL32.dll
 0002:0000015c       __imp__GetSystemDirectoryA@8 004bc15c     kernel32:KERNEL32.dll
 0002:00000160       __imp__RaiseException@16   004bc160     kernel32:KERNEL32.dll
 0002:00000164       __imp__GetACP@0            004bc164     kernel32:KERNEL32.dll
 0002:00000168       __imp__GetStringTypeW@16   004bc168     kernel32:KERNEL32.dll
 0002:0000016c       __imp__GetStringTypeA@20   004bc16c     kernel32:KERNEL32.dll
 0002:00000170       __imp__SetEnvironmentVariableW@8 004bc170     kernel32:KERNEL32.dll
 0002:00000174       __imp__SetEnvironmentVariableA@8 004bc174     kernel32:KERNEL32.dll
 0002:00000178       __imp__GetEnvironmentStringsW@0 004bc178     kernel32:KERNEL32.dll
 0002:0000017c       __imp__FreeEnvironmentStringsW@4 004bc17c     kernel32:KERNEL32.dll
 0002:00000180       __imp__GetEnvironmentStrings@0 004bc180     kernel32:KERNEL32.dll
 0002:00000184       __imp__GetCPInfo@8         004bc184     kernel32:KERNEL32.dll
 0002:00000188       __imp__FreeEnvironmentStringsA@4 004bc188     kernel32:KERNEL32.dll
 0002:0000018c       __imp__UnhandledExceptionFilter@4 004bc18c     kernel32:KERNEL32.dll
 0002:00000190       \177KERNEL32_NULL_THUNK_DATA 004bc190     kernel32:KERNEL32.dll
 0002:00000194       __imp__GetWindowLongA@8    004bc194     user32:USER32.dll
 0002:00000198       __imp__RegisterWindowMessageA@4 004bc198     user32:USER32.dll
 0002:0000019c       __imp__UnregisterHotKey@8  004bc19c     user32:USER32.dll
 0002:000001a0       __imp__RegisterHotKey@16   004bc1a0     user32:USER32.dll
 0002:000001a4       __imp__SystemParametersInfoA@16 004bc1a4     user32:USER32.dll
 0002:000001a8       __imp__LoadIconA@8         004bc1a8     user32:USER32.dll
 0002:000001ac       __imp__RegisterClassA@4    004bc1ac     user32:USER32.dll
 0002:000001b0       __imp__AdjustWindowRect@12 004bc1b0     user32:USER32.dll
 0002:000001b4       __imp__GetDesktopWindow@0  004bc1b4     user32:USER32.dll
 0002:000001b8       __imp__GetDC@4             004bc1b8     user32:USER32.dll
 0002:000001bc       __imp__ReleaseDC@8         004bc1bc     user32:USER32.dll
 0002:000001c0       __imp__SetWindowLongA@12   004bc1c0     user32:USER32.dll
 0002:000001c4       __imp__SetForegroundWindow@4 004bc1c4     user32:USER32.dll
 0002:000001c8       __imp__PostQuitMessage@4   004bc1c8     user32:USER32.dll
 0002:000001cc       __imp__DefWindowProcA@16   004bc1cc     user32:USER32.dll
 0002:000001d0       __imp__SetTimer@16         004bc1d0     user32:USER32.dll
 0002:000001d4       __imp__InvalidateRect@12   004bc1d4     user32:USER32.dll
 0002:000001d8       __imp__UpdateWindow@4      004bc1d8     user32:USER32.dll
 0002:000001dc       __imp__CreateWindowExA@48  004bc1dc     user32:USER32.dll
 0002:000001e0       __imp__SendMessageA@16     004bc1e0     user32:USER32.dll
 0002:000001e4       __imp__ShowWindow@8        004bc1e4     user32:USER32.dll
 0002:000001e8       __imp__CloseWindow@4       004bc1e8     user32:USER32.dll
 0002:000001ec       __imp__DestroyWindow@4     004bc1ec     user32:USER32.dll
 0002:000001f0       __imp__GetWindowTextA@12   004bc1f0     user32:USER32.dll
 0002:000001f4       __imp__SetWindowTextA@8    004bc1f4     user32:USER32.dll
 0002:000001f8       __imp__CallWindowProcA@20  004bc1f8     user32:USER32.dll
 0002:000001fc       __imp__SetFocus@4          004bc1fc     user32:USER32.dll
 0002:00000200       __imp__PeekMessageA@20     004bc200     user32:USER32.dll
 0002:00000204       __imp__MessageBoxExA@20    004bc204     user32:USER32.dll
 0002:00000208       __imp__OpenClipboard@4     004bc208     user32:USER32.dll
 0002:0000020c       __imp__GetClipboardData@4  004bc20c     user32:USER32.dll
 0002:00000210       __imp__CloseClipboard@0    004bc210     user32:USER32.dll
 0002:00000214       __imp__GetMessageA@16      004bc214     user32:USER32.dll
 0002:00000218       __imp__TranslateMessage@4  004bc218     user32:USER32.dll
 0002:0000021c       __imp__DispatchMessageA@4  004bc21c     user32:USER32.dll
 0002:00000220       __imp__GetCursorPos@4      004bc220     user32:USER32.dll
 0002:00000224       __imp__ReleaseCapture@0    004bc224     user32:USER32.dll
 0002:00000228       __imp__GetSystemMetrics@4  004bc228     user32:USER32.dll
 0002:0000022c       __imp__GetWindowRect@8     004bc22c     user32:USER32.dll
 0002:00000230       __imp__SetCursorPos@8      004bc230     user32:USER32.dll
 0002:00000234       __imp__SetCapture@4        004bc234     user32:USER32.dll
 0002:00000238       __imp__ClipCursor@4        004bc238     user32:USER32.dll
 0002:0000023c       __imp__ShowCursor@4        004bc23c     user32:USER32.dll
 0002:00000240       __imp__EnumDisplaySettingsA@12 004bc240     user32:USER32.dll
 0002:00000244       __imp__ChangeDisplaySettingsA@8 004bc244     user32:USER32.dll
 0002:00000248       __imp__MessageBoxA@16      004bc248     user32:USER32.dll
 0002:0000024c       __imp__LoadCursorA@8       004bc24c     user32:USER32.dll
 0002:00000250       \177USER32_NULL_THUNK_DATA 004bc250     user32:USER32.dll
 0002:00000254       __imp__midiInStart@4       004bc254     winmm:WINMM.dll
 0002:00000258       __imp__joyGetNumDevs@0     004bc258     winmm:WINMM.dll
 0002:0000025c       __imp__joyGetPosEx@8       004bc25c     winmm:WINMM.dll
 0002:00000260       __imp__midiInGetDevCapsA@12 004bc260     winmm:WINMM.dll
 0002:00000264       __imp__midiInGetNumDevs@0  004bc264     winmm:WINMM.dll
 0002:00000268       __imp__midiInClose@4       004bc268     winmm:WINMM.dll
 0002:0000026c       __imp__timeEndPeriod@4     004bc26c     winmm:WINMM.dll
 0002:00000270       __imp__timeGetTime@0       004bc270     winmm:WINMM.dll
 0002:00000274       __imp__timeBeginPeriod@4   004bc274     winmm:WINMM.dll
 0002:00000278       __imp__joyGetDevCapsA@12   004bc278     winmm:WINMM.dll
 0002:0000027c       __imp__midiInOpen@20       004bc27c     winmm:WINMM.dll
 0002:00000280       \177WINMM_NULL_THUNK_DATA  004bc280     winmm:WINMM.dll
 0002:00000284       __imp__WSAGetLastError@0   004bc284     wsock32:WSOCK32.dll
 0002:00000288       __imp__WSACleanup@0        004bc288     wsock32:WSOCK32.dll
 0002:0000028c       __imp__WSAStartup@8        004bc28c     wsock32:WSOCK32.dll
 0002:00000290       __imp__gethostname@8       004bc290     wsock32:WSOCK32.dll
 0002:00000294       __imp__ntohl@4             004bc294     wsock32:WSOCK32.dll
 0002:00000298       __imp__connect@12          004bc298     wsock32:WSOCK32.dll
 0002:0000029c       __imp__send@16             004bc29c     wsock32:WSOCK32.dll
 0002:000002a0       __imp__recv@16             004bc2a0     wsock32:WSOCK32.dll
 0002:000002a4       __imp__socket@12           004bc2a4     wsock32:WSOCK32.dll
 0002:000002a8       __imp__ioctlsocket@12      004bc2a8     wsock32:WSOCK32.dll
 0002:000002ac       __imp__setsockopt@20       004bc2ac     wsock32:WSOCK32.dll
 0002:000002b0       __imp__htons@4             004bc2b0     wsock32:WSOCK32.dll
 0002:000002b4       __imp__bind@12             004bc2b4     wsock32:WSOCK32.dll
 0002:000002b8       __imp__closesocket@4       004bc2b8     wsock32:WSOCK32.dll
 0002:000002bc       __imp__sendto@24           004bc2bc     wsock32:WSOCK32.dll
 0002:000002c0       __imp__recvfrom@24         004bc2c0     wsock32:WSOCK32.dll
 0002:000002c4       __imp__inet_addr@4         004bc2c4     wsock32:WSOCK32.dll
 0002:000002c8       __imp__gethostbyname@4     004bc2c8     wsock32:WSOCK32.dll
 0002:000002cc       \177WSOCK32_NULL_THUNK_DATA 004bc2cc     wsock32:WSOCK32.dll
 0002:000002d0       __imp__CoInitialize@4      004bc2d0     ole32:ole32.dll
 0002:000002d4       __imp__CoUninitialize@0    004bc2d4     ole32:ole32.dll
 0002:000002d8       __imp__CoCreateInstance@20 004bc2d8     ole32:ole32.dll
 0002:000002dc       \177ole32_NULL_THUNK_DATA  004bc2dc     ole32:ole32.dll
 0002:000002fc       ??_C@_0BI@GFBIMDFO@CL_GetUserCmd?3?5?$CFi?5?$DO?$DN?5?$CFi?$AA@ 004bc2fc     cl_cgame.obj
 0002:00000314       ??_C@_0CB@KNGFLOML@CL_GetParseEntityState?3?5?$CFi?5?$DO?$DN?5?$CFi@ 004bc314     cl_cgame.obj
 0002:00000338       ??_C@_0CN@NFLCIAJJ@CL_GetSnapshot?3?5truncated?5?$CFi?5ent@ 004bc338     cl_cgame.obj
 0002:00000368       ??_C@_0DI@DMJPFKEN@CL_GetSnapshot?3?5snapshotNumber?5?$DO@ 004bc368     cl_cgame.obj
 0002:000003a0       ??_C@_02DKCKIIND@?$CFs?$AA@ 004bc3a0     cl_cgame.obj
 0002:000003a4       ??_C@_0BN@EHLDLIPD@MAX_GAMESTATE_CHARS?5exceeded?$AA@ 004bc3a4     cl_cgame.obj
 0002:000003c4       ??_C@_0CB@GKLEHILN@configstring?5?$DO?5MAX_CONFIGSTRINGS@ 004bc3c4     cl_cgame.obj
 0002:000003e8       ??_C@_0DC@GKPOBHJK@wait?5?$DL?5wait?5?$DL?5wait?5?$DL?5wait?5?$DL?5scre@ 004bc3e8     cl_cgame.obj
 0002:0000041c       ??_C@_0BA@GNMFKLDC@clientLevelShot?$AA@ 004bc41c     cl_cgame.obj
 0002:0000042c       ??_C@_0M@NBIMEKNE@map_restart?$AA@ 004bc42c     cl_cgame.obj
 0002:00000438       ??_C@_02EODNHJKB@cs?$AA@   004bc438     cl_cgame.obj
 0002:0000043c       ??_C@_09PHKADKGH@cs?5?$CFs?5?$CC?$CFs?$AA@ 004bc43c     cl_cgame.obj
 0002:00000448       ??_C@_01BJJEKLCA@?$CC?$AA@ 004bc448     cl_cgame.obj
 0002:0000044c       ??_C@_0BN@DLAPMAAP@bcs?5exceeded?5BIG_INFO_STRING?$AA@ 004bc44c     cl_cgame.obj
 0002:0000046c       ??_C@_04EIHLPGFK@bcs2?$AA@ 004bc46c     cl_cgame.obj
 0002:00000474       ??_C@_04GDFGKFJJ@bcs1?$AA@ 004bc474     cl_cgame.obj
 0002:0000047c       ??_C@_04HKENJENI@bcs0?$AA@ 004bc47c     cl_cgame.obj
 0002:00000484       ??_C@_0BF@PHOEELOB@Server?5disconnected?6?$AA@ 004bc484     cl_cgame.obj
 0002:0000049c       ??_C@_0BJ@FDEBGBPO@Server?5Disconnected?5?9?5?$CFs?$AA@ 004bc49c     cl_cgame.obj
 0002:000004b8       ??_C@_0L@KKPFIJOL@disconnect?$AA@ 004bc4b8     cl_cgame.obj
 0002:000004c4       ??_C@_0BI@JLIEJCCP@serverCommand?3?5?$CFi?5?3?5?$CFs?6?$AA@ 004bc4c4     cl_cgame.obj
 0002:000004dc       ??_C@_0DG@FOCFKOFN@CL_GetServerCommand?3?5requested?5a@ 004bc4dc     cl_cgame.obj
 0002:00000514       ??_C@_0DH@KEKKOLLD@CL_GetServerCommand?3?5a?5reliable?5@ 004bc514     cl_cgame.obj
 0002:0000054c       ??_C@_0BK@HMDPIKIJ@Bad?5cgame?5system?5trap?3?5?$CFi?$AA@ 004bc54c     cl_cgame.obj
 0002:00000568       ??_C@_0BN@IDOJBIPH@CL_InitCGame?3?5?$CF5?42f?5seconds?6?$AA@ 004bc568     cl_cgame.obj
 0002:00000588       __real@3f50624dd2f1a9fc    004bc588     cl_cgame.obj
 0002:00000590       ??_C@_0BK@DNNCDOHF@VM_Create?5on?5cgame?5failed?$AA@ 004bc590     cl_cgame.obj
 0002:000005ac       ??_C@_05DAFANPAC@cgame?$AA@ 004bc5ac     cl_cgame.obj
 0002:000005b4       ??_C@_08HKFBPMGE@vm_cgame?$AA@ 004bc5b4     cl_cgame.obj
 0002:000005c0       ??_C@_0M@DKNJHPLK@maps?1?$CFs?4bsp?$AA@ 004bc5c0     cl_cgame.obj
 0002:000005cc       ??_C@_07KMNEBLH@mapname?$AA@ 004bc5cc     cl_cgame.obj
 0002:000005d4       ??_C@_03JLNFKLOC@?$CFi?5?$AA@ 004bc5d4     cl_cgame.obj
 0002:000005d8       __real@00000000            004bc5d8     cl_cgame.obj
 0002:000005dc       ??_C@_07CLMNDOPI@?$DMFAST?$DO?5?$AA@ 004bc5dc     cl_cgame.obj
 0002:000005e4       ??_C@_08DFNEKPFP@?$DMRESET?$DO?5?$AA@ 004bc5e4     cl_cgame.obj
 0002:000005f0       ??_C@_0N@JKAMCJJO@activeAction?$AA@ 004bc5f0     cl_cgame.obj
 0002:000005fd       ??_C@_00CNPNBAHC@?$AA@     004bc5fd     cl_cgame.obj
 0002:00000600       ??_C@_0CL@NEIPEDIE@cl?4snap?4serverTime?5?$DM?5cl?4oldFrame@ 004bc600     cl_cgame.obj
 0002:0000062c       ??_C@_0CA@FIEOEIEM@CL_SetCGameTime?3?5?$CBcl?4snap?4valid?$AA@ 004bc62c     cl_cgame.obj
 0002:0000064c       ??_C@_0BO@EBCDHAOB@CIN_HandleForVideo?3?5none?5free?$AA@ 004bc64c     cl_cin.obj
 0002:0000066c       __real@c1bad1e1            004bc66c     cl_cin.obj
 0002:00000670       __real@c138331e            004bc670     cl_cin.obj
 0002:00000674       __real@423574bc            004bc674     cl_cin.obj
 0002:00000678       __real@42000000            004bc678     cl_cin.obj
 0002:0000067c       __real@4264d0e5            004bc67c     cl_cin.obj
 0002:00000680       ??_C@_0DH@BGGOKGDB@HACK?3?5approxmimating?5cinematic?5f@ 004bc680     cl_cin.obj
 0002:000006b8       ??_C@_03OFAPEBGM@?$CFs?6?$AA@ 004bc6b8     cl_cin.obj
 0002:000006bc       ??_C@_07MCHHMPMB@nextmap?$AA@ 004bc6bc     cl_cin.obj
 0002:000006c4       ??_C@_0BE@JMMOLKGP@finished?5cinematic?6?$AA@ 004bc6c4     cl_cin.obj
 0002:000006d8       ??_C@_0BL@ODCKOIHE@trFMV?3?3stop?$CI?$CJ?0?5closing?5?$CFs?6?$AA@ 004bc6d8     cl_cin.obj
 0002:000006f4       ??_C@_0CA@PBEAEEHD@roq_size?$DO65536?$HM?$HMroq_id?$DN?$DN0x1084?6?$AA@ 004bc6f4     cl_cin.obj
 0002:00000714       __real@3c23d70a            004bc714     cl_cin.obj
 0002:00000718       __real@40400000            004bc718     cl_cin.obj
 0002:0000071c       __real@4f800000            004bc71c     cl_cin.obj
 0002:00000720       ??_C@_0BP@ONKNDCKB@trFMV?3?3play?$CI?$CJ?0?5invalid?5RoQ?5ID?6?$AA@ 004bc720     cl_cin.obj
 0002:00000740       ??_C@_0BL@NOJKJAEE@trFMV?3?3play?$CI?$CJ?0?5playing?5?$CFs?6?$AA@ 004bc740     cl_cin.obj
 0002:0000075c       ??_C@_0BG@CHLIAINM@play?$CI?$CFs?$CJ?0?5ROQSize?$DM?$DN0?6?$AA@ 004bc75c     cl_cin.obj
 0002:00000774       ??_C@_0BJ@PGHMMNHI@SCR_PlayCinematic?$CI?5?$CFs?5?$CJ?6?$AA@ 004bc774     cl_cin.obj
 0002:00000790       ??_C@_08KLIMONEL@video?1?$CFs?$AA@ 004bc790     cl_cin.obj
 0002:0000079c       ??_C@_01KICIPPFI@?2?$AA@   004bc79c     cl_cin.obj
 0002:000007a0       ??_C@_01KMDKNFGN@?1?$AA@   004bc7a0     cl_cin.obj
 0002:000007a4       ??_C@_07IAFCMJGF@end?4roq?$AA@ 004bc7a4     cl_cin.obj
 0002:000007ac       ??_C@_0M@DDLBHMNL@demoend?4roq?$AA@ 004bc7ac     cl_cin.obj
 0002:000007b8       ??_C@_0BE@DDELHFMC@CL_PlayCinematic_f?6?$AA@ 004bc7b8     cl_cin.obj
 0002:000007cc       ??_C@_01EEMJAFIK@?6?$AA@   004bc7cc     cl_console.obj
 0002:000007d0       ??_C@_0BH@DBPHKMFK@ERROR?3?5couldn?8t?5open?4?6?$AA@ 004bc7d0     cl_console.obj
 0002:000007e8       ??_C@_0BM@HNBBHJDG@Dumped?5console?5text?5to?5?$CFs?4?6?$AA@ 004bc7e8     cl_console.obj
 0002:00000804       ??_C@_0BL@FAHDMBMK@usage?3?5condump?5?$DMfilename?$DO?6?$AA@ 004bc804     cl_console.obj
 0002:00000820       ??_C@_0N@BFMOJDMP@?$FLskipnotify?$FN?$AA@ 004bc820     cl_console.obj
 0002:00000830       __real@41800000            004bc830     cl_console.obj
 0002:00000834       __real@41000000            004bc834     cl_console.obj
 0002:00000838       ??_C@_04HKLMIPDN@say?3?$AA@ 004bc838     cl_console.obj
 0002:00000840       ??_C@_09LMMIOJG@say_team?3?$AA@ 004bc840     cl_console.obj
 0002:0000084c       __real@447a0000            004bc84c     cl_console.obj
 0002:00000850       ??_C@_08JLENPJJP@Q3?51?432b?$AA@ 004bc850     cl_console.obj
 0002:0000085c       __real@40000000            004bc85c     cl_console.obj
 0002:00000860       __real@43f00000            004bc860     cl_console.obj
 0002:00000864       ??_C@_07NENKHFEO@condump?$AA@ 004bc864     cl_console.obj
 0002:0000086c       ??_C@_05MEHLAELG@clear?$AA@ 004bc86c     cl_console.obj
 0002:00000874       ??_C@_0N@NFNJCLFL@messagemode4?$AA@ 004bc874     cl_console.obj
 0002:00000884       ??_C@_0N@JKJILNJM@messagemode3?$AA@ 004bc884     cl_console.obj
 0002:00000894       ??_C@_0N@IDIDIMNN@messagemode2?$AA@ 004bc894     cl_console.obj
 0002:000008a4       ??_C@_0M@JINOELJH@messagemode?$AA@ 004bc8a4     cl_console.obj
 0002:000008b0       ??_C@_0O@JJBKLGLG@toggleconsole?$AA@ 004bc8b0     cl_console.obj
 0002:000008c0       ??_C@_0N@MGJFCGAP@scr_conspeed?$AA@ 004bc8c0     cl_console.obj
 0002:000008d0       ??_C@_0P@INMLCMIF@con_notifytime?$AA@ 004bc8d0     cl_console.obj
 0002:000008e0       ??_C@_01EKENIIDA@3?$AA@    004bc8e0     cl_console.obj
 0002:000008e4       ??_C@_0BP@KKNANIBM@Three?5keys?5down?5for?5a?5button?$CB?6?$AA@ 004bc8e4     cl_input.obj
 0002:00000904       __real@3f800000            004bc904     cl_input.obj
 0002:00000908       __real@3f76800000000000    004bc908     cl_input.obj
 0002:00000910       ??_C@_0BO@PJHINAKI@CL_JoystickEvent?3?5bad?5axis?5?$CFi?$AA@ 004bc910     cl_input.obj
 0002:00000930       ??_C@_08ENNALHMG@?$CFf?5?3?5?$CFf?6?$AA@ 004bc930     cl_input.obj
 0002:00000940       __real@3fe0000000000000    004bc940     cl_input.obj
 0002:00000948       __real@43360b61            004bc948     cl_input.obj
 0002:0000094c       __real@42b40000            004bc94c     cl_input.obj
 0002:00000950       ??_C@_0O@FAEBFPEP@cl_maxpackets?$AA@ 004bc950     cl_input.obj
 0002:00000960       ??_C@_03BDPCEMGP@125?$AA@  004bc960     cl_input.obj
 0002:00000964       ??_C@_02IHCGGLPM@15?$AA@   004bc964     cl_input.obj
 0002:00000968       ??_C@_0DK@ONGDGOPA@WARNING?3?5?$CD462?5unsent?5fragments?5?$CI@ 004bc968     cl_input.obj
 0002:000009a4       ??_C@_04FMMAFMGP@?$CI?$CFi?$CJ?$AA@ 004bc9a4     cl_input.obj
 0002:000009ac       ??_C@_0BF@IEGIFLHJ@MAX_PACKET_USERCMDS?6?$AA@ 004bc9ac     cl_input.obj
 0002:000009c4       ??_C@_0N@HCACMDEB@cl_packetdup?$AA@ 004bc9c4     cl_input.obj
 0002:000009d4       ??_C@_01BMBHCPLG@5?$AA@    004bc9d4     cl_input.obj
 0002:000009d8       ??_C@_01GBGANLPD@0?$AA@    004bc9d8     cl_input.obj
 0002:000009dc       ??_C@_02KHOJGJKF@?4?5?$AA@ 004bc9dc     cl_input.obj
 0002:000009e0       ??_C@_0N@PJOLPAGC@cl_debugMove?$AA@ 004bc9e0     cl_input.obj
 0002:000009f0       ??_C@_0L@BPLIDNFG@cl_nodelta?$AA@ 004bc9f0     cl_input.obj
 0002:000009fc       ??_C@_06ICJGCHDB@?9mlook?$AA@ 004bc9fc     cl_input.obj
 0002:00000a04       ??_C@_06OBEGBCAL@?$CLmlook?$AA@ 004bca04     cl_input.obj
 0002:00000a0c       ??_C@_09OGHPIOCM@?9button14?$AA@ 004bca0c     cl_input.obj
 0002:00000a18       ??_C@_09OLGBPOGL@?$CLbutton14?$AA@ 004bca18     cl_input.obj
 0002:00000a24       ??_C@_09KJDOBIOL@?9button13?$AA@ 004bca24     cl_input.obj
 0002:00000a30       ??_C@_09KECAGIKM@?$CLbutton13?$AA@ 004bca30     cl_input.obj
 0002:00000a3c       ??_C@_09LACFCJKK@?9button12?$AA@ 004bca3c     cl_input.obj
 0002:00000a48       ??_C@_09LNDLFJON@?$CLbutton12?$AA@ 004bca48     cl_input.obj
 0002:00000a54       ??_C@_09JLAIHKGJ@?9button11?$AA@ 004bca54     cl_input.obj
 0002:00000a60       ??_C@_09JGBGAKCO@?$CLbutton11?$AA@ 004bca60     cl_input.obj
 0002:00000a6c       ??_C@_09ICBDELCI@?9button10?$AA@ 004bca6c     cl_input.obj
 0002:00000a78       ??_C@_09IPANDLGP@?$CLbutton10?$AA@ 004bca78     cl_input.obj
 0002:00000a84       ??_C@_08PFLPFDPC@?9button9?$AA@ 004bca84     cl_input.obj
 0002:00000a90       ??_C@_08IGKFCKHI@?$CLbutton9?$AA@ 004bca90     cl_input.obj
 0002:00000a9c       ??_C@_08OMKEGCLD@?9button8?$AA@ 004bca9c     cl_input.obj
 0002:00000aa8       ??_C@_08JPLOBLDJ@?$CLbutton8?$AA@ 004bcaa8     cl_input.obj
 0002:00000ab4       ??_C@_08GLDMHOHM@?9button7?$AA@ 004bcab4     cl_input.obj
 0002:00000ac0       ??_C@_08BICGAHPG@?$CLbutton7?$AA@ 004bcac0     cl_input.obj
 0002:00000acc       ??_C@_08HCCHEPDN@?9button6?$AA@ 004bcacc     cl_input.obj
 0002:00000ad8       ??_C@_08BDNDGLH@?$CLbutton6?$AA@ 004bcad8     cl_input.obj
 0002:00000ae4       ??_C@_08FJAKBMPO@?9button5?$AA@ 004bcae4     cl_input.obj
 0002:00000af0       ??_C@_08CKBAGFHE@?$CLbutton5?$AA@ 004bcaf0     cl_input.obj
 0002:00000afc       ??_C@_08EABBCNLP@?9button4?$AA@ 004bcafc     cl_input.obj
 0002:00000b08       ??_C@_08DDALFEDF@?$CLbutton4?$AA@ 004bcb08     cl_input.obj
 0002:00000b14       ??_C@_08PFALLHI@?9button3?$AA@ 004bcb14     cl_input.obj
 0002:00000b20       ??_C@_08HMEKMCPC@?$CLbutton3?$AA@ 004bcb20     cl_input.obj
 0002:00000b2c       ??_C@_08BGELIKDJ@?9button2?$AA@ 004bcb2c     cl_input.obj
 0002:00000b38       ??_C@_08GFFBPDLD@?$CLbutton2?$AA@ 004bcb38     cl_input.obj
 0002:00000b44       ??_C@_08DNGGNJPK@?9button1?$AA@ 004bcb44     cl_input.obj
 0002:00000b50       ??_C@_08EOHMKAHA@?$CLbutton1?$AA@ 004bcb50     cl_input.obj
 0002:00000b5c       ??_C@_08CEHNOILL@?9button0?$AA@ 004bcb5c     cl_input.obj
 0002:00000b68       ??_C@_08FHGHJBDB@?$CLbutton0?$AA@ 004bcb68     cl_input.obj
 0002:00000b74       ??_C@_07GIMEOOL@?9attack?$AA@ 004bcb74     cl_input.obj
 0002:00000b7c       ??_C@_07MAODEHGM@?$CLattack?$AA@ 004bcb7c     cl_input.obj
 0002:00000b84       ??_C@_06PLOIEHCE@?9speed?$AA@ 004bcb84     cl_input.obj
 0002:00000b8c       ??_C@_06JIDIHCBO@?$CLspeed?$AA@ 004bcb8c     cl_input.obj
 0002:00000b94       ??_C@_0L@LEKMOGAF@?9moveright?$AA@ 004bcb94     cl_input.obj
 0002:00000ba0       ??_C@_0L@FMBJCMEG@?$CLmoveright?$AA@ 004bcba0     cl_input.obj
 0002:00000bac       ??_C@_09ICIDCGOI@?9moveleft?$AA@ 004bcbac     cl_input.obj
 0002:00000bb8       ??_C@_09IPJNFGKP@?$CLmoveleft?$AA@ 004bcbb8     cl_input.obj
 0002:00000bc4       ??_C@_07OBMFNJMJ@?9strafe?$AA@ 004bcbc4     cl_input.obj
 0002:00000bcc       ??_C@_07CHKKNAEO@?$CLstrafe?$AA@ 004bcbcc     cl_input.obj
 0002:00000bd4       ??_C@_09KPLABCPP@?9lookdown?$AA@ 004bcbd4     cl_input.obj
 0002:00000be0       ??_C@_09KCKOGCLI@?$CLlookdown?$AA@ 004bcbe0     cl_input.obj
 0002:00000bec       ??_C@_07MHFKIPNM@?9lookup?$AA@ 004bcbec     cl_input.obj
 0002:00000bf4       ??_C@_07BDFIGFL@?$CLlookup?$AA@ 004bcbf4     cl_input.obj
 0002:00000bfc       ??_C@_05FJPPDLOK@?9back?$AA@ 004bcbfc     cl_input.obj
 0002:00000c04       ??_C@_05IPKGNIPH@?$CLback?$AA@ 004bcc04     cl_input.obj
 0002:00000c0c       ??_C@_08NJFEAJHL@?9forward?$AA@ 004bcc0c     cl_input.obj
 0002:00000c18       ??_C@_08KKEOHAPB@?$CLforward?$AA@ 004bcc18     cl_input.obj
 0002:00000c24       ??_C@_06LFFHCIPL@?9right?$AA@ 004bcc24     cl_input.obj
 0002:00000c2c       ??_C@_06NGIHBNMB@?$CLright?$AA@ 004bcc2c     cl_input.obj
 0002:00000c34       ??_C@_05KCDMNOKJ@?9left?$AA@ 004bcc34     cl_input.obj
 0002:00000c3c       ??_C@_05HEGFDNLE@?$CLleft?$AA@ 004bcc3c     cl_input.obj
 0002:00000c44       ??_C@_09HAIHLONB@?9movedown?$AA@ 004bcc44     cl_input.obj
 0002:00000c50       ??_C@_09HNJJMOJG@?$CLmovedown?$AA@ 004bcc50     cl_input.obj
 0002:00000c5c       ??_C@_07OMACAGKI@?9moveup?$AA@ 004bcc5c     cl_input.obj
 0002:00000c64       ??_C@_07CKGNAPCP@?$CLmoveup?$AA@ 004bcc64     cl_input.obj
 0002:00000c6c       ??_C@_0L@FHIBDANG@centerview?$AA@ 004bcc6c     cl_input.obj
 0002:00000c78       ??_C@_09COMJPDLF@SEMICOLON?$AA@ 004bcc78     cl_keys.obj
 0002:00000c84       ??_C@_05DIAHPDGL@PAUSE?$AA@ 004bcc84     cl_keys.obj
 0002:00000c8c       ??_C@_09GONHEPJO@KP_EQUALS?$AA@ 004bcc8c     cl_keys.obj
 0002:00000c98       ??_C@_07PCCOFIHH@KP_STAR?$AA@ 004bcc98     cl_keys.obj
 0002:00000ca0       ??_C@_0L@LEPHIPFO@KP_NUMLOCK?$AA@ 004bcca0     cl_keys.obj
 0002:00000cac       ??_C@_07CCBHGHDK@KP_PLUS?$AA@ 004bccac     cl_keys.obj
 0002:00000cb4       ??_C@_08KDIFPCFL@KP_MINUS?$AA@ 004bccb4     cl_keys.obj
 0002:00000cc0       ??_C@_08KHGBLJLO@KP_SLASH?$AA@ 004bccc0     cl_keys.obj
 0002:00000ccc       ??_C@_06KMLJNBKH@KP_DEL?$AA@ 004bcccc     cl_keys.obj
 0002:00000cd4       ??_C@_06JPNMOIAF@KP_INS?$AA@ 004bccd4     cl_keys.obj
 0002:00000cdc       ??_C@_08MHGPIJOM@KP_ENTER?$AA@ 004bccdc     cl_keys.obj
 0002:00000ce8       ??_C@_07BHJOEFGA@KP_PGDN?$AA@ 004bcce8     cl_keys.obj
 0002:00000cf0       ??_C@_0N@MJLAPIEJ@KP_DOWNARROW?$AA@ 004bccf0     cl_keys.obj
 0002:00000d00       ??_C@_06NAIJNDCL@KP_END?$AA@ 004bcd00     cl_keys.obj
 0002:00000d08       ??_C@_0O@NLCDAJLA@KP_RIGHTARROW?$AA@ 004bcd08     cl_keys.obj
 0002:00000d18       ??_C@_04BICCMFCD@KP_5?$AA@ 004bcd18     cl_keys.obj
 0002:00000d20       ??_C@_0N@DMPGMABG@KP_LEFTARROW?$AA@ 004bcd20     cl_keys.obj
 0002:00000d30       ??_C@_07NODLLDPI@KP_PGUP?$AA@ 004bcd30     cl_keys.obj
 0002:00000d38       ??_C@_0L@CCBCEPGH@KP_UPARROW?$AA@ 004bcd38     cl_keys.obj
 0002:00000d44       ??_C@_07GOJPFDII@KP_HOME?$AA@ 004bcd44     cl_keys.obj
 0002:00000d4c       ??_C@_05NIMGPOLB@AUX16?$AA@ 004bcd4c     cl_keys.obj
 0002:00000d54       ??_C@_05PDOLKNHC@AUX15?$AA@ 004bcd54     cl_keys.obj
 0002:00000d5c       ??_C@_05OKPAJMDD@AUX14?$AA@ 004bcd5c     cl_keys.obj
 0002:00000d64       ??_C@_05KFLBAKPE@AUX13?$AA@ 004bcd64     cl_keys.obj
 0002:00000d6c       ??_C@_05LMKKDLLF@AUX12?$AA@ 004bcd6c     cl_keys.obj
 0002:00000d74       ??_C@_05JHIHGIHG@AUX11?$AA@ 004bcd74     cl_keys.obj
 0002:00000d7c       ??_C@_05IOJMFJDH@AUX10?$AA@ 004bcd7c     cl_keys.obj
 0002:00000d84       ??_C@_04MMLGHEDJ@AUX9?$AA@ 004bcd84     cl_keys.obj
 0002:00000d8c       ??_C@_04NFKNEFHI@AUX8?$AA@ 004bcd8c     cl_keys.obj
 0002:00000d94       ??_C@_04FCDFFJLH@AUX7?$AA@ 004bcd94     cl_keys.obj
 0002:00000d9c       ??_C@_04ELCOGIPG@AUX6?$AA@ 004bcd9c     cl_keys.obj
 0002:00000da4       ??_C@_04GAADDLDF@AUX5?$AA@ 004bcda4     cl_keys.obj
 0002:00000dac       ??_C@_04HJBIAKHE@AUX4?$AA@ 004bcdac     cl_keys.obj
 0002:00000db4       ??_C@_04DGFJJMLD@AUX3?$AA@ 004bcdb4     cl_keys.obj
 0002:00000dbc       ??_C@_04CPECKNPC@AUX2?$AA@ 004bcdbc     cl_keys.obj
 0002:00000dc4       ??_C@_04EGPPODB@AUX1?$AA@  004bcdc4     cl_keys.obj
 0002:00000dcc       ??_C@_05EHAFPHFO@JOY32?$AA@ 004bcdcc     cl_keys.obj
 0002:00000dd4       ??_C@_05GMCIKEJN@JOY31?$AA@ 004bcdd4     cl_keys.obj
 0002:00000ddc       ??_C@_05HFDDJFNM@JOY30?$AA@ 004bcddc     cl_keys.obj
 0002:00000de4       ??_C@_05KFDDEEKC@JOY29?$AA@ 004bcde4     cl_keys.obj
 0002:00000dec       ??_C@_05LMCIHFOD@JOY28?$AA@ 004bcdec     cl_keys.obj
 0002:00000df4       ??_C@_05DLLAGJCM@JOY27?$AA@ 004bcdf4     cl_keys.obj
 0002:00000dfc       ??_C@_05CCKLFIGN@JOY26?$AA@ 004bcdfc     cl_keys.obj
 0002:00000e04       ??_C@_05JIGALKO@JOY25?$AA@ 004bce04     cl_keys.obj
 0002:00000e0c       ??_C@_05BAJNDKOP@JOY24?$AA@ 004bce0c     cl_keys.obj
 0002:00000e14       ??_C@_05FPNMKMCI@JOY23?$AA@ 004bce14     cl_keys.obj
 0002:00000e1c       ??_C@_05EGMHJNGJ@JOY22?$AA@ 004bce1c     cl_keys.obj
 0002:00000e24       ??_C@_05GNOKMOKK@JOY21?$AA@ 004bce24     cl_keys.obj
 0002:00000e2c       ??_C@_05HEPBPPOL@JOY20?$AA@ 004bce2c     cl_keys.obj
 0002:00000e34       ??_C@_05KHHFPKPL@JOY19?$AA@ 004bce34     cl_keys.obj
 0002:00000e3c       ??_C@_05LOGOMLLK@JOY18?$AA@ 004bce3c     cl_keys.obj
 0002:00000e44       ??_C@_05DJPGNHHF@JOY17?$AA@ 004bce44     cl_keys.obj
 0002:00000e4c       ??_C@_05CAONOGDE@JOY16?$AA@ 004bce4c     cl_keys.obj
 0002:00000e54       ??_C@_05LMALFPH@JOY15?$AA@ 004bce54     cl_keys.obj
 0002:00000e5c       ??_C@_05BCNLIELG@JOY14?$AA@ 004bce5c     cl_keys.obj
 0002:00000e64       ??_C@_05FNJKBCHB@JOY13?$AA@ 004bce64     cl_keys.obj
 0002:00000e6c       ??_C@_05EEIBCDDA@JOY12?$AA@ 004bce6c     cl_keys.obj
 0002:00000e74       ??_C@_05GPKMHAPD@JOY11?$AA@ 004bce74     cl_keys.obj
 0002:00000e7c       ??_C@_05HGLHEBLC@JOY10?$AA@ 004bce7c     cl_keys.obj
 0002:00000e84       ??_C@_04IFAAJIOE@JOY9?$AA@ 004bce84     cl_keys.obj
 0002:00000e8c       ??_C@_04JMBLKJKF@JOY8?$AA@ 004bce8c     cl_keys.obj
 0002:00000e94       ??_C@_04BLIDLFGK@JOY7?$AA@ 004bce94     cl_keys.obj
 0002:00000e9c       ??_C@_04CJIIECL@JOY6?$AA@  004bce9c     cl_keys.obj
 0002:00000ea4       ??_C@_04CJLFNHOI@JOY5?$AA@ 004bcea4     cl_keys.obj
 0002:00000eac       ??_C@_04DAKOOGKJ@JOY4?$AA@ 004bceac     cl_keys.obj
 0002:00000eb4       ??_C@_04HPOPHAGO@JOY3?$AA@ 004bceb4     cl_keys.obj
 0002:00000ebc       ??_C@_04GGPEEBCP@JOY2?$AA@ 004bcebc     cl_keys.obj
 0002:00000ec4       ??_C@_04ENNJBCOM@JOY1?$AA@ 004bcec4     cl_keys.obj
 0002:00000ecc       ??_C@_0L@NBPPJGMJ@MWHEELDOWN?$AA@ 004bcecc     cl_keys.obj
 0002:00000ed8       ??_C@_08NAKENEKM@MWHEELUP?$AA@ 004bced8     cl_keys.obj
 0002:00000ee4       ??_C@_06EEGKOBOL@MOUSE5?$AA@ 004bcee4     cl_keys.obj
 0002:00000eec       ??_C@_06FNHBNAKK@MOUSE4?$AA@ 004bceec     cl_keys.obj
 0002:00000ef4       ??_C@_06BCDAEGGN@MOUSE3?$AA@ 004bcef4     cl_keys.obj
 0002:00000efc       ??_C@_06LCLHHCM@MOUSE2?$AA@ 004bcefc     cl_keys.obj
 0002:00000f04       ??_C@_06CAAGCEOP@MOUSE1?$AA@ 004bcf04     cl_keys.obj
 0002:00000f0c       ??_C@_03JMGAKCCH@END?$AA@  004bcf0c     cl_keys.obj
 0002:00000f10       ??_C@_04GHGFPGNC@HOME?$AA@ 004bcf10     cl_keys.obj
 0002:00000f18       ??_C@_04NHMBBGKC@PGUP?$AA@ 004bcf18     cl_keys.obj
 0002:00000f20       ??_C@_04BOGEOADK@PGDN?$AA@ 004bcf20     cl_keys.obj
 0002:00000f28       ??_C@_03OAFAKAKL@DEL?$AA@  004bcf28     cl_keys.obj
 0002:00000f2c       ??_C@_03NDDFJJAJ@INS?$AA@  004bcf2c     cl_keys.obj
 0002:00000f30       ??_C@_03KIBNPMNE@F12?$AA@  004bcf30     cl_keys.obj
 0002:00000f34       ??_C@_03IDDAKPBH@F11?$AA@  004bcf34     cl_keys.obj
 0002:00000f38       ??_C@_03JKCLJOFG@F10?$AA@  004bcf38     cl_keys.obj
 0002:00000f3c       ??_C@_02HKCNFKCF@F9?$AA@   004bcf3c     cl_keys.obj
 0002:00000f40       ??_C@_02GDDGGLGE@F8?$AA@   004bcf40     cl_keys.obj
 0002:00000f44       ??_C@_02OEKOHHKL@F7?$AA@   004bcf44     cl_keys.obj
 0002:00000f48       ??_C@_02PNLFEGOK@F6?$AA@   004bcf48     cl_keys.obj
 0002:00000f4c       ??_C@_02NGJIBFCJ@F5?$AA@   004bcf4c     cl_keys.obj
 0002:00000f50       ??_C@_02MPIDCEGI@F4?$AA@   004bcf50     cl_keys.obj
 0002:00000f54       ??_C@_02IAMCLCKP@F3?$AA@   004bcf54     cl_keys.obj
 0002:00000f58       ??_C@_02JJNJIDOO@F2?$AA@   004bcf58     cl_keys.obj
 0002:00000f5c       ??_C@_02LCPENACN@F1?$AA@   004bcf5c     cl_keys.obj
 0002:00000f60       ??_C@_08INDENNHK@CAPSLOCK?$AA@ 004bcf60     cl_keys.obj
 0002:00000f6c       ??_C@_07FBJAHANB@COMMAND?$AA@ 004bcf6c     cl_keys.obj
 0002:00000f74       ??_C@_05OAHIEJBI@SHIFT?$AA@ 004bcf74     cl_keys.obj
 0002:00000f7c       ??_C@_04FBBFEIFJ@CTRL?$AA@ 004bcf7c     cl_keys.obj
 0002:00000f84       ??_C@_03FKEEPDEP@ALT?$AA@  004bcf84     cl_keys.obj
 0002:00000f88       ??_C@_0L@CIPLPPIL@RIGHTARROW?$AA@ 004bcf88     cl_keys.obj
 0002:00000f94       ??_C@_09FNHBLDAE@LEFTARROW?$AA@ 004bcf94     cl_keys.obj
 0002:00000fa0       ??_C@_09KIDHILFL@DOWNARROW?$AA@ 004bcfa0     cl_keys.obj
 0002:00000fac       ??_C@_07MNCBLHKG@UPARROW?$AA@ 004bcfac     cl_keys.obj
 0002:00000fb4       ??_C@_09MALOLBMO@BACKSPACE?$AA@ 004bcfb4     cl_keys.obj
 0002:00000fc0       ??_C@_05CAEOFMEP@SPACE?$AA@ 004bcfc0     cl_keys.obj
 0002:00000fc8       ??_C@_06CDPDIIDH@ESCAPE?$AA@ 004bcfc8     cl_keys.obj
 0002:00000fd0       ??_C@_05EMNIMLKD@ENTER?$AA@ 004bcfd0     cl_keys.obj
 0002:00000fd8       ??_C@_03CJMDHCGG@TAB?$AA@  004bcfd8     cl_keys.obj
 0002:00000fdc       ??_C@_0BM@MHAABCMH@drawLen?5?$DO?$DN?5MAX_STRING_CHARS?$AA@ 004bcfdc     cl_keys.obj
 0002:00000ff8       ??_C@_0P@IGICGKLH@?$DMOUT?5OF?5RANGE?$DO?$AA@ 004bcff8     cl_keys.obj
 0002:00001008       ??_C@_0BA@FLLJDFDJ@?$DMKEY?5NOT?5FOUND?$DO?$AA@ 004bd008     cl_keys.obj
 0002:00001018       ??_C@_0BI@PLEALGJH@?$CC?$CFs?$CC?5isn?8t?5a?5valid?5key?6?$AA@ 004bd018     cl_keys.obj
 0002:00001030       ??_C@_0CL@OCGCHGGL@unbind?5?$DMkey?$DO?5?3?5remove?5commands?5f@ 004bd030     cl_keys.obj
 0002:0000105c       ??_C@_01CLKCMJKC@?5?$AA@   004bd05c     cl_keys.obj
 0002:00001060       ??_C@_0BD@BAINEHPI@?$CC?$CFs?$CC?5is?5not?5bound?6?$AA@ 004bd060     cl_keys.obj
 0002:00001074       ??_C@_0N@CHDOIAJI@?$CC?$CFs?$CC?5?$DN?5?$CC?$CFs?$CC?6?$AA@ 004bd074     cl_keys.obj
 0002:00001084       ??_C@_0DC@GHIPCCCE@bind?5?$DMkey?$DO?5?$FLcommand?$FN?5?3?5attach?5a?5@ 004bd084     cl_keys.obj
 0002:000010b8       ??_C@_0O@HKEPFNEK@bind?5?$CFs?5?$CC?$CFs?$CC?6?$AA@ 004bd0b8     cl_keys.obj
 0002:000010c8       ??_C@_0L@EPHOCAKP@unbindall?6?$AA@ 004bd0c8     cl_keys.obj
 0002:000010d4       ??_C@_08MHBLPCGN@?$CFs?5?$CC?$CFs?$CC?6?$AA@ 004bd0d4     cl_keys.obj
 0002:000010e0       ??_C@_08OLCDMLCJ@bindlist?$AA@ 004bd0e0     cl_keys.obj
 0002:000010ec       ??_C@_09EBAHBELN@unbindall?$AA@ 004bd0ec     cl_keys.obj
 0002:000010f8       ??_C@_06IDJGFAK@unbind?$AA@ 004bd0f8     cl_keys.obj
 0002:00001100       ??_C@_04NPNJNMMP@bind?$AA@ 004bd100     cl_keys.obj
 0002:00001108       ??_C@_0L@BJOGPJJF@?9?$CFs?5?$CFi?5?$CFi?6?$AA@ 004bd108     cl_keys.obj
 0002:00001114       ??_C@_08LMOPPDJO@cmd?5say?5?$AA@ 004bd114     cl_keys.obj
 0002:00001120       ??_C@_04MCOKGCBH@?$FN?$CFs?6?$AA@ 004bd120     cl_keys.obj
 0002:00001128       ??_C@_03GFPEDOMH@?2?$CFs?$AA@ 004bd128     cl_keys.obj
 0002:0000112c       ??_C@_06NICJIFDH@clear?6?$AA@ 004bd12c     cl_keys.obj
 0002:00001134       ??_C@_09MNFIPOON@say?5?$CC?$CFs?$CC?6?$AA@ 004bd134     cl_keys.obj
 0002:00001140       ??_C@_0P@BAMGBHOI@say_team?5?$CC?$CFs?$CC?6?$AA@ 004bd140     cl_keys.obj
 0002:00001150       ??_C@_0O@MFAGMBFC@tell?5?$CFi?5?$CC?$CFs?$CC?6?$AA@ 004bd150     cl_keys.obj
 0002:00001160       ??_C@_09NMODOCNP@?$CFs?5?$CFi?5?$CFi?6?$AA@ 004bd160     cl_keys.obj
 0002:0000116c       ??_C@_0CK@GMJFPAOO@?$CFs?5is?5unbound?0?5use?5controls?5menu@ 004bd16c     cl_keys.obj
 0002:00001198       ??_C@_08JIEIDHIE@nextdemo?$AA@ 004bd198     cl_keys.obj
 0002:000011a4       ??_C@_0P@EIAPFKBF@com_cameraMode?$AA@ 004bd1a4     cl_keys.obj
 0002:000011b4       ??_C@_0BI@EAPJOGJE@Client?5command?5overflow?$AA@ 004bd1b4     cl_main.obj
 0002:000011cc       ??_C@_0P@JFMMMOHN@Stopped?5demo?4?6?$AA@ 004bd1cc     cl_main.obj
 0002:000011dc       ??_C@_0BH@FJJDMOAC@Not?5recording?5a?5demo?4?6?$AA@ 004bd1dc     cl_main.obj
 0002:000011f4       ??_C@_0N@JINADPLJ@demo9999?4tga?$AA@ 004bd1f4     cl_main.obj
 0002:00001204       ??_C@_0N@EFJGOOKC@demo?$CFi?$CFi?$CFi?$CFi?$AA@ 004bd204     cl_main.obj
 0002:00001214       ??_C@_0BA@OHINOCDN@ui_recordSPDemo?$AA@ 004bd214     cl_main.obj
 0002:00001224       ??_C@_0BC@PMCLPAOL@recording?5to?5?$CFs?4?6?$AA@ 004bd224     cl_main.obj
 0002:00001238       ??_C@_0P@JBKMAJI@demos?1?$CFs?4dm_?$CFd?$AA@ 004bd238     cl_main.obj
 0002:00001248       ??_C@_0FA@PLJDEPGO@?$FO3WARNING?3?5You?5should?5set?5?8g_syn@ 004bd248     cl_main.obj
 0002:00001298       ??_C@_0BF@LICFCALK@g_synchronousClients?$AA@ 004bd298     cl_main.obj
 0002:000012b0       ??_C@_0CD@JLOAFGIP@You?5must?5be?5in?5a?5level?5to?5record@ 004bd2b0     cl_main.obj
 0002:000012d4       ??_C@_0BE@GOGLPLDO@Already?5recording?4?6?$AA@ 004bd2d4     cl_main.obj
 0002:000012e8       ??_C@_0BD@PGNLAEFI@record?5?$DMdemoname?$DO?6?$AA@ 004bd2e8     cl_main.obj
 0002:000012fc       ??_C@_0P@NIDHDKPC@Demo?5file?3?5?$CFs?6?$AA@ 004bd2fc     cl_main.obj
 0002:0000130c       ??_C@_0P@HACEFMAG@Not?5found?3?5?$CFs?6?$AA@ 004bd30c     cl_main.obj
 0002:0000131c       ??_C@_03LFLJCHJK@d1?6?$AA@ 004bd31c     cl_main.obj
 0002:00001320       ??_C@_0BB@HGODKPPP@CL_NextDemo?3?5?$CFs?6?$AA@ 004bd320     cl_main.obj
 0002:00001334       ??_C@_09NFOPKLIK@sv_cheats?$AA@ 004bd334     cl_main.obj
 0002:00001340       ??_C@_0BA@MIMGFFNE@cl_downloadName?$AA@ 004bd340     cl_main.obj
 0002:00001350       ??_C@_0P@FABCFONG@r_uiFullScreen?$AA@ 004bd350     cl_main.obj
 0002:00001360       ??_C@_01HIHLOKLC@1?$AA@    004bd360     cl_main.obj
 0002:00001364       ??_C@_0BG@NHOAAIGH@Unknown?5command?5?$CC?$CFs?$CC?6?$AA@ 004bd364     cl_main.obj
 0002:0000137c       ??_C@_0O@IFNCIAOO@getmotd?5?$CC?$CFs?$CC?6?$AA@ 004bd37c     cl_main.obj
 0002:0000138c       ??_C@_07CPCPJPKL@version?$AA@ 004bd38c     cl_main.obj
 0002:00001394       ??_C@_08NELFFGLM@renderer?$AA@ 004bd394     cl_main.obj
 0002:000013a0       ??_C@_09DBEGHIJJ@challenge?$AA@ 004bd3a0     cl_main.obj
 0002:000013ac       ??_C@_02IKAHHCAI@?$CFi?$AA@ 004bd3ac     cl_main.obj
 0002:000013b0       ??_C@_0BP@FPDCKHM@?$CFs?5resolved?5to?5?$CFi?4?$CFi?4?$CFi?4?$CFi?3?$CFi?6?$AA@ 004bd3b0     cl_main.obj
 0002:000013d0       ??_C@_0BK@PDDCGPDI@Couldn?8t?5resolve?5address?6?$AA@ 004bd3d0     cl_main.obj
 0002:000013ec       ??_C@_0O@NIMOHCFP@Resolving?5?$CFs?6?$AA@ 004bd3ec     cl_main.obj
 0002:000013fc       ??_C@_0BH@CEAMHKGJ@update?4quake3arena?4com?$AA@ 004bd3fc     cl_main.obj
 0002:00001414       ??_C@_0BG@FGGNFFEK@getKeyAuthorize?5?$CFi?5?$CFs?$AA@ 004bd414     cl_main.obj
 0002:0000142c       ??_C@_0N@IFIIDPHP@cl_anonymous?$AA@ 004bd42c     cl_main.obj
 0002:0000143c       ??_C@_06GIKKBIFN@demota?$AA@ 004bd43c     cl_main.obj
 0002:00001444       ??_C@_0M@KDAJBLAP@fs_restrict?$AA@ 004bd444     cl_main.obj
 0002:00001450       ??_C@_0BK@MNOBFHCL@authorize?4quake3arena?4com?$AA@ 004bd450     cl_main.obj
 0002:0000146c       ??_C@_0BM@PIMKCOAK@Not?5connected?5to?5a?5server?4?6?$AA@ 004bd46c     cl_main.obj
 0002:00001488       ??_C@_0O@PJAFINBM@?$CFs?5undefined?6?$AA@ 004bd488     cl_main.obj
 0002:00001498       ??_C@_06BAKFFEGN@?$CFs?$DN?$CFs?6?$AA@ 004bd498     cl_main.obj
 0002:000014a0       ??_C@_01NEMOKFLO@?$DN?$AA@ 004bd4a0     cl_main.obj
 0002:000014a4       ??_C@_0BJ@EBHAICOP@Disconnected?5from?5server?$AA@ 004bd4a4     cl_main.obj
 0002:000014c0       ??_C@_0BG@JDIGCOKJ@ui_singlePlayerActive?$AA@ 004bd4c0     cl_main.obj
 0002:000014d8       ??_C@_0BP@KAEALGFM@Can?8t?5reconnect?5to?5localhost?4?6?$AA@ 004bd4d8     cl_main.obj
 0002:000014f8       ??_C@_0M@LNGHCJI@connect?5?$CFs?6?$AA@ 004bd4f8     cl_main.obj
 0002:00001504       ??_C@_09IPAEKDAI@localhost?$AA@ 004bd504     cl_main.obj
 0002:00001510       ??_C@_0BI@OBPNNDLP@cl_currentServerAddress?$AA@ 004bd510     cl_main.obj
 0002:00001528       ??_C@_0BE@BMPNGILO@Bad?5server?5address?6?$AA@ 004bd528     cl_main.obj
 0002:0000153c       ??_C@_0O@JEEKIFAP@sv_killserver?$AA@ 004bd53c     cl_main.obj
 0002:0000154c       ??_C@_0N@IAGKKNPJ@Server?5quit?6?$AA@ 004bd54c     cl_main.obj
 0002:0000155c       ??_C@_0BJ@JGJJEKBC@usage?3?5connect?5?$FLserver?$FN?6?$AA@ 004bd55c     cl_main.obj
 0002:00001578       ??_C@_0FE@GKHHMJFK@You?5must?5either?5be?5connected?0?6or@ 004bd578     cl_main.obj
 0002:000015cc       ??_C@_05GCMNNKNG@rcon?5?$AA@ 004bd5cc     cl_main.obj
 0002:000015d4       ??_C@_0DN@LCHLNDDC@You?5must?5set?5?8rconpassword?8?5befo@ 004bd5d4     cl_main.obj
 0002:00001614       ??_C@_03JDANDILB@?$CFd?5?$AA@ 004bd614     cl_main.obj
 0002:00001618       ??_C@_03LBGAPDPL@Yf?5?$AA@ 004bd618     cl_main.obj
 0002:0000161c       ??_C@_03MCDIKHCL@vdr?$AA@  004bd61c     cl_main.obj
 0002:00001620       ??_C@_0BG@KJOBEGLE@Opened?5PK3?5Names?3?5?$CFs?6?$AA@ 004bd620     cl_main.obj
 0002:00001638       ??_C@_0BK@GENIKODO@Referenced?5PK3?5Names?3?5?$CFs?6?$AA@ 004bd638     cl_main.obj
 0002:00001654       ??_C@_08JBKNBCEM@?$CF4i?3?5?$CFs?6?$AA@ 004bd654     cl_main.obj
 0002:00001660       ??_C@_0CI@DBDLLCJO@?9?9?9?9?9?9?9?9?9?9?9?9?9?9?9?9?9?9?9?9?9?9?9?9?9?9?9?9?9?9?9?9@ 004bd660     cl_main.obj
 0002:00001688       ??_C@_0BF@CNHFFNEA@User?5info?5settings?3?6?$AA@ 004bd688     cl_main.obj
 0002:000016a0       ??_C@_0M@CDCBGBHB@Server?3?5?$CFs?6?$AA@ 004bd6a0     cl_main.obj
 0002:000016ac       ??_C@_0L@PILDHKCK@state?3?5?$CFi?6?$AA@ 004bd6ac     cl_main.obj
 0002:000016b8       ??_C@_0CI@OGJFLPIM@?9?9?9?9?9?9?9?9?9?5Client?5Information?5?9?9?9@ 004bd6b8     cl_main.obj
 0002:000016e0       ??_C@_0M@CDGAENEE@download?5?$CFs?$AA@ 004bd6e0     cl_main.obj
 0002:000016ec       ??_C@_0BA@CHCCPCBI@cl_downloadTime?$AA@ 004bd6ec     cl_main.obj
 0002:000016fc       ??_C@_0BB@FAHDFBEE@cl_downloadCount?$AA@ 004bd6fc     cl_main.obj
 0002:00001710       ??_C@_0BA@IMGLJLPN@cl_downloadSize?$AA@ 004bd710     cl_main.obj
 0002:00001720       ??_C@_06IHDMMOPO@?$CFs?4tmp?$AA@ 004bd720     cl_main.obj
 0002:00001728       ??_C@_0FI@OJLPOMHD@?$CK?$CK?$CK?$CK?$CK?5CL_BeginDownload?5?$CK?$CK?$CK?$CK?$CK?6Loc@ 004bd728     cl_main.obj
 0002:00001780       ??_C@_0N@FADCLAAC@getchallenge?$AA@ 004bd780     cl_main.obj
 0002:00001790       ??_C@_08CCJJPJEL@connect?5?$AA@ 004bd790     cl_main.obj
 0002:0000179c       ??_C@_05IPCIHGO@qport?$AA@ 004bd79c     cl_main.obj
 0002:000017a4       ??_C@_08FCFPNNHF@protocol?$AA@ 004bd7a4     cl_main.obj
 0002:000017b0       ??_C@_09HOOHLIKH@net_qport?$AA@ 004bd7b0     cl_main.obj
 0002:000017bc       ??_C@_0CB@JLKOHGFD@CL_CheckForResend?3?5bad?5cls?4state@ 004bd7bc     cl_main.obj
 0002:000017e0       ??_C@_0BB@GDGLAKGE@com_errorMessage?$AA@ 004bd7e0     cl_main.obj
 0002:000017f4       ??_C@_0CI@POLDFEDD@Server?5disconnected?5for?5unknown?5@ 004bd7f4     cl_main.obj
 0002:0000181c       ??_C@_0O@GJFLJONJ@cl_motdString?$AA@ 004bd81c     cl_main.obj
 0002:0000182c       ??_C@_04GJFDDCGE@motd?$AA@ 004bd82c     cl_main.obj
 0002:00001834       ??_C@_0BO@DIFEDBKJ@?$CFd?5servers?5parsed?5?$CItotal?5?$CFd?$CJ?6?$AA@ 004bd834     cl_main.obj
 0002:00001854       ??_C@_0BP@DMDBGEFJ@server?3?5?$CFd?5ip?3?5?$CFd?4?$CFd?4?$CFd?4?$CFd?3?$CFd?6?$AA@ 004bd854     cl_main.obj
 0002:00001874       ??_C@_0BK@BOAAMPMC@CL_ServersResponsePacket?6?$AA@ 004bd874     cl_main.obj
 0002:00001890       ??_C@_0BP@CBAODGNF@?6Server?5connection?5timed?5out?4?6?$AA@ 004bd890     cl_main.obj
 0002:000018b0       ??_C@_0O@FJGEONLL@userinfo?5?$CC?$CFs?$CC?$AA@ 004bd8b0     cl_main.obj
 0002:000018c0       __real@3fd0000000000000    004bd8c0     cl_main.obj
 0002:000018c8       ??_C@_0BD@MBKJOELF@screenshot?5silent?6?$AA@ 004bd8c8     cl_main.obj
 0002:000018dc       ??_C@_04MMPNEILC@?$FO1?$CFs?$AA@ 004bd8dc     cl_main.obj
 0002:000018e4       ??_C@_04GGPEIADJ@?$FO3?$CFs?$AA@ 004bd8e4     cl_main.obj
 0002:000018ec       ??_C@_07PMJAFAE@console?$AA@ 004bd8ec     cl_main.obj
 0002:000018f4       ??_C@_05PMAELIEO@white?$AA@ 004bd8f4     cl_main.obj
 0002:000018fc       ??_C@_0BA@FILGFBEK@gfx?12d?1bigchars?$AA@ 004bd8fc     cl_main.obj
 0002:0000190c       ??_C@_09DIABHAFB@cl_paused?$AA@ 004bd90c     cl_main.obj
 0002:00001918       ??_C@_0BM@BKBAAMDA@Couldn?8t?5initialize?5refresh?$AA@ 004bd918     cl_main.obj
 0002:00001934       ??_C@_0CB@LHLKLKOG@?9?9?9?9?9?9?9?9?9?9?9?9?9?9?9?9?9?9?9?9?9?9?9?9?9?9?9?9?9?9?9?6@ 004bd934     cl_main.obj
 0002:00001958       ??_C@_0CC@CKFOOPEI@?9?9?9?9?9?5Initializing?5Renderer?5?9?9?9?9@ 004bd958     cl_main.obj
 0002:0000197c       ??_C@_0BE@BOKBONJL@model?5is?5set?5to?5?$CFs?6?$AA@ 004bd97c     cl_main.obj
 0002:00001990       ??_C@_09DHBBGOBJ@headmodel?$AA@ 004bd990     cl_main.obj
 0002:0000199c       ??_C@_05NCCFOPHA@model?$AA@ 004bd99c     cl_main.obj
 0002:000019a4       ??_C@_0BJ@NDLHEOCN@?9?9?9?9?9?9?9?9?9?9?9?9?9?9?9?9?9?9?9?9?9?9?9?6?$AA@ 004bd9a4     cl_main.obj
 0002:000019c0       ??_C@_0L@FBHMLJNH@cl_running?$AA@ 004bd9c0     cl_main.obj
 0002:000019cc       ??_C@_06NOAHJGOA@showip?$AA@ 004bd9cc     cl_main.obj
 0002:000019d4       ??_C@_0N@LJMIJCBN@serverstatus?$AA@ 004bd9d4     cl_main.obj
 0002:000019e4       ??_C@_04OONEELOO@ping?$AA@ 004bd9e4     cl_main.obj
 0002:000019ec       ??_C@_06NMKMANLK@setenv?$AA@ 004bd9ec     cl_main.obj
 0002:000019f4       ??_C@_04CLKJCJJE@rcon?$AA@ 004bd9f4     cl_main.obj
 0002:000019fc       ??_C@_0O@BBKHNMKE@globalservers?$AA@ 004bd9fc     cl_main.obj
 0002:00001a0c       ??_C@_0N@OHPGBJMI@localservers?$AA@ 004bda0c     cl_main.obj
 0002:00001a1c       ??_C@_07KAIBNCHO@connect?$AA@ 004bda1c     cl_main.obj
 0002:00001a24       ??_C@_0L@OLGNCHFI@stoprecord?$AA@ 004bda24     cl_main.obj
 0002:00001a30       ??_C@_09DHDJHDLH@cinematic?$AA@ 004bda30     cl_main.obj
 0002:00001a3c       ??_C@_04PLPNPBEF@demo?$AA@ 004bda3c     cl_main.obj
 0002:00001a44       ??_C@_06KKGOIHDP@record?$AA@ 004bda44     cl_main.obj
 0002:00001a4c       ??_C@_0M@DIIAMDPB@vid_restart?$AA@ 004bda4c     cl_main.obj
 0002:00001a58       ??_C@_0M@IJBIKBGC@snd_restart?$AA@ 004bda58     cl_main.obj
 0002:00001a64       ??_C@_08PPJNGBMG@userinfo?$AA@ 004bda64     cl_main.obj
 0002:00001a70       ??_C@_0O@OBMKKPAG@configstrings?$AA@ 004bda70     cl_main.obj
 0002:00001a80       ??_C@_03LGLGIONO@cmd?$AA@  004bda80     cl_main.obj
 0002:00001a84       ??_C@_0BE@LMHMEFGD@recursive?5shutdown?6?$AA@ 004bda84     cl_main.obj
 0002:00001a98       ??_C@_0BJ@EPBBJNIE@?9?9?9?9?9?5CL_Shutdown?5?9?9?9?9?9?6?$AA@ 004bda98     cl_main.obj
 0002:00001ab4       ??_C@_0L@CNOGMKDC@punkbuster?$AA@ 004bdab4     cl_main.obj
 0002:00001ac0       ??_C@_07MMIKBOAN@maxping?$AA@ 004bdac0     cl_main.obj
 0002:00001ac8       ??_C@_07CKOKLBOM@minping?$AA@ 004bdac8     cl_main.obj
 0002:00001ad0       ??_C@_07EAJPOACB@nettype?$AA@ 004bdad0     cl_main.obj
 0002:00001ad8       ??_C@_08NJPDEKHO@gametype?$AA@ 004bdad8     cl_main.obj
 0002:00001ae4       ??_C@_04MJNAPEEI@game?$AA@ 004bdae4     cl_main.obj
 0002:00001aec       ??_C@_0O@OCOCOONB@sv_maxclients?$AA@ 004bdaec     cl_main.obj
 0002:00001afc       ??_C@_08EHKIGBEA@hostname?$AA@ 004bdafc     cl_main.obj
 0002:00001b08       ??_C@_07HKJFGNHJ@clients?$AA@ 004bdb08     cl_main.obj
 0002:00001b10       ??_C@_06DJHOIPC@?$CFs?3?5?$CFs?$AA@ 004bdb10     cl_main.obj
 0002:00001b18       ??_C@_02DPKJAMEF@?$CFd?$AA@ 004bdb18     cl_main.obj
 0002:00001b1c       ??_C@_0BI@DBADJLIK@ping?5time?5?$CFdms?5from?5?$CFs?6?$AA@ 004bdb1c     cl_main.obj
 0002:00001b34       ??_C@_0CO@PDOECEBD@MAX_OTHER_SERVERS?5hit?0?5dropping?5@ 004bdb34     cl_main.obj
 0002:00001b64       ??_C@_0CE@BMBLKOLI@Different?5protocol?5info?5packet?3?5@ 004bdb64     cl_main.obj
 0002:00001b88       ??_C@_09EKLELPNI@getstatus?$AA@ 004bdb88     cl_main.obj
 0002:00001b94       ??_C@_0BK@GJAGDIHH@?$CF?92d?5?5?5?$CF?93d?5?5?5?5?$CF?93d?5?5?5?$CFs?6?$AA@ 004bdb94     cl_main.obj
 0002:00001bb0       ??_C@_07CIFAGBMG@unknown?$AA@ 004bdbb0     cl_main.obj
 0002:00001bb8       ??_C@_05OKMLJOMC@?$CFd?5?$CFd?$AA@ 004bdbb8     cl_main.obj
 0002:00001bc0       ??_C@_0BJ@FOGFOPMO@num?3?5score?3?5ping?3?5name?3?6?$AA@ 004bdbc0     cl_main.obj
 0002:00001bdc       ??_C@_0L@GBJHHNEK@?6Players?3?6?$AA@ 004bdbdc     cl_main.obj
 0002:00001be8       ??_C@_05FNFPHGDP@?$CF?924s?$AA@ 004bdbe8     cl_main.obj
 0002:00001bf0       ??_C@_0BC@KPIAKMPH@Server?5settings?3?6?$AA@ 004bdbf0     cl_main.obj
 0002:00001c04       ??_C@_0BA@HEMALGFI@?$PP?$PP?$PP?$PPgetinfo?5xxx?$AA@ 004bdc04     cl_main.obj
 0002:00001c14       ??_C@_0CO@LIFGMECC@Scanning?5for?5servers?5on?5the?5loca@ 004bdc14     cl_main.obj
 0002:00001c44       ??_C@_05ILLBKCMN@?5demo?$AA@ 004bdc44     cl_main.obj
 0002:00001c4c       ??_C@_03EEBNCBOD@?5?$CFs?$AA@ 004bdc4c     cl_main.obj
 0002:00001c50       ??_C@_0O@KMBAKMAC@getservers?5?$CFs?$AA@ 004bdc50     cl_main.obj
 0002:00001c60       ??_C@_0BH@HJHKJDCC@master?4quake3arena?4com?$AA@ 004bdc60     cl_main.obj
 0002:00001c78       ??_C@_0CH@IJAABCGN@Requesting?5servers?5from?5the?5mast@ 004bdc78     cl_main.obj
 0002:00001ca0       ??_C@_0DK@CEAJIEBF@usage?3?5globalservers?5?$DMmaster?$CD?50?9@ 004bdca0     cl_main.obj
 0002:00001cdc       ??_C@_0L@KMOIMFOM@cl_maxPing?$AA@ 004bdcdc     cl_main.obj
 0002:00001ce8       ??_C@_0M@PAOKIPMI@getinfo?5xxx?$AA@ 004bdce8     cl_main.obj
 0002:00001cf4       ??_C@_0BG@GCANHGBC@usage?3?5ping?5?$FLserver?$FN?6?$AA@ 004bdcf4     cl_main.obj
 0002:00001d0c       ??_C@_0BO@PKCGGDHB@Usage?3?5serverstatus?5?$FLserver?$FN?6?$AA@ 004bdd0c     cl_main.obj
 0002:00001d2c       ??_C@_04NOJCDH@?$CF02x?$AA@ 004bdd2c     cl_main.obj
 0002:00001d34       ??_C@_0CF@PCNJDKKO@?$CFi?5frames?0?5?$CF3?41f?5seconds?3?5?$CF3?41f?5@ 004bdd34     cl_main.obj
 0002:00001d60       __real@408f400000000000    004bdd60     cl_main.obj
 0002:00001d68       ??_C@_0BK@CDNCLIJC@Demo?5file?5was?5truncated?4?6?$AA@ 004bdd68     cl_main.obj
 0002:00001d84       ??_C@_0CM@CDKKAHKA@CL_ReadDemoMessage?3?5demoMsglen?5?$DO@ 004bdd84     cl_main.obj
 0002:00001db0       ??_C@_0BB@OONEJEGE@couldn?8t?5open?5?$CFs?$AA@ 004bddb0     cl_main.obj
 0002:00001dc4       ??_C@_0CF@NNMMABBB@Protocol?5?$CFd?5not?5supported?5for?5de@ 004bddc4     cl_main.obj
 0002:00001dec       ??_C@_08OPAGIOMF@demos?1?$CFs?$AA@ 004bddec     cl_main.obj
 0002:00001df8       ??_C@_0BF@LAJFIGGG@playdemo?5?$DMdemoname?$DO?6?$AA@ 004bddf8     cl_main.obj
 0002:00001e10       ??_C@_06EIKEHMLC@donedl?$AA@ 004bde10     cl_main.obj
 0002:00001e18       ??_C@_0P@LAKMDNN@Need?5paks?3?5?$CFs?6?$AA@ 004bde18     cl_main.obj
 0002:00001e28       ??_C@_0LE@HBLDLCIC@?6WARNING?3?5You?5are?5missing?5some?5f@ 004bde28     cl_main.obj
 0002:00001edc       ??_C@_0CI@KFHENOL@Unknown?5connectionless?5packet?5co@ 004bdedc     cl_main.obj
 0002:00001f04       ??_C@_0BD@BBKFKIHA@getserversResponse?$AA@ 004bdf04     cl_main.obj
 0002:00001f18       ??_C@_05IJDJACGD@print?$AA@ 004bdf18     cl_main.obj
 0002:00001f20       ??_C@_0N@KFCBIMP@keyAuthorize?$AA@ 004bdf20     cl_main.obj
 0002:00001f30       ??_C@_04OFDNEFMC@echo?$AA@ 004bdf30     cl_main.obj
 0002:00001f38       ??_C@_0P@DGEHCAPG@statusResponse?$AA@ 004bdf38     cl_main.obj
 0002:00001f48       ??_C@_0N@LMKIPMEE@infoResponse?$AA@ 004bdf48     cl_main.obj
 0002:00001f58       ??_C@_0BI@OHPKCELG@?$CFs?5should?5have?5been?5?$CFs?6?$AA@ 004bdf58     cl_main.obj
 0002:00001f70       ??_C@_0DF@MNDPKCCL@connectResponse?5from?5a?5different@ 004bdf70     cl_main.obj
 0002:00001fa8       ??_C@_0DI@LOEOILK@connectResponse?5packet?5while?5not@ 004bdfa8     cl_main.obj
 0002:00001fe0       ??_C@_0CB@DAMFFBNO@Dup?5connect?5received?4?5?5Ignored?4?6@ 004bdfe0     cl_main.obj
 0002:00002004       ??_C@_0BA@LMOGOADK@connectResponse?$AA@ 004be004     cl_main.obj
 0002:00002014       ??_C@_0BH@HJNMAMEA@challengeResponse?3?5?$CFd?6?$AA@ 004be014     cl_main.obj
 0002:0000202c       ??_C@_0DB@NPIBIHLP@Unwanted?5challenge?5response?5rece@ 004be02c     cl_main.obj
 0002:00002060       ??_C@_0BC@DGKDGAMO@challengeResponse?$AA@ 004be060     cl_main.obj
 0002:00002074       ??_C@_0BC@IFKLHAPC@CL?5packet?5?$CFs?3?5?$CFs?6?$AA@ 004be074     cl_main.obj
 0002:00002088       ??_C@_0CI@KKHCEKLL@?$CFs?3sequenced?5packet?5without?5conn@ 004be088     cl_main.obj
 0002:000020b0       ??_C@_0BB@JCENNPDP@?$CFs?3?5Runt?5packet?6?$AA@ 004be0b0     cl_main.obj
 0002:000020c4       ??_C@_0CM@KNFCNAPG@?9?9?9?9?9?5Client?5Initialization?5Comp@ 004be0c4     cl_main.obj
 0002:000020f0       ??_C@_0BC@GPOKHKHA@fs_referencedList?$AA@ 004be0f0     cl_main.obj
 0002:00002104       ??_C@_0O@HJFIEPKA@fs_openedList?$AA@ 004be104     cl_main.obj
 0002:00002114       ??_C@_09MCGBPECP@reconnect?$AA@ 004be114     cl_main.obj
 0002:00002120       ??_C@_0L@FEIAOOGN@clientinfo?$AA@ 004be120     cl_main.obj
 0002:0000212c       ??_C@_0M@NABCNGBA@cg_viewsize?$AA@ 004be12c     cl_main.obj
 0002:00002138       ??_C@_0BA@PKAEEJJB@cg_predictItems?$AA@ 004be138     cl_main.obj
 0002:00002148       ??_C@_08NLHBPEGP@password?$AA@ 004be148     cl_main.obj
 0002:00002154       ??_C@_03OMLNFKE@sex?$AA@   004be154     cl_main.obj
 0002:00002158       ??_C@_04ICKCIGNO@male?$AA@ 004be158     cl_main.obj
 0002:00002160       ??_C@_08OKGPDOIO@teamtask?$AA@ 004be160     cl_main.obj
 0002:0000216c       ??_C@_08HBHLIHAM@handicap?$AA@ 004be16c     cl_main.obj
 0002:00002178       ??_C@_03GNABGMEE@100?$AA@  004be178     cl_main.obj
 0002:0000217c       ??_C@_06KEONFOCA@color2?$AA@ 004be17c     cl_main.obj
 0002:00002184       ??_C@_06IPMAANOD@color1?$AA@ 004be184     cl_main.obj
 0002:0000218c       ??_C@_01FAMBOPH@4?$AA@     004be18c     cl_main.obj
 0002:00002190       ??_C@_0L@OOBNLHBJ@g_blueTeam?$AA@ 004be190     cl_main.obj
 0002:0000219c       ??_C@_06GMDNOCON@Pagans?$AA@ 004be19c     cl_main.obj
 0002:000021a4       ??_C@_09HOBGGEAD@g_redTeam?$AA@ 004be1a4     cl_main.obj
 0002:000021b0       ??_C@_07OLKAFEPH@Stroggs?$AA@ 004be1b0     cl_main.obj
 0002:000021b8       ??_C@_0P@JMIBMNM@team_headmodel?$AA@ 004be1b8     cl_main.obj
 0002:000021c8       ??_C@_06IHCBDILC@?$CKjames?$AA@ 004be1c8     cl_main.obj
 0002:000021d0       ??_C@_0L@KEDOKIKJ@team_model?$AA@ 004be1d0     cl_main.obj
 0002:000021dc       ??_C@_05MAECCALN@james?$AA@ 004be1dc     cl_main.obj
 0002:000021e4       ??_C@_05PDPNFFJO@sarge?$AA@ 004be1e4     cl_main.obj
 0002:000021ec       ??_C@_05DGPADKBM@snaps?$AA@ 004be1ec     cl_main.obj
 0002:000021f4       ??_C@_02PIBHCBOA@20?$AA@   004be1f4     cl_main.obj
 0002:000021f8       ??_C@_04HCCHHEEF@rate?$AA@ 004be1f8     cl_main.obj
 0002:00002200       ??_C@_04NEFKOBHG@3000?$AA@ 004be200     cl_main.obj
 0002:00002208       ??_C@_04MEMAJGDJ@name?$AA@ 004be208     cl_main.obj
 0002:00002210       ??_C@_0O@PCBPGDGA@UnnamedPlayer?$AA@ 004be210     cl_main.obj
 0002:00002220       ??_C@_03BAAJCDMO@800?$AA@  004be220     cl_main.obj
 0002:00002224       ??_C@_08BEMLPELN@m_filter?$AA@ 004be224     cl_main.obj
 0002:00002230       ??_C@_06NKCCGJAO@m_side?$AA@ 004be230     cl_main.obj
 0002:00002238       ??_C@_09CGJLBBDA@m_forward?$AA@ 004be238     cl_main.obj
 0002:00002244       ??_C@_04FNMPJLCB@0?425?$AA@ 004be244     cl_main.obj
 0002:0000224c       ??_C@_05HPEILLPC@m_yaw?$AA@ 004be24c     cl_main.obj
 0002:00002254       ??_C@_07JIEGLHEC@m_pitch?$AA@ 004be254     cl_main.obj
 0002:0000225c       ??_C@_05OACFFLK@0?4022?$AA@ 004be25c     cl_main.obj
 0002:00002264       ??_C@_0O@JKEEFDLF@cg_autoswitch?$AA@ 004be264     cl_main.obj
 0002:00002274       ??_C@_0BK@NLNALACG@cl_serverStatusResendTime?$AA@ 004be274     cl_main.obj
 0002:00002290       ??_C@_03EOKBPBHD@750?$AA@  004be290     cl_main.obj
 0002:00002294       ??_C@_0O@EPDAEHAE@r_inGameVideo?$AA@ 004be294     cl_main.obj
 0002:000022a4       ??_C@_0O@PJLPEGOC@cl_conXOffset?$AA@ 004be2a4     cl_main.obj
 0002:000022b4       ??_C@_0BB@MLOALJHK@cl_allowDownload?$AA@ 004be2b4     cl_main.obj
 0002:000022c8       ??_C@_0BB@JAAMCGDF@cl_showmouserate?$AA@ 004be2c8     cl_main.obj
 0002:000022dc       ??_C@_0M@HDIJIOFC@cl_freelook?$AA@ 004be2dc     cl_main.obj
 0002:000022e8       ??_C@_0O@EKMGNMKC@cl_mouseAccel?$AA@ 004be2e8     cl_main.obj
 0002:000022f8       ??_C@_0M@JFLMCFNC@sensitivity?$AA@ 004be2f8     cl_main.obj
 0002:00002304       ??_C@_06HFMKGFEH@cl_run?$AA@ 004be304     cl_main.obj
 0002:0000230c       ??_C@_02PJNFELNH@30?$AA@   004be30c     cl_main.obj
 0002:00002310       ??_C@_0BB@FCKNHEAF@cl_anglespeedkey?$AA@ 004be310     cl_main.obj
 0002:00002324       ??_C@_03GMOBGHL@1?45?$AA@  004be324     cl_main.obj
 0002:00002328       ??_C@_0O@KLONPPKB@cl_pitchspeed?$AA@ 004be328     cl_main.obj
 0002:00002338       ??_C@_0M@JHKIFKKF@cl_yawspeed?$AA@ 004be338     cl_main.obj
 0002:00002344       ??_C@_03GKAIMEJI@140?$AA@  004be344     cl_main.obj
 0002:00002348       ??_C@_0M@OFMEHMGC@rconAddress?$AA@ 004be348     cl_main.obj
 0002:00002354       ??_C@_0BA@HFABJKOC@cl_forceavidemo?$AA@ 004be354     cl_main.obj
 0002:00002364       ??_C@_0L@EFFMDGHC@cl_avidemo?$AA@ 004be364     cl_main.obj
 0002:00002370       ??_C@_08LGFIIHD@timedemo?$AA@ 004be370     cl_main.obj
 0002:0000237c       ??_C@_0N@DJJLAFOK@rconPassword?$AA@ 004be37c     cl_main.obj
 0002:0000238c       ??_C@_0O@NDLMCONH@cl_freezeDemo?$AA@ 004be38c     cl_main.obj
 0002:0000239c       ??_C@_0BB@FEJGPFPP@cl_showTimeDelta?$AA@ 004be39c     cl_main.obj
 0002:000023b0       ??_C@_0M@FIFNOBJK@cl_showSend?$AA@ 004be3b0     cl_main.obj
 0002:000023bc       ??_C@_0L@MNBOPENL@cl_shownet?$AA@ 004be3bc     cl_main.obj
 0002:000023c8       ??_C@_0N@PNJIOFAD@cl_timeNudge?$AA@ 004be3c8     cl_main.obj
 0002:000023d8       ??_C@_0L@JCNOFHIK@cl_timeout?$AA@ 004be3d8     cl_main.obj
 0002:000023e4       ??_C@_03HPLEMDKK@200?$AA@  004be3e4     cl_main.obj
 0002:000023e8       ??_C@_07CFPJCBPL@cl_motd?$AA@ 004be3e8     cl_main.obj
 0002:000023f0       ??_C@_0L@EEOFAGMJ@cl_noprint?$AA@ 004be3f0     cl_main.obj
 0002:000023fc       ??_C@_0CD@IPKBNFJ@?9?9?9?9?9?5Client?5Initialization?5?9?9?9?9@ 004be3fc     cl_main.obj
 0002:00002420       ??_C@_0N@NPHPNCMK@svc_snapshot?$AA@ 004be420     cl_parse.obj
 0002:00002430       ??_C@_0N@NJJNDAEC@svc_download?$AA@ 004be430     cl_parse.obj
 0002:00002440       ??_C@_0BC@MPNLMMMD@svc_serverCommand?$AA@ 004be440     cl_parse.obj
 0002:00002454       ??_C@_0N@BGKJKGIK@svc_baseline?$AA@ 004be454     cl_parse.obj
 0002:00002464       ??_C@_0BB@FCKFJGAJ@svc_configstring?$AA@ 004be464     cl_parse.obj
 0002:00002478       ??_C@_0O@LFJOIOEL@svc_gamestate?$AA@ 004be478     cl_parse.obj
 0002:00002488       ??_C@_07LENEADMB@svc_nop?$AA@ 004be488     cl_parse.obj
 0002:00002490       ??_C@_07NKDCEGCG@svc_bad?$AA@ 004be490     cl_parse.obj
 0002:00002498       ??_C@_07ENBOGMFB@?$CF3i?3?$CFs?6?$AA@ 004be498     cl_parse.obj
 0002:000024a0       ??_C@_0BE@HJHAKBFM@?$CF3i?3?5?5baseline?3?5?$CFi?6?$AA@ 004be4a0     cl_parse.obj
 0002:000024b4       ??_C@_0BB@PEEFLBGI@?$CF3i?3?5?5delta?3?5?$CFi?6?$AA@ 004be4b4     cl_parse.obj
 0002:000024c8       ??_C@_0BF@DMOLEINN@?$CF3i?3?5?5unchanged?3?5?$CFi?6?$AA@ 004be4c8     cl_parse.obj
 0002:000024e0       ??_C@_0CH@FIOHCEPK@CL_ParsePacketEntities?3?5end?5of?5m@ 004be4e0     cl_parse.obj
 0002:00002508       ??_C@_0CD@OFCDBLEN@?5?5?5snapshot?3?$CFi?5?5delta?3?$CFi?5?5ping?3?$CF@ 004be508     cl_parse.obj
 0002:0000252c       ??_C@_0BA@HLANGOLO@packet?5entities?$AA@ 004be52c     cl_parse.obj
 0002:0000253c       ??_C@_0CB@DKGPPJCN@Delta?5parseEntitiesNum?5too?5old?4?6@ 004be53c     cl_parse.obj
 0002:00002560       ??_C@_0BG@KNOBNHLI@Delta?5frame?5too?5old?4?6?$AA@ 004be560     cl_parse.obj
 0002:00002578       ??_C@_0DF@IPHEMKHH@Delta?5from?5invalid?5frame?5?$CInot?5su@ 004be578     cl_parse.obj
 0002:000025b0       ??_C@_0M@DCHLDPOO@playerstate?$AA@ 004be5b0     cl_parse.obj
 0002:000025bc       ??_C@_07CAKOHKGL@sv_pure?$AA@ 004be5bc     cl_parse.obj
 0002:000025c4       ??_C@_07FMAMAFJE@fs_game?$AA@ 004be5c4     cl_parse.obj
 0002:000025cc       ??_C@_0BG@GLEJBOHO@sv_referencedPakNames?$AA@ 004be5cc     cl_parse.obj
 0002:000025e4       ??_C@_0BC@GMMNJNGA@sv_referencedPaks?$AA@ 004be5e4     cl_parse.obj
 0002:000025f8       ??_C@_0M@POGHGNMP@sv_pakNames?$AA@ 004be5f8     cl_parse.obj
 0002:00002604       ??_C@_07PALKJHIL@sv_paks?$AA@ 004be604     cl_parse.obj
 0002:0000260c       ??_C@_0M@KIKMJPNG@sv_serverid?$AA@ 004be60c     cl_parse.obj
 0002:00002618       ??_C@_0CE@PAKDFLME@CL_ParseGamestate?3?5bad?5command?5b@ 004be618     cl_parse.obj
 0002:0000263c       ??_C@_0CB@MJAKJKGN@Baseline?5number?5out?5of?5range?3?5?$CFi@ 004be63c     cl_parse.obj
 0002:00002660       ??_C@_09PCLPELCK@nextdl?5?$CFd?$AA@ 004be660     cl_parse.obj
 0002:0000266c       ??_C@_0BF@FEBHKNJL@Could?5not?5create?5?$CFs?6?$AA@ 004be66c     cl_parse.obj
 0002:00002684       ??_C@_06NJGLKCLH@stopdl?$AA@ 004be684     cl_parse.obj
 0002:0000268c       ??_C@_0DI@JKPJCOJB@Server?5sending?5download?0?5but?5no?5@ 004be68c     cl_parse.obj
 0002:000026c4       ??_C@_0CN@HEADJFOK@CL_ParseDownload?3?5Expected?5block@ 004be6c4     cl_parse.obj
 0002:000026f4       ??_C@_0P@OAODPOMK@END?5OF?5MESSAGE?$AA@ 004be6f4     cl_parse.obj
 0002:00002704       ??_C@_0DH@BBFPEAJH@CL_ParseServerMessage?3?5read?5past@ 004be704     cl_parse.obj
 0002:0000273c       ??_C@_0DB@FPIIIAAE@CL_ParseServerMessage?3?5Illegible@ 004be73c     cl_parse.obj
 0002:00002770       ??_C@_0BA@JPKIBJNA@?$CF3i?3BAD?5CMD?5?$CFi?6?$AA@ 004be770     cl_parse.obj
 0002:00002780       ??_C@_0BE@OPHJAJHM@?9?9?9?9?9?9?9?9?9?9?9?9?9?9?9?9?9?9?6?$AA@ 004be780     cl_parse.obj
 0002:00002798       __real@3f61111111111111    004be798     cl_scrn.obj
 0002:000027a0       __real@3f5999999999999a    004be7a0     cl_scrn.obj
 0002:000027a8       __real@3d800000            004be7a8     cl_scrn.obj
 0002:000027b0       __real@3fb0000000000000    004be7b0     cl_scrn.obj
 0002:000027b8       ??_C@_0BC@LNEGBKC@RECORDING?5?$CFs?3?5?$CFik?$AA@ 004be7b8     cl_scrn.obj
 0002:000027cc       ??_C@_0L@CFOJGOPC@graphshift?$AA@ 004be7cc     cl_scrn.obj
 0002:000027d8       ??_C@_0L@MJMDNBMK@graphscale?$AA@ 004be7d8     cl_scrn.obj
 0002:000027e4       ??_C@_0M@GMACCADH@graphheight?$AA@ 004be7e4     cl_scrn.obj
 0002:000027f0       ??_C@_02MLODCJFF@32?$AA@   004be7f0     cl_scrn.obj
 0002:000027f4       ??_C@_0L@HHCDLFPE@debuggraph?$AA@ 004be7f4     cl_scrn.obj
 0002:00002800       ??_C@_09GNNLMGGI@timegraph?$AA@ 004be800     cl_scrn.obj
 0002:0000280c       ??_C@_0CD@LIPOMDOG@SCR_DrawScreenField?3?5bad?5cls?4sta@ 004be80c     cl_scrn.obj
 0002:00002830       ??_C@_0BP@GMBCBCMM@draw?5screen?5without?5UI?5loaded?6?$AA@ 004be830     cl_scrn.obj
 0002:00002850       ??_C@_0CF@GEKBNHMI@SCR_UpdateScreen?3?5recursively?5ca@ 004be850     cl_scrn.obj
 0002:00002878       ??_C@_0BA@JEMDJBMB@servercache?4dat?$AA@ 004be878     cl_ui.obj
 0002:00002888       ??_C@_04HLBMEOMD@addr?$AA@ 004be888     cl_ui.obj
 0002:00002890       ??_C@_0BH@PNNHGENL@Bad?5UI?5system?5trap?3?5?$CFi?$AA@ 004be890     cl_ui.obj
 0002:000028a8       ??_C@_0BG@JBIBCIPI@UI_CIN_PlayCinematic?6?$AA@ 004be8a8     cl_ui.obj
 0002:000028c0       ??_C@_0CK@FNGBPDDH@User?5Interface?5is?5version?5?$CFd?0?5ex@ 004be8c0     cl_ui.obj
 0002:000028ec       ??_C@_0BH@ECPNONCF@VM_Create?5on?5UI?5failed?$AA@ 004be8ec     cl_ui.obj
 0002:00002904       ??_C@_02OGLLFMLI@ui?$AA@   004be904     cl_ui.obj
 0002:00002908       ??_C@_05IHIPGGNN@vm_ui?$AA@ 004be908     cl_ui.obj
 0002:00002910       ??_C@_0BE@ELELOBLD@Map?5with?5no?5shaders?$AA@ 004be910     cm_load.obj
 0002:00002924       ??_C@_0CC@IBCMNOCH@CMod_LoadShaders?3?5funny?5lump?5siz@ 004be924     cm_load.obj
 0002:00002948       ??_C@_0BH@CCEOEHI@MAX_SUBMODELS?5exceeded?$AA@ 004be948     cm_load.obj
 0002:00002960       ??_C@_0BD@MKELOBFD@Map?5with?5no?5models?$AA@ 004be960     cm_load.obj
 0002:00002974       ??_C@_0CE@MGJNCBPJ@CMod_LoadSubmodels?3?5funny?5lump?5s@ 004be974     cm_load.obj
 0002:00002998       ??_C@_0BB@GPGCHEBB@Map?5has?5no?5nodes?$AA@ 004be998     cm_load.obj
 0002:000029ac       ??_C@_0CA@CGOMLOLO@MOD_LoadBmodel?3?5funny?5lump?5size?$AA@ 004be9ac     cm_load.obj
 0002:000029cc       ??_C@_0CE@NNCDCDMG@CMod_LoadBrushes?3?5bad?5shaderNum?3@ 004be9cc     cm_load.obj
 0002:000029f0       ??_C@_0BC@EBABHCIG@Map?5with?5no?5leafs?$AA@ 004be9f0     cm_load.obj
 0002:00002a08       __real@3ff0000000000000    004bea08     cm_load.obj
 0002:00002a10       ??_C@_0BD@FKOGFNAN@Map?5with?5no?5planes?$AA@ 004bea10     cm_load.obj
 0002:00002a24       ??_C@_0CH@MJKOBAAK@CMod_LoadBrushSides?3?5bad?5shaderN@ 004bea24     cm_load.obj
 0002:00002a4c       ??_C@_0BL@GCIBIODK@ParseMesh?3?5MAX_PATCH_VERTS?$AA@ 004bea4c     cm_load.obj
 0002:00002a68       ??_C@_0CO@INDKCALG@CM_ClipHandleToModel?3?5bad?5handle@ 004bea68     cm_load.obj
 0002:00002a98       ??_C@_0CE@IDDBKAAE@CM_ClipHandleToModel?3?5bad?5handle@ 004bea98     cm_load.obj
 0002:00002abc       ??_C@_0BL@CFOECHKA@CM_InlineModel?3?5bad?5number?$AA@ 004beabc     cm_load.obj
 0002:00002ad8       ??_C@_0BL@NKFJNPCM@CM_LeafCluster?3?5bad?5number?$AA@ 004bead8     cm_load.obj
 0002:00002af4       ??_C@_0BI@LLPODCBJ@CM_LeafArea?3?5bad?5number?$AA@ 004beaf4     cm_load.obj
 0002:00002b0c       ??_C@_0DK@KJOJIHED@CM_LoadMap?3?5?$CFs?5has?5wrong?5version@ 004beb0c     cm_load.obj
 0002:00002b48       ??_C@_0BB@OEPBHON@Couldn?8t?5load?5?$CFs?$AA@ 004beb48     cm_load.obj
 0002:00002b5c       ??_C@_0BG@FOHJEOAK@CM_LoadMap?$CI?5?$CFs?0?5?$CFi?5?$CJ?6?$AA@ 004beb5c     cm_load.obj
 0002:00002b74       ??_C@_0BD@GHKOGBLC@cm_playerCurveClip?$AA@ 004beb74     cm_load.obj
 0002:00002b88       ??_C@_0M@DMJHPFDE@cm_noCurves?$AA@ 004beb88     cm_load.obj
 0002:00002b94       ??_C@_0L@GKMKNHLN@cm_noAreas?$AA@ 004beb94     cm_load.obj
 0002:00002ba0       ??_C@_0BG@KOPIJPGC@CM_LoadMap?3?5NULL?5name?$AA@ 004beba0     cm_load.obj
 0002:00002bb8       __real@3fb999999999999a    004bebb8     cm_patch.obj
 0002:00002bc0       __real@bfb999999999999a    004bebc0     cm_patch.obj
 0002:00002bc8       __real@3f947ae147ae147b    004bebc8     cm_patch.obj
 0002:00002bd0       __real@3f1a36e2eb1c432d    004bebd0     cm_patch.obj
 0002:00002bd8       __real@bf800000            004bebd8     cm_patch.obj
 0002:00002bdc       ??_C@_0BB@JNELFKGE@MAX_PATCH_PLANES?$AA@ 004bebdc     cm_patch.obj
 0002:00002bf0       ??_C@_0CE@NJNBHFJK@WARNING?3?5CM_GridPlane?5unresolvab@ 004bebf0     cm_patch.obj
 0002:00002c14       ??_C@_0DA@PCDKAIPH@WARNING?3?5CM_SetBorderInward?3?5mix@ 004bec14     cm_patch.obj
 0002:00002c44       ??_C@_0CC@BGGAAOHM@CM_SetBorderInward?3?5bad?5paramete@ 004bec44     cm_patch.obj
 0002:00002c68       __real@c77fff00            004bec68     cm_patch.obj
 0002:00002c6c       __real@477fff00            004bec6c     cm_patch.obj
 0002:00002c70       ??_C@_0CN@BPJNCPGM@WARNING?3?5CM_AddFacetBevels?4?4?4?5in@ 004bec70     cm_patch.obj
 0002:00002ca0       ??_C@_0CD@OEGHCJEG@WARNING?3?5bevel?5plane?5already?5use@ 004beca0     cm_patch.obj
 0002:00002cc4       ??_C@_0BI@JFDENLMJ@ERROR?3?5too?5many?5bevels?6?$AA@ 004becc4     cm_patch.obj
 0002:00002ce0       __real@3fc0000000000000    004bece0     cm_patch.obj
 0002:00002ce8       ??_C@_0BF@BAKLCMON@r_debugSurfaceUpdate?$AA@ 004bece8     cm_patch.obj
 0002:00002d00       ??_C@_0CH@BLOEEIKO@winding?5chopped?5away?5by?5border?5p@ 004bed00     cm_patch.obj
 0002:00002d28       ??_C@_0N@JBOPDDFG@cm_debugSize?$AA@ 004bed28     cm_patch.obj
 0002:00002d38       ??_C@_01FDFGLJHB@2?$AA@    004bed38     cm_patch.obj
 0002:00002d3c       ??_C@_0P@ENOIJBKF@r_debugSurface?$AA@ 004bed3c     cm_patch.obj
 0002:00002d4c       ??_C@_0BH@LLNEMILC@CM_EdgePlaneNum?3?5bad?5k?$AA@ 004bed4c     cm_patch.obj
 0002:00002d64       __real@40800000            004bed64     cm_patch.obj
 0002:00002d68       ??_C@_0L@BHDFOPIG@MAX_FACETS?$AA@ 004bed68     cm_patch.obj
 0002:00002d74       ??_C@_0DC@BHAKBNNN@CM_GeneratePatchFacets?3?5source?5i@ 004bed74     cm_patch.obj
 0002:00002da8       ??_C@_0EE@IBFPNDNH@CM_GeneratePatchFacets?3?5even?5siz@ 004beda8     cm_patch.obj
 0002:00002dec       ??_C@_0DF@ODLAAPCB@CM_GeneratePatchFacets?3?5bad?5para@ 004bedec     cm_patch.obj
 0002:00002e24       ??_C@_0BH@LNMPEGNH@?$CI?$CF5?41f?0?5?$CF5?41f?0?5?$CF5?41f?$CJ?6?$AA@ 004bee24     cm_polylib.obj
 0002:00002e3c       ??_C@_0CD@BOFJFDD@FreeWinding?3?5freed?5a?5freed?5windi@ 004bee3c     cm_polylib.obj
 0002:00002e60       __real@3feff7ced916872b    004bee60     cm_polylib.obj
 0002:00002e68       ??_C@_0CD@BHBKGNIF@BaseWindingForPlane?3?5no?5axis?5fou@ 004bee68     cm_polylib.obj
 0002:00002e8c       ??_C@_0CD@PEDPMDOJ@ClipWinding?3?5MAX_POINTS_ON_WINDI@ 004bee8c     cm_polylib.obj
 0002:00002eb0       ??_C@_0CG@OLJCNKCC@ClipWinding?3?5points?5exceeded?5est@ 004beeb0     cm_polylib.obj
 0002:00002ed8       __real@3dcccccd            004beed8     cm_polylib.obj
 0002:00002edc       __real@bdcccccd            004beedc     cm_polylib.obj
 0002:00002ee0       ??_C@_0BJ@OGJJAGOO@CheckWinding?3?5non?9convex?$AA@ 004beee0     cm_polylib.obj
 0002:00002efc       ??_C@_0BO@BKAOIPNM@CheckWinding?3?5degenerate?5edge?$AA@ 004beefc     cm_polylib.obj
 0002:00002f1c       ??_C@_0BO@IFHIHAOC@CheckWinding?3?5point?5off?5plane?$AA@ 004bef1c     cm_polylib.obj
 0002:00002f3c       ??_C@_0BL@MEPEMAFE@CheckFace?3?5BUGUS_RANGE?3?5?$CFf?$AA@ 004bef3c     cm_polylib.obj
 0002:00002f58       ??_C@_0BG@EFPIHBAE@CheckWinding?3?5?$CFf?5area?$AA@ 004bef58     cm_polylib.obj
 0002:00002f70       ??_C@_0BI@CIEPJPFG@CheckWinding?3?5?$CFi?5points?$AA@ 004bef70     cm_polylib.obj
 0002:00002f88       ??_C@_0BH@BFMDHBGF@FloodArea_r?3?5reflooded?$AA@ 004bef88     cm_test.obj
 0002:00002fa0       ??_C@_0DD@NONPJOAP@CM_AdjustAreaPortalState?3?5negati@ 004befa0     cm_test.obj
 0002:00002fd4       ??_C@_0CK@BFFNFBLN@CM_ChangeAreaPortalState?3?5bad?5ar@ 004befd4     cm_test.obj
 0002:00003000       ??_C@_0BE@NBHJNIOB@area?5?$DO?$DN?5cm?4numAreas?$AA@ 004bf000     cm_test.obj
 0002:00003014       __real@3fc00000            004bf014     cm_trace.obj
 0002:00003018       __real@3f000000            004bf018     cm_trace.obj
 0002:0000301c       __real@45000000            004bf01c     cm_trace.obj
 0002:00003020       ??_C@_0BI@JOMBKBLK@Cbuf_AddText?3?5overflow?6?$AA@ 004bf020     cmd.obj
 0002:00003038       ??_C@_0BM@KMPIOOIF@Cbuf_InsertText?5overflowed?6?$AA@ 004bf038     cmd.obj
 0002:00003054       ??_C@_0CE@BLDHFDBK@Cmd_AddCommand?3?5?$CFs?5already?5defin@ 004bf054     cmd.obj
 0002:00003078       ??_C@_0N@IIIOLKJI@?$CFi?5commands?6?$AA@ 004bf078     cmd.obj
 0002:00003088       ??_C@_0M@NJLDBOCK@execing?5?$CFs?6?$AA@ 004bf088     cmd.obj
 0002:00003094       ??_C@_0BC@EKILBLKK@couldn?8t?5exec?5?$CFs?6?$AA@ 004bf094     cmd.obj
 0002:000030a8       ??_C@_04IFJILJI@?4cfg?$AA@ 004bf0a8     cmd.obj
 0002:000030b0       ??_C@_0CJ@HNMBJIBF@exec?5?$DMfilename?$DO?5?3?5execute?5a?5scri@ 004bf0b0     cmd.obj
 0002:000030dc       ??_C@_0DC@EJOKMNAB@vstr?5?$DMvariablename?$DO?5?3?5execute?5a?5@ 004bf0dc     cmd.obj
 0002:00003110       ??_C@_03IKGEINEE@?$CFs?5?$AA@ 004bf110     cmd.obj
 0002:00003114       ??_C@_04PNOAOIAG@wait?$AA@ 004bf114     cmd.obj
 0002:0000311c       ??_C@_04HIDEMJAH@vstr?$AA@ 004bf11c     cmd.obj
 0002:00003124       ??_C@_04MGEIEJAD@exec?$AA@ 004bf124     cmd.obj
 0002:0000312c       ??_C@_07LKLFKPJJ@cmdlist?$AA@ 004bf12c     cmd.obj
 0002:00003134       ??_C@_0CA@HHKKPMIM@Cbuf_ExecuteText?3?5bad?5exec_when?$AA@ 004bf134     cmd.obj
 0002:00003154       ??_C@_0BG@HNINGLEK@logfile?5opened?5on?5?$CFs?6?$AA@ 004bf154     common.obj
 0002:0000316c       ??_C@_0N@HGNLKJGF@qconsole?4log?$AA@ 004bf16c     common.obj
 0002:0000317c       ??_C@_0N@GPGLOFGG@cvar_restart?$AA@ 004bf17c     common.obj
 0002:0000318c       ??_C@_04FAOFCKOL@safe?$AA@ 004bf18c     common.obj
 0002:00003194       ??_C@_03KCHOJKKI@set?$AA@  004bf194     common.obj
 0002:00003198       ??_C@_0BI@MAFPOHOH@?$CFd?5?$CFs?5memory?5overhead?$AN?6?$AA@ 004bf198     common.obj
 0002:000031b0       ??_C@_0BM@BAHOBDOG@?$CFd?5?$CFs?5memory?5in?5?$CFd?5blocks?$AN?6?$AA@ 004bf1b0     common.obj
 0002:000031cc       ??_C@_0CP@MANOLJKG@?$AN?6?$DN?$DN?$DN?$DN?$DN?$DN?$DN?$DN?$DN?$DN?$DN?$DN?$DN?$DN?$DN?$DN?$AN?6?$CFs?5log?$AN?6?$DN?$DN?$DN?$DN@ 004bf1cc     common.obj
 0002:000031fc       ??_C@_05GCKAPDAI@SMALL?$AA@ 004bf1fc     common.obj
 0002:00003204       ??_C@_04KLKHHPIG@MAIN?$AA@ 004bf204     common.obj
 0002:0000320c       ??_C@_0CI@OANEJCJB@?5?5?5?5?5?5?5?5?$CF8i?5bytes?5in?5small?5Zone?5@ 004bf20c     common.obj
 0002:00003234       ??_C@_0CE@NPDILPEO@?5?5?5?5?5?5?5?5?$CF8i?5bytes?5in?5dynamic?5oth@ 004bf234     common.obj
 0002:00003258       ??_C@_0CH@EOLLDOAN@?5?5?5?5?5?5?5?5?$CF8i?5bytes?5in?5dynamic?5ren@ 004bf258     common.obj
 0002:00003280       ??_C@_0CF@CNFAILNA@?5?5?5?5?5?5?5?5?$CF8i?5bytes?5in?5dynamic?5bot@ 004bf280     common.obj
 0002:000032a8       ??_C@_0BN@HAFIPPM@?$CF8i?5bytes?5in?5?$CFi?5zone?5blocks?6?$AA@ 004bf2a8     common.obj
 0002:000032c8       ??_C@_0BG@FENEFIEO@?$CF8i?5unused?5highwater?6?$AA@ 004bf2c8     common.obj
 0002:000032e0       ??_C@_0BH@CLOMEGOK@?$CF8i?5total?5hunk?5in?5use?6?$AA@ 004bf2e0     common.obj
 0002:000032f8       ??_C@_0BI@GFEBGNFI@?$CF8i?5high?5tempHighwater?6?$AA@ 004bf2f8     common.obj
 0002:00003310       ??_C@_0P@PNBADBH@?$CF8i?5high?5temp?6?$AA@ 004bf310     common.obj
 0002:00003320       ??_C@_0BE@HHMLFLFC@?$CF8i?5high?5permanent?6?$AA@ 004bf320     common.obj
 0002:00003334       ??_C@_0P@MGIBPNNM@?$CF8i?5high?5mark?6?$AA@ 004bf334     common.obj
 0002:00003344       ??_C@_0BH@FCECDNPG@?$CF8i?5low?5tempHighwater?6?$AA@ 004bf344     common.obj
 0002:0000335c       ??_C@_0O@IOIEGEPB@?$CF8i?5low?5temp?6?$AA@ 004bf35c     common.obj
 0002:0000336c       ??_C@_0BD@DOEBODMG@?$CF8i?5low?5permanent?6?$AA@ 004bf36c     common.obj
 0002:00003380       ??_C@_0O@EHNEJKDK@?$CF8i?5low?5mark?6?$AA@ 004bf380     common.obj
 0002:00003390       ??_C@_0BG@OCFDAFBB@?$CF8i?5bytes?5total?5zone?6?$AA@ 004bf390     common.obj
 0002:000033a8       ??_C@_0BG@IMIDAEKI@?$CF8i?5bytes?5total?5hunk?6?$AA@ 004bf3a8     common.obj
 0002:000033c0       ??_C@_0CE@BLFCFJMN@ERROR?3?5two?5consecutive?5free?5bloc@ 004bf3c0     common.obj
 0002:000033e4       ??_C@_0DB@INBMMEOG@ERROR?3?5next?5block?5doesn?8t?5have?5p@ 004bf3e4     common.obj
 0002:00003418       ??_C@_0DB@EJEJBDEF@ERROR?3?5block?5size?5does?5not?5touch@ 004bf418     common.obj
 0002:0000344c       ??_C@_0CB@IHMKPJJG@block?3?$CFp?5?5?5?5size?3?$CF7i?5?5?5?5tag?3?$CF3i?6@ 004bf44c     common.obj
 0002:00003470       ??_C@_0BB@PCMLDEB@?$CFd?5hunk?5blocks?$AN?6?$AA@ 004bf470     common.obj
 0002:00003484       ??_C@_0BB@OAKONLKG@?$CFd?5Hunk?5memory?$AN?6?$AA@ 004bf484     common.obj
 0002:00003498       ??_C@_0DB@BHMHHFJ@?$AN?6?$DN?$DN?$DN?$DN?$DN?$DN?$DN?$DN?$DN?$DN?$DN?$DN?$DN?$DN?$DN?$DN?$AN?6Hunk?5log?$AN?6?$DN?$DN@ 004bf498     common.obj
 0002:000034cc       ??_C@_0DH@MKFMPAEL@?$AN?6?$DN?$DN?$DN?$DN?$DN?$DN?$DN?$DN?$DN?$DN?$DN?$DN?$DN?$DN?$DN?$DN?$AN?6Hunk?5Small?5l@ 004bf4cc     common.obj
 0002:00003504       ??_C@_0BP@KPGLMOBC@Hunk_Clear?3?5reset?5the?5hunk?5ok?6?$AA@ 004bf504     common.obj
 0002:00003524       ??_C@_0BN@MJLDDPNI@Couldn?8t?5open?5journal?5files?6?$AA@ 004bf524     common.obj
 0002:00003544       ??_C@_0M@COLEEONP@com_journal?$AA@ 004bf544     common.obj
 0002:00003550       ??_C@_0BM@POMPJIOA@Replaying?5journaled?5events?6?$AA@ 004bf550     common.obj
 0002:0000356c       ??_C@_0BA@OJDELHBG@journaldata?4dat?$AA@ 004bf56c     common.obj
 0002:0000357c       ??_C@_0M@BEDDKMKF@journal?4dat?$AA@ 004bf57c     common.obj
 0002:00003588       ??_C@_0BD@MBEKCKFD@Journaling?5events?6?$AA@ 004bf588     common.obj
 0002:0000359c       ??_C@_07CFFBIKLI@journal?$AA@ 004bf59c     common.obj
 0002:000035a4       ??_C@_0BJ@GPNJLJPC@SV_PacketEvent?5time?3?5?$CFi?6?$AA@ 004bf5a4     common.obj
 0002:000035c0       ??_C@_0EM@CPHPFGMM@?1?1?5id?5Software?5and?5Activision?5wi@ 004bf5c0     common.obj
 0002:0000360c       ??_C@_0CG@ILMLHNJJ@?1?1?5Do?5not?5give?5this?5file?5to?5ANYO@ 004bf60c     common.obj
 0002:00003634       ??_C@_0CI@PFGDDHBG@?6?1?1?5generated?5by?5quake?0?5do?5not?5m@ 004bf634     common.obj
 0002:0000365c       ??_C@_0BE@JKCFDMJK@Couldn?8t?5write?5?$CFs?4?6?$AA@ 004bf65c     common.obj
 0002:00003670       ??_C@_08LAIDFEPP@?$CFs?1q3key?$AA@ 004bf670     common.obj
 0002:0000367c       ??_C@_0CG@FPKFBBME@?1?1?5generated?5by?5quake?0?5do?5not?5mo@ 004bf67c     common.obj
 0002:000036a4       ??_C@_06KOMAFLML@baseq3?$AA@ 004bf6a4     common.obj
 0002:000036ac       ??_C@_0N@KFPKBBOI@q3config?4cfg?$AA@ 004bf6ac     common.obj
 0002:000036bc       ??_C@_0N@FMLDMECN@Writing?5?$CFs?4?6?$AA@ 004bf6bc     common.obj
 0002:000036cc       ??_C@_0BP@JAAMJFGO@Usage?3?5writeconfig?5?$DMfilename?$DO?6?$AA@ 004bf6cc     common.obj
 0002:000036ec       ??_C@_0CD@IHBFIHBI@Hitch?5warning?3?5?$CFi?5msec?5frame?5tim@ 004bf6ec     common.obj
 0002:00003710       __real@c0490fdb            004bf710     common.obj
 0002:00003714       __real@40490fdb            004bf714     common.obj
 0002:00003718       ??_C@_07FBMPDAOB@?5?5?5?5?$CFs?6?$AA@ 004bf718     common.obj
 0002:00003720       ??_C@_0BE@FIJAKBIE@Server?5crashed?3?5?$CFs?6?$AA@ 004bf720     common.obj
 0002:00003734       ??_C@_0DF@NMNFBMEP@?$CK?$CK?$CK?$CK?$CK?$CK?$CK?$CK?$CK?$CK?$CK?$CK?$CK?$CK?$CK?$CK?$CK?$CK?$CK?$CK?6ERROR?3?5?$CFs?6?$CK@ 004bf734     common.obj
 0002:0000376c       ??_C@_0BK@MPNLHLAM@Server?5fatal?5crashed?3?5?$CFs?6?$AA@ 004bf76c     common.obj
 0002:00003788       ??_C@_0BH@PKJLOEHK@Server?5didn?8t?5have?5CD?6?$AA@ 004bf788     common.obj
 0002:000037a0       ??_C@_0BK@DDHCKPII@recursive?5error?5after?3?5?$CFs?$AA@ 004bf7a0     common.obj
 0002:000037bc       ??_C@_0P@JAPNKEH@MISSING?5VALUE?6?$AA@ 004bf7bc     common.obj
 0002:000037cc       ??_C@_0CE@FGOINGFL@Z_Free?3?5memory?5block?5wrote?5past?5@ 004bf7cc     common.obj
 0002:000037f0       ??_C@_0BO@KPDAKNIP@Z_Free?3?5freed?5a?5freed?5pointer?$AA@ 004bf7f0     common.obj
 0002:00003810       ??_C@_0CH@OJFIIOIA@Z_Free?3?5freed?5a?5pointer?5without?5@ 004bf810     common.obj
 0002:00003838       ??_C@_0BF@IBBHAAHI@Z_Free?3?5NULL?5pointer?$AA@ 004bf838     common.obj
 0002:00003850       ??_C@_0DM@CJFCFDMA@Z_Malloc?3?5failed?5on?5allocation?5o@ 004bf850     common.obj
 0002:0000388c       ??_C@_04GHJNJNPO@main?$AA@ 004bf88c     common.obj
 0002:00003894       ??_C@_05KJDGBEEG@small?$AA@ 004bf894     common.obj
 0002:0000389c       ??_C@_0CC@LIMDBBOP@Z_TagMalloc?3?5tried?5to?5use?5a?50?5ta@ 004bf89c     common.obj
 0002:000038c0       ??_C@_0CK@MHBJLLKL@Z_CheckHeap?3?5two?5consecutive?5fre@ 004bf8c0     common.obj
 0002:000038ec       ??_C@_0DH@DHOAKNHO@Z_CheckHeap?3?5next?5block?5doesn?8t?5@ 004bf8ec     common.obj
 0002:00003924       ??_C@_0DH@PDLFHKNN@Z_CheckHeap?3?5block?5size?5does?5not@ 004bf924     common.obj
 0002:0000395c       ??_C@_0BK@CDNNLLKC@Com_TouchMemory?3?5?$CFi?5msec?6?$AA@ 004bf95c     common.obj
 0002:00003978       ??_C@_0CO@GEDAJKNP@Small?5zone?5data?5failed?5to?5alloca@ 004bf978     common.obj
 0002:000039a8       __real@35800000            004bf9a8     common.obj
 0002:000039ac       ??_C@_0CF@OPBLBLPA@Zone?5data?5failed?5to?5allocate?5?$CFi?5@ 004bf9ac     common.obj
 0002:000039d4       ??_C@_0N@MAMMMEDK@com_zoneMegs?$AA@ 004bf9d4     common.obj
 0002:000039e4       ??_C@_02KMALDIDP@16?$AA@   004bf9e4     common.obj
 0002:000039e8       ??_C@_07FNDDLPMM@meminfo?$AA@ 004bf9e8     common.obj
 0002:000039f0       ??_C@_0CF@BDKJHKGO@Hunk?5data?5failed?5to?5allocate?5?$CFi?5@ 004bf9f0     common.obj
 0002:00003a18       ??_C@_0DB@DJODFHPN@Minimum?5com_hunkMegs?5is?5?$CFi?0?5allo@ 004bfa18     common.obj
 0002:00003a50       ??_C@_0EI@EOGOECDI@Minimum?5com_hunkMegs?5for?5a?5dedic@ 004bfa50     common.obj
 0002:00003a98       ??_C@_0N@JFILOCFO@com_hunkMegs?$AA@ 004bfa98     common.obj
 0002:00003aa8       ??_C@_02KLACJAOD@56?$AA@   004bfaa8     common.obj
 0002:00003aac       ??_C@_0DM@JGPFFDMA@Hunk?5initialization?5failed?4?5File@ 004bfaac     common.obj
 0002:00003ae8       ??_C@_0BI@DFDJEDO@Hunk_Alloc?5failed?5on?5?$CFi?$AA@ 004bfae8     common.obj
 0002:00003b00       ??_C@_0CP@BHLCFLCK@Hunk_Alloc?3?5Hunk?5memory?5system?5n@ 004bfb00     common.obj
 0002:00003b30       ??_C@_0CG@IDCIPPIH@Hunk_AllocateTempMemory?3?5failed?5@ 004bfb30     common.obj
 0002:00003b58       ??_C@_0CK@KPLCADKN@Hunk_FreeTempMemory?3?5not?5the?5fin@ 004bfb58     common.obj
 0002:00003b84       ??_C@_0BP@DFPHFPJG@Hunk_FreeTempMemory?3?5bad?5magic?$AA@ 004bfb84     common.obj
 0002:00003ba4       ??_C@_0BO@GBMLCFPO@Error?5writing?5to?5journal?5file?$AA@ 004bfba4     common.obj
 0002:00003bc4       ??_C@_0CA@BFODPKNC@Error?5reading?5from?5journal?5file?$AA@ 004bfbc4     common.obj
 0002:00003be4       ??_C@_0CB@OJGNBCMC@WARNING?3?5Com_PushEvent?5overflow?6@ 004bfbe4     common.obj
 0002:00003c08       ??_C@_0BE@PFFNONJO@Testing?5fatal?5error?$AA@ 004bfc08     common.obj
 0002:00003c1c       ??_C@_0BD@DDPCEAL@Testing?5drop?5error?$AA@ 004bfc1c     common.obj
 0002:00003c30       ??_C@_0BC@DJHDECHL@freeze?5?$DMseconds?$DO?6?$AA@ 004bfc30     common.obj
 0002:00003c44       ??_C@_0BB@FHAPCDKO@?5?5?5?5?5?5?5?5?5?5?5?5?5?5?5?5?$AA@ 004bfc44     common.obj
 0002:00003c58       ??_C@_0CI@HOGAMGJF@?9?9?9?5Common?5Initialization?5Comple@ 004bfc58     common.obj
 0002:00003c80       ??_C@_0BE@DIBMBDCC@cinematic?5intro?4RoQ?$AA@ 004bfc80     common.obj
 0002:00003c94       ??_C@_0BG@DLPIPEDG@cinematic?5idlogo?4RoQ?6?$AA@ 004bfc94     common.obj
 0002:00003cac       ??_C@_08EPEHIMMI@?$CFs?5?$CFs?5?$CFs?$AA@ 004bfcac     common.obj
 0002:00003cb8       ??_C@_0M@HMAJCOKO@writeconfig?$AA@ 004bfcb8     common.obj
 0002:00003cc4       ??_C@_0O@OGEFLAOE@changeVectors?$AA@ 004bfcc4     common.obj
 0002:00003cd4       ??_C@_04KNNLNNGO@quit?$AA@ 004bfcd4     common.obj
 0002:00003cdc       ??_C@_06NANJHIPM@freeze?$AA@ 004bfcdc     common.obj
 0002:00003ce4       ??_C@_05DLEGDHMH@crash?$AA@ 004bfce4     common.obj
 0002:00003cec       ??_C@_05KKCIMGE@error?$AA@ 004bfcec     common.obj
 0002:00003cf4       ??_C@_0BA@PBHFIIBP@com_introplayed?$AA@ 004bfcf4     common.obj
 0002:00003d04       ??_C@_0BA@MOHNLIKA@com_buildScript?$AA@ 004bfd04     common.obj
 0002:00003d14       ??_C@_0L@MPAGGMDN@sv_running?$AA@ 004bfd14     common.obj
 0002:00003d20       ??_C@_09CGEBDJFG@sv_paused?$AA@ 004bfd20     common.obj
 0002:00003d2c       ??_C@_0L@JMMMBHPM@com_speeds?$AA@ 004bfd2c     common.obj
 0002:00003d38       ??_C@_07OFMACKEH@viewlog?$AA@ 004bfd38     common.obj
 0002:00003d40       ??_C@_0M@FAMBDMMF@com_dropsim?$AA@ 004bfd40     common.obj
 0002:00003d4c       ??_C@_0O@LCCBKALF@com_showtrace?$AA@ 004bfd4c     common.obj
 0002:00003d5c       ??_C@_09BHOLEJHN@fixedtime?$AA@ 004bfd5c     common.obj
 0002:00003d68       ??_C@_09IIOBMIO@timescale?$AA@ 004bfd68     common.obj
 0002:00003d74       ??_C@_07HMINABEO@logfile?$AA@ 004bfd74     common.obj
 0002:00003d7c       ??_C@_09DKNLLEN@com_blood?$AA@ 004bfd7c     common.obj
 0002:00003d88       ??_C@_0L@PCENNGCA@com_maxfps?$AA@ 004bfd88     common.obj
 0002:00003d94       ??_C@_02IIPHFAHD@85?$AA@   004bfd94     common.obj
 0002:00003d98       ??_C@_09BJOAODLF@dedicated?$AA@ 004bfd98     common.obj
 0002:00003da4       ??_C@_0BD@PHEIHMPD@exec?5autoexec?4cfg?6?$AA@ 004bfda4     common.obj
 0002:00003db8       ??_C@_0BD@MLBAFJNC@exec?5q3config?4cfg?6?$AA@ 004bfdb8     common.obj
 0002:00003dcc       ??_C@_0BC@FDOILEKD@exec?5default?4cfg?6?$AA@ 004bfdcc     common.obj
 0002:00003de0       ??_C@_09DNECJBKD@developer?$AA@ 004bfde0     common.obj
 0002:00003dec       ??_C@_0BM@JMOBJEDO@Error?5during?5initialization?$AA@ 004bfdec     common.obj
 0002:00003e08       ??_C@_09GPBPOFIE@?$CFs?5?$CFs?5?$CFs?6?$AA@ 004bfe08     common.obj
 0002:00003e14       ??_C@_07CECGJJJI@win?9x86?$AA@ 004bfe14     common.obj
 0002:00003e1c       ??_C@_0M@BBDAHLGI@May?525?52008?$AA@ 004bfe1c     common.obj
 0002:00003e28       ??_C@_0CB@HFEJCBKA@Com_EventLoop?3?5bad?5event?5type?5?$CFi@ 004bfe28     common.obj
 0002:00003e4c       ??_C@_0CA@ENDIPNNF@Com_EventLoop?3?5oversize?5packet?6?$AA@ 004bfe4c     common.obj
 0002:00003e6c       ??_C@_0CC@HBLLGKBA@?$CF4i?5traces?5?5?$CI?$CFib?5?$CFip?$CJ?5?$CF4i?5points@ 004bfe6c     common.obj
 0002:00003e90       ??_C@_0DM@DEOKJHOL@frame?3?$CFi?5all?3?$CF3i?5sv?3?$CF3i?5ev?3?$CF3i?5c@ 004bfe90     common.obj
 0002:00003ecc       ??_C@_0DI@GOCCEMPD@Warning?3?5cvar?5?$CC?$CFs?$CC?5given?5initial@ 004bfecc     cvar.obj
 0002:00003f04       ??_C@_09OBPPEEI@MAX_CVARS?$AA@ 004bff04     cvar.obj
 0002:00003f10       ??_C@_07LGPHKPBC@BADNAME?$AA@ 004bff10     cvar.obj
 0002:00003f18       ??_C@_0BO@HIEMFHPL@invalid?5cvar?5name?5string?3?5?$CFs?6?$AA@ 004bff18     cvar.obj
 0002:00003f38       ??_C@_0BJ@EGPKCOBM@Cvar_Get?3?5NULL?5parameter?$AA@ 004bff38     cvar.obj
 0002:00003f54       ??_C@_0BI@NNDBDFOI@?$CFs?5is?5cheat?5protected?4?6?$AA@ 004bff54     cvar.obj
 0002:00003f6c       ??_C@_0CF@MMBKLCAG@?$CFs?5will?5be?5changed?5upon?5restarti@ 004bff6c     cvar.obj
 0002:00003f94       ??_C@_0BI@PGDNNHME@?$CFs?5is?5write?5protected?4?6?$AA@ 004bff94     cvar.obj
 0002:00003fac       ??_C@_0BC@PCJCNELF@?$CFs?5is?5read?5only?4?6?$AA@ 004bffac     cvar.obj
 0002:00003fc0       ??_C@_0BC@MNGANAJN@Cvar_Set2?3?5?$CFs?5?$CFs?6?$AA@ 004bffc0     cvar.obj
 0002:00003fd4       ??_C@_02NJPGOMH@?$CFf?$AA@ 004bffd4     cvar.obj
 0002:00003fd8       ??_C@_0P@OHLLLJFN@latched?3?5?$CC?$CFs?$CC?6?$AA@ 004bffd8     cvar.obj
 0002:00003fe8       ??_C@_0BP@BMGCKJHO@?$CC?$CFs?$CC?5is?3?$CC?$CFs?$FO7?$CC?5default?3?$CC?$CFs?$FO7?$CC?6?$AA@ 004bffe8     cvar.obj
 0002:00004008       ??_C@_0BK@FDJCCMFA@usage?3?5toggle?5?$DMvariable?$DO?6?$AA@ 004c0008     cvar.obj
 0002:00004024       ??_C@_0BP@JNHFCPJL@usage?3?5set?5?$DMvariable?$DO?5?$DMvalue?$DO?6?$AA@ 004c0024     cvar.obj
 0002:00004044       ??_C@_0CA@BBMGOBNI@usage?3?5setu?5?$DMvariable?$DO?5?$DMvalue?$DO?6?$AA@ 004c0044     cvar.obj
 0002:00004064       ??_C@_0CA@GDDHLLFI@usage?3?5sets?5?$DMvariable?$DO?5?$DMvalue?$DO?6?$AA@ 004c0064     cvar.obj
 0002:00004084       ??_C@_0CA@OEJADIJJ@usage?3?5seta?5?$DMvariable?$DO?5?$DMvalue?$DO?6?$AA@ 004c0084     cvar.obj
 0002:000040a4       ??_C@_0BJ@HCHIPOJA@usage?3?5reset?5?$DMvariable?$DO?6?$AA@ 004c00a4     cvar.obj
 0002:000040c0       ??_C@_0O@IMDAJAHE@seta?5?$CFs?5?$CC?$CFs?$CC?6?$AA@ 004c00c0     cvar.obj
 0002:000040d0       ??_C@_08JANFGNJF@cl_cdkey?$AA@ 004c00d0     cvar.obj
 0002:000040dc       ??_C@_0BB@ELMIENAI@?$CFi?5cvar?5indexes?6?$AA@ 004c00dc     cvar.obj
 0002:000040f0       ??_C@_0BB@CNBPFGFL@?6?$CFi?5total?5cvars?6?$AA@ 004c00f0     cvar.obj
 0002:00004104       ??_C@_09INMFINGF@?5?$CFs?5?$CC?$CFs?$CC?6?$AA@ 004c0104     cvar.obj
 0002:00004110       ??_C@_01GFHCPBMG@C?$AA@    004c0110     cvar.obj
 0002:00004114       ??_C@_01OCOKONAJ@L?$AA@    004c0114     cvar.obj
 0002:00004118       ??_C@_01FHEEJDEE@A?$AA@    004c0118     cvar.obj
 0002:0000411c       ??_C@_01JPJNBJEM@I?$AA@    004c011c     cvar.obj
 0002:00004120       ??_C@_01DGKLNCNG@R?$AA@    004c0120     cvar.obj
 0002:00004124       ??_C@_01HJOKEEBB@U?$AA@    004c0124     cvar.obj
 0002:00004128       ??_C@_01CPLAODJH@S?$AA@    004c0128     cvar.obj
 0002:0000412c       ??_C@_0DM@CADHDAHP@Cvar_Update?3?5src?5?$CFs?5length?5?$CFd?5ex@ 004c012c     cvar.obj
 0002:00004168       ??_C@_0CB@LCNMLEBG@Cvar_Update?3?5handle?5out?5of?5range@ 004c0168     cvar.obj
 0002:0000418c       ??_C@_08HKAEGNIC@cvarlist?$AA@ 004c018c     cvar.obj
 0002:00004198       ??_C@_05CFMALAOA@reset?$AA@ 004c0198     cvar.obj
 0002:000041a0       ??_C@_04KEEJAPKG@seta?$AA@ 004c01a0     cvar.obj
 0002:000041a8       ??_C@_04IKOHNIPD@setu?$AA@ 004c01a8     cvar.obj
 0002:000041b0       ??_C@_04NMLNHPHF@sets?$AA@ 004c01b0     cvar.obj
 0002:000041b8       ??_C@_06FHLCKAHH@toggle?$AA@ 004c01b8     cvar.obj
 0002:000041c0       ??_C@_0BM@PCLMEAKM@FS_HandleForFile?3?5none?5free?$AA@ 004c01c0     files.obj
 0002:000041dc       ??_C@_0BH@ENNDMPLD@FS_FileForHandle?3?5NULL?$AA@ 004c01dc     files.obj
 0002:000041f4       ??_C@_0CN@FJPHMIMA@FS_FileForHandle?3?5can?8t?5get?5FILE@ 004c01f4     files.obj
 0002:00004224       ??_C@_0CA@KPOIDJBD@FS_FileForHandle?3?5out?5of?5reange?$AA@ 004c0224     files.obj
 0002:00004244       ??_C@_04HDOCAJNK@?$CFs?$CFs?$AA@ 004c0244     files.obj
 0002:0000424c       ??_C@_06HALAHGDI@?1?$CFs?1?$CFs?$AA@ 004c024c     files.obj
 0002:00004254       ??_C@_0DA@OPJLIFHH@WARNING?3?5refusing?5to?5create?5rela@ 004c0254     files.obj
 0002:00004284       ??_C@_02MOLJINC@?3?3?$AA@  004c0284     files.obj
 0002:00004288       ??_C@_02DJGKEECL@?4?4?$AA@ 004c0288     files.obj
 0002:0000428c       ??_C@_0BI@CAOFAEDB@Ignoring?5journal?5files?6?$AA@ 004c028c     files.obj
 0002:000042a4       ??_C@_0BP@DCHMDBJP@Short?5write?5in?5FS_Copyfiles?$CI?$CJ?6?$AA@ 004c02a4     files.obj
 0002:000042c4       ??_C@_02GMLFBBN@wb?$AA@    004c02c4     files.obj
 0002:000042c8       ??_C@_0BO@PEGACBP@Short?5read?5in?5FS_Copyfiles?$CI?$CJ?6?$AA@ 004c02c8     files.obj
 0002:000042e8       ??_C@_02JDPG@rb?$AA@       004c02e8     files.obj
 0002:000042ec       ??_C@_0P@KGHBPCIF@copy?5?$CFs?5to?5?$CFs?6?$AA@ 004c02ec     files.obj
 0002:000042fc       ??_C@_0BA@MLCEENKL@writing?5to?3?5?$CFs?6?$AA@ 004c02fc     files.obj
 0002:0000430c       ??_C@_0BK@KMAALCKD@FS_SV_FOpenFileWrite?3?5?$CFs?6?$AA@ 004c030c     files.obj
 0002:00004328       ??_C@_0CN@OMHGMFID@Filesystem?5call?5made?5without?5ini@ 004c0328     files.obj
 0002:00004358       ??_C@_0CG@FLINNLBK@FS_SV_FOpenFileRead?5?$CIfs_cdpath?$CJ?5@ 004c0358     files.obj
 0002:00004380       ??_C@_0CH@DIDGHCFB@FS_SV_FOpenFileRead?5?$CIfs_basepath@ 004c0380     files.obj
 0002:000043a8       ??_C@_0CH@NKEDPAKN@FS_SV_FOpenFileRead?5?$CIfs_homepath@ 004c03a8     files.obj
 0002:000043d0       ??_C@_0BJ@HAKJFOOE@FS_SV_Rename?3?5?$CFs?5?9?9?$DO?5?$CFs?6?$AA@ 004c03d0     files.obj
 0002:000043ec       ??_C@_0BG@PNPFEECE@FS_Rename?3?5?$CFs?5?9?9?$DO?5?$CFs?6?$AA@ 004c03ec     files.obj
 0002:00004404       ??_C@_0BH@DHOJCMAJ@FS_FOpenFileWrite?3?5?$CFs?6?$AA@ 004c0404     files.obj
 0002:0000441c       ??_C@_02BOGAIONP@ab?$AA@   004c041c     files.obj
 0002:00004420       ??_C@_0BI@KJCGJHFP@FS_FOpenFileAppend?3?5?$CFs?6?$AA@ 004c0420     files.obj
 0002:00004438       ??_C@_0CJ@MGIOFJMI@FS_FOpenFileRead?3?5?$CFs?5?$CIfound?5in?5?8@ 004c0438     files.obj
 0002:00004464       __real@38000100            004c0464     files.obj
 0002:00004468       ??_C@_0CG@BBPIBMKO@FS_FOpenFileRead?3?5?$CFs?5?$CIfound?5in?5?8@ 004c0468     files.obj
 0002:00004490       ??_C@_0BD@NBMLGLPG@Couldn?8t?5reopen?5?$CFs?$AA@ 004c0490     files.obj
 0002:000044a4       ??_C@_06FIKIFLOA@pd?$CJlqh?$AA@ 004c04a4     files.obj
 0002:000044ac       ??_C@_09KOGMCLPC@?2?$GAZf?$FO?8jof?$AA@ 004c04ac     files.obj
 0002:000044b8       ??_C@_0L@PDOPIANI@dTZT?$GAX?$CBdi?$GA?$AA@ 004c04b8     files.obj
 0002:000044c4       ??_C@_06IPPMLGON@?4arena?$AA@ 004c04c4     files.obj
 0002:000044cc       ??_C@_04NONLJGOA@?4bot?$AA@ 004c04cc     files.obj
 0002:000044d4       ??_C@_0L@LOIHPJMG@levelshots?$AA@ 004c04d4     files.obj
 0002:000044e0       ??_C@_07GACINHDJ@?4config?$AA@ 004c04e0     files.obj
 0002:000044e8       ??_C@_04LCMACLFG@?4txt?$AA@ 004c04e8     files.obj
 0002:000044f0       ??_C@_07MAFDLGF@?4shader?$AA@ 004c04f0     files.obj
 0002:000044f8       ??_C@_04PBCOOEDG@?4dat?$AA@ 004c04f8     files.obj
 0002:00004500       ??_C@_05IDJGMGLA@?4game?$AA@ 004c0500     files.obj
 0002:00004508       ??_C@_05OMAOFEO@?4menu?$AA@ 004c0508     files.obj
 0002:00004510       ??_C@_0P@CJCGDCLK@Can?8t?5find?5?$CFs?6?$AA@ 004c0510     files.obj
 0002:00004520       ??_C@_05DEAEPJBI@q3key?$AA@ 004c0520     files.obj
 0002:00004528       ??_C@_06KDKPKJKM@?4dm_?$CFd?$AA@ 004c0528     files.obj
 0002:00004530       ??_C@_0DE@FPPDNFFA@FS_FOpenFileRead?3?5NULL?5?8filename@ 004c0530     files.obj
 0002:00004564       ??_C@_0BH@JBMACPMK@FS_Read?3?5?91?5bytes?5read?$AA@ 004c0564     files.obj
 0002:0000457c       ??_C@_0BM@KBJOLIDM@FS_Write?3?5?91?5bytes?5written?6?$AA@ 004c057c     files.obj
 0002:00004598       ??_C@_0BL@MHLILIO@FS_Write?3?50?5bytes?5written?6?$AA@ 004c0598     files.obj
 0002:000045b4       ??_C@_0BH@JLADNIGI@Bad?5origin?5in?5FS_Seek?6?$AA@ 004c05b4     files.obj
 0002:000045cc       ??_C@_0CE@PCHLGHBN@ZIP?5FILE?5FSEEK?5NOT?5YET?5IMPLEMENT@ 004c05cc     files.obj
 0002:000045f0       ??_C@_0BE@HILOFDOP@FS_FreeFile?$CI?5NULL?5?$CJ?$AA@ 004c05f0     files.obj
 0002:00004604       ??_C@_0BD@LDIONFIK@Failed?5to?5open?5?$CFs?6?$AA@ 004c0604     files.obj
 0002:00004618       ??_C@_0BN@HEBINHD@FS_WriteFile?3?5NULL?5parameter?$AA@ 004c0618     files.obj
 0002:00004638       ??_C@_04JMPKHIOK@?4pk3?$AA@ 004c0638     files.obj
 0002:00004640       ??_C@_0BB@NEJIHPJO@?1description?4txt?$AA@ 004c0640     files.obj
 0002:00004654       ??_C@_01LFCBOECM@?4?$AA@   004c0654     files.obj
 0002:00004658       ??_C@_0CE@GOHPFEGA@usage?3?5dir?5?$DMdirectory?$DO?5?$FLextensio@ 004c0658     files.obj
 0002:0000467c       ??_C@_0BB@DKKMKEBK@?9?9?9?9?9?9?9?9?9?9?9?9?9?9?9?6?$AA@ 004c067c     files.obj
 0002:00004690       ??_C@_0BE@MKJFMONH@Directory?5of?5?$CFs?5?$CFs?6?$AA@ 004c0690     files.obj
 0002:000046a4       ??_C@_0BB@EGMCJFKN@?$CFd?5files?5listed?6?$AA@ 004c06a4     files.obj
 0002:000046b8       ??_C@_0BK@BBJDOPOH@example?3?5fdir?5?$CKq3dm?$CK?4bsp?6?$AA@ 004c06b8     files.obj
 0002:000046d4       ??_C@_0BG@OINMOPNJ@usage?3?5fdir?5?$DMfilter?$DO?6?$AA@ 004c06d4     files.obj
 0002:000046ec       ??_C@_0P@HENFNMJG@handle?5?$CFi?3?5?$CFs?6?$AA@ 004c06ec     files.obj
 0002:000046fc       ??_C@_06KIFJAIP@?$CFs?1?$CFs?6?$AA@ 004c06fc     files.obj
 0002:00004704       ??_C@_0BG@CENCGGPF@?5?5?5?5on?5the?5pure?5list?6?$AA@ 004c0704     files.obj
 0002:0000471c       ??_C@_0BK@MCAEBIFK@?5?5?5?5not?5on?5the?5pure?5list?6?$AA@ 004c071c     files.obj
 0002:00004738       ??_C@_0P@GCFMIPGN@?$CFs?5?$CI?$CFi?5files?$CJ?6?$AA@ 004c0738     files.obj
 0002:00004748       ??_C@_0BG@HPKHMA@Current?5search?5path?3?6?$AA@ 004c0748     files.obj
 0002:00004760       ??_C@_0BJ@GCFEINHC@Usage?3?5touchFile?5?$DMfile?$DO?6?$AA@ 004c0760     files.obj
 0002:0000477c       ??_C@_08LGPKPKCN@?$CFs?1pak?$CFd?$AA@ 004c077c     files.obj
 0002:00004788       ??_C@_0CJ@MOAKOHNN@?5?$CIlocal?5file?5exists?5with?5wrong?5c@ 004c0788     files.obj
 0002:000047b4       ??_C@_0M@KGJNBCOJ@?$CFs?4?$CF08x?4pk3?$AA@ 004c07b4     files.obj
 0002:000047c0       ??_C@_06NHIHDJNN@?$CFs?4pk3?$AA@ 004c07c0     files.obj
 0002:000047c8       ??_C@_01EOFPKCAF@?$EA?$AA@ 004c07c8     files.obj
 0002:000047cc       ??_C@_0M@PLGKGDEK@missionpack?$AA@ 004c07cc     files.obj
 0002:000047d8       ??_C@_09BCJOAAGD@touchFile?$AA@ 004c07d8     files.obj
 0002:000047e4       ??_C@_04MBOEABIA@fdir?$AA@ 004c07e4     files.obj
 0002:000047ec       ??_C@_03DAPAKLGM@dir?$AA@  004c07ec     files.obj
 0002:000047f0       ??_C@_04LNEJFJGI@path?$AA@ 004c07f0     files.obj
 0002:000047f8       ??_C@_0BH@ENGIAIMF@?$CFd?5files?5in?5pk3?5files?6?$AA@ 004c07f8     files.obj
 0002:00004810       ??_C@_0BI@FLKKINBM@?9?9?9?9?9?9?9?9?9?9?9?9?9?9?9?9?9?9?9?9?9?9?6?$AA@ 004c0810     files.obj
 0002:00004828       ??_C@_0M@LECGGKKC@fs_homepath?$AA@ 004c0828     files.obj
 0002:00004834       ??_C@_0M@HHPKLILN@fs_basegame?$AA@ 004c0834     files.obj
 0002:00004840       ??_C@_0M@DGDBFJN@fs_basepath?$AA@ 004c0840     files.obj
 0002:0000484c       ??_C@_09CIALLHHK@fs_cdpath?$AA@ 004c084c     files.obj
 0002:00004858       ??_C@_0N@PLNEKBEI@fs_copyfiles?$AA@ 004c0858     files.obj
 0002:00004868       ??_C@_08OKNDMBHA@fs_debug?$AA@ 004c0868     files.obj
 0002:00004874       ??_C@_0BI@LBEJILEG@?9?9?9?9?9?5FS_Startup?5?9?9?9?9?9?6?$AA@ 004c0874     files.obj
 0002:0000488c       ??_C@_0BP@JOGJAID@FS?5search?5reorder?5is?5required?6?$AA@ 004c088c     files.obj
 0002:000048ac       ??_C@_0BN@HAHOMMJP@Connected?5to?5a?5pure?5server?4?6?$AA@ 004c08ac     files.obj
 0002:000048cc       ??_C@_0BI@PIKLIGCP@FSH_FOpenFile?3?5bad?5mode?$AA@ 004c08cc     files.obj
 0002:000048e4       ??_C@_0BN@IBAOHAGH@Writing?5?$CFs?5to?5journal?5file?4?6?$AA@ 004c08e4     files.obj
 0002:00004904       ??_C@_0CF@GJHFIHLC@Writing?5len?5for?5?$CFs?5to?5journal?5fi@ 004c0904     files.obj
 0002:0000492c       ??_C@_0CG@JNPHIOFB@Writing?5zero?5for?5?$CFs?5to?5journal?5f@ 004c092c     files.obj
 0002:00004954       ??_C@_0CB@MAKFKKPM@Read?5from?5journalDataFile?5failed@ 004c0954     files.obj
 0002:00004978       ??_C@_0BP@DLEFKJEB@Loading?5?$CFs?5from?5journal?5file?4?6?$AA@ 004c0978     files.obj
 0002:00004998       ??_C@_0BN@KJKCEPNA@FS_ReadFile?5with?5empty?5name?6?$AA@ 004c0998     files.obj
 0002:000049b8       ??_C@_08GEJGLEOK@$modlist?$AA@ 004c09b8     files.obj
 0002:000049c4       ??_C@_0BH@KPMEDBPE@Corrupted?5pak0?4pk3?3?5?$CFu?$AA@ 004c09c4     files.obj
 0002:000049dc       ??_C@_0CE@KPCDGPCC@?6Running?5in?5restricted?5demo?5mode@ 004c09dc     files.obj
 0002:00004a00       ??_C@_0BP@LCBBIFIA@Invalid?5product?5identification?$AA@ 004c0a00     files.obj
 0002:00004a20       ??_C@_0O@PPIKOBGI@productid?4txt?$AA@ 004c0a20     files.obj
 0002:00004a30       ??_C@_0BK@EGLLFLGB@Couldn?8t?5load?5default?4cfg?$AA@ 004c0a30     files.obj
 0002:00004a4c       ??_C@_0M@BAINMAIF@default?4cfg?$AA@ 004c0a4c     files.obj
 0002:00004a58       ??_C@_0BF@BLDAMEAN@Invalid?5game?5folder?6?$AA@ 004c0a58     files.obj
 0002:00004a70       ??_C@_0O@KIDPHDKB@fs_gamedirvar?$AA@ 004c0a70     files.obj
 0002:00004a80       ??_C@_0M@LANFJBCD@jumppad_ent?$AA@ 004c0a80     msg.obj
 0002:00004a8c       ??_C@_0BA@PEKHLKLH@grapplePoint?$FL2?$FN?$AA@ 004c0a8c     msg.obj
 0002:00004a9c       ??_C@_0BA@PGOBAEOO@grapplePoint?$FL1?$FN?$AA@ 004c0a9c     msg.obj
 0002:00004aac       ??_C@_0BA@PHCDGONJ@grapplePoint?$FL0?$FN?$AA@ 004c0aac     msg.obj
 0002:00004abc       ??_C@_0O@DMGGNGOM@viewangles?$FL2?$FN?$AA@ 004c0abc     msg.obj
 0002:00004acc       ??_C@_0O@FIJGMFDG@eventParms?$FL1?$FN?$AA@ 004c0acc     msg.obj
 0002:00004adc       ??_C@_0O@FJFEKPAB@eventParms?$FL0?$FN?$AA@ 004c0adc     msg.obj
 0002:00004aec       ??_C@_0L@OCHPBDAP@torsoTimer?$AA@ 004c0aec     msg.obj
 0002:00004af8       ??_C@_0BA@OFFIKLKI@delta_angles?$FL2?$FN?$AA@ 004c0af8     msg.obj
 0002:00004b08       ??_C@_0BA@OGNMHPMG@delta_angles?$FL0?$FN?$AA@ 004c0b08     msg.obj
 0002:00004b18       ??_C@_07HHCKHIKK@pm_type?$AA@ 004c0b18     msg.obj
 0002:00004b20       ??_C@_0M@JFNAGFPA@damageCount?$AA@ 004c0b20     msg.obj
 0002:00004b2c       ??_C@_0M@MJMBEJAO@damagePitch?$AA@ 004c0b2c     msg.obj
 0002:00004b38       ??_C@_09DCADJNIO@damageYaw?$AA@ 004c0b38     msg.obj
 0002:00004b44       ??_C@_0M@HOGACEIB@damageEvent?$AA@ 004c0b44     msg.obj
 0002:00004b50       ??_C@_0L@MAFIMFPM@viewheight?$AA@ 004c0b50     msg.obj
 0002:00004b5c       ??_C@_0BC@GBAGMPPC@externalEventParm?$AA@ 004c0b5c     msg.obj
 0002:00004b70       ??_C@_0BA@OHBOBFPB@delta_angles?$FL1?$FN?$AA@ 004c0b70     msg.obj
 0002:00004b80       ??_C@_05HJCMGBKF@speed?$AA@ 004c0b80     msg.obj
 0002:00004b88       ??_C@_07GFBFDLBM@gravity?$AA@ 004c0b88     msg.obj
 0002:00004b90       ??_C@_0O@NKKNBCBK@externalEvent?$AA@ 004c0b90     msg.obj
 0002:00004ba0       ??_C@_0M@KALDLEMN@weaponstate?$AA@ 004c0ba0     msg.obj
 0002:00004bac       ??_C@_08DPFJBFEN@pm_flags?$AA@ 004c0bac     msg.obj
 0002:00004bb8       ??_C@_09PDPBIKFA@events?$FL1?$FN?$AA@ 004c0bb8     msg.obj
 0002:00004bc4       ??_C@_09PCDDOAGH@events?$FL0?$FN?$AA@ 004c0bc4     msg.obj
 0002:00004bd0       ??_C@_0M@POONNNAA@movementDir?$AA@ 004c0bd0     msg.obj
 0002:00004bdc       ??_C@_0O@GLMOEBPG@eventSequence?$AA@ 004c0bdc     msg.obj
 0002:00004bec       ??_C@_07DDMNBPBG@pm_time?$AA@ 004c0bec     msg.obj
 0002:00004bf4       ??_C@_09FPJALGDE@legsTimer?$AA@ 004c0bf4     msg.obj
 0002:00004c00       ??_C@_0M@DGBCHEDG@velocity?$FL2?$FN?$AA@ 004c0c00     msg.obj
 0002:00004c0c       ??_C@_0L@PNPIGBF@weaponTime?$AA@ 004c0c0c     msg.obj
 0002:00004c18       ??_C@_0O@DPOCACIC@viewangles?$FL0?$FN?$AA@ 004c0c18     msg.obj
 0002:00004c28       ??_C@_0O@DOCAGILF@viewangles?$FL1?$FN?$AA@ 004c0c28     msg.obj
 0002:00004c38       ??_C@_0M@DEFEMKGP@velocity?$FL1?$FN?$AA@ 004c0c38     msg.obj
 0002:00004c44       ??_C@_0M@DFJGKAFI@velocity?$FL0?$FN?$AA@ 004c0c44     msg.obj
 0002:00004c50       ??_C@_08HDFLKCJP@bobCycle?$AA@ 004c0c50     msg.obj
 0002:00004c5c       ??_C@_0M@BGGKMAGH@commandTime?$AA@ 004c0c5c     msg.obj
 0002:00004c68       ??_C@_05MIJNFGED@frame?$AA@ 004c0c68     msg.obj
 0002:00004c70       ??_C@_0O@HPPKGIAK@constantLight?$AA@ 004c0c70     msg.obj
 0002:00004c80       ??_C@_0L@MOGFAHDO@angles2?$FL2?$FN?$AA@ 004c0c80     msg.obj
 0002:00004c8c       ??_C@_0L@MNOBNDFA@angles2?$FL0?$FN?$AA@ 004c0c8c     msg.obj
 0002:00004c98       ??_C@_09PCHELDHA@angles?$FL2?$FN?$AA@ 004c0c98     msg.obj
 0002:00004ca4       ??_C@_05CAIMHGND@time2?$AA@ 004c0ca4     msg.obj
 0002:00004cac       ??_C@_0BA@EFHFHEJM@apos?4trDelta?$FL2?$FN?$AA@ 004c0cac     msg.obj
 0002:00004cbc       ??_C@_0BA@EHDDMKMF@apos?4trDelta?$FL1?$FN?$AA@ 004c0cbc     msg.obj
 0002:00004ccc       ??_C@_0BA@EGPBKAPC@apos?4trDelta?$FL0?$FN?$AA@ 004c0ccc     msg.obj
 0002:00004cdc       ??_C@_0P@BICHHIIO@apos?4trBase?$FL2?$FN?$AA@ 004c0cdc     msg.obj
 0002:00004cec       ??_C@_0BA@DPBJMBAH@apos?4trDuration?$AA@ 004c0cec     msg.obj
 0002:00004cfc       ??_C@_0M@EBDENFGM@apos?4trTime?$AA@ 004c0cfc     msg.obj
 0002:00004d08       ??_C@_04CLCEDBPF@time?$AA@ 004c0d08     msg.obj
 0002:00004d10       ??_C@_09PBPAGHBO@angles?$FL0?$FN?$AA@ 004c0d10     msg.obj
 0002:00004d1c       ??_C@_0M@EDEPDPKE@modelindex2?$AA@ 004c0d1c     msg.obj
 0002:00004d28       ??_C@_0L@EOIHEPPC@origin2?$FL1?$FN?$AA@ 004c0d28     msg.obj
 0002:00004d34       ??_C@_0L@EPEFCFMF@origin2?$FL0?$FN?$AA@ 004c0d34     msg.obj
 0002:00004d40       ??_C@_0L@EMMBPBKL@origin2?$FL2?$FN?$AA@ 004c0d40     msg.obj
 0002:00004d4c       ??_C@_08HDLPHJFP@generic1?$AA@ 004c0d4c     msg.obj
 0002:00004d58       ??_C@_09DPJGNNNM@loopSound?$AA@ 004c0d58     msg.obj
 0002:00004d64       ??_C@_0BA@GEGLLMHD@otherEntityNum2?$AA@ 004c0d64     msg.obj
 0002:00004d74       ??_C@_0L@OOABJPOI@modelindex?$AA@ 004c0d74     msg.obj
 0002:00004d80       ??_C@_08BOHIELLL@powerups?$AA@ 004c0d80     msg.obj
 0002:00004d8c       ??_C@_05OPIONHBI@solid?$AA@ 004c0d8c     msg.obj
 0002:00004d94       ??_C@_09FOHGOHCG@origin?$FL2?$FN?$AA@ 004c0d94     msg.obj
 0002:00004da0       ??_C@_09FMDAFJHP@origin?$FL1?$FN?$AA@ 004c0da0     msg.obj
 0002:00004dac       ??_C@_09FNPCDDEI@origin?$FL0?$FN?$AA@ 004c0dac     msg.obj
 0002:00004db8       ??_C@_0M@FNDLCNA@apos?4trType?$AA@ 004c0db8     msg.obj
 0002:00004dc4       ??_C@_0P@JDFIJFKD@pos?4trDuration?$AA@ 004c0dc4     msg.obj
 0002:00004dd4       ??_C@_09PADCANCJ@angles?$FL1?$FN?$AA@ 004c0dd4     msg.obj
 0002:00004de0       ??_C@_09ENNGDKOC@clientNum?$AA@ 004c0de0     msg.obj
 0002:00004dec       ??_C@_06GEPNGEJI@weapon?$AA@ 004c0dec     msg.obj
 0002:00004df4       ??_C@_0P@MIMDOCJJ@otherEntityNum?$AA@ 004c0df4     msg.obj
 0002:00004e04       ??_C@_06PEMOFHAI@eFlags?$AA@ 004c0e04     msg.obj
 0002:00004e0c       ??_C@_0L@KGHGOFDE@pos?4trType?$AA@ 004c0e0c     msg.obj
 0002:00004e18       ??_C@_0BA@GCAPFJDJ@groundEntityNum?$AA@ 004c0e18     msg.obj
 0002:00004e28       ??_C@_08NBDCCOLG@legsAnim?$AA@ 004c0e28     msg.obj
 0002:00004e34       ??_C@_09EHJMMCCL@eventParm?$AA@ 004c0e34     msg.obj
 0002:00004e40       ??_C@_09IDGFAJEG@torsoAnim?$AA@ 004c0e40     msg.obj
 0002:00004e4c       ??_C@_05IBNLLBBK@eType?$AA@ 004c0e4c     msg.obj
 0002:00004e54       ??_C@_0L@MMCDLJGH@angles2?$FL1?$FN?$AA@ 004c0e54     msg.obj
 0002:00004e60       ??_C@_05GFHEIIDD@event?$AA@ 004c0e60     msg.obj
 0002:00004e68       ??_C@_0P@BLKDKMOA@apos?4trBase?$FL0?$FN?$AA@ 004c0e68     msg.obj
 0002:00004e78       ??_C@_0P@OJDECADI@pos?4trDelta?$FL2?$FN?$AA@ 004c0e78     msg.obj
 0002:00004e88       ??_C@_0P@BKGBMGNH@apos?4trBase?$FL1?$FN?$AA@ 004c0e88     msg.obj
 0002:00004e98       ??_C@_0O@OFIKJMKF@pos?4trBase?$FL2?$FN?$AA@ 004c0e98     msg.obj
 0002:00004ea8       ??_C@_0P@OLHCJOGB@pos?4trDelta?$FL1?$FN?$AA@ 004c0ea8     msg.obj
 0002:00004eb8       ??_C@_0P@OKLAPEFG@pos?4trDelta?$FL0?$FN?$AA@ 004c0eb8     msg.obj
 0002:00004ec8       ??_C@_0O@OHMMCCPM@pos?4trBase?$FL1?$FN?$AA@ 004c0ec8     msg.obj
 0002:00004ed8       ??_C@_0O@OGAOEIML@pos?4trBase?$FL0?$FN?$AA@ 004c0ed8     msg.obj
 0002:00004ee8       ??_C@_0L@OCJBICII@pos?4trTime?$AA@ 004c0ee8     msg.obj
 0002:00004ef4       ??_C@_0DB@CDCFBJOH@MSG_Copy?3?5can?8t?5copy?5into?5a?5smal@ 004c0ef4     msg.obj
 0002:00004f28       ??_C@_0BE@HBLHKMBF@can?8t?5read?5?$CFd?5bits?6?$AA@ 004c0f28     msg.obj
 0002:00004f3c       ??_C@_0BL@JPLBKHNB@MSG_WriteBits?3?5bad?5bits?5?$CFi?$AA@ 004c0f3c     msg.obj
 0002:00004f58       ??_C@_0CC@BCAHGEKN@MSG_WriteString?3?5MAX_STRING_CHAR@ 004c0f58     msg.obj
 0002:00004f7c       ??_C@_0CB@FEBBBOCP@MSG_WriteString?3?5BIG_INFO_STRING@ 004c0f7c     msg.obj
 0002:00004fa0       __real@3f360b61            004c0fa0     msg.obj
 0002:00004fa4       ??_C@_0M@JKPELGIL@?$CFd?5used?5?$CFd?6?$AA@ 004c0fa4     msg.obj
 0002:00004fb0       ??_C@_0CM@EJOMBCBE@MSG_WriteDeltaEntity?3?5Bad?5entity@ 004c0fb0     msg.obj
 0002:00004fdc       ??_C@_0M@ILPPMOAB@?5?$CI?$CFi?5bits?$CJ?6?$AA@ 004c0fdc     msg.obj
 0002:00004fe8       ??_C@_06NMFPGCPD@?$CFs?3?$CFi?5?$AA@ 004c0fe8     msg.obj
 0002:00004ff0       ??_C@_06NHADCFMO@?$CFs?3?$CFf?5?$AA@ 004c0ff0     msg.obj
 0002:00004ff8       ??_C@_0M@HKNCGALG@?$CF3i?3?5?$CD?$CF?93i?5?$AA@ 004c0ff8     msg.obj
 0002:00005004       ??_C@_0BD@NOLCAOLH@?$CF3i?3?5?$CD?$CF?93i?5remove?6?$AA@ 004c1004     msg.obj
 0002:00005018       ??_C@_0BM@MHCCEDBM@Bad?5delta?5entity?5number?3?5?$CFi?$AA@ 004c1018     msg.obj
 0002:00005034       ??_C@_0M@GJDAJLLB@PS_POWERUPS?$AA@ 004c1034     msg.obj
 0002:00005040       ??_C@_07CDFACGBI@PS_AMMO?$AA@ 004c1040     msg.obj
 0002:00005048       ??_C@_0O@GFKBHLEI@PS_PERSISTANT?$AA@ 004c1048     msg.obj
 0002:00005058       ??_C@_08PLJCGDKN@PS_STATS?$AA@ 004c1058     msg.obj
 0002:00005064       ??_C@_0BC@OLEJBHLP@?$CF3i?3?5playerstate?5?$AA@ 004c1064     msg.obj
 0002:00005078       ??_C@_06HJHJCKIO@server?$AA@ 004c1078     net_chan.obj
 0002:00005080       ??_C@_06DGDLPBAN@client?$AA@ 004c1080     net_chan.obj
 0002:00005088       ??_C@_08HJDPOCEL@showdrop?$AA@ 004c1088     net_chan.obj
 0002:00005094       ??_C@_0M@DDMGOMOJ@showpackets?$AA@ 004c1094     net_chan.obj
 0002:000050a0       ??_C@_0CG@BDGJLBKO@NET_CompareBaseAdr?3?5bad?5address?5@ 004c10a0     net_chan.obj
 0002:000050c8       ??_C@_0CO@DHMLBJGH@?$CF02x?$CF02x?$CF02x?$CF02x?4?$CF02x?$CF02x?$CF02x?$CF02@ 004c10c8     net_chan.obj
 0002:000050f8       ??_C@_0BA@OMBGEIBN@?$CFi?4?$CFi?4?$CFi?4?$CFi?3?$CFhu?$AA@ 004c10f8     net_chan.obj
 0002:00005108       ??_C@_03EHEMCPIE@bot?$AA@  004c1108     net_chan.obj
 0002:0000510c       ??_C@_08HAEGGJGF@loopback?$AA@ 004c110c     net_chan.obj
 0002:00005118       ??_C@_0CC@DHFIOJGP@NET_CompareAdr?3?5bad?5address?5type@ 004c1118     net_chan.obj
 0002:0000513c       ??_C@_0BB@NGJDDNAF@send?5packet?5?$CF4i?6?$AA@ 004c113c     net_chan.obj
 0002:00005150       ??_C@_01JLIPDDHJ@?3?$AA@   004c1150     net_chan.obj
 0002:00005154       ??_C@_0CD@LNBJCMMG@?$CFs?5send?5?$CF4i?5?3?5s?$DN?$CFi?5fragment?$DN?$CFi?0?$CF@ 004c1154     net_chan.obj
 0002:00005178       ??_C@_0BL@BFLOIGMD@?$CFs?5send?5?$CF4i?5?3?5s?$DN?$CFi?5ack?$DN?$CFi?6?$AA@ 004c1178     net_chan.obj
 0002:00005194       ??_C@_0BO@OIBNDEGJ@Netchan_Transmit?3?5length?5?$DN?5?$CFi?$AA@ 004c1194     net_chan.obj
 0002:000051b4       ??_C@_0BM@KGOPCCAH@?$CFs?3illegal?5fragment?5length?6?$AA@ 004c11b4     net_chan.obj
 0002:000051d0       ??_C@_0CF@FNEEAEAE@?$CFs?3fragmentLength?5?$CFi?5?$DO?5msg?9?$DOmaxs@ 004c11d0     net_chan.obj
 0002:000051f8       ??_C@_0BP@NNNGGON@?$CFs?3Dropped?5a?5message?5fragment?6?$AA@ 004c11f8     net_chan.obj
 0002:00005218       ??_C@_0BN@CDDCLPO@?$CFs?3Dropped?5?$CFi?5packets?5at?5?$CFi?6?$AA@ 004c1218     net_chan.obj
 0002:00005238       ??_C@_0CB@IKJIFCCO@?$CFs?3Out?5of?5order?5packet?5?$CFi?5at?5?$CFi?6@ 004c1238     net_chan.obj
 0002:0000525c       ??_C@_0BE@NEBCOCEH@?$CFs?5recv?5?$CF4i?5?3?5s?$DN?$CFi?6?$AA@ 004c125c     net_chan.obj
 0002:00005270       ??_C@_0CD@PJJBGHAI@?$CFs?5recv?5?$CF4i?5?3?5s?$DN?$CFi?5fragment?$DN?$CFi?0?$CF@ 004c1270     net_chan.obj
 0002:00005294       __real@37800000            004c1294     q_math.obj
 0002:00005298       __real@437f0000            004c1298     q_math.obj
 0002:0000529c       __real@43b40000            004c129c     q_math.obj
 0002:000052a0       __real@404ca5dc0d03cf25    004c12a0     q_math.obj
 0002:000052a8       __real@43870000            004c12a8     q_math.obj
 0002:000052ac       __real@c3340000            004c12ac     q_math.obj
 0002:000052b0       __real@43340000            004c12b0     q_math.obj
 0002:000052b8       __real@4066c16c16c16c17    004c12b8     q_math.obj
 0002:000052c0       __real@4076800000000000    004c12c0     q_math.obj
 0002:000052c8       __real@4066800000000000    004c12c8     q_math.obj
 0002:000052d0       __real@3c8efa35            004c12d0     q_math.obj
 0002:000052d4       __real@3bb60b61            004c12d4     q_math.obj
 0002:000052d8       ??_C@_0BI@KPLEBEJF@ERROR?3?5?$CFs?0?5line?5?$CFd?3?5?$CFs?6?$AA@ 004c12d8     q_shared.obj
 0002:000052f0       ??_C@_0BK@DJMKDJBL@WARNING?3?5?$CFs?0?5line?5?$CFd?3?5?$CFs?6?$AA@ 004c12f0     q_shared.obj
 0002:0000530c       ??_C@_0BJ@OLBOPICM@Q_strncpyz?3?5destsize?5?$DM?51?$AA@ 004c130c     q_shared.obj
 0002:00005328       ??_C@_0BF@BJHHBLMD@Q_strncpyz?3?5NULL?5src?$AA@ 004c1328     q_shared.obj
 0002:00005340       ??_C@_0BG@EKAPNPCH@Q_strncpyz?3?5NULL?5dest?$AA@ 004c1340     q_shared.obj
 0002:00005358       ??_C@_0BN@EFOOAHFL@Q_strcat?3?5already?5overflowed?$AA@ 004c1358     q_shared.obj
 0002:00005378       ??_C@_0CD@GIPJKOOD@Com_sprintf?3?5overflow?5of?5?$CFi?5in?5?$CF@ 004c1378     q_shared.obj
 0002:0000539c       ??_C@_0CC@GMEFDOKA@Com_sprintf?3?5overflowed?5bigbuffe@ 004c139c     q_shared.obj
 0002:000053c0       ??_C@_0CG@FLHABLN@Info_ValueForKey?3?5oversize?5infos@ 004c13c0     q_shared.obj
 0002:000053e8       ??_C@_0CE@HMPLGKDK@Info_RemoveKey?3?5oversize?5infostr@ 004c13e8     q_shared.obj
 0002:0000540c       ??_C@_0CI@CPIEPBLO@Info_RemoveKey_Big?3?5oversize?5inf@ 004c140c     q_shared.obj
 0002:00005434       ??_C@_0CD@JIDDAEOO@Can?8t?5use?5keys?5or?5values?5with?5a?5@ 004c1434     q_shared.obj
 0002:00005458       ??_C@_0CL@JCFAGLFD@Can?8t?5use?5keys?5or?5values?5with?5a?5@ 004c1458     q_shared.obj
 0002:00005484       ??_C@_0CD@MGFMEBLE@Can?8t?5use?5keys?5or?5values?5with?5a?5@ 004c1484     q_shared.obj
 0002:000054a8       ??_C@_0BN@CAOBGKLE@Info?5string?5length?5exceeded?6?$AA@ 004c14a8     q_shared.obj
 0002:000054c8       ??_C@_06NELKLDPM@?2?$CFs?2?$CFs?$AA@ 004c14c8     q_shared.obj
 0002:000054d0       ??_C@_0CJ@CEEBDGNA@Info_SetValueForKey?3?5oversize?5in@ 004c14d0     q_shared.obj
 0002:000054fc       ??_C@_0CB@EMDOOGBI@BIG?5Info?5string?5length?5exceeded?6@ 004c14fc     q_shared.obj
 0002:00005520       ??_C@_0BF@BFEJCABG@MatchToken?3?5?$CFs?5?$CB?$DN?5?$CFs?$AA@ 004c1520     q_shared.obj
 0002:00005538       ??_C@_01PKGAHCOL@?$CJ?$AA@ 004c1538     q_shared.obj
 0002:0000553c       ??_C@_01ODHLEDKK@?$CI?$AA@ 004c153c     q_shared.obj
 0002:00005540       ??_C@_0BF@PIJCDGGI@No?5background?5file?4?6?$AA@ 004c1540     snd_dma.obj
 0002:00005558       ??_C@_0BF@DBAKANBB@Background?5file?3?5?$CFs?6?$AA@ 004c1558     snd_dma.obj
 0002:00005570       ??_C@_0BB@DLHOOLMA@0x?$CFx?5dma?5buffer?6?$AA@ 004c1570     snd_dma.obj
 0002:00005584       ??_C@_0L@CLCJCFAJ@?$CF5d?5speed?6?$AA@ 004c1584     snd_dma.obj
 0002:00005590       ??_C@_0BG@FOGLIFDD@?$CF5d?5submission_chunk?6?$AA@ 004c1590     snd_dma.obj
 0002:000055a8       ??_C@_0BA@HGOIHECG@?$CF5d?5samplebits?6?$AA@ 004c15a8     snd_dma.obj
 0002:000055b8       ??_C@_0N@LFEODKMK@?$CF5d?5samples?6?$AA@ 004c15b8     snd_dma.obj
 0002:000055c8       ??_C@_0M@FDDHHICE@?$CF5d?5stereo?6?$AA@ 004c15c8     snd_dma.obj
 0002:000055d4       ??_C@_0BH@MEMPFHHG@sound?5system?5is?5muted?6?$AA@ 004c15d4     snd_dma.obj
 0002:000055ec       ??_C@_0BK@NEOOOKPB@sound?5system?5not?5started?6?$AA@ 004c15ec     snd_dma.obj
 0002:00005608       ??_C@_0BI@JEHEKKKP@?9?9?9?9?9?5Sound?5Info?5?9?9?9?9?9?6?$AA@ 004c1608     snd_dma.obj
 0002:00005620       ??_C@_0CA@PLLGIKIN@Channel?5memory?5manager?5started?6?$AA@ 004c1620     snd_dma.obj
 0002:00005640       ??_C@_09MPGJFHJB@soundinfo?$AA@ 004c1640     snd_dma.obj
 0002:0000564c       ??_C@_09CJIFEKFJ@soundlist?$AA@ 004c164c     snd_dma.obj
 0002:00005658       ??_C@_09MAAKNOCD@stopsound?$AA@ 004c1658     snd_dma.obj
 0002:00005664       ??_C@_05LLDJOKNO@music?$AA@ 004c1664     snd_dma.obj
 0002:0000566c       ??_C@_04GBHMDDO@play?$AA@  004c166c     snd_dma.obj
 0002:00005674       ??_C@_0BJ@ONEALDEO@S_FindName?3?5out?5of?5sfx_t?$AA@ 004c1674     snd_dma.obj
 0002:00005690       ??_C@_0BI@FNMGDFHG@Sound?5name?5too?5long?3?5?$CFs?$AA@ 004c1690     snd_dma.obj
 0002:000056a8       ??_C@_0BI@MBEBGPGI@S_FindName?3?5empty?5name?6?$AA@ 004c16a8     snd_dma.obj
 0002:000056c0       ??_C@_0BC@JMCPOJBP@S_FindName?3?5NULL?6?$AA@ 004c16c0     snd_dma.obj
 0002:000056d4       __real@3a51b717            004c16d4     snd_dma.obj
 0002:000056d8       __real@42a00000            004c16d8     snd_dma.obj
 0002:000056dc       ??_C@_02JCPHEAGH@?$FO3?$AA@ 004c16dc     snd_dma.obj
 0002:000056e0       ??_C@_0CG@MHCEPADK@S_StartSound?3?5handle?5?$CFi?5out?5of?5r@ 004c16e0     snd_dma.obj
 0002:00005708       ??_C@_0BA@EKACNJLN@dropping?5sound?6?$AA@ 004c1708     snd_dma.obj
 0002:00005718       ??_C@_08IOBNMEPB@?$CFi?5?3?5?$CFs?6?$AA@ 004c1718     snd_dma.obj
 0002:00005724       ??_C@_0BP@PLEMPNLH@S_StartSound?3?5bad?5entitynum?5?$CFi?$AA@ 004c1724     snd_dma.obj
 0002:00005744       ??_C@_0CL@JCKKLMHG@S_StartLocalSound?3?5handle?5?$CFi?5out@ 004c1744     snd_dma.obj
 0002:00005770       ??_C@_0CL@NOGDPHFG@S_AddLoopingSound?3?5handle?5?$CFi?5out@ 004c1770     snd_dma.obj
 0002:0000579c       __real@42c80000            004c179c     snd_dma.obj
 0002:000057a0       __real@0000000000000000    004c17a0     snd_dma.obj
 0002:000057a8       ??_C@_0BA@JCBCPJHP@?$CFs?5has?5length?50?$AA@ 004c17a8     snd_dma.obj
 0002:000057b8       ??_C@_0CP@ECDOCLA@S_AddRealLoopingSound?3?5handle?5?$CFi@ 004c17b8     snd_dma.obj
 0002:000057e8       ??_C@_0CC@BJECBNFP@S_RawSamples?3?5overflowed?5?$CFi?5?$DO?5?$CFi@ 004c17e8     snd_dma.obj
 0002:0000580c       ??_C@_0CK@EAFGMFOG@S_RawSamples?3?5resetting?5minimum?3@ 004c180c     snd_dma.obj
 0002:00005838       __real@43800000            004c1838     snd_dma.obj
 0002:0000583c       ??_C@_0CJ@FABAALOF@S_UpdateEntityPosition?3?5bad?5enti@ 004c183c     snd_dma.obj
 0002:00005868       ??_C@_0BE@FOMELIJC@Total?5resident?3?5?$CFi?6?$AA@ 004c1868     snd_dma.obj
 0002:0000587c       ??_C@_0BC@HICHNCDI@?$CF6i?$FL?$CFs?$FN?5?3?5?$CFs?$FL?$CFs?$FN?6?$AA@ 004c187c     snd_dma.obj
 0002:00005890       ??_C@_09BLPOEION@resident?5?$AA@ 004c1890     snd_dma.obj
 0002:0000589c       ??_C@_09IKAMNOEC@paged?5out?$AA@ 004c189c     snd_dma.obj
 0002:000058a8       ??_C@_05NFJCPBPK@daub4?$AA@ 004c18a8     snd_dma.obj
 0002:000058b0       ??_C@_05JDPOCLPK@mulaw?$AA@ 004c18b0     snd_dma.obj
 0002:000058b8       ??_C@_05BANKJDCB@adpcm?$AA@ 004c18b8     snd_dma.obj
 0002:000058c0       ??_C@_05DCAALEKH@16bit?$AA@ 004c18c0     snd_dma.obj
 0002:000058c8       ??_C@_0BF@OFMFCFOH@No?5data?5chunk?5in?5?$CFs?6?$AA@ 004c18c8     snd_dma.obj
 0002:000058e0       ??_C@_04PJOLNDGD@data?$AA@ 004c18e0     snd_dma.obj
 0002:000058e8       ??_C@_0CM@GEAHPJEC@?$FO3WARNING?3?5music?5file?5?$CFs?5is?5not?5@ 004c18e8     snd_dma.obj
 0002:00005914       ??_C@_0CE@GKPHMJFG@Not?5a?5microsoft?5PCM?5format?5wav?3?5@ 004c1914     snd_dma.obj
 0002:00005938       ??_C@_0BE@CADIOBKC@No?5fmt?5chunk?5in?5?$CFs?6?$AA@ 004c1938     snd_dma.obj
 0002:0000594c       ??_C@_04CAJPEBPP@fmt?5?$AA@ 004c194c     snd_dma.obj
 0002:00005954       ??_C@_0CI@BJIPAJDD@?$FO3WARNING?3?5couldn?8t?5open?5music?5f@ 004c1954     snd_dma.obj
 0002:0000597c       ??_C@_04IBLEHOMF@?4wav?$AA@ 004c197c     snd_dma.obj
 0002:00005984       ??_C@_0CC@NGKFCGIG@S_StartBackgroundTrack?$CI?5?$CFs?0?5?$CFs?5?$CJ@ 004c1984     snd_dma.obj
 0002:000059a8       ??_C@_0CF@BHKHLDOB@StreamedRead?5failure?5on?5music?5tr@ 004c19a8     snd_dma.obj
 0002:000059d0       __real@3e800000            004c19d0     snd_dma.obj
 0002:000059d4       ??_C@_0CF@BDGBFLDG@S_FreeOldestSound?3?5freeing?5sound@ 004c19d4     snd_dma.obj
 0002:000059fc       ??_C@_0CO@KFOCFNID@?$FO3WARNING?3?5could?5not?5find?5?$CFs?5?9?5u@ 004c19fc     snd_dma.obj
 0002:00005a2c       ??_C@_0BO@KNMPIDHG@Sound?5name?5exceeds?5MAX_QPATH?6?$AA@ 004c1a2c     snd_dma.obj
 0002:00005a50       __real@3f847ae147ae147b    004c1a50     snd_dma.obj
 0002:00005a58       __real@41300000            004c1a58     snd_dma.obj
 0002:00005a5c       ??_C@_06MKMJDPPC@?$CFs?4wav?$AA@ 004c1a5c     snd_dma.obj
 0002:00005a64       ??_C@_0BO@IEIFFKHL@music?5?$DMmusicfile?$DO?5?$FLloopfile?$FN?6?$AA@ 004c1a64     snd_dma.obj
 0002:00005a84       ??_C@_06HEFAAICK@s_stop?$AA@ 004c1a84     snd_dma.obj
 0002:00005a8c       ??_C@_06KDCPAFOD@s_info?$AA@ 004c1a8c     snd_dma.obj
 0002:00005a94       ??_C@_06EFMDBICL@s_list?$AA@ 004c1a94     snd_dma.obj
 0002:00005a9c       ??_C@_0CG@KGENGPKN@?9?9?9?9?9?9?9?9?9?9?9?9?9?9?9?9?9?9?9?9?9?9?9?9?9?9?9?9?9?9?9?9@ 004c1a9c     snd_dma.obj
 0002:00005ac4       ??_C@_0BD@FJHCPMAJ@not?5initializing?4?6?$AA@ 004c1ac4     snd_dma.obj
 0002:00005ad8       ??_C@_0M@NLIFPOIG@s_initsound?$AA@ 004c1ad8     snd_dma.obj
 0002:00005ae4       ??_C@_0M@GGPLEHOA@s_testsound?$AA@ 004c1ae4     snd_dma.obj
 0002:00005af0       ??_C@_06CBNOHGMK@s_show?$AA@ 004c1af0     snd_dma.obj
 0002:00005af8       ??_C@_0N@MILGKHMC@s_mixPreStep?$AA@ 004c1af8     snd_dma.obj
 0002:00005b08       ??_C@_04FOELEPEP@0?405?$AA@ 004c1b08     snd_dma.obj
 0002:00005b10       ??_C@_0L@CIDOAMPN@s_mixahead?$AA@ 004c1b10     snd_dma.obj
 0002:00005b1c       ??_C@_03PBDDOHNJ@0?42?$AA@ 004c1b1c     snd_dma.obj
 0002:00005b20       ??_C@_05GPLACMP@s_khz?$AA@ 004c1b20     snd_dma.obj
 0002:00005b28       ??_C@_02MKCBEDGC@22?$AA@   004c1b28     snd_dma.obj
 0002:00005b2c       ??_C@_09FFKKACPC@s_doppler?$AA@ 004c1b2c     snd_dma.obj
 0002:00005b38       ??_C@_0N@EPGANNDD@s_separation?$AA@ 004c1b38     snd_dma.obj
 0002:00005b48       ??_C@_03LOHCHBBO@0?45?$AA@ 004c1b48     snd_dma.obj
 0002:00005b4c       ??_C@_0O@DCFOJKGE@s_musicvolume?$AA@ 004c1b4c     snd_dma.obj
 0002:00005b5c       ??_C@_08HCGCKAMG@s_volume?$AA@ 004c1b5c     snd_dma.obj
 0002:00005b68       ??_C@_03LNMAPFD@0?48?$AA@  004c1b68     snd_dma.obj
 0002:00005b6c       ??_C@_0CH@FFLNOAMN@?6?9?9?9?9?9?9?9?5sound?5initialization?5?9?9@ 004c1b6c     snd_dma.obj
 0002:00005b94       ??_C@_0BH@PPLJNIIB@sound?1feedback?1hit?4wav?$AA@ 004c1b94     snd_dma.obj
 0002:00005bac       ??_C@_0BG@BFIOFFAA@not?5started?5or?5muted?6?$AA@ 004c1bac     snd_dma.obj
 0002:00005bc4       ??_C@_0BK@LAAFJK@?9?9?9?9?$CI?$CFi?$CJ?9?9?9?9?5painted?3?5?$CFi?6?$AA@ 004c1bc4     snd_dma.obj
 0002:00005be0       ??_C@_09NKFDHBJC@?$CFf?5?$CFf?5?$CFs?6?$AA@ 004c1be0     snd_dma.obj
 0002:00005bec       ??_C@_0BO@JLIKIDHN@Sound?5memory?5manager?5started?6?$AA@ 004c1bec     snd_mem.obj
 0002:00005c0c       ??_C@_0O@HNCJJOBC@com_soundMegs?$AA@ 004c1c0c     snd_mem.obj
 0002:00005c1c       ??_C@_01KJLJFBPL@8?$AA@    004c1c1c     snd_mem.obj
 0002:00005c20       ??_C@_0BK@HIFIFFLN@Missing?5RIFF?1WAVE?5chunks?6?$AA@ 004c1c20     snd_mem.obj
 0002:00005c3c       ??_C@_0BE@DOAIJNHB@Missing?5data?5chunk?6?$AA@ 004c1c3c     snd_mem.obj
 0002:00005c50       ??_C@_0BL@LLPLMHJH@Microsoft?5PCM?5format?5only?6?$AA@ 004c1c50     snd_mem.obj
 0002:00005c6c       ??_C@_0BD@FLDJFMEC@Missing?5fmt?5chunk?6?$AA@ 004c1c6c     snd_mem.obj
 0002:00005c80       ??_C@_04HFHJMNCD@WAVE?$AA@ 004c1c80     snd_mem.obj
 0002:00005c88       ??_C@_04EPCGJKAP@RIFF?$AA@ 004c1c88     snd_mem.obj
 0002:00005c90       ??_C@_0CH@DLPNPMAK@?$FO3WARNING?3?5?$CFs?5is?5not?5a?522kHz?5wav@ 004c1c90     snd_mem.obj
 0002:00005cb8       ??_C@_0CD@BHGEJMMG@?$FO3WARNING?3?5?$CFs?5is?5a?58?5bit?5wav?5fil@ 004c1cb8     snd_mem.obj
 0002:00005cdc       ??_C@_0BJ@LNMLELKA@?$CFs?5is?5a?5stereo?5wav?5file?6?$AA@ 004c1cdc     snd_mem.obj
 0002:00005cf8       ??_C@_0DC@PNBPCCNC@?$CFd?5bytes?5free?5sound?5buffer?5memor@ 004c1cf8     snd_mem.obj
 0002:00005d30       __real@4153880000000000    004c1d30     snd_mix.obj
 0002:00005d38       __real@44800000            004c1d38     snd_mix.obj
 0002:00005d40       __real@3fdee8dd4748bf14    004c1d40     snd_wavelet.obj
 0002:00005d48       __real@3feac4bdd6e3fd71    004c1d48     snd_wavelet.obj
 0002:00005d50       __real@3fc0907dc1930691    004c1d50     snd_wavelet.obj
 0002:00005d58       __real@3fccb0bf0b6b7109    004c1d58     snd_wavelet.obj
 0002:00005d60       __real@c7000000            004c1d60     snd_wavelet.obj
 0002:00005d64       __real@46fffe00            004c1d64     snd_wavelet.obj
 0002:00005d68       ??_C@_0CE@GNNEKHHF@SV_BotFreeClient?3?5bad?5clientNum?3@ 004c1d68     sv_bot.obj
 0002:00005d8c       ??_C@_0BC@KEMOOJ@bot_highlightarea?$AA@ 004c1d8c     sv_bot.obj
 0002:00005da0       ??_C@_0P@PHABANOG@bot_groundonly?$AA@ 004c1da0     sv_bot.obj
 0002:00005db0       ??_C@_0BB@GFMPGHPP@bot_reachability?$AA@ 004c1db0     sv_bot.obj
 0002:00005dc4       ??_C@_09JMCENGKH@bot_debug?$AA@ 004c1dc4     sv_bot.obj
 0002:00005dd0       ??_C@_0BE@HKMNOMAG@unknown?5print?5type?6?$AA@ 004c1dd0     sv_bot.obj
 0002:00005de4       ??_C@_0L@CNJLHKJM@?$FO1Exit?3?5?$CFs?$AA@ 004c1de4     sv_bot.obj
 0002:00005df0       ??_C@_0M@GLOCHAGD@?$FO1Fatal?3?5?$CFs?$AA@ 004c1df0     sv_bot.obj
 0002:00005dfc       ??_C@_0M@LKBEKEOF@?$FO1Error?3?5?$CFs?$AA@ 004c1dfc     sv_bot.obj
 0002:00005e08       ??_C@_0O@LHCIHOMB@?$FO3Warning?3?5?$CFs?$AA@ 004c1e08     sv_bot.obj
 0002:00005e18       ??_C@_0DA@ONPNGPHE@SV_Bot_HunkAlloc?3?5Alloc?5with?5mar@ 004c1e18     sv_bot.obj
 0002:00005e48       __real@bfefae147ae147ae    004c1e48     sv_bot.obj
 0002:00005e50       __real@3fefae147ae147ae    004c1e50     sv_bot.obj
 0002:00005e58       ??_C@_0DC@ICCMFCJF@?$FO1Error?3?5SV_BotLibSetup?5without?5@ 004c1e58     sv_bot.obj
 0002:00005e8c       ??_C@_0BE@IDNEOHBL@bot_interbreedwrite?$AA@ 004c1e8c     sv_bot.obj
 0002:00005ea0       ??_C@_0BE@BBMLIECL@bot_interbreedcycle?$AA@ 004c1ea0     sv_bot.obj
 0002:00005eb4       ??_C@_0BD@GLHGHIJE@bot_interbreedbots?$AA@ 004c1eb4     sv_bot.obj
 0002:00005ec8       ??_C@_02PKFBJPLJ@10?$AA@   004c1ec8     sv_bot.obj
 0002:00005ecc       ??_C@_0BD@MIDHDJEH@bot_interbreedchar?$AA@ 004c1ecc     sv_bot.obj
 0002:00005ee0       ??_C@_0P@IGNPDGBD@bot_minplayers?$AA@ 004c1ee0     sv_bot.obj
 0002:00005ef0       ??_C@_0O@ILENLOKO@bot_challenge?$AA@ 004c1ef0     sv_bot.obj
 0002:00005f00       ??_C@_0P@OLNMGHML@bot_rocketjump?$AA@ 004c1f00     sv_bot.obj
 0002:00005f10       ??_C@_0M@HIPNFLBG@bot_grapple?$AA@ 004c1f10     sv_bot.obj
 0002:00005f1c       ??_C@_0L@DIBKBFBJ@bot_report?$AA@ 004c1f1c     sv_bot.obj
 0002:00005f28       ??_C@_09KJGEBPM@bot_pause?$AA@ 004c1f28     sv_bot.obj
 0002:00005f34       ??_C@_0L@JNAIAIAH@bot_nochat?$AA@ 004c1f34     sv_bot.obj
 0002:00005f40       ??_C@_0N@JOELMLFL@bot_fastchat?$AA@ 004c1f40     sv_bot.obj
 0002:00005f50       ??_C@_0BB@LICKAML@bot_testclusters?$AA@ 004c1f50     sv_bot.obj
 0002:00005f64       ??_C@_0O@NEGDFLLI@bot_testsolid?$AA@ 004c1f64     sv_bot.obj
 0002:00005f74       ??_C@_0O@BBHMLBKC@bot_testrchat?$AA@ 004c1f74     sv_bot.obj
 0002:00005f84       ??_C@_0O@HIGNEDPK@bot_testichat?$AA@ 004c1f84     sv_bot.obj
 0002:00005f94       ??_C@_0BF@BBFOCAKO@bot_reloadcharacters?$AA@ 004c1f94     sv_bot.obj
 0002:00005fac       ??_C@_0O@NKIABNEG@bot_thinktime?$AA@ 004c1fac     sv_bot.obj
 0002:00005fbc       ??_C@_0BF@MDEDPJEF@bot_saveroutingcache?$AA@ 004c1fbc     sv_bot.obj
 0002:00005fd4       ??_C@_0BA@CHMPBPHA@bot_aasoptimize?$AA@ 004c1fd4     sv_bot.obj
 0002:00005fe4       ??_C@_0P@HFCEKFCE@bot_forcewrite?$AA@ 004c1fe4     sv_bot.obj
 0002:00005ff4       ??_C@_0BG@GJKIOMNG@bot_forcereachability?$AA@ 004c1ff4     sv_bot.obj
 0002:0000600c       ??_C@_0BE@HANIKEON@bot_forceclustering?$AA@ 004c200c     sv_bot.obj
 0002:00006020       ??_C@_0BG@HILKKLKJ@bot_visualizejumppads?$AA@ 004c2020     sv_bot.obj
 0002:00006038       ??_C@_0BC@OFKLJGBH@bot_maxdebugpolys?$AA@ 004c2038     sv_bot.obj
 0002:0000604c       ??_C@_0O@IHEJFHJE@bot_developer?$AA@ 004c204c     sv_bot.obj
 0002:0000605c       ??_C@_0L@BKCPIMBP@bot_enable?$AA@ 004c205c     sv_bot.obj
 0002:00006068       ??_C@_0BF@NJDIPJLA@Game?5CD?5not?5in?5drive?$AA@ 004c2068     sv_bot.obj
 0002:00006080       ??_C@_0CA@COHLGPJ@Player?5?$CFs?5is?5not?5on?5the?5server?6?$AA@ 004c2080     sv_ccmds.obj
 0002:000060a0       ??_C@_0BG@FMLKELB@No?5player?5specified?4?6?$AA@ 004c20a0     sv_ccmds.obj
 0002:000060b8       ??_C@_0BF@BEBENGBA@Bad?5client?5slot?3?5?$CFi?6?$AA@ 004c20b8     sv_ccmds.obj
 0002:000060d0       ??_C@_0BF@GAKLMKPI@Bad?5slot?5number?3?5?$CFs?6?$AA@ 004c20d0     sv_ccmds.obj
 0002:000060e8       ??_C@_0BJ@PDNIBEAG@Client?5?$CFi?5is?5not?5active?6?$AA@ 004c20e8     sv_ccmds.obj
 0002:00006104       ??_C@_08ICLMJBJO@spdevmap?$AA@ 004c2104     sv_ccmds.obj
 0002:00006110       ??_C@_06JMKHDEMO@devmap?$AA@ 004c2110     sv_ccmds.obj
 0002:00006118       ??_C@_0L@LPENDGCI@g_doWarmup?$AA@ 004c2118     sv_ccmds.obj
 0002:00006124       ??_C@_02HJDGIJBC@sp?$AA@   004c2124     sv_ccmds.obj
 0002:00006128       ??_C@_0L@GFINLBEC@g_gametype?$AA@ 004c2128     sv_ccmds.obj
 0002:00006134       ??_C@_0BD@IOLJLANL@Can?8t?5find?5map?5?$CFs?6?$AA@ 004c2134     sv_ccmds.obj
 0002:00006148       ??_C@_0CA@KCGHPPMG@variable?5change?5?9?9?5restarting?4?6?$AA@ 004c2148     sv_ccmds.obj
 0002:00006168       ??_C@_0DC@HPLLIPAB@SV_MapRestart_f?$CI?$CFd?$CJ?3?5dropped?5cli@ 004c2168     sv_ccmds.obj
 0002:0000619c       ??_C@_0N@HLIAHCAN@map_restart?6?$AA@ 004c219c     sv_ccmds.obj
 0002:000061ac       ??_C@_0BI@BNNKLCPB@Server?5is?5not?5running?4?6?$AA@ 004c21ac     sv_ccmds.obj
 0002:000061c4       ??_C@_0L@GPCEIOHM@print?5?$CC?$CFs?$CC?$AA@ 004c21c4     sv_ccmds.obj
 0002:000061d0       ??_C@_0BJ@BPEGMFB@Cannot?5kick?5host?5player?6?$AA@ 004c21d0     sv_ccmds.obj
 0002:000061ec       ??_C@_07GCOBEAMC@allbots?$AA@ 004c21ec     sv_ccmds.obj
 0002:000061f4       ??_C@_0L@JGGOGHBB@was?5kicked?$AA@ 004c21f4     sv_ccmds.obj
 0002:00006200       ??_C@_03NFKEKGGK@all?$AA@  004c2200     sv_ccmds.obj
 0002:00006208       ??_C@_0FB@IAPOMDOC@Usage?3?5kick?5?$DMplayer?5name?$DO?6kick?5a@ 004c2208     sv_ccmds.obj
 0002:0000625c       ??_C@_0CA@IHMFJNLM@?$CFs?5was?5banned?5from?5coming?5back?6?$AA@ 004c225c     sv_ccmds.obj
 0002:0000627c       ??_C@_0BE@LNHBPGBP@banUser?5?$CFi?4?$CFi?4?$CFi?4?$CFi?$AA@ 004c227c     sv_ccmds.obj
 0002:00006290       ??_C@_0BO@JNCGGNFP@Usage?3?5banUser?5?$DMplayer?5name?$DO?6?$AA@ 004c2290     sv_ccmds.obj
 0002:000062b0       ??_C@_0CC@FHLBNCJE@Usage?3?5banClient?5?$DMclient?5number?$DO@ 004c22b0     sv_ccmds.obj
 0002:000062d4       ??_C@_0CA@OMEFHEIE@Usage?3?5kicknum?5?$DMclient?5number?$DO?6?$AA@ 004c22d4     sv_ccmds.obj
 0002:000062f4       ??_C@_04PJGPIPHP@?5?$CF5i?$AA@ 004c22f4     sv_ccmds.obj
 0002:000062fc       ??_C@_03NPMIIIHK@?$CF5i?$AA@ 004c22fc     sv_ccmds.obj
 0002:00006300       ??_C@_04IPICLMID@?$CF7i?5?$AA@ 004c2300     sv_ccmds.obj
 0002:00006308       ??_C@_02PGJLIFGD@?$FO7?$AA@ 004c2308     sv_ccmds.obj
 0002:0000630c       ??_C@_04JNDHBDGN@?$CF4i?5?$AA@ 004c230c     sv_ccmds.obj
 0002:00006314       ??_C@_05JIJJOLGO@ZMBI?5?$AA@ 004c2314     sv_ccmds.obj
 0002:0000631c       ??_C@_05FHKCJFKL@CNCT?5?$AA@ 004c231c     sv_ccmds.obj
 0002:00006324       ??_C@_04CFILHEAI@?$CF5i?5?$AA@ 004c2324     sv_ccmds.obj
 0002:0000632c       ??_C@_04OACLNE@?$CF3i?5?$AA@ 004c232c     sv_ccmds.obj
 0002:00006338       ??_C@_0EK@MBPBHBBK@?9?9?9?5?9?9?9?9?9?5?9?9?9?9?5?9?9?9?9?9?9?9?9?9?9?9?9?9?9?9?5?9@ 004c2338     sv_ccmds.obj
 0002:00006388       ??_C@_0EJ@JCNPBNOM@num?5score?5ping?5name?5?5?5?5?5?5?5?5?5?5?5?5l@ 004c2388     sv_ccmds.obj
 0002:000063d4       ??_C@_08BLGHJHOM@map?3?5?$CFs?6?$AA@ 004c23d4     sv_ccmds.obj
 0002:000063e0       ??_C@_0L@KDCLABHC@chat?5?$CC?$CFs?6?$CC?$AA@ 004c23e0     sv_ccmds.obj
 0002:000063ec       ??_C@_09KIHOHKKG@console?3?5?$AA@ 004c23ec     sv_ccmds.obj
 0002:000063f8       ??_C@_0BH@LAHBCPJF@Server?5info?5settings?3?6?$AA@ 004c23f8     sv_ccmds.obj
 0002:00006410       ??_C@_0BH@HBKMNNLG@System?5info?5settings?3?6?$AA@ 004c2410     sv_ccmds.obj
 0002:00006428       ??_C@_09DDAOCEB@?9?9?9?9?9?9?9?9?6?$AA@ 004c2428     sv_ccmds.obj
 0002:00006434       ??_C@_09IIBHBCGO@userinfo?6?$AA@ 004c2434     sv_ccmds.obj
 0002:00006440       ??_C@_0BG@NIEOENOA@Usage?3?5info?5?$DMuserid?$DO?6?$AA@ 004c2440     sv_ccmds.obj
 0002:00006458       ??_C@_0L@OMIGLNJO@killserver?$AA@ 004c2458     sv_ccmds.obj
 0002:00006464       ??_C@_03BANJEMDJ@say?$AA@  004c2464     sv_ccmds.obj
 0002:00006468       ??_C@_05JFDPDGMD@spmap?$AA@ 004c2468     sv_ccmds.obj
 0002:00006470       ??_C@_03HBNNNHNM@map?$AA@  004c2470     sv_ccmds.obj
 0002:00006474       ??_C@_0L@LFJOEPCG@sectorlist?$AA@ 004c2474     sv_ccmds.obj
 0002:00006480       ??_C@_08GCHPGJL@dumpuser?$AA@ 004c2480     sv_ccmds.obj
 0002:0000648c       ??_C@_0L@JENAJOPJ@systeminfo?$AA@ 004c248c     sv_ccmds.obj
 0002:00006498       ??_C@_0L@OJMFMOP@serverinfo?$AA@ 004c2498     sv_ccmds.obj
 0002:000064a4       ??_C@_06DJIHEMFI@status?$AA@ 004c24a4     sv_ccmds.obj
 0002:000064ac       ??_C@_0L@NBDAICFL@clientkick?$AA@ 004c24ac     sv_ccmds.obj
 0002:000064b8       ??_C@_09NMALIMLK@banClient?$AA@ 004c24b8     sv_ccmds.obj
 0002:000064c4       ??_C@_07MNEAPDFN@banUser?$AA@ 004c24c4     sv_ccmds.obj
 0002:000064cc       ??_C@_04FNIJDBCC@kick?$AA@ 004c24cc     sv_ccmds.obj
 0002:000064d4       ??_C@_09NCPIAHOP@heartbeat?$AA@ 004c24d4     sv_ccmds.obj
 0002:000064e0       ??_C@_06EKEKFCEC@nextdl?$AA@ 004c24e0     sv_client.obj
 0002:000064e8       ??_C@_08HNIAHLMM@download?$AA@ 004c24e8     sv_client.obj
 0002:000064f4       ??_C@_02GFBACKGC@cp?$AA@   004c24f4     sv_client.obj
 0002:000064f8       ??_C@_0CE@IHINFNJF@print?6Someone?5is?5using?5this?5CD?5K@ 004c24f8     sv_client.obj
 0002:0000651c       ??_C@_09MBPDEDJD@print?6?$CFs?6?$AA@ 004c251c     sv_client.obj
 0002:00006528       ??_C@_0CF@DFLDHJDB@print?6Awaiting?5CD?5key?5authorizat@ 004c2528     sv_client.obj
 0002:00006550       ??_C@_0BF@JLJINJFC@challengeResponse?5?$CFi?$AA@ 004c2550     sv_client.obj
 0002:00006568       ??_C@_06MPKMECK@accept?$AA@ 004c2568     sv_client.obj
 0002:00006570       ??_C@_0CD@NLEENFLL@print?6Server?5is?5not?5a?5demo?5serve@ 004c2570     sv_client.obj
 0002:00006594       ??_C@_0CL@OHKPCOFN@SV_AuthorizeIpPacket?3?5challenge?5@ 004c2594     sv_client.obj
 0002:000065c0       ??_C@_0DB@LGFOIHIH@SV_AuthorizeIpPacket?3?5not?5from?5a@ 004c25c0     sv_client.obj
 0002:000065f4       ??_C@_0CN@KDBDIPIK@Going?5from?5CS_CONNECTED?5to?5CS_PR@ 004c25f4     sv_client.obj
 0002:00006624       ??_C@_0CB@EAILJHJ@SV_SendClientGameState?$CI?$CJ?5for?5?$CFs?6@ 004c2624     sv_client.obj
 0002:00006648       ??_C@_0CK@GAFGMNPI@Going?5from?5CS_PRIMED?5to?5CS_ACTIV@ 004c2648     sv_client.obj
 0002:00006674       ??_C@_0CI@MOHODIAH@clientDownload?3?5?$CFd?5?3?5file?5?$CC?$CFs?$CC?5a@ 004c2674     sv_client.obj
 0002:0000669c       ??_C@_0BJ@GCBEGMAA@clientDownload?3?5?$CFs?5Done?6?$AA@ 004c269c     sv_client.obj
 0002:000066b8       ??_C@_0CH@KLJBEJLM@clientDownload?3?5?$CFd?5?3?5writing?5blo@ 004c26b8     sv_client.obj
 0002:000066e0       ??_C@_0L@FHBHENPL@sv_MaxRate?$AA@ 004c26e0     sv_client.obj
 0002:000066ec       ??_C@_04KOJKLCBG@1000?$AA@ 004c26ec     sv_client.obj
 0002:000066f4       ??_C@_0DE@NDHILGPJ@File?5?$CC?$CFs?$CC?5not?5found?5on?5server?5fo@ 004c26f4     sv_client.obj
 0002:00006728       ??_C@_0DE@PKCFFLAA@clientDownload?3?5?$CFd?5?3?5?$CC?$CFs?$CC?5file?5n@ 004c2728     sv_client.obj
 0002:00006760       ??_C@_0NL@DHILMFMH@Could?5not?5download?5?$CC?$CFs?$CC?5because?5@ 004c2760     sv_client.obj
 0002:00006840       ??_C@_0KC@PMIAHGNA@Could?5not?5download?5?$CC?$CFs?$CC?5because?5@ 004c2840     sv_client.obj
 0002:000068e4       ??_C@_0CM@JNECMCJP@clientDownload?3?5?$CFd?5?3?5?$CC?$CFs?$CC?5downlo@ 004c28e4     sv_client.obj
 0002:00006910       ??_C@_0CF@NHMNKNNJ@Cannot?5autodownload?5id?5pk3?5file?5@ 004c2910     sv_client.obj
 0002:00006938       ??_C@_0GM@IJEBFDBA@Cannot?5autodownload?5Team?5Arena?5f@ 004c2938     sv_client.obj
 0002:000069a4       ??_C@_0DI@PLGAONGI@clientDownload?3?5?$CFd?5?3?5?$CC?$CFs?$CC?5cannot@ 004c29a4     sv_client.obj
 0002:000069dc       ??_C@_0CE@JIBLCLMP@clientDownload?3?5?$CFd?5?3?5begining?5?$CC?$CF@ 004c29dc     sv_client.obj
 0002:00006a00       ??_C@_02GIIHKPLE@ip?$AA@   004c2a00     sv_client.obj
 0002:00006a04       ??_C@_0CA@PLBLJOEE@client?5text?5ignored?5for?5?$CFs?3?5?$CFs?6?$AA@ 004c2a04     sv_client.obj
 0002:00006a24       ??_C@_0CG@IHMMCKIP@getIpAuthorize?5?$CFi?5?$CFi?4?$CFi?4?$CFi?4?$CFi?5?$CFs@ 004c2a24     sv_client.obj
 0002:00006a4c       ??_C@_0BP@ECBEJKDB@sending?5getIpAuthorize?5for?5?$CFs?6?$AA@ 004c2a4c     sv_client.obj
 0002:00006a6c       ??_C@_0BM@KDJKNJFI@authorize?5server?5timed?5out?6?$AA@ 004c2a6c     sv_client.obj
 0002:00006a88       ??_C@_0BA@PCPGFMFA@disconnect?5?$CC?$CFs?$CC?$AA@ 004c2a88     sv_client.obj
 0002:00006a98       ??_C@_0BL@IKHIFDGN@Going?5to?5CS_ZOMBIE?5for?5?$CFs?6?$AA@ 004c2a98     sv_client.obj
 0002:00006ab4       ??_C@_0BB@FFPEABPI@print?5?$CC?$CFs?$FO7?5?$CFs?6?$CC?$AA@ 004c2ab4     sv_client.obj
 0002:00006ac8       ??_C@_0BA@KJHEBMDK@broken?5download?$AA@ 004c2ac8     sv_client.obj
 0002:00006ad8       ??_C@_0CK@EEKHNEKF@clientDownload?3?5?$CFd?5?3?5file?5?$CC?$CFs?$CC?5c@ 004c2ad8     sv_client.obj
 0002:00006b04       ??_C@_0DF@CGGBKJAN@clientDownload?3?5?$CFd?5?3?5client?5ackn@ 004c2b04     sv_client.obj
 0002:00006b3c       ??_C@_0N@GGGDBMDO@disconnected?$AA@ 004c2b3c     sv_client.obj
 0002:00006b4c       ??_C@_0DH@DJILMAML@Unpure?5client?5detected?4?5Invalid?5@ 004c2b4c     sv_client.obj
 0002:00006b84       ??_C@_0CN@FCJKPEIK@ignoring?5outdated?5cp?5command?5fro@ 004c2b84     sv_client.obj
 0002:00006bb4       ??_C@_09NGKOICNF@vm?1ui?4qvm?$AA@ 004c2bb4     sv_client.obj
 0002:00006bc0       ??_C@_0N@MIJFBLLA@vm?1cgame?4qvm?$AA@ 004c2bc0     sv_client.obj
 0002:00006bd0       ??_C@_0BH@DJCJEPBJ@Lost?5reliable?5commands?$AA@ 004c2bd0     sv_client.obj
 0002:00006be8       ??_C@_0CC@POHIDIAI@Client?5?$CFs?5lost?5?$CFi?5clientCommands@ 004c2be8     sv_client.obj
 0002:00006c0c       ??_C@_0BN@CDEFJJCC@clientCommand?3?5?$CFs?5?3?5?$CFi?5?3?5?$CFs?6?$AA@ 004c2c0c     sv_client.obj
 0002:00006c2c       ??_C@_0BN@OHAOFFFB@Cannot?5validate?5pure?5client?$CB?$AA@ 004c2c2c     sv_client.obj
 0002:00006c4c       ??_C@_0DA@HCALNAD@?$CFs?3?5didn?8t?5get?5cp?5command?0?5resen@ 004c2c4c     sv_client.obj
 0002:00006c7c       ??_C@_0CA@MHDHEKFF@cmdCount?5?$DO?5MAX_PACKET_USERCMDS?6?$AA@ 004c2c7c     sv_client.obj
 0002:00006c9c       ??_C@_0O@KIEOLJAH@cmdCount?5?$DM?51?6?$AA@ 004c2c9c     sv_client.obj
 0002:00006cac       ??_C@_0CJ@KKMJLOKN@WARNING?3?5bad?5command?5byte?5for?5cl@ 004c2cac     sv_client.obj
 0002:00006cd8       ??_C@_0CD@KEGKAOCA@?$CFs?5?3?5dropped?5gamestate?0?5resendin@ 004c2cd8     sv_client.obj
 0002:00006cfc       ??_C@_0DJ@EAHJJJGJ@?$CFs?5?3?5ignoring?5pre?5map_restart?5?1?5@ 004c2cfc     sv_client.obj
 0002:00006d38       ??_C@_0CL@DFDOECNK@Going?5from?5CS_FREE?5to?5CS_CONNECT@ 004c2d38     sv_client.obj
 0002:00006d64       ??_C@_0BI@BLKLCACF@Rejected?5a?5connection?4?6?$AA@ 004c2d64     sv_client.obj
 0002:00006d7c       ??_C@_0BH@NCFENBBP@print?6Server?5is?5full?4?6?$AA@ 004c2d7c     sv_client.obj
 0002:00006d94       ??_C@_0CB@OMBNPOIO@server?5is?5full?5on?5local?5connect?6@ 004c2d94     sv_client.obj
 0002:00006db8       ??_C@_0CB@GOGCKONC@Game?5rejected?5a?5connection?3?5?$CFs?4?6@ 004c2db8     sv_client.obj
 0002:00006ddc       ??_C@_0BE@HMGKIAJD@only?5bots?5on?5server?$AA@ 004c2ddc     sv_client.obj
 0002:00006df0       ??_C@_0O@FLCHKEJG@?$CFs?3reconnect?6?$AA@ 004c2df0     sv_client.obj
 0002:00006e00       ??_C@_0CH@PHCNAHEM@Client?5?$CFi?5rejected?5on?5a?5too?5high@ 004c2e00     sv_client.obj
 0002:00006e28       ??_C@_0CE@KINDDLDA@print?6Server?5is?5for?5low?5pings?5on@ 004c2e28     sv_client.obj
 0002:00006e4c       ??_C@_0CG@PNAAMAJH@Client?5?$CFi?5rejected?5on?5a?5too?5low?5@ 004c2e4c     sv_client.obj
 0002:00006e74       ??_C@_0CF@JPLKPOEC@print?6Server?5is?5for?5high?5pings?5o@ 004c2e74     sv_client.obj
 0002:00006e9c       ??_C@_0CN@CCHCPFHI@Client?5?$CFi?5connecting?5with?5?$CFi?5cha@ 004c2e9c     sv_client.obj
 0002:00006ecc       ??_C@_0CC@CIJKAFKI@?$CFs?3reconnect?5rejected?5?3?5too?5soon@ 004c2ecc     sv_client.obj
 0002:00006ef0       ??_C@_0CI@EIEGJKNB@print?6No?5or?5bad?5challenge?5for?5ad@ 004c2ef0     sv_client.obj
 0002:00006f18       ??_C@_0CG@NFNEGGLD@?5?5?5?5rejected?5connect?5from?5versio@ 004c2f18     sv_client.obj
 0002:00006f40       ??_C@_0CI@CNIPOKOM@print?6Server?5uses?5protocol?5versi@ 004c2f40     sv_client.obj
 0002:00006f68       ??_C@_0BG@MHNPDKDO@SVC_DirectConnect?5?$CI?$CJ?6?$AA@ 004c2f68     sv_client.obj
 0002:00006f80       ??_C@_0CA@HBFCCGAO@SV_SvEntityForGentity?3?5bad?5gEnt?$AA@ 004c2f80     sv_game.obj
 0002:00006fa0       ??_C@_0CJ@BCMBPMHM@SV_SetBrushModel?3?5?$CFs?5isn?8t?5a?5bru@ 004c2fa0     sv_game.obj
 0002:00006fcc       ??_C@_0BH@MHCNIHPH@SV_SetBrushModel?3?5NULL?$AA@ 004c2fcc     sv_game.obj
 0002:00006fe4       ??_C@_0CD@INNMELOE@SV_GetServerinfo?3?5bufferSize?5?$DN?$DN?5@ 004c2fe4     sv_game.obj
 0002:00007008       ??_C@_0CA@HGKJAJPL@SV_GetUsercmd?3?5bad?5clientNum?3?$CFi?$AA@ 004c3008     sv_game.obj
 0002:00007028       ??_C@_0BJ@HAMMCDKL@Bad?5game?5system?5trap?3?5?$CFi?$AA@ 004c3028     sv_game.obj
 0002:00007044       ??_C@_0BK@FFDIGEEK@VM_Restart?5on?5game?5failed?$AA@ 004c3044     sv_game.obj
 0002:00007060       ??_C@_0BJ@EAOELJMB@VM_Create?5on?5game?5failed?$AA@ 004c3060     sv_game.obj
 0002:0000707c       ??_C@_06BLCJNLEL@qagame?$AA@ 004c307c     sv_game.obj
 0002:00007084       ??_C@_07BHFGNDCM@vm_game?$AA@ 004c3084     sv_game.obj
 0002:0000708c       ??_C@_0M@MAONIEJF@cs?5?$CFi?5?$CC?$CFs?$CC?6?$AA@ 004c308c     sv_init.obj
 0002:00007098       ??_C@_0M@BPLDJGIF@?$CFs?5?$CFi?5?$CC?$CFs?$CC?6?$AA@ 004c3098     sv_init.obj
 0002:000070a4       ??_C@_0CC@NDBLLBPI@SV_SetConfigstring?3?5bad?5index?5?$CFi@ 004c30a4     sv_init.obj
 0002:000070c8       ??_C@_0CC@GPKJPKM@SV_GetConfigstring?3?5bad?5index?5?$CFi@ 004c30c8     sv_init.obj
 0002:000070ec       ??_C@_0CF@GDNLOPIJ@SV_GetConfigstring?3?5bufferSize?5?$DN@ 004c30ec     sv_init.obj
 0002:00007114       ??_C@_0BO@HKNINECJ@SV_SetUserinfo?3?5bad?5index?5?$CFi?6?$AA@ 004c3114     sv_init.obj
 0002:00007134       ??_C@_0BO@EFONBEDJ@SV_GetUserinfo?3?5bad?5index?5?$CFi?6?$AA@ 004c3134     sv_init.obj
 0002:00007154       ??_C@_0CB@MDKHFBJG@SV_GetUserinfo?3?5bufferSize?5?$DN?$DN?5?$CFi@ 004c3154     sv_init.obj
 0002:00007178       ??_C@_0BM@HIHCAEOD@SV_Startup?3?5svs?4initialized?$AA@ 004c3178     sv_init.obj
 0002:00007194       ??_C@_09FHDGEKJP@vm?1?$CFs?4qvm?$AA@ 004c3194     sv_init.obj
 0002:000071a0       ??_C@_0CF@MLCIJBNO@?9?9?9?9?9?9?9?9?9?9?9?9?9?9?9?9?9?9?9?9?9?9?9?9?9?9?9?9?9?9?9?9@ 004c31a0     sv_init.obj
 0002:000071c8       ??_C@_0CO@LKBABFKA@WARNING?3?5sv_pure?5set?5but?5no?5PK3?5@ 004c31c8     sv_init.obj
 0002:000071f8       ??_C@_0P@HEEKJLPJ@sv_mapChecksum?$AA@ 004c31f8     sv_init.obj
 0002:00007208       ??_C@_0O@JEFGAJAK@map_restart?50?$AA@ 004c3208     sv_init.obj
 0002:00007218       ??_C@_0CF@OFBEAHFI@?9?9?9?9?9?9?5Server?5Initialization?5?9?9?9@ 004c3218     sv_init.obj
 0002:00007240       ??_C@_0O@IIGECOIK@sv_strictAuth?$AA@ 004c3240     sv_init.obj
 0002:00007250       ??_C@_0BA@DJIAIMF@sv_lanForceRate?$AA@ 004c3250     sv_init.obj
 0002:00007260       ??_C@_0O@GOELPJCA@sv_padPackets?$AA@ 004c3260     sv_init.obj
 0002:00007270       ??_C@_0M@EFKNOLKP@sv_showloss?$AA@ 004c3270     sv_init.obj
 0002:0000727c       ??_C@_0BC@MCFEMHMF@sv_reconnectlimit?$AA@ 004c327c     sv_init.obj
 0002:00007290       ??_C@_0L@LLHDLDHL@sv_master5?$AA@ 004c3290     sv_init.obj
 0002:0000729c       ??_C@_0L@KCGIICDK@sv_master4?$AA@ 004c329c     sv_init.obj
 0002:000072a8       ??_C@_0L@ONCJBEPN@sv_master3?$AA@ 004c32a8     sv_init.obj
 0002:000072b4       ??_C@_0L@PEDCCFLM@sv_master2?$AA@ 004c32b4     sv_init.obj
 0002:000072c0       ??_C@_0L@NPBPHGHP@sv_master1?$AA@ 004c32c0     sv_init.obj
 0002:000072cc       ??_C@_0BB@MOCFKELF@sv_allowDownload?$AA@ 004c32cc     sv_init.obj
 0002:000072e0       ??_C@_0O@LLNJEMPF@sv_zombietime?$AA@ 004c32e0     sv_init.obj
 0002:000072f0       ??_C@_0L@MKEICGA@sv_timeout?$AA@ 004c32f0     sv_init.obj
 0002:000072fc       ??_C@_06JGIFLGEL@sv_fps?$AA@ 004c32fc     sv_init.obj
 0002:00007304       ??_C@_0BD@HGHMKODF@sv_privatePassword?$AA@ 004c3304     sv_init.obj
 0002:00007318       ??_C@_0BA@HMJAMCL@sv_floodProtect?$AA@ 004c3318     sv_init.obj
 0002:00007328       ??_C@_0L@DCJCBAAG@sv_maxPing?$AA@ 004c3328     sv_init.obj
 0002:00007334       ??_C@_0L@NEPCLPOH@sv_minPing?$AA@ 004c3334     sv_init.obj
 0002:00007340       ??_C@_0L@KOGBCPKN@sv_maxRate?$AA@ 004c3340     sv_init.obj
 0002:0000734c       ??_C@_0M@NHCIKFPA@sv_hostname?$AA@ 004c334c     sv_init.obj
 0002:00007358       ??_C@_06LNKFDEGN@noname?$AA@ 004c3358     sv_init.obj
 0002:00007360       ??_C@_0BC@BAEHHBBD@sv_privateClients?$AA@ 004c3360     sv_init.obj
 0002:00007374       ??_C@_05MIMHCHNF@nomap?$AA@ 004c3374     sv_init.obj
 0002:0000737c       ??_C@_0M@DBAEPHIE@sv_keywords?$AA@ 004c337c     sv_init.obj
 0002:00007388       ??_C@_09KPHKOKCC@timelimit?$AA@ 004c3388     sv_init.obj
 0002:00007394       ??_C@_09GCIEGDDN@fraglimit?$AA@ 004c3394     sv_init.obj
 0002:000073a0       ??_C@_07GMGCLCAP@dmflags?$AA@ 004c33a0     sv_init.obj
 0002:000073a8       ??_C@_0BN@CHNIPINJ@?9?9?9?9?9?9?9?9?9?9?9?9?9?9?9?9?9?9?9?9?9?9?9?9?9?9?9?6?$AA@ 004c33a8     sv_init.obj
 0002:000073c8       ??_C@_0BN@MINIHLBM@?9?9?9?9?9?5Server?5Shutdown?5?9?9?9?9?9?6?$AA@ 004c33c8     sv_init.obj
 0002:000073e8       ??_C@_05FEKEECGM@cs?5?$CFi?$AA@ 004c33e8     sv_main.obj
 0002:000073f0       ??_C@_0BI@BCMAPBDO@Server?5command?5overflow?$AA@ 004c33f0     sv_main.obj
 0002:00007408       ??_C@_0N@HPDJBMCC@cmd?5?$CF5d?3?5?$CFs?6?$AA@ 004c3408     sv_main.obj
 0002:00007418       ??_C@_0CF@DKJKGIEJ@?$DN?$DN?$DN?$DN?$DN?5pending?5server?5commands?5?$DN?$DN@ 004c3418     sv_main.obj
 0002:00007440       ??_C@_0P@KHEIJHKL@broadcast?3?5?$CFs?6?$AA@ 004c3440     sv_main.obj
 0002:00007450       ??_C@_0O@MFJONBCN@heartbeat?5?$CFs?6?$AA@ 004c3450     sv_main.obj
 0002:00007460       ??_C@_0N@KDHOMFCK@QuakeArena?91?$AA@ 004c3460     sv_main.obj
 0002:00007470       ??_C@_0BJ@FPIJBFOP@Sending?5heartbeat?5to?5?$CFs?6?$AA@ 004c3470     sv_main.obj
 0002:0000748c       ??_C@_0BO@EBNPOCKC@Couldn?8t?5resolve?5address?3?5?$CFs?6?$AA@ 004c348c     sv_main.obj
 0002:000074ac       ??_C@_0BF@DMGFDDCI@statusResponse?6?$CFs?6?$CFs?$AA@ 004c34ac     sv_main.obj
 0002:000074c4       ??_C@_0M@FDOKAKMK@?$CFi?5?$CFi?5?$CC?$CFs?$CC?6?$AA@ 004c34c4     sv_main.obj
 0002:000074d0       ??_C@_07CCFMBAIN@demo?5?$CFs?$AA@ 004c34d0     sv_main.obj
 0002:000074d8       ??_C@_0BA@ECLOOOJB@infoResponse?6?$CFs?$AA@ 004c34d8     sv_main.obj
 0002:000074e8       ??_C@_07NELDBAJ@maxPing?$AA@ 004c34e8     sv_main.obj
 0002:000074f0       ??_C@_07OLCLJOOI@minPing?$AA@ 004c34f0     sv_main.obj
 0002:000074f8       ??_C@_04NDBBJLFP@pure?$AA@ 004c34f8     sv_main.obj
 0002:00007500       ??_C@_08HCILNBCA@print?6?$CFs?$AA@ 004c3500     sv_main.obj
 0002:0000750c       ??_C@_0BD@LBHHIPJJ@Bad?5rconpassword?4?6?$AA@ 004c350c     sv_main.obj
 0002:00007520       ??_C@_0CE@LDGIIONG@No?5rconpassword?5set?5on?5the?5serve@ 004c3520     sv_main.obj
 0002:00007544       ??_C@_0BG@IKEHJABJ@Bad?5rcon?5from?5?$CFs?3?6?$CFs?6?$AA@ 004c3544     sv_main.obj
 0002:0000755c       ??_C@_0BC@EHLDDKCE@Rcon?5from?5?$CFs?3?6?$CFs?6?$AA@ 004c355c     sv_main.obj
 0002:00007570       ??_C@_0CH@NHBAICIE@bad?5connectionless?5packet?5from?5?$CF@ 004c3570     sv_main.obj
 0002:00007598       ??_C@_0M@OJIOIONL@ipAuthorize?$AA@ 004c3598     sv_main.obj
 0002:000075a4       ??_C@_07OICKPAFH@getinfo?$AA@ 004c35a4     sv_main.obj
 0002:000075ac       ??_C@_0BD@JKPIBMPL@SV?5packet?5?$CFs?5?3?5?$CFs?6?$AA@ 004c35ac     sv_main.obj
 0002:000075c0       ??_C@_0CN@BLLAHKEO@SV_PacketEvent?3?5fixing?5up?5a?5tran@ 004c35c0     sv_main.obj
 0002:000075f0       ??_C@_09KJPPMAOI@timed?5out?$AA@ 004c35f0     sv_main.obj
 0002:000075fc       ??_C@_0CP@OAICOBIP@Going?5from?5CS_ZOMBIE?5to?5CS_FREE?5@ 004c35fc     sv_main.obj
 0002:0000762c       ??_C@_0P@BKKOFHJN@map_restart?50?6?$AA@ 004c362c     sv_main.obj
 0002:0000763c       ??_C@_0DG@CKJAOBCN@Restarting?5server?5due?5to?5numSnap@ 004c363c     sv_main.obj
 0002:00007674       ??_C@_0O@PKDALKNK@vstr?5nextmap?6?$AA@ 004c3674     sv_main.obj
 0002:00007684       ??_C@_0CH@OOPAJFOA@Restarting?5server?5due?5to?5time?5wr@ 004c3684     sv_main.obj
 0002:000076ac       ??_C@_0BE@KDNEMLAA@Server?5was?5killed?4?6?$AA@ 004c36ac     sv_main.obj
 0002:000076c0       ??_C@_0DN@JABDKDJO@?$CD462?5Netchan_TransmitNextFragmen@ 004c36c0     sv_net_chan.obj
 0002:00007700       ??_C@_0DC@LPKBFGIK@?$CD462?5Netchan_TransmitNextFragmen@ 004c3700     sv_net_chan.obj
 0002:00007738       ??_C@_0EK@ODEKMBHH@?$CD462?5Netchan_TransmitNextFragmen@ 004c3738     sv_net_chan.obj
 0002:00007788       ??_C@_0EO@MKKMHFAL@netchan?5queue?5is?5not?5properly?5in@ 004c3788     sv_net_chan.obj
 0002:000077d8       ??_C@_0DF@MDAEODOK@?$CD462?5SV_Netchan_Transmit?3?5unsent@ 004c37d8     sv_net_chan.obj
 0002:00007810       ??_C@_0CO@GHMJABCI@?$CFs?3?5Delta?5request?5from?5out?5of?5da@ 004c3810     sv_snapshot.obj
 0002:00007840       ??_C@_0CM@DLGJFOOO@?$CFs?3?5Delta?5request?5from?5out?5of?5da@ 004c3840     sv_snapshot.obj
 0002:0000786c       ??_C@_0CI@IHBPJMCI@SV_QsortEntityStates?3?5duplicated@ 004c386c     sv_snapshot.obj
 0002:00007894       ??_C@_0BP@KFJNHKJA@SVF_CLIENTMASK?3?5cientNum?5?$DO?532?6?$AA@ 004c3894     sv_snapshot.obj
 0002:000078b4       ??_C@_0BJ@OGOHIIMC@FIXING?5ENT?9?$DOS?4NUMBER?$CB?$CB?$CB?6?$AA@ 004c38b4     sv_snapshot.obj
 0002:000078d0       ??_C@_0CB@DGHKPLAI@svs?4nextSnapshotEntities?5wrapped@ 004c38d0     sv_snapshot.obj
 0002:000078f4       ??_C@_0CA@BILMKJDC@WARNING?3?5msg?5overflowed?5for?5?$CFs?6?$AA@ 004c38f4     sv_snapshot.obj
 0002:00007914       ??_C@_0BI@IINMPMIE@sector?5?$CFi?3?5?$CFi?5entities?6?$AA@ 004c3914     sv_world.obj
 0002:0000792c       ??_C@_0DE@NOEMPBKJ@WARNING?3?5SV_UnlinkEntity?3?5not?5fo@ 004c392c     sv_world.obj
 0002:00007960       ??_C@_0CI@LMCDEPAK@Object?5?$CFi?5touching?53?5areas?5at?5?$CFf@ 004c3960     sv_world.obj
 0002:00007988       ??_C@_0BL@IPEAAEPI@SV_AreaEntities?3?5MAXCOUNT?6?$AA@ 004c3988     sv_world.obj
 0002:00007c18       ??_C@_0CE@LOHAHEGK@incomplete?5dynamic?5bit?5lengths?5t@ 004c3c18     unzip.obj
 0002:00007c3c       ??_C@_0CI@CGMOPDPD@oversubscribed?5dynamic?5bit?5lengt@ 004c3c3c     unzip.obj
 0002:00007c64       ??_C@_0BP@NEEEJJNA@incomplete?5literal?1length?5tree?$AA@ 004c3c64     unzip.obj
 0002:00007c84       ??_C@_0CD@GJIDGCKE@oversubscribed?5literal?1length?5tr@ 004c3c84     unzip.obj
 0002:00007ca8       ??_C@_0CB@KPKKKLFO@empty?5distance?5tree?5with?5lengths@ 004c3ca8     unzip.obj
 0002:00007ccc       ??_C@_0BJ@CBCPDPJF@incomplete?5distance?5tree?$AA@ 004c3ccc     unzip.obj
 0002:00007ce8       ??_C@_0BN@KBLCDIAI@oversubscribed?5distance?5tree?$AA@ 004c3ce8     unzip.obj
 0002:00007d08       ??_C@_0BM@FFFLPBBC@invalid?5literal?1length?5code?$AA@ 004c3d08     unzip.obj
 0002:00007d24       ??_C@_0BG@LBKINIKP@invalid?5distance?5code?$AA@ 004c3d24     unzip.obj
 0002:00007d3c       ??_C@_0BK@BMMPFBBH@invalid?5bit?5length?5repeat?$AA@ 004c3d3c     unzip.obj
 0002:00007d58       ??_C@_0CE@GMIGFPBB@too?5many?5length?5or?5distance?5symb@ 004c3d58     unzip.obj
 0002:00007d7c       ??_C@_0BN@LGAADGOK@invalid?5stored?5block?5lengths?$AA@ 004c3d7c     unzip.obj
 0002:00007d9c       ??_C@_0BD@PJCBIDD@invalid?5block?5type?$AA@ 004c3d9c     unzip.obj
 0002:00007db0       ??_C@_0BA@MOKMMFOD@need?5dictionary?$AA@ 004c3db0     unzip.obj
 0002:00007dc0       ??_C@_0BF@MEIGEHBE@incorrect?5data?5check?$AA@ 004c3dc0     unzip.obj
 0002:00007dd8       ??_C@_0BH@LIBMMIGA@incorrect?5header?5check?$AA@ 004c3dd8     unzip.obj
 0002:00007df0       ??_C@_0BE@EMOGCLGO@invalid?5window?5size?$AA@ 004c3df0     unzip.obj
 0002:00007e04       ??_C@_0BL@IHKGDAEE@unknown?5compression?5method?$AA@ 004c3e04     unzip.obj
 0002:00007e20       ??_C@_05HBMFIKCP@1?41?43?$AA@ 004c3e20     unzip.obj
 0002:00007e28       ??_C@_05FKKECMBM@?$CFs?$CL?$CFi?$AA@ 004c3e28     vm.obj
 0002:00007e30       ??_C@_0L@CKHGNKPG@NO?5SYMBOLS?$AA@ 004c3e30     vm.obj
 0002:00007e3c       ??_C@_0BB@MJCHPEFI@After?5code?5block?$AA@ 004c3e3c     vm.obj
 0002:00007e50       ??_C@_0BC@NFLMMLOB@Before?5code?5block?$AA@ 004c3e50     vm.obj
 0002:00007e64       ??_C@_0BL@FKOJLOGO@?$CFi?5symbols?5parsed?5from?5?$CFs?6?$AA@ 004c3e64     vm.obj
 0002:00007e80       ??_C@_0CJ@KBFNJAIO@WARNING?3?5incomplete?5line?5at?5end?5@ 004c3e80     vm.obj
 0002:00007eac       ??_C@_0BP@EJCGAFI@Couldn?8t?5load?5symbol?5file?3?5?$CFs?6?$AA@ 004c3eac     vm.obj
 0002:00007ecc       ??_C@_09KLPMHLFB@vm?1?$CFs?4map?$AA@ 004c3ecc     vm.obj
 0002:00007ed8       ??_C@_0P@LAPBOIJN@VM_Call?$CI?5?$CFi?5?$CJ?6?$AA@ 004c3ed8     vm.obj
 0002:00007ee8       ??_C@_0BF@GNADHAJC@VM_Call?5with?5NULL?5vm?$AA@ 004c3ee8     vm.obj
 0002:00007f00       ??_C@_0BB@NCIFAMHB@?5?5?5?5?$CF9?40f?5total?6?$AA@ 004c3f00     vm.obj
 0002:00007f14       ??_C@_0O@DAPAGLHI@?$CF2i?$CF?$CF?5?$CF9i?5?$CFs?6?$AA@ 004c3f14     vm.obj
 0002:00007f24       ??_C@_0BH@DGKALKOH@?5?5?5?5data?5length?5?3?5?$CF7i?6?$AA@ 004c3f24     vm.obj
 0002:00007f3c       ??_C@_0BH@PPKCIMFO@?5?5?5?5table?5length?3?5?$CF7i?6?$AA@ 004c3f3c     vm.obj
 0002:00007f54       ??_C@_0BH@KGNDPGNP@?5?5?5?5code?5length?5?3?5?$CF7i?6?$AA@ 004c3f54     vm.obj
 0002:00007f6c       ??_C@_0N@CFOLNHPI@interpreted?6?$AA@ 004c3f6c     vm.obj
 0002:00007f7c       ??_C@_0BC@GEADELFK@compiled?5on?5load?6?$AA@ 004c3f7c     vm.obj
 0002:00007f90       ??_C@_07IMELJBKE@native?6?$AA@ 004c3f90     vm.obj
 0002:00007f98       ??_C@_05LLGELLBM@?$CFs?5?3?5?$AA@ 004c3f98     vm.obj
 0002:00007fa0       ??_C@_0BO@GJPNKMOM@Registered?5virtual?5machines?3?6?$AA@ 004c3fa0     vm.obj
 0002:00007fc0       ??_C@_0BL@KGOIDDFO@?$CFi?3?5?$CFi?5?$CI?$CFi?$CJ?5?$DN?5?$CFi?5?$CFi?5?$CFi?5?$CFi?6?$AA@ 004c3fc0     vm.obj
 0002:00007fdc       ??_C@_0N@HIIMEIJN@syscalls?4log?$AA@ 004c3fdc     vm.obj
 0002:00007fec       ??_C@_01NOFIACDB@w?$AA@    004c3fec     vm.obj
 0002:00007ff0       ??_C@_06LIKFIMOC@vminfo?$AA@ 004c3ff0     vm.obj
 0002:00007ff8       ??_C@_09GNBAHOHK@vmprofile?$AA@ 004c3ff8     vm.obj
 0002:00008004       ??_C@_0CD@GEPNAEEP@?$CFs?5loaded?5in?5?$CFd?5bytes?5on?5the?5hun@ 004c4004     vm.obj
 0002:00008028       ??_C@_0BC@OPCEGJFC@?$CFs?5has?5bad?5header?$AA@ 004c4028     vm.obj
 0002:0000803c       ??_C@_08OEINOMOH@Failed?4?6?$AA@ 004c403c     vm.obj
 0002:00008048       ??_C@_0BF@IGPEJINO@Loading?5vm?5file?5?$CFs?4?6?$AA@ 004c4048     vm.obj
 0002:00008060       ??_C@_0CG@KNDPANGF@Failed?5to?5load?5dll?0?5looking?5for?5@ 004c4060     vm.obj
 0002:00008088       ??_C@_0BG@JJIBCGPE@Loading?5dll?5file?5?$CFs?4?6?$AA@ 004c4088     vm.obj
 0002:000080a0       ??_C@_0BI@IOGIAGHC@VM_Create?3?5no?5free?5vm_t?$AA@ 004c40a0     vm.obj
 0002:000080b8       ??_C@_0BF@IGDBCBGP@VM_Create?3?5bad?5parms?$AA@ 004c40b8     vm.obj
 0002:000080d0       ??_C@_0BE@OFKMANMD@VM_Restart?5failed?4?6?$AA@ 004c40d0     vm.obj
 0002:000080e4       ??_C@_0O@HMGHEGLA@VM_Restart?$CI?$CJ?6?$AA@ 004c40e4     vm.obj
 0002:000080f4       ??_C@_0CJ@PMEMCJLI@?5?5?5?5?5?5?5?5?5?5?5?5?5?5?5?5?5?5?5?5?5?5?5?5?5?5?5?5?5?5?5?5@ 004c40f4     vm_interpreted.obj
 0002:00008120       ??_C@_0CP@GJNCCGPN@VM_PrepareInterpreter?3?5pc?5?$DO?5head@ 004c4120     vm_interpreted.obj
 0002:00008150       ??_C@_0CA@CCJDPMLL@Interpreter?5error?3?5opStack?5?$DN?5?$CFi?$AA@ 004c4150     vm_interpreted.obj
 0002:00008170       ??_C@_0CA@KLAFBCCD@OP_BLOCK_COPY?5not?5dword?5aligned?$AA@ 004c4170     vm_interpreted.obj
 0002:00008190       ??_C@_0BD@LHJDCNBD@Hex?3?5bad?5char?5?8?$CFc?8?$AA@ 004c4190     vm_x86.obj
 0002:000081a4       ??_C@_05BOHLOLPB@89?507?$AA@ 004c41a4     vm_x86.obj
 0002:000081ac       ??_C@_08PPLFGLPG@83?5EF?504?$AA@ 004c41ac     vm_x86.obj
 0002:000081b8       ??_C@_08FDAACEPK@83?5EF?508?$AA@ 004c41b8     vm_x86.obj
 0002:000081c4       ??_C@_08ONFOEBJE@83?5C7?504?$AA@ 004c41c4     vm_x86.obj
 0002:000081d0       ??_C@_05JAHJDKCP@8B?507?$AA@ 004c41d0     vm_x86.obj
 0002:000081d8       ??_C@_02GEDPMDLI@B8?$AA@   004c41d8     vm_x86.obj
 0002:000081dc       ??_C@_05KHJPBIKP@8B?51F?$AA@ 004c41dc     vm_x86.obj
 0002:000081e4       ??_C@_02LBOPFCME@BB?$AA@   004c41e4     vm_x86.obj
 0002:000081e8       ??_C@_05EEBJOGGM@8B?5D8?$AA@ 004c41e8     vm_x86.obj
 0002:000081f0       ??_C@_0CJ@IMEHDLPA@VM?5file?5?$CFs?5compiled?5to?5?$CFi?5bytes?5@ 004c41f0     vm_x86.obj
 0002:0000821c       ??_C@_0CK@EFPLJADG@VM_CompileX86?3?5bad?5opcode?5?$CFi?5at?5@ 004c421c     vm_x86.obj
 0002:00008248       ??_C@_08KBFJACGK@FF?524?585?$AA@ 004c4248     vm_x86.obj
 0002:00008254       ??_C@_02KPBALKNG@5E?$AA@   004c4254     vm_x86.obj
 0002:00008258       ??_C@_02IEDNOJBF@5F?$AA@   004c4258     vm_x86.obj
 0002:0000825c       ??_C@_05COGPPAE@F3?5A5?$AA@ 004c425c     vm_x86.obj
 0002:00008264       ??_C@_05LKKMOIGM@03?5FB?$AA@ 004c4264     vm_x86.obj
 0002:0000826c       ??_C@_05CCLENIBL@23?5F8?$AA@ 004c426c     vm_x86.obj
 0002:00008274       ??_C@_05IMIIKANL@03?5F3?$AA@ 004c4274     vm_x86.obj
 0002:0000827c       ??_C@_05OKGNFCBD@23?5F0?$AA@ 004c427c     vm_x86.obj
 0002:00008284       ??_C@_02HNCEPCPJ@B9?$AA@   004c4284     vm_x86.obj
 0002:00008288       ??_C@_08OJKHKNOB@8B?57F?5FC?$AA@ 004c4288     vm_x86.obj
 0002:00008294       ??_C@_05JCDPIEHG@8B?537?$AA@ 004c4294     vm_x86.obj
 0002:0000829c       ??_C@_02LCBJKBKC@57?$AA@   004c429c     vm_x86.obj
 0002:000082a0       ??_C@_08JGPFDFGB@0F?5BF?507?$AA@ 004c42a0     vm_x86.obj
 0002:000082ac       ??_C@_08NBFFEPLB@0F?5BE?507?$AA@ 004c42ac     vm_x86.obj
 0002:000082b8       ??_C@_05OMJJPHJF@DB?507?$AA@ 004c42b8     vm_x86.obj
 0002:000082c0       ??_C@_08LFPHLGAB@D8?54f?504?$AA@ 004c42c0     vm_x86.obj
 0002:000082cc       ??_C@_08DGBACCNE@D8?577?504?$AA@ 004c42cc     vm_x86.obj
 0002:000082d8       ??_C@_08PNEMPBHB@D8?567?504?$AA@ 004c42d8     vm_x86.obj
 0002:000082e4       ??_C@_08EDMCLBON@D9?55F?5FC?$AA@ 004c42e4     vm_x86.obj
 0002:000082f0       ??_C@_05FPPLAPPL@D8?507?$AA@ 004c42f0     vm_x86.obj
 0002:000082f8       ??_C@_08EMCMKLDH@D9?547?5FC?$AA@ 004c42f8     vm_x86.obj
 0002:00008304       ??_C@_05FFHNAEML@D9?51F?$AA@ 004c4304     vm_x86.obj
 0002:0000830c       ??_C@_05HPOABKDH@D9?5E0?$AA@ 004c430c     vm_x86.obj
 0002:00008314       ??_C@_05GCJLCGEL@D9?507?$AA@ 004c4314     vm_x86.obj
 0002:0000831c       ??_C@_08FEJGNPIL@D3?56F?5FC?$AA@ 004c431c     vm_x86.obj
 0002:00008328       ??_C@_08JPMKAMCO@D3?57F?5FC?$AA@ 004c4328     vm_x86.obj
 0002:00008334       ??_C@_08JACEBGPE@D3?567?5FC?$AA@ 004c4334     vm_x86.obj
 0002:00008340       ??_C@_05KGFNHCJI@8B?50F?$AA@ 004c4340     vm_x86.obj
 0002:00008348       ??_C@_05JBKBFDBG@F7?517?$AA@ 004c4348     vm_x86.obj
 0002:00008350       ??_C@_08LALBOJO@31?547?5FC?$AA@ 004c4350     vm_x86.obj
 0002:0000835c       ??_C@_08OBGDDJOO@09?547?5FC?$AA@ 004c435c     vm_x86.obj
 0002:00008368       ??_C@_08BMHAAKNN@21?547?5FC?$AA@ 004c4368     vm_x86.obj
 0002:00008374       ??_C@_05JDOHONEP@F7?527?$AA@ 004c4374     vm_x86.obj
 0002:0000837c       ??_C@_05KFMDKFPI@F7?52F?$AA@ 004c437c     vm_x86.obj
 0002:00008384       ??_C@_08JBOHEIFD@89?557?5FC?$AA@ 004c4384     vm_x86.obj
 0002:00008390       ??_C@_05JCCFIHHI@F7?537?$AA@ 004c4390     vm_x86.obj
 0002:00008398       ??_C@_05BAIDDHFK@33?5D2?$AA@ 004c4398     vm_x86.obj
 0002:000083a0       ??_C@_08FKLLJLPG@89?547?5FC?$AA@ 004c43a0     vm_x86.obj
 0002:000083ac       ??_C@_05KEABMPMP@F7?53F?$AA@ 004c43ac     vm_x86.obj
 0002:000083b4       ??_C@_02CFIAHFEI@99?$AA@   004c43b4     vm_x86.obj
 0002:000083b8       ??_C@_08KLIBBGDA@8B?547?5FC?$AA@ 004c43b8     vm_x86.obj
 0002:000083c4       ??_C@_08MPJFBBGI@29?547?5FC?$AA@ 004c43c4     vm_x86.obj
 0002:000083d0       ??_C@_08DCIGCCFL@01?547?5FC?$AA@ 004c43d0     vm_x86.obj
 0002:000083dc       ??_C@_05KHIFBLKB@F7?51F?$AA@ 004c43dc     vm_x86.obj
 0002:000083e4       ??_C@_08KAABHBPO@F6?5C4?541?$AA@ 004c43e4     vm_x86.obj
 0002:000083f0       ??_C@_08KHAINJCC@F6?5C4?501?$AA@ 004c43f0     vm_x86.obj
 0002:000083fc       ??_C@_08LJBKEALP@F6?5C4?540?$AA@ 004c43fc     vm_x86.obj
 0002:00008408       ??_C@_05EGCGNCJ@DF?5E0?$AA@ 004c4408     vm_x86.obj
 0002:00008410       ??_C@_08BDNPAFKM@D8?55F?508?$AA@ 004c4410     vm_x86.obj
 0002:0000841c       ??_C@_08HMCOFAOE@D9?547?504?$AA@ 004c441c     vm_x86.obj
 0002:00008428       ??_C@_05IBOGFJHE@72?506?$AA@ 004c4428     vm_x86.obj
 0002:00008430       ??_C@_05HEGGPPLE@76?506?$AA@ 004c4430     vm_x86.obj
 0002:00008438       ??_C@_05EJAGNGAE@77?506?$AA@ 004c4438     vm_x86.obj
 0002:00008440       ??_C@_05LMIGHAME@73?506?$AA@ 004c4440     vm_x86.obj
 0002:00008448       ??_C@_05EFFEJAAL@7C?506?$AA@ 004c4448     vm_x86.obj
 0002:00008450       ??_C@_05MKBEGFKL@7E?506?$AA@ 004c4450     vm_x86.obj
 0002:00008458       ??_C@_05GFGDEGLC@FF?525?$AA@ 004c4458     vm_x86.obj
 0002:00008460       ??_C@_05INLEBPHL@7F?506?$AA@ 004c4460     vm_x86.obj
 0002:00008468       ??_C@_05PHHEEMBL@7D?506?$AA@ 004c4468     vm_x86.obj
 0002:00008470       ??_C@_05OKGKMNE@74?506?$AA@ 004c4470     vm_x86.obj
 0002:00008478       ??_C@_05DDMGIFGE@75?506?$AA@ 004c4478     vm_x86.obj
 0002:00008480       ??_C@_08LFGDDMDC@3B?547?508?$AA@ 004c4480     vm_x86.obj
 0002:0000848c       ??_C@_08JLIDONOD@8B?547?504?$AA@ 004c448c     vm_x86.obj
 0002:00008498       ??_C@_08KEGPAMOK@8B?55F?5FC?$AA@ 004c4498     vm_x86.obj
 0002:000084a4       ??_C@_08FFIEBBC@0F?5B6?583?$AA@ 004c44a4     vm_x86.obj
 0002:000084b0       ??_C@_08DIDIGIKC@0F?5B7?583?$AA@ 004c44b0     vm_x86.obj
 0002:000084bc       ??_C@_05NBCLPNFA@8B?580?$AA@ 004c44bc     vm_x86.obj
 0002:000084c4       ??_C@_02LDEEJNBC@2D?$AA@   004c44c4     vm_x86.obj
 0002:000084c8       ??_C@_05IIKCMFF@FF?58B?$AA@ 004c44c8     vm_x86.obj
 0002:000084d0       ??_C@_02IGOEABML@05?$AA@   004c44d0     vm_x86.obj
 0002:000084d4       ??_C@_05PKAGKOJD@8B?583?$AA@ 004c44d4     vm_x86.obj
 0002:000084dc       ??_C@_05DOKOGEOC@FF?583?$AA@ 004c44dc     vm_x86.obj
 0002:000084e4       ??_C@_02IGAJHAEE@C3?$AA@   004c44e4     vm_x86.obj
 0002:000084e8       ??_C@_05GBKHEHHI@81?5C6?$AA@ 004c44e8     vm_x86.obj
 0002:000084f0       ??_C@_05GHCFPIOL@FF?515?$AA@ 004c44f0     vm_x86.obj
 0002:000084f8       ??_C@_05NHKGMIGL@C7?586?$AA@ 004c44f8     vm_x86.obj
 0002:00008500       ??_C@_05JHDILAI@89?586?$AA@ 004c4500     vm_x86.obj
 0002:00008508       ??_C@_05IDBKPHG@8D?586?$AA@ 004c4508     vm_x86.obj
 0002:00008510       ??_C@_05MAKOKIJC@C7?507?$AA@ 004c4510     vm_x86.obj
 0002:00008518       ??_C@_05BLKLDMOJ@81?52F?$AA@ 004c4518     vm_x86.obj
 0002:00008520       ??_C@_05COALKADA@81?507?$AA@ 004c4520     vm_x86.obj
 0002:00008528       ??_C@_05EJGEFGPN@88?583?$AA@ 004c4528     vm_x86.obj
 0002:00008530       ??_C@_08PCPLBAHO@66?589?583?$AA@ 004c4530     vm_x86.obj
 0002:0000853c       ??_C@_05HEAEHPEN@89?583?$AA@ 004c453c     vm_x86.obj
 0002:00008544       ??_C@_08LELBAKK@0F?5B6?503?$AA@ 004c4544     vm_x86.obj
 0002:00008550       ??_C@_08DGCLDJBK@0F?5B7?503?$AA@ 004c4550     vm_x86.obj
 0002:0000855c       ??_C@_05PEBFPPCL@8B?503?$AA@ 004c455c     vm_x86.obj
 0002:00008564       ??_C@_05GBDIBBPP@81?5EE?$AA@ 004c4564     vm_x86.obj
 0002:0000856c       ??_C@_02KJDGAJLC@CC?$AA@   004c456c     vm_x86.obj
 0002:00008570       ??_C@_0CH@KBPAIEIJ@VM_CompileX86?3?5pc?5?$DO?5header?9?$DOcode@ 004c4570     vm_x86.obj
 0002:00008598       ??_C@_0CC@BBOPGMCE@VM_CompileX86?3?5maxLength?5exceede@ 004c4598     vm_x86.obj
 0002:000085bc       ??_C@_0CI@DJIHNOJD@programStack?5corrupted?5in?5compil@ 004c45bc     vm_x86.obj
 0002:000085e4       ??_C@_0CD@CEBALJKM@opStack?5corrupted?5in?5compiled?5co@ 004c45e4     vm_x86.obj
 0002:00008608       _GUID_SysMouse             004c4608     win_input.obj
 0002:00008618       _GUID_XAxis                004c4618     win_input.obj
 0002:00008628       _GUID_YAxis                004c4628     win_input.obj
 0002:00008638       _GUID_ZAxis                004c4638     win_input.obj
 0002:00008648       ??_C@_07EMFEJGAN@no?5POV?6?$AA@ 004c4648     win_input.obj
 0002:00008650       ??_C@_07GBHJMAHC@HASPOV?6?$AA@ 004c4650     win_input.obj
 0002:00008658       ??_C@_0M@EMGDDLAE@Caps?3?50x?$CFx?6?$AA@ 004c4658     win_input.obj
 0002:00008664       ??_C@_0P@IHBPICK@Axis?3?5?$CFi?5?1?5?$CFi?6?$AA@ 004c4664     win_input.obj
 0002:00008674       ??_C@_0BF@PJBJAPDP@Numbuttons?3?5?$CFi?5?1?5?$CFi?6?$AA@ 004c4674     win_input.obj
 0002:0000868c       ??_C@_0M@KEHKBEMN@RegKey?3?5?$CFs?6?$AA@ 004c468c     win_input.obj
 0002:00008698       ??_C@_0M@FCGKCNFI@OemVxD?3?5?$CFs?6?$AA@ 004c4698     win_input.obj
 0002:000086a4       ??_C@_0L@KFAEIOHL@Pname?3?5?$CFs?6?$AA@ 004c46a4     win_input.obj
 0002:000086b0       ??_C@_0BB@MPGIOLMD@Joystick?5found?4?6?$AA@ 004c46b0     win_input.obj
 0002:000086c4       ??_C@_0DK@KEFPCM@joystick?5not?5found?5?9?9?5invalid?5jo@ 004c46c4     win_input.obj
 0002:00008700       ??_C@_0CP@LGEKEFDA@joystick?5not?5found?5?9?9?5no?5valid?5j@ 004c4700     win_input.obj
 0002:00008730       ??_C@_0CK@HJHGOPLD@joystick?5not?5found?5?9?9?5driver?5not@ 004c4730     win_input.obj
 0002:0000875c       ??_C@_0BJ@HFLDAPPJ@Joystick?5is?5not?5active?4?6?$AA@ 004c475c     win_input.obj
 0002:00008778       __real@3f00000000000000    004c4778     win_input.obj
 0002:00008780       ??_C@_0CJ@POKLHOLL@?$CF8x?5?$CF5i?5?$CF5?42f?5?$CF5?42f?5?$CF5?42f?5?$CF5?42f?5@ 004c4780     win_input.obj
 0002:000087ac       ??_C@_0BL@JNGNJJBL@?4?4?4product?5ID?3?5?5?5?5?5?50x?$CFhx?6?$AA@ 004c47ac     win_input.obj
 0002:000087c8       ??_C@_0BL@MLLFNMAG@?4?4?4manufacturer?5ID?3?50x?$CFhx?6?$AA@ 004c47c8     win_input.obj
 0002:000087e4       ??_C@_0BG@IFDHOHKE@device?5?$CF2d?3?5?5?5?5?5?5?5?$CFs?6?$AA@ 004c47e4     win_input.obj
 0002:000087fc       ??_C@_03KHICJKCI@?4?4?4?$AA@ 004c47fc     win_input.obj
 0002:00008800       ??_C@_03ELIFGAKH@?$CK?$CK?$CK?$AA@ 004c4800     win_input.obj
 0002:00008804       ??_C@_0O@ILMLMLBN@in_mididevice?$AA@ 004c4804     win_input.obj
 0002:00008814       ??_C@_0BI@MOFLADHH@number?5of?5devices?3?5?5?$CFd?6?$AA@ 004c4814     win_input.obj
 0002:0000882c       ??_C@_0BI@JCNHHIF@current?5device?3?5?5?5?5?5?$CFd?6?$AA@ 004c482c     win_input.obj
 0002:00008844       ??_C@_0BI@MNCPBAID@channel?3?5?5?5?5?5?5?5?5?5?5?5?5?$CFd?6?$AA@ 004c4844     win_input.obj
 0002:0000885c       ??_C@_0BI@ONOGGNGI@port?3?5?5?5?5?5?5?5?5?5?5?5?5?5?5?5?$CFd?6?$AA@ 004c485c     win_input.obj
 0002:00008874       ??_C@_0BJ@JEGLDNKE@?6MIDI?5control?3?5?5?5?5?5?5?5?$CFs?6?$AA@ 004c4874     win_input.obj
 0002:00008890       ??_C@_07MHHIKOPA@enabled?$AA@ 004c4890     win_input.obj
 0002:00008898       ??_C@_08BEHKFNNO@disabled?$AA@ 004c4898     win_input.obj
 0002:000088a4       ??_C@_0CO@BDCKEEAF@WARNING?3?5could?5not?5open?5MIDI?5dev@ 004c48a4     win_input.obj
 0002:000088d4       ??_C@_07KPEFKOPL@in_midi?$AA@ 004c48d4     win_input.obj
 0002:000088dc       ??_C@_0BK@CCEBLJCF@DirectInput?5initialized?4?6?$AA@ 004c48dc     win_input.obj
 0002:000088f8       ??_C@_0BM@EODFEMCB@Couldn?8t?5set?5DI?5buffersize?6?$AA@ 004c48f8     win_input.obj
 0002:00008914       ??_C@_0BM@NMAODKLJ@Couldn?8t?5set?5DI?5coop?5level?6?$AA@ 004c4914     win_input.obj
 0002:00008930       ??_C@_0BO@BNCCIHMP@Couldn?8t?5set?5DI?5mouse?5format?6?$AA@ 004c4930     win_input.obj
 0002:00008950       ??_C@_0BP@DAFJNOPB@Couldn?8t?5open?5DI?5mouse?5device?6?$AA@ 004c4950     win_input.obj
 0002:00008970       ??_C@_0BL@ICIGFMME@iDirectInputCreate?5failed?6?$AA@ 004c4970     win_input.obj
 0002:0000898c       ??_C@_0BL@FLLJFGNK@Couldn?8t?5get?5DI?5proc?5addr?6?$AA@ 004c498c     win_input.obj
 0002:000089a8       ??_C@_0BD@BGJEDEPJ@DirectInputCreateA?$AA@ 004c49a8     win_input.obj
 0002:000089bc       ??_C@_0BK@IKANOGNK@Couldn?8t?5load?5dinput?4dll?6?$AA@ 004c49bc     win_input.obj
 0002:000089d8       ??_C@_0L@NKFBIDA@dinput?4dll?$AA@ 004c49d8     win_input.obj
 0002:000089e4       ??_C@_0BN@PJMDGECC@Initializing?5DirectInput?4?4?4?6?$AA@ 004c49e4     win_input.obj
 0002:00008a04       ??_C@_08EEBOBCCE@in_mouse?$AA@ 004c4a04     win_input.obj
 0002:00008a10       ??_C@_02PGHGPEOM@?91?$AA@  004c4a10     win_input.obj
 0002:00008a14       ??_C@_0CI@FHJNIMCC@Falling?5back?5to?5Win32?5mouse?5supp@ 004c4a14     win_input.obj
 0002:00008a3c       ??_C@_0DA@FHIPFOFL@No?5window?5for?5DirectInput?5mouse?5@ 004c4a3c     win_input.obj
 0002:00008a6c       ??_C@_0CA@JLJBCBHD@Skipping?5check?5for?5DirectInput?6?$AA@ 004c4a6c     win_input.obj
 0002:00008a8c       ??_C@_0CD@NBEAJIAO@Disallowing?5DirectInput?5on?5NT?54?4@ 004c4a8c     win_input.obj
 0002:00008ab0       ??_C@_0BL@CONMJMEO@Mouse?5control?5not?5active?4?6?$AA@ 004c4ab0     win_input.obj
 0002:00008acc       ??_C@_0CH@JLLNFJIJ@?6?9?9?9?9?9?9?9?5Input?5Initialization?5?9?9@ 004c4acc     win_input.obj
 0002:00008af4       ??_C@_08MKJIFFKA@midiinfo?$AA@ 004c4af4     win_input.obj
 0002:00008b00       ??_C@_0O@CDIHIFMG@joy_threshold?$AA@ 004c4b00     win_input.obj
 0002:00008b10       ??_C@_04FPIJCFHI@0?415?$AA@ 004c4b10     win_input.obj
 0002:00008b18       ??_C@_0BB@KLDPJBGL@in_debugjoystick?$AA@ 004c4b18     win_input.obj
 0002:00008b2c       ??_C@_0BA@FGPJKNGC@in_joyBallScale?$AA@ 004c4b2c     win_input.obj
 0002:00008b3c       ??_C@_04BBAKNJII@0?402?$AA@ 004c4b3c     win_input.obj
 0002:00008b44       ??_C@_0M@MJEIGFNL@in_joystick?$AA@ 004c4b44     win_input.obj
 0002:00008b50       ??_C@_0P@GHEMCIPL@in_logitechbug?$AA@ 004c4b50     win_input.obj
 0002:00008b60       ??_C@_0P@JPEONNIO@in_midichannel?$AA@ 004c4b60     win_input.obj
 0002:00008b70       ??_C@_0M@MPFHODKD@in_midiport?$AA@ 004c4b70     win_input.obj
 0002:00008b7c       ??_C@_07DDONFNPJ@3dfxvgl?$AA@ 004c4b7c     win_input.obj
 0002:00008b84       ??_C@_0L@LKKCCEBO@r_glDriver?$AA@ 004c4b84     win_input.obj
 0002:00008b90       ??_C@_0N@JILGCMBC@r_fullscreen?$AA@ 004c4b90     win_input.obj
 0002:00008ba0       ??_C@_0CE@IAFBHFFK@Proceeding?5with?5delayed?5mouse?5in@ 004c4ba0     win_input.obj
 0002:00008bc4       ??_C@_05BMGBEOOC@?$CFs?2?$CFs?$AA@ 004c4bc4     win_main.obj
 0002:00008bcc       ??_C@_04EDLLLMBI@?$CFs?2?$CK?$AA@ 004c4bcc     win_main.obj
 0002:00008bd4       ??_C@_07PHOBPKGE@?$CFs?2?$CFs?2?$CK?$AA@ 004c4bd4     win_main.obj
 0002:00008bdc       ??_C@_06HKFIIKHL@?$CFs?2?$CK?$CFs?$AA@ 004c4bdc     win_main.obj
 0002:00008be4       ??_C@_0BC@PEIHHIKI@bin?2x86?2glibc?92?41?$AA@ 004c4be4     win_main.obj
 0002:00008bf8       ??_C@_01KDCPPGHE@r?$AA@    004c4bf8     win_main.obj
 0002:00008bfc       ??_C@_0L@BGCMICOJ@quake3?4exe?$AA@ 004c4bfc     win_main.obj
 0002:00008c08       ??_C@_06IBGBCFGI@quake3?$AA@ 004c4c08     win_main.obj
 0002:00008c10       ??_C@_03HBAHNJNM@?6?$AN?$AI?$AA@ 004c4c10     win_main.obj
 0002:00008c14       ??_C@_0CB@NFLEJIB@Sys_UnloadDll?5FreeLibrary?5failed@ 004c4c14     win_main.obj
 0002:00008c38       ??_C@_06MGMAGDAM@vmMain?$AA@ 004c4c38     win_main.obj
 0002:00008c40       ??_C@_08OHGJLDCF@dllEntry?$AA@ 004c4c40     win_main.obj
 0002:00008c50       ??_C@_0MP@OOOFDFBE@You?5are?5about?5to?5load?5a?5?4DLL?5exe@ 004c4c50     win_main.obj
 0002:00008d20       ??_C@_0BB@MEBOOCBB@Security?5Warning?$AA@ 004c4d20     win_main.obj
 0002:00008d34       ??_C@_0BE@FKPJANIK@com_blindlyLoadDLLs?$AA@ 004c4d34     win_main.obj
 0002:00008d48       ??_C@_09IAFMCHD@?$CFsx86?4dll?$AA@ 004c4d48     win_main.obj
 0002:00008d54       ??_C@_0BI@PJPKIIL@Sys_QueEvent?3?5overflow?6?$AA@ 004c4d54     win_main.obj
 0002:00008d6c       ??_C@_08ODGEKKOL@username?$AA@ 004c4d6c     win_main.obj
 0002:00008d78       ??_C@_09MHINEACI@sys_cpuid?$AA@ 004c4d78     win_main.obj
 0002:00008d84       ??_C@_0CF@BFIMMDPC@WARNING?3?5unknown?5sys_cpustring?5?8@ 004c4d84     win_main.obj
 0002:00008dac       ??_C@_03CIPMPAJL@axp?$AA@  004c4dac     win_main.obj
 0002:00008db0       ??_C@_0L@PLDMOKFD@PentiumIII?$AA@ 004c4db0     win_main.obj
 0002:00008dbc       ??_C@_05FIGNBJMO@3dnow?$AA@ 004c4dbc     win_main.obj
 0002:00008dc4       ??_C@_03LABOKELA@mmx?$AA@  004c4dc4     win_main.obj
 0002:00008dc8       ??_C@_03MKEPLMIM@x87?$AA@  004c4dc8     win_main.obj
 0002:00008dcc       ??_C@_0BI@JHAKIADL@?4?4?4forcing?5CPU?5type?5to?5?$AA@ 004c4dcc     win_main.obj
 0002:00008de4       ??_C@_0BF@GOCLOPNN@Unknown?5cpu?5type?5?$CFd?6?$AA@ 004c4de4     win_main.obj
 0002:00008dfc       ??_C@_09DKIGPEEK@Alpha?5AXP?$AA@ 004c4dfc     win_main.obj
 0002:00008e08       ??_C@_0O@FJOEEOAJ@AMD?5w?1?53DNow?$CB?$AA@ 004c4e08     win_main.obj
 0002:00008e18       ??_C@_0BC@EEDJECOE@Intel?5Pentium?5III?$AA@ 004c4e18     win_main.obj
 0002:00008e2c       ??_C@_0BH@CIDJJMAD@x86?5?$CIP5?1Pentium2?0?5MMX?$CJ?$AA@ 004c4e2c     win_main.obj
 0002:00008e44       ??_C@_0BH@DEPNLFPE@x86?5?$CIP5?1PPro?0?5non?9MMX?$CJ?$AA@ 004c4e44     win_main.obj
 0002:00008e5c       ??_C@_0BC@MJACFOKB@x86?5?$CIpre?9Pentium?$CJ?$AA@ 004c4e5c     win_main.obj
 0002:00008e70       ??_C@_07DCLBNMLN@generic?$AA@ 004c4e70     win_main.obj
 0002:00008e78       ??_C@_0BJ@GBJNEBBH@?4?4?4detecting?5CPU?0?5found?5?$AA@ 004c4e78     win_main.obj
 0002:00008e94       ??_C@_0O@PDIAGKHD@sys_cpustring?$AA@ 004c4e94     win_main.obj
 0002:00008ea4       ??_C@_06EEDLFOCL@detect?$AA@ 004c4ea4     win_main.obj
 0002:00008eac       ??_C@_0M@EGGCJNOO@win_wndproc?$AA@ 004c4eac     win_main.obj
 0002:00008eb8       ??_C@_0O@JFLHKJDK@win_hinstance?$AA@ 004c4eb8     win_main.obj
 0002:00008ec8       ??_C@_04LLAMKKNO@arch?$AA@ 004c4ec8     win_main.obj
 0002:00008ed0       ??_C@_0BI@LPAECBNN@unknown?5Windows?5variant?$AA@ 004c4ed0     win_main.obj
 0002:00008ee8       ??_C@_05JOEKOKIA@win95?$AA@ 004c4ee8     win_main.obj
 0002:00008ef0       ??_C@_0N@HFCODOMN@win95?5osr2?4x?$AA@ 004c4ef0     win_main.obj
 0002:00008f00       ??_C@_05CLOEJEMN@win98?$AA@ 004c4f00     win_main.obj
 0002:00008f08       ??_C@_05BONLKMPB@winnt?$AA@ 004c4f08     win_main.obj
 0002:00008f10       ??_C@_0BN@CHAFMCKP@Quake3?5doesn?8t?5run?5on?5Win32s?$AA@ 004c4f10     win_main.obj
 0002:00008f30       ??_C@_0CN@HNJMBKHO@Quake3?5requires?5Windows?5version?5@ 004c4f30     win_main.obj
 0002:00008f60       ??_C@_0BF@JBGMMOFJ@Couldn?8t?5get?5OS?5info?$AA@ 004c4f60     win_main.obj
 0002:00008f78       ??_C@_0M@BPCAELNM@net_restart?$AA@ 004c4f78     win_main.obj
 0002:00008f84       ??_C@_0L@PEIHAAKP@in_restart?$AA@ 004c4f84     win_main.obj
 0002:00008f90       ??_C@_0BH@ECMEJIDF@Working?5directory?3?5?$CFs?6?$AA@ 004c4f90     win_main.obj
 0002:00008fa8       ??_C@_0N@LHDAEOPK@WSATRY_AGAIN?$AA@ 004c4fa8     win_net.obj
 0002:00008fb8       ??_C@_0P@HLNEBJNJ@WSANO_RECOVERY?$AA@ 004c4fb8     win_net.obj
 0002:00008fc8       ??_C@_0L@CBLHPKCP@WSANO_DATA?$AA@ 004c4fc8     win_net.obj
 0002:00008fd4       ??_C@_08LPKPOPGP@NO?5ERROR?$AA@ 004c4fd4     win_net.obj
 0002:00008fe0       ??_C@_0BC@JCJCFNAO@WSAHOST_NOT_FOUND?$AA@ 004c4fe0     win_net.obj
 0002:00008ff4       ??_C@_0BD@PKACBPOA@WSAVERNOTSUPPORTED?$AA@ 004c4ff4     win_net.obj
 0002:00009008       ??_C@_0BC@CLCHBKPK@WSANOTINITIALISED?$AA@ 004c5008     win_net.obj
 0002:0000901c       ??_C@_0L@EEHHIAEC@WSAEDISCON?$AA@ 004c501c     win_net.obj
 0002:00009028       ??_C@_0P@MDJAKAKC@WSASYSNOTREADY?$AA@ 004c5028     win_net.obj
 0002:00009038       ??_C@_0N@NJBKCOKK@WSAEHOSTDOWN?$AA@ 004c5038     win_net.obj
 0002:00009048       ??_C@_0BA@PCKIJCGI@WSAENAMETOOLONG?$AA@ 004c5048     win_net.obj
 0002:00009058       ??_C@_08PGIMLMFD@WSAELOOP?$AA@ 004c5058     win_net.obj
 0002:00009064       ??_C@_0BA@ECEEDLKJ@WSAECONNREFUSED?$AA@ 004c5064     win_net.obj
 0002:00009074       ??_C@_0N@BJEDIOFA@WSAETIMEDOUT?$AA@ 004c5074     win_net.obj
 0002:00009084       ??_C@_0BA@COKPFEMB@WSAETOOMANYREFS?$AA@ 004c5084     win_net.obj
 0002:00009094       ??_C@_0N@JOJKMOCF@WSAESHUTDOWN?$AA@ 004c5094     win_net.obj
 0002:000090a4       ??_C@_0M@BJHJCMPN@WSAENOTCONN?$AA@ 004c50a4     win_net.obj
 0002:000090b0       ??_C@_0L@KMBJICHC@WSAEISCONN?$AA@ 004c50b0     win_net.obj
 0002:000090bc       ??_C@_0L@OOBBNNPD@WSAENOBUFS?$AA@ 004c50bc     win_net.obj
 0002:000090c8       ??_C@_0O@CIPFFFJE@WSAECONNRESET?$AA@ 004c50c8     win_net.obj
 0002:000090d8       ??_C@_0BI@NPIHFCBB@WSWSAECONNABORTEDAEINTR?$AA@ 004c50d8     win_net.obj
 0002:000090f0       ??_C@_0N@KABONKCJ@WSAENETRESET?$AA@ 004c50f0     win_net.obj
 0002:00009100       ??_C@_0P@MMGFNLEA@WSAENETUNREACH?$AA@ 004c5100     win_net.obj
 0002:00009110       ??_C@_0M@BMNODHFM@WSAENETDOWN?$AA@ 004c5110     win_net.obj
 0002:0000911c       ??_C@_0BB@MBBPJMGK@WSAEADDRNOTAVAIL?$AA@ 004c511c     win_net.obj
 0002:00009130       ??_C@_0O@OPDDJBEB@WSAEADDRINUSE?$AA@ 004c5130     win_net.obj
 0002:00009140       ??_C@_0BA@DNDGDCNF@WSAEAFNOSUPPORT?$AA@ 004c5140     win_net.obj
 0002:00009150       ??_C@_0BA@KKILJDEG@WSAEPFNOSUPPORT?$AA@ 004c5150     win_net.obj
 0002:00009160       ??_C@_0O@IFNEEJHC@WSAEOPNOTSUPP?$AA@ 004c5160     win_net.obj
 0002:00009170       ??_C@_0BD@KNONLHOA@WSAESOCKTNOSUPPORT?$AA@ 004c5170     win_net.obj
 0002:00009184       ??_C@_0BD@EDJBJFH@WSAEPROTONOSUPPORT?$AA@ 004c5184     win_net.obj
 0002:00009198       ??_C@_0P@KODINEND@WSAENOPROTOOPT?$AA@ 004c5198     win_net.obj
 0002:000091a8       ??_C@_0O@HCKGAENP@WSAEPROTOTYPE?$AA@ 004c51a8     win_net.obj
 0002:000091b8       ??_C@_0M@PJKLHKI@WSAEMSGSIZE?$AA@ 004c51b8     win_net.obj
 0002:000091c4       ??_C@_0BA@BLGPIJAD@WSAEDESTADDRREQ?$AA@ 004c51c4     win_net.obj
 0002:000091d4       ??_C@_0M@MDGNMGJ@WSAENOTSOCK?$AA@ 004c51d4     win_net.obj
 0002:000091e0       ??_C@_0M@EAGDEEAC@WSAEALREADY?$AA@ 004c51e0     win_net.obj
 0002:000091ec       ??_C@_0P@FHEJEBJC@WSAEINPROGRESS?$AA@ 004c51ec     win_net.obj
 0002:000091fc       ??_C@_0P@BLDHJENA@WSAEWOULDBLOCK?$AA@ 004c51fc     win_net.obj
 0002:0000920c       ??_C@_09IJIBIDKO@WSAEMFILE?$AA@ 004c520c     win_net.obj
 0002:00009218       ??_C@_09PDAAOFKK@WSAEINVAL?$AA@ 004c5218     win_net.obj
 0002:00009224       ??_C@_09BIHAGEEK@WSAEFAULT?$AA@ 004c5224     win_net.obj
 0002:00009230       ??_C@_09EKFHKCJJ@WSAEACCES?$AA@ 004c5230     win_net.obj
 0002:0000923c       ??_C@_08LJKOCPDH@WSAEBADF?$AA@ 004c523c     win_net.obj
 0002:00009248       ??_C@_08KEJFHKFF@WSAEINTR?$AA@ 004c5248     win_net.obj
 0002:00009254       ??_C@_02NJNOFBBI@?$CFx?$AA@ 004c5254     win_net.obj
 0002:00009258       ??_C@_0BJ@NDNBFPLK@Oversize?5packet?5from?5?$CFs?6?$AA@ 004c5258     win_net.obj
 0002:00009274       ??_C@_0BD@GIOPKJNJ@NET_GetPacket?3?5?$CFs?6?$AA@ 004c5274     win_net.obj
 0002:00009288       ??_C@_0CB@JKHJHNNL@Sys_SendPacket?3?5bad?5address?5type@ 004c5288     win_net.obj
 0002:000092ac       ??_C@_0BE@DDOALEHF@NET_SendPacket?3?5?$CFs?6?$AA@ 004c52ac     win_net.obj
 0002:000092c0       ??_C@_0BB@DIPHJIFE@IP?3?5?$CFi?4?$CFi?4?$CFi?4?$CFi?6?$AA@ 004c52c0     win_net.obj
 0002:000092d4       ??_C@_0CD@BCJMGHPJ@WARNING?3?5UDP_OpenSocket?3?5bind?3?5?$CF@ 004c52d4     win_net.obj
 0002:000092f8       ??_C@_0DG@CIGPJCJC@WARNING?3?5UDP_OpenSocket?3?5setsock@ 004c52f8     win_net.obj
 0002:00009330       ??_C@_0CM@DLFGJOIC@WARNING?3?5UDP_OpenSocket?3?5ioctl?5F@ 004c5330     win_net.obj
 0002:0000935c       ??_C@_0CF@MBEBDLFC@WARNING?3?5UDP_OpenSocket?3?5socket?3@ 004c535c     win_net.obj
 0002:00009384       ??_C@_0CB@EGLAFCKD@Opening?5IP?5socket?3?5localhost?3?$CFi?6@ 004c5384     win_net.obj
 0002:000093a8       ??_C@_0BK@FBACENIG@Opening?5IP?5socket?3?5?$CFs?3?$CFi?6?$AA@ 004c53a8     win_net.obj
 0002:000093c4       ??_C@_0BN@JGAEDBBB@NET_OpenSocks?3?5bad?5response?6?$AA@ 004c53c4     win_net.obj
 0002:000093e4       ??_C@_0CO@JGEDJDD@NET_OpenSocks?3?5relay?5address?5is?5@ 004c53e4     win_net.obj
 0002:00009414       ??_C@_0CD@BALIMEMG@NET_OpenSocks?3?5request?5denied?3?5?$CF@ 004c5414     win_net.obj
 0002:00009438       ??_C@_0BJ@GIBPKBJF@NET_OpenSocks?3?5recv?3?5?$CFs?6?$AA@ 004c5438     win_net.obj
 0002:00009454       ??_C@_0BJ@OMJJFCJN@NET_OpenSocks?3?5send?3?5?$CFs?6?$AA@ 004c5454     win_net.obj
 0002:00009470       ??_C@_0CG@OEEMKDKJ@NET_OpenSocks?3?5authentication?5fa@ 004c5470     win_net.obj
 0002:00009498       ??_C@_0BP@MFAELAIP@NET_OpenSocks?3?5request?5denied?6?$AA@ 004c5498     win_net.obj
 0002:000094b8       ??_C@_0BM@KKEOEFCP@NET_OpenSocks?3?5connect?3?5?$CFs?6?$AA@ 004c54b8     win_net.obj
 0002:000094d8       ??_C@_0EF@JDPHELLH@WARNING?3?5NET_OpenSocks?3?5gethostb@ 004c54d8     win_net.obj
 0002:00009520       ??_C@_0CL@NFJLJMMA@WARNING?3?5NET_OpenSocks?3?5gethostb@ 004c5520     win_net.obj
 0002:0000954c       ??_C@_0CE@LFANBIPO@WARNING?3?5NET_OpenSocks?3?5socket?3?5@ 004c554c     win_net.obj
 0002:00009570       ??_C@_0CF@BHILGHLE@Opening?5connection?5to?5SOCKS?5serv@ 004c5570     win_net.obj
 0002:00009598       ??_C@_0L@CGPAFLOO@Alias?3?5?$CFs?6?$AA@ 004c5598     win_net.obj
 0002:000095a4       ??_C@_0O@CBMKAPKN@Hostname?3?5?$CFs?6?$AA@ 004c55a4     win_net.obj
 0002:000095b4       ??_C@_0CE@KJBINNKI@WARNING?3?5Couldn?8t?5allocate?5IP?5po@ 004c55b4     win_net.obj
 0002:000095d8       ??_C@_08HGBCFGPE@net_port?$AA@ 004c55d8     win_net.obj
 0002:000095e4       ??_C@_06BGCGFJHC@net_ip?$AA@ 004c55e4     win_net.obj
 0002:000095ec       ??_C@_0BP@HGPMDKOP@WARNING?3?5IPX_Socket?3?5bind?3?5?$CFs?6?$AA@ 004c55ec     win_net.obj
 0002:0000960c       ??_C@_0DC@FPOBNHBG@WARNING?3?5IPX_Socket?3?5setsockopt?5@ 004c560c     win_net.obj
 0002:00009640       ??_C@_0CI@DCHMECMH@WARNING?3?5IPX_Socket?3?5ioctl?5FIONB@ 004c5640     win_net.obj
 0002:00009668       ??_C@_0CB@MIADMHKM@WARNING?3?5IPX_Socket?3?5socket?3?5?$CFs?6@ 004c5668     win_net.obj
 0002:0000968c       ??_C@_0BC@POLDBMKP@net_socksPassword?$AA@ 004c568c     win_net.obj
 0002:000096a0       ??_C@_0BC@MGKGECCL@net_socksUsername?$AA@ 004c56a0     win_net.obj
 0002:000096b4       ??_C@_0O@DFGDDOCB@net_socksPort?$AA@ 004c56b4     win_net.obj
 0002:000096c4       ??_C@_04KAIJODKO@1080?$AA@ 004c56c4     win_net.obj
 0002:000096cc       ??_C@_0BA@CEJBNOOE@net_socksServer?$AA@ 004c56cc     win_net.obj
 0002:000096dc       ??_C@_0BB@GKECMOEC@net_socksEnabled?$AA@ 004c56dc     win_net.obj
 0002:000096f0       ??_C@_09OEINMMAE@net_noipx?$AA@ 004c56f0     win_net.obj
 0002:000096fc       ??_C@_09CNLEKFIH@net_noudp?$AA@ 004c56fc     win_net.obj
 0002:00009708       ??_C@_0BF@DNHJMPMJ@Winsock?5Initialized?6?$AA@ 004c5708     win_net.obj
 0002:00009720       ??_C@_0DF@DFODMHFF@WARNING?3?5Winsock?5initialization?5@ 004c5720     win_net.obj
 0002:00009758       ??_C@_06BALNJMNP@player?$AA@ 004c5758     win_shared.obj
 0002:00009760       _CLSID_DirectSound         004c5760     win_snd.obj
 0002:00009770       _CLSID_DirectSound8        004c5770     win_snd.obj
 0002:00009780       _IID_IDirectSound8         004c5780     win_snd.obj
 0002:00009790       _IID_IDirectSound          004c5790     win_snd.obj
 0002:000097a0       ??_C@_0BB@MLKAOHBD@DSERR_BUFFERLOST?$AA@ 004c57a0     win_snd.obj
 0002:000097b4       ??_C@_0BG@FGFOLLAI@DSERR_PRIOLEVELNEEDED?$AA@ 004c57b4     win_snd.obj
 0002:000097cc       ??_C@_0BD@MODBPMIE@DSERR_INVALIDPARAM?$AA@ 004c57cc     win_snd.obj
 0002:000097e0       ??_C@_0BD@CHCMAAJB@DSERR_INVALIDCALLS?$AA@ 004c57e0     win_snd.obj
 0002:000097f4       ??_C@_0BH@JMLLEGNC@?4?4?4freeing?5DSOUND?4DLL?6?$AA@ 004c57f4     win_snd.obj
 0002:0000980c       ??_C@_0BI@ONFOIEFD@?4?4?4releasing?5DS?5object?6?$AA@ 004c580c     win_snd.obj
 0002:00009824       ??_C@_0BN@HLLBEHBP@?4?4?4releasing?5primary?5buffer?6?$AA@ 004c5824     win_snd.obj
 0002:00009844       ??_C@_0CI@NDEOJEHM@?4?4?4stopping?5and?5releasing?5sound?5@ 004c5844     win_snd.obj
 0002:0000986c       ??_C@_0BO@IJKEIGDF@?4?4?4setting?5NORMAL?5coop?5level?6?$AA@ 004c586c     win_snd.obj
 0002:0000988c       ??_C@_0BH@FLIOGFIE@Destroying?5DS?5buffers?6?$AA@ 004c588c     win_snd.obj
 0002:000098a4       ??_C@_0BM@OJIPGJEH@Shutting?5down?5sound?5system?6?$AA@ 004c58a4     win_snd.obj
 0002:000098c0       ??_C@_0DD@BGCOLCPM@SNDDMA_BeginPainting?3?5Lock?5faile@ 004c58c0     win_snd.obj
 0002:000098f4       ??_C@_0CC@OAOFCFJN@Couldn?8t?5get?5sound?5buffer?5status@ 004c58f4     win_snd.obj
 0002:00009918       ??_C@_0CC@PKGMOMAO@sound?5SetCooperativeLevel?5failed@ 004c5918     win_snd.obj
 0002:0000993c       ??_C@_0BI@JNPGMFHC@?$CK?$CK?$CK?5GetCaps?5failed?5?$CK?$CK?$CK?6?$AA@ 004c593c     win_snd.obj
 0002:00009954       ??_C@_0CC@IFPHFPKL@?$CK?$CK?$CK?5Looped?5sound?5play?5failed?5?$CK?$CK?$CK@ 004c5954     win_snd.obj
 0002:00009978       ??_C@_0BJ@HLPNNPFF@forced?5to?5software?4?5?5ok?6?$AA@ 004c5978     win_snd.obj
 0002:00009994       ??_C@_07GLGIIGGC@failed?6?$AA@ 004c5994     win_snd.obj
 0002:0000999c       ??_C@_0BG@MMNAOEAM@locked?5hardware?4?5?5ok?6?$AA@ 004c599c     win_snd.obj
 0002:000099b4       ??_C@_0BP@HGFEGEHO@?4?4?4creating?5secondary?5buffer?3?5?$AA@ 004c59b4     win_snd.obj
 0002:000099d4       ??_C@_0CH@HGNPMEEH@?4?4?4setting?5DSSCL_PRIORITY?5coop?5l@ 004c59d4     win_snd.obj
 0002:000099fc       ??_C@_03DJDALPN@ok?6?$AA@  004c59fc     win_snd.obj
 0002:00009a00       ??_C@_0BK@NKEBHAFI@Initializing?5DirectSound?6?$AA@ 004c5a00     win_snd.obj
 0002:00009a1c       ??_C@_0BI@GGLFCNB@Completed?5successfully?6?$AA@ 004c5a1c     win_snd.obj
 0002:00009a34       ??_C@_0CN@FPBLKFON@Invalid?5visLevel?5?$CFd?5sent?5to?5Sys_@ 004c5a34     win_syscon.obj
 0002:00009a64       ??_C@_06GGHJAEBN@static?$AA@ 004c5a64     win_syscon.obj
 0002:00009a6c       ??_C@_04COAGEIMF@copy?$AA@ 004c5a6c     win_syscon.obj
 0002:00009a74       ??_C@_06HFKPFKMP@button?$AA@ 004c5a74     win_syscon.obj
 0002:00009a7c       ??_C@_04NABONMNG@edit?$AA@ 004c5a7c     win_syscon.obj
 0002:00009a84       ??_C@_0M@KGGAJAJ@Courier?5New?$AA@ 004c5a84     win_syscon.obj
 0002:00009a90       ??_C@_0BA@ODHMOKEJ@Quake?53?5Console?$AA@ 004c5a90     win_syscon.obj
 0002:00009aa0       ??_C@_0O@LCHGAMCF@Q3?5WinConsole?$AA@ 004c5aa0     win_syscon.obj
 0002:00009ab0       ??_C@_0BF@JDMIOBEC@VID_AppActivate?3?5?$CFi?6?$AA@ 004c5ab0     win_wndproc.obj
 0002:00009ac8       ??_C@_0N@DAGNKKMD@vid_restart?6?$AA@ 004c5ac8     win_wndproc.obj
 0002:00009ad8       ??_C@_0BA@NAALPGKC@MSWHEEL_ROLLMSG?$AA@ 004c5ad8     win_wndproc.obj
 0002:00009ae8       ??_C@_08PKOLMEA@vid_ypos?$AA@ 004c5ae8     win_wndproc.obj
 0002:00009af4       ??_C@_08DCMOJFPA@vid_xpos?$AA@ 004c5af4     win_wndproc.obj
 0002:00009b00       ??_C@_0BI@OEAPLIMI@Mode?511?3?5856x480?5?$CIwide?$CJ?$AA@ 004c5b00     renderer:tr_init.obj
 0002:00009b18       ??_C@_0BD@HLKNJPO@Mode?510?3?52048x1536?$AA@ 004c5b18     renderer:tr_init.obj
 0002:00009b2c       ??_C@_0BD@JNNBKNHO@Mode?5?59?3?51600x1200?$AA@ 004c5b2c     renderer:tr_init.obj
 0002:00009b40       ??_C@_0BD@DKPOHKD@Mode?5?58?3?51280x1024?$AA@ 004c5b40     renderer:tr_init.obj
 0002:00009b54       ??_C@_0BC@MHGKJHNA@Mode?5?57?3?51152x864?$AA@ 004c5b54     renderer:tr_init.obj
 0002:00009b68       ??_C@_0BC@HHENFJOI@Mode?5?56?3?51024x768?$AA@ 004c5b68     renderer:tr_init.obj
 0002:00009b7c       ??_C@_0BB@IJBLHFE@Mode?5?55?3?5960x720?$AA@ 004c5b7c     renderer:tr_init.obj
 0002:00009b90       ??_C@_0BB@NNFNOODL@Mode?5?54?3?5800x600?$AA@ 004c5b90     renderer:tr_init.obj
 0002:00009ba4       ??_C@_0BB@LBLJFEKK@Mode?5?53?3?5640x480?$AA@ 004c5ba4     renderer:tr_init.obj
 0002:00009bb8       ??_C@_0BB@BIPDPPJI@Mode?5?52?3?5512x384?$AA@ 004c5bb8     renderer:tr_init.obj
 0002:00009bcc       ??_C@_0BB@MMHLKHAE@Mode?5?51?3?5400x300?$AA@ 004c5bcc     renderer:tr_init.obj
 0002:00009be0       ??_C@_0BB@CPBKKPEN@Mode?5?50?3?5320x240?$AA@ 004c5be0     renderer:tr_init.obj
 0002:00009bf4       ??_C@_0CL@BOALOAHK@WARNING?3?5cvar?5?8?$CFs?8?5out?5of?5range?5@ 004c5bf4     renderer:tr_init.obj
 0002:00009c20       ??_C@_0CL@IJJEPBFD@WARNING?3?5cvar?5?8?$CFs?8?5out?5of?5range?5@ 004c5c20     renderer:tr_init.obj
 0002:00009c4c       ??_C@_0CK@MCFFPBMM@WARNING?3?5cvar?5?8?$CFs?8?5must?5be?5integ@ 004c5c4c     renderer:tr_init.obj
 0002:00009c78       ??_C@_0BD@GFONGFHN@GL_CheckErrors?3?5?$CFs?$AA@ 004c5c78     renderer:tr_init.obj
 0002:00009c8c       ??_C@_0BB@JMBJBKGI@GL_OUT_OF_MEMORY?$AA@ 004c5c8c     renderer:tr_init.obj
 0002:00009ca0       ??_C@_0BD@KAJAFKFC@GL_STACK_UNDERFLOW?$AA@ 004c5ca0     renderer:tr_init.obj
 0002:00009cb4       ??_C@_0BC@DLCDMCHH@GL_STACK_OVERFLOW?$AA@ 004c5cb4     renderer:tr_init.obj
 0002:00009cc8       ??_C@_0BF@NFNGKHIL@GL_INVALID_OPERATION?$AA@ 004c5cc8     renderer:tr_init.obj
 0002:00009ce0       ??_C@_0BB@HDIPJELP@GL_INVALID_VALUE?$AA@ 004c5ce0     renderer:tr_init.obj
 0002:00009cf4       ??_C@_0BA@LLPLHEDK@GL_INVALID_ENUM?$AA@ 004c5cf4     renderer:tr_init.obj
 0002:00009d04       ??_C@_0BJ@GLPJAIDL@screenshots?1shot9999?4tga?$AA@ 004c5d04     renderer:tr_init.obj
 0002:00009d20       ??_C@_0BN@MIOHCEKC@screenshots?1shot?$CFi?$CFi?$CFi?$CFi?4tga?$AA@ 004c5d20     renderer:tr_init.obj
 0002:00009d40       ??_C@_0BJ@JEAMDKOE@screenshots?1shot9999?4jpg?$AA@ 004c5d40     renderer:tr_init.obj
 0002:00009d5c       ??_C@_0BN@DHBCBGHN@screenshots?1shot?$CFi?$CFi?$CFi?$CFi?4jpg?$AA@ 004c5d5c     renderer:tr_init.obj
 0002:00009d7c       ??_C@_09CKEIHHKG@Wrote?5?$CFs?6?$AA@ 004c5d7c     renderer:tr_init.obj
 0002:00009d88       __real@3b2aaaab            004c5d88     renderer:tr_init.obj
 0002:00009d8c       __real@3b000000            004c5d8c     renderer:tr_init.obj
 0002:00009d90       ??_C@_0BC@PIIMIPAI@levelshots?1?$CFs?4tga?$AA@ 004c5d90     renderer:tr_init.obj
 0002:00009da4       ??_C@_0CE@KCEHNJII@ScreenShot?3?5Couldn?8t?5create?5a?5fi@ 004c5da4     renderer:tr_init.obj
 0002:00009dc8       ??_C@_0BD@HBDKKBCK@screenshots?1?$CFs?4tga?$AA@ 004c5dc8     renderer:tr_init.obj
 0002:00009ddc       ??_C@_06MJMIHDAA@silent?$AA@ 004c5ddc     renderer:tr_init.obj
 0002:00009de4       ??_C@_09EFOFPGPE@levelshot?$AA@ 004c5de4     renderer:tr_init.obj
 0002:00009df0       ??_C@_0BD@IOMPJDPF@screenshots?1?$CFs?4jpg?$AA@ 004c5df0     renderer:tr_init.obj
 0002:00009e04       ??_C@_0BC@IFPCCECI@Forcing?5glFinish?6?$AA@ 004c5e04     renderer:tr_init.obj
 0002:00009e18       ??_C@_0CD@ECDDMNLK@Using?5dual?5processor?5acceleratio@ 004c5e18     renderer:tr_init.obj
 0002:00009e3c       ??_C@_0BO@MIJCEOJG@HACK?3?5riva128?5approximations?6?$AA@ 004c5e3c     renderer:tr_init.obj
 0002:00009e5c       ??_C@_0BO@BGGGCGOF@HACK?3?5ragePro?5approximations?6?$AA@ 004c5e5c     renderer:tr_init.obj
 0002:00009e7c       ??_C@_0CL@DPDADBAH@HACK?3?5using?5vertex?5lightmap?5appr@ 004c5e7c     renderer:tr_init.obj
 0002:00009ea8       ??_C@_0BJ@OONJCCFB@compressed?5textures?3?5?$CFs?6?$AA@ 004c5ea8     renderer:tr_init.obj
 0002:00009ec4       ??_C@_0BA@EDNGJAE@texenv?5add?3?5?$CFs?6?$AA@ 004c5ec4     renderer:tr_init.obj
 0002:00009ed4       ??_C@_0BM@JNLAHAFE@compiled?5vertex?5arrays?3?5?$CFs?6?$AA@ 004c5ed4     renderer:tr_init.obj
 0002:00009ef0       ??_C@_0BC@IPPCAGDE@multitexture?3?5?$CFs?6?$AA@ 004c5ef0     renderer:tr_init.obj
 0002:00009f04       ??_C@_0BC@OJIGLCBE@texture?5bits?3?5?$CFd?6?$AA@ 004c5f04     renderer:tr_init.obj
 0002:00009f18       ??_C@_0M@HJDEHNFH@picmip?3?5?$CFd?6?$AA@ 004c5f18     renderer:tr_init.obj
 0002:00009f24       ??_C@_0BB@GDPDBBGK@texturemode?3?5?$CFs?6?$AA@ 004c5f24     renderer:tr_init.obj
 0002:00009f38       ??_C@_0DE@COMDCGLO@multiple?5glColor4ubv?5?$CL?5glTexCoor@ 004c5f38     renderer:tr_init.obj
 0002:00009f6c       ??_C@_0BH@GKJMINED@single?5glDrawElements?6?$AA@ 004c5f6c     renderer:tr_init.obj
 0002:00009f84       ??_C@_05IKLLBJL@none?6?$AA@ 004c5f84     renderer:tr_init.obj
 0002:00009f8c       ??_C@_0BJ@OLJGLICH@multiple?5glArrayElement?6?$AA@ 004c5f8c     renderer:tr_init.obj
 0002:00009fa8       ??_C@_0BH@MKBIGIHK@rendering?5primitives?3?5?$AA@ 004c5fa8     renderer:tr_init.obj
 0002:00009fc0       ??_C@_08IFLGILAF@CPU?3?5?$CFs?6?$AA@ 004c5fc0     renderer:tr_init.obj
 0002:00009fcc       ??_C@_0CH@DOFMLBBC@GAMMA?3?5software?5w?1?5?$CFd?5overbright@ 004c5fcc     renderer:tr_init.obj
 0002:00009ff4       ??_C@_0CH@FPMGOKFJ@GAMMA?3?5hardware?5w?1?5?$CFd?5overbright@ 004c5ff4     renderer:tr_init.obj
 0002:0000a01c       ??_C@_04KNPIFONP@N?1A?6?$AA@ 004c601c     renderer:tr_init.obj
 0002:0000a024       ??_C@_03PMGGPEJJ@?$CFd?6?$AA@ 004c6024     renderer:tr_init.obj
 0002:0000a028       ??_C@_0BJ@PKACHHCP@MODE?3?5?$CFd?0?5?$CFd?5x?5?$CFd?5?$CFs?5hz?3?$AA@ 004c6028     renderer:tr_init.obj
 0002:0000a044       ??_C@_0DJ@HCPGCGMA@?6PIXELFORMAT?3?5color?$CI?$CFd?9bits?$CJ?5Z?$CI?$CF@ 004c6044     renderer:tr_init.obj
 0002:0000a080       ??_C@_0CA@JDLIPENJ@GL_MAX_ACTIVE_TEXTURES_ARB?3?5?$CFd?6?$AA@ 004c6080     renderer:tr_init.obj
 0002:0000a0a0       ??_C@_0BJ@DOKOKCEC@GL_MAX_TEXTURE_SIZE?3?5?$CFd?6?$AA@ 004c60a0     renderer:tr_init.obj
 0002:0000a0bc       ??_C@_0BD@KJCGIEGA@GL_EXTENSIONS?3?5?$CFs?6?$AA@ 004c60bc     renderer:tr_init.obj
 0002:0000a0d0       ??_C@_0BA@IECAGHEM@GL_VERSION?3?5?$CFs?6?$AA@ 004c60d0     renderer:tr_init.obj
 0002:0000a0e0       ??_C@_0BB@GPBJMNCI@GL_RENDERER?3?5?$CFs?6?$AA@ 004c60e0     renderer:tr_init.obj
 0002:0000a0f4       ??_C@_0L@GIACNHMO@fullscreen?$AA@ 004c60f4     renderer:tr_init.obj
 0002:0000a100       ??_C@_08KIHLFLPI@windowed?$AA@ 004c6100     renderer:tr_init.obj
 0002:0000a10c       ??_C@_0BA@JPIMJDLP@?6GL_VENDOR?3?5?$CFs?6?$AA@ 004c610c     renderer:tr_init.obj
 0002:0000a11c       ??_C@_07KOAACKLB@gfxinfo?$AA@ 004c611c     renderer:tr_init.obj
 0002:0000a124       ??_C@_0P@HMAPNEDH@screenshotJPEG?$AA@ 004c6124     renderer:tr_init.obj
 0002:0000a134       ??_C@_0L@CMHOPIGK@screenshot?$AA@ 004c6134     renderer:tr_init.obj
 0002:0000a140       ??_C@_08JNNJIBJE@modelist?$AA@ 004c6140     renderer:tr_init.obj
 0002:0000a14c       ??_C@_09EOKHBMCA@modellist?$AA@ 004c614c     renderer:tr_init.obj
 0002:0000a158       ??_C@_08HGIBIHIO@skinlist?$AA@ 004c6158     renderer:tr_init.obj
 0002:0000a164       ??_C@_0L@LGFNICHF@shaderlist?$AA@ 004c6164     renderer:tr_init.obj
 0002:0000a170       ??_C@_09JBMKNKFJ@imagelist?$AA@ 004c6170     renderer:tr_init.obj
 0002:0000a17c       ??_C@_0P@NIPCLOBB@r_maxpolyverts?$AA@ 004c617c     renderer:tr_init.obj
 0002:0000a18c       ??_C@_0L@CKEBPMHC@r_maxpolys?$AA@ 004c618c     renderer:tr_init.obj
 0002:0000a198       ??_C@_0L@MAOLAFLC@cg_shadows?$AA@ 004c6198     renderer:tr_init.obj
 0002:0000a1a4       ??_C@_0M@LGLKLKOB@r_noportals?$AA@ 004c61a4     renderer:tr_init.obj
 0002:0000a1b0       ??_C@_09OGELGAJA@r_lockpvs?$AA@ 004c61b0     renderer:tr_init.obj
 0002:0000a1bc       ??_C@_0N@EIKBMIBB@r_drawBuffer?$AA@ 004c61bc     renderer:tr_init.obj
 0002:0000a1cc       ??_C@_07KHDMNPGL@GL_BACK?$AA@ 004c61cc     renderer:tr_init.obj
 0002:0000a1d4       ??_C@_0O@BAMKGKDI@r_offsetunits?$AA@ 004c61d4     renderer:tr_init.obj
 0002:0000a1e4       ??_C@_02NNFLKHCP@?92?$AA@  004c61e4     renderer:tr_init.obj
 0002:0000a1e8       ??_C@_0P@MNPHBPLD@r_offsetfactor?$AA@ 004c61e8     renderer:tr_init.obj
 0002:0000a1f8       ??_C@_07CLHDHFMP@r_clear?$AA@ 004c61f8     renderer:tr_init.obj
 0002:0000a200       ??_C@_0O@FPMANPKI@r_shownormals?$AA@ 004c6200     renderer:tr_init.obj
 0002:0000a210       ??_C@_09KIABLACG@r_showsky?$AA@ 004c6210     renderer:tr_init.obj
 0002:0000a21c       ??_C@_0L@FFKAMJAN@r_showtris?$AA@ 004c621c     renderer:tr_init.obj
 0002:0000a228       ??_C@_08IPIKLPHC@r_nobind?$AA@ 004c6228     renderer:tr_init.obj
 0002:0000a234       ??_C@_09GELDECFH@r_logFile?$AA@ 004c6234     renderer:tr_init.obj
 0002:0000a240       ??_C@_09HIPDJBIH@r_verbose?$AA@ 004c6240     renderer:tr_init.obj
 0002:0000a24c       ??_C@_08ILOBJANK@r_speeds?$AA@ 004c624c     renderer:tr_init.obj
 0002:0000a258       ??_C@_0O@EGPFGENM@r_showcluster?$AA@ 004c6258     renderer:tr_init.obj
 0002:0000a268       ??_C@_07IFOJIEEJ@r_novis?$AA@ 004c6268     renderer:tr_init.obj
 0002:0000a270       ??_C@_08GDHICAID@r_nocull?$AA@ 004c6270     renderer:tr_init.obj
 0002:0000a27c       ??_C@_08EKMCNKBJ@r_ignore?$AA@ 004c627c     renderer:tr_init.obj
 0002:0000a288       ??_C@_0P@JAKGJBEE@r_drawentities?$AA@ 004c6288     renderer:tr_init.obj
 0002:0000a298       ??_C@_0M@HGMGOPHP@r_norefresh?$AA@ 004c6298     renderer:tr_init.obj
 0002:0000a2a4       ??_C@_0L@DPLFJPIH@r_lodscale?$AA@ 004c62a4     renderer:tr_init.obj
 0002:0000a2b0       ??_C@_0BC@NCGFPEJB@r_measureOverdraw?$AA@ 004c62b0     renderer:tr_init.obj
 0002:0000a2c4       ??_C@_0O@DPCGOEGM@r_skipBackEnd?$AA@ 004c62c4     renderer:tr_init.obj
 0002:0000a2d4       ??_C@_09NNHMNIOD@r_showSmp?$AA@ 004c62d4     renderer:tr_init.obj
 0002:0000a2e0       ??_C@_0M@PNEBDHMB@r_flareFade?$AA@ 004c62e0     renderer:tr_init.obj
 0002:0000a2ec       ??_C@_01COCBENDE@7?$AA@    004c62ec     renderer:tr_init.obj
 0002:0000a2f0       ??_C@_0M@IGENIJKG@r_flareSize?$AA@ 004c62f0     renderer:tr_init.obj
 0002:0000a2fc       ??_C@_02PMJKFNFC@40?$AA@   004c62fc     renderer:tr_init.obj
 0002:0000a300       ??_C@_0N@KANAPLNL@r_portalOnly?$AA@ 004c6300     renderer:tr_init.obj
 0002:0000a310       ??_C@_0L@GFIPPKI@r_lightmap?$AA@ 004c6310     renderer:tr_init.obj
 0002:0000a31c       ??_C@_0M@BIOFCHNF@r_drawworld?$AA@ 004c631c     renderer:tr_init.obj
 0002:0000a328       ??_C@_0L@IBLKDFNO@r_nocurves?$AA@ 004c6328     renderer:tr_init.obj
 0002:0000a334       ??_C@_0P@IMHHMLJH@r_saveFontData?$AA@ 004c6334     renderer:tr_init.obj
 0002:0000a344       ??_C@_0P@FPGBOPOJ@r_printShaders?$AA@ 004c6344     renderer:tr_init.obj
 0002:0000a354       ??_C@_0M@FAFKFKNC@r_debugSort?$AA@ 004c6354     renderer:tr_init.obj
 0002:0000a360       ??_C@_0N@CLEJOIDB@r_debuglight?$AA@ 004c6360     renderer:tr_init.obj
 0002:0000a370       ??_C@_0N@MJCHINNC@r_showImages?$AA@ 004c6370     renderer:tr_init.obj
 0002:0000a380       ??_C@_0BA@JKEOFBGN@r_directedScale?$AA@ 004c6380     renderer:tr_init.obj
 0002:0000a390       ??_C@_0P@PCFMEOGO@r_ambientScale?$AA@ 004c6390     renderer:tr_init.obj
 0002:0000a3a0       ??_C@_03JFFPCCNN@0?46?$AA@ 004c63a0     renderer:tr_init.obj
 0002:0000a3a4       ??_C@_0N@MNJJLPGP@r_primitives?$AA@ 004c63a4     renderer:tr_init.obj
 0002:0000a3b4       ??_C@_0BE@JCAJHBHI@r_railSegmentLength?$AA@ 004c63b4     renderer:tr_init.obj
 0002:0000a3c8       ??_C@_0BA@KIFPEIFH@r_railCoreWidth?$AA@ 004c63c8     renderer:tr_init.obj
 0002:0000a3d8       ??_C@_01DHDKHMHF@6?$AA@    004c63d8     renderer:tr_init.obj
 0002:0000a3dc       ??_C@_0M@FCDKDOFO@r_railWidth?$AA@ 004c63dc     renderer:tr_init.obj
 0002:0000a3e8       ??_C@_0BA@BPCDNPON@r_facePlaneCull?$AA@ 004c63e8     renderer:tr_init.obj
 0002:0000a3f8       ??_C@_07OFDDGDHB@r_gamma?$AA@ 004c63f8     renderer:tr_init.obj
 0002:0000a400       ??_C@_0P@HNMDPIEI@r_swapInterval?$AA@ 004c6400     renderer:tr_init.obj
 0002:0000a410       ??_C@_0O@BGKNIDHM@r_textureMode?$AA@ 004c6410     renderer:tr_init.obj
 0002:0000a420       ??_C@_0BJ@PCPDHFJH@GL_LINEAR_MIPMAP_NEAREST?$AA@ 004c6420     renderer:tr_init.obj
 0002:0000a43c       ??_C@_08BHIHIACG@r_finish?$AA@ 004c643c     renderer:tr_init.obj
 0002:0000a448       ??_C@_0O@PLDNGPHO@r_dlightBacks?$AA@ 004c6448     renderer:tr_init.obj
 0002:0000a458       ??_C@_0P@CEODIJEF@r_dynamiclight?$AA@ 004c6458     renderer:tr_init.obj
 0002:0000a468       ??_C@_09JENCIPDG@r_drawSun?$AA@ 004c6468     renderer:tr_init.obj
 0002:0000a474       ??_C@_09DKHGHCIK@r_fastsky?$AA@ 004c6474     renderer:tr_init.obj
 0002:0000a480       ??_C@_0BB@FAMAENF@r_ignoreGLErrors?$AA@ 004c6480     renderer:tr_init.obj
 0002:0000a494       ??_C@_07HFGKHFPM@r_znear?$AA@ 004c6494     renderer:tr_init.obj
 0002:0000a49c       ??_C@_08PDJPECIC@r_flares?$AA@ 004c649c     renderer:tr_init.obj
 0002:0000a4a8       ??_C@_09MCCGJPLJ@r_lodbias?$AA@ 004c64a8     renderer:tr_init.obj
 0002:0000a4b4       ??_C@_0BA@EEHBLFFN@r_lodCurveError?$AA@ 004c64b4     renderer:tr_init.obj
 0002:0000a4c4       ??_C@_03HJHPABEB@250?$AA@  004c64c4     renderer:tr_init.obj
 0002:0000a4c8       ??_C@_0P@ODPAICMO@r_singleShader?$AA@ 004c64c8     renderer:tr_init.obj
 0002:0000a4d8       ??_C@_0M@IIHNMIDC@r_intensity?$AA@ 004c64d8     renderer:tr_init.obj
 0002:0000a4e4       ??_C@_0BE@MNKOGJGK@r_mapOverBrightBits?$AA@ 004c64e4     renderer:tr_init.obj
 0002:0000a4f8       ??_C@_0N@JEFJGNMG@r_fullbright?$AA@ 004c64f8     renderer:tr_init.obj
 0002:0000a508       ??_C@_0BB@FFCENIEG@r_displayRefresh?$AA@ 004c6508     renderer:tr_init.obj
 0002:0000a51c       ??_C@_0BB@JLILKIBL@r_ignoreFastPath?$AA@ 004c651c     renderer:tr_init.obj
 0002:0000a530       ??_C@_05KECOIEHL@r_smp?$AA@ 004c6530     renderer:tr_init.obj
 0002:0000a538       ??_C@_0P@CEFBGCNE@r_subdivisions?$AA@ 004c6538     renderer:tr_init.obj
 0002:0000a548       ??_C@_0P@BJDDOIJN@r_uifullscreen?$AA@ 004c6548     renderer:tr_init.obj
 0002:0000a558       ??_C@_0O@LOOKMMOO@r_vertexLight?$AA@ 004c6558     renderer:tr_init.obj
 0002:0000a568       ??_C@_0BA@MPIFMBGH@r_simpleMipMaps?$AA@ 004c6568     renderer:tr_init.obj
 0002:0000a578       ??_C@_0P@PMHAFEHO@r_customaspect?$AA@ 004c6578     renderer:tr_init.obj
 0002:0000a588       ??_C@_0P@HHMLCCLC@r_customheight?$AA@ 004c6588     renderer:tr_init.obj
 0002:0000a598       ??_C@_04MJHCKDHM@1024?$AA@ 004c6598     renderer:tr_init.obj
 0002:0000a5a0       ??_C@_0O@EAAAAJJP@r_customwidth?$AA@ 004c65a0     renderer:tr_init.obj
 0002:0000a5b0       ??_C@_04ILPBONMK@1600?$AA@ 004c65b0     renderer:tr_init.obj
 0002:0000a5b8       ??_C@_06LBAPPDBG@r_mode?$AA@ 004c65b8     renderer:tr_init.obj
 0002:0000a5c0       ??_C@_0BA@EIFIPMEJ@r_ignorehwgamma?$AA@ 004c65c0     renderer:tr_init.obj
 0002:0000a5d0       ??_C@_0BB@FCPGIIJJ@r_overBrightBits?$AA@ 004c65d0     renderer:tr_init.obj
 0002:0000a5e4       ??_C@_0M@MLADPBHK@r_depthbits?$AA@ 004c65e4     renderer:tr_init.obj
 0002:0000a5f0       ??_C@_0O@HILFODLB@r_stencilbits?$AA@ 004c65f0     renderer:tr_init.obj
 0002:0000a600       ??_C@_08DKALIKIA@r_stereo?$AA@ 004c6600     renderer:tr_init.obj
 0002:0000a60c       ??_C@_0M@FAHBKNDA@r_colorbits?$AA@ 004c660c     renderer:tr_init.obj
 0002:0000a618       ??_C@_0O@HAOJHCNC@r_texturebits?$AA@ 004c6618     renderer:tr_init.obj
 0002:0000a628       ??_C@_0BB@OJJFINJB@r_detailtextures?$AA@ 004c6628     renderer:tr_init.obj
 0002:0000a63c       ??_C@_0BB@PCBDDBLH@r_colorMipLevels?$AA@ 004c663c     renderer:tr_init.obj
 0002:0000a650       ??_C@_0BC@PNEOFHC@r_roundImagesDown?$AA@ 004c6650     renderer:tr_init.obj
 0002:0000a664       ??_C@_08PHNBMEML@r_picmip?$AA@ 004c6664     renderer:tr_init.obj
 0002:0000a670       ??_C@_0BG@OKHMCNAA@r_ext_texture_env_add?$AA@ 004c6670     renderer:tr_init.obj
 0002:0000a688       ??_C@_0BM@FKPHHJJN@r_ext_compiled_vertex_array?$AA@ 004c6688     renderer:tr_init.obj
 0002:0000a6a4       ??_C@_0BD@DEGOFCOI@r_ext_multitexture?$AA@ 004c66a4     renderer:tr_init.obj
 0002:0000a6b8       ??_C@_0BE@GKOFPKJD@r_ext_gamma_control?$AA@ 004c66b8     renderer:tr_init.obj
 0002:0000a6cc       ??_C@_0BK@GPIDLLEE@r_ext_compressed_textures?$AA@ 004c66cc     renderer:tr_init.obj
 0002:0000a6e8       ??_C@_0BC@HJALDEG@r_allowExtensions?$AA@ 004c66e8     renderer:tr_init.obj
 0002:0000a6fc       ??_C@_08EMLDNFIC@opengl32?$AA@ 004c66fc     renderer:tr_init.obj
 0002:0000a708       ??_C@_0M@KILDDLLK@shaderstate?$AA@ 004c6708     renderer:tr_init.obj
 0002:0000a714       ??_C@_0BD@IGCMANBD@RE_Shutdown?$CI?5?$CFi?5?$CJ?6?$AA@ 004c6714     renderer:tr_init.obj
 0002:0000a728       ??_C@_0DB@JNEJBLCB@Mismatched?5REF_API_VERSION?3?5expe@ 004c6728     renderer:tr_init.obj
 0002:0000a75c       ??_C@_0BN@PMHALLBM@?9?9?9?9?9?5finished?5R_Init?5?9?9?9?9?9?6?$AA@ 004c675c     renderer:tr_init.obj
 0002:0000a77c       ??_C@_0BF@GNBIIAHE@glGetError?$CI?$CJ?5?$DN?50x?$CFx?6?$AA@ 004c677c     renderer:tr_init.obj
 0002:0000a794       __real@3b800000            004c6794     renderer:tr_init.obj
 0002:0000a798       __real@3a800000            004c6798     renderer:tr_init.obj
 0002:0000a79c       __real@3eb42d0b            004c679c     renderer:tr_init.obj
 0002:0000a7a0       ??_C@_0CH@LEDEAOCO@WARNING?3?5tess?4xyz?5not?516?5byte?5al@ 004c67a0     renderer:tr_init.obj
 0002:0000a7c8       ??_C@_0BE@MDHPNILD@?9?9?9?9?9?5R_Init?5?9?9?9?9?9?6?$AA@ 004c67c8     renderer:tr_init.obj
 0002:0000a7dc       __real@c0000000            004c67dc     renderer:tr_main.obj
 0002:0000a7e0       __real@3c0efa35            004c67e0     renderer:tr_main.obj
 0002:0000a7e4       __real@3b449ba6            004c67e4     renderer:tr_main.obj
 0002:0000a7e8       __real@3a83126f            004c67e8     renderer:tr_main.obj
 0002:0000a7ec       __real@c2800000            004c67ec     renderer:tr_main.obj
 0002:0000a7f0       __real@42800000            004c67f0     renderer:tr_main.obj
 0002:0000a7f4       ??_C@_0CA@HFCHICEL@R_AddEntitySurfaces?3?5Bad?5reType?$AA@ 004c67f4     renderer:tr_main.obj
 0002:0000a814       ??_C@_0CD@MFJALMLM@R_AddEntitySurfaces?3?5Bad?5modelty@ 004c6814     renderer:tr_main.obj
 0002:0000a838       ??_C@_0CI@MGFPEFGD@WARNING?3?5recursive?5mirror?1portal@ 004c6838     renderer:tr_main.obj
 0002:0000a860       ??_C@_0BP@DEDPBGDJ@Shader?5?8?$CFs?8with?5sort?5?$DN?$DN?5SS_BAD?$AA@ 004c6860     renderer:tr_main.obj
 0002:0000a880       ??_C@_0BJ@JDBKNKDM@OUT?5OF?5RANGE?5FOR?5BOOLEAN?$AA@ 004c6880     renderer:win_qgl.obj
 0002:0000a89c       ??_C@_07IMBILHHE@GL_TRUE?$AA@ 004c689c     renderer:win_qgl.obj
 0002:0000a8a4       ??_C@_08IGAOJPMH@GL_FALSE?$AA@ 004c68a4     renderer:win_qgl.obj
 0002:0000a8b0       ??_C@_0BA@GHBGOAFD@?$CB?$CB?$CB?5UNKNOWN?5?$CB?$CB?$CB?$AA@ 004c68b0     renderer:win_qgl.obj
 0002:0000a8c0       ??_C@_0M@OOEKJBLI@GL_NOTEQUAL?$AA@ 004c68c0     renderer:win_qgl.obj
 0002:0000a8cc       ??_C@_09NOLOLEBE@GL_GEQUAL?$AA@ 004c68cc     renderer:win_qgl.obj
 0002:0000a8d8       ??_C@_0L@FFMBBKLC@GL_GREATER?$AA@ 004c68d8     renderer:win_qgl.obj
 0002:0000a8e4       ??_C@_08IDALKOKJ@GL_EQUAL?$AA@ 004c68e4     renderer:win_qgl.obj
 0002:0000a8f0       ??_C@_07JFDMNHE@GL_LESS?$AA@ 004c68f0     renderer:win_qgl.obj
 0002:0000a8f8       ??_C@_09NMLJOAOO@GL_LEQUAL?$AA@ 004c68f8     renderer:win_qgl.obj
 0002:0000a904       ??_C@_08LNFBFHMF@GL_NEVER?$AA@ 004c6904     renderer:win_qgl.obj
 0002:0000a910       ??_C@_09BFDFBJNI@GL_ALWAYS?$AA@ 004c6910     renderer:win_qgl.obj
 0002:0000a91c       ??_C@_04OPBHEPOC@0x?$CFx?$AA@ 004c691c     renderer:win_qgl.obj
 0002:0000a924       ??_C@_0N@FABIPFMG@GL_LINE_LOOP?$AA@ 004c6924     renderer:win_qgl.obj
 0002:0000a934       ??_C@_0O@JMNICDEE@GL_LINE_STRIP?$AA@ 004c6934     renderer:win_qgl.obj
 0002:0000a944       ??_C@_08LJNPFFPO@GL_LINES?$AA@ 004c6944     renderer:win_qgl.obj
 0002:0000a950       ??_C@_09NNGDFGOK@GL_POINTS?$AA@ 004c6950     renderer:win_qgl.obj
 0002:0000a95c       ??_C@_0L@PLGFHCPP@GL_POLYGON?$AA@ 004c695c     renderer:win_qgl.obj
 0002:0000a968       ??_C@_0O@NHDLAEKB@GL_QUAD_STRIP?$AA@ 004c6968     renderer:win_qgl.obj
 0002:0000a978       ??_C@_08PKCGEEFJ@GL_QUADS?$AA@ 004c6978     renderer:win_qgl.obj
 0002:0000a984       ??_C@_0BA@JPEIIGD@GL_TRIANGLE_FAN?$AA@ 004c6984     renderer:win_qgl.obj
 0002:0000a994       ??_C@_0BC@IJJHLCGE@GL_TRIANGLE_STRIP?$AA@ 004c6994     renderer:win_qgl.obj
 0002:0000a9a8       ??_C@_0N@DPCLFMKI@GL_TRIANGLES?$AA@ 004c69a8     renderer:win_qgl.obj
 0002:0000a9b8       ??_C@_0BH@LLLOJEAO@GL_TEXTURE_COORD_ARRAY?$AA@ 004c69b8     renderer:win_qgl.obj
 0002:0000a9d0       ??_C@_0P@IEOMEBHC@GL_COLOR_ARRAY?$AA@ 004c69d0     renderer:win_qgl.obj
 0002:0000a9e0       ??_C@_0P@NHDEGKDG@GL_CLIP_PLANE0?$AA@ 004c69e0     renderer:win_qgl.obj
 0002:0000a9f0       ??_C@_0BA@JFHJMJII@GL_VERTEX_ARRAY?$AA@ 004c69f0     renderer:win_qgl.obj
 0002:0000aa00       ??_C@_0O@ELNGFGOK@GL_TEXTURE_2D?$AA@ 004c6a00     renderer:win_qgl.obj
 0002:0000aa10       ??_C@_0BA@OMMJCFDD@GL_STENCIL_TEST?$AA@ 004c6a10     renderer:win_qgl.obj
 0002:0000aa20       ??_C@_0O@LGFCICFJ@GL_ALPHA_TEST?$AA@ 004c6a20     renderer:win_qgl.obj
 0002:0000aa30       ??_C@_0N@KIJKCNGC@GL_CULL_FACE?$AA@ 004c6a30     renderer:win_qgl.obj
 0002:0000aa40       ??_C@_0O@IFJMGEGG@GL_DEPTH_TEST?$AA@ 004c6a40     renderer:win_qgl.obj
 0002:0000aa50       ??_C@_08JFOCFHII@GL_BLEND?$AA@ 004c6a50     renderer:win_qgl.obj
 0002:0000aa5c       ??_C@_09KPJJGMBD@GL_DOUBLE?$AA@ 004c6a5c     renderer:win_qgl.obj
 0002:0000aa68       ??_C@_08CAFAKAJG@GL_FLOAT?$AA@ 004c6a68     renderer:win_qgl.obj
 0002:0000aa74       ??_C@_0BA@IMMELLJG@GL_UNSIGNED_INT?$AA@ 004c6a74     renderer:win_qgl.obj
 0002:0000aa84       ??_C@_06GDCJNGFG@GL_INT?$AA@ 004c6a84     renderer:win_qgl.obj
 0002:0000aa8c       ??_C@_0BC@GAFCKNBB@GL_UNSIGNED_SHORT?$AA@ 004c6a8c     renderer:win_qgl.obj
 0002:0000aaa0       ??_C@_08JIKLIIFH@GL_SHORT?$AA@ 004c6aa0     renderer:win_qgl.obj
 0002:0000aaac       ??_C@_0BB@COPABHLN@GL_UNSIGNED_BYTE?$AA@ 004c6aac     renderer:win_qgl.obj
 0002:0000aac0       ??_C@_07LFHLDIGA@GL_BYTE?$AA@ 004c6ac0     renderer:win_qgl.obj
 0002:0000aac8       ??_C@_08PCDPFMDL@glAccum?6?$AA@ 004c6ac8     renderer:win_qgl.obj
 0002:0000aad4       ??_C@_0BJ@HDENBGFH@glAlphaFunc?$CI?50x?$CFx?0?5?$CFf?5?$CJ?6?$AA@ 004c6ad4     renderer:win_qgl.obj
 0002:0000aaf0       ??_C@_0BH@BMLLFOBA@glAreTexturesResident?6?$AA@ 004c6af0     renderer:win_qgl.obj
 0002:0000ab08       ??_C@_0BA@NIMHNGKH@glArrayElement?6?$AA@ 004c6b08     renderer:win_qgl.obj
 0002:0000ab18       ??_C@_0P@JLNLBFBE@glBegin?$CI?5?$CFs?5?$CJ?6?$AA@ 004c6b18     renderer:win_qgl.obj
 0002:0000ab28       ??_C@_0BL@HPKHNJKH@glBindTexture?$CI?50x?$CFx?0?5?$CFu?5?$CJ?6?$AA@ 004c6b28     renderer:win_qgl.obj
 0002:0000ab44       ??_C@_09DMBKNKAB@glBitmap?6?$AA@ 004c6b44     renderer:win_qgl.obj
 0002:0000ab50       ??_C@_0N@DDMEICAJ@GL_DST_ALPHA?$AA@ 004c6b50     renderer:win_qgl.obj
 0002:0000ab60       ??_C@_0N@EHMDOGOC@GL_DST_COLOR?$AA@ 004c6b60     renderer:win_qgl.obj
 0002:0000ab70       ??_C@_0BH@GMGAKMMA@GL_ONE_MINUS_DST_COLOR?$AA@ 004c6b70     renderer:win_qgl.obj
 0002:0000ab88       ??_C@_0BH@LMBAHOML@GL_ONE_MINUS_SRC_ALPHA?$AA@ 004c6b88     renderer:win_qgl.obj
 0002:0000aba0       ??_C@_07BEGJIDM@GL_ZERO?$AA@ 004c6ba0     renderer:win_qgl.obj
 0002:0000aba8       ??_C@_06BFJLKKJK@GL_ONE?$AA@ 004c6ba8     renderer:win_qgl.obj
 0002:0000abb0       ??_C@_0N@JHLDDEOJ@GL_SRC_ALPHA?$AA@ 004c6bb0     renderer:win_qgl.obj
 0002:0000abc0       ??_C@_0BH@LNGGJGMM@glBlendFunc?$CI?5?$CFs?0?5?$CFs?5?$CJ?6?$AA@ 004c6bc0     renderer:win_qgl.obj
 0002:0000abd8       ??_C@_0BC@PGBDBDGL@glCallList?$CI?5?$CFu?5?$CJ?6?$AA@ 004c6bd8     renderer:win_qgl.obj
 0002:0000abec       ??_C@_0N@LIOIEBNO@glCallLists?6?$AA@ 004c6bec     renderer:win_qgl.obj
 0002:0000abfc       ??_C@_02MNMNLDAI@?$CJ?6?$AA@ 004c6bfc     renderer:win_qgl.obj
 0002:0000ac00       ??_C@_0BF@BIJIMNGE@GL_ACCUM_BUFFER_BIT?5?$AA@ 004c6c00     renderer:win_qgl.obj
 0002:0000ac18       ??_C@_0BH@KKNFMDIJ@GL_STENCIL_BUFFER_BIT?5?$AA@ 004c6c18     renderer:win_qgl.obj
 0002:0000ac30       ??_C@_0BF@KJOBCEGC@GL_DEPTH_BUFFER_BIT?5?$AA@ 004c6c30     renderer:win_qgl.obj
 0002:0000ac48       ??_C@_0BF@BFPFMDEP@GL_COLOR_BUFFER_BIT?5?$AA@ 004c6c48     renderer:win_qgl.obj
 0002:0000ac60       ??_C@_0BB@IDDIBIDC@glClear?$CI?50x?$CFx?5?$DN?5?$AA@ 004c6c60     renderer:win_qgl.obj
 0002:0000ac74       ??_C@_0O@IIACIDEG@glClearAccum?6?$AA@ 004c6c74     renderer:win_qgl.obj
 0002:0000ac84       ??_C@_0O@MCNBJGHD@glClearColor?6?$AA@ 004c6c84     renderer:win_qgl.obj
 0002:0000ac94       ??_C@_0BE@FCIHELMM@glClearDepth?$CI?5?$CFf?5?$CJ?6?$AA@ 004c6c94     renderer:win_qgl.obj
 0002:0000aca8       ??_C@_0O@PPKHDEOL@glClearIndex?6?$AA@ 004c6ca8     renderer:win_qgl.obj
 0002:0000acb8       ??_C@_0BG@MJOLJGGJ@glClearStencil?$CI?5?$CFd?5?$CJ?6?$AA@ 004c6cb8     renderer:win_qgl.obj
 0002:0000acd0       ??_C@_0N@OBAJGAJH@glClipPlane?6?$AA@ 004c6cd0     renderer:win_qgl.obj
 0002:0000ace0       ??_C@_0L@KNBMCMLJ@glColor3b?6?$AA@ 004c6ce0     renderer:win_qgl.obj
 0002:0000acec       ??_C@_0M@BFBEGOLK@glColor3bv?6?$AA@ 004c6cec     renderer:win_qgl.obj
 0002:0000acf8       ??_C@_0L@KJJBFAAL@glColor3d?6?$AA@ 004c6cf8     renderer:win_qgl.obj
 0002:0000ad04       ??_C@_0M@DAHPDBGG@glColor3dv?6?$AA@ 004c6d04     renderer:win_qgl.obj
 0002:0000ad10       ??_C@_0L@KKBFIEGF@glColor3f?6?$AA@ 004c6d10     renderer:win_qgl.obj
 0002:0000ad1c       ??_C@_0M@JKHGPJON@glColor3fv?6?$AA@ 004c6d1c     renderer:win_qgl.obj
 0002:0000ad28       ??_C@_0L@KBEJMDFI@glColor3i?6?$AA@ 004c6d28     renderer:win_qgl.obj
 0002:0000ad34       ??_C@_0M@MCBFOJLL@glColor3iv?6?$AA@ 004c6d34     renderer:win_qgl.obj
 0002:0000ad40       ??_C@_0L@LAPIOFPO@glColor3s?6?$AA@ 004c6d40     renderer:win_qgl.obj
 0002:0000ad4c       ??_C@_0M@PNLBFOEA@glColor3sv?6?$AA@ 004c6d4c     renderer:win_qgl.obj
 0002:0000ad58       ??_C@_0M@MDPFAKDA@glColor3ub?6?$AA@ 004c6d58     renderer:win_qgl.obj
 0002:0000ad64       ??_C@_0N@IBBOLMBI@glColor3ubv?6?$AA@ 004c6d64     renderer:win_qgl.obj
 0002:0000ad74       ??_C@_0M@MPKAOFNB@glColor3ui?6?$AA@ 004c6d74     renderer:win_qgl.obj
 0002:0000ad80       ??_C@_0N@FGBPDLBJ@glColor3uiv?6?$AA@ 004c6d80     renderer:win_qgl.obj
 0002:0000ad90       ??_C@_0M@NOBBMDHH@glColor3us?6?$AA@ 004c6d90     renderer:win_qgl.obj
 0002:0000ad9c       ??_C@_0N@GJLLIMOC@glColor3usv?6?$AA@ 004c6d9c     renderer:win_qgl.obj
 0002:0000adac       ??_C@_0L@DAMLBEAA@glColor4b?6?$AA@ 004c6dac     renderer:win_qgl.obj
 0002:0000adb8       ??_C@_0M@KHDELCKK@glColor4bv?6?$AA@ 004c6db8     renderer:win_qgl.obj
 0002:0000adc4       ??_C@_0L@DEEGGILC@glColor4d?6?$AA@ 004c6dc4     renderer:win_qgl.obj
 0002:0000add0       ??_C@_0M@ICFPONHG@glColor4dv?6?$AA@ 004c6dd0     renderer:win_qgl.obj
 0002:0000addc       ??_C@_0BK@GLHDEOI@glColor4f?$CI?5?$CFf?0?$CFf?0?$CFf?0?$CFf?5?$CJ?6?$AA@ 004c6ddc     renderer:win_qgl.obj
 0002:0000adf8       ??_C@_0BL@NGEGGGIG@glColor4fv?$CI?5?$CFf?0?$CFf?0?$CFf?0?$CFf?5?$CJ?6?$AA@ 004c6df8     renderer:win_qgl.obj
 0002:0000ae14       ??_C@_0L@DMJOPLOB@glColor4i?6?$AA@ 004c6e14     renderer:win_qgl.obj
 0002:0000ae20       ??_C@_0M@HADFDFKL@glColor4iv?6?$AA@ 004c6e20     renderer:win_qgl.obj
 0002:0000ae2c       ??_C@_0L@CNCPNNEH@glColor4s?6?$AA@ 004c6e2c     renderer:win_qgl.obj
 0002:0000ae38       ??_C@_0M@EPJBICFA@glColor4sv?6?$AA@ 004c6e38     renderer:win_qgl.obj
 0002:0000ae44       ??_C@_0N@JMBLIMKA@glColor4ubv?6?$AA@ 004c6e44     renderer:win_qgl.obj
 0002:0000ae54       ??_C@_0M@HNIADJMB@glColor4ui?6?$AA@ 004c6e54     renderer:win_qgl.obj
 0002:0000ae60       ??_C@_0N@ELBKALKB@glColor4uiv?6?$AA@ 004c6e60     renderer:win_qgl.obj
 0002:0000ae70       ??_C@_0M@GMDBBPGH@glColor4us?6?$AA@ 004c6e70     renderer:win_qgl.obj
 0002:0000ae7c       ??_C@_0N@HELOLMFK@glColor4usv?6?$AA@ 004c6e7c     renderer:win_qgl.obj
 0002:0000ae8c       ??_C@_0N@NJANOBDC@glColorMask?6?$AA@ 004c6e8c     renderer:win_qgl.obj
 0002:0000ae9c       ??_C@_0BB@KJLCDMPM@glColorMaterial?6?$AA@ 004c6e9c     renderer:win_qgl.obj
 0002:0000aeb0       ??_C@_0CD@MDNBONKN@glColorPointer?$CI?5?$CFd?0?5?$CFs?0?5?$CFd?0?5MEM?5@ 004c6eb0     renderer:win_qgl.obj
 0002:0000aed4       ??_C@_0O@FNIGMMMF@glCopyPixels?6?$AA@ 004c6ed4     renderer:win_qgl.obj
 0002:0000aee4       ??_C@_0BC@NAEEIAAJ@glCopyTexImage1D?6?$AA@ 004c6ee4     renderer:win_qgl.obj
 0002:0000aef8       ??_C@_0BC@MCPBCPOH@glCopyTexImage2D?6?$AA@ 004c6ef8     renderer:win_qgl.obj
 0002:0000af0c       ??_C@_0BF@LJHMNDOI@glCopyTexSubImage1D?6?$AA@ 004c6f0c     renderer:win_qgl.obj
 0002:0000af24       ??_C@_0BF@KLMJHMAG@glCopyTexSubImage2D?6?$AA@ 004c6f24     renderer:win_qgl.obj
 0002:0000af3c       ??_C@_0BC@HLKMMCBJ@glCullFace?$CI?5?$CFs?5?$CJ?6?$AA@ 004c6f3c     renderer:win_qgl.obj
 0002:0000af50       ??_C@_08PENMMOEI@GL_FRONT?$AA@ 004c6f50     renderer:win_qgl.obj
 0002:0000af5c       ??_C@_0P@JIJNGNMF@glDeleteLists?6?$AA@ 004c6f5c     renderer:win_qgl.obj
 0002:0000af6c       ??_C@_0BC@PJPFPBNP@glDeleteTextures?6?$AA@ 004c6f6c     renderer:win_qgl.obj
 0002:0000af80       ??_C@_0BD@KINJHKOL@glDepthFunc?$CI?5?$CFs?5?$CJ?6?$AA@ 004c6f80     renderer:win_qgl.obj
 0002:0000af94       ??_C@_0BD@KOOMMBOM@glDepthMask?$CI?5?$CFs?5?$CJ?6?$AA@ 004c6f94     renderer:win_qgl.obj
 0002:0000afa8       ??_C@_0BI@GLOECODG@glDepthRange?$CI?5?$CFf?0?5?$CFf?5?$CJ?6?$AA@ 004c6fa8     renderer:win_qgl.obj
 0002:0000afc0       ??_C@_0BB@JJCKFOMA@glDisable?$CI?5?$CFs?5?$CJ?6?$AA@ 004c6fc0     renderer:win_qgl.obj
 0002:0000afd4       ??_C@_0BM@DMNJOMNK@glDisableClientState?$CI?5?$CFs?5?$CJ?6?$AA@ 004c6fd4     renderer:win_qgl.obj
 0002:0000aff0       ??_C@_0O@KKMGEGEI@glDrawArrays?6?$AA@ 004c6ff0     renderer:win_qgl.obj
 0002:0000b000       ??_C@_0O@NAIEGBKI@glDrawBuffer?6?$AA@ 004c7000     renderer:win_qgl.obj
 0002:0000b010       ??_C@_0CD@GPAGANOP@glDrawElements?$CI?5?$CFs?0?5?$CFd?0?5?$CFs?0?5MEM?5@ 004c7010     renderer:win_qgl.obj
 0002:0000b034       ??_C@_0O@EMNCJNMC@glDrawPixels?6?$AA@ 004c7034     renderer:win_qgl.obj
 0002:0000b044       ??_C@_0M@EJLMLIDA@glEdgeFlag?6?$AA@ 004c7044     renderer:win_qgl.obj
 0002:0000b050       ??_C@_0BD@CIGMNIB@glEdgeFlagPointer?6?$AA@ 004c7050     renderer:win_qgl.obj
 0002:0000b064       ??_C@_0N@IBJEPFKK@glEdgeFlagv?6?$AA@ 004c7064     renderer:win_qgl.obj
 0002:0000b074       ??_C@_0BA@OGCEDJJI@glEnable?$CI?5?$CFs?5?$CJ?6?$AA@ 004c7074     renderer:win_qgl.obj
 0002:0000b084       ??_C@_0BL@HACNJHBM@glEnableClientState?$CI?5?$CFs?5?$CJ?6?$AA@ 004c7084     renderer:win_qgl.obj
 0002:0000b0a0       ??_C@_06KNGPEBLE@glEnd?6?$AA@ 004c70a0     renderer:win_qgl.obj
 0002:0000b0a8       ??_C@_0L@DEPEENDO@glEndList?6?$AA@ 004c70a8     renderer:win_qgl.obj
 0002:0000b0b4       ??_C@_0P@CCLLNLGD@glEvalCoord1d?6?$AA@ 004c70b4     renderer:win_qgl.obj
 0002:0000b0c4       ??_C@_0BA@HDJNPCIH@glEvalCoord1dv?6?$AA@ 004c70c4     renderer:win_qgl.obj
 0002:0000b0d4       ??_C@_0P@CBDPAPAN@glEvalCoord1f?6?$AA@ 004c70d4     renderer:win_qgl.obj
 0002:0000b0e4       ??_C@_0BA@NJJEDKAM@glEvalCoord1fv?6?$AA@ 004c70e4     renderer:win_qgl.obj
 0002:0000b0f4       ??_C@_0P@DAAOHEIN@glEvalCoord2d?6?$AA@ 004c70f4     renderer:win_qgl.obj
 0002:0000b104       ??_C@_0BA@DEDNIIFH@glEvalCoord2dv?6?$AA@ 004c7104     renderer:win_qgl.obj
 0002:0000b114       ??_C@_0P@DDIKKAOD@glEvalCoord2f?6?$AA@ 004c7114     renderer:win_qgl.obj
 0002:0000b124       ??_C@_0BA@JODEEANM@glEvalCoord2fv?6?$AA@ 004c7124     renderer:win_qgl.obj
 0002:0000b134       ??_C@_0N@NMAEIMBN@glEvalMesh1?6?$AA@ 004c7134     renderer:win_qgl.obj
 0002:0000b144       ??_C@_0N@NOECDCEE@glEvalMesh2?6?$AA@ 004c7144     renderer:win_qgl.obj
 0002:0000b154       ??_C@_0O@HDACINEI@glEvalPoint1?6?$AA@ 004c7154     renderer:win_qgl.obj
 0002:0000b164       ??_C@_0O@HBEEDDBB@glEvalPoint2?6?$AA@ 004c7164     renderer:win_qgl.obj
 0002:0000b174       ??_C@_0BC@LPBOOEHF@glFeedbackBuffer?6?$AA@ 004c7174     renderer:win_qgl.obj
 0002:0000b188       ??_C@_09HLIDOBK@glFinish?6?$AA@ 004c7188     renderer:win_qgl.obj
 0002:0000b194       ??_C@_08KMOCPHF@glFlush?6?$AA@ 004c7194     renderer:win_qgl.obj
 0002:0000b1a0       ??_C@_07NOMCDGOK@glFogf?6?$AA@ 004c71a0     renderer:win_qgl.obj
 0002:0000b1a8       ??_C@_08OHAFLAOO@glFogfv?6?$AA@ 004c71a8     renderer:win_qgl.obj
 0002:0000b1b4       ??_C@_07NFJOHBNH@glFogi?6?$AA@ 004c71b4     renderer:win_qgl.obj
 0002:0000b1bc       ??_C@_08LPGGKALI@glFogiv?6?$AA@ 004c71bc     renderer:win_qgl.obj
 0002:0000b1c8       ??_C@_0N@NMLNMEBP@glFrontFace?6?$AA@ 004c71c8     renderer:win_qgl.obj
 0002:0000b1d8       ??_C@_0L@LMAEODIN@glFrustum?6?$AA@ 004c71d8     renderer:win_qgl.obj
 0002:0000b1e4       ??_C@_0M@HHPKAAJL@glGenLists?6?$AA@ 004c71e4     renderer:win_qgl.obj
 0002:0000b1f0       ??_C@_0P@JMFCBDJL@glGenTextures?6?$AA@ 004c71f0     renderer:win_qgl.obj
 0002:0000b200       ??_C@_0P@LIIGLEFN@glGetBooleanv?6?$AA@ 004c7200     renderer:win_qgl.obj
 0002:0000b210       ??_C@_0BA@IPIJIHMN@glGetClipPlane?6?$AA@ 004c7210     renderer:win_qgl.obj
 0002:0000b220       ??_C@_0O@ECLHFBEH@glGetDoublev?6?$AA@ 004c7220     renderer:win_qgl.obj
 0002:0000b230       ??_C@_0M@NNLCAJOK@glGetError?6?$AA@ 004c7230     renderer:win_qgl.obj
 0002:0000b23c       ??_C@_0N@HLHLNAFJ@glGetFloatv?6?$AA@ 004c723c     renderer:win_qgl.obj
 0002:0000b24c       ??_C@_0P@EBNDNMKL@glGetIntegerv?6?$AA@ 004c724c     renderer:win_qgl.obj
 0002:0000b25c       ??_C@_0O@CMPPCHPE@glGetLightfv?6?$AA@ 004c725c     renderer:win_qgl.obj
 0002:0000b26c       ??_C@_0O@HEJMDHKC@glGetLightiv?6?$AA@ 004c726c     renderer:win_qgl.obj
 0002:0000b27c       ??_C@_0M@MBNHELAF@glGetMapdv?6?$AA@ 004c727c     renderer:win_qgl.obj
 0002:0000b288       ??_C@_0M@GLNOIDIO@glGetMapfv?6?$AA@ 004c7288     renderer:win_qgl.obj
 0002:0000b294       ??_C@_0M@DDLNJDNI@glGetMapiv?6?$AA@ 004c7294     renderer:win_qgl.obj
 0002:0000b2a0       ??_C@_0BB@NFOCGLEJ@glGetMaterialfv?6?$AA@ 004c72a0     renderer:win_qgl.obj
 0002:0000b2b4       ??_C@_0BB@INIBHLBP@glGetMaterialiv?6?$AA@ 004c72b4     renderer:win_qgl.obj
 0002:0000b2c8       ??_C@_0BB@BAHJMCIF@glGetPixelMapfv?6?$AA@ 004c72c8     renderer:win_qgl.obj
 0002:0000b2dc       ??_C@_0BC@BFPMNNEI@glGetPixelMapuiv?6?$AA@ 004c72dc     renderer:win_qgl.obj
 0002:0000b2f0       ??_C@_0BC@CKFIGKLD@glGetPixelMapusv?6?$AA@ 004c72f0     renderer:win_qgl.obj
 0002:0000b304       ??_C@_0P@ONOIGCPP@glGetPointerv?6?$AA@ 004c7304     renderer:win_qgl.obj
 0002:0000b314       ??_C@_0BF@EMKGEEI@glGetPolygonStipple?6?$AA@ 004c7314     renderer:win_qgl.obj
 0002:0000b32c       ??_C@_0N@LGGJBJIH@glGetString?6?$AA@ 004c732c     renderer:win_qgl.obj
 0002:0000b33c       ??_C@_0P@FGPABIKP@glGetTexEnvfv?6?$AA@ 004c733c     renderer:win_qgl.obj
 0002:0000b34c       ??_C@_0P@OJDAIPJ@glGetTexEnviv?6?$AA@ 004c734c     renderer:win_qgl.obj
 0002:0000b35c       ??_C@_0P@FBDBONIN@glGetTexGendv?6?$AA@ 004c735c     renderer:win_qgl.obj
 0002:0000b36c       ??_C@_0P@PLDICFAG@glGetTexGenfv?6?$AA@ 004c736c     renderer:win_qgl.obj
 0002:0000b37c       ??_C@_0P@KDFLDFFA@glGetTexGeniv?6?$AA@ 004c737c     renderer:win_qgl.obj
 0002:0000b38c       ??_C@_0P@GDNIDBKL@glGetTexImage?6?$AA@ 004c738c     renderer:win_qgl.obj
 0002:0000b39c       ??_C@_0BK@OBIOIGJJ@glGetTexLevelParameterfv?6?$AA@ 004c739c     renderer:win_qgl.obj
 0002:0000b3b8       ??_C@_0BK@LJONJGMP@glGetTexLevelParameteriv?6?$AA@ 004c73b8     renderer:win_qgl.obj
 0002:0000b3d4       ??_C@_0BF@IPLIDKOM@glGetTexParameterfv?6?$AA@ 004c73d4     renderer:win_qgl.obj
 0002:0000b3ec       ??_C@_0BF@NHNLCKLK@glGetTexParameteriv?6?$AA@ 004c73ec     renderer:win_qgl.obj
 0002:0000b404       ??_C@_0BG@MNKJGBKM@glHint?$CI?50x?$CFx?0?50x?$CFx?5?$CJ?6?$AA@ 004c7404     renderer:win_qgl.obj
 0002:0000b41c       ??_C@_0N@FKAIDDBG@glIndexMask?6?$AA@ 004c741c     renderer:win_qgl.obj
 0002:0000b42c       ??_C@_0BA@NOPNNKJG@glIndexPointer?6?$AA@ 004c742c     renderer:win_qgl.obj
 0002:0000b43c       ??_C@_09KBEPKCDK@glIndexd?6?$AA@ 004c743c     renderer:win_qgl.obj
 0002:0000b448       ??_C@_0L@GBKJOPKO@glIndexdv?6?$AA@ 004c7448     renderer:win_qgl.obj
 0002:0000b454       ??_C@_09KCMLHGFE@glIndexf?6?$AA@ 004c7454     renderer:win_qgl.obj
 0002:0000b460       ??_C@_0L@MLKACHCF@glIndexfv?6?$AA@ 004c7460     renderer:win_qgl.obj
 0002:0000b46c       ??_C@_09KJJHDBGJ@glIndexi?6?$AA@ 004c746c     renderer:win_qgl.obj
 0002:0000b478       ??_C@_0L@JDMDDHHD@glIndexiv?6?$AA@ 004c7478     renderer:win_qgl.obj
 0002:0000b484       ??_C@_09LICGBHMP@glIndexs?6?$AA@ 004c7484     renderer:win_qgl.obj
 0002:0000b490       ??_C@_0L@KMGHIAII@glIndexsv?6?$AA@ 004c7490     renderer:win_qgl.obj
 0002:0000b49c       ??_C@_0L@JCCDNEPI@glIndexub?6?$AA@ 004c749c     renderer:win_qgl.obj
 0002:0000b4a8       ??_C@_0M@BEPACAEE@glIndexubv?6?$AA@ 004c74a8     renderer:win_qgl.obj
 0002:0000b4b4       ??_C@_0N@CDMKHFL@glInitNames?6?$AA@ 004c74b4     renderer:win_qgl.obj
 0002:0000b4c4       ??_C@_0BF@DPBGJABO@glInterleavedArrays?6?$AA@ 004c74c4     renderer:win_qgl.obj
 0002:0000b4dc       ??_C@_0N@MCLKFGMJ@glIsEnabled?6?$AA@ 004c74dc     renderer:win_qgl.obj
 0002:0000b4ec       ??_C@_09ECGOBBBP@glIsList?6?$AA@ 004c74ec     renderer:win_qgl.obj
 0002:0000b4f8       ??_C@_0N@KCFONENE@glIsTexture?6?$AA@ 004c74f8     renderer:win_qgl.obj
 0002:0000b508       ??_C@_0P@BJPDMKCI@glLightModelf?6?$AA@ 004c7508     renderer:win_qgl.obj
 0002:0000b518       ??_C@_0BA@JCKICCIO@glLightModelfv?6?$AA@ 004c7518     renderer:win_qgl.obj
 0002:0000b528       ??_C@_0P@BCKPINBF@glLightModeli?6?$AA@ 004c7528     renderer:win_qgl.obj
 0002:0000b538       ??_C@_0BA@MKMLDCNI@glLightModeliv?6?$AA@ 004c7538     renderer:win_qgl.obj
 0002:0000b548       ??_C@_09BLFOEPBJ@glLightf?6?$AA@ 004c7548     renderer:win_qgl.obj
 0002:0000b554       ??_C@_0L@MDHEIPDB@glLightfv?6?$AA@ 004c7554     renderer:win_qgl.obj
 0002:0000b560       ??_C@_09BAACAICE@glLighti?6?$AA@ 004c7560     renderer:win_qgl.obj
 0002:0000b56c       ??_C@_0L@JLBHJPGH@glLightiv?6?$AA@ 004c756c     renderer:win_qgl.obj
 0002:0000b578       ??_C@_0P@LKIDALDN@glLineStipple?6?$AA@ 004c7578     renderer:win_qgl.obj
 0002:0000b588       ??_C@_0N@KOBEAJHG@glLineWidth?6?$AA@ 004c7588     renderer:win_qgl.obj
 0002:0000b598       ??_C@_0M@OHCLBBNL@glListBase?6?$AA@ 004c7598     renderer:win_qgl.obj
 0002:0000b5a4       ??_C@_0BA@KAKDDCOF@glLoadIdentity?6?$AA@ 004c75a4     renderer:win_qgl.obj
 0002:0000b5b4       ??_C@_0P@IBFFJEIA@glLoadMatrixd?6?$AA@ 004c75b4     renderer:win_qgl.obj
 0002:0000b5c4       ??_C@_0P@ICNBEAOO@glLoadMatrixf?6?$AA@ 004c75c4     renderer:win_qgl.obj
 0002:0000b5d4       ??_C@_0M@KHFCCBO@glLoadName?6?$AA@ 004c75d4     renderer:win_qgl.obj
 0002:0000b5e0       ??_C@_0L@MFDAICIH@glLogicOp?6?$AA@ 004c75e0     renderer:win_qgl.obj
 0002:0000b5ec       ??_C@_08EELAIOPD@glMap1d?6?$AA@ 004c75ec     renderer:win_qgl.obj
 0002:0000b5f8       ??_C@_08EHDEFKJN@glMap1f?6?$AA@ 004c75f8     renderer:win_qgl.obj
 0002:0000b604       ??_C@_08FGAFCBBN@glMap2d?6?$AA@ 004c7604     renderer:win_qgl.obj
 0002:0000b610       ??_C@_08FFIBPFHD@glMap2f?6?$AA@ 004c7610     renderer:win_qgl.obj
 0002:0000b61c       ??_C@_0N@JLEJCNNK@glMapGrid1d?6?$AA@ 004c761c     renderer:win_qgl.obj
 0002:0000b62c       ??_C@_0N@JIMNPJLE@glMapGrid1f?6?$AA@ 004c762c     renderer:win_qgl.obj
 0002:0000b63c       ??_C@_0N@IJPMICDE@glMapGrid2d?6?$AA@ 004c763c     renderer:win_qgl.obj
 0002:0000b64c       ??_C@_0N@IKHIFGFK@glMapGrid2f?6?$AA@ 004c764c     renderer:win_qgl.obj
 0002:0000b65c       ??_C@_0N@IPPFJFJM@glMaterialf?6?$AA@ 004c765c     renderer:win_qgl.obj
 0002:0000b66c       ??_C@_0O@FODCFDEE@glMaterialfv?6?$AA@ 004c766c     renderer:win_qgl.obj
 0002:0000b67c       ??_C@_0N@IEKJNCKB@glMateriali?6?$AA@ 004c767c     renderer:win_qgl.obj
 0002:0000b68c       ??_C@_0O@GFBEDBC@glMaterialiv?6?$AA@ 004c768c     renderer:win_qgl.obj
 0002:0000b69c       ??_C@_0O@PFEMKMME@glMatrixMode?6?$AA@ 004c769c     renderer:win_qgl.obj
 0002:0000b6ac       ??_C@_0P@FGNGIEHH@glMultMatrixd?6?$AA@ 004c76ac     renderer:win_qgl.obj
 0002:0000b6bc       ??_C@_0P@FFFCFABJ@glMultMatrixf?6?$AA@ 004c76bc     renderer:win_qgl.obj
 0002:0000b6cc       ??_C@_0L@LNPNEJOG@glNewList?6?$AA@ 004c76cc     renderer:win_qgl.obj
 0002:0000b6d8       ??_C@_0M@EJNLJMHO@glNormal3b?6?$AA@ 004c76d8     renderer:win_qgl.obj
 0002:0000b6e4       ??_C@_0N@BAPAPOBJ@glNormal3bv?6?$AA@ 004c76e4     renderer:win_qgl.obj
 0002:0000b6f4       ??_C@_0M@ENFGOAMM@glNormal3d?6?$AA@ 004c76f4     renderer:win_qgl.obj
 0002:0000b700       ??_C@_0N@DFJLKBMF@glNormal3dv?6?$AA@ 004c7700     renderer:win_qgl.obj
 0002:0000b710       ??_C@_0M@EONCDEKC@glNormal3f?6?$AA@ 004c7710     renderer:win_qgl.obj
 0002:0000b71c       ??_C@_0N@JPJCGJEO@glNormal3fv?6?$AA@ 004c771c     renderer:win_qgl.obj
 0002:0000b72c       ??_C@_0M@EFIOHDJP@glNormal3i?6?$AA@ 004c772c     renderer:win_qgl.obj
 0002:0000b738       ??_C@_0N@MHPBHJBI@glNormal3iv?6?$AA@ 004c7738     renderer:win_qgl.obj
 0002:0000b748       ??_C@_0M@FEDPFFDJ@glNormal3s?6?$AA@ 004c7748     renderer:win_qgl.obj
 0002:0000b754       ??_C@_0N@PIFFMOOD@glNormal3sv?6?$AA@ 004c7754     renderer:win_qgl.obj
 0002:0000b764       ??_C@_0BB@MKGIKLEH@glNormalPointer?6?$AA@ 004c7764     renderer:win_qgl.obj
 0002:0000b778       ??_C@_08BJLNOGOG@glOrtho?6?$AA@ 004c7778     renderer:win_qgl.obj
 0002:0000b784       ??_C@_0P@BCPFLAHE@glPassThrough?6?$AA@ 004c7784     renderer:win_qgl.obj
 0002:0000b794       ??_C@_0O@JLKJPKII@glPixelMapfv?6?$AA@ 004c7794     renderer:win_qgl.obj
 0002:0000b7a4       ??_C@_0P@GLMGHBMN@glPixelMapuiv?6?$AA@ 004c77a4     renderer:win_qgl.obj
 0002:0000b7b4       ??_C@_0P@FEGCMGDG@glPixelMapusv?6?$AA@ 004c77b4     renderer:win_qgl.obj
 0002:0000b7c4       ??_C@_0P@CBEBJBCL@glPixelStoref?6?$AA@ 004c77c4     renderer:win_qgl.obj
 0002:0000b7d4       ??_C@_0P@CKBNNGBG@glPixelStorei?6?$AA@ 004c77d4     renderer:win_qgl.obj
 0002:0000b7e4       ??_C@_0BC@PCIFIHCI@glPixelTransferf?6?$AA@ 004c77e4     renderer:win_qgl.obj
 0002:0000b7f8       ??_C@_0BC@PJNJMABF@glPixelTransferi?6?$AA@ 004c77f8     renderer:win_qgl.obj
 0002:0000b80c       ??_C@_0N@LKLMDEO@glPixelZoom?6?$AA@ 004c780c     renderer:win_qgl.obj
 0002:0000b81c       ??_C@_0N@HFMOHJLJ@glPointSize?6?$AA@ 004c781c     renderer:win_qgl.obj
 0002:0000b82c       ??_C@_0BN@GGKAIPLL@glPolygonMode?$CI?50x?$CFx?0?50x?$CFx?5?$CJ?6?$AA@ 004c782c     renderer:win_qgl.obj
 0002:0000b84c       ??_C@_0BB@JCDHAKOE@glPolygonOffset?6?$AA@ 004c784c     renderer:win_qgl.obj
 0002:0000b860       ??_C@_0BC@CHIKJHAK@glPolygonStipple?6?$AA@ 004c7860     renderer:win_qgl.obj
 0002:0000b874       ??_C@_0N@BPIBIAIA@glPopAttrib?6?$AA@ 004c7874     renderer:win_qgl.obj
 0002:0000b884       ??_C@_0BD@ECDMKECN@glPopClientAttrib?6?$AA@ 004c7884     renderer:win_qgl.obj
 0002:0000b898       ??_C@_0N@GMHJAAAA@glPopMatrix?6?$AA@ 004c7898     renderer:win_qgl.obj
 0002:0000b8a8       ??_C@_0L@FNACPBGC@glPopName?6?$AA@ 004c78a8     renderer:win_qgl.obj
 0002:0000b8b4       ??_C@_0BG@BHACENHH@glPrioritizeTextures?6?$AA@ 004c78b4     renderer:win_qgl.obj
 0002:0000b8cc       ??_C@_0O@DPFPMJA@glPushAttrib?6?$AA@ 004c78cc     renderer:win_qgl.obj
 0002:0000b8dc       ??_C@_0BE@IMKJMGKH@glPushClientAttrib?6?$AA@ 004c78dc     renderer:win_qgl.obj
 0002:0000b8f0       ??_C@_0O@HAANHMBA@glPushMatrix?6?$AA@ 004c78f0     renderer:win_qgl.obj
 0002:0000b900       ??_C@_0M@PHDHNHLF@glPushName?6?$AA@ 004c7900     renderer:win_qgl.obj
 0002:0000b90c       ??_C@_0P@NEMPOAMF@glRasterPot2d?6?$AA@ 004c790c     renderer:win_qgl.obj
 0002:0000b91c       ??_C@_0BA@FBNLLANJ@glRasterPos2dv?6?$AA@ 004c791c     renderer:win_qgl.obj
 0002:0000b92c       ??_C@_0P@GFGLOILL@glRasterPos2f?6?$AA@ 004c792c     renderer:win_qgl.obj
 0002:0000b93c       ??_C@_0BA@LPJHMLHE@glRasterPos2if?6?$AA@ 004c793c     renderer:win_qgl.obj
 0002:0000b94c       ??_C@_0BA@KDLBGIAE@glRasterPos2iv?6?$AA@ 004c794c     renderer:win_qgl.obj
 0002:0000b95c       ??_C@_0P@HPIGIJCA@glRasterPos2s?6?$AA@ 004c795c     renderer:win_qgl.obj
 0002:0000b96c       ??_C@_0BA@JMBFNPPP@glRasterPos2sv?6?$AA@ 004c796c     renderer:win_qgl.obj
 0002:0000b97c       ??_C@_0P@NOFDFLLA@glRasterPos3d?6?$AA@ 004c797c     renderer:win_qgl.obj
 0002:0000b98c       ??_C@_0BA@GMLLJJGJ@glRasterPos3dv?6?$AA@ 004c798c     renderer:win_qgl.obj
 0002:0000b99c       ??_C@_0P@NNNHIPNO@glRasterPos3f?6?$AA@ 004c799c     renderer:win_qgl.obj
 0002:0000b9ac       ??_C@_0BA@MGLCFBOC@glRasterPos3fv?6?$AA@ 004c79ac     renderer:win_qgl.obj
 0002:0000b9bc       ??_C@_0P@NGILMIOD@glRasterPos3i?6?$AA@ 004c79bc     renderer:win_qgl.obj
 0002:0000b9cc       ??_C@_0BA@JONBEBLE@glRasterPos3iv?6?$AA@ 004c79cc     renderer:win_qgl.obj
 0002:0000b9dc       ??_C@_0P@MHDKOOEF@glRasterPos3s?6?$AA@ 004c79dc     renderer:win_qgl.obj
 0002:0000b9ec       ??_C@_0BA@KBHFPGEP@glRasterPos3sv?6?$AA@ 004c79ec     renderer:win_qgl.obj
 0002:0000b9fc       ??_C@_0P@EDIEGDAJ@glRasterPos4d?6?$AA@ 004c79fc     renderer:win_qgl.obj
 0002:0000ba0c       ??_C@_0BA@NOJLEFHJ@glRasterPos4dv?6?$AA@ 004c7a0c     renderer:win_qgl.obj
 0002:0000ba1c       ??_C@_0P@EAAALHGH@glRasterPos4f?6?$AA@ 004c7a1c     renderer:win_qgl.obj
 0002:0000ba2c       ??_C@_0BA@HEJCINPC@glRasterPos4fv?6?$AA@ 004c7a2c     renderer:win_qgl.obj
 0002:0000ba3c       ??_C@_0P@ELFMPAFK@glRasterPos4i?6?$AA@ 004c7a3c     renderer:win_qgl.obj
 0002:0000ba4c       ??_C@_0BA@CMPBJNKE@glRasterPos4iv?6?$AA@ 004c7a4c     renderer:win_qgl.obj
 0002:0000ba5c       ??_C@_0P@FKONNGPM@glRasterPos4s?6?$AA@ 004c7a5c     renderer:win_qgl.obj
 0002:0000ba6c       ??_C@_0BA@BDFFCKFP@glRasterPos4sv?6?$AA@ 004c7a6c     renderer:win_qgl.obj
 0002:0000ba7c       ??_C@_0O@CBCBIGEI@glReadBuffer?6?$AA@ 004c7a7c     renderer:win_qgl.obj
 0002:0000ba8c       ??_C@_0O@LNHHHKCC@glReadPixels?6?$AA@ 004c7a8c     renderer:win_qgl.obj
 0002:0000ba9c       ??_C@_08MFDNGFJP@glRectd?6?$AA@ 004c7a9c     renderer:win_qgl.obj
 0002:0000baa8       ??_C@_09MHHBMKAO@glRectdv?6?$AA@ 004c7aa8     renderer:win_qgl.obj
 0002:0000bab4       ??_C@_08MGLJLBPB@glRectf?6?$AA@ 004c7ab4     renderer:win_qgl.obj
 0002:0000bac0       ??_C@_09GNHIACIF@glRectfv?6?$AA@ 004c7ac0     renderer:win_qgl.obj
 0002:0000bacc       ??_C@_08MNOFPGMM@glRecti?6?$AA@ 004c7acc     renderer:win_qgl.obj
 0002:0000bad8       ??_C@_09DFBLBCND@glRectiv?6?$AA@ 004c7ad8     renderer:win_qgl.obj
 0002:0000bae4       ??_C@_08NMFENAGK@glRects?6?$AA@ 004c7ae4     renderer:win_qgl.obj
 0002:0000baf0       ??_C@_09KLPKFCI@glRectsv?6?$AA@ 004c7af0     renderer:win_qgl.obj
 0002:0000bafc       ??_C@_0O@CHJAMNBA@glRenderMode?6?$AA@ 004c7afc     renderer:win_qgl.obj
 0002:0000bb0c       ??_C@_0L@BNDHBADO@glRotated?6?$AA@ 004c7b0c     renderer:win_qgl.obj
 0002:0000bb18       ??_C@_0L@BOLDMEFA@glRotatef?6?$AA@ 004c7b18     renderer:win_qgl.obj
 0002:0000bb24       ??_C@_09NCENJCJJ@glScaled?6?$AA@ 004c7b24     renderer:win_qgl.obj
 0002:0000bb30       ??_C@_09NBMJEGPH@glScalef?6?$AA@ 004c7b30     renderer:win_qgl.obj
 0002:0000bb3c       ??_C@_0BN@PMDENLCH@glScissor?$CI?5?$CFd?0?5?$CFd?0?5?$CFd?0?5?$CFd?5?$CJ?6?$AA@ 004c7b3c     renderer:win_qgl.obj
 0002:0000bb5c       ??_C@_0BA@LPJAJLDO@glSelectBuffer?6?$AA@ 004c7b5c     renderer:win_qgl.obj
 0002:0000bb6c       ??_C@_0O@FCFIILII@glShadeModel?6?$AA@ 004c7b6c     renderer:win_qgl.obj
 0002:0000bb7c       ??_C@_0P@EPHCPMAF@glStencilFunc?6?$AA@ 004c7b7c     renderer:win_qgl.obj
 0002:0000bb8c       ??_C@_0P@BMLFODHO@glStencilMask?6?$AA@ 004c7b8c     renderer:win_qgl.obj
 0002:0000bb9c       ??_C@_0N@MHDGPGEA@glStencilOp?6?$AA@ 004c7b9c     renderer:win_qgl.obj
 0002:0000bbac       ??_C@_0O@OMKJIGDN@glTexCoord1d?6?$AA@ 004c7bac     renderer:win_qgl.obj
 0002:0000bbbc       ??_C@_0P@PPIAJMCJ@glTexCoord1dv?6?$AA@ 004c7bbc     renderer:win_qgl.obj
 0002:0000bbcc       ??_C@_0O@OPCNFCFD@glTexCoord1f?6?$AA@ 004c7bcc     renderer:win_qgl.obj
 0002:0000bbdc       ??_C@_0P@FFIJFEKC@glTexCoord1fv?6?$AA@ 004c7bdc     renderer:win_qgl.obj
 0002:0000bbec       ??_C@_0O@OEHBBFGO@glTexCoord1i?6?$AA@ 004c7bec     renderer:win_qgl.obj
 0002:0000bbfc       ??_C@_0P@NOKEEPE@glTexCoord1iv?6?$AA@ 004c7bfc     renderer:win_qgl.obj
 0002:0000bc0c       ??_C@_0O@PFMADDMI@glTexCoord1s?6?$AA@ 004c7c0c     renderer:win_qgl.obj
 0002:0000bc1c       ??_C@_0P@DCEOPDAP@glTexCoord1sv?6?$AA@ 004c7c1c     renderer:win_qgl.obj
 0002:0000bc2c       ??_C@_0O@POBMCJND@glTexCoord2d?6?$AA@ 004c7c2c     renderer:win_qgl.obj
 0002:0000bc3c       ??_C@_0P@LICAOGPJ@glTexCoord2dv?6?$AA@ 004c7c3c     renderer:win_qgl.obj
 0002:0000bc4c       ??_C@_0O@PNJIPNLN@glTexCoord2f?6?$AA@ 004c7c4c     renderer:win_qgl.obj
 0002:0000bc5c       ??_C@_0P@BCCJCOHC@glTexCoord2fv?6?$AA@ 004c7c5c     renderer:win_qgl.obj
 0002:0000bc6c       ??_C@_0O@PGMELKIA@glTexCoord2i?6?$AA@ 004c7c6c     renderer:win_qgl.obj
 0002:0000bc7c       ??_C@_0P@EKEKDOCE@glTexCoord2iv?6?$AA@ 004c7c7c     renderer:win_qgl.obj
 0002:0000bc8c       ??_C@_0O@OHHFJMCG@glTexCoord2s?6?$AA@ 004c7c8c     renderer:win_qgl.obj
 0002:0000bc9c       ??_C@_0P@HFOOIJNP@glTexCoord2sv?6?$AA@ 004c7c9c     renderer:win_qgl.obj
 0002:0000bcac       ??_C@_0O@EGKAEOLG@glTexCoord3d?6?$AA@ 004c7cac     renderer:win_qgl.obj
 0002:0000bcbc       ??_C@_0P@IFEAMPEJ@glTexCoord3dv?6?$AA@ 004c7cbc     renderer:win_qgl.obj
 0002:0000bccc       ??_C@_0O@EFCEJKNI@glTexCoord3f?6?$AA@ 004c7ccc     renderer:win_qgl.obj
 0002:0000bcdc       ??_C@_0P@CPEJAHMC@glTexCoord3fv?6?$AA@ 004c7cdc     renderer:win_qgl.obj
 0002:0000bcec       ??_C@_0O@EOHINNOF@glTexCoord3i?6?$AA@ 004c7cec     renderer:win_qgl.obj
 0002:0000bcfc       ??_C@_0P@HHCKBHJE@glTexCoord3iv?6?$AA@ 004c7cfc     renderer:win_qgl.obj
 0002:0000bd0c       ??_C@_0O@FPMJPLED@glTexCoord3s?6?$AA@ 004c7d0c     renderer:win_qgl.obj
 0002:0000bd1c       ??_C@_0P@EIIOKAGP@glTexCoord3sv?6?$AA@ 004c7d1c     renderer:win_qgl.obj
 0002:0000bd2c       ??_C@_0O@NLHHHGAP@glTexCoord4d?6?$AA@ 004c7d2c     renderer:win_qgl.obj
 0002:0000bd3c       ??_C@_0P@DHGABDFJ@glTexCoord4dv?6?$AA@ 004c7d3c     renderer:win_qgl.obj
 0002:0000bd4c       ??_C@_0O@NIPDKCGB@glTexCoord4f?6?$AA@ 004c7d4c     renderer:win_qgl.obj
 0002:0000bd5c       ??_C@_0P@JNGJNLNC@glTexCoord4fv?6?$AA@ 004c7d5c     renderer:win_qgl.obj
 0002:0000bd6c       ??_C@_0O@NDKPOFFM@glTexCoord4i?6?$AA@ 004c7d6c     renderer:win_qgl.obj
 0002:0000bd7c       ??_C@_0P@MFAKMLIE@glTexCoord4iv?6?$AA@ 004c7d7c     renderer:win_qgl.obj
 0002:0000bd8c       ??_C@_0O@MCBOMDPK@glTexCoord4s?6?$AA@ 004c7d8c     renderer:win_qgl.obj
 0002:0000bd9c       ??_C@_0P@PKKOHMHP@glTexCoord4sv?6?$AA@ 004c7d9c     renderer:win_qgl.obj
 0002:0000bdac       ??_C@_0CG@PCDFCPLA@glTexCoordPointer?$CI?5?$CFd?0?5?$CFs?0?5?$CFd?0?5M@ 004c7dac     renderer:win_qgl.obj
 0002:0000bdd4       ??_C@_0BN@OFAECEEA@glTexEnvf?$CI?50x?$CFx?0?50x?$CFx?0?5?$CFf?5?$CJ?6?$AA@ 004c7dd4     renderer:win_qgl.obj
 0002:0000bdf4       ??_C@_0M@LNBBKFDI@glTexEnvfv?6?$AA@ 004c7df4     renderer:win_qgl.obj
 0002:0000be00       ??_C@_0BP@OOICOAPD@glTexEnvi?$CI?50x?$CFx?0?50x?$CFx?0?50x?$CFx?5?$CJ?6?$AA@ 004c7e00     renderer:win_qgl.obj
 0002:0000be20       ??_C@_0M@OFHCLFGO@glTexEnviv?6?$AA@ 004c7e20     renderer:win_qgl.obj
 0002:0000be2c       ??_C@_0L@GDDJMABA@glTexGend?6?$AA@ 004c7e2c     renderer:win_qgl.obj
 0002:0000be38       ??_C@_0M@LKNAFABK@glTexGendv?6?$AA@ 004c7e38     renderer:win_qgl.obj
 0002:0000be44       ??_C@_0L@GALNBEHO@glTexGenf?6?$AA@ 004c7e44     renderer:win_qgl.obj
 0002:0000be50       ??_C@_0M@BANJJIJB@glTexGenfv?6?$AA@ 004c7e50     renderer:win_qgl.obj
 0002:0000be5c       ??_C@_0L@GLOBFDED@glTexGeni?6?$AA@ 004c7e5c     renderer:win_qgl.obj
 0002:0000be68       ??_C@_0M@EILKIIMH@glTexGeniv?6?$AA@ 004c7e68     renderer:win_qgl.obj
 0002:0000be74       ??_C@_0O@DNKLIMPL@glTexImage1D?6?$AA@ 004c7e74     renderer:win_qgl.obj
 0002:0000be84       ??_C@_0O@CPBOCDBF@glTexImage2D?6?$AA@ 004c7e84     renderer:win_qgl.obj
 0002:0000be94       ??_C@_0CD@PAPIOALP@glTexParameterf?$CI?50x?$CFx?0?50x?$CFx?0?5?$CFf?5@ 004c7e94     renderer:win_qgl.obj
 0002:0000beb8       ??_C@_0BC@KMPIMJKO@glTexParameterfv?6?$AA@ 004c7eb8     renderer:win_qgl.obj
 0002:0000becc       ??_C@_0CF@OBKPAONE@glTexParameteri?$CI?50x?$CFx?0?50x?$CFx?0?50x?$CF@ 004c7ecc     renderer:win_qgl.obj
 0002:0000bef4       ??_C@_0BC@PEJLNJPI@glTexParameteriv?6?$AA@ 004c7ef4     renderer:win_qgl.obj
 0002:0000bf08       ??_C@_0BB@JDDMMEFO@glTexSubImage1D?6?$AA@ 004c7f08     renderer:win_qgl.obj
 0002:0000bf1c       ??_C@_0BB@IBIJGLLA@glTexSubImage2D?6?$AA@ 004c7f1c     renderer:win_qgl.obj
 0002:0000bf30       ??_C@_0O@HIFANJBI@glTranslated?6?$AA@ 004c7f30     renderer:win_qgl.obj
 0002:0000bf40       ??_C@_0O@HLNEANHG@glTranslatef?6?$AA@ 004c7f40     renderer:win_qgl.obj
 0002:0000bf50       ??_C@_0M@KIAKGGGC@glVertex2d?6?$AA@ 004c7f50     renderer:win_qgl.obj
 0002:0000bf5c       ??_C@_0N@EBAHDKM@glVertex2dv?6?$AA@ 004c7f5c     renderer:win_qgl.obj
 0002:0000bf6c       ??_C@_0M@KLIOLCAM@glVertex2f?6?$AA@ 004c7f6c     renderer:win_qgl.obj
 0002:0000bf78       ??_C@_0N@KOBJLLCH@glVertex2fv?6?$AA@ 004c7f78     renderer:win_qgl.obj
 0002:0000bf88       ??_C@_0M@KANCPFDB@glVertex2i?6?$AA@ 004c7f88     renderer:win_qgl.obj
 0002:0000bf94       ??_C@_0N@PGHKKLHB@glVertex2iv?6?$AA@ 004c7f94     renderer:win_qgl.obj
 0002:0000bfa4       ??_C@_0M@LBGDNDJH@glVertex2s?6?$AA@ 004c7fa4     renderer:win_qgl.obj
 0002:0000bfb0       ??_C@_0N@MJNOBMIK@glVertex2sv?6?$AA@ 004c7fb0     renderer:win_qgl.obj
 0002:0000bfc0       ??_C@_0M@BALGABAH@glVertex3d?6?$AA@ 004c7fc0     renderer:win_qgl.obj
 0002:0000bfcc       ??_C@_0N@DJHAFKBM@glVertex3dv?6?$AA@ 004c7fcc     renderer:win_qgl.obj
 0002:0000bfdc       ??_C@_0M@BDDCNFGJ@glVertex3f?6?$AA@ 004c7fdc     renderer:win_qgl.obj
 0002:0000bfe8       ??_C@_0N@JDHJJCJH@glVertex3fv?6?$AA@ 004c7fe8     renderer:win_qgl.obj
 0002:0000bff8       ??_C@_0M@BIGOJCFE@glVertex3i?6?$AA@ 004c7ff8     renderer:win_qgl.obj
 0002:0000c004       ??_C@_0N@MLBKICMB@glVertex3iv?6?$AA@ 004c8004     renderer:win_qgl.obj
 0002:0000c014       ??_C@_0M@JNPLEPC@glVertex3s?6?$AA@ 004c8014     renderer:win_qgl.obj
 0002:0000c020       ??_C@_0N@PELODFDK@glVertex3sv?6?$AA@ 004c8020     renderer:win_qgl.obj
 0002:0000c030       ??_C@_0M@INGBDJLO@glVertex4d?6?$AA@ 004c8030     renderer:win_qgl.obj
 0002:0000c03c       ??_C@_0N@ILFAIGAM@glVertex4dv?6?$AA@ 004c803c     renderer:win_qgl.obj
 0002:0000c04c       ??_C@_0M@IOOFONNA@glVertex4f?6?$AA@ 004c804c     renderer:win_qgl.obj
 0002:0000c058       ??_C@_0N@CBFJEOIH@glVertex4fv?6?$AA@ 004c8058     renderer:win_qgl.obj
 0002:0000c068       ??_C@_0M@IFLJKKON@glVertex4i?6?$AA@ 004c8068     renderer:win_qgl.obj
 0002:0000c074       ??_C@_0N@HJDKFONB@glVertex4iv?6?$AA@ 004c8074     renderer:win_qgl.obj
 0002:0000c084       ??_C@_0M@JEAIIMEL@glVertex4s?6?$AA@ 004c8084     renderer:win_qgl.obj
 0002:0000c090       ??_C@_0N@EGJOOJCK@glVertex4sv?6?$AA@ 004c8090     renderer:win_qgl.obj
 0002:0000c0a0       ??_C@_0CE@FOOALGBI@glVertexPointer?$CI?5?$CFd?0?5?$CFs?0?5?$CFd?0?5MEM@ 004c80a0     renderer:win_qgl.obj
 0002:0000c0c4       ??_C@_0BO@LKDIICAC@glViewport?$CI?5?$CFd?0?5?$CFd?0?5?$CFd?0?5?$CFd?5?$CJ?6?$AA@ 004c80c4     renderer:win_qgl.obj
 0002:0000c0e4       ??_C@_0BJ@IIAEBML@?4?4?4unloading?5OpenGL?5DLL?6?$AA@ 004c80e4     renderer:win_qgl.obj
 0002:0000c100       ??_C@_0BG@MCOGEHEL@?4?4?4shutting?5down?5QGL?6?$AA@ 004c8100     renderer:win_qgl.obj
 0002:0000c118       ??_C@_07OOGNMJEI@Glide3X?$AA@ 004c8118     renderer:win_qgl.obj
 0002:0000c120       ??_C@_0BF@HHBGLCOH@?$CK?$CK?$CK?5CLOSING?5LOG?5?$CK?$CK?$CK?6?$AA@ 004c8120     renderer:win_qgl.obj
 0002:0000c138       ??_C@_02BKFDOEMK@wt?$AA@   004c8138     renderer:win_qgl.obj
 0002:0000c13c       ??_C@_09LGIMFBO@?$CFs?1gl?4log?$AA@ 004c813c     renderer:win_qgl.obj
 0002:0000c148       ??_C@_0P@NIPKMJHJ@wglSwapBuffers?$AA@ 004c8148     renderer:win_qgl.obj
 0002:0000c158       ??_C@_0BC@GFMMJIBD@wglSetPixelFormat?$AA@ 004c8158     renderer:win_qgl.obj
 0002:0000c16c       ??_C@_0BC@KLNCGCDP@wglGetPixelFormat?$AA@ 004c816c     renderer:win_qgl.obj
 0002:0000c180       ??_C@_0BH@EEFLPPJN@wglDescribePixelFormat?$AA@ 004c8180     renderer:win_qgl.obj
 0002:0000c198       ??_C@_0BF@KOEIAGCE@wglChoosePixelFormat?$AA@ 004c8198     renderer:win_qgl.obj
 0002:0000c1b0       ??_C@_0BE@CJLPKDLH@wglUseFontOutlinesA?$AA@ 004c81b0     renderer:win_qgl.obj
 0002:0000c1c4       ??_C@_0BD@DNLKODH@wglUseFontBitmapsA?$AA@ 004c81c4     renderer:win_qgl.obj
 0002:0000c1d8       ??_C@_0BE@JEAIHNHB@wglSwapLayerBuffers?$AA@ 004c81d8     renderer:win_qgl.obj
 0002:0000c1ec       ??_C@_0O@GCGJMHDL@wglShareLists?$AA@ 004c81ec     renderer:win_qgl.obj
 0002:0000c1fc       ??_C@_0BK@IDIDCPAL@wglSetLayerPaletteEntries?$AA@ 004c81fc     renderer:win_qgl.obj
 0002:0000c218       ??_C@_0BH@KGAMHPCJ@wglRealizeLayerPalette?$AA@ 004c8218     renderer:win_qgl.obj
 0002:0000c230       ??_C@_0P@BBBFNDGG@wglMakeCurrent?$AA@ 004c8230     renderer:win_qgl.obj
 0002:0000c240       ??_C@_0BC@FFKMKEGM@wglGetProcAddress?$AA@ 004c8240     renderer:win_qgl.obj
 0002:0000c254       ??_C@_0BK@ICKNAINE@wglGetLayerPaletteEntries?$AA@ 004c8254     renderer:win_qgl.obj
 0002:0000c270       ??_C@_0BA@BMKCDCKD@wglGetCurrentDC?$AA@ 004c8270     renderer:win_qgl.obj
 0002:0000c280       ??_C@_0BF@HABDPBMA@wglGetCurrentContext?$AA@ 004c8280     renderer:win_qgl.obj
 0002:0000c298       ??_C@_0BG@CJLCKGBL@wglDescribeLayerPlane?$AA@ 004c8298     renderer:win_qgl.obj
 0002:0000c2b0       ??_C@_0BB@OGAIJNNO@wglDeleteContext?$AA@ 004c82b0     renderer:win_qgl.obj
 0002:0000c2c4       ??_C@_0BG@JIDGNHOC@wglCreateLayerContext?$AA@ 004c82c4     renderer:win_qgl.obj
 0002:0000c2dc       ??_C@_0BB@GHMBNOIP@wglCreateContext?$AA@ 004c82dc     renderer:win_qgl.obj
 0002:0000c2f0       ??_C@_0P@BPLJMLAG@wglCopyContext?$AA@ 004c82f0     renderer:win_qgl.obj
 0002:0000c300       ??_C@_0L@KBLIPDFH@glViewport?$AA@ 004c8300     renderer:win_qgl.obj
 0002:0000c30c       ??_C@_0BA@HAHECJNK@glVertexPointer?$AA@ 004c830c     renderer:win_qgl.obj
 0002:0000c31c       ??_C@_0M@BHICLKLB@glVertex4sv?$AA@ 004c831c     renderer:win_qgl.obj
 0002:0000c328       ??_C@_0L@IMGCCGJH@glVertex4s?$AA@ 004c8328     renderer:win_qgl.obj
 0002:0000c334       ??_C@_0M@GDDJMBH@glVertex4iv?$AA@ 004c8334     renderer:win_qgl.obj
 0002:0000c340       ??_C@_0L@DMEPNMEM@glVertex4i?$AA@ 004c8340     renderer:win_qgl.obj
 0002:0000c34c       ??_C@_0M@NGPNLCK@glVertex4fv?$AA@ 004c834c     renderer:win_qgl.obj
 0002:0000c358       ??_C@_0L@LLNHMAID@glVertex4f?$AA@ 004c8358     renderer:win_qgl.obj
 0002:0000c364       ??_C@_0M@OOLAPEE@glVertex4dv?$AA@ 004c8364     renderer:win_qgl.obj
 0002:0000c370       ??_C@_0L@IJOBKCAB@glVertex4d?$AA@ 004c8370     renderer:win_qgl.obj
 0002:0000c37c       ??_C@_0M@IKFFICAI@glVertex3sv?$AA@ 004c837c     renderer:win_qgl.obj
 0002:0000c388       ??_C@_0L@IJCNDABC@glVertex3s?$AA@ 004c8388     renderer:win_qgl.obj
 0002:0000c394       ??_C@_0M@JLOEKEKO@glVertex3iv?$AA@ 004c8394     renderer:win_qgl.obj
 0002:0000c3a0       ??_C@_0L@DJAAMKMJ@glVertex3i?$AA@ 004c83a0     renderer:win_qgl.obj
 0002:0000c3ac       ??_C@_0M@JALIODJD@glVertex3fv?$AA@ 004c83ac     renderer:win_qgl.obj
 0002:0000c3b8       ??_C@_0L@LOJINGAG@glVertex3f?$AA@ 004c83b8     renderer:win_qgl.obj
 0002:0000c3c4       ??_C@_0M@JDDMDHPN@glVertex3dv?$AA@ 004c83c4     renderer:win_qgl.obj
 0002:0000c3d0       ??_C@_0L@IMKOLEIE@glVertex3d?$AA@ 004c83d0     renderer:win_qgl.obj
 0002:0000c3dc       ??_C@_0M@DCOJOFGN@glVertex2sv?$AA@ 004c83dc     renderer:win_qgl.obj
 0002:0000c3e8       ??_C@_0L@IIOPFKCF@glVertex2s?$AA@ 004c83e8     renderer:win_qgl.obj
 0002:0000c3f4       ??_C@_0M@CDFIMDML@glVertex2iv?$AA@ 004c83f4     renderer:win_qgl.obj
 0002:0000c400       ??_C@_0L@DIMCKAPO@glVertex2i?$AA@ 004c8400     renderer:win_qgl.obj
 0002:0000c40c       ??_C@_0M@CIAEIEPG@glVertex2fv?$AA@ 004c840c     renderer:win_qgl.obj
 0002:0000c418       ??_C@_0L@LPFKLMDB@glVertex2f?$AA@ 004c8418     renderer:win_qgl.obj
 0002:0000c424       ??_C@_0M@CLIAFAJI@glVertex2dv?$AA@ 004c8424     renderer:win_qgl.obj
 0002:0000c430       ??_C@_0L@INGMNOLD@glVertex2d?$AA@ 004c8430     renderer:win_qgl.obj
 0002:0000c43c       ??_C@_0N@IFPDDBNE@glTranslatef?$AA@ 004c843c     renderer:win_qgl.obj
 0002:0000c44c       ??_C@_0N@LHMFFDFG@glTranslated?$AA@ 004c844c     renderer:win_qgl.obj
 0002:0000c45c       ??_C@_0BA@NHKIJEMK@glTexSubImage2D?$AA@ 004c845c     renderer:win_qgl.obj
 0002:0000c46c       ??_C@_0BA@NFOOCKJD@glTexSubImage1D?$AA@ 004c846c     renderer:win_qgl.obj
 0002:0000c47c       ??_C@_0BB@KPLJEAAI@glTexParameteriv?$AA@ 004c847c     renderer:win_qgl.obj
 0002:0000c490       ??_C@_0BA@KDNJAKA@glTexParameteri?$AA@ 004c8490     renderer:win_qgl.obj
 0002:0000c4a0       ??_C@_0BB@KEOFAHDF@glTexParameterfv?$AA@ 004c84a0     renderer:win_qgl.obj
 0002:0000c4b4       ??_C@_0BA@INKFIMGP@glTexParameterf?$AA@ 004c84b4     renderer:win_qgl.obj
 0002:0000c4c4       ??_C@_0N@JBIKHLCC@glTexImage2D?$AA@ 004c84c4     renderer:win_qgl.obj
 0002:0000c4d4       ??_C@_0N@JDMMMFHL@glTexImage1D?$AA@ 004c84d4     renderer:win_qgl.obj
 0002:0000c4e4       ??_C@_0L@OIGLGFLJ@glTexGeniv?$AA@ 004c84e4     renderer:win_qgl.obj
 0002:0000c4f0       ??_C@_09GKNHFOEO@glTexGeni?$AA@ 004c84f0     renderer:win_qgl.obj
 0002:0000c4fc       ??_C@_0L@ODDHCCIE@glTexGenfv?$AA@ 004c84fc     renderer:win_qgl.obj
 0002:0000c508       ??_C@_09ONEPECIB@glTexGenf?$AA@ 004c8508     renderer:win_qgl.obj
 0002:0000c514       ??_C@_0L@OALDPGOK@glTexGendv?$AA@ 004c8514     renderer:win_qgl.obj
 0002:0000c520       ??_C@_09NPHJCAAD@glTexGend?$AA@ 004c8520     renderer:win_qgl.obj
 0002:0000c52c       ??_C@_0L@EHNOIKND@glTexEnviv?$AA@ 004c852c     renderer:win_qgl.obj
 0002:0000c538       ??_C@_09NFCDHIOH@glTexEnvi?$AA@ 004c8538     renderer:win_qgl.obj
 0002:0000c544       ??_C@_0L@EMICMNOO@glTexEnvfv?$AA@ 004c8544     renderer:win_qgl.obj
 0002:0000c550       ??_C@_09FCLLGECI@glTexEnvf?$AA@ 004c8550     renderer:win_qgl.obj
 0002:0000c55c       ??_C@_0BC@DAOMILMO@glTexCoordPointer?$AA@ 004c855c     renderer:win_qgl.obj
 0002:0000c570       ??_C@_0O@EBJEPFAA@glTexCoord4sv?$AA@ 004c8570     renderer:win_qgl.obj
 0002:0000c580       ??_C@_0N@CJOJLEKC@glTexCoord4s?$AA@ 004c8580     renderer:win_qgl.obj
 0002:0000c590       ??_C@_0O@FACFNDKG@glTexCoord4iv?$AA@ 004c8590     renderer:win_qgl.obj
 0002:0000c5a0       ??_C@_0N@JJMEEOHJ@glTexCoord4i?$AA@ 004c85a0     renderer:win_qgl.obj
 0002:0000c5b0       ??_C@_0O@FLHJJEJL@glTexCoord4fv?$AA@ 004c85b0     renderer:win_qgl.obj
 0002:0000c5c0       ??_C@_0N@BOFMFCLG@glTexCoord4f?$AA@ 004c85c0     renderer:win_qgl.obj
 0002:0000c5d0       ??_C@_0O@FIPNEAPF@glTexCoord4dv?$AA@ 004c85d0     renderer:win_qgl.obj
 0002:0000c5e0       ??_C@_0N@CMGKDADE@glTexCoord4d?$AA@ 004c85e0     renderer:win_qgl.obj
 0002:0000c5f0       ??_C@_0O@NMEDMNLJ@glTexCoord3sv?$AA@ 004c85f0     renderer:win_qgl.obj
 0002:0000c600       ??_C@_0N@CMKGKCCH@glTexCoord3s?$AA@ 004c8600     renderer:win_qgl.obj
 0002:0000c610       ??_C@_0O@MNPCOLBP@glTexCoord3iv?$AA@ 004c8610     renderer:win_qgl.obj
 0002:0000c620       ??_C@_0N@JMILFIPM@glTexCoord3i?$AA@ 004c8620     renderer:win_qgl.obj
 0002:0000c630       ??_C@_0O@MGKOKMCC@glTexCoord3fv?$AA@ 004c8630     renderer:win_qgl.obj
 0002:0000c640       ??_C@_0N@BLBDEEDD@glTexCoord3f?$AA@ 004c8640     renderer:win_qgl.obj
 0002:0000c650       ??_C@_0O@MFCKHIEM@glTexCoord3dv?$AA@ 004c8650     renderer:win_qgl.obj
 0002:0000c660       ??_C@_0N@CJCFCGLB@glTexCoord3d?$AA@ 004c8660     renderer:win_qgl.obj
 0002:0000c670       ??_C@_0O@GEPPKKNM@glTexCoord2sv?$AA@ 004c8670     renderer:win_qgl.obj
 0002:0000c680       ??_C@_0N@CNGEMIBA@glTexCoord2s?$AA@ 004c8680     renderer:win_qgl.obj
 0002:0000c690       ??_C@_0O@HFEOIMHK@glTexCoord2iv?$AA@ 004c8690     renderer:win_qgl.obj
 0002:0000c6a0       ??_C@_0N@JNEJDCML@glTexCoord2i?$AA@ 004c86a0     renderer:win_qgl.obj
 0002:0000c6b0       ??_C@_0O@HOBCMLEH@glTexCoord2fv?$AA@ 004c86b0     renderer:win_qgl.obj
 0002:0000c6c0       ??_C@_0N@BKNBCOAE@glTexCoord2f?$AA@ 004c86c0     renderer:win_qgl.obj
 0002:0000c6d0       ??_C@_0O@HNJGBPCJ@glTexCoord2dv?$AA@ 004c86d0     renderer:win_qgl.obj
 0002:0000c6e0       ??_C@_0N@CIOHEMIG@glTexCoord2d?$AA@ 004c86e0     renderer:win_qgl.obj
 0002:0000c6f0       ??_C@_0O@HGEKAFDC@glTexCoord1sv?$AA@ 004c86f0     renderer:win_qgl.obj
 0002:0000c700       ??_C@_0N@CPCCHGEJ@glTexCoord1s?$AA@ 004c8700     renderer:win_qgl.obj
 0002:0000c710       ??_C@_0O@GHPLCDJE@glTexCoord1iv?$AA@ 004c8710     renderer:win_qgl.obj
 0002:0000c720       ??_C@_0N@JPAPIMJC@glTexCoord1i?$AA@ 004c8720     renderer:win_qgl.obj
 0002:0000c730       ??_C@_0O@GMKHGEKJ@glTexCoord1fv?$AA@ 004c8730     renderer:win_qgl.obj
 0002:0000c740       ??_C@_0N@BIJHJAFN@glTexCoord1f?$AA@ 004c8740     renderer:win_qgl.obj
 0002:0000c750       ??_C@_0O@GPCDLAMH@glTexCoord1dv?$AA@ 004c8750     renderer:win_qgl.obj
 0002:0000c760       ??_C@_0N@CKKBPCNP@glTexCoord1d?$AA@ 004c8760     renderer:win_qgl.obj
 0002:0000c770       ??_C@_0M@BILBNGF@glStencilOp?$AA@ 004c8770     renderer:win_qgl.obj
 0002:0000c77c       ??_C@_0O@DJFHPFEP@glStencilMask?$AA@ 004c877c     renderer:win_qgl.obj
 0002:0000c78c       ??_C@_0O@ENNLLOLN@glStencilFunc?$AA@ 004c878c     renderer:win_qgl.obj
 0002:0000c79c       ??_C@_0N@NALMFHKN@glShadeModel?$AA@ 004c879c     renderer:win_qgl.obj
 0002:0000c7ac       ??_C@_0P@KACPMBCN@glSelectBuffer?$AA@ 004c87ac     renderer:win_qgl.obj
 0002:0000c7bc       ??_C@_09ECGPAEPL@glScissor?$AA@ 004c87bc     renderer:win_qgl.obj
 0002:0000c7c8       ??_C@_08JCPEOPLK@glScalef?$AA@ 004c87c8     renderer:win_qgl.obj
 0002:0000c7d4       ??_C@_08KAMCINDI@glScaled?$AA@ 004c87d4     renderer:win_qgl.obj
 0002:0000c7e0       ??_C@_09FCODNBIM@glRotatef?$AA@ 004c87e0     renderer:win_qgl.obj
 0002:0000c7ec       ??_C@_09GANFLDAO@glRotated?$AA@ 004c87ec     renderer:win_qgl.obj
 0002:0000c7f8       ??_C@_0N@HCFJFDGP@glRenderMode?$AA@ 004c87f8     renderer:win_qgl.obj
 0002:0000c808       ??_C@_08FPNOOGJA@glRectsv?$AA@ 004c8808     renderer:win_qgl.obj
 0002:0000c814       ??_C@_07GCAIEMDA@glRects?$AA@ 004c8814     renderer:win_qgl.obj
 0002:0000c81c       ??_C@_08EOGPMADG@glRectiv?$AA@ 004c881c     renderer:win_qgl.obj
 0002:0000c828       ??_C@_07NCCFLGOL@glRecti?$AA@ 004c8828     renderer:win_qgl.obj
 0002:0000c830       ??_C@_08EFDDIHAL@glRectfv?$AA@ 004c8830     renderer:win_qgl.obj
 0002:0000c83c       ??_C@_07FFLNKKCE@glRectf?$AA@ 004c883c     renderer:win_qgl.obj
 0002:0000c844       ??_C@_08EGLHFDGF@glRectdv?$AA@ 004c8844     renderer:win_qgl.obj
 0002:0000c850       ??_C@_07GHILMIKG@glRectd?$AA@ 004c8850     renderer:win_qgl.obj
 0002:0000c858       ??_C@_0N@CKFNNHOO@glReadPixels?$AA@ 004c8858     renderer:win_qgl.obj
 0002:0000c868       ??_C@_0N@HFKHBECK@glReadBuffer?$AA@ 004c8868     renderer:win_qgl.obj
 0002:0000c878       ??_C@_0P@NJGHOAAG@glRasterPos4sv?$AA@ 004c8878     renderer:win_qgl.obj
 0002:0000c888       ??_C@_0O@INMAOOA@glRasterPos4s?$AA@ 004c8888     renderer:win_qgl.obj
 0002:0000c898       ??_C@_0P@MINGMGKA@glRasterPos4iv?$AA@ 004c8898     renderer:win_qgl.obj
 0002:0000c8a8       ??_C@_0O@LIPBPEDL@glRasterPos4i?$AA@ 004c88a8     renderer:win_qgl.obj
 0002:0000c8b8       ??_C@_0P@MDIKIBJN@glRasterPos4fv?$AA@ 004c88b8     renderer:win_qgl.obj
 0002:0000c8c8       ??_C@_0O@DPGJOIPE@glRasterPos4f?$AA@ 004c88c8     renderer:win_qgl.obj
 0002:0000c8d8       ??_C@_0P@MAAOFFPD@glRasterPos4dv?$AA@ 004c88d8     renderer:win_qgl.obj
 0002:0000c8e8       ??_C@_0O@NFPIKHG@glRasterPos4d?$AA@ 004c88e8     renderer:win_qgl.obj
 0002:0000c8f8       ??_C@_0P@EELANILP@glRasterPos3sv?$AA@ 004c88f8     renderer:win_qgl.obj
 0002:0000c908       ??_C@_0O@NJDBIGF@glRasterPos3s?$AA@ 004c8908     renderer:win_qgl.obj
 0002:0000c918       ??_C@_0P@FFABPOBJ@glRasterPos3iv?$AA@ 004c8918     renderer:win_qgl.obj
 0002:0000c928       ??_C@_0O@LNLOOCLO@glRasterPos3i?$AA@ 004c8928     renderer:win_qgl.obj
 0002:0000c938       ??_C@_0P@FOFNLJCE@glRasterPos3fv?$AA@ 004c8938     renderer:win_qgl.obj
 0002:0000c948       ??_C@_0O@DKCGPOHB@glRasterPos3f?$AA@ 004c8948     renderer:win_qgl.obj
 0002:0000c958       ??_C@_0P@FNNJGNEK@glRasterPos3dv?$AA@ 004c8958     renderer:win_qgl.obj
 0002:0000c968       ??_C@_0O@IBAJMPD@glRasterPos3d?$AA@ 004c8968     renderer:win_qgl.obj
 0002:0000c978       ??_C@_0P@PMAMLPNK@glRasterPos2sv?$AA@ 004c8978     renderer:win_qgl.obj
 0002:0000c988       ??_C@_0O@MFBHCFC@glRasterPos2s?$AA@ 004c8988     renderer:win_qgl.obj
 0002:0000c998       ??_C@_0P@ONLNJJHM@glRasterPos2iv?$AA@ 004c8998     renderer:win_qgl.obj
 0002:0000c9a8       ??_C@_0O@LMHMIIIJ@glRasterPos2i?$AA@ 004c89a8     renderer:win_qgl.obj
 0002:0000c9b8       ??_C@_0P@OGOBNOEB@glRasterPos2fv?$AA@ 004c89b8     renderer:win_qgl.obj
 0002:0000c9c8       ??_C@_0O@DLOEJEEG@glRasterPos2f?$AA@ 004c89c8     renderer:win_qgl.obj
 0002:0000c9d8       ??_C@_0P@OFGFAKCP@glRasterPos2dv?$AA@ 004c89d8     renderer:win_qgl.obj
 0002:0000c9e8       ??_C@_0O@JNCPGME@glRasterPos2d?$AA@ 004c89e8     renderer:win_qgl.obj
 0002:0000c9f8       ??_C@_0L@LFFFABIK@glPushName?$AA@ 004c89f8     renderer:win_qgl.obj
 0002:0000ca04       ??_C@_0N@IHFNHGBL@glPushMatrix?$AA@ 004c8a04     renderer:win_qgl.obj
 0002:0000ca14       ??_C@_0BD@JKGPLNEA@glPushClientAttrib?$AA@ 004c8a14     renderer:win_qgl.obj
 0002:0000ca28       ??_C@_0N@KDMLHFJM@glPushAttrib?$AA@ 004c8a28     renderer:win_qgl.obj
 0002:0000ca38       ??_C@_0BF@FFCGNNIA@glPrioritizeTextures?$AA@ 004c8a38     renderer:win_qgl.obj
 0002:0000ca50       ??_C@_09IKDPIJOE@glPopName?$AA@ 004c8a50     renderer:win_qgl.obj
 0002:0000ca5c       ??_C@_0M@JPEAAEEK@glPopMatrix?$AA@ 004c8a5c     renderer:win_qgl.obj
 0002:0000ca68       ??_C@_0BC@GOOJKIDH@glPopClientAttrib?$AA@ 004c8a68     renderer:win_qgl.obj
 0002:0000ca7c       ??_C@_0M@LLNGAHMN@glPopAttrib?$AA@ 004c8a7c     renderer:win_qgl.obj
 0002:0000ca88       ??_C@_0BB@GIADEJGP@glPolygonStipple?$AA@ 004c8a88     renderer:win_qgl.obj
 0002:0000ca9c       ??_C@_0BA@FFBJGNC@glPolygonOffset?$AA@ 004c8a9c     renderer:win_qgl.obj
 0002:0000caac       ??_C@_0O@DKMNBFMB@glPolygonMode?$AA@ 004c8aac     renderer:win_qgl.obj
 0002:0000cabc       ??_C@_0M@EEAPMMNM@glPointSize?$AA@ 004c8abc     renderer:win_qgl.obj
 0002:0000cac8       ??_C@_0M@JAMJIGNB@glPixelZoom?$AA@ 004c8ac8     renderer:win_qgl.obj
 0002:0000cad4       ??_C@_0BB@IAMKJDIC@glPixelTransferi?$AA@ 004c8ad4     renderer:win_qgl.obj
 0002:0000cae8       ??_C@_0BB@HFCIPEN@glPixelTransferf?$AA@ 004c8ae8     renderer:win_qgl.obj
 0002:0000cafc       ??_C@_0O@JCCIGLOF@glPixelStorei?$AA@ 004c8afc     renderer:win_qgl.obj
 0002:0000cb0c       ??_C@_0O@BFLAHHCK@glPixelStoref?$AA@ 004c8b0c     renderer:win_qgl.obj
 0002:0000cb1c       ??_C@_0O@FMEEPGOI@glPixelMapusv?$AA@ 004c8b1c     renderer:win_qgl.obj
 0002:0000cb2c       ??_C@_0O@ENPFNAEO@glPixelMapuiv?$AA@ 004c8b2c     renderer:win_qgl.obj
 0002:0000cb3c       ??_C@_0N@CNONNBNO@glPixelMapfv?$AA@ 004c8b3c     renderer:win_qgl.obj
 0002:0000cb4c       ??_C@_0O@KCIMMNEH@glPassThrough?$AA@ 004c8b4c     renderer:win_qgl.obj
 0002:0000cb5c       ??_C@_07DBAFHOII@glOrtho?$AA@ 004c8b5c     renderer:win_qgl.obj
 0002:0000cb64       ??_C@_0BA@DCLMCEOP@glNormalPointer?$AA@ 004c8b64     renderer:win_qgl.obj
 0002:0000cb74       ??_C@_0M@NHLFGDMD@glNormal3sv?$AA@ 004c8b74     renderer:win_qgl.obj
 0002:0000cb80       ??_C@_0L@BNHPJOI@glNormal3s?$AA@ 004c8b80     renderer:win_qgl.obj
 0002:0000cb8c       ??_C@_0M@MGAEEFGF@glNormal3iv?$AA@ 004c8b8c     renderer:win_qgl.obj
 0002:0000cb98       ??_C@_0L@LBPKADDD@glNormal3i?$AA@ 004c8b98     renderer:win_qgl.obj
 0002:0000cba4       ??_C@_0M@MNFIACFI@glNormal3fv?$AA@ 004c8ba4     renderer:win_qgl.obj
 0002:0000cbb0       ??_C@_0L@DGGCBPPM@glNormal3f?$AA@ 004c8bb0     renderer:win_qgl.obj
 0002:0000cbbc       ??_C@_0M@MONMNGDG@glNormal3dv?$AA@ 004c8bbc     renderer:win_qgl.obj
 0002:0000cbc8       ??_C@_0L@EFEHNHO@glNormal3d?$AA@ 004c8bc8     renderer:win_qgl.obj
 0002:0000cbd4       ??_C@_0M@MKFBKKIE@glNormal3bv?$AA@ 004c8bd4     renderer:win_qgl.obj
 0002:0000cbe0       ??_C@_0L@FCAONKPI@glNormal3b?$AA@ 004c8be0     renderer:win_qgl.obj
 0002:0000cbec       ??_C@_09KAGOBDOO@glNewList?$AA@ 004c8bec     renderer:win_qgl.obj
 0002:0000cbf8       ??_C@_0O@LHKDNPKJ@glMultMatrixf?$AA@ 004c8bf8     renderer:win_qgl.obj
 0002:0000cc08       ??_C@_0O@IFJFLNCL@glMultMatrixd?$AA@ 004c8c08     renderer:win_qgl.obj
 0002:0000cc18       ??_C@_0N@KDLNHKEJ@glMatrixMode?$AA@ 004c8c18     renderer:win_qgl.obj
 0002:0000cc28       ??_C@_0N@HCDOEFL@glMaterialiv?$AA@ 004c8c28     renderer:win_qgl.obj
 0002:0000cc38       ??_C@_0M@PHEGJGAN@glMateriali?$AA@ 004c8c38     renderer:win_qgl.obj
 0002:0000cc44       ??_C@_0N@MHPKDGG@glMaterialfv?$AA@ 004c8c44     renderer:win_qgl.obj
 0002:0000cc54       ??_C@_0M@HANOIKMC@glMaterialf?$AA@ 004c8c54     renderer:win_qgl.obj
 0002:0000cc60       ??_C@_0M@PNEKFPAF@glMapGrid2f?$AA@ 004c8c60     renderer:win_qgl.obj
 0002:0000cc6c       ??_C@_0M@MPHMDNIH@glMapGrid2d?$AA@ 004c8c6c     renderer:win_qgl.obj
 0002:0000cc78       ??_C@_0M@PPAMOBFM@glMapGrid1f?$AA@ 004c8c78     renderer:win_qgl.obj
 0002:0000cc84       ??_C@_0M@MNDKIDNO@glMapGrid1d?$AA@ 004c8c84     renderer:win_qgl.obj
 0002:0000cc90       ??_C@_07GEAGLFKJ@glMap2f?$AA@ 004c8c90     renderer:win_qgl.obj
 0002:0000cc98       ??_C@_07FGDANHCL@glMap2d?$AA@ 004c8c98     renderer:win_qgl.obj
 0002:0000cca0       ??_C@_07GGEAALPA@glMap1f?$AA@ 004c8ca0     renderer:win_qgl.obj
 0002:0000cca8       ??_C@_07FEHGGJHC@glMap1d?$AA@ 004c8ca8     renderer:win_qgl.obj
 0002:0000ccb0       ??_C@_09GKGMNAKG@glLogicOp?$AA@ 004c8cb0     renderer:win_qgl.obj
 0002:0000ccbc       ??_C@_0L@JFFJNAJA@glLoadName?$AA@ 004c8cbc     renderer:win_qgl.obj
 0002:0000ccc8       ??_C@_0O@DJGBMGEI@glLoadMatrixf?$AA@ 004c8cc8     renderer:win_qgl.obj
 0002:0000ccd8       ??_C@_0O@LFHKEMK@glLoadMatrixd?$AA@ 004c8cd8     renderer:win_qgl.obj
 0002:0000cce8       ??_C@_0P@EJAFHEPO@glLoadIdentity?$AA@ 004c8ce8     renderer:win_qgl.obj
 0002:0000ccf8       ??_C@_0L@HDOJDFBA@glListBase?$AA@ 004c8cf8     renderer:win_qgl.obj
 0002:0000cd04       ??_C@_0M@CFLGNFPG@glLineWidth?$AA@ 004c8d04     renderer:win_qgl.obj
 0002:0000cd10       ??_C@_0O@LDOINBOK@glLineStipple?$AA@ 004c8d10     renderer:win_qgl.obj
 0002:0000cd20       ??_C@_09JDIIDONO@glLightiv?$AA@ 004c8d20     renderer:win_qgl.obj
 0002:0000cd2c       ??_C@_08DIKHJHIE@glLighti?$AA@ 004c8d2c     renderer:win_qgl.obj
 0002:0000cd38       ??_C@_09JINEHJOD@glLightfv?$AA@ 004c8d38     renderer:win_qgl.obj
 0002:0000cd44       ??_C@_08LPDPILEL@glLightf?$AA@ 004c8d44     renderer:win_qgl.obj
 0002:0000cd50       ??_C@_0P@JBCFLLOP@glLightModeliv?$AA@ 004c8d50     renderer:win_qgl.obj
 0002:0000cd60       ??_C@_0O@PILBKMEH@glLightModeli?$AA@ 004c8d60     renderer:win_qgl.obj
 0002:0000cd70       ??_C@_0P@JKHJPMNC@glLightModelfv?$AA@ 004c8d70     renderer:win_qgl.obj
 0002:0000cd80       ??_C@_0O@HPCJLAII@glLightModelf?$AA@ 004c8d80     renderer:win_qgl.obj
 0002:0000cd90       ??_C@_0M@NJHAEPDN@glIsTexture?$AA@ 004c8d90     renderer:win_qgl.obj
 0002:0000cd9c       ??_C@_08DMFMJKDH@glIsList?$AA@ 004c8d9c     renderer:win_qgl.obj
 0002:0000cda8       ??_C@_0M@INHMIHKC@glIsEnabled?$AA@ 004c8da8     renderer:win_qgl.obj
 0002:0000cdb4       ??_C@_0BE@EDEDCKLI@glInterleavedArrays?$AA@ 004c8db4     renderer:win_qgl.obj
 0002:0000cdc8       ??_C@_0M@LBOBLINN@glInitNames?$AA@ 004c8dc8     renderer:win_qgl.obj
 0002:0000cdd4       ??_C@_0L@BBKJOCAC@glIndexubv?$AA@ 004c8dd4     renderer:win_qgl.obj
 0002:0000cde0       ??_C@_09BBIPIKNC@glIndexub?$AA@ 004c8de0     renderer:win_qgl.obj
 0002:0000cdec       ??_C@_09DLKMCBDF@glIndexsv?$AA@ 004c8dec     renderer:win_qgl.obj
 0002:0000cdf8       ??_C@_08HLGHCJCJ@glIndexs?$AA@ 004c8df8     renderer:win_qgl.obj
 0002:0000ce04       ??_C@_09CKBNAHJD@glIndexiv?$AA@ 004c8e04     renderer:win_qgl.obj
 0002:0000ce10       ??_C@_08MLEKNDPC@glIndexi?$AA@ 004c8e10     renderer:win_qgl.obj
 0002:0000ce1c       ??_C@_09CBEBEAKO@glIndexfv?$AA@ 004c8e1c     renderer:win_qgl.obj
 0002:0000ce28       ??_C@_08EMNCMPDN@glIndexf?$AA@ 004c8e28     renderer:win_qgl.obj
 0002:0000ce34       ??_C@_09CCMFJEMA@glIndexdv?$AA@ 004c8e34     renderer:win_qgl.obj
 0002:0000ce40       ??_C@_08HOOEKNLP@glIndexd?$AA@ 004c8e40     renderer:win_qgl.obj
 0002:0000ce4c       ??_C@_0P@KGJBLKPD@glIndexPointer?$AA@ 004c8e4c     renderer:win_qgl.obj
 0002:0000ce5c       ??_C@_0M@ONDJOEOA@glIndexMask?$AA@ 004c8e5c     renderer:win_qgl.obj
 0002:0000ce68       ??_C@_06HEADGMBC@glHint?$AA@ 004c8e68     renderer:win_qgl.obj
 0002:0000ce70       ??_C@_0BE@DGCNLNPP@glGetTexParameteriv?$AA@ 004c8e70     renderer:win_qgl.obj
 0002:0000ce84       ??_C@_0BE@DNHBPKMC@glGetTexParameterfv?$AA@ 004c8e84     renderer:win_qgl.obj
 0002:0000ce98       ??_C@_0O@DOIIJLAD@glGetTexImage?$AA@ 004c8e98     renderer:win_qgl.obj
 0002:0000cea8       ??_C@_0O@HOAMNHM@glGetTexGeniv?$AA@ 004c8ea8     renderer:win_qgl.obj
 0002:0000ceb8       ??_C@_0O@MLMIKEB@glGetTexGenfv?$AA@ 004c8eb8     renderer:win_qgl.obj
 0002:0000cec8       ??_C@_0O@PDIFOCP@glGetTexGendv?$AA@ 004c8ec8     renderer:win_qgl.obj
 0002:0000ced8       ??_C@_0O@KIFFCCBG@glGetTexEnviv?$AA@ 004c8ed8     renderer:win_qgl.obj
 0002:0000cee8       ??_C@_0O@KDAJGFCL@glGetTexEnvfv?$AA@ 004c8ee8     renderer:win_qgl.obj
 0002:0000cef8       ??_C@_0M@OPOBFDCB@glGetString?$AA@ 004c8ef8     renderer:win_qgl.obj
 0002:0000cf04       ??_C@_0BE@PBJHLEJI@glGetPolygonStipple?$AA@ 004c8f04     renderer:win_qgl.obj
 0002:0000cf18       ??_C@_0O@LADEDGJO@glGetPointerv?$AA@ 004c8f18     renderer:win_qgl.obj
 0002:0000cf28       ??_C@_0BB@NHJEMOOF@glGetPixelMapusv?$AA@ 004c8f28     renderer:win_qgl.obj
 0002:0000cf3c       ??_C@_0BB@MGCFOIED@glGetPixelMapuiv?$AA@ 004c8f3c     renderer:win_qgl.obj
 0002:0000cf50       ??_C@_0BA@EDGNDGIE@glGetPixelMapfv?$AA@ 004c8f50     renderer:win_qgl.obj
 0002:0000cf60       ??_C@_0BA@GJKDADAB@glGetMaterialiv?$AA@ 004c8f60     renderer:win_qgl.obj
 0002:0000cf70       ??_C@_0BA@GCPPEEDM@glGetMaterialfv?$AA@ 004c8f70     renderer:win_qgl.obj
 0002:0000cf80       ??_C@_0L@FOFLNEHD@glGetMapiv?$AA@ 004c8f80     renderer:win_qgl.obj
 0002:0000cf8c       ??_C@_0L@FFAHJDEO@glGetMapfv?$AA@ 004c8f8c     renderer:win_qgl.obj
 0002:0000cf98       ??_C@_0L@FGIDEHCA@glGetMapdv?$AA@ 004c8f98     renderer:win_qgl.obj
 0002:0000cfa4       ??_C@_0N@MNDANBJN@glGetLightiv?$AA@ 004c8fa4     renderer:win_qgl.obj
 0002:0000cfb4       ??_C@_0N@MGGMJGKA@glGetLightfv?$AA@ 004c8fb4     renderer:win_qgl.obj
 0002:0000cfc4       ??_C@_0O@DHHDCCLF@glGetIntegerv?$AA@ 004c8fc4     renderer:win_qgl.obj
 0002:0000cfd4       ??_C@_0M@CKCOBONE@glGetFloatv?$AA@ 004c8fd4     renderer:win_qgl.obj
 0002:0000cfe0       ??_C@_0L@FPKAMKHB@glGetError?$AA@ 004c8fe0     renderer:win_qgl.obj
 0002:0000cfec       ??_C@_0N@OFBMMCDH@glGetDoublev?$AA@ 004c8fec     renderer:win_qgl.obj
 0002:0000cffc       ??_C@_0P@MMMNLMC@glGetClipPlane?$AA@ 004c8ffc     renderer:win_qgl.obj
 0002:0000d00c       ??_C@_0O@NLMELLCJ@glGetBooleanv?$AA@ 004c900c     renderer:win_qgl.obj
 0002:0000d01c       ??_C@_0O@LLMANLNK@glGenTextures?$AA@ 004c901c     renderer:win_qgl.obj
 0002:0000d02c       ??_C@_0L@BNOFOEBP@glGenLists?$AA@ 004c902c     renderer:win_qgl.obj
 0002:0000d038       ??_C@_09ICLFHOKP@glFrustum?$AA@ 004c9038     renderer:win_qgl.obj
 0002:0000d044       ??_C@_0M@ILBMDJDA@glFrontFace?$AA@ 004c9044     renderer:win_qgl.obj
 0002:0000d050       ??_C@_07FGBEEHCN@glFogiv?$AA@ 004c9050     renderer:win_qgl.obj
 0002:0000d058       ??_C@_06BOOFNKDM@glFogi?$AA@ 004c9058     renderer:win_qgl.obj
 0002:0000d060       ??_C@_07FNEIAABA@glFogfv?$AA@ 004c9060     renderer:win_qgl.obj
 0002:0000d068       ??_C@_06JJHNMGPD@glFogf?$AA@ 004c9068     renderer:win_qgl.obj
 0002:0000d070       ??_C@_07COFELLJA@glFlush?$AA@ 004c9070     renderer:win_qgl.obj
 0002:0000d078       ??_C@_08DFCPOKBK@glFinish?$AA@ 004c9078     renderer:win_qgl.obj
 0002:0000d084       ??_C@_0BB@COFAIKCN@glFeedbackBuffer?$AA@ 004c9084     renderer:win_qgl.obj
 0002:0000d098       ??_C@_0N@BFGDHBFK@glEvalPoint2?$AA@ 004c9098     renderer:win_qgl.obj
 0002:0000d0a8       ??_C@_0N@DOEOCCJJ@glEvalPoint1?$AA@ 004c90a8     renderer:win_qgl.obj
 0002:0000d0b8       ??_C@_0M@BJHJGIPD@glEvalMesh2?$AA@ 004c90b8     renderer:win_qgl.obj
 0002:0000d0c4       ??_C@_0M@DCFEDLDA@glEvalMesh1?$AA@ 004c90c4     renderer:win_qgl.obj
 0002:0000d0d0       ??_C@_0P@LAAAJGBJ@glEvalCoord2fv?$AA@ 004c90d0     renderer:win_qgl.obj
 0002:0000d0e0       ??_C@_0O@GJGIOPHD@glEvalCoord2f?$AA@ 004c90e0     renderer:win_qgl.obj
 0002:0000d0f0       ??_C@_0P@LDIEECHH@glEvalCoord2dv?$AA@ 004c90f0     renderer:win_qgl.obj
 0002:0000d100       ??_C@_0O@FLFOINPB@glEvalCoord2d?$AA@ 004c9100     renderer:win_qgl.obj
 0002:0000d110       ??_C@_0P@KCLFDJPH@glEvalCoord1fv?$AA@ 004c9110     renderer:win_qgl.obj
 0002:0000d120       ??_C@_0O@GLCOFBCK@glEvalCoord1f?$AA@ 004c9120     renderer:win_qgl.obj
 0002:0000d130       ??_C@_0P@KBDBONJJ@glEvalCoord1dv?$AA@ 004c9130     renderer:win_qgl.obj
 0002:0000d140       ??_C@_0O@FJBIDDKI@glEvalCoord1d?$AA@ 004c9140     renderer:win_qgl.obj
 0002:0000d150       ??_C@_09HKEBCLHH@glEndList?$AA@ 004c9150     renderer:win_qgl.obj
 0002:0000d15c       ??_C@_05OIBMBLHE@glEnd?$AA@ 004c915c     renderer:win_qgl.obj
 0002:0000d164       ??_C@_0BE@KECPKGNE@glEnableClientState?$AA@ 004c9164     renderer:win_qgl.obj
 0002:0000d178       ??_C@_08OOEHEKOP@glEnable?$AA@ 004c9178     renderer:win_qgl.obj
 0002:0000d184       ??_C@_0M@MKDGIOMK@glEdgeFlagv?$AA@ 004c9184     renderer:win_qgl.obj
 0002:0000d190       ??_C@_0BC@LILGCNN@glEdgeFlagPointer?$AA@ 004c9190     renderer:win_qgl.obj
 0002:0000d1a4       ??_C@_0L@DFCKJEPI@glEdgeFlag?$AA@ 004c91a4     renderer:win_qgl.obj
 0002:0000d1b0       ??_C@_0N@FLFIHFDP@glDrawPixels?$AA@ 004c91b0     renderer:win_qgl.obj
 0002:0000d1c0       ??_C@_0P@MENFIFGE@glDrawElements?$AA@ 004c91c0     renderer:win_qgl.obj
 0002:0000d1d0       ??_C@_0N@EKCLGPL@glDrawBuffer?$AA@ 004c91d0     renderer:win_qgl.obj
 0002:0000d1e0       ??_C@_0N@CMNPPOHA@glDrawArrays?$AA@ 004c91e0     renderer:win_qgl.obj
 0002:0000d1f0       ??_C@_0BF@LJDHBNBP@glDisableClientState?$AA@ 004c91f0     renderer:win_qgl.obj
 0002:0000d208       ??_C@_09MHGMIMKN@glDisable?$AA@ 004c9208     renderer:win_qgl.obj
 0002:0000d214       ??_C@_0N@PEBDIKOA@glDepthRange?$AA@ 004c9214     renderer:win_qgl.obj
 0002:0000d224       ??_C@_0M@KABMFLLN@glDepthMask?$AA@ 004c9224     renderer:win_qgl.obj
 0002:0000d230       ??_C@_0M@NEJABAEP@glDepthFunc?$AA@ 004c9230     renderer:win_qgl.obj
 0002:0000d23c       ??_C@_0BB@KMPLFJIC@glDeleteTextures?$AA@ 004c923c     renderer:win_qgl.obj
 0002:0000d250       ??_C@_0O@KPJIJAFM@glDeleteLists?$AA@ 004c9250     renderer:win_qgl.obj
 0002:0000d260       ??_C@_0L@BAPBLHME@glCullFace?$AA@ 004c9260     renderer:win_qgl.obj
 0002:0000d26c       ??_C@_0BE@PIJELGDB@glCopyTexSubImage2D?$AA@ 004c926c     renderer:win_qgl.obj
 0002:0000d280       ??_C@_0BE@PKNCAIGI@glCopyTexSubImage1D?$AA@ 004c9280     renderer:win_qgl.obj
 0002:0000d294       ??_C@_0BB@MGAFKJKC@glCopyTexImage2D?$AA@ 004c9294     renderer:win_qgl.obj
 0002:0000d2a8       ??_C@_0BB@MEEDBHPL@glCopyTexImage1D?$AA@ 004c92a8     renderer:win_qgl.obj
 0002:0000d2bc       ??_C@_0N@OACCOOE@glCopyPixels?$AA@ 004c92bc     renderer:win_qgl.obj
 0002:0000d2cc       ??_C@_0P@DPKEGLKI@glColorPointer?$AA@ 004c92cc     renderer:win_qgl.obj
 0002:0000d2dc       ??_C@_0BA@OOEHEGPC@glColorMaterial?$AA@ 004c92dc     renderer:win_qgl.obj
 0002:0000d2ec       ??_C@_0M@DLGOAHPH@glColorMask?$AA@ 004c92ec     renderer:win_qgl.obj
 0002:0000d2f8       ??_C@_0M@OPLLCJJN@glColor4usv?$AA@ 004c92f8     renderer:win_qgl.obj
 0002:0000d304       ??_C@_0L@NHFPGDEK@glColor4us?$AA@ 004c9304     renderer:win_qgl.obj
 0002:0000d310       ??_C@_0M@POAKAPDL@glColor4uiv?$AA@ 004c9310     renderer:win_qgl.obj
 0002:0000d31c       ??_C@_0L@GHHCJJJB@glColor4ui?$AA@ 004c931c     renderer:win_qgl.obj
 0002:0000d328       ??_C@_0M@PCFPOANK@glColor4ubv?$AA@ 004c9328     renderer:win_qgl.obj
 0002:0000d334       ??_C@_0L@IEIGEAFK@glColor4ub?$AA@ 004c9334     renderer:win_qgl.obj
 0002:0000d340       ??_C@_0L@KOKFOLLN@glColor4sv?$AA@ 004c9340     renderer:win_qgl.obj
 0002:0000d34c       ??_C@_09MNOHCDOB@glColor4s?$AA@ 004c934c     renderer:win_qgl.obj
 0002:0000d358       ??_C@_0L@LPBEMNBL@glColor4iv?$AA@ 004c9358     renderer:win_qgl.obj
 0002:0000d364       ??_C@_09HNMKNJDK@glColor4i?$AA@ 004c9364     renderer:win_qgl.obj
 0002:0000d370       ??_C@_0L@LEEIIKCG@glColor4fv?$AA@ 004c9370     renderer:win_qgl.obj
 0002:0000d37c       ??_C@_09PKFCMFPF@glColor4f?$AA@ 004c937c     renderer:win_qgl.obj
 0002:0000d388       ??_C@_0L@LHMMFOEI@glColor4dv?$AA@ 004c9388     renderer:win_qgl.obj
 0002:0000d394       ??_C@_09MIGEKHHH@glColor4d?$AA@ 004c9394     renderer:win_qgl.obj
 0002:0000d3a0       ??_C@_0L@LDEBCCPK@glColor4bv?$AA@ 004c93a0     renderer:win_qgl.obj
 0002:0000d3ac       ??_C@_09JODOAAPB@glColor4b?$AA@ 004c93ac     renderer:win_qgl.obj
 0002:0000d3b8       ??_C@_0M@FNJLPFIN@glColor3usv?$AA@ 004c93b8     renderer:win_qgl.obj
 0002:0000d3c4       ??_C@_0L@EKIIFLPD@glColor3us?$AA@ 004c93c4     renderer:win_qgl.obj
 0002:0000d3d0       ??_C@_0M@EMCKNDCL@glColor3uiv?$AA@ 004c93d0     renderer:win_qgl.obj
 0002:0000d3dc       ??_C@_0L@PKKFKBCI@glColor3ui?$AA@ 004c93dc     renderer:win_qgl.obj
 0002:0000d3e8       ??_C@_0M@EAHPDMMK@glColor3ubv?$AA@ 004c93e8     renderer:win_qgl.obj
 0002:0000d3f4       ??_C@_0L@BJFBHIOD@glColor3ub?$AA@ 004c93f4     renderer:win_qgl.obj
 0002:0000d400       ??_C@_0L@DDHCNDAE@glColor3sv?$AA@ 004c9400     renderer:win_qgl.obj
 0002:0000d40c       ??_C@_09MIKIDFGE@glColor3s?$AA@ 004c940c     renderer:win_qgl.obj
 0002:0000d418       ??_C@_0L@CCMDPFKC@glColor3iv?$AA@ 004c9418     renderer:win_qgl.obj
 0002:0000d424       ??_C@_09HIIFMPLP@glColor3i?$AA@ 004c9424     renderer:win_qgl.obj
 0002:0000d430       ??_C@_0L@CJJPLCJP@glColor3fv?$AA@ 004c9430     renderer:win_qgl.obj
 0002:0000d43c       ??_C@_09PPBNNDHA@glColor3f?$AA@ 004c943c     renderer:win_qgl.obj
 0002:0000d448       ??_C@_0L@CKBLGGPB@glColor3dv?$AA@ 004c9448     renderer:win_qgl.obj
 0002:0000d454       ??_C@_09MNCLLBPC@glColor3d?$AA@ 004c9454     renderer:win_qgl.obj
 0002:0000d460       ??_C@_0L@COJGBKED@glColor3bv?$AA@ 004c9460     renderer:win_qgl.obj
 0002:0000d46c       ??_C@_09JLHBBGHE@glColor3b?$AA@ 004c946c     renderer:win_qgl.obj
 0002:0000d478       ??_C@_0M@OHCNGGFF@glClipPlane?$AA@ 004c9478     renderer:win_qgl.obj
 0002:0000d484       ??_C@_0P@KBLPBBFP@glClearStencil?$AA@ 004c9484     renderer:win_qgl.obj
 0002:0000d494       ??_C@_0N@EIILHCMH@glClearIndex?$AA@ 004c9494     renderer:win_qgl.obj
 0002:0000d4a4       ??_C@_0N@LJIELNG@glClearDepth?$AA@ 004c94a4     renderer:win_qgl.obj
 0002:0000d4b4       ??_C@_0N@OGLMDNKC@glClearColor?$AA@ 004c94b4     renderer:win_qgl.obj
 0002:0000d4c4       ??_C@_0N@OKAMEJMG@glClearAccum?$AA@ 004c94c4     renderer:win_qgl.obj
 0002:0000d4d4       ??_C@_07IBAPPAHJ@glClear?$AA@ 004c94d4     renderer:win_qgl.obj
 0002:0000d4dc       ??_C@_0M@LFDBDICJ@glCallLists?$AA@ 004c94dc     renderer:win_qgl.obj
 0002:0000d4e8       ??_C@_0L@CIPLDIDL@glCallList?$AA@ 004c94e8     renderer:win_qgl.obj
 0002:0000d4f4       ??_C@_0M@PFBKOKOH@glBlendFunc?$AA@ 004c94f4     renderer:win_qgl.obj
 0002:0000d500       ??_C@_08PJOLDJDK@glBitmap?$AA@ 004c9500     renderer:win_qgl.obj
 0002:0000d50c       ??_C@_0O@JKKCIBGC@glBindTexture?$AA@ 004c950c     renderer:win_qgl.obj
 0002:0000d51c       ??_C@_07FCOIFMD@glBegin?$AA@ 004c951c     renderer:win_qgl.obj
 0002:0000d524       ??_C@_0P@CKCIJELG@glArrayElement?$AA@ 004c9524     renderer:win_qgl.obj
 0002:0000d534       ??_C@_0BG@DHOKJLEP@glAreTexturesResident?$AA@ 004c9534     renderer:win_qgl.obj
 0002:0000d54c       ??_C@_0M@BJGLMKCC@glAlphaFunc?$AA@ 004c954c     renderer:win_qgl.obj
 0002:0000d558       ??_C@_07LNIJJMEN@glAccum?$AA@ 004c9558     renderer:win_qgl.obj
 0002:0000d560       ??_C@_0L@IMJOIOGF@succeeded?6?$AA@ 004c9560     renderer:win_qgl.obj
 0002:0000d56c       ??_C@_0CF@ECPGGODN@?4?4?4calling?5LoadLibrary?$CI?5?8?$CFs?4dll?8@ 004c956c     renderer:win_qgl.obj
 0002:0000d598       ??_C@_0EE@CEOMEOHB@?4?4?4WARNING?3?5missing?5Glide?5instal@ 004c9598     renderer:win_qgl.obj
 0002:0000d5dc       ??_C@_0BF@OEJFCMGM@?4?4?4initializing?5QGL?6?$AA@ 004c95dc     renderer:win_qgl.obj
 0002:0000d5f4       ??_C@_0BI@EMKCPMIG@GL_LINEAR_MIPMAP_LINEAR?$AA@ 004c95f4     renderer:tr_image.obj
 0002:0000d60c       ??_C@_0BJ@HEAOEMHH@GL_NEAREST_MIPMAP_LINEAR?$AA@ 004c960c     renderer:tr_image.obj
 0002:0000d628       ??_C@_0BK@DIHBBLKN@GL_NEAREST_MIPMAP_NEAREST?$AA@ 004c9628     renderer:tr_image.obj
 0002:0000d644       ??_C@_09MNJDEIIG@GL_LINEAR?$AA@ 004c9644     renderer:tr_image.obj
 0002:0000d650       ??_C@_0L@PCHCEECD@GL_NEAREST?$AA@ 004c9650     renderer:tr_image.obj
 0002:0000d65c       ??_C@_0BB@GBGIGKBA@bad?5filter?5name?6?$AA@ 004c965c     renderer:tr_image.obj
 0002:0000d670       ??_C@_0CI@FNBBMLKI@Refusing?5to?5set?5trilinear?5on?5a?5v@ 004c9670     renderer:tr_image.obj
 0002:0000d698       ??_C@_0BD@GJNNOEIC@?5?$CFi?5total?5images?6?6?$AA@ 004c9698     renderer:tr_image.obj
 0002:0000d6ac       ??_C@_0CK@EIAOBKGB@?5?$CFi?5total?5texels?5?$CInot?5including?5@ 004c96ac     renderer:tr_image.obj
 0002:0000d6d8       ??_C@_0M@MOFGFFHA@?5?9?9?9?9?9?9?9?9?9?6?$AA@ 004c96d8     renderer:tr_image.obj
 0002:0000d6e4       ??_C@_04MDKIEGGJ@?5?$CFs?6?$AA@ 004c96e4     renderer:tr_image.obj
 0002:0000d6ec       ??_C@_05JEKGNKMI@clmp?5?$AA@ 004c96ec     renderer:tr_image.obj
 0002:0000d6f4       ??_C@_05PEEGEOBJ@rept?5?$AA@ 004c96f4     renderer:tr_image.obj
 0002:0000d6fc       ??_C@_05IBJBGJJN@S3TC?5?$AA@ 004c96fc     renderer:tr_image.obj
 0002:0000d704       ??_C@_05IKJLKKIL@?$DP?$DP?$DP?$DP?5?$AA@ 004c9704     renderer:tr_image.obj
 0002:0000d70c       ??_C@_05LCHCLIED@RGBA8?$AA@ 004c970c     renderer:tr_image.obj
 0002:0000d714       ??_C@_04BJEMBBJI@RGB8?$AA@ 004c9714     renderer:tr_image.obj
 0002:0000d71c       ??_C@_05BOMHPHEP@RGBA4?$AA@ 004c971c     renderer:tr_image.obj
 0002:0000d724       ??_C@_05GDJBOAJG@RGB5?5?$AA@ 004c9724     renderer:tr_image.obj
 0002:0000d72c       ??_C@_05DAGJCABK@RGBA?5?$AA@ 004c972c     renderer:tr_image.obj
 0002:0000d734       ??_C@_05HJHMIBAN@RGB?5?5?$AA@ 004c9734     renderer:tr_image.obj
 0002:0000d73c       ??_C@_05OACLJHN@IA?5?5?5?$AA@ 004c973c     renderer:tr_image.obj
 0002:0000d744       ??_C@_05KKFAOHIA@I?5?5?5?5?$AA@ 004c9744     renderer:tr_image.obj
 0002:0000d74c       ??_C@_0BJ@LLKIDIMA@?$CF4i?3?5?$CF4i?5?$CF4i?5?5?$CFs?5?5?5?$CFd?5?5?5?$AA@ 004c974c     renderer:tr_image.obj
 0002:0000d768       ??_C@_03ICICOMAL@yes?$AA@  004c9768     renderer:tr_image.obj
 0002:0000d76c       ??_C@_03NDENAIGM@no?5?$AA@ 004c976c     renderer:tr_image.obj
 0002:0000d770       ??_C@_0DG@JCJHFFAO@?6?5?5?5?5?5?5?9w?9?9?5?9h?9?9?5?9mm?9?5?9TMU?9?5?9if?9@ 004c9770     renderer:tr_image.obj
 0002:0000d7a8       __real@3fe8000000000000    004c97a8     renderer:tr_image.obj
 0002:0000d7b0       ??_C@_0BL@CFNJBMFH@ResampleTexture?3?5max?5width?$AA@ 004c97b0     renderer:tr_image.obj
 0002:0000d7cc       ??_C@_0CD@JDGPJFMH@R_CreateImage?3?5MAX_DRAWIMAGES?5hi@ 004c97cc     renderer:tr_image.obj
 0002:0000d7f0       ??_C@_09DIHLIDNM@?$CKlightmap?$AA@ 004c97f0     renderer:tr_image.obj
 0002:0000d7fc       ??_C@_0CB@COPOFLLF@R_CreateImage?3?5?$CC?$CFs?$CC?5is?5too?5long?6@ 004c97fc     renderer:tr_image.obj
 0002:0000d820       ??_C@_0CP@HFFCJEDA@LoadBMP?3?5illegal?5pixel_size?5?8?$CFd?8@ 004c9820     renderer:tr_image.obj
 0002:0000d850       ??_C@_0DM@FILABPHO@LoadBMP?3?5monochrome?5and?54?9bit?5BM@ 004c9850     renderer:tr_image.obj
 0002:0000d88c       ??_C@_0DF@KOIMKIGD@LoadBMP?3?5only?5uncompressed?5BMP?5f@ 004c988c     renderer:tr_image.obj
 0002:0000d8c8       ??_C@_0EA@NGPBBGNH@LoadBMP?3?5header?5size?5does?5not?5ma@ 004c98c8     renderer:tr_image.obj
 0002:0000d908       ??_C@_0DG@EEIFLDDF@LoadBMP?3?5only?5Windows?9style?5BMP?5@ 004c9908     renderer:tr_image.obj
 0002:0000d940       ??_C@_0CF@ENHIPICL@Bad?5pcx?5file?5?$CFs?5?$CI?$CFi?5x?5?$CFi?$CJ?5?$CI?$CFi?5x?5@ 004c9940     renderer:tr_image.obj
 0002:0000d968       ??_C@_0BK@PFOMPPID@PCX?5file?5?$CFs?5was?5malformed?$AA@ 004c9968     renderer:tr_image.obj
 0002:0000d988       ??_C@_0EB@OLGCIND@WARNING?3?5?8?$CFs?8?5TGA?5file?5header?5de@ 004c9988     renderer:tr_image.obj
 0002:0000d9cc       ??_C@_0CP@LECNENMO@LoadTGA?3?5illegal?5pixel_size?5?8?$CFd?8@ 004c99cc     renderer:tr_image.obj
 0002:0000d9fc       ??_C@_0DM@DMKLIHNL@LoadTGA?3?5Only?532?5or?524?5bit?5image@ 004c99fc     renderer:tr_image.obj
 0002:0000da38       ??_C@_0CC@LANFMKPP@LoadTGA?3?5colormaps?5not?5supported@ 004c9a38     renderer:tr_image.obj
 0002:0000da60       ??_C@_0EJ@MFOPHNJO@LoadTGA?3?5Only?5type?52?5?$CIRGB?$CJ?0?53?5?$CIg@ 004c9a60     renderer:tr_image.obj
 0002:0000daac       ??_C@_04GNPKBLNA@?4jpg?$AA@ 004c9aac     renderer:tr_image.obj
 0002:0000dab4       ??_C@_04LJDDIHIK@?4bmp?$AA@ 004c9ab4     renderer:tr_image.obj
 0002:0000dabc       ??_C@_04IBGELPJM@?4pcx?$AA@ 004c9abc     renderer:tr_image.obj
 0002:0000dac4       ??_C@_04JCAPCJAP@?4tga?$AA@ 004c9ac4     renderer:tr_image.obj
 0002:0000dacc       ??_C@_0DK@MNCNIICN@WARNING?3?5reused?5image?5?$CFs?5with?5mi@ 004c9acc     renderer:tr_image.obj
 0002:0000db08       ??_C@_0DG@MEFHLIGB@WARNING?3?5reused?5image?5?$CFs?5with?5mi@ 004c9b08     renderer:tr_image.obj
 0002:0000db40       ??_C@_0DB@JBEOHFBI@WARNING?3?5reused?5image?5?$CFs?5with?5mi@ 004c9b40     renderer:tr_image.obj
 0002:0000db74       ??_C@_06LLGHKAEB@?$CKwhite?$AA@ 004c9b74     renderer:tr_image.obj
 0002:0000db7c       ??_C@_0O@HNBMHJNF@trying?5?$CFs?4?4?4?6?$AA@ 004c9b7c     renderer:tr_image.obj
 0002:0000db8c       ??_C@_07MNOAAFDD@?$CKdlight?$AA@ 004c9b8c     renderer:tr_image.obj
 0002:0000db94       __real@457a0000            004c9b94     renderer:tr_image.obj
 0002:0000db98       __real@40f00000            004c9b98     renderer:tr_image.obj
 0002:0000db9c       __real@3b808081            004c9b9c     renderer:tr_image.obj
 0002:0000dba0       __real@c37f0000            004c9ba0     renderer:tr_image.obj
 0002:0000dba4       __real@3f888889            004c9ba4     renderer:tr_image.obj
 0002:0000dba8       __real@3d000000            004c9ba8     renderer:tr_image.obj
 0002:0000dbb0       __real@3fef000000000000    004c9bb0     renderer:tr_image.obj
 0002:0000dbb8       __real@3fa0000000000000    004c9bb8     renderer:tr_image.obj
 0002:0000dbc0       __real@3f60000000000000    004c9bc0     renderer:tr_image.obj
 0002:0000dbc8       ??_C@_04MFNGOGOF@?$CKfog?$AA@ 004c9bc8     renderer:tr_image.obj
 0002:0000dbd0       ??_C@_08KPIGECMN@?$CKdefault?$AA@ 004c9bd0     renderer:tr_image.obj
 0002:0000dbdc       ??_C@_08HHPIHCEN@?$CKscratch?$AA@ 004c9bdc     renderer:tr_image.obj
 0002:0000dbe8       ??_C@_0P@IACCPHGD@?$CKidentityLight?$AA@ 004c9be8     renderer:tr_image.obj
 0002:0000dbf8       __real@406fe00000000000    004c9bf8     renderer:tr_image.obj
 0002:0000dc00       ??_C@_03NBLACKLF@3?40?$AA@ 004c9c00     renderer:tr_image.obj
 0002:0000dc04       ??_C@_0CG@DBBAHOML@Empty?5name?5passed?5to?5RE_Register@ 004c9c04     renderer:tr_image.obj
 0002:0000dc2c       ??_C@_04MGKOECLF@tag_?$AA@ 004c9c2c     renderer:tr_image.obj
 0002:0000dc34       ??_C@_05JNLGGGIB@?4skin?$AA@ 004c9c34     renderer:tr_image.obj
 0002:0000dc3c       ??_C@_0DA@INLCLALN@WARNING?3?5RE_RegisterSkin?$CI?5?8?$CFs?8?5?$CJ@ 004c9c3c     renderer:tr_image.obj
 0002:0000dc6c       ??_C@_0BN@KCHDLGKI@Skin?5name?5exceeds?5MAX_QPATH?6?$AA@ 004c9c6c     renderer:tr_image.obj
 0002:0000dc8c       ??_C@_0P@BKIAPLDF@?$DMdefault?5skin?$DO?$AA@ 004c9c8c     renderer:tr_image.obj
 0002:0000dc9c       ??_C@_0BA@EEMBKHGA@?5?5?5?5?5?5?5?$CFs?5?$DN?5?$CFs?6?$AA@ 004c9c9c     renderer:tr_image.obj
 0002:0000dcac       ??_C@_0CD@NLAAGEFK@flare?5adds?3?$CFi?5tests?3?$CFi?5renders?3?$CF@ 004c9cac     renderer:tr_cmds.obj
 0002:0000dcd0       ??_C@_0M@CAGENDME@zFar?3?5?$CF?40f?6?$AA@ 004c9cd0     renderer:tr_cmds.obj
 0002:0000dcdc       ??_C@_0CN@IIFCDMCN@dlight?5srf?3?$CFi?5?5culled?3?$CFi?5?5verts?3@ 004c9cdc     renderer:tr_cmds.obj
 0002:0000dd0c       ??_C@_0BB@ODENPAFM@viewcluster?3?5?$CFi?6?$AA@ 004c9d0c     renderer:tr_cmds.obj
 0002:0000dd20       ??_C@_0DI@CLNINGCE@?$CImd3?$CJ?5?$CFi?5sin?5?$CFi?5sclip?5?5?$CFi?5sout?5?$CF@ 004c9d20     renderer:tr_cmds.obj
 0002:0000dd58       ??_C@_0DK@PDABEOHF@?$CIpatch?$CJ?5?$CFi?5sin?5?$CFi?5sclip?5?5?$CFi?5sout@ 004c9d58     renderer:tr_cmds.obj
 0002:0000dd98       ??_C@_0EE@IJFCGEK@?$CFi?1?$CFi?5shaders?1surfs?5?$CFi?5leafs?5?$CFi?5@ 004c9d98     renderer:tr_cmds.obj
 0002:0000dddc       __real@358637bd            004c9ddc     renderer:tr_cmds.obj
 0002:0000dde0       ??_C@_0M@IPNOCDNB@?4?4?4failed?4?6?$AA@ 004c9de0     renderer:tr_cmds.obj
 0002:0000ddec       ??_C@_0P@HOCIIEJB@?4?4?4succeeded?4?6?$AA@ 004c9dec     renderer:tr_cmds.obj
 0002:0000ddfc       ??_C@_0BM@JMNGBMDE@Trying?5SMP?5acceleration?4?4?4?6?$AA@ 004c9dfc     renderer:tr_cmds.obj
 0002:0000de18       ??_C@_0CA@BOMALFJA@R_GetCommandBuffer?3?5bad?5size?5?$CFi?$AA@ 004c9e18     renderer:tr_cmds.obj
 0002:0000de38       ??_C@_0DK@NPPAJLCP@RE_BeginFrame?3?5Stereo?5is?5disable@ 004c9e38     renderer:tr_cmds.obj
 0002:0000de74       ??_C@_0DJ@HLGALEHO@RE_BeginFrame?3?5Stereo?5is?5enabled@ 004c9e74     renderer:tr_cmds.obj
 0002:0000deb0       ??_C@_0CP@PGCGPPGN@RE_BeginFrame?$CI?$CJ?5?9?5glGetError?$CI?$CJ?5f@ 004c9eb0     renderer:tr_cmds.obj
 0002:0000dee0       ??_C@_0EK@OFLLHINH@Warning?3?5stencil?5shadows?5and?5ove@ 004c9ee0     renderer:tr_cmds.obj
 0002:0000df2c       ??_C@_0DK@JPMHOIDD@Warning?3?5not?5enough?5stencil?5bits@ 004c9f2c     renderer:tr_cmds.obj
 0002:0000df68       ??_C@_0BF@OHALGONN@GL_Bind?3?5NULL?5image?6?$AA@ 004c9f68     renderer:tr_backend.obj
 0002:0000df80       ??_C@_0BM@MKDPKBLD@GL_SelectTexture?3?5unit?5?$DN?5?$CFi?$AA@ 004c9f80     renderer:tr_backend.obj
 0002:0000df9c       ??_C@_0CN@JJAMLFKM@glClientActiveTextureARB?$CI?5GL_TEX@ 004c9f9c     renderer:tr_backend.obj
 0002:0000dfcc       ??_C@_0CH@EBJBHDDO@glActiveTextureARB?$CI?5GL_TEXTURE1_@ 004c9fcc     renderer:tr_backend.obj
 0002:0000dff4       ??_C@_0CN@IOHHKBOP@glClientActiveTextureARB?$CI?5GL_TEX@ 004c9ff4     renderer:tr_backend.obj
 0002:0000e024       ??_C@_0CH@FGOKGHHN@glActiveTextureARB?$CI?5GL_TEXTURE0_@ 004ca024     renderer:tr_backend.obj
 0002:0000e04c       ??_C@_0CE@DIKCONAP@GL_TexEnv?3?5invalid?5env?5?8?$CFd?8?5pass@ 004ca04c     renderer:tr_backend.obj
 0002:0000e070       ??_C@_0CI@MPNHLHAM@GL_State?3?5invalid?5dst?5blend?5stat@ 004ca070     renderer:tr_backend.obj
 0002:0000e098       ??_C@_0CI@JNKBENCF@GL_State?3?5invalid?5src?5blend?5stat@ 004ca098     renderer:tr_backend.obj
 0002:0000e0c0       __real@3fd3333333333333    004ca0c0     renderer:tr_backend.obj
 0002:0000e0c8       ??_C@_0CC@BHAIMEHO@qglTexSubImage2D?5?$CFi?0?5?$CFi?3?5?$CFi?5msec@ 004ca0c8     renderer:tr_backend.obj
 0002:0000e0ec       ??_C@_0DB@BADIHKNP@Draw_StretchRaw?3?5size?5not?5a?5powe@ 004ca0ec     renderer:tr_backend.obj
 0002:0000e120       ??_C@_0BM@CDGHDPNH@?$CFi?5msec?5to?5draw?5all?5images?6?$AA@ 004ca120     renderer:tr_backend.obj
 0002:0000e13c       ??_C@_0DG@CHHALGE@?$CK?$CK?$CK?$CK?$CK?$CK?$CK?$CK?$CK?$CK?$CK?$CK?$CK?$CK?$CK?$CK?$CK?5RB_SwapBuffers@ 004ca13c     renderer:tr_backend.obj
 0002:0000e174       ??_C@_0DL@BKDLJMAM@R_LoadMD3?3?5?$CFs?5has?5more?5than?5?$CFi?5t@ 004ca174     renderer:tr_model.obj
 0002:0000e1b0       ??_C@_0DH@KLLOOHPD@R_LoadMD3?3?5?$CFs?5has?5more?5than?5?$CFi?5v@ 004ca1b0     renderer:tr_model.obj
 0002:0000e1e8       ??_C@_0BN@JENBICHP@R_LoadMD3?3?5?$CFs?5has?5no?5frames?6?$AA@ 004ca1e8     renderer:tr_model.obj
 0002:0000e208       ??_C@_0DD@KHJJKPOK@R_LoadMD3?3?5?$CFs?5has?5wrong?5version?5@ 004ca208     renderer:tr_model.obj
 0002:0000e23c       ??_C@_0BN@PNDGAECH@R_LoadMD4?3?5?$CFs?5has?5no?5frames?6?$AA@ 004ca23c     renderer:tr_model.obj
 0002:0000e25c       ??_C@_0DD@KJJDGJEK@R_LoadMD4?3?5?$CFs?5has?5wrong?5version?5@ 004ca25c     renderer:tr_model.obj
 0002:0000e290       ??_C@_0BE@IACJADAH@?$CF8i?5?3?5Total?5models?6?$AA@ 004ca290     renderer:tr_model.obj
 0002:0000e2a4       ??_C@_0P@FDGJGCED@?$CF8i?5?3?5?$CI?$CFi?$CJ?5?$CFs?6?$AA@ 004ca2a4     renderer:tr_model.obj
 0002:0000e2b4       ??_C@_0BN@KFFAINND@RE_RegisterModel?3?5NULL?5name?6?$AA@ 004ca2b4     renderer:tr_model.obj
 0002:0000e2d4       ??_C@_0CJ@CAIMAAFD@RE_RegisterModel?3?5unknown?5fileid@ 004ca2d4     renderer:tr_model.obj
 0002:0000e300       ??_C@_0DC@CLACIFFN@RE_RegisterModel?3?5R_AllocModel?$CI?$CJ@ 004ca300     renderer:tr_model.obj
 0002:0000e334       ??_C@_07BEDDCCPM@_?$CFd?4md3?$AA@ 004ca334     renderer:tr_model.obj
 0002:0000e33c       ??_C@_0BO@FCMCBBHN@Model?5name?5exceeds?5MAX_QPATH?6?$AA@ 004ca33c     renderer:tr_model.obj
 0002:0000e35c       ??_C@_04BEGKODDK@dust?$AA@ 004ca35c     renderer:tr_shader.obj
 0002:0000e364       ??_C@_08LLBHFIEL@nodlight?$AA@ 004ca364     renderer:tr_shader.obj
 0002:0000e370       ??_C@_0L@MKEHCLJM@nolightmap?$AA@ 004ca370     renderer:tr_shader.obj
 0002:0000e37c       ??_C@_0L@CHECABJO@pointlight?$AA@ 004ca37c     renderer:tr_shader.obj
 0002:0000e388       ??_C@_06MEFHFNAK@nodraw?$AA@ 004ca388     renderer:tr_shader.obj
 0002:0000e390       ??_C@_07PPLNNCCH@nosteps?$AA@ 004ca390     renderer:tr_shader.obj
 0002:0000e398       ??_C@_05DLDJBIMA@flesh?$AA@ 004ca398     renderer:tr_shader.obj
 0002:0000e3a0       ??_C@_0L@BIBBDCEB@metalsteps?$AA@ 004ca3a0     renderer:tr_shader.obj
 0002:0000e3ac       ??_C@_08IPOHNGKE@nodamage?$AA@ 004ca3ac     renderer:tr_shader.obj
 0002:0000e3b8       ??_C@_06GGMOHJIJ@ladder?$AA@ 004ca3b8     renderer:tr_shader.obj
 0002:0000e3c0       ??_C@_07LDNMIKIJ@nomarks?$AA@ 004ca3c0     renderer:tr_shader.obj
 0002:0000e3c8       ??_C@_08FFFCKPOA@noimpact?$AA@ 004ca3c8     renderer:tr_shader.obj
 0002:0000e3d4       ??_C@_05BFPPMEOD@slick?$AA@ 004ca3d4     renderer:tr_shader.obj
 0002:0000e3dc       ??_C@_04NPKLNGDP@hint?$AA@ 004ca3dc     renderer:tr_shader.obj
 0002:0000e3e4       ??_C@_0M@GKGEABAN@alphashadow?$AA@ 004ca3e4     renderer:tr_shader.obj
 0002:0000e3f0       ??_C@_0M@FCGGILAO@lightfilter?$AA@ 004ca3f0     renderer:tr_shader.obj
 0002:0000e3fc       ??_C@_03BNEOMJOP@sky?$AA@  004ca3fc     renderer:tr_shader.obj
 0002:0000e400       ??_C@_03KJMBPJEB@fog?$AA@  004ca400     renderer:tr_shader.obj
 0002:0000e404       ??_C@_0L@BIKHJKPM@donotenter?$AA@ 004ca404     renderer:tr_shader.obj
 0002:0000e410       ??_C@_0O@GEGDJGOB@clusterportal?$AA@ 004ca410     renderer:tr_shader.obj
 0002:0000e420       ??_C@_0L@PPDFKPM@areaportal?$AA@ 004ca420     renderer:tr_shader.obj
 0002:0000e42c       ??_C@_0L@GMELLABP@structural?$AA@ 004ca42c     renderer:tr_shader.obj
 0002:0000e438       ??_C@_06EENFNEPD@detail?$AA@ 004ca438     renderer:tr_shader.obj
 0002:0000e440       ??_C@_05JIFNPOFN@trans?$AA@ 004ca440     renderer:tr_shader.obj
 0002:0000e448       ??_C@_06NHCMNMEH@origin?$AA@ 004ca448     renderer:tr_shader.obj
 0002:0000e450       ??_C@_08POKGLNIM@nonsolid?$AA@ 004ca450     renderer:tr_shader.obj
 0002:0000e45c       ??_C@_06IBIIOGMH@nodrop?$AA@ 004ca45c     renderer:tr_shader.obj
 0002:0000e464       ??_C@_0M@IHNOGBMG@monsterclip?$AA@ 004ca464     renderer:tr_shader.obj
 0002:0000e470       ??_C@_0L@BLJOELF@playerclip?$AA@ 004ca470     renderer:tr_shader.obj
 0002:0000e47c       ??_C@_04MKBPEMMM@lava?$AA@ 004ca47c     renderer:tr_shader.obj
 0002:0000e484       ??_C@_05IBOCMEGH@slime?$AA@ 004ca484     renderer:tr_shader.obj
 0002:0000e48c       ??_C@_05ELAABIKM@water?$AA@ 004ca48c     renderer:tr_shader.obj
 0002:0000e494       ??_C@_02LEBOADDI@dn?$AA@   004ca494     renderer:tr_shader.obj
 0002:0000e498       ??_C@_02HNLLPFKA@up?$AA@   004ca498     renderer:tr_shader.obj
 0002:0000e49c       ??_C@_02HLHCNIN@ft?$AA@    004ca49c     renderer:tr_shader.obj
 0002:0000e4a0       ??_C@_02HCNENIII@lf?$AA@   004ca4a0     renderer:tr_shader.obj
 0002:0000e4a4       ??_C@_02MNOEILMP@bk?$AA@   004ca4a4     renderer:tr_shader.obj
 0002:0000e4a8       ??_C@_02BMJICGCB@rt?$AA@   004ca4a8     renderer:tr_shader.obj
 0002:0000e4ac       ??_C@_0DA@MPCOKHDD@WARNING?3?5missing?5vector?5element?5@ 004ca4ac     renderer:tr_shader.obj
 0002:0000e4dc       ??_C@_0CN@BPDNDCOG@WARNING?3?5missing?5parenthesis?5in?5@ 004ca4dc     renderer:tr_shader.obj
 0002:0000e50c       ??_C@_0DF@FIOFMDKK@WARNING?3?5invalid?5alphaFunc?5name?5@ 004ca50c     renderer:tr_shader.obj
 0002:0000e544       ??_C@_05LEJEKBHA@GE128?$AA@ 004ca544     renderer:tr_shader.obj
 0002:0000e54c       ??_C@_05IDNDOPIB@LT128?$AA@ 004ca54c     renderer:tr_shader.obj
 0002:0000e554       ??_C@_03GMILPAPI@GT0?$AA@  004ca554     renderer:tr_shader.obj
 0002:0000e558       ??_C@_0EG@NFEMCCHE@WARNING?3?5unknown?5blend?5mode?5?8?$CFs?8@ 004ca558     renderer:tr_shader.obj
 0002:0000e5a0       ??_C@_0BG@GMACLBML@GL_SRC_ALPHA_SATURATE?$AA@ 004ca5a0     renderer:tr_shader.obj
 0002:0000e5b8       ??_C@_0BH@BIGHMICL@GL_ONE_MINUS_DST_ALPHA?$AA@ 004ca5b8     renderer:tr_shader.obj
 0002:0000e5d0       ??_C@_0BH@MIBHBKCA@GL_ONE_MINUS_SRC_COLOR?$AA@ 004ca5d0     renderer:tr_shader.obj
 0002:0000e5e8       ??_C@_0N@ODLEFAAC@GL_SRC_COLOR?$AA@ 004ca5e8     renderer:tr_shader.obj
 0002:0000e5f8       ??_C@_0DD@DLNAFJMK@WARNING?3?5invalid?5genfunc?5name?5?8?$CF@ 004ca5f8     renderer:tr_shader.obj
 0002:0000e62c       ??_C@_05GPLCCBII@noise?$AA@ 004ca62c     renderer:tr_shader.obj
 0002:0000e634       ??_C@_0BA@CLNFMHNL@inversesawtooth?$AA@ 004ca634     renderer:tr_shader.obj
 0002:0000e644       ??_C@_08PDBODDPM@sawtooth?$AA@ 004ca644     renderer:tr_shader.obj
 0002:0000e650       ??_C@_08FOPOJBJM@triangle?$AA@ 004ca650     renderer:tr_shader.obj
 0002:0000e65c       ??_C@_06ICDKOIFG@square?$AA@ 004ca65c     renderer:tr_shader.obj
 0002:0000e664       ??_C@_03BLEJJJBH@sin?$AA@  004ca664     renderer:tr_shader.obj
 0002:0000e668       ??_C@_0CP@DKEEEEHD@WARNING?3?5missing?5waveform?5parm?5i@ 004ca668     renderer:tr_shader.obj
 0002:0000e698       ??_C@_0CM@BIKEMJGH@WARNING?3?5unknown?5tcMod?5?8?$CFs?8?5in?5s@ 004ca698     renderer:tr_shader.obj
 0002:0000e6c4       ??_C@_0BA@JHGJPDGP@entityTranslate?$AA@ 004ca6c4     renderer:tr_shader.obj
 0002:0000e6d4       ??_C@_0DE@CPIKJPCO@WARNING?3?5missing?5tcMod?5rotate?5pa@ 004ca6d4     renderer:tr_shader.obj
 0002:0000e708       ??_C@_06CEHMNFAL@rotate?$AA@ 004ca708     renderer:tr_shader.obj
 0002:0000e710       ??_C@_0DB@HCGDEMJB@WARNING?3?5missing?5transform?5parms@ 004ca710     renderer:tr_shader.obj
 0002:0000e744       ??_C@_09IFONHNKG@transform?$AA@ 004ca744     renderer:tr_shader.obj
 0002:0000e750       ??_C@_0CP@GCKFKABP@WARNING?3?5missing?5stretch?5parms?5i@ 004ca750     renderer:tr_shader.obj
 0002:0000e780       ??_C@_07LEPFLFDH@stretch?$AA@ 004ca780     renderer:tr_shader.obj
 0002:0000e788       ??_C@_0DE@KNBGFEPJ@WARNING?3?5missing?5scale?5scroll?5pa@ 004ca788     renderer:tr_shader.obj
 0002:0000e7bc       ??_C@_06FJKBNFNG@scroll?$AA@ 004ca7bc     renderer:tr_shader.obj
 0002:0000e7c4       ??_C@_0CN@BBMLEDFN@WARNING?3?5missing?5scale?5parms?5in?5@ 004ca7c4     renderer:tr_shader.obj
 0002:0000e7f4       ??_C@_05MHMEBBGO@scale?$AA@ 004ca7f4     renderer:tr_shader.obj
 0002:0000e7fc       ??_C@_0CM@KOGGLEIE@WARNING?3?5missing?5tcMod?5turb?5in?5s@ 004ca7fc     renderer:tr_shader.obj
 0002:0000e828       ??_C@_0DC@NOBDKEOI@WARNING?3?5missing?5tcMod?5turb?5parm@ 004ca828     renderer:tr_shader.obj
 0002:0000e85c       ??_C@_04GJNAKLFI@turb?$AA@ 004ca85c     renderer:tr_shader.obj
 0002:0000e864       ??_C@_0CN@JIBKBGGH@ERROR?3?5too?5many?5tcMod?5stages?5in?5@ 004ca864     renderer:tr_shader.obj
 0002:0000e894       ??_C@_0DA@LHNAOODG@WARNING?3?5unknown?5parameter?5?8?$CFs?8?5@ 004ca894     renderer:tr_shader.obj
 0002:0000e8c8       ??_C@_0ED@GFKIPHND@WARNING?3?5missing?5parameter?5for?5?8@ 004ca8c8     renderer:tr_shader.obj
 0002:0000e910       ??_C@_0ED@OOIKPLLE@WARNING?3?5missing?5parameter?5for?5?8@ 004ca910     renderer:tr_shader.obj
 0002:0000e958       ??_C@_0ED@JEBNHGPN@WARNING?3?5missing?5parameter?5for?5?8@ 004ca958     renderer:tr_shader.obj
 0002:0000e9a0       ??_C@_0EC@PDBNEELC@WARNING?3?5missing?5parameter?5for?5?8@ 004ca9a0     renderer:tr_shader.obj
 0002:0000e9e8       ??_C@_0EC@FAEJMGED@WARNING?3?5missing?5parameter?5for?5?8@ 004ca9e8     renderer:tr_shader.obj
 0002:0000ea2c       ??_C@_0DN@CLBKOKJO@WARNING?3?5missing?5parameter?5for?5?8@ 004caa2c     renderer:tr_shader.obj
 0002:0000ea6c       ??_C@_0CA@OOLPPJGG@WARNING?3?5no?5matching?5?8?$HN?8?5found?6?$AA@ 004caa6c     renderer:tr_shader.obj
 0002:0000ea8c       ??_C@_0CN@BFINHNOM@WARNING?3?5unknown?5texgen?5parm?5in?5@ 004caa8c     renderer:tr_shader.obj
 0002:0000eabc       ??_C@_06NBFPPGEG@vector?$AA@ 004caabc     renderer:tr_shader.obj
 0002:0000eac4       ??_C@_04BHIIPFEC@base?$AA@ 004caac4     renderer:tr_shader.obj
 0002:0000eacc       ??_C@_07JDHEGGGP@texture?$AA@ 004caacc     renderer:tr_shader.obj
 0002:0000ead4       ??_C@_08GFIHGMBN@lightmap?$AA@ 004caad4     renderer:tr_shader.obj
 0002:0000eae0       ??_C@_0M@PINLHHEI@environment?$AA@ 004caae0     renderer:tr_shader.obj
 0002:0000eaec       ??_C@_0CN@NPBJMNFM@WARNING?3?5missing?5texgen?5parm?5in?5@ 004caaec     renderer:tr_shader.obj
 0002:0000eb1c       ??_C@_0L@LLDCFDJB@depthwrite?$AA@ 004cab1c     renderer:tr_shader.obj
 0002:0000eb28       ??_C@_05CLHILOEI@tcMod?$AA@ 004cab28     renderer:tr_shader.obj
 0002:0000eb30       ??_C@_05LDLNDDHA@tcGen?$AA@ 004cab30     renderer:tr_shader.obj
 0002:0000eb38       ??_C@_06PILMGBAG@texgen?$AA@ 004cab38     renderer:tr_shader.obj
 0002:0000eb40       ??_C@_0DJ@CNPGHDHL@WARNING?3?5unknown?5alphaGen?5parame@ 004cab40     renderer:tr_shader.obj
 0002:0000eb80       ??_C@_0FI@HDECGDLN@WARNING?3?5missing?5range?5parameter@ 004cab80     renderer:tr_shader.obj
 0002:0000ebd8       ??_C@_06JAELEMPN@portal?$AA@ 004cabd8     renderer:tr_shader.obj
 0002:0000ebe0       ??_C@_0BB@IPMOEOM@lightingSpecular?$AA@ 004cabe0     renderer:tr_shader.obj
 0002:0000ebf4       ??_C@_0DJ@COAGBCFB@WARNING?3?5missing?5parameters?5for?5@ 004cabf4     renderer:tr_shader.obj
 0002:0000ec30       ??_C@_08MKJGOHMF@alphaGen?$AA@ 004cac30     renderer:tr_shader.obj
 0002:0000ec3c       ??_C@_0DH@IFLDHGBE@WARNING?3?5unknown?5rgbGen?5paramete@ 004cac3c     renderer:tr_shader.obj
 0002:0000ec74       ??_C@_0P@GOBJMPDO@oneMinusVertex?$AA@ 004cac74     renderer:tr_shader.obj
 0002:0000ec84       ??_C@_0BA@JGIIOMOF@lightingDiffuse?$AA@ 004cac84     renderer:tr_shader.obj
 0002:0000ec94       ??_C@_0M@NFGCOAEO@exactVertex?$AA@ 004cac94     renderer:tr_shader.obj
 0002:0000eca0       ??_C@_06HLKHCFCI@vertex?$AA@ 004caca0     renderer:tr_shader.obj
 0002:0000eca8       ??_C@_0P@HLCEDLEK@oneMinusEntity?$AA@ 004caca8     renderer:tr_shader.obj
 0002:0000ecb8       ??_C@_06GOJKNBFM@entity?$AA@ 004cacb8     renderer:tr_shader.obj
 0002:0000ecc0       ??_C@_0BB@LOAKDOL@identityLighting?$AA@ 004cacc0     renderer:tr_shader.obj
 0002:0000ecd4       ??_C@_08LBJOIDDC@identity?$AA@ 004cacd4     renderer:tr_shader.obj
 0002:0000ece0       ??_C@_05BNCCCJPP@const?$AA@ 004cace0     renderer:tr_shader.obj
 0002:0000ece8       ??_C@_04LJEDCPFL@wave?$AA@ 004cace8     renderer:tr_shader.obj
 0002:0000ecf0       ??_C@_0DH@BMDJGBJJ@WARNING?3?5missing?5parameters?5for?5@ 004cacf0     renderer:tr_shader.obj
 0002:0000ed28       ??_C@_06FMMGNFCK@rgbGen?$AA@ 004cad28     renderer:tr_shader.obj
 0002:0000ed30       ??_C@_0DE@LHICOKDF@WARNING?3?5missing?5parm?5for?5blendF@ 004cad30     renderer:tr_shader.obj
 0002:0000ed64       ??_C@_05BIODCFPJ@blend?$AA@ 004cad64     renderer:tr_shader.obj
 0002:0000ed6c       ??_C@_06EOIELIPE@filter?$AA@ 004cad6c     renderer:tr_shader.obj
 0002:0000ed74       ??_C@_03BDGOHNNK@add?$AA@  004cad74     renderer:tr_shader.obj
 0002:0000ed78       ??_C@_09OFNNOJFC@blendfunc?$AA@ 004cad78     renderer:tr_shader.obj
 0002:0000ed84       ??_C@_0DA@BIDNCEP@WARNING?3?5unknown?5depthfunc?5?8?$CFs?8?5@ 004cad84     renderer:tr_shader.obj
 0002:0000edb4       ??_C@_05OAKNMNI@equal?$AA@ 004cadb4     renderer:tr_shader.obj
 0002:0000edbc       ??_C@_06GOLCIEJE@lequal?$AA@ 004cadbc     renderer:tr_shader.obj
 0002:0000edc4       ??_C@_09MEFHBDPK@depthfunc?$AA@ 004cadc4     renderer:tr_shader.obj
 0002:0000edd0       ??_C@_09MIGNOGJD@alphaFunc?$AA@ 004cadd0     renderer:tr_shader.obj
 0002:0000eddc       ??_C@_08GGBNKEBM@videoMap?$AA@ 004caddc     renderer:tr_shader.obj
 0002:0000ede8       ??_C@_07BMBIACGE@animMap?$AA@ 004cade8     renderer:tr_shader.obj
 0002:0000edf0       ??_C@_08DEEDKPOB@clampmap?$AA@ 004cadf0     renderer:tr_shader.obj
 0002:0000edfc       ??_C@_0DN@EAKLECLL@WARNING?3?5R_FindImageFile?5could?5n@ 004cadfc     renderer:tr_shader.obj
 0002:0000ee3c       ??_C@_09CGLCLDGP@$lightmap?$AA@ 004cae3c     renderer:tr_shader.obj
 0002:0000ee48       ??_C@_0M@BDLBCOHL@$whiteimage?$AA@ 004cae48     renderer:tr_shader.obj
 0002:0000ee58       ??_C@_0ED@LOPFOKI@WARNING?3?5unknown?5deformVertexes?5@ 004cae58     renderer:tr_shader.obj
 0002:0000ee9c       ??_C@_04HDMMNHEL@move?$AA@ 004cae9c     renderer:tr_shader.obj
 0002:0000eea4       ??_C@_06IKLLLDHL@normal?$AA@ 004caea4     renderer:tr_shader.obj
 0002:0000eeb0       ??_C@_0EL@ODFGAGPK@WARNING?3?5illegal?5div?5value?5of?50?5@ 004caeb0     renderer:tr_shader.obj
 0002:0000eefc       ??_C@_0DF@DFJPIOJM@WARNING?3?5missing?5deformVertexes?5@ 004caefc     renderer:tr_shader.obj
 0002:0000ef34       ??_C@_0DL@MGCKFNID@WARNING?3?5missing?5deformVertexes?5@ 004caf34     renderer:tr_shader.obj
 0002:0000ef70       ??_C@_05BONBJFEO@bulge?$AA@ 004caf70     renderer:tr_shader.obj
 0002:0000ef78       ??_C@_04CIMGMMMG@text?$AA@ 004caf78     renderer:tr_shader.obj
 0002:0000ef80       ??_C@_0M@JPJOBJAO@autosprite2?$AA@ 004caf80     renderer:tr_shader.obj
 0002:0000ef8c       ??_C@_0L@OJCKPKMG@autosprite?$AA@ 004caf8c     renderer:tr_shader.obj
 0002:0000ef98       ??_C@_0BB@OOOFIDJN@projectionShadow?$AA@ 004caf98     renderer:tr_shader.obj
 0002:0000efac       ??_C@_0CF@BCAMFONL@WARNING?3?5MAX_SHADER_DEFORMS?5in?5?8@ 004cafac     renderer:tr_shader.obj
 0002:0000efd4       ??_C@_0CN@BAHOFFDJ@WARNING?3?5missing?5deform?5parm?5in?5@ 004cafd4     renderer:tr_shader.obj
 0002:0000f004       ??_C@_09ELMIAJNO@?$CFs_?$CFs?4tga?$AA@ 004cb004     renderer:tr_shader.obj
 0002:0000f010       ??_C@_01JOAMLHOP@?9?$AA@   004cb010     renderer:tr_shader.obj
 0002:0000f014       ??_C@_0DG@PHBLMGGL@WARNING?3?5?8skyParms?8?5missing?5para@ 004cb014     renderer:tr_shader.obj
 0002:0000f04c       ??_C@_0L@DDGNHNOE@underwater?$AA@ 004cb04c     renderer:tr_shader.obj
 0002:0000f058       ??_C@_07NHJEPDMH@nearest?$AA@ 004cb058     renderer:tr_shader.obj
 0002:0000f060       ??_C@_08FEMHJDBF@additive?$AA@ 004cb060     renderer:tr_shader.obj
 0002:0000f06c       ??_C@_06BDPMPKBB@banner?$AA@ 004cb06c     renderer:tr_shader.obj
 0002:0000f074       ??_C@_0L@FKGCKOHC@seeThrough?$AA@ 004cb074     renderer:tr_shader.obj
 0002:0000f080       ??_C@_05CFEEDGHM@decal?$AA@ 004cb080     renderer:tr_shader.obj
 0002:0000f088       ??_C@_06CJCOLNBB@opaque?$AA@ 004cb088     renderer:tr_shader.obj
 0002:0000f090       ??_C@_0DA@IOEIMDIA@WARNING?3?5missing?5sort?5parameter?5@ 004cb090     renderer:tr_shader.obj
 0002:0000f0c0       ??_C@_0DI@PJHAFAJB@WARNING?3?5unknown?5general?5shader?5@ 004cb0c0     renderer:tr_shader.obj
 0002:0000f0f8       ??_C@_0CJ@CFIAOEJP@WARNING?3?5no?5concluding?5?8?$HN?8?5in?5sh@ 004cb0f8     renderer:tr_shader.obj
 0002:0000f124       ??_C@_04PIMMHFGE@sort?$AA@ 004cb124     renderer:tr_shader.obj
 0002:0000f12c       ??_C@_0DA@HDFMABOL@WARNING?3?5invalid?5cull?5parm?5?8?$CFs?8?5@ 004cb12c     renderer:tr_shader.obj
 0002:0000f15c       ??_C@_09LHPHMEAL@backsided?$AA@ 004cb15c     renderer:tr_shader.obj
 0002:0000f168       ??_C@_08EHJFDP@backside?$AA@ 004cb168     renderer:tr_shader.obj
 0002:0000f174       ??_C@_04JFCNHLLM@back?$AA@ 004cb174     renderer:tr_shader.obj
 0002:0000f17c       ??_C@_07DBNODEFN@disable?$AA@ 004cb17c     renderer:tr_shader.obj
 0002:0000f184       ??_C@_08INIPHAGC@twosided?$AA@ 004cb184     renderer:tr_shader.obj
 0002:0000f190       ??_C@_04CGFJFPFD@none?$AA@ 004cb190     renderer:tr_shader.obj
 0002:0000f198       ??_C@_0CM@CKHAANCG@WARNING?3?5missing?5cull?5parms?5in?5s@ 004cb198     renderer:tr_shader.obj
 0002:0000f1c4       ??_C@_04DDCLEDDO@cull?$AA@ 004cb1c4     renderer:tr_shader.obj
 0002:0000f1cc       ??_C@_05OEPGNJB@light?$AA@ 004cb1cc     renderer:tr_shader.obj
 0002:0000f1d4       ??_C@_08OPCHEDJ@skyparms?$AA@ 004cb1d4     renderer:tr_shader.obj
 0002:0000f1e0       ??_C@_0DN@BCDJHKBE@WARNING?3?5missing?5parm?5for?5?8fogPa@ 004cb1e0     renderer:tr_shader.obj
 0002:0000f220       ??_C@_08FMKCJPFI@fogParms?$AA@ 004cb220     renderer:tr_shader.obj
 0002:0000f22c       ??_C@_0P@CACIGKMN@entityMergable?$AA@ 004cb22c     renderer:tr_shader.obj
 0002:0000f23c       ??_C@_0O@DGEGEFGN@polygonOffset?$AA@ 004cb23c     renderer:tr_shader.obj
 0002:0000f24c       ??_C@_08DIOICGND@nopicmip?$AA@ 004cb24c     renderer:tr_shader.obj
 0002:0000f258       ??_C@_09LMLIDNFN@nomipmaps?$AA@ 004cb258     renderer:tr_shader.obj
 0002:0000f264       ??_C@_0M@EHMHKHGD@surfaceParm?$AA@ 004cb264     renderer:tr_shader.obj
 0002:0000f270       ??_C@_05MHKELFFB@q3map?$AA@ 004cb270     renderer:tr_shader.obj
 0002:0000f278       ??_C@_09LCMIMMJI@clampTime?$AA@ 004cb278     renderer:tr_shader.obj
 0002:0000f284       ??_C@_08MFDEDCHM@tesssize?$AA@ 004cb284     renderer:tr_shader.obj
 0002:0000f290       ??_C@_0P@FJMHOEJC@deformVertexes?$AA@ 004cb290     renderer:tr_shader.obj
 0002:0000f2a0       ??_C@_09BFMCMBDI@q3map_sun?$AA@ 004cb2a0     renderer:tr_shader.obj
 0002:0000f2ac       ??_C@_03FOCNPFKF@qer?$AA@  004cb2ac     renderer:tr_shader.obj
 0002:0000f2b0       ??_C@_0DL@HHKDKKCO@WARNING?3?5expecting?5?8?$HL?8?0?5found?5?8?$CF@ 004cb2b0     renderer:tr_shader.obj
 0002:0000f2ec       ??_C@_0DE@FPIJLKBK@WARNING?3?5GeneratePermanentShader@ 004cb2ec     renderer:tr_shader.obj
 0002:0000f320       ??_C@_0DK@CGNDAAJI@WARNING?3?5shader?5?8?$CFs?8?5has?5lightma@ 004cb320     renderer:tr_shader.obj
 0002:0000f35c       ??_C@_0CF@HBDBMHII@Shader?5?$CFs?5has?5a?5stage?5with?5no?5im@ 004cb35c     renderer:tr_shader.obj
 0002:0000f384       ??_C@_0CD@LPOFEGPO@Couldn?8t?5find?5image?5for?5shader?5?$CF@ 004cb384     renderer:tr_shader.obj
 0002:0000f3a8       ??_C@_0N@CFLHIGKB@?$CKSHADER?$CK?5?$CFs?6?$AA@ 004cb3a8     renderer:tr_shader.obj
 0002:0000f3b8       ??_C@_0BP@BKKCKGLL@Shader?5name?5exceeds?5MAX_QPATH?6?$AA@ 004cb3b8     renderer:tr_shader.obj
 0002:0000f3d8       ??_C@_0DA@NIHGGMJL@R_GetShaderByHandle?3?5out?5of?5rang@ 004cb3d8     renderer:tr_shader.obj
 0002:0000f408       ??_C@_0BC@OGEMBECL@?$CFi?5total?5shaders?6?$AA@ 004cb408     renderer:tr_shader.obj
 0002:0000f41c       ??_C@_05BBKJDEBM@?3?5?$CFs?6?$AA@ 004cb41c     renderer:tr_shader.obj
 0002:0000f424       ??_C@_0BC@HCKKJGI@?3?5?$CFs?5?$CIDEFAULTED?$CJ?6?$AA@ 004cb424     renderer:tr_shader.obj
 0002:0000f438       ??_C@_04PFOHOKJK@?5?5?5?5?$AA@ 004cb438     renderer:tr_shader.obj
 0002:0000f440       ??_C@_04PIMDLBBI@vlt?5?$AA@ 004cb440     renderer:tr_shader.obj
 0002:0000f448       ??_C@_04KHAPFJPB@lmmt?$AA@ 004cb448     renderer:tr_shader.obj
 0002:0000f450       ??_C@_04KFCMJFIC@sky?5?$AA@ 004cb450     renderer:tr_shader.obj
 0002:0000f458       ??_C@_04MJPKGGAG@gen?5?$AA@ 004cb458     renderer:tr_shader.obj
 0002:0000f460       ??_C@_02ODGLENGE@E?5?$AA@  004cb460     renderer:tr_shader.obj
 0002:0000f464       ??_C@_06GGLIPOFD@?5?5?5?5?5?5?$AA@ 004cb464     renderer:tr_shader.obj
 0002:0000f46c       ??_C@_06DHLNCDIF@MT?$CId?$CJ?5?$AA@ 004cb46c     renderer:tr_shader.obj
 0002:0000f474       ??_C@_06EKLFGMAP@MT?$CIm?$CJ?5?$AA@ 004cb474     renderer:tr_shader.obj
 0002:0000f47c       ??_C@_06GDNDLH@MT?$CIa?$CJ?5?$AA@ 004cb47c     renderer:tr_shader.obj
 0002:0000f484       ??_C@_02KNHHEEKP@?5?5?$AA@ 004cb484     renderer:tr_shader.obj
 0002:0000f488       ??_C@_02OMLKHGOL@L?5?$AA@  004cb488     renderer:tr_shader.obj
 0002:0000f48c       ??_C@_0CA@KEAFAHPN@WARNING?3?5no?5shader?5files?5found?6?$AA@ 004cb48c     renderer:tr_shader.obj
 0002:0000f4ac       ??_C@_0BB@NGOCHMHE@?4?4?4loading?5?8?$CFs?8?6?$AA@ 004cb4ac     renderer:tr_shader.obj
 0002:0000f4c0       ??_C@_0L@NIPFIBOE@scripts?1?$CFs?$AA@ 004cb4c0     renderer:tr_shader.obj
 0002:0000f4cc       ??_C@_07OMEBBDEO@scripts?$AA@ 004cb4cc     renderer:tr_shader.obj
 0002:0000f4d4       ??_C@_0BB@GHMCCJHM@?$DMstencil?5shadow?$DO?$AA@ 004cb4d4     renderer:tr_shader.obj
 0002:0000f4e8       ??_C@_09IOAPNCJN@?$DMdefault?$DO?$AA@ 004cb4e8     renderer:tr_shader.obj
 0002:0000f4f4       ??_C@_03OHFMDAD@sun?$AA@   004cb4f4     renderer:tr_shader.obj
 0002:0000f4f8       ??_C@_0M@NEGJIMEO@flareShader?$AA@ 004cb4f8     renderer:tr_shader.obj
 0002:0000f504       ??_C@_0BG@IIJFOJD@Initializing?5Shaders?6?$AA@ 004cb504     renderer:tr_shader.obj
 0002:0000f51c       ??_C@_0CN@KBGEEHMK@WARNING?3?5R_RemapShader?3?5shader?5?$CF@ 004cb51c     renderer:tr_shader.obj
 0002:0000f54c       ??_C@_0DB@FEBDLGIJ@WARNING?3?5R_RemapShader?3?5new?5shad@ 004cb54c     renderer:tr_shader.obj
 0002:0000f580       ??_C@_0CA@FJLHLOEE@?4?4?4hardware?5acceleration?5found?6?$AA@ 004cb580     renderer:win_glimp.obj
 0002:0000f5a0       ??_C@_0BL@GLEAHEND@?4?4?4MCD?5acceleration?5found?6?$AA@ 004cb5a0     renderer:win_glimp.obj
 0002:0000f5bc       ??_C@_0BN@NPGHGFAF@?4?4?4using?5software?5emulation?6?$AA@ 004cb5bc     renderer:win_glimp.obj
 0002:0000f5dc       ??_C@_0CD@MIKCGIGN@?4?4?4no?5hardware?5acceleration?5foun@ 004cb5dc     renderer:win_glimp.obj
 0002:0000f600       ??_C@_0DH@LPNFLFIF@?4?4?4PFD?5?$CFd?5rejected?0?5improper?5fla@ 004cb600     renderer:win_glimp.obj
 0002:0000f638       ??_C@_0BO@IIFIFIHJ@?4?4?4PFD?5?$CFd?5rejected?0?5not?5RGBA?6?$AA@ 004cb638     renderer:win_glimp.obj
 0002:0000f658       ??_C@_0CL@NNOBGMMI@?4?4?4PFD?5?$CFd?5rejected?0?5software?5acc@ 004cb658     renderer:win_glimp.obj
 0002:0000f684       ??_C@_0BC@PCEJAFPG@?4?4?4?$CFd?5PFDs?5found?6?$AA@ 004cb684     renderer:win_glimp.obj
 0002:0000f698       ??_C@_0CB@BNBOIMIK@?4?4?4numPFDs?5?$DO?5MAX_PFDS?5?$CI?$CFd?5?$DO?5?$CFd?$CJ?6@ 004cb698     renderer:win_glimp.obj
 0002:0000f6bc       ??_C@_0CA@MIGGKPBC@?4?4?4GLW_ChoosePFD?$CI?5?$CFd?0?5?$CFd?0?5?$CFd?5?$CJ?6?$AA@ 004cb6bc     renderer:win_glimp.obj
 0002:0000f6dc       ??_C@_0BN@HOGCJCBA@?4?4?4attempting?5to?5use?5stereo?6?$AA@ 004cb6dc     renderer:win_glimp.obj
 0002:0000f6fc       ??_C@_0BM@NECBPBKH@?4?4?4making?5context?5current?3?5?$AA@ 004cb6fc     renderer:win_glimp.obj
 0002:0000f718       ??_C@_0BJ@JOAMHKMN@?4?4?4creating?5GL?5context?3?5?$AA@ 004cb718     renderer:win_glimp.obj
 0002:0000f734       ??_C@_0BK@HLFJBFLM@?4?4?4SetPixelFormat?5failed?6?$AA@ 004cb734     renderer:win_glimp.obj
 0002:0000f750       ??_C@_0BO@GMOIKBFJ@?4?4?4qwglSetPixelFormat?5failed?6?$AA@ 004cb750     renderer:win_glimp.obj
 0002:0000f770       ??_C@_0BM@PDCKOEHH@?4?4?4PIXELFORMAT?5?$CFd?5selected?6?$AA@ 004cb770     renderer:win_glimp.obj
 0002:0000f78c       ??_C@_0BJ@NAMOHALF@?4?4?4GLW_ChoosePFD?5failed?6?$AA@ 004cb78c     renderer:win_glimp.obj
 0002:0000f7a8       ??_C@_0CJ@LGOKIJGB@?4?4?4failed?5to?5select?5stereo?5pixel@ 004cb7a8     renderer:win_glimp.obj
 0002:0000f7d4       ??_C@_0CO@OKBCOKJN@?4?4?4failed?5to?5find?5an?5appropriate@ 004cb7d4     renderer:win_glimp.obj
 0002:0000f804       ??_C@_0BA@DAJDIPF@?4?4?4failed?5hard?6?$AA@ 004cb804     renderer:win_glimp.obj
 0002:0000f814       ??_C@_0BA@NBCOEONH@?4?4?4getting?5DC?3?5?$AA@ 004cb814     renderer:win_glimp.obj
 0002:0000f824       ??_C@_0BM@FJOJLJJF@Initializing?5OpenGL?5driver?6?$AA@ 004cb824     renderer:win_glimp.obj
 0002:0000f840       ??_C@_0DD@ODIDMMC@?4?4?4window?5already?5present?0?5Creat@ 004cb840     renderer:win_glimp.obj
 0002:0000f874       ??_C@_0CB@HNOFCKCK@?4?4?4created?5window?$EA?$CFd?0?$CFd?5?$CI?$CFdx?$CFd?$CJ?6@ 004cb874     renderer:win_glimp.obj
 0002:0000f898       ??_C@_0CM@COMDHHBB@GLW_CreateWindow?$CI?$CJ?5?9?5Couldn?8t?5cr@ 004cb898     renderer:win_glimp.obj
 0002:0000f8c4       ??_C@_0BM@HPOGBHED@?4?4?4registered?5window?5class?6?$AA@ 004cb8c4     renderer:win_glimp.obj
 0002:0000f8e0       ??_C@_0DC@PEKLGHAL@GLW_CreateWindow?3?5could?5not?5regi@ 004cb8e0     renderer:win_glimp.obj
 0002:0000f914       ??_C@_0P@CMLELHDI@Quake?53?3?5Arena?$AA@ 004cb914     renderer:win_glimp.obj
 0002:0000f924       ??_C@_0BC@MOLHDJNJ@unknown?5error?5?$CFd?6?$AA@ 004cb924     renderer:win_glimp.obj
 0002:0000f938       ??_C@_0N@EAFANHAA@not?5updated?6?$AA@ 004cb938     renderer:win_glimp.obj
 0002:0000f948       ??_C@_09LGNMDMPD@bad?5mode?6?$AA@ 004cb948     renderer:win_glimp.obj
 0002:0000f954       ??_C@_0BE@MJDAFIPL@DISP_CHANGE_FAILED?6?$AA@ 004cb954     renderer:win_glimp.obj
 0002:0000f968       ??_C@_0L@GDLHKFGA@bad?5flags?6?$AA@ 004cb968     renderer:win_glimp.obj
 0002:0000f974       ??_C@_0L@MPLECDLO@bad?5param?6?$AA@ 004cb974     renderer:win_glimp.obj
 0002:0000f980       ??_C@_0BC@OMPFMAKF@restart?5required?6?$AA@ 004cb980     renderer:win_glimp.obj
 0002:0000f994       ??_C@_04CFDEAMPI@?5ok?6?$AA@ 004cb994     renderer:win_glimp.obj
 0002:0000f99c       ??_C@_09EAENAJAK@?5failed?0?5?$AA@ 004cb99c     renderer:win_glimp.obj
 0002:0000f9a8       ??_C@_0CC@JHAFIJOJ@?4?4?4trying?5next?5higher?5resolution@ 004cb9a8     renderer:win_glimp.obj
 0002:0000f9cc       ??_C@_08KJDHGAC@failed?0?5?$AA@ 004cb9cc     renderer:win_glimp.obj
 0002:0000f9d8       ??_C@_0BB@LCGMGEBN@?4?4?4calling?5CDS?3?5?$AA@ 004cb9d8     renderer:win_glimp.obj
 0002:0000f9ec       ??_C@_0BP@IICPPCNA@?4?4?4restoring?5display?5settings?6?$AA@ 004cb9ec     renderer:win_glimp.obj
 0002:0000fa0c       ??_C@_0CP@IJJINLOI@?4?4?4already?5fullscreen?0?5avoiding?5@ 004cba0c     renderer:win_glimp.obj
 0002:0000fa3c       ??_C@_0CG@CGPOLEAL@?4?4?4using?5desktop?5display?5depth?5o@ 004cba3c     renderer:win_glimp.obj
 0002:0000fa68       ??_C@_0EA@MNHMDDEA@WARNING?3?4?4?4changing?5depth?5not?5su@ 004cba68     renderer:win_glimp.obj
 0002:0000faa8       ??_C@_0BL@OCIMBLIP@?4?4?4using?5colorsbits?5of?5?$CFd?6?$AA@ 004cbaa8     renderer:win_glimp.obj
 0002:0000fac8       ??_C@_0BAN@LMLOHOBE@It?5is?5highly?5unlikely?5that?5a?5cor@ 004cbac8     renderer:win_glimp.obj
 0002:0000fbd8       ??_C@_0BI@JLHDKHCN@Low?5Desktop?5Color?5Depth?$AA@ 004cbbd8     renderer:win_glimp.obj
 0002:0000fbf0       ??_C@_0L@LHPMKOFC@?5?$CFd?5?$CFd?5?$CFs?6?$AA@ 004cbbf0     renderer:win_glimp.obj
 0002:0000fbfc       ??_C@_0P@CDOCDADM@?5invalid?5mode?6?$AA@ 004cbbfc     renderer:win_glimp.obj
 0002:0000fc0c       ??_C@_02OFDPNJAI@FS?$AA@   004cbc0c     renderer:win_glimp.obj
 0002:0000fc10       ??_C@_01ELNMCGJD@W?$AA@    004cbc10     renderer:win_glimp.obj
 0002:0000fc14       ??_C@_0BE@MPKDPDGP@?4?4?4setting?5mode?5?$CFd?3?$AA@ 004cbc14     renderer:win_glimp.obj
 0002:0000fc28       ??_C@_0CF@IOEIOODM@?4?4?4WGL_3DFX_gamma_control?5not?5fo@ 004cbc28     renderer:win_glimp.obj
 0002:0000fc50       ??_C@_0CE@PEHNJLME@?4?4?4ignoring?5WGL_3DFX_gamma_contr@ 004cbc50     renderer:win_glimp.obj
 0002:0000fc74       ??_C@_0CB@NILMOBGI@?4?4?4using?5WGL_3DFX_gamma_control?6@ 004cbc74     renderer:win_glimp.obj
 0002:0000fc98       ??_C@_0BK@KFCHIHMN@wglSetDeviceGammaRamp3DFX?$AA@ 004cbc98     renderer:win_glimp.obj
 0002:0000fcb4       ??_C@_0BK@KEAJKABC@wglGetDeviceGammaRamp3DFX?$AA@ 004cbcb4     renderer:win_glimp.obj
 0002:0000fcd0       ??_C@_0BH@FENLDGLL@WGL_3DFX_gamma_control?$AA@ 004cbcd0     renderer:win_glimp.obj
 0002:0000fce8       ??_C@_0CL@NDHIPFLH@?4?4?4GL_EXT_compiled_vertex_array?5@ 004cbce8     renderer:win_glimp.obj
 0002:0000fd14       ??_C@_0CK@OCNDKECL@?4?4?4ignoring?5GL_EXT_compiled_vert@ 004cbd14     renderer:win_glimp.obj
 0002:0000fd40       ??_C@_0BD@GEBMCHJI@bad?5getprocaddress?$AA@ 004cbd40     renderer:win_glimp.obj
 0002:0000fd54       ??_C@_0BC@CIFHOEOG@glUnlockArraysEXT?$AA@ 004cbd54     renderer:win_glimp.obj
 0002:0000fd68       ??_C@_0BA@FALFDEFM@glLockArraysEXT?$AA@ 004cbd68     renderer:win_glimp.obj
 0002:0000fd78       ??_C@_0CH@MAMJLLDH@?4?4?4using?5GL_EXT_compiled_vertex_@ 004cbd78     renderer:win_glimp.obj
 0002:0000fda0       ??_C@_0BN@LBNKGIPJ@GL_EXT_compiled_vertex_array?$AA@ 004cbda0     renderer:win_glimp.obj
 0002:0000fdc0       ??_C@_0CC@BHBHALAE@?4?4?4GL_ARB_multitexture?5not?5found@ 004cbdc0     renderer:win_glimp.obj
 0002:0000fde4       ??_C@_0CB@EPJPPON@?4?4?4ignoring?5GL_ARB_multitexture?6@ 004cbde4     renderer:win_glimp.obj
 0002:0000fe08       ??_C@_0DF@HBIOMIEF@?4?4?4not?5using?5GL_ARB_multitexture@ 004cbe08     renderer:win_glimp.obj
 0002:0000fe40       ??_C@_0BO@NHKDBIBP@?4?4?4using?5GL_ARB_multitexture?6?$AA@ 004cbe40     renderer:win_glimp.obj
 0002:0000fe60       ??_C@_0BJ@PBJNGLJH@glClientActiveTextureARB?$AA@ 004cbe60     renderer:win_glimp.obj
 0002:0000fe7c       ??_C@_0BD@IKCKKKNH@glActiveTextureARB?$AA@ 004cbe7c     renderer:win_glimp.obj
 0002:0000fe90       ??_C@_0BF@GFGCIEPA@glMultiTexCoord2fARB?$AA@ 004cbe90     renderer:win_glimp.obj
 0002:0000fea8       ??_C@_0BE@MEMOPMEA@GL_ARB_multitexture?$AA@ 004cbea8     renderer:win_glimp.obj
 0002:0000febc       ??_C@_0CD@FCNOKLOJ@?4?4?4WGL_EXT_swap_control?5not?5foun@ 004cbebc     renderer:win_glimp.obj
 0002:0000fee0       ??_C@_0BP@OPLBKLEE@?4?4?4using?5WGL_EXT_swap_control?6?$AA@ 004cbee0     renderer:win_glimp.obj
 0002:0000ff00       ??_C@_0BD@IINOPBDD@wglSwapIntervalEXT?$AA@ 004cbf00     renderer:win_glimp.obj
 0002:0000ff14       ??_C@_0CF@GHBNFILH@?4?4?4GL_EXT_texture_env_add?5not?5fo@ 004cbf14     renderer:win_glimp.obj
 0002:0000ff3c       ??_C@_0CE@CLIBMNDC@?4?4?4ignoring?5GL_EXT_texture_env_a@ 004cbf3c     renderer:win_glimp.obj
 0002:0000ff60       ??_C@_0CB@HEALHJO@?4?4?4using?5GL_EXT_texture_env_add?6@ 004cbf60     renderer:win_glimp.obj
 0002:0000ff84       ??_C@_0BE@BKNIHLLE@EXT_texture_env_add?$AA@ 004cbf84     renderer:win_glimp.obj
 0002:0000ff98       ??_C@_0BJ@PEHOEDEJ@?4?4?4GL_S3_s3tc?5not?5found?6?$AA@ 004cbf98     renderer:win_glimp.obj
 0002:0000ffb4       ??_C@_0BI@EOFEGDJG@?4?4?4ignoring?5GL_S3_s3tc?6?$AA@ 004cbfb4     renderer:win_glimp.obj
 0002:0000ffcc       ??_C@_0BF@DKAGBHJJ@?4?4?4using?5GL_S3_s3tc?6?$AA@ 004cbfcc     renderer:win_glimp.obj
 0002:0000ffe4       ??_C@_0L@LMFIOPIG@GL_S3_s3tc?$AA@ 004cbfe4     renderer:win_glimp.obj
 0002:0000fff0       ??_C@_0CA@PKLDCBMC@Initializing?5OpenGL?5extensions?6?$AA@ 004cbff0     renderer:win_glimp.obj
 0002:00010010       ??_C@_0CE@KMKFALLM@?$CK?$CK?$CK?5IGNORING?5OPENGL?5EXTENSIONS?5?$CK@ 004cc010     renderer:win_glimp.obj
 0002:00010034       ??_C@_0CM@FMNDEFGP@GLW_CheckOSVersion?$CI?$CJ?5?9?5GetVersio@ 004cc034     renderer:win_glimp.obj
 0002:00010060       ??_C@_0CK@JALFOIED@GLimp_EndFrame?$CI?$CJ?5?9?5SwapBuffers?$CI?$CJ@ 004cc060     renderer:win_glimp.obj
 0002:0001008c       ??_C@_0BG@EPMPCICE@?4?4?4resetting?5display?6?$AA@ 004cc08c     renderer:win_glimp.obj
 0002:000100a4       ??_C@_0BG@IPNGMJMJ@?4?4?4destroying?5window?6?$AA@ 004cc0a4     renderer:win_glimp.obj
 0002:000100bc       ??_C@_0BF@HIPDEIDH@?4?4?4releasing?5DC?3?5?$CFs?6?$AA@ 004cc0bc     renderer:win_glimp.obj
 0002:000100d4       ??_C@_0BM@DJONDHEF@?4?4?4deleting?5GL?5context?3?5?$CFs?6?$AA@ 004cc0d4     renderer:win_glimp.obj
 0002:000100f0       ??_C@_0CF@DDBFDAN@?4?4?4wglMakeCurrent?$CI?5NULL?0?5NULL?5?$CJ?3@ 004cc0f0     renderer:win_glimp.obj
 0002:00010118       ??_C@_0CA@JNAAMPLK@Shutting?5down?5OpenGL?5subsystem?6?$AA@ 004cc118     renderer:win_glimp.obj
 0002:00010138       ??_C@_07IPNMCAN@success?$AA@ 004cc138     renderer:win_glimp.obj
 0002:00010140       ??_C@_06ODACHPEO@failed?$AA@ 004cc140     renderer:win_glimp.obj
 0002:00010148       ??_C@_0DB@OOIIKJEH@?4?4?4WARNING?3?5fullscreen?5unavailab@ 004cc148     renderer:win_glimp.obj
 0002:0001017c       ??_C@_0CP@LOAGJHPF@?4?4?4WARNING?3?5could?5not?5set?5the?5gi@ 004cc17c     renderer:win_glimp.obj
 0002:000101ac       ??_C@_0BF@HNMFJNCH@FX_GLIDE_NO_SPLASH?$DN0?$AA@ 004cc1ac     renderer:win_glimp.obj
 0002:000101c4       ??_C@_0CJ@LKNJIDNA@?4?4?4assuming?5?8?$CFs?8?5is?5a?5standalone@ 004cc1c4     renderer:win_glimp.obj
 0002:000101f0       ??_C@_0DF@FDLDJCGG@GLW_StartOpenGL?$CI?$CJ?5?9?5could?5not?5lo@ 004cc1f0     renderer:win_glimp.obj
 0002:00010228       ??_C@_09EPIMANLC@riva?5tnt?5?$AA@ 004cc228     renderer:win_glimp.obj
 0002:00010234       ??_C@_08PNDBLPLJ@riva?5128?$AA@ 004cc234     renderer:win_glimp.obj
 0002:00010240       ??_C@_09COBMGPLJ@permedia2?$AA@ 004cc240     renderer:win_glimp.obj
 0002:0001024c       ??_C@_07MDGFFNDP@ragepro?$AA@ 004cc24c     renderer:win_glimp.obj
 0002:00010254       ??_C@_08PAOHCFPG@Rage?5Pro?$AA@ 004cc254     renderer:win_glimp.obj
 0002:00010260       ??_C@_08NCCEAIGL@rage?5pro?$AA@ 004cc260     renderer:win_glimp.obj
 0002:0001026c       ??_C@_06ONPIAGPG@glzicd?$AA@ 004cc26c     renderer:win_glimp.obj
 0002:00010274       ??_C@_07MMKJOGPH@voodoo3?$AA@ 004cc274     renderer:win_glimp.obj
 0002:0001027c       ??_C@_07BFKHNPB@banshee?$AA@ 004cc27c     renderer:win_glimp.obj
 0002:00010284       ??_C@_0O@NHGMKMHI@r_texturemode?$AA@ 004cc284     renderer:win_glimp.obj
 0002:00010294       ??_C@_0L@NHHNJFPM@s3?5savage4?$AA@ 004cc294     renderer:win_glimp.obj
 0002:000102a0       ??_C@_08IANPNEIM@savage3d?$AA@ 004cc2a0     renderer:win_glimp.obj
 0002:000102ac       ??_C@_07GFKNCEDE@rage128?$AA@ 004cc2ac     renderer:win_glimp.obj
 0002:000102b4       ??_C@_08HEOMHBGA@rage?5128?$AA@ 004cc2b4     renderer:win_glimp.obj
 0002:000102c0       ??_C@_0BL@NGHEFHNP@voodoo?5graphics?11?5tmu?12?5mb?$AA@ 004cc2c0     renderer:win_glimp.obj
 0002:000102dc       ??_C@_0BB@OKGMNIFP@r_maskMinidriver?$AA@ 004cc2dc     renderer:win_glimp.obj
 0002:000102f0       ??_C@_0BC@BNBBBHDE@r_allowSoftwareGL?$AA@ 004cc2f0     renderer:win_glimp.obj
 0002:00010304       ??_C@_0CL@HLGCEFDK@GLimp_Init?$CI?$CJ?5?9?5incorrect?5operati@ 004cc304     renderer:win_glimp.obj
 0002:00010330       ??_C@_0BP@CDHFKDJO@Initializing?5OpenGL?5subsystem?6?$AA@ 004cc330     renderer:win_glimp.obj
 0002:00010350       ??_C@_0BE@NPAMJJ@r_lastValidRenderer?$AA@ 004cc350     renderer:win_glimp.obj
 0002:00010364       ??_C@_0BA@KCKFOAHI@?$CIuninitialized?$CJ?$AA@ 004cc364     renderer:win_glimp.obj
 0002:00010374       ??_C@_0CO@EOJAGHCM@RE_RegisterFont?3?5FreeType?5code?5n@ 004cc374     renderer:tr_font.obj
 0002:000103a4       ??_C@_0BH@EJJGLAMJ@fonts?1fontImage_?$CFi?4dat?$AA@ 004cc3a4     renderer:tr_font.obj
 0002:000103bc       ??_C@_0DF@KGACFLBL@RE_RegisterFont?3?5Too?5many?5fonts?5@ 004cc3bc     renderer:tr_font.obj
 0002:000103f4       ??_C@_0BJ@ONIEGCNG@R_PointInLeaf?3?5bad?5model?$AA@ 004cc3f4     renderer:tr_world.obj
 0002:00010410       ??_C@_0BF@BAHPENBA@cluster?3?$CFi?5?5area?3?$CFi?6?$AA@ 004cc410     renderer:tr_world.obj
 0002:00010428       __real@40a00000            004cc428     renderer:tr_bsp.obj
 0002:0001042c       ??_C@_0BO@HMCELCP@Brightest?5lightmap?5value?3?5?$CFd?6?$AA@ 004cc42c     renderer:tr_bsp.obj
 0002:0001044c       ??_C@_0M@GGCLEKFK@?$CKlightmap?$CFd?$AA@ 004cc44c     renderer:tr_bsp.obj
 0002:00010458       __real@3f2f5c29            004cc458     renderer:tr_bsp.obj
 0002:0001045c       __real@3d810625            004cc45c     renderer:tr_bsp.obj
 0002:00010460       __real@3ea8f5c3            004cc460     renderer:tr_bsp.obj
 0002:00010464       ??_C@_0BP@JJDMICKK@ShaderForShaderNum?3?5bad?5num?5?$CFi?$AA@ 004cc464     renderer:tr_bsp.obj
 0002:00010484       ??_C@_0CH@FEFMAIEG@WARNING?3?5MAX_FACE_POINTS?5exceede@ 004cc484     renderer:tr_bsp.obj
 0002:000104ac       ??_C@_0BO@KFEJELLI@Bad?5index?5in?5triangle?5surface?$AA@ 004cc4ac     renderer:tr_bsp.obj
 0002:000104cc       ??_C@_0BI@IDNDEPDA@stitched?5?$CFd?5LoD?5cracks?6?$AA@ 004cc4cc     renderer:tr_bsp.obj
 0002:000104e4       ??_C@_0DH@BPCGGBHH@?4?4?4loaded?5?$CFd?5faces?0?5?$CFi?5meshes?0?5?$CF@ 004cc4e4     renderer:tr_bsp.obj
 0002:0001051c       ??_C@_0BA@PMNKLNK@Bad?5surfaceType?$AA@ 004cc51c     renderer:tr_bsp.obj
 0002:0001052c       ??_C@_0BP@LNMBABNB@LoadMap?3?5funny?5lump?5size?5in?5?$CFs?$AA@ 004cc52c     renderer:tr_bsp.obj
 0002:0001054c       ??_C@_03COCDEFBB@?$CK?$CFd?$AA@ 004cc54c     renderer:tr_bsp.obj
 0002:00010550       ??_C@_0CC@KODOEMIA@fog?5brush?5sideNumber?5out?5of?5rang@ 004cc550     renderer:tr_bsp.obj
 0002:00010574       ??_C@_0BN@GDFIOGDD@fog?5brushNumber?5out?5of?5range?$AA@ 004cc574     renderer:tr_bsp.obj
 0002:00010594       ??_C@_0BO@IHAFNPEE@WARNING?3?5light?5grid?5mismatch?6?$AA@ 004cc594     renderer:tr_bsp.obj
 0002:000105b4       ??_C@_0CM@EJOCAFMB@WARNING?3?5no?5semi?5colon?5in?5shader@ 004cc5b4     renderer:tr_bsp.obj
 0002:000105e0       ??_C@_0DC@JPJBKBBA@WARNING?3?5no?5semi?5colon?5in?5vertex@ 004cc5e0     renderer:tr_bsp.obj
 0002:00010614       ??_C@_08OEKJENGB@?$CFf?5?$CFf?5?$CFf?$AA@ 004cc614     renderer:tr_bsp.obj
 0002:00010620       ??_C@_08PLHKIFFJ@gridsize?$AA@ 004cc620     renderer:tr_bsp.obj
 0002:0001062c       ??_C@_0M@NEKNPMKB@remapshader?$AA@ 004cc62c     renderer:tr_bsp.obj
 0002:00010638       ??_C@_0BC@LEFDABNE@vertexremapshader?$AA@ 004cc638     renderer:tr_bsp.obj
 0002:0001064c       ??_C@_0DP@JCKGEGMK@RE_LoadWorldMap?3?5?$CFs?5has?5wrong?5ve@ 004cc64c     renderer:tr_bsp.obj
 0002:0001068c       ??_C@_0BO@FKKONKDO@RE_LoadWorldMap?3?5?$CFs?5not?5found?$AA@ 004cc68c     renderer:tr_bsp.obj
 0002:000106ac       ??_C@_0DA@HFMADLDH@ERROR?3?5attempted?5to?5redundantly?5@ 004cc6ac     renderer:tr_bsp.obj
 0002:000106e0       ??_C@_0EE@FBLEADKI@WARNING?3?5RE_AddPolyToScene?3?5r_ma@ 004cc6e0     renderer:tr_scene.obj
 0002:00010724       ??_C@_0CO@ICFMIPOA@WARNING?3?5RE_AddPolyToScene?3?5NULL@ 004cc724     renderer:tr_scene.obj
 0002:00010754       ??_C@_0CG@DEMNJENN@RE_AddRefEntityToScene?3?5bad?5reTy@ 004cc754     renderer:tr_scene.obj
 0002:0001077c       ??_C@_0BP@KOPNJDAJ@R_RenderScene?3?5NULL?5worldmodel?$AA@ 004cc77c     renderer:tr_scene.obj
 0002:0001079c       ??_C@_0BN@KPIPFFIJ@?$DN?$DN?$DN?$DN?$DN?$DN?5RE_RenderScene?5?$DN?$DN?$DN?$DN?$DN?6?$AA@ 004cc79c     renderer:tr_scene.obj
 0002:000107bc       ??_C@_0BA@MBJODGEL@amb?3?$CFi?5?5dir?3?$CFi?6?$AA@ 004cc7bc     renderer:tr_light.obj
 0002:000107cc       __real@43160000            004cc7cc     renderer:tr_light.obj
 0002:000107d0       __real@bfe0000000000000    004cc7d0     renderer:tr_marks.obj
 0002:000107d8       __real@bfa999999999999a    004cc7d8     renderer:tr_marks.obj
 0002:000107e0       __real@41a00000            004cc7e0     renderer:tr_marks.obj
 0002:000107e4       __real@3bff01fe            004cc7e4     renderer:tr_noise.obj
 0002:000107e8       ??_C@_0BD@LDKOPICD@glUnlockArraysEXT?6?$AA@ 004cc7e8     renderer:tr_shade.obj
 0002:000107fc       ??_C@_0BB@JIGCEAGB@glLockArraysEXT?6?$AA@ 004cc7fc     renderer:tr_shade.obj
 0002:00010810       ??_C@_0CL@KIMCIKPC@ERROR?3?5unknown?5texmod?5?8?$CFd?8?5in?5sh@ 004cc810     renderer:tr_shade.obj
 0002:0001083c       ??_C@_0CH@KLPBLGIL@?9?9?9?5RB_StageIteratorGeneric?$CI?5?$CFs?5@ 004cc83c     renderer:tr_shade.obj
 0002:00010864       ??_C@_0DJ@BJEEMKDD@?9?9?9?5RB_StageIteratorVertexLitTex@ 004cc864     renderer:tr_shade.obj
 0002:000108a0       ??_C@_0DH@IFGPEEH@?9?9?9?5RB_StageIteratorLightmappedM@ 004cc8a0     renderer:tr_shade.obj
 0002:000108d8       ??_C@_0M@FAPJFEJO@?9?9?9?9?9?9?9?9?9?9?6?$AA@ 004cc8d8     renderer:tr_shade.obj
 0002:000108e4       ??_C@_0CK@MBNGEIEM@RB_EndSurface?$CI?$CJ?5?9?5SHADER_MAX_VER@ 004cc8e4     renderer:tr_shade.obj
 0002:00010910       ??_C@_0CJ@GNPNENL@RB_EndSurface?$CI?$CJ?5?9?5SHADER_MAX_IND@ 004cc910     renderer:tr_shade.obj
 0002:0001093c       ??_C@_0CJ@IAOLBLPF@WARNING?3?5shader?5?$CFs?5in?5skin?5?$CFs?5no@ 004cc93c     renderer:tr_mesh.obj
 0002:00010968       ??_C@_0CO@IEHCNJOK@WARNING?3?5no?5shader?5for?5surface?5?$CF@ 004cc968     renderer:tr_mesh.obj
 0002:00010998       ??_C@_0DD@DEGFOKKF@R_AddMD3Surfaces?3?5no?5such?5frame?5@ 004cc998     renderer:tr_mesh.obj
 0002:000109cc       ??_C@_0CK@PCOMEKCP@RB_CheckOverflow?3?5indices?5?$DO?5MAX?5@ 004cc9cc     renderer:tr_surface.obj
 0002:000109f8       ??_C@_0CI@FEFGMFPL@RB_CheckOverflow?3?5verts?5?$DO?5MAX?5?$CI?$CF@ 004cc9f8     renderer:tr_surface.obj
 0002:00010a20       __real@404e000000000000    004cca20     renderer:tr_surface.obj
 0002:00010a28       __real@3f90000000000000    004cca28     renderer:tr_surface.obj
 0002:00010a30       ??_C@_0BJ@FAJDOIKM@Bad?5surface?5tesselated?4?6?$AA@ 004cca30     renderer:tr_surface.obj
 0002:00010a50       _jpeg_std_message_table    004cca50     renderer:jerror.obj
 0002:00010c2c       ??_C@_0CL@OCGBAKPF@Application?5transferred?5too?5many@ 004ccc2c     renderer:jerror.obj
 0002:00010c58       ??_C@_0CL@BAKCGOKJ@Invalid?5SOS?5parameters?5for?5seque@ 004ccc58     renderer:jerror.obj
 0002:00010c84       ??_C@_0DI@NFMBADOH@Corrupt?5JPEG?5data?3?5found?5marker?5@ 004ccc84     renderer:jerror.obj
 0002:00010cbc       ??_C@_0BL@DPFPFMLM@Premature?5end?5of?5JPEG?5file?$AA@ 004cccbc     renderer:jerror.obj
 0002:00010cd8       ??_C@_0CO@ODCCEDLN@Warning?3?5unknown?5JFIF?5revision?5n@ 004cccd8     renderer:jerror.obj
 0002:00010d08       ??_C@_0CE@PBLDOPKB@Corrupt?5JPEG?5data?3?5bad?5Huffman?5c@ 004ccd08     renderer:jerror.obj
 0002:00010d2c       ??_C@_0DB@PGMEPGHN@Corrupt?5JPEG?5data?3?5premature?5end@ 004ccd2c     renderer:jerror.obj
 0002:00010d60       ??_C@_0DM@PCOGCKJB@Corrupt?5JPEG?5data?3?5?$CFu?5extraneous@ 004ccd60     renderer:jerror.obj
 0002:00010da0       ??_C@_0EC@CBCJOINE@Inconsistent?5progression?5sequenc@ 004ccda0     renderer:jerror.obj
 0002:00010de4       ??_C@_0CG@KEGHCDOM@Unknown?5Adobe?5color?5transform?5co@ 004ccde4     renderer:jerror.obj
 0002:00010e0c       ??_C@_0BH@LJLGPEFF@Obtained?5XMS?5handle?5?$CFu?$AA@ 004cce0c     renderer:jerror.obj
 0002:00010e24       ??_C@_0BE@FOGGKKAO@Freed?5XMS?5handle?5?$CFu?$AA@ 004cce24     renderer:jerror.obj
 0002:00010e38       ??_C@_0DE@EEJCDLOO@Unrecognized?5component?5IDs?5?$CFd?5?$CFd@ 004cce38     renderer:jerror.obj
 0002:00010e6c       ??_C@_0BJ@GOCABEP@Opened?5temporary?5file?5?$CFs?$AA@ 004cce6c     renderer:jerror.obj
 0002:00010e88       ??_C@_0BJ@KDCGAOJB@Closed?5temporary?5file?5?$CFs?$AA@ 004cce88     renderer:jerror.obj
 0002:00010ea4       ??_C@_0BN@GAMIJLDC@?5?5Ss?$DN?$CFd?0?5Se?$DN?$CFd?0?5Ah?$DN?$CFd?0?5Al?$DN?$CFd?$AA@ 004ccea4     renderer:jerror.obj
 0002:00010ec4       ??_C@_0BO@CDEKFGLC@?5?5?5?5Component?5?$CFd?3?5dc?$DN?$CFd?5ac?$DN?$CFd?$AA@ 004ccec4     renderer:jerror.obj
 0002:00010ee4       ??_C@_0BN@BLOOHNC@Start?5Of?5Scan?3?5?$CFd?5components?$AA@ 004ccee4     renderer:jerror.obj
 0002:00010f04       ??_C@_0P@JLCHJELA@Start?5of?5Image?$AA@ 004ccf04     renderer:jerror.obj
 0002:00010f14       ??_C@_0BP@EDCAMHHE@?5?5?5?5Component?5?$CFd?3?5?$CFdhx?$CFdv?5q?$DN?$CFd?$AA@ 004ccf14     renderer:jerror.obj
 0002:00010f34       ??_C@_0DK@DMINKOGN@Start?5Of?5Frame?50x?$CF02x?3?5width?$DN?$CFu?0@ 004ccf34     renderer:jerror.obj
 0002:00010f70       ??_C@_0DJ@PCBCLFML@Smoothing?5not?5supported?5with?5non@ 004ccf70     renderer:jerror.obj
 0002:00010fac       ??_C@_05LLAPAOG@RST?$CFd?$AA@ 004ccfac     renderer:jerror.obj
 0002:00010fb4       ??_C@_0CF@NIMOLBCP@At?5marker?50x?$CF02x?0?5recovery?5actio@ 004ccfb4     renderer:jerror.obj
 0002:00010fdc       ??_C@_0CE@FDPBEAOO@Selected?5?$CFd?5colors?5for?5quantizat@ 004ccfdc     renderer:jerror.obj
 0002:00011000       ??_C@_0BI@NEIBNACE@Quantizing?5to?5?$CFd?5colors?$AA@ 004cd000     renderer:jerror.obj
 0002:00011018       ??_C@_0CD@CNNAOOFA@Quantizing?5to?5?$CFd?5?$DN?5?$CFd?$CK?$CFd?$CK?$CFd?5colo@ 004cd018     renderer:jerror.obj
 0002:0001103c       ??_C@_0CI@GHPOCOCL@?5?5?5?5?5?5?5?5?$CF4u?5?$CF4u?5?$CF4u?5?$CF4u?5?$CF4u?5?$CF4u?5@ 004cd03c     renderer:jerror.obj
 0002:00011064       ??_C@_0BJ@COPODLDN@Unexpected?5marker?50x?$CF02x?$AA@ 004cd064     renderer:jerror.obj
 0002:00011080       ??_C@_0CC@KHCAAFMC@Skipping?5marker?50x?$CF02x?0?5length?5?$CF@ 004cd080     renderer:jerror.obj
 0002:000110a4       ??_C@_0CB@BADBMAAB@?5?5?5?5with?5?$CFd?5x?5?$CFd?5thumbnail?5image@ 004cd0a4     renderer:jerror.obj
 0002:000110c8       ??_C@_0CL@BJMGIDLN@Unknown?5JFIF?5minor?5revision?5numb@ 004cd0c8     renderer:jerror.obj
 0002:000110f4       ??_C@_0DM@JLHNPIBE@Warning?3?5thumbnail?5image?5size?5do@ 004cd0f4     renderer:jerror.obj
 0002:00011130       ??_C@_0CE@MKDBBMLI@JFIF?5APP0?5marker?0?5density?5?$CFdx?$CFd?5@ 004cd130     renderer:jerror.obj
 0002:00011154       ??_C@_0CI@FKGPAJC@?5?5?5?5?5?5?5?5?$CF3d?5?$CF3d?5?$CF3d?5?$CF3d?5?$CF3d?5?$CF3d?5@ 004cd154     renderer:jerror.obj
 0002:0001117c       ??_C@_0N@HJHFKELG@End?5Of?5Image?$AA@ 004cd17c     renderer:jerror.obj
 0002:0001118c       ??_C@_0BH@GIPOLIGC@Obtained?5EMS?5handle?5?$CFu?$AA@ 004cd18c     renderer:jerror.obj
 0002:000111a4       ??_C@_0BE@IPCOOGDJ@Freed?5EMS?5handle?5?$CFu?$AA@ 004cd1a4     renderer:jerror.obj
 0002:000111b8       ??_C@_0BL@EMFIKBEK@Define?5Restart?5Interval?5?$CFu?$AA@ 004cd1b8     renderer:jerror.obj
 0002:000111d4       ??_C@_0CL@KLDOJIKN@Define?5Quantization?5Table?5?$CFd?5?5pr@ 004cd1d4     renderer:jerror.obj
 0002:00011200       ??_C@_0BM@MDIEILCE@Define?5Huffman?5Table?50x?$CF02x?$AA@ 004cd200     renderer:jerror.obj
 0002:0001121c       ??_C@_0CH@KIJGKPAA@Define?5Arithmetic?5Table?50x?$CF02x?3?5@ 004cd21c     renderer:jerror.obj
 0002:00011244       ??_C@_0CM@CAEPHFAA@Unknown?5APP14?5marker?5?$CInot?5Adobe?$CJ@ 004cd244     renderer:jerror.obj
 0002:00011270       ??_C@_0CK@HCPFFNKJ@Unknown?5APP0?5marker?5?$CInot?5JFIF?$CJ?0?5@ 004cd270     renderer:jerror.obj
 0002:000112a0       ??_C@_0EC@EHPKAOHA@Adobe?5APP14?5marker?3?5version?5?$CFd?0?5@ 004cd2a0     renderer:jerror.obj
 0002:000112e4       ??_C@_0DO@EGLODMBB@Caution?3?5quantization?5tables?5are@ 004cd2e4     renderer:jerror.obj
 0002:00011324       ??_C@_0M@JNBJJLAI@6?5?52?9Aug?995?$AA@ 004cd324     renderer:jerror.obj
 0002:00011330       ??_C@_0CD@HPLBEMMI@Copyright?5?$CIC?$CJ?51995?0?5Thomas?5G?4?5La@ 004cd330     renderer:jerror.obj
 0002:00011354       ??_C@_0BE@FDPDCBIN@Write?5to?5XMS?5failed?$AA@ 004cd354     renderer:jerror.obj
 0002:00011368       ??_C@_0BF@EKLGFGNM@Read?5from?5XMS?5failed?$AA@ 004cd368     renderer:jerror.obj
 0002:00011380       ??_C@_0CH@LJLHCCHC@Image?5too?5wide?5for?5this?5implemen@ 004cd380     renderer:jerror.obj
 0002:000113a8       ??_C@_0CD@GCLFJCHC@Virtual?5array?5controller?5messed?5@ 004cd3a8     renderer:jerror.obj
 0002:000113cc       ??_C@_0BP@BPKOBOIP@Unsupported?5marker?5type?50x?$CF02x?$AA@ 004cd3cc     renderer:jerror.obj
 0002:000113ec       ??_C@_0CK@EPADOAKC@Application?5transferred?5too?5few?5@ 004cd3ec     renderer:jerror.obj
 0002:00011418       ??_C@_0DG@KALDLIJB@Write?5failed?5on?5temporary?5file?5?9@ 004cd418     renderer:jerror.obj
 0002:00011450       ??_C@_0BO@GOBJOAAI@Seek?5failed?5on?5temporary?5file?$AA@ 004cd450     renderer:jerror.obj
 0002:00011470       ??_C@_0BO@EEPJGHHI@Read?5failed?5on?5temporary?5file?$AA@ 004cd470     renderer:jerror.obj
 0002:00011490       ??_C@_0CD@POKNOPOF@Failed?5to?5create?5temporary?5file?5@ 004cd490     renderer:jerror.obj
 0002:000114b4       ??_C@_0CM@HONLBDPH@Invalid?5JPEG?5file?5structure?3?5SOS@ 004cd4b4     renderer:jerror.obj
 0002:000114e0       ??_C@_0CN@HGJCMLNE@Invalid?5JPEG?5file?5structure?3?5two@ 004cd4e0     renderer:jerror.obj
 0002:00011510       ??_C@_0CK@HMKECJK@Unsupported?5JPEG?5process?3?5SOF?5ty@ 004cd510     renderer:jerror.obj
 0002:0001153c       ??_C@_0DA@GJIJGINK@Invalid?5JPEG?5file?5structure?3?5mis@ 004cd53c     renderer:jerror.obj
 0002:0001156c       ??_C@_0CN@IHJJJAFJ@Invalid?5JPEG?5file?5structure?3?5two@ 004cd56c     renderer:jerror.obj
 0002:0001159c       ??_C@_0CH@NHMNHHIB@Cannot?5quantize?5to?5more?5than?5?$CFd?5@ 004cd59c     renderer:jerror.obj
 0002:000115c4       ??_C@_0CI@PLMPLCNO@Cannot?5quantize?5to?5fewer?5than?5?$CFd@ 004cd5c4     renderer:jerror.obj
 0002:000115ec       ??_C@_0CO@HPDBAEEA@Cannot?5quantize?5more?5than?5?$CFd?5col@ 004cd5ec     renderer:jerror.obj
 0002:0001161c       ??_C@_0BO@DJPLELIB@Insufficient?5memory?5?$CIcase?5?$CFd?$CJ?$AA@ 004cd61c     renderer:jerror.obj
 0002:0001163c       ??_C@_0CL@GNLFDFCL@Not?5a?5JPEG?5file?3?5starts?5with?50x?$CF@ 004cd63c     renderer:jerror.obj
 0002:00011668       ??_C@_0CK@CCHKIENB@Quantization?5table?50x?$CF02x?5was?5no@ 004cd668     renderer:jerror.obj
 0002:00011694       ??_C@_0CC@BKPLBDLJ@JPEG?5datastream?5contains?5no?5imag@ 004cd694     renderer:jerror.obj
 0002:000116b8       ??_C@_0CF@BKANFCCL@Huffman?5table?50x?$CF02x?5was?5not?5def@ 004cd6b8     renderer:jerror.obj
 0002:000116e0       ??_C@_0BM@HJHFKLAF@Backing?5store?5not?5supported?$AA@ 004cd6e0     renderer:jerror.obj
 0002:000116fc       ??_C@_0CO@BEHINNOI@Requested?5feature?5was?5omitted?5at@ 004cd6fc     renderer:jerror.obj
 0002:0001172c       ??_C@_0BE@EOAAHHJ@Not?5implemented?5yet?$AA@ 004cd72c     renderer:jerror.obj
 0002:00011740       ??_C@_0CH@EFBBPPCK@Invalid?5color?5quantization?5mode?5@ 004cd740     renderer:jerror.obj
 0002:00011768       ??_C@_0CH@NIBDNILP@Scan?5script?5does?5not?5transmit?5al@ 004cd768     renderer:jerror.obj
 0002:00011790       ??_C@_0DO@OPNPKGO@Cannot?5transcode?5due?5to?5multiple@ 004cd790     renderer:jerror.obj
 0002:000117d0       ??_C@_0BM@KEKMMNGA@Premature?5end?5of?5input?5file?$AA@ 004cd7d0     renderer:jerror.obj
 0002:000117ec       ??_C@_0BB@JJAIKFBB@Empty?5input?5file?$AA@ 004cd7ec     renderer:jerror.obj
 0002:00011800       ??_C@_0CP@EKFPGPNP@Maximum?5supported?5image?5dimensio@ 004cd800     renderer:jerror.obj
 0002:00011830       ??_C@_0CB@LFBMFPHI@Missing?5Huffman?5code?5table?5entry@ 004cd830     renderer:jerror.obj
 0002:00011854       ??_C@_0CB@LLDOGNPJ@Huffman?5code?5size?5table?5overflow@ 004cd854     renderer:jerror.obj
 0002:00011878       ??_C@_0CI@EKDDDHFF@Fractional?5sampling?5not?5implemen@ 004cd878     renderer:jerror.obj
 0002:000118a0       ??_C@_0CP@IDOBLGGD@Output?5file?5write?5error?5?9?9?9?5out?5@ 004cd8a0     renderer:jerror.obj
 0002:000118d0       ??_C@_0BG@BALCKDNL@Input?5file?5read?5error?$AA@ 004cd8d0     renderer:jerror.obj
 0002:000118e8       ??_C@_0CB@DMGINPNE@Didn?8t?5expect?5more?5than?5one?5scan@ 004cd8e8     renderer:jerror.obj
 0002:0001190c       ??_C@_0BE@DGJBKIEB@Write?5to?5EMS?5failed?$AA@ 004cd90c     renderer:jerror.obj
 0002:00011920       ??_C@_0BF@CPNENPBA@Read?5from?5EMS?5failed?$AA@ 004cd920     renderer:jerror.obj
 0002:00011938       ??_C@_0CF@DAGGEAPM@Empty?5JPEG?5image?5?$CIDNL?5not?5suppor@ 004cd938     renderer:jerror.obj
 0002:00011960       ??_C@_0BD@DIMECAOP@Bogus?5DQT?5index?5?$CFd?$AA@ 004cd960     renderer:jerror.obj
 0002:00011974       ??_C@_0BD@KJHFPHIC@Bogus?5DHT?5index?5?$CFd?$AA@ 004cd974     renderer:jerror.obj
 0002:00011988       ??_C@_0BB@GDNEPMHL@Bogus?5DHT?5counts?$AA@ 004cd988     renderer:jerror.obj
 0002:0001199c       ??_C@_0BF@CLIOOJFM@Bogus?5DAC?5value?50x?$CFx?$AA@ 004cd99c     renderer:jerror.obj
 0002:000119b4       ??_C@_0BD@LDBBBMFL@Bogus?5DAC?5index?5?$CFd?$AA@ 004cd9b4     renderer:jerror.obj
 0002:000119c8       ??_C@_0CF@JDLOPNGO@Unsupported?5color?5conversion?5req@ 004cd9c8     renderer:jerror.obj
 0002:000119f0       ??_C@_0CG@BEBDNOCG@Too?5many?5color?5components?3?5?$CFd?0?5m@ 004cd9f0     renderer:jerror.obj
 0002:00011a18       ??_C@_0CF@LAEFHNAH@CCIR601?5sampling?5not?5implemented@ 004cda18     renderer:jerror.obj
 0002:00011a40       ??_C@_0BM@PKHCPJDH@Suspension?5not?5allowed?5here?$AA@ 004cda40     renderer:jerror.obj
 0002:00011a5c       ??_C@_0CL@JKHIPJLJ@Buffer?5passed?5to?5JPEG?5library?5is@ 004cda5c     renderer:jerror.obj
 0002:00011a88       ??_C@_0BL@CBOEEPLK@Bogus?5virtual?5array?5access?$AA@ 004cda88     renderer:jerror.obj
 0002:00011aa4       ??_C@_0CK@BAMFIBMM@Improper?5call?5to?5JPEG?5library?5in@ 004cdaa4     renderer:jerror.obj
 0002:00011ad0       ??_C@_0CA@MJDDICLK@Invalid?5scan?5script?5at?5entry?5?$CFd?$AA@ 004cdad0     renderer:jerror.obj
 0002:00011af0       ??_C@_0BH@HMMHPOPE@Bogus?5sampling?5factors?$AA@ 004cdaf0     renderer:jerror.obj
 0002:00011b08       ??_C@_0DH@HIKEGPKP@Invalid?5progressive?5parameters?5a@ 004cdb08     renderer:jerror.obj
 0002:00011b40       ??_C@_0DH@LNGGEGOL@Invalid?5progressive?5parameters?5S@ 004cdb40     renderer:jerror.obj
 0002:00011b78       ??_C@_0CD@LDBDNLHK@Unsupported?5JPEG?5data?5precision?5@ 004cdb78     renderer:jerror.obj
 0002:00011b9c       ??_C@_0BM@OEMICEFD@Invalid?5memory?5pool?5code?5?$CFd?$AA@ 004cdb9c     renderer:jerror.obj
 0002:00011bb8       ??_C@_0DA@HLEOHNPA@Sampling?5factors?5too?5large?5for?5i@ 004cdbb8     renderer:jerror.obj
 0002:00011be8       ??_C@_0BE@OGLAEMOG@Bogus?5marker?5length?$AA@ 004cdbe8     renderer:jerror.obj
 0002:00011bfc       ??_C@_0BG@NEGIHEMC@Bogus?5JPEG?5colorspace?$AA@ 004cdbfc     renderer:jerror.obj
 0002:00011c14       ??_C@_0BH@BGDIGLHC@Bogus?5input?5colorspace?$AA@ 004cdc14     renderer:jerror.obj
 0002:00011c2c       ??_C@_0CI@MBJANLAP@IDCT?5output?5block?5size?5?$CFd?5not?5su@ 004cdc2c     renderer:jerror.obj
 0002:00011c54       ??_C@_0BP@ONFLCDHG@Invalid?5component?5ID?5?$CFd?5in?5SOS?$AA@ 004cdc54     renderer:jerror.obj
 0002:00011c74       ??_C@_0BK@DKALDNKG@Bogus?5buffer?5control?5mode?$AA@ 004cdc74     renderer:jerror.obj
 0002:00011c90       ??_C@_0CF@DENLILGA@MAX_ALLOC_CHUNK?5is?5wrong?0?5please@ 004cdc90     renderer:jerror.obj
 0002:00011cb8       ??_C@_0CA@FDMPGPNI@ALIGN_TYPE?5is?5wrong?0?5please?5fix?$AA@ 004cdcb8     renderer:jerror.obj
 0002:00011cd8       ??_C@_0DJ@KONAFFHE@Sorry?0?5there?5are?5legal?5restricti@ 004cdcd8     renderer:jerror.obj
 0002:00011d14       ??_C@_0BG@MIBALFBH@Bogus?5message?5code?5?$CFd?$AA@ 004cdd14     renderer:jerror.obj
 0002:000120e8       ??_C@_0EF@OOLKDLBP@WARNING?3?5suspicious?5gamma?5tables@ 004ce0e8     renderer:win_gamma.obj
 0002:00012130       ??_C@_0DP@KHIKMCPB@WARNING?3?5device?5has?5broken?5gamma@ 004ce130     renderer:win_gamma.obj
 0002:00012170       ??_C@_0BM@HCCAHBCJ@SetDeviceGammaRamp?5failed?4?6?$AA@ 004ce170     renderer:win_gamma.obj
 0002:0001218c       ??_C@_0BL@LBLAAGEL@skipping?5W2K?5gamma?5clamp?4?6?$AA@ 004ce18c     renderer:win_gamma.obj
 0002:000121a8       ??_C@_0BN@EINPLPO@performing?5W2K?5gamma?5clamp?4?6?$AA@ 004ce1a8     renderer:win_gamma.obj
 0002:000121c8       __real@41c00000            004ce1c8     renderer:tr_flares.obj
 0002:000121cc       __real@3acccccd            004ce1cc     renderer:tr_flares.obj
 0002:000121d0       __real@c0f869f000000000    004ce1d0     renderer:tr_flares.obj
 0002:000121d8       __real@40f869f000000000    004ce1d8     renderer:tr_flares.obj
 0002:000121e0       __real@44000000            004ce1e0     renderer:tr_shadows.obj
 0002:000121e4       ??_C@_0BP@OIODLEAK@ClipSkyPolygon?3?5MAX_CLIP_VERTS?$AA@ 004ce1e4     renderer:tr_sky.obj
 0002:00012208       __real@3fe2492492492492    004ce208     renderer:tr_sky.obj
 0002:00012210       ??_C@_0DA@DJLPNMLL@SHADER_MAX_VERTEXES?5hit?5in?5FillC@ 004ce210     renderer:tr_sky.obj
 0002:00012240       __real@c0800000            004ce240     renderer:tr_sky.obj
 0002:00012244       __real@45800000            004ce244     renderer:tr_sky.obj
 0002:00012248       __real@46000000            004ce248     renderer:tr_sky.obj
 0002:0001224c       __real@4b800000            004ce24c     renderer:tr_sky.obj
 0002:00012250       __real@3fd999999999999a    004ce250     renderer:tr_sky.obj
 0002:00012258       ??_C@_0DP@KCJNMMFJ@TableForFunc?5called?5with?5invalid@ 004ce258     renderer:tr_shade_calc.obj
 0002:00012298       __real@43480000            004ce298     renderer:tr_shade_calc.obj
 0002:0001229c       __real@3f7ae148            004ce29c     renderer:tr_shade_calc.obj
 0002:000122a0       __real@4322f983            004ce2a0     renderer:tr_shade_calc.obj
 0002:000122a4       __real@bf400000            004ce2a4     renderer:tr_shade_calc.obj
 0002:000122a8       __real@497423f0            004ce2a8     renderer:tr_shade_calc.obj
 0002:000122ac       __real@c97423f0            004ce2ac     renderer:tr_shade_calc.obj
 0002:000122b0       __real@3f34fdf4            004ce2b0     renderer:tr_shade_calc.obj
 0002:000122b4       ??_C@_0CJ@LIFBHBKN@Autosprite?5shader?5?$CFs?5had?5odd?5ind@ 004ce2b4     renderer:tr_shade_calc.obj
 0002:000122e0       ??_C@_0CK@OKNCJKLI@Autosprite?5shader?5?$CFs?5had?5odd?5ver@ 004ce2e0     renderer:tr_shade_calc.obj
 0002:0001230c       ??_C@_0CK@NPHOOAGM@Autosprite2?5shader?5?$CFs?5had?5odd?5in@ 004ce30c     renderer:tr_shade_calc.obj
 0002:00012338       ??_C@_0CL@GNGEHAP@Autosprite2?5shader?5?$CFs?5had?5odd?5ve@ 004ce338     renderer:tr_shade_calc.obj
 0002:00012364       __real@3f780000            004ce364     renderer:tr_shade_calc.obj
 0002:00012368       __real@3fee000000000000    004ce368     renderer:tr_shade_calc.obj
 0002:00012370       __real@4090000000000000    004ce370     renderer:tr_shade_calc.obj
 0002:00012378       __real@3f50000000000000    004ce378     renderer:tr_shade_calc.obj
 0002:00012380       __real@40360b61            004ce380     renderer:tr_shade_calc.obj
 0002:00012394       ??_C@_05IBIMIMKO@?$CFld?$CFc?$AA@ 004ce394     renderer:jmemmgr.obj
 0002:0001239c       ??_C@_07OOOLPGAB@JPEGMEM?$AA@ 004ce39c     renderer:jmemmgr.obj
 0002:000123e8       __real@4001a855de72ab5d    004ce3e8     renderer:jcdctmgr.obj
 0002:000123f0       __real@4011517a7bc720bb    004ce3f0     renderer:jcdctmgr.obj
 0002:000123f8       __real@40192469c0a7bf3b    004ce3f8     renderer:jcdctmgr.obj
 0002:00012400       __real@4022d062ef6c11aa    004ce400     renderer:jcdctmgr.obj
 0002:00012408       __real@4024e7ae914d6fca    004ce408     renderer:jcdctmgr.obj
 0002:00012410       __real@40263150b14861ef    004ce410     renderer:jcdctmgr.obj
 0002:00012418       __real@4020000000000000    004ce418     renderer:jcdctmgr.obj
 0002:00012420       __real@46800100            004ce420     renderer:jcdctmgr.obj
 0002:00012428       _jpeg_zigzag_order         004ce428     renderer:jutils.obj
 0002:00012528       _jpeg_natural_order        004ce528     renderer:jutils.obj
 0002:00012728       __real@3fd1a855de72ab5d    004ce728     renderer:jddctmgr.obj
 0002:00012730       __real@3fe1517a7bc720bb    004ce730     renderer:jddctmgr.obj
 0002:00012738       __real@3fe92469c0a7bf3b    004ce738     renderer:jddctmgr.obj
 0002:00012740       __real@3ff2d062ef6c11aa    004ce740     renderer:jddctmgr.obj
 0002:00012748       __real@3ff4e7ae914d6fca    004ce748     renderer:jddctmgr.obj
 0002:00012750       __real@3ff63150b14861ef    004ce750     renderer:jddctmgr.obj
 0002:00012758       __real@3fa73d75            004ce758     renderer:jfdctflt.obj
 0002:0001275c       __real@3f0a8bd4            004ce75c     renderer:jfdctflt.obj
 0002:00012760       __real@3ec3ef15            004ce760     renderer:jfdctflt.obj
 0002:00012764       __real@3f3504f3            004ce764     renderer:jfdctflt.obj
 0002:00012768       __real@3f8a8bd4            004ce768     renderer:jidctflt.obj
 0002:0001276c       __real@40273d75            004ce76c     renderer:jidctflt.obj
 0002:00012770       __real@3fec835e            004ce770     renderer:jidctflt.obj
 0002:00012774       __real@3fb504f3            004ce774     renderer:jidctflt.obj
 0002:00012778       ??_C@_0CH@HHAFFDBM@?$CFs?3?5invalid?5client?5number?5?$CFd?0?5?$FL0@ 004ce778     botlib:be_interface.obj
 0002:000127a0       ??_C@_0CH@FBKAEODK@?$CFs?3?5invalid?5entity?5number?5?$CFd?0?5?$FL0@ 004ce7a0     botlib:be_interface.obj
 0002:000127c8       ??_C@_0CJ@LEPGCBMF@?$CFs?3?5bot?5library?5used?5before?5bein@ 004ce7c8     botlib:be_interface.obj
 0002:000127f4       ??_C@_0M@KCCINJFC@maxentities?$AA@ 004ce7f4     botlib:be_interface.obj
 0002:00012800       ??_C@_0L@JKCONGEA@maxclients?$AA@ 004ce800     botlib:be_interface.obj
 0002:0001280c       ??_C@_03KGFMDCCC@128?$AA@  004ce80c     botlib:be_interface.obj
 0002:00012810       ??_C@_0CH@HACDNLAK@?9?9?9?9?9?9?9?5BotLib?5Initialization?5?9?9@ 004ce810     botlib:be_interface.obj
 0002:00012838       ??_C@_0L@KLADBGPO@botlib?4log?$AA@ 004ce838     botlib:be_interface.obj
 0002:00012844       ??_C@_0P@OCLCOFHK@BotLibShutdown?$AA@ 004ce844     botlib:be_interface.obj
 0002:00012854       ??_C@_0O@KCOEGEFI@BotStartFrame?$AA@ 004ce854     botlib:be_interface.obj
 0002:00012864       ??_C@_0CH@GPCMCKNF@?9?9?9?9?9?9?9?9?9?9?9?9?9?9?9?9?9?9?9?9?9?9?9?9?9?9?9?9?9?9?9?9@ 004ce864     botlib:be_interface.obj
 0002:0001288c       ??_C@_0CH@NEJLIBNP@?9?9?9?9?9?9?9?9?9?9?9?9?5Map?5Loading?5?9?9?9?9?9?9?9@ 004ce88c     botlib:be_interface.obj
 0002:000128b4       ??_C@_0L@DEHNJNME@BotLoadMap?$AA@ 004ce8b4     botlib:be_interface.obj
 0002:000128c0       ??_C@_0BA@EHNIKGDG@BotUpdateEntity?$AA@ 004ce8c0     botlib:be_interface.obj
 0002:000128d0       ??_C@_0DE@FKKHEABJ@Mismatched?5BOTLIB_API_VERSION?3?5e@ 004ce8d0     botlib:be_interface.obj
 0002:00012904       ??_C@_0CD@LBGJLEMH@move?5state?5handle?5?$CFd?5out?5of?5rang@ 004ce904     botlib:be_ai_move.obj
 0002:00012928       ??_C@_0BH@MIGCOJAJ@invalid?5move?5state?5?$CFd?6?$AA@ 004ce928     botlib:be_ai_move.obj
 0002:00012940       __real@c066800000000000    004ce940     botlib:be_ai_move.obj
 0002:00012948       __real@44480000            004ce948     botlib:be_ai_move.obj
 0002:0001294c       __real@42400000            004ce94c     botlib:be_ai_move.obj
 0002:00012950       ??_C@_0BJ@OFCFCBJP@no?5entity?5with?5model?5?$CFd?6?$AA@ 004ce950     botlib:be_ai_move.obj
 0002:0001296c       ??_C@_0CF@KPCLGMGH@entity?5?$CFs?5model?5number?5out?5of?5ra@ 004ce96c     botlib:be_ai_move.obj
 0002:00012994       ??_C@_0M@OOBMECJN@func_static?$AA@ 004ce994     botlib:be_ai_move.obj
 0002:000129a0       ??_C@_09KJCKJKEG@func_door?$AA@ 004ce9a0     botlib:be_ai_move.obj
 0002:000129ac       ??_C@_09HCDLIOGG@func_plat?$AA@ 004ce9ac     botlib:be_ai_move.obj
 0002:000129b8       ??_C@_0N@BAMIHEIF@func_bobbing?$AA@ 004ce9b8     botlib:be_ai_move.obj
 0002:000129c8       ??_C@_09CNJINBGN@classname?$AA@ 004ce9c8     botlib:be_ai_move.obj
 0002:000129d4       __real@42700000            004ce9d4     botlib:be_ai_move.obj
 0002:000129d8       __real@42480000            004ce9d8     botlib:be_ai_move.obj
 0002:000129dc       __real@41200000            004ce9dc     botlib:be_ai_move.obj
 0002:000129e0       __real@3fe6666666666666    004ce9e0     botlib:be_ai_move.obj
 0002:000129e8       __real@43c80000            004ce9e8     botlib:be_ai_move.obj
 0002:000129ec       __real@40c00000            004ce9ec     botlib:be_ai_move.obj
 0002:000129f0       __real@41100000            004ce9f0     botlib:be_ai_move.obj
 0002:000129f4       __real@437a0000            004ce9f4     botlib:be_ai_move.obj
 0002:000129f8       __real@42200000            004ce9f8     botlib:be_ai_move.obj
 0002:00012a00       __real@402e000000000000    004cea00     botlib:be_ai_move.obj
 0002:00012a08       __real@4044000000000000    004cea08     botlib:be_ai_move.obj
 0002:00012a10       __real@4051800000000000    004cea10     botlib:be_ai_move.obj
 0002:00012a18       __real@4024000000000000    004cea18     botlib:be_ai_move.obj
 0002:00012a20       __real@41500000            004cea20     botlib:be_ai_move.obj
 0002:00012a28       __real@bfe999999999999a    004cea28     botlib:be_ai_move.obj
 0002:00012a30       __real@41f00000            004cea30     botlib:be_ai_move.obj
 0002:00012a34       ??_C@_0CN@FCEPHGNO@BotFuncBobStartEnd?3?5no?5entity?5wi@ 004cea34     botlib:be_ai_move.obj
 0002:00012a64       __real@43960000            004cea64     botlib:be_ai_move.obj
 0002:00012a68       __real@428c0000            004cea68     botlib:be_ai_move.obj
 0002:00012a70       __real@4000000000000000    004cea70     botlib:be_ai_move.obj
 0002:00012a78       __real@4014000000000000    004cea78     botlib:be_ai_move.obj
 0002:00012a80       ??_C@_0CE@HLPLILDO@travel?5type?5?$CFd?5not?5implemented?5y@ 004cea80     botlib:be_ai_move.obj
 0002:00012aa4       ??_C@_0CL@OINLALFH@?$CIlast?$CJ?5travel?5type?5?$CFd?5not?5implem@ 004ceaa4     botlib:be_ai_move.obj
 0002:00012ad0       ??_C@_0CM@EECBHCFO@client?5?$CFd?5didn?8t?5find?5jumppad?5re@ 004cead0     botlib:be_ai_move.obj
 0002:00012afc       ??_C@_0DB@HHOLNPFB@client?5?$CFd?3?5on?5func_bobbing?5witho@ 004ceafc     botlib:be_ai_move.obj
 0002:00012b30       ??_C@_0CO@IHIDPMNN@client?5?$CFd?3?5on?5func_plat?5without?5@ 004ceb30     botlib:be_ai_move.obj
 0002:00012b60       ??_C@_0P@HCMCPAPN@cmd_grappleoff?$AA@ 004ceb60     botlib:be_ai_move.obj
 0002:00012b70       ??_C@_0L@CGFHOHKL@grappleoff?$AA@ 004ceb70     botlib:be_ai_move.obj
 0002:00012b7c       ??_C@_0O@KJJPDGKD@cmd_grappleon?$AA@ 004ceb7c     botlib:be_ai_move.obj
 0002:00012b8c       ??_C@_09OCNPEJFF@grappleon?$AA@ 004ceb8c     botlib:be_ai_move.obj
 0002:00012b98       ??_C@_0P@DMONFFLF@offhandgrapple?$AA@ 004ceb98     botlib:be_ai_move.obj
 0002:00012ba8       ??_C@_0BC@GDFOAKDA@entitytypemissile?$AA@ 004ceba8     botlib:be_ai_move.obj
 0002:00012bbc       ??_C@_0BC@JLHLAKEN@weapindex_grapple?$AA@ 004cebbc     botlib:be_ai_move.obj
 0002:00012bd0       ??_C@_0BB@HLFMNGMC@weapindex_bfg10k?$AA@ 004cebd0     botlib:be_ai_move.obj
 0002:00012be4       ??_C@_01LAKCGALK@9?$AA@    004cebe4     botlib:be_ai_move.obj
 0002:00012be8       ??_C@_0BJ@HPPOPPGN@weapindex_rocketlauncher?$AA@ 004cebe8     botlib:be_ai_move.obj
 0002:00012c04       ??_C@_0L@FKMMBKBD@sv_gravity?$AA@ 004cec04     botlib:be_ai_move.obj
 0002:00012c10       ??_C@_0O@GNGGPGPK@sv_maxbarrier?$AA@ 004cec10     botlib:be_ai_move.obj
 0002:00012c20       ??_C@_07PBGODEDP@sv_step?$AA@ 004cec20     botlib:be_ai_move.obj
 0002:00012c28       ??_C@_02DCIIBFLB@18?$AA@   004cec28     botlib:be_ai_move.obj
 0002:00012c2c       ??_C@_0CD@PNOBECBL@chat?5state?5handle?5?$CFd?5out?5of?5rang@ 004cec2c     botlib:be_ai_chat.obj
 0002:00012c50       ??_C@_0BH@BOBFFKKN@invalid?5chat?5state?5?$CFd?6?$AA@ 004cec50     botlib:be_ai_chat.obj
 0002:00012c68       ??_C@_0N@CLOBICAF@max_messages?$AA@ 004cec68     botlib:be_ai_chat.obj
 0002:00012c78       ??_C@_0BM@BPJKPONG@empty?5console?5message?5heap?6?$AA@ 004cec78     botlib:be_ai_chat.obj
 0002:00012c94       ??_C@_02JODFHDIE@?$FN?6?$AA@ 004cec94     botlib:be_ai_chat.obj
 0002:00012c98       ??_C@_02KEGNLNML@?0?5?$AA@ 004cec98     botlib:be_ai_chat.obj
 0002:00012c9c       ??_C@_0O@EMHOANHL@?$CI?$CC?$CFs?$CC?0?5?$CF1?42f?$CJ?$AA@ 004cec9c     botlib:be_ai_chat.obj
 0002:00012cac       ??_C@_07MLGNNCMH@?$CFld?5?3?5?$FL?$AA@ 004cecac     botlib:be_ai_chat.obj
 0002:00012cb4       ??_C@_09DKCHGKCM@missing?5?$HN?$AA@ 004cecb4     botlib:be_ai_chat.obj
 0002:00012cc0       ??_C@_0O@EIFOHJCH@unexpected?5?$CFs?$AA@ 004cecc0     botlib:be_ai_chat.obj
 0002:00012cd0       ??_C@_0CI@PKNFOMEN@synonym?5must?5have?5at?5least?5two?5e@ 004cecd0     botlib:be_ai_chat.obj
 0002:00012cf8       ??_C@_0N@BBKGEIBC@empty?5string?$AA@ 004cecf8     botlib:be_ai_chat.obj
 0002:00012d08       ??_C@_0L@DLODIKAH@too?5many?5?$HN?$AA@ 004ced08     botlib:be_ai_chat.obj
 0002:00012d14       ??_C@_0BM@OMAMOJNI@more?5than?532?5context?5levels?$AA@ 004ced14     botlib:be_ai_chat.obj
 0002:00012d30       ??_C@_0BD@IJKNLBNC@counldn?8t?5load?5?$CFs?6?$AA@ 004ced30     botlib:be_ai_chat.obj
 0002:00012d44       ??_C@_0L@EBHNEODC@loaded?5?$CFs?6?$AA@ 004ced44     botlib:be_ai_chat.obj
 0002:00012d50       ??_C@_01LBDDMOBJ@?$FN?$AA@ 004ced50     botlib:be_ai_chat.obj
 0002:00012d54       ??_C@_01IHBHIGKO@?0?$AA@   004ced54     botlib:be_ai_chat.obj
 0002:00012d58       ??_C@_01OHGJGJJP@?$FL?$AA@ 004ced58     botlib:be_ai_chat.obj
 0002:00012d5c       ??_C@_01CELHOKLL@?$HN?$AA@ 004ced5c     botlib:be_ai_chat.obj
 0002:00012d60       ??_C@_01HCONENDN@?$HL?$AA@ 004ced60     botlib:be_ai_chat.obj
 0002:00012d64       ??_C@_08LPOJGGC@botfiles?$AA@ 004ced64     botlib:be_ai_chat.obj
 0002:00012d70       ??_C@_0BO@IKGHDNCH@unknown?5message?5component?5?$CFs?6?$AA@ 004ced70     botlib:be_ai_chat.obj
 0002:00012d90       ??_C@_0BH@MIBABKMH@chat?5message?5too?5long?6?$AA@ 004ced90     botlib:be_ai_chat.obj
 0002:00012da8       ??_C@_01ICJEACDI@?$DL?$AA@ 004ceda8     botlib:be_ai_chat.obj
 0002:00012dac       ??_C@_07NHACKFHP@?$CFcr?$CFs?$CFc?$AA@ 004cedac     botlib:be_ai_chat.obj
 0002:00012db4       ??_C@_08MPPNLMAG@?$CFcv?$CFld?$CFc?$AA@ 004cedb4     botlib:be_ai_chat.obj
 0002:00012dc0       ??_C@_02KGHIDFGE@?$HN?6?$AA@ 004cedc0     botlib:be_ai_chat.obj
 0002:00012dc4       ??_C@_04OEDFLLKD@?$CC?$CFs?$CC?$AA@ 004cedc4     botlib:be_ai_chat.obj
 0002:00012dcc       ??_C@_06EFKGKAHA@?$CFs?5?$DN?5?$HL?$AA@ 004cedcc     botlib:be_ai_chat.obj
 0002:00012dd4       ??_C@_0BC@BAMLPFKF@unknown?5random?5?$CFs?$AA@ 004cedd4     botlib:be_ai_chat.obj
 0002:00012de8       ??_C@_0P@OACPPOMP@?5?$DN?5?$CI?$CFd?0?5?$CFd?$CJ?$DL?$HN?6?$AA@ 004cede8     botlib:be_ai_chat.obj
 0002:00012df8       ??_C@_01DNKMNLPK@?$HM?$AA@ 004cedf8     botlib:be_ai_chat.obj
 0002:00012dfc       ??_C@_02MNJOIFPO@?$HL?5?$AA@ 004cedfc     botlib:be_ai_chat.obj
 0002:00012e00       ??_C@_0BC@KAKFIJOK@invalid?5token?5?$CFs?6?$AA@ 004cee00     botlib:be_ai_chat.obj
 0002:00012e14       ??_C@_0CJ@LJIMHIAM@can?8t?5have?5more?5than?5?$CFd?5match?5va@ 004cee14     botlib:be_ai_chat.obj
 0002:00012e40       ??_C@_0CI@ELCFAGFH@not?5allowed?5to?5have?5adjacent?5var@ 004cee40     botlib:be_ai_chat.obj
 0002:00012e68       ??_C@_0BM@HHFBANAI@expected?5integer?0?5found?5?$CFs?6?$AA@ 004cee68     botlib:be_ai_chat.obj
 0002:00012e84       ??_C@_0CJ@BGCLGFPJ@BotMatchVariable?3?5variable?5out?5o@ 004cee84     botlib:be_ai_chat.obj
 0002:00012eb0       ??_C@_0BP@IFMKLFPG@?$CFs?5?$DN?5?$HL?$CC?$CFs?$CC?$HN?5?1?1MISSING?5RANDOM?$AN?6?$AA@ 004ceeb0     botlib:be_ai_chat.obj
 0002:00012ed0       ??_C@_0EA@MFJADLPG@BotCheckChatMessageIntegrety?3?5me@ 004ceed0     botlib:be_ai_chat.obj
 0002:00012f10       ??_C@_07OMEJJINM@?7?$CC?$CFs?$CC?$DL?6?$AA@ 004cef10     botlib:be_ai_chat.obj
 0002:00012f18       ??_C@_02KCPFEJNG@?$HL?6?$AA@ 004cef18     botlib:be_ai_chat.obj
 0002:00012f1c       ??_C@_0L@CEMLGMNM@?$FN?5?$DN?5?$CF1?40f?6?$AA@ 004cef1c     botlib:be_ai_chat.obj
 0002:00012f28       ??_C@_02MOLGKLA@it?$AA@    004cef28     botlib:be_ai_chat.obj
 0002:00012f2c       ??_C@_06GJLDEJIL@female?$AA@ 004cef2c     botlib:be_ai_chat.obj
 0002:00012f34       ??_C@_01DCLJPIOD@?$CB?$AA@ 004cef34     botlib:be_ai_chat.obj
 0002:00012f38       ??_C@_01HNPIGOCE@?$CG?$AA@ 004cef38     botlib:be_ai_chat.obj
 0002:00012f3c       ??_C@_0BD@FIJOIEDC@BotDumpReplyChat?3?6?$AA@ 004cef3c     botlib:be_ai_chat.obj
 0002:00012f50       ??_C@_0FP@CMPNKFLO@variables?5from?5the?5match?5templat@ 004cef50     botlib:be_ai_chat.obj
 0002:00012fb0       ??_C@_0BO@PNMCIEEB@all?5keys?5have?5a?5?$CG?5or?5?$CB?5prefix?$AA@ 004cefb0     botlib:be_ai_chat.obj
 0002:00012fd0       ??_C@_0EA@FPBKDDJB@the?5key?5?$CFs?5with?5prefix?5?$CB?5is?5insi@ 004cefd0     botlib:be_ai_chat.obj
 0002:00013010       ??_C@_0CO@FOMEJLFB@the?5key?5?$CFs?5with?5prefix?5?$CB?5is?5insi@ 004cf010     botlib:be_ai_chat.obj
 0002:00013040       ??_C@_0FB@GIBDPBLM@one?5of?5the?5match?5templates?5does?5@ 004cf040     botlib:be_ai_chat.obj
 0002:00013094       ??_C@_0BF@NHLDPIBI@expected?5?$FL?0?5found?5?$CFs?$AA@ 004cf094     botlib:be_ai_chat.obj
 0002:000130ac       ??_C@_0L@GIBMDEGE@no?5rchats?6?$AA@ 004cf0ac     botlib:be_ai_chat.obj
 0002:000130b8       ??_C@_01PPODPGHN@?$DO?$AA@ 004cf0b8     botlib:be_ai_chat.obj
 0002:000130bc       ??_C@_01MNNFJEPP@?$DM?$AA@ 004cf0bc     botlib:be_ai_chat.obj
 0002:000130c0       ??_C@_02KCGCGHLG@?5?$HN?$AA@ 004cf0c0     botlib:be_ai_chat.obj
 0002:000130c4       ??_C@_06HHGKKPGK@?5?5?$CC?$CFs?$CC?$AA@ 004cf0c4     botlib:be_ai_chat.obj
 0002:000130cc       ??_C@_0BH@BCOGOEDC@?5?5numchatmessages?5?$DN?5?$CFd?$AA@ 004cf0cc     botlib:be_ai_chat.obj
 0002:000130e4       ??_C@_02PEDIMADA@?5?$HL?$AA@ 004cf0e4     botlib:be_ai_chat.obj
 0002:000130e8       ??_C@_0L@BONMNFAN@?5type?5?$CC?$CFs?$CC?$AA@ 004cf0e8     botlib:be_ai_chat.obj
 0002:000130f4       ??_C@_0BN@OAGFKFDD@couldn?8t?5find?5chat?5?$CFs?5in?5?$CFs?6?$AA@ 004cf0f4     botlib:be_ai_chat.obj
 0002:00013114       ??_C@_0BH@JEMDOFNP@unknown?5definition?5?$CFs?6?$AA@ 004cf114     botlib:be_ai_chat.obj
 0002:0001312c       ??_C@_0BI@CHLNDHKD@expected?5type?5found?5?$CFs?6?$AA@ 004cf12c     botlib:be_ai_chat.obj
 0002:00013144       ??_C@_0BD@KLGBKGBL@loaded?5?$CFs?5from?5?$CFs?6?$AA@ 004cf144     botlib:be_ai_chat.obj
 0002:00013158       ??_C@_04GPMDFGEJ@type?$AA@ 004cf158     botlib:be_ai_chat.obj
 0002:00013160       ??_C@_04BLJLMHHG@chat?$AA@ 004cf160     botlib:be_ai_chat.obj
 0002:00013168       ??_C@_0BP@MBDJBKIB@couldn?8t?5load?5chat?5?$CFs?5from?5?$CFs?6?$AA@ 004cf168     botlib:be_ai_chat.obj
 0002:00013188       ??_C@_0DF@IIKAMBDG@ichatdata?5table?5full?$DL?5couldn?8t?5l@ 004cf188     botlib:be_ai_chat.obj
 0002:000131c0       ??_C@_0CJ@EDLCIPGI@BotConstructChat?3?5message?5?$CC?$CFs?$CC?5t@ 004cf1c0     botlib:be_ai_chat.obj
 0002:000131ec       ??_C@_0CM@GBHEGLKK@BotConstructChat?3?5unknown?5random@ 004cf1ec     botlib:be_ai_chat.obj
 0002:00013218       ??_C@_0CH@JOHLJANI@BotConstructChat?3?5message?5?$CFs?5too@ 004cf218     botlib:be_ai_chat.obj
 0002:00013240       ??_C@_0DH@JNLFODLL@BotConstructChat?3?5message?5?$CFs?5var@ 004cf240     botlib:be_ai_chat.obj
 0002:00013278       ??_C@_0DE@BBIMJEKM@BotConstructChat?3?5message?5?$CC?$CFs?$CC?5i@ 004cf278     botlib:be_ai_chat.obj
 0002:000132ac       ??_C@_0CF@FFFEONNP@too?5many?5expansions?5in?5chat?5mess@ 004cf2ac     botlib:be_ai_chat.obj
 0002:000132d4       ??_C@_0BF@JOLBPMPB@?9?9?9?9?9?9?9?9?9?9?9?9?9?9?9?9?9?9?9?6?$AA@ 004cf2d4     botlib:be_ai_chat.obj
 0002:000132ec       ??_C@_0BG@DAIPIBLI@?$CFs?5has?5?$CFd?5chat?5lines?6?$AA@ 004cf2ec     botlib:be_ai_chat.obj
 0002:00013304       ??_C@_0M@CICLJBLC@say_team?5?$CFs?$AA@ 004cf304     botlib:be_ai_chat.obj
 0002:00013310       ??_C@_0L@LOJGBKIG@tell?5?$CFd?5?$CFs?$AA@ 004cf310     botlib:be_ai_chat.obj
 0002:0001331c       ??_C@_06BCNPLFHG@say?5?$CFs?$AA@ 004cf31c     botlib:be_ai_chat.obj
 0002:00013324       ??_C@_09DMEAFLAH@rchatfile?$AA@ 004cf324     botlib:be_ai_chat.obj
 0002:00013330       ??_C@_07BGFNFHIM@rchat?4c?$AA@ 004cf330     botlib:be_ai_chat.obj
 0002:00013338       ??_C@_06GCPOGFCC@nochat?$AA@ 004cf338     botlib:be_ai_chat.obj
 0002:00013340       ??_C@_09MIMFOEJ@matchfile?$AA@ 004cf340     botlib:be_ai_chat.obj
 0002:0001334c       ??_C@_07DAECBMIF@match?4c?$AA@ 004cf34c     botlib:be_ai_chat.obj
 0002:00013354       ??_C@_07DFFPFLEN@rndfile?$AA@ 004cf354     botlib:be_ai_chat.obj
 0002:0001335c       ??_C@_05OGJCAIGA@rnd?4c?$AA@ 004cf35c     botlib:be_ai_chat.obj
 0002:00013364       ??_C@_07PKBHNKPF@synfile?$AA@ 004cf364     botlib:be_ai_chat.obj
 0002:0001336c       ??_C@_05JALDHADD@syn?4c?$AA@ 004cf36c     botlib:be_ai_chat.obj
 0002:00013374       ??_C@_04IFBFDIKF@maxs?$AA@ 004cf374     botlib:be_ai_goal.obj
 0002:0001337c       ??_C@_04FIAKMPII@mins?$AA@ 004cf37c     botlib:be_ai_goal.obj
 0002:00013384       ??_C@_0M@JFIMPIHC@respawntime?$AA@ 004cf384     botlib:be_ai_goal.obj
 0002:00013390       ??_C@_05FKHKFDID@index?$AA@ 004cf390     botlib:be_ai_goal.obj
 0002:00013398       ??_C@_0CD@HELJPMIG@goal?5state?5handle?5?$CFd?5out?5of?5rang@ 004cf398     botlib:be_ai_goal.obj
 0002:000133bc       ??_C@_0BH@PLLAAOAM@invalid?5goal?5state?5?$CFd?6?$AA@ 004cf3bc     botlib:be_ai_goal.obj
 0002:000133d4       ??_C@_0CA@FLCFPAIO@more?5than?5?$CFd?5item?5info?5defined?6?$AA@ 004cf3d4     botlib:be_ai_goal.obj
 0002:000133f4       ??_C@_0BF@PNCKGICK@no?5item?5info?5loaded?6?$AA@ 004cf3f4     botlib:be_ai_goal.obj
 0002:0001340c       ??_C@_08ENCMGJPE@iteminfo?$AA@ 004cf40c     botlib:be_ai_goal.obj
 0002:00013418       ??_C@_0BD@IBDAAGDO@max_iteminfo?5?$DN?5?$CFd?6?$AA@ 004cf418     botlib:be_ai_goal.obj
 0002:0001342c       ??_C@_0N@FCIHMPOM@max_iteminfo?$AA@ 004cf42c     botlib:be_ai_goal.obj
 0002:0001343c       ??_C@_03CPCFKGMH@256?$AA@  004cf43c     botlib:be_ai_goal.obj
 0002:00013440       ??_C@_0CI@LHHPPLNO@item?5info?5?$CFd?5?$CC?$CFs?$CC?5has?5no?5fuzzy?5w@ 004cf440     botlib:be_ai_goal.obj
 0002:00013468       ??_C@_0P@HIDOFLAM@max_levelitems?$AA@ 004cf468     botlib:be_ai_goal.obj
 0002:00013478       ??_C@_0BE@OPAGCKFM@out?5of?5level?5items?6?$AA@ 004cf478     botlib:be_ai_goal.obj
 0002:0001348c       ??_C@_0P@NDPOMACK@?$CFd?5camp?5spots?6?$AA@ 004cf48c     botlib:be_ai_goal.obj
 0002:0001349c       ??_C@_0BC@GDDPKONG@?$CFd?5map?5locations?6?$AA@ 004cf49c     botlib:be_ai_goal.obj
 0002:000134b0       ??_C@_0CJ@BCICAJAI@camp?5spot?5at?5?$CF1?41f?5?$CF1?41f?5?$CF1?41f?5i@ 004cf4b0     botlib:be_ai_goal.obj
 0002:000134dc       ??_C@_06NLFCANPD@random?$AA@ 004cf4dc     botlib:be_ai_goal.obj
 0002:000134e4       ??_C@_06CMCBKMCB@weight?$AA@ 004cf4e4     botlib:be_ai_goal.obj
 0002:000134ec       ??_C@_05CCGOGOBM@range?$AA@ 004cf4ec     botlib:be_ai_goal.obj
 0002:000134f4       ??_C@_09BLMHBGJ@info_camp?$AA@ 004cf4f4     botlib:be_ai_goal.obj
 0002:00013500       ??_C@_07ONPBMBOP@message?$AA@ 004cf500     botlib:be_ai_goal.obj
 0002:00013508       ??_C@_0BA@BFKBOHOP@target_location?$AA@ 004cf508     botlib:be_ai_goal.obj
 0002:00013518       ??_C@_0BG@FGIAGNA@found?5?$CFd?5level?5items?6?$AA@ 004cf518     botlib:be_ai_goal.obj
 0002:00013530       ??_C@_0DC@LLNGFMLL@?$CFs?5not?5reachable?5for?5bots?5at?5?$CI?$CF1@ 004cf530     botlib:be_ai_goal.obj
 0002:00013564       ??_C@_0CE@GABHNCEE@?$CFs?5in?5solid?5at?5?$CI?$CF1?41f?5?$CF1?41f?5?$CF1?41@ 004cf564     botlib:be_ai_goal.obj
 0002:00013588       ??_C@_0N@PAECNMEH@item_botroam?$AA@ 004cf588     botlib:be_ai_goal.obj
 0002:00013598       ??_C@_06NFBNODNO@notbot?$AA@ 004cf598     botlib:be_ai_goal.obj
 0002:000135a0       ??_C@_09FDFEENEB@notsingle?$AA@ 004cf5a0     botlib:be_ai_goal.obj
 0002:000135ac       ??_C@_07CLBNBEAH@notteam?$AA@ 004cf5ac     botlib:be_ai_goal.obj
 0002:000135b4       ??_C@_07DDCDJNBH@notfree?$AA@ 004cf5b4     botlib:be_ai_goal.obj
 0002:000135bc       ??_C@_0CJ@NOFKLOEA@item?5?$CFs?5reachable?5from?5jumppad?5a@ 004cf5bc     botlib:be_ai_goal.obj
 0002:000135e8       ??_C@_0BI@INFPJMMC@item?5?$CFs?5without?5origin?6?$AA@ 004cf5e8     botlib:be_ai_goal.obj
 0002:00013600       ??_C@_0BJ@KFHJJGAI@entity?5?$CFs?5unknown?5item?$AN?6?$AA@ 004cf600     botlib:be_ai_goal.obj
 0002:0001361c       ??_C@_0L@HLIKNEFC@spawnflags?$AA@ 004cf61c     botlib:be_ai_goal.obj
 0002:00013628       ??_C@_0BJ@GPKBNKNM@item?5?$CFs?5has?5modelindex?50?$AA@ 004cf628     botlib:be_ai_goal.obj
 0002:00013644       ??_C@_0CI@HLDADGI@avoid?5goal?5?$CFs?0?5number?5?$CFd?5for?5?$CFf?5@ 004cf644     botlib:be_ai_goal.obj
 0002:0001366c       ??_C@_06BNEENKNB@?$CFd?3?5?$CFs?$AA@ 004cf66c     botlib:be_ai_goal.obj
 0002:00013674       ??_C@_0BE@BBIKOMDL@goal?5heap?5overflow?6?$AA@ 004cf674     botlib:be_ai_goal.obj
 0002:00013688       __real@3f826e978d4fdf3b    004cf688     botlib:be_ai_goal.obj
 0002:00013690       ??_C@_0BH@LPPOHIHL@couldn?8t?5load?5weights?6?$AA@ 004cf690     botlib:be_ai_goal.obj
 0002:000136a8       ??_C@_0BO@OFOCDAPF@invalid?5goal?5state?5handle?5?$CFd?6?$AA@ 004cf6a8     botlib:be_ai_goal.obj
 0002:000136c8       ??_C@_0O@DPNHINNN@droppedweight?$AA@ 004cf6c8     botlib:be_ai_goal.obj
 0002:000136d8       ??_C@_0BL@DEFNFIDM@couldn?8t?5load?5item?5config?6?$AA@ 004cf6d8     botlib:be_ai_goal.obj
 0002:000136f4       ??_C@_0L@LFADFAG@itemconfig?$AA@ 004cf6f4     botlib:be_ai_goal.obj
 0002:00013700       ??_C@_07HBEMBONH@items?4c?$AA@ 004cf700     botlib:be_ai_goal.obj
 0002:00013708       ??_C@_0L@BHIFJKKK@bouncestop?$AA@ 004cf708     botlib:be_ai_weap.obj
 0002:00013714       ??_C@_0L@PPIMOAKE@bouncefric?$AA@ 004cf714     botlib:be_ai_weap.obj
 0002:00013720       ??_C@_06DPMIMFNG@bounce?$AA@ 004cf720     botlib:be_ai_weap.obj
 0002:00013728       ??_C@_0L@NJHJLKG@detonation?$AA@ 004cf728     botlib:be_ai_weap.obj
 0002:00013734       ??_C@_04GHHNIPCF@push?$AA@ 004cf734     botlib:be_ai_weap.obj
 0002:0001373c       ??_C@_09OLKAIEMO@healthinc?$AA@ 004cf73c     botlib:be_ai_weap.obj
 0002:00013748       ??_C@_0L@LLALLABI@damagetype?$AA@ 004cf748     botlib:be_ai_weap.obj
 0002:00013754       ??_C@_09DOEGBGAO@visdamage?$AA@ 004cf754     botlib:be_ai_weap.obj
 0002:00013760       ??_C@_06KGHINEPG@radius?$AA@ 004cf760     botlib:be_ai_weap.obj
 0002:00013768       ??_C@_06GJOIPFFF@damage?$AA@ 004cf768     botlib:be_ai_weap.obj
 0002:00013770       ??_C@_08PFGPOMOJ@spindown?$AA@ 004cf770     botlib:be_ai_weap.obj
 0002:0001377c       ??_C@_06IGOPKBLH@spinup?$AA@ 004cf77c     botlib:be_ai_weap.obj
 0002:00013784       ??_C@_06DGFOANMH@reload?$AA@ 004cf784     botlib:be_ai_weap.obj
 0002:0001378c       ??_C@_08IFCMKJCD@activate?$AA@ 004cf78c     botlib:be_ai_weap.obj
 0002:00013798       ??_C@_09KNCLBKIN@ammoindex?$AA@ 004cf798     botlib:be_ai_weap.obj
 0002:000137a4       ??_C@_0L@FCOOONPA@ammoamount?$AA@ 004cf7a4     botlib:be_ai_weap.obj
 0002:000137b0       ??_C@_0P@NJBBMHGK@extrazvelocity?$AA@ 004cf7b0     botlib:be_ai_weap.obj
 0002:000137c0       ??_C@_0M@ONPMIPEC@angleoffset?$AA@ 004cf7c0     botlib:be_ai_weap.obj
 0002:000137cc       ??_C@_06KLHHMIGM@offset?$AA@ 004cf7cc     botlib:be_ai_weap.obj
 0002:000137d4       ??_C@_06HCMEEBKG@recoil?$AA@ 004cf7d4     botlib:be_ai_weap.obj
 0002:000137dc       ??_C@_0N@OKFAMOHD@acceleration?$AA@ 004cf7dc     botlib:be_ai_weap.obj
 0002:000137ec       ??_C@_07OBCOMENM@vspread?$AA@ 004cf7ec     botlib:be_ai_weap.obj
 0002:000137f4       ??_C@_07IIBPOHMF@hspread?$AA@ 004cf7f4     botlib:be_ai_weap.obj
 0002:000137fc       ??_C@_0P@NGONDBIO@numprojectiles?$AA@ 004cf7fc     botlib:be_ai_weap.obj
 0002:0001380c       ??_C@_0L@BOMCPGNF@projectile?$AA@ 004cf80c     botlib:be_ai_weap.obj
 0002:00013818       ??_C@_05GECEPKB@flags?$AA@ 004cf818     botlib:be_ai_weap.obj
 0002:00013820       ??_C@_0M@PNPIEPHK@weaponindex?$AA@ 004cf820     botlib:be_ai_weap.obj
 0002:0001382c       ??_C@_05KJNJLLGA@level?$AA@ 004cf82c     botlib:be_ai_weap.obj
 0002:00013834       ??_C@_06EBGNBFIA@number?$AA@ 004cf834     botlib:be_ai_weap.obj
 0002:0001383c       ??_C@_0BM@JHOEFCAC@weapon?5number?5out?5of?5range?6?$AA@ 004cf83c     botlib:be_ai_weap.obj
 0002:00013858       ??_C@_0CL@PNIBMIGN@weapon?5?$CFs?5uses?5undefined?5project@ 004cf858     botlib:be_ai_weap.obj
 0002:00013884       ??_C@_0CD@BOCMCBMN@weapon?5?$CFs?5has?5no?5projectile?5in?5?$CF@ 004cf884     botlib:be_ai_weap.obj
 0002:000138a8       ??_C@_0BN@NFAIFCED@weapon?5?$CFd?5has?5no?5name?5in?5?$CFs?6?$AA@ 004cf8a8     botlib:be_ai_weap.obj
 0002:000138c8       ??_C@_0BH@BCLPAAIH@no?5weapon?5info?5loaded?6?$AA@ 004cf8c8     botlib:be_ai_weap.obj
 0002:000138e0       ??_C@_0BN@CDKNOAJI@unknown?5definition?5?$CFs?5in?5?$CFs?6?$AA@ 004cf8e0     botlib:be_ai_weap.obj
 0002:00013900       ??_C@_0CI@CKKHFCFJ@more?5than?5?$CFd?5projectiles?5defined@ 004cf900     botlib:be_ai_weap.obj
 0002:00013928       ??_C@_0CK@BMAKINJL@weapon?5info?5number?5?$CFd?5out?5of?5ran@ 004cf928     botlib:be_ai_weap.obj
 0002:00013954       ??_C@_0P@ECOEJLJA@projectileinfo?$AA@ 004cf954     botlib:be_ai_weap.obj
 0002:00013964       ??_C@_0L@DNADMFPA@weaponinfo?$AA@ 004cf964     botlib:be_ai_weap.obj
 0002:00013970       ??_C@_0BJ@DEOLMOJN@max_projectileinfo?5?$DN?5?$CFd?6?$AA@ 004cf970     botlib:be_ai_weap.obj
 0002:0001398c       ??_C@_0BD@NPBGALBJ@max_projectileinfo?$AA@ 004cf98c     botlib:be_ai_weap.obj
 0002:000139a0       ??_C@_0BF@IEGKFMLK@max_weaponinfo?5?$DN?5?$CFd?6?$AA@ 004cf9a0     botlib:be_ai_weap.obj
 0002:000139b8       ??_C@_0P@IAKNEENP@max_weaponinfo?$AA@ 004cf9b8     botlib:be_ai_weap.obj
 0002:000139c8       ??_C@_0CA@KGGEKGMG@couldn?8t?5load?5weapon?5config?5?$CFs?6?$AA@ 004cf9c8     botlib:be_ai_weap.obj
 0002:000139e8       ??_C@_0CB@OGKBNMGI@couldn?8t?5load?5the?5weapon?5config?6@ 004cf9e8     botlib:be_ai_weap.obj
 0002:00013a0c       ??_C@_0N@LAFMGPOO@weaponconfig?$AA@ 004cfa0c     botlib:be_ai_weap.obj
 0002:00013a1c       ??_C@_09DEBEJFNC@weapons?4c?$AA@ 004cfa1c     botlib:be_ai_weap.obj
 0002:00013a28       ??_C@_0M@JKGINFAL@tell?5?$CFd?0?5?$CFs?$AA@ 004cfa28     botlib:be_ea.obj
 0002:00013a34       ??_C@_06JKABFJFP@use?5?$CFs?$AA@ 004cfa34     botlib:be_ea.obj
 0002:00013a3c       ??_C@_07CPFNBDJF@drop?5?$CFs?$AA@ 004cfa3c     botlib:be_ea.obj
 0002:00013a44       ??_C@_09DHILADMM@invuse?5?$CFs?$AA@ 004cfa44     botlib:be_ea.obj
 0002:00013a50       ??_C@_0L@EGPGFLDB@invdrop?5?$CFs?$AA@ 004cfa50     botlib:be_ea.obj
 0002:00013a5c       __real@c3c80000            004cfa5c     botlib:be_ea.obj
 0002:00013a60       ??_C@_0BL@LKJOCOEM@?$CFs?3?5index?5?$CFd?5out?5of?5range?6?$AA@ 004cfa60     botlib:be_aas_main.obj
 0002:00013a7c       ??_C@_0CC@NOMCHAJ@?$CFs?3?5reference?5to?5unused?5index?5?$CFd@ 004cfa7c     botlib:be_aas_main.obj
 0002:00013aa0       ??_C@_0BI@OOMOACGM@?$CFs?3?5index?5?$CFd?5not?5setup?6?$AA@ 004cfaa0     botlib:be_aas_main.obj
 0002:00013ab8       ??_C@_0BK@IEPMPCKO@?$CFs?3?5index?5not?5setup?5?$CC?$CFs?$CC?6?$AA@ 004cfab8     botlib:be_aas_main.obj
 0002:00013ad4       ??_C@_0P@FNFFGKPG@ModelFromIndex?$AA@ 004cfad4     botlib:be_aas_main.obj
 0002:00013ae4       ??_C@_0P@NMFGOFFJ@IndexFromModel?$AA@ 004cfae4     botlib:be_aas_main.obj
 0002:00013af4       ??_C@_0BC@CLICPINC@AAS?5initialized?4?6?$AA@ 004cfaf4     botlib:be_aas_main.obj
 0002:00013b08       ??_C@_0BD@KNDGFCCN@couldn?8t?5write?5?$CFs?6?$AA@ 004cfb08     botlib:be_aas_main.obj
 0002:00013b1c       ??_C@_0BI@PECGHGFB@?$CFs?5written?5succesfully?6?$AA@ 004cfb1c     botlib:be_aas_main.obj
 0002:00013b34       ??_C@_0M@MFMPGCMK@aasoptimize?$AA@ 004cfb34     botlib:be_aas_main.obj
 0002:00013b40       ??_C@_0L@MNCDALON@forcewrite?$AA@ 004cfb40     botlib:be_aas_main.obj
 0002:00013b4c       ??_C@_0BB@GMCJAANP@saveroutingcache?$AA@ 004cfb4c     botlib:be_aas_main.obj
 0002:00013b60       ??_C@_0L@JEKILDFB@memorydump?$AA@ 004cfb60     botlib:be_aas_main.obj
 0002:00013b6c       ??_C@_0BA@OBLODKFG@showmemoryusage?$AA@ 004cfb6c     botlib:be_aas_main.obj
 0002:00013b7c       ??_C@_0BB@FOPILIHM@showcacheupdates?$AA@ 004cfb7c     botlib:be_aas_main.obj
 0002:00013b90       ??_C@_0M@BMODPEIJ@maps?1?$CFs?4aas?$AA@ 004cfb90     botlib:be_aas_main.obj
 0002:00013b9c       ??_C@_0P@MCFJEJDN@AAS?5shutdown?4?6?$AA@ 004cfb9c     botlib:be_aas_main.obj
 0002:00013bac       ??_C@_0BE@DPLJFOML@openlog?5?$DMfilename?$DO?6?$AA@ 004cfbac     botlib:l_log.obj
 0002:00013bc0       ??_C@_0P@OAMPMFKE@Opened?5log?5?$CFs?6?$AA@ 004cfbc0     botlib:l_log.obj
 0002:00013bd0       ??_C@_0BM@MCGFOLNG@can?8t?5open?5the?5log?5file?5?$CFs?6?$AA@ 004cfbd0     botlib:l_log.obj
 0002:00013bec       ??_C@_0BP@DENECPGL@log?5file?5?$CFs?5is?5already?5opened?6?$AA@ 004cfbec     botlib:l_log.obj
 0002:00013c0c       ??_C@_03MGHMBJCF@log?$AA@  004cfc0c     botlib:l_log.obj
 0002:00013c10       ??_C@_0P@EBJFELDF@Closed?5log?5?$CFs?6?$AA@ 004cfc10     botlib:l_log.obj
 0002:00013c20       ??_C@_0BJ@GMGFLNFJ@can?8t?5close?5log?5file?5?$CFs?6?$AA@ 004cfc20     botlib:l_log.obj
 0002:00013c3c       ??_C@_02PCIJFNDE@?$AN?6?$AA@ 004cfc3c     botlib:l_log.obj
 0002:00013c40       ??_C@_0BM@IGDCFNDJ@?$CFd?5?5?5?$CF02d?3?$CF02d?3?$CF02d?3?$CF02d?5?5?5?$AA@ 004cfc40     botlib:l_log.obj
 0002:00013c5c       __real@3991a2b4            004cfc5c     botlib:l_log.obj
 0002:00013c60       __real@3c888889            004cfc60     botlib:l_log.obj
 0002:00013c64       __real@c2c80000            004cfc64     botlib:l_log.obj
 0002:00013c68       ??_C@_07FNDAMPLK@evalint?$AA@ 004cfc68     botlib:l_precomp.obj
 0002:00013c70       ??_C@_09BLDJOION@evalfloat?$AA@ 004cfc70     botlib:l_precomp.obj
 0002:00013c7c       ??_C@_04KGAGIKCD@eval?$AA@ 004cfc7c     botlib:l_precomp.obj
 0002:00013c84       ??_C@_06PGFLMPLC@pragma?$AA@ 004cfc84     botlib:l_precomp.obj
 0002:00013c8c       ??_C@_04HJPCFDOP@line?$AA@ 004cfc8c     botlib:l_precomp.obj
 0002:00013c94       ??_C@_05PKCPKOLM@undef?$AA@ 004cfc94     botlib:l_precomp.obj
 0002:00013c9c       ??_C@_06EPMMJFDC@define?$AA@ 004cfc9c     botlib:l_precomp.obj
 0002:00013ca4       ??_C@_07FHOHOHLG@include?$AA@ 004cfca4     botlib:l_precomp.obj
 0002:00013cac       ??_C@_05PAODFFED@endif?$AA@ 004cfcac     botlib:l_precomp.obj
 0002:00013cb4       ??_C@_04FHMCPBIP@else?$AA@ 004cfcb4     botlib:l_precomp.obj
 0002:00013cbc       ??_C@_04GNFOIEOK@elif?$AA@ 004cfcbc     botlib:l_precomp.obj
 0002:00013cc4       ??_C@_06ENONKJGC@ifndef?$AA@ 004cfcc4     botlib:l_precomp.obj
 0002:00013ccc       ??_C@_05LOELCHJN@ifdef?$AA@ 004cfccc     botlib:l_precomp.obj
 0002:00013cd4       ??_C@_02HEBPBKGD@if?$AA@   004cfcd4     botlib:l_precomp.obj
 0002:00013cd8       ??_C@_0BG@GBKGLIDE@file?5?$CFs?0?5line?5?$CFd?3?5?$CFs?6?$AA@ 004cfcd8     botlib:l_precomp.obj
 0002:00013cf0       ??_C@_0BI@DBGANKKJ@?$CFs?5recursively?5included?$AA@ 004cfcf0     botlib:l_precomp.obj
 0002:00013d08       ??_C@_0BE@PFGKJJGH@out?5of?5token?5space?6?$AA@ 004cfd08     botlib:l_precomp.obj
 0002:00013d1c       ??_C@_0P@IFDFMCIL@missing?5?$CDendif?$AA@ 004cfd1c     botlib:l_precomp.obj
 0002:00013d2c       ??_C@_0BF@PPHAFKBJ@define?5?$CFs?5incomplete?$AA@ 004cfd2c     botlib:l_precomp.obj
 0002:00013d44       ??_C@_0BN@LKHLCMOF@define?5?$CFs?5has?5too?5many?5parms?$AA@ 004cfd44     botlib:l_precomp.obj
 0002:00013d64       ??_C@_0BO@CIDPMME@define?5?$CFs?5with?5too?5many?5parms?$AA@ 004cfd64     botlib:l_precomp.obj
 0002:00013d84       ??_C@_0BF@GHJFDBAE@too?5few?5define?5parms?$AA@ 004cfd84     botlib:l_precomp.obj
 0002:00013d9c       ??_C@_0BB@HBCKCGHH@too?5many?5comma?8s?$AA@ 004cfd9c     botlib:l_precomp.obj
 0002:00013db0       ??_C@_0CE@LBMAFIHE@define?5with?5more?5than?5?$CFd?5paramet@ 004cfdb0     botlib:l_precomp.obj
 0002:00013dd4       ??_C@_0BI@CAHOPMH@define?5?$CFs?5missing?5parms?$AA@ 004cfdd4     botlib:l_precomp.obj
 0002:00013dec       ??_C@_04CFMCHKOF@?$CF4d?3?$AA@ 004cfdec     botlib:l_precomp.obj
 0002:00013df4       ??_C@_08JBLMAOHN@__TIME__?$AA@ 004cfdf4     botlib:l_precomp.obj
 0002:00013e00       ??_C@_08HHMBOFCN@__DATE__?$AA@ 004cfe00     botlib:l_precomp.obj
 0002:00013e0c       ??_C@_08FMJNKKCK@__FILE__?$AA@ 004cfe0c     botlib:l_precomp.obj
 0002:00013e18       ??_C@_08ICCNKGAE@__LINE__?$AA@ 004cfe18     botlib:l_precomp.obj
 0002:00013e24       ??_C@_0BH@DDBOIAKK@can?8t?5merge?5?$CFs?5with?5?$CFs?$AA@ 004cfe24     botlib:l_precomp.obj
 0002:00013e3c       ??_C@_0BH@FGJBFJMP@can?8t?5stringize?5tokens?$AA@ 004cfe3c     botlib:l_precomp.obj
 0002:00013e54       ??_C@_0CO@FIAHGJJO@stringizing?5operator?5without?5def@ 004cfe54     botlib:l_precomp.obj
 0002:00013e84       ??_C@_0BC@ELACKGMC@file?5?$CFs?5not?5found?$AA@ 004cfe84     botlib:l_precomp.obj
 0002:00013e98       ??_C@_0CH@BILCEFJF@?$CDinclude?5without?5file?5name?5betwe@ 004cfe98     botlib:l_precomp.obj
 0002:00013ec0       ??_C@_0BM@MKHAAFFA@?$CDinclude?5missing?5trailing?5?$DO?$AA@ 004cfec0     botlib:l_precomp.obj
 0002:00013edc       ??_C@_0BL@MDEODINB@?$CDinclude?5without?5file?5name?$AA@ 004cfedc     botlib:l_precomp.obj
 0002:00013ef8       ??_C@_0P@CHOGDKAE@can?8t?5undef?5?$CFs?$AA@ 004cfef8     botlib:l_precomp.obj
 0002:00013f08       ??_C@_0BI@LCFFDKMI@expected?5name?0?5found?5?$CFs?$AA@ 004cff08     botlib:l_precomp.obj
 0002:00013f20       ??_C@_0BD@IELPOLI@undef?5without?5name?$AA@ 004cff20     botlib:l_precomp.obj
 0002:00013f34       ??_C@_0CF@NLPAJGLD@expected?5name?5after?5?$CDifdef?0?5foun@ 004cff34     botlib:l_precomp.obj
 0002:00013f5c       ??_C@_0BE@IMBJDEPK@?$CDifdef?5without?5name?$AA@ 004cff5c     botlib:l_precomp.obj
 0002:00013f70       ??_C@_0BC@LGACBGNI@?$CDelse?5after?5?$CDelse?$AA@ 004cff70     botlib:l_precomp.obj
 0002:00013f84       ??_C@_0BA@NPOEMJCD@misplaced?5?$CDelse?$AA@ 004cff84     botlib:l_precomp.obj
 0002:00013f94       ??_C@_0BB@CPALJMLI@misplaced?5?$CDendif?$AA@ 004cff94     botlib:l_precomp.obj
 0002:00013fa8       ??_C@_0BH@CHBBNAOH@?$DP?5after?5?$DP?5in?5?$CDif?1?$CDelif?$AA@ 004cffa8     botlib:l_precomp.obj
 0002:00013fc0       ??_C@_0BJ@JILHHGIH@?3?5without?5?$DP?5in?5?$CDif?1?$CDelif?$AA@ 004cffc0     botlib:l_precomp.obj
 0002:00013fdc       ??_C@_0BN@HMNACNG@divide?5by?5zero?5in?5?$CDif?1?$CDelif?6?$AA@ 004cffdc     botlib:l_precomp.obj
 0002:00013ffc       ??_C@_0BL@BNPPJONA@mising?5values?5in?5?$CDif?1?$CDelif?$AA@ 004cfffc     botlib:l_precomp.obj
 0002:00014018       ??_C@_0BI@MJMEGLFD@too?5many?5?$CI?5in?5?$CDif?1?$CDelif?$AA@ 004d0018     botlib:l_precomp.obj
 0002:00014030       ??_C@_0BP@NIBGGAAE@trailing?5operator?5in?5?$CDif?1?$CDelif?$AA@ 004d0030     botlib:l_precomp.obj
 0002:00014050       ??_C@_0BE@PAMHPFIE@out?5of?5value?5space?6?$AA@ 004d0050     botlib:l_precomp.obj
 0002:00014064       ??_C@_0BK@PKFCEECE@syntax?5error?5in?5?$CDif?1?$CDelif?$AA@ 004d0064     botlib:l_precomp.obj
 0002:00014080       ??_C@_0CC@OHHFNCNF@defined?5without?5name?5in?5?$CDif?1?$CDeli@ 004d0080     botlib:l_precomp.obj
 0002:000140a4       ??_C@_0BP@FNAPCIDI@defined?5without?5?$CJ?5in?5?$CDif?1?$CDelif?$AA@ 004d00a4     botlib:l_precomp.obj
 0002:000140c4       ??_C@_0BP@FCIAONAD@undefined?5name?5?$CFs?5in?5?$CDif?1?$CDelif?$AA@ 004d00c4     botlib:l_precomp.obj
 0002:000140e4       ??_C@_0BH@OFGCJCOE@out?5of?5operator?5space?6?$AA@ 004d00e4     botlib:l_precomp.obj
 0002:000140fc       ??_C@_0CB@PFAFLJI@invalid?5operator?5?$CFs?5in?5?$CDif?1?$CDelif@ 004d00fc     botlib:l_precomp.obj
 0002:00014120       ??_C@_0CI@GGOHGOKI@operator?5?$CFs?5after?5operator?5in?5?$CDi@ 004d0120     botlib:l_precomp.obj
 0002:00014148       ??_C@_0DA@OGPMIBNF@illigal?5operator?5?$CFs?5on?5floating?5@ 004d0148     botlib:l_precomp.obj
 0002:00014178       ??_C@_0CC@DNHHPAPI@misplaced?5minus?5sign?5in?5?$CDif?1?$CDeli@ 004d0178     botlib:l_precomp.obj
 0002:0001419c       ??_C@_0BI@ONNIJHPK@unknown?5?$CFs?5in?5?$CDif?1?$CDelif?$AA@ 004d019c     botlib:l_precomp.obj
 0002:000141b4       ??_C@_07MJAJDDLG@defined?$AA@ 004d01b4     botlib:l_precomp.obj
 0002:000141bc       ??_C@_0BL@GBPPHEGE@?$CL?$CL?5or?5?9?9?5used?5in?5?$CDif?1?$CDelif?$AA@ 004d01bc     botlib:l_precomp.obj
 0002:000141d8       ??_C@_0CA@FEDLLKBK@?$CB?5or?5?$HO?5after?5value?5in?5?$CDif?1?$CDelif?$AA@ 004d01d8     botlib:l_precomp.obj
 0002:000141f8       ??_C@_0BJ@FLJMGJFD@too?5many?5?$CJ?5in?5?$CDif?1?$CDelsif?$AA@ 004d01f8     botlib:l_precomp.obj
 0002:00014214       ??_C@_0BC@JLPCHENH@can?8t?5evaluate?5?$CFs?$AA@ 004d0214     botlib:l_precomp.obj
 0002:00014228       ??_C@_0BP@GDBMMIIP@can?8t?5evaluate?5?$CFs?0?5not?5defined?$AA@ 004d0228     botlib:l_precomp.obj
 0002:00014248       ??_C@_0BJ@GGKGDEMC@no?5value?5after?5?$CDif?1?$CDelif?$AA@ 004d0248     botlib:l_precomp.obj
 0002:00014264       ??_C@_0BE@NEDCJHGJ@nothing?5to?5evaluate?$AA@ 004d0264     botlib:l_precomp.obj
 0002:00014278       ??_C@_0CH@DDGJDDBD@no?5leading?5?$CI?5after?5$evalint?1$eva@ 004d0278     botlib:l_precomp.obj
 0002:000142a0       ??_C@_0BA@OFHILMEG@misplaced?5?$CDelif?$AA@ 004d02a0     botlib:l_precomp.obj
 0002:000142b0       ??_C@_0BO@PLIOJNDH@?$CDline?5directive?5not?5supported?$AA@ 004d02b0     botlib:l_precomp.obj
 0002:000142d0       ??_C@_0BF@PIGJJAAO@?$CDerror?5directive?3?5?$CFs?$AA@ 004d02d0     botlib:l_precomp.obj
 0002:000142e8       ??_C@_0CA@KICMIAFO@?$CDpragma?5directive?5not?5supported?$AA@ 004d02e8     botlib:l_precomp.obj
 0002:00014308       ??_C@_05NBLIHODN@?$CF1?42f?$AA@ 004d0308     botlib:l_precomp.obj
 0002:00014310       ??_C@_0CB@OMHFNJIL@unknown?5precompiler?5directive?5?$CFs@ 004d0310     botlib:l_precomp.obj
 0002:00014334       ??_C@_0BH@CKLPJCIG@found?5?$CD?5at?5end?5of?5line?$AA@ 004d0334     botlib:l_precomp.obj
 0002:0001434c       ??_C@_0BF@PIJDPBJF@found?5?$CD?5without?5name?$AA@ 004d034c     botlib:l_precomp.obj
 0002:00014364       ??_C@_0BH@KCNOOMN@found?5$?5at?5end?5of?5line?$AA@ 004d0364     botlib:l_precomp.obj
 0002:0001437c       ??_C@_0BF@GDJCPOIP@found?5$?5without?5name?$AA@ 004d037c     botlib:l_precomp.obj
 0002:00014394       ??_C@_0CD@DCDKNJKM@file?5?$CFs?5still?5open?5in?5precompile@ 004d0394     botlib:l_precomp.obj
 0002:000143b8       ??_C@_0CB@GIDBGAHO@string?5longer?5than?5MAX_TOKEN?5?$CFd?6@ 004d03b8     botlib:l_precomp.obj
 0002:000143dc       ??_C@_0BG@PHOMHNKB@expected?5?$CFs?0?5found?5?$CFs?$AA@ 004d03dc     botlib:l_precomp.obj
 0002:000143f4       ??_C@_0BK@JEDPJDDM@couldn?8t?5find?5expected?5?$CFs?$AA@ 004d03f4     botlib:l_precomp.obj
 0002:00014410       ??_C@_08EFPOOAED@found?5?$CFs?$AA@ 004d0410     botlib:l_precomp.obj
 0002:0001441c       ??_C@_08LLKPIPDF@?5integer?$AA@ 004d041c     botlib:l_precomp.obj
 0002:00014428       ??_C@_06EOECJFKG@?5float?$AA@ 004d0428     botlib:l_precomp.obj
 0002:00014430       ??_C@_09GBGALIGL@?5unsigned?$AA@ 004d0430     botlib:l_precomp.obj
 0002:0001443c       ??_C@_05BOODDNDJ@?5long?$AA@ 004d043c     botlib:l_precomp.obj
 0002:00014444       ??_C@_06FNFBAEBE@binary?$AA@ 004d0444     botlib:l_precomp.obj
 0002:0001444c       ??_C@_05NANFMDJ@octal?$AA@ 004d044c     botlib:l_precomp.obj
 0002:00014454       ??_C@_07EEKBCPDP@decimal?$AA@ 004d0454     botlib:l_precomp.obj
 0002:0001445c       ??_C@_0BI@DOMAOFAI@expected?5a?5?$CFs?0?5found?5?$CFs?$AA@ 004d045c     botlib:l_precomp.obj
 0002:00014474       ??_C@_0M@CCLOEHNM@punctuation?$AA@ 004d0474     botlib:l_precomp.obj
 0002:00014480       ??_C@_07IDLNMGBF@literal?$AA@ 004d0480     botlib:l_precomp.obj
 0002:00014488       ??_C@_06ICGJLFIM@string?$AA@ 004d0488     botlib:l_precomp.obj
 0002:00014490       ??_C@_0BN@ECGBICMG@couldn?8t?5read?5expected?5token?$AA@ 004d0490     botlib:l_precomp.obj
 0002:000144b0       ??_C@_0BJ@FCHLMCOB@define?5with?5misplaced?5?$CD?$CD?$AA@ 004d04b0     botlib:l_precomp.obj
 0002:000144cc       ??_C@_02IEBMKJDF@?$CD?$CD?$AA@ 004d04cc     botlib:l_precomp.obj
 0002:000144d0       ??_C@_0CF@FNOAJAKF@recursive?5define?5?$CIremoved?5recurs@ 004d04d0     botlib:l_precomp.obj
 0002:000144f8       ??_C@_0BG@PHCEBIF@define?5not?5terminated?$AA@ 004d04f8     botlib:l_precomp.obj
 0002:00014510       ??_C@_0CB@JHGJFPBB@define?5parameters?5not?5terminated@ 004d0510     botlib:l_precomp.obj
 0002:00014534       ??_C@_0BP@HPJAJOKD@two?5the?5same?5define?5parameters?$AA@ 004d0534     botlib:l_precomp.obj
 0002:00014554       ??_C@_0BJ@CDAIKNHD@invalid?5define?5parameter?$AA@ 004d0554     botlib:l_precomp.obj
 0002:00014570       ??_C@_0BK@OHINAMCG@expected?5define?5parameter?$AA@ 004d0570     botlib:l_precomp.obj
 0002:0001458c       ??_C@_0BD@PFJBIMHG@redefinition?5of?5?$CFs?$AA@ 004d058c     botlib:l_precomp.obj
 0002:000145a0       ??_C@_0BC@PNHKPGCD@can?8t?5redefine?5?$CFs?$AA@ 004d05a0     botlib:l_precomp.obj
 0002:000145b4       ??_C@_0CG@PGNFJILG@expected?5name?5after?5?$CDdefine?0?5fou@ 004d05b4     botlib:l_precomp.obj
 0002:000145dc       ??_C@_0BF@EDHDDJPD@?$CDdefine?5without?5name?$AA@ 004d05dc     botlib:l_precomp.obj
 0002:000145f4       ??_C@_07GADFAJMP@?$CKextern?$AA@ 004d05f4     botlib:l_precomp.obj
 0002:000145fc       ??_C@_0CC@MOFCJGCF@character?5handle?5?$CFd?5out?5of?5range@ 004d05fc     botlib:be_ai_char.obj
 0002:00014620       ??_C@_0BG@MOINIJPL@invalid?5character?5?$CFd?6?$AA@ 004d0620     botlib:be_ai_char.obj
 0002:00014638       ??_C@_08GMEDCLD@?5?$CF4d?5?$CFd?6?$AA@ 004d0638     botlib:be_ai_char.obj
 0002:00014644       ??_C@_08FEAOGNN@?5?$CF4d?5?$CFf?6?$AA@ 004d0644     botlib:be_ai_char.obj
 0002:00014650       ??_C@_08BPKNIHEG@?5?$CF4d?5?$CFs?6?$AA@ 004d0650     botlib:be_ai_char.obj
 0002:0001465c       ??_C@_09MAKFBPDF@skill?5?$CFd?6?$AA@ 004d065c     botlib:be_ai_char.obj
 0002:00014668       ??_C@_0CC@HINMPLM@expected?5integer?5index?0?5found?5?$CFs@ 004d0668     botlib:be_ai_char.obj
 0002:0001468c       ??_C@_0CL@PPLBNLNK@characteristic?5index?5out?5of?5rang@ 004d068c     botlib:be_ai_char.obj
 0002:000146b8       ??_C@_0CN@FGECCABF@expected?5integer?0?5float?5or?5strin@ 004d06b8     botlib:be_ai_char.obj
 0002:000146e8       ??_C@_0CH@LHHMLMDG@characteristic?5?$CFd?5already?5initia@ 004d06e8     botlib:be_ai_char.obj
 0002:00014710       ??_C@_05ODMCMJAJ@skill?$AA@ 004d0710     botlib:be_ai_char.obj
 0002:00014718       ??_C@_0CB@MKGIENMG@couldn?8t?5load?5any?5skill?5from?5?$CFs?6@ 004d0718     botlib:be_ai_char.obj
 0002:0001473c       ??_C@_0CB@OBHKNOIO@loaded?5default?5skill?5?$CFf?5from?5?$CFs?6@ 004d073c     botlib:be_ai_char.obj
 0002:00014760       ??_C@_0CI@NPODPODE@loaded?5cached?5default?5skill?5?$CFf?5f@ 004d0760     botlib:be_ai_char.obj
 0002:00014788       ??_C@_0BJ@EMLEGOCJ@loaded?5skill?5?$CFf?5from?5?$CFs?6?$AA@ 004d0788     botlib:be_ai_char.obj
 0002:000147a4       ??_C@_0CA@CAABAEMN@loaded?5cached?5skill?5?$CFf?5from?5?$CFs?6?$AA@ 004d07a4     botlib:be_ai_char.obj
 0002:000147c4       ??_C@_0CB@LJBGGHEP@loaded?5default?5skill?5?$CFd?5from?5?$CFs?6@ 004d07c4     botlib:be_ai_char.obj
 0002:000147e8       ??_C@_0CI@IHIPEHPF@loaded?5cached?5default?5skill?5?$CFd?5f@ 004d07e8     botlib:be_ai_char.obj
 0002:00014810       ??_C@_0BB@OCLCLNLB@bots?1default_c?4c?$AA@ 004d0810     botlib:be_ai_char.obj
 0002:00014824       ??_C@_0BO@KHBDCBON@couldn?8t?5find?5skill?5?$CFd?5in?5?$CFs?6?$AA@ 004d0824     botlib:be_ai_char.obj
 0002:00014844       ??_C@_0BJ@BENINHOI@loaded?5skill?5?$CFd?5from?5?$CFs?6?$AA@ 004d0844     botlib:be_ai_char.obj
 0002:00014860       __real@4010000000000000    004d0860     botlib:be_ai_char.obj
 0002:00014868       ??_C@_0CC@FCGCALKF@characteristic?5?$CFd?5does?5not?5exist@ 004d0868     botlib:be_ai_char.obj
 0002:0001488c       ??_C@_0CG@PKODDELM@characteristic?5?$CFd?5is?5not?5initial@ 004d088c     botlib:be_ai_char.obj
 0002:000148b4       ??_C@_0CC@DHDJPPBG@characteristic?5?$CFd?5is?5not?5a?5float@ 004d08b4     botlib:be_ai_char.obj
 0002:000148d8       ??_C@_0DC@DHJFBIJH@cannot?5bound?5characteristic?5?$CFd?5b@ 004d08d8     botlib:be_ai_char.obj
 0002:0001490c       ??_C@_0CE@LLNBHBFO@characteristic?5?$CFd?5is?5not?5a?5integ@ 004d090c     botlib:be_ai_char.obj
 0002:00014930       ??_C@_0DC@DAOEBMME@cannot?5bound?5characteristic?5?$CFd?5b@ 004d0930     botlib:be_ai_char.obj
 0002:00014964       ??_C@_0CD@JOPFDMMO@characteristic?5?$CFd?5is?5not?5a?5strin@ 004d0964     botlib:be_ai_char.obj
 0002:00014988       ??_C@_0BJ@GLODEBJK@invalid?5return?5value?5?$CFs?6?$AA@ 004d0988     botlib:be_ai_weight.obj
 0002:000149a4       ??_C@_0BM@HDMBEFIO@negative?5value?5set?5to?5zero?6?$AA@ 004d09a4     botlib:be_ai_weight.obj
 0002:000149c0       ??_C@_07HHFEDLHG@balance?$AA@ 004d09c0     botlib:be_ai_weight.obj
 0002:000149c8       ??_C@_0BO@EHFJJING@switch?5already?5has?5a?5default?6?$AA@ 004d09c8     botlib:be_ai_weight.obj
 0002:000149e8       ??_C@_0BB@EGNLBCLO@invalid?5name?5?$CFs?6?$AA@ 004d09e8     botlib:be_ai_weight.obj
 0002:000149fc       ??_C@_0BI@OGAGPDGB@switch?5without?5default?6?$AA@ 004d09fc     botlib:be_ai_weight.obj
 0002:00014a14       ??_C@_06DOPOGBGP@switch?$AA@ 004d0a14     botlib:be_ai_weight.obj
 0002:00014a1c       ??_C@_06LNOFJDNM@return?$AA@ 004d0a1c     botlib:be_ai_weight.obj
 0002:00014a24       ??_C@_04CKOINMPC@case?$AA@ 004d0a24     botlib:be_ai_weight.obj
 0002:00014a2c       ??_C@_07DLHCIBDH@default?$AA@ 004d0a2c     botlib:be_ai_weight.obj
 0002:00014a34       ??_C@_0BI@EPKIMGGL@too?5many?5fuzzy?5weights?6?$AA@ 004d0a34     botlib:be_ai_weight.obj
 0002:00014a4c       ??_C@_0CL@HHMEIDHK@weightFileList?5was?5full?5trying?5t@ 004d0a4c     botlib:be_ai_weight.obj
 0002:00014a78       ??_C@_0DA@LJPOKDON@cannot?5interbreed?5weight?5configs@ 004d0a78     botlib:be_ai_weight.obj
 0002:00014aa8       ??_C@_0DD@CNDDMNEB@cannot?5interbreed?5weight?5configs@ 004d0aa8     botlib:be_ai_weight.obj
 0002:00014adc       ??_C@_0DB@HDMANNJK@cannot?5interbreed?5weight?5configs@ 004d0adc     botlib:be_ai_weight.obj
 0002:00014b10       ??_C@_0DG@IEMEEKLE@cannot?5interbreed?5weight?5configs@ 004d0b10     botlib:be_ai_weight.obj
 0002:00014b48       ??_C@_0CI@DHABDHGE@AAS_EntityInfo?3?5entnum?5?$CFd?5out?5of@ 004d0b48     botlib:be_aas_entity.obj
 0002:00014b70       ??_C@_0CK@IABHHEBM@AAS_EntityInfo?3?5aasworld?5not?5ini@ 004d0b70     botlib:be_aas_entity.obj
 0002:00014b9c       ??_C@_0CK@DFLNBMPC@AAS_EntityOrigin?3?5entnum?5?$CFd?5out?5@ 004d0b9c     botlib:be_aas_entity.obj
 0002:00014bc8       ??_C@_0CO@GOHMBDIM@AAS_EntityModelindex?3?5entnum?5?$CFd?5@ 004d0bc8     botlib:be_aas_entity.obj
 0002:00014bf8       ??_C@_0CI@MHKPMBGB@AAS_EntityType?3?5entnum?5?$CFd?5out?5of@ 004d0bf8     botlib:be_aas_entity.obj
 0002:00014c20       ??_C@_0CM@KBCKFNEI@AAS_EntityModelNum?3?5entnum?5?$CFd?5ou@ 004d0c20     botlib:be_aas_entity.obj
 0002:00014c4c       ??_C@_0CI@PKIBPHIO@AAS_EntitySize?3?5entnum?5?$CFd?5out?5of@ 004d0c4c     botlib:be_aas_entity.obj
 0002:00014c74       ??_C@_0BO@MBNJNHCC@AAS_UpdateEntity?3?5not?5loaded?6?$AA@ 004d0c74     botlib:be_aas_entity.obj
 0002:00014c94       ??_C@_0BF@BABOLIN@rs_maxjumpfallheight?$AA@ 004d0c94     botlib:be_aas_move.obj
 0002:00014cac       ??_C@_03FMBEFOJN@450?$AA@  004d0cac     botlib:be_aas_move.obj
 0002:00014cb0       ??_C@_0BB@EFAOPOH@rs_maxfallheight?$AA@ 004d0cb0     botlib:be_aas_move.obj
 0002:00014cc4       ??_C@_0BA@EIMKLMOE@rs_falldamage10?$AA@ 004d0cc4     botlib:be_aas_move.obj
 0002:00014cd4       ??_C@_0P@DKDPFKAP@rs_falldamage5?$AA@ 004d0cd4     botlib:be_aas_move.obj
 0002:00014ce4       ??_C@_0BB@CHLHBMFH@rs_startelevator?$AA@ 004d0ce4     botlib:be_aas_move.obj
 0002:00014cf8       ??_C@_0L@EDHEJKKK@rs_funcbob?$AA@ 004d0cf8     botlib:be_aas_move.obj
 0002:00014d04       ??_C@_0BI@BFCKOPFL@rs_aircontrolledjumppad?$AA@ 004d0d04     botlib:be_aas_move.obj
 0002:00014d1c       ??_C@_0L@BDNLAFIB@rs_jumppad?$AA@ 004d0d1c     botlib:be_aas_move.obj
 0002:00014d28       ??_C@_0L@NKJOKCB@rs_bfgjump?$AA@ 004d0d28     botlib:be_aas_move.obj
 0002:00014d34       ??_C@_0O@KLDHKDPG@rs_rocketjump?$AA@ 004d0d34     botlib:be_aas_move.obj
 0002:00014d44       ??_C@_0N@DFNGJGCB@rs_startjump?$AA@ 004d0d44     botlib:be_aas_move.obj
 0002:00014d54       ??_C@_0BF@EEBNNHGL@rs_startwalkoffledge?$AA@ 004d0d54     botlib:be_aas_move.obj
 0002:00014d6c       ??_C@_02PONMODAL@70?$AA@   004d0d6c     botlib:be_aas_move.obj
 0002:00014d70       ??_C@_0BA@GKDMJAIB@rs_startgrapple?$AA@ 004d0d70     botlib:be_aas_move.obj
 0002:00014d80       ??_C@_03OCGDPLBD@500?$AA@  004d0d80     botlib:be_aas_move.obj
 0002:00014d84       ??_C@_0P@LHMFFEKL@rs_startcrouch?$AA@ 004d0d84     botlib:be_aas_move.obj
 0002:00014d94       ??_C@_03MHAIKEMP@300?$AA@  004d0d94     botlib:be_aas_move.obj
 0002:00014d98       ??_C@_0P@PHELIMLJ@rs_barrierjump?$AA@ 004d0d98     botlib:be_aas_move.obj
 0002:00014da8       ??_C@_0M@MEFOEMOE@rs_teleport?$AA@ 004d0da8     botlib:be_aas_move.obj
 0002:00014db4       ??_C@_02PNFIDHGF@50?$AA@   004d0db4     botlib:be_aas_move.obj
 0002:00014db8       ??_C@_0N@JKBBEPHH@rs_waterjump?$AA@ 004d0db8     botlib:be_aas_move.obj
 0002:00014dc8       ??_C@_0BB@HAKLBAKB@phys_falldelta10?$AA@ 004d0dc8     botlib:be_aas_move.obj
 0002:00014ddc       ??_C@_02PPBOIJDM@60?$AA@   004d0ddc     botlib:be_aas_move.obj
 0002:00014de0       ??_C@_0BA@IDFBNLKN@phys_falldelta5?$AA@ 004d0de0     botlib:be_aas_move.obj
 0002:00014df0       ??_C@_0N@CKBIGONB@phys_jumpvel?$AA@ 004d0df0     botlib:be_aas_move.obj
 0002:00014e00       ??_C@_03HKPLNFCP@270?$AA@  004d0e00     botlib:be_aas_move.obj
 0002:00014e04       ??_C@_0BA@MNKPJHJN@phys_maxbarrier?$AA@ 004d0e04     botlib:be_aas_move.obj
 0002:00014e14       ??_C@_02NCPIBIBE@33?$AA@   004d0e14     botlib:be_aas_move.obj
 0002:00014e18       ??_C@_0BC@BGLDKCMB@phys_maxwaterjump?$AA@ 004d0e18     botlib:be_aas_move.obj
 0002:00014e2c       ??_C@_0BC@JMNKLJNN@phys_maxsteepness?$AA@ 004d0e2c     botlib:be_aas_move.obj
 0002:00014e40       ??_C@_03IMEEBDJM@0?47?$AA@ 004d0e40     botlib:be_aas_move.obj
 0002:00014e44       ??_C@_0N@OLIJKDDL@phys_maxstep?$AA@ 004d0e44     botlib:be_aas_move.obj
 0002:00014e54       ??_C@_02CLJDCEPA@19?$AA@   004d0e54     botlib:be_aas_move.obj
 0002:00014e58       ??_C@_0BE@LDJBDLBF@phys_swimaccelerate?$AA@ 004d0e58     botlib:be_aas_move.obj
 0002:00014e6c       ??_C@_0BD@NNGBBLHI@phys_airaccelerate?$AA@ 004d0e6c     botlib:be_aas_move.obj
 0002:00014e80       ??_C@_0BE@FFIPDPFP@phys_walkaccelerate?$AA@ 004d0e80     botlib:be_aas_move.obj
 0002:00014e94       ??_C@_0BF@PMDEEHNA@phys_maxswimvelocity?$AA@ 004d0e94     botlib:be_aas_move.obj
 0002:00014eac       ??_C@_03GLMKKOKP@150?$AA@  004d0eac     botlib:be_aas_move.obj
 0002:00014eb0       ??_C@_0BH@IOAMOCDB@phys_maxcrouchvelocity?$AA@ 004d0eb0     botlib:be_aas_move.obj
 0002:00014ec8       ??_C@_0BF@KDOBLJFP@phys_maxwalkvelocity?$AA@ 004d0ec8     botlib:be_aas_move.obj
 0002:00014ee0       ??_C@_0BB@IJKKLCCL@phys_maxvelocity?$AA@ 004d0ee0     botlib:be_aas_move.obj
 0002:00014ef4       ??_C@_03MEIMHAKB@320?$AA@  004d0ef4     botlib:be_aas_move.obj
 0002:00014ef8       ??_C@_0BC@IMACIKDE@phys_watergravity?$AA@ 004d0ef8     botlib:be_aas_move.obj
 0002:00014f0c       ??_C@_03FKNPJMHG@400?$AA@  004d0f0c     botlib:be_aas_move.obj
 0002:00014f10       ??_C@_0BD@IPGBHKKJ@phys_waterfriction?$AA@ 004d0f10     botlib:be_aas_move.obj
 0002:00014f24       ??_C@_0N@KOBDBIMP@phys_gravity?$AA@ 004d0f24     botlib:be_aas_move.obj
 0002:00014f34       ??_C@_0P@HGIEEKKG@phys_stopspeed?$AA@ 004d0f34     botlib:be_aas_move.obj
 0002:00014f44       ??_C@_0O@KFCMEAKP@phys_friction?$AA@ 004d0f44     botlib:be_aas_move.obj
 0002:00014f54       __real@43fa0000            004d0f54     botlib:be_aas_move.obj
 0002:00014f58       __real@41b00000            004d0f58     botlib:be_aas_move.obj
 0002:00014f5c       ??_C@_0BO@BLKMJPOB@PredictMovement?3?5start?5solid?6?$AA@ 004d0f5c     botlib:be_aas_move.obj
 0002:00014f7c       __real@c3960000            004d0f7c     botlib:be_aas_move.obj
 0002:00014f80       ??_C@_0O@IMGOLFOH@leave?5ground?6?$AA@ 004d0f80     botlib:be_aas_move.obj
 0002:00014f90       ??_C@_0BE@ICPCLNOB@?$CFd?5midrange?5area?5?$CFd?$AA@ 004d0f90     botlib:be_aas_routealt.obj
 0002:00014fa4       __real@3f4ccccd            004d0fa4     botlib:be_aas_routealt.obj
 0002:00014fa8       __real@3f8ccccd            004d0fa8     botlib:be_aas_routealt.obj
 0002:00014fac       ??_C@_0BI@PLPAKMFI@?$CFd?5bytes?5routing?5cache?6?$AA@ 004d0fac     botlib:be_aas_route.obj
 0002:00014fc4       ??_C@_0BJ@FFMFFMFH@?$CFd?5portal?5cache?5updates?6?$AA@ 004d0fc4     botlib:be_aas_route.obj
 0002:00014fe0       ??_C@_0BH@IMJGLBBE@?$CFd?5area?5cache?5updates?6?$AA@ 004d0fe0     botlib:be_aas_route.obj
 0002:00014ff8       ??_C@_0DA@BGBJJEEH@AAS_EnableRoutingArea?3?5areanum?5?$CF@ 004d0ff8     botlib:be_aas_route.obj
 0002:00015028       ??_C@_0CK@NIAJBAAO@area?5?$CFd?5has?5more?5than?5128?5reacha@ 004d1028     botlib:be_aas_route.obj
 0002:00015054       __real@3fa66666            004d1054     botlib:be_aas_route.obj
 0002:00015058       ??_C@_0CD@PPPFMKKL@written?5?$CFd?5bytes?5of?5routing?5cach@ 004d1058     botlib:be_aas_route.obj
 0002:0001507c       ??_C@_0BM@DAFGPIEG@?6route?5cache?5written?5to?5?$CFs?6?$AA@ 004d107c     botlib:be_aas_route.obj
 0002:00015098       ??_C@_0BJ@HCPGIGFI@Unable?5to?5open?5file?3?5?$CFs?6?$AA@ 004d1098     botlib:be_aas_route.obj
 0002:000150b4       ??_C@_0M@FIEIFMAA@maps?1?$CFs?4rcd?$AA@ 004d10b4     botlib:be_aas_route.obj
 0002:000150c0       ??_C@_0DE@BIPEEDLP@route?5cache?5dump?5has?5wrong?5versi@ 004d10c0     botlib:be_aas_route.obj
 0002:000150f4       ??_C@_0BO@JKLJGLEA@?$CFs?5is?5not?5a?5route?5cache?5dump?6?$AA@ 004d10f4     botlib:be_aas_route.obj
 0002:00015114       ??_C@_0BB@KOMOOHGO@max_routingcache?$AA@ 004d1114     botlib:be_aas_route.obj
 0002:00015128       ??_C@_04DPPBKBGP@4096?$AA@ 004d1128     botlib:be_aas_route.obj
 0002:00015130       ??_C@_0DH@NEAPKHCH@AAS_AreaTravelTimeToGoalArea?3?5ar@ 004d1130     botlib:be_aas_route.obj
 0002:00015168       ??_C@_0DL@EBFGAMIN@AAS_AreaTravelTimeToGoalArea?3?5go@ 004d1168     botlib:be_aas_route.obj
 0002:000151a4       ??_C@_0DD@INGMKBAA@AAS_NextAreaReachability?3?5areanu@ 004d11a4     botlib:be_aas_route.obj
 0002:000151d8       ??_C@_0EB@MCKKKILC@AAS_NextAreaReachability?3?5reachn@ 004d11d8     botlib:be_aas_route.obj
 0002:0001521c       ??_C@_0CC@HHIKNNJF@area?5?$CFd?5center?5?$CFf?5?$CFf?5?$CFf?5in?5solid@ 004d121c     botlib:be_aas_route.obj
 0002:00015240       ??_C@_0BL@PJMGPMOB@AAS_CreateAllRoutingCache?6?$AA@ 004d1240     botlib:be_aas_route.obj
 0002:0001525c       ??_C@_0BL@CJDBHLDC@trigger_push?5without?5time?6?$AA@ 004d125c     botlib:be_aas_reach.obj
 0002:00015278       ??_C@_0CH@FACFDAAG@trigger_push?5without?5target?5enti@ 004d1278     botlib:be_aas_reach.obj
 0002:000152a0       ??_C@_0L@FEPNPAJD@targetname?$AA@ 004d12a0     botlib:be_aas_reach.obj
 0002:000152ac       ??_C@_06JJLAMBGK@target?$AA@ 004d12ac     botlib:be_aas_reach.obj
 0002:000152b4       ??_C@_0BK@JKILNG@trigger_push?5start?5solid?6?$AA@ 004d12b4     botlib:be_aas_reach.obj
 0002:000152d0       ??_C@_0BJ@PIPGKHBD@AAS_MAX_REACHABILITYSIZE?$AA@ 004d12d0     botlib:be_aas_reach.obj
 0002:000152ec       ??_C@_0CO@CAIPEICN@AAS_AreaReachability?3?5areanum?5?$CFd@ 004d12ec     botlib:be_aas_reach.obj
 0002:00015320       __real@41124f8000000000    004d1320     botlib:be_aas_reach.obj
 0002:00015328       __real@4049000000000000    004d1328     botlib:be_aas_reach.obj
 0002:00015330       __real@41700000            004d1330     botlib:be_aas_reach.obj
 0002:00015334       __real@43700000            004d1334     botlib:be_aas_reach.obj
 0002:00015338       __real@3f866666            004d1338     botlib:be_aas_reach.obj
 0002:0001533c       __real@3f99999a            004d133c     botlib:be_aas_reach.obj
 0002:00015340       ??_C@_0M@GAOGDGCN@bot_notteam?$AA@ 004d1340     botlib:be_aas_reach.obj
 0002:0001534c       ??_C@_0CC@HLGOOKDO@trigger_multiple?5not?5in?5any?5area@ 004d134c     botlib:be_aas_reach.obj
 0002:00015370       ??_C@_0CK@HGLAMBGC@teleported?5into?5slime?5or?5lava?5at@ 004d1370     botlib:be_aas_reach.obj
 0002:0001539c       ??_C@_05FECBCJJD@angle?$AA@ 004d139c     botlib:be_aas_reach.obj
 0002:000153a4       ??_C@_0CG@CEMGMOAN@teleporter?5destination?5?$CI?$CFs?$CJ?5in?5s@ 004d13a4     botlib:be_aas_reach.obj
 0002:000153cc       ??_C@_0CM@CLBMAOHE@teleporter?5destination?5?$CI?$CFs?$CJ?5with@ 004d13cc     botlib:be_aas_reach.obj
 0002:000153f8       ??_C@_0CO@NOOGBJFD@teleporter?5without?5misc_teleport@ 004d13f8     botlib:be_aas_reach.obj
 0002:00015428       ??_C@_0DG@PNPCBHNC@trigger_teleport?5at?5?$CF1?40f?5?$CF1?40f?5@ 004d1428     botlib:be_aas_reach.obj
 0002:00015460       ??_C@_0BP@MFGNJEFC@trigger_teleport?5model?5?$DN?5?$CC?$CFs?$CC?6?$AA@ 004d1460     botlib:be_aas_reach.obj
 0002:00015480       ??_C@_0BB@COMMHECA@trigger_teleport?$AA@ 004d1480     botlib:be_aas_reach.obj
 0002:00015494       ??_C@_0CC@NGDNGGBL@target_teleporter?5without?5target@ 004d1494     botlib:be_aas_reach.obj
 0002:000154b8       ??_C@_0BC@GJLLMIEM@target_teleporter?$AA@ 004d14b8     botlib:be_aas_reach.obj
 0002:000154cc       ??_C@_0DG@BADEBAMF@trigger_multiple?5at?5?$CF1?40f?5?$CF1?40f?5@ 004d14cc     botlib:be_aas_reach.obj
 0002:00015504       ??_C@_0BP@HIGEPBIN@trigger_multiple?5model?5?$DN?5?$CC?$CFs?$CC?6?$AA@ 004d1504     botlib:be_aas_reach.obj
 0002:00015524       ??_C@_0BB@LKHFHPEP@trigger_multiple?$AA@ 004d1524     botlib:be_aas_reach.obj
 0002:00015538       ??_C@_06LNLHEAAG@height?$AA@ 004d1538     botlib:be_aas_reach.obj
 0002:00015540       ??_C@_03MHHCOBAB@lip?$AA@  004d1540     botlib:be_aas_reach.obj
 0002:00015544       ??_C@_0CF@BDBFALFG@func_plat?5with?5invalid?5model?5num@ 004d1544     botlib:be_aas_reach.obj
 0002:0001556c       ??_C@_0BJ@LDMJPEKH@func_plat?5without?5model?6?$AA@ 004d156c     botlib:be_aas_reach.obj
 0002:00015588       __real@43000000            004d1588     botlib:be_aas_reach.obj
 0002:0001558c       __real@43400000            004d158c     botlib:be_aas_reach.obj
 0002:00015590       ??_C@_0CC@PCNLLMDF@funcbob?5reach?5from?5area?5?$CFd?5to?5?$CFd@ 004d1590     botlib:be_aas_reach.obj
 0002:000155b8       ??_C@_0EN@JGFDJKIH@funcbob?5model?5?$CFd?0?5start?5?$DN?5?$HL?$CF1?41f@ 004d15b8     botlib:be_aas_reach.obj
 0002:00015608       ??_C@_0CI@BJOEBEBE@func_bobbing?5with?5invalid?5model?5@ 004d1608     botlib:be_aas_reach.obj
 0002:00015630       ??_C@_0BM@HGBLGKHA@func_bobbing?5without?5model?6?$AA@ 004d1630     botlib:be_aas_reach.obj
 0002:00015650       __real@4059000000000000    004d1650     botlib:be_aas_reach.obj
 0002:00015658       ??_C@_0CN@NDLDAEHG@found?5a?5trigger_push?5with?5veloci@ 004d1658     botlib:be_aas_reach.obj
 0002:00015688       ??_C@_0CH@EKLAGLOI@trigger_push?5not?5in?5any?5jump?5pad@ 004d1688     botlib:be_aas_reach.obj
 0002:000156b0       ??_C@_0N@CCJDLJOF@trigger_push?$AA@ 004d16b0     botlib:be_aas_reach.obj
 0002:000156c0       __real@3fd0c15240000000    004d16c0     botlib:be_aas_reach.obj
 0002:000156c8       __real@44fa0000            004d16c8     botlib:be_aas_reach.obj
 0002:000156cc       ??_C@_0CE@GGDNMGF@area?5?$CFd?5center?5?$CFf?5?$CFf?5?$CFf?5in?5solid@ 004d16cc     botlib:be_aas_reach.obj
 0002:000156f0       __real@3eaaaaab            004d16f0     botlib:be_aas_reach.obj
 0002:000156f4       ??_C@_0CH@PFPOMNKK@AAS_BestReachableArea?3?5aas?5not?5l@ 004d16f4     botlib:be_aas_reach.obj
 0002:0001571c       __real@47c34f80            004d171c     botlib:be_aas_reach.obj
 0002:00015720       ??_C@_0BG@HCGBEFOB@?$CFd?5weapon?5jump?5areas?6?$AA@ 004d1720     botlib:be_aas_reach.obj
 0002:00015738       ??_C@_0BF@ILDMGFED@item_invulnerability?$AA@ 004d1738     botlib:be_aas_reach.obj
 0002:00015750       ??_C@_0L@MMGPPPDM@item_regen?$AA@ 004d1750     botlib:be_aas_reach.obj
 0002:0001575c       ??_C@_09MDKNIFFH@item_quad?$AA@ 004d175c     botlib:be_aas_reach.obj
 0002:00015768       ??_C@_0L@JBGNLNGG@weapon_bfg?$AA@ 004d1768     botlib:be_aas_reach.obj
 0002:00015774       ??_C@_0P@FEPBKEBF@weapon_railgun?$AA@ 004d1774     botlib:be_aas_reach.obj
 0002:00015784       ??_C@_0BB@LBHAKENA@weapon_plasmagun?$AA@ 004d1784     botlib:be_aas_reach.obj
 0002:00015798       ??_C@_0BB@OCCEAFCD@weapon_lightning?$AA@ 004d1798     botlib:be_aas_reach.obj
 0002:000157ac       ??_C@_0BG@HJKONAJE@weapon_rocketlauncher?$AA@ 004d17ac     botlib:be_aas_reach.obj
 0002:000157c4       ??_C@_0BH@DGCCJPLM@weapon_grenadelauncher?$AA@ 004d17c4     botlib:be_aas_reach.obj
 0002:000157dc       ??_C@_0BB@PBGAONGH@item_health_mega?$AA@ 004d17dc     botlib:be_aas_reach.obj
 0002:000157f0       ??_C@_0BC@FPPLPJIL@item_armor_combat?$AA@ 004d17f0     botlib:be_aas_reach.obj
 0002:00015804       ??_C@_0BA@EKKMHIH@item_armor_body?$AA@ 004d1804     botlib:be_aas_reach.obj
 0002:00015814       ??_C@_0BJ@MGEPEAF@calculating?5clusters?4?4?4?6?$AA@ 004d1814     botlib:be_aas_reach.obj
 0002:00015830       ??_C@_0CM@JBJKNNFH@?6please?5wait?5while?5storing?5reach@ 004d1830     botlib:be_aas_reach.obj
 0002:0001585c       ??_C@_08PLEDPJBP@?$AN?$CF6?41f?$CF?$CF?$AA@ 004d185c     botlib:be_aas_reach.obj
 0002:00015868       ??_C@_0BN@PENKEBEJ@calculating?5reachability?4?4?4?6?$AA@ 004d1868     botlib:be_aas_reach.obj
 0002:00015888       ??_C@_0N@PBBHPDFE@grapplereach?$AA@ 004d1888     botlib:be_aas_reach.obj
 0002:00015898       ??_C@_0BC@HJNNPMHF@forcereachability?$AA@ 004d1898     botlib:be_aas_reach.obj
 0002:000158ac       ??_C@_0BJ@JBOKGNLE@bsp?5entity?5out?5of?5range?6?$AA@ 004d18ac     botlib:be_aas_bspq3.obj
 0002:000158c8       ??_C@_0M@HBEEPJK@?$CFlf?5?$CFlf?5?$CFlf?$AA@ 004d18c8     botlib:be_aas_bspq3.obj
 0002:000158d4       ??_C@_0L@MIANKDAD@missing?5?$HN?6?$AA@ 004d18d4     botlib:be_aas_bspq3.obj
 0002:000158e0       ??_C@_0M@HDEGANAK@invalid?5?$CFs?6?$AA@ 004d18e0     botlib:be_aas_bspq3.obj
 0002:000158ec       ??_C@_0BP@POHMEOEC@too?5many?5entities?5in?5BSP?5file?6?$AA@ 004d18ec     botlib:be_aas_bspq3.obj
 0002:0001590c       ??_C@_07IJNKCNKH@entdata?$AA@ 004d190c     botlib:be_aas_bspq3.obj
 0002:00015914       ??_C@_0DE@DAMFACPE@AAS_PresenceTypeBoundingBox?3?5unk@ 004d1914     botlib:be_aas_sample.obj
 0002:00015948       ??_C@_0N@PMPJOGOE@max_aaslinks?$AA@ 004d1948     botlib:be_aas_sample.obj
 0002:00015958       ??_C@_04MHGDGELL@6144?$AA@ 004d1958     botlib:be_aas_sample.obj
 0002:00015960       ??_C@_0BF@KNNPFKDB@empty?5aas?5link?5heap?6?$AA@ 004d1960     botlib:be_aas_sample.obj
 0002:00015978       ??_C@_0CC@DPIPPCFJ@AAS_PointAreaNum?3?5aas?5not?5loaded@ 004d1978     botlib:be_aas_sample.obj
 0002:0001599c       ??_C@_0CG@BJGNCCMO@AAS_AreaCluster?3?5invalid?5area?5nu@ 004d199c     botlib:be_aas_sample.obj
 0002:000159c4       ??_C@_0CL@HEHPOKDE@AAS_AreaPresenceType?3?5invalid?5ar@ 004d19c4     botlib:be_aas_sample.obj
 0002:000159f0       __real@bf50624dd2f1a9fc    004d19f0     botlib:be_aas_sample.obj
 0002:000159f8       ??_C@_0CG@KBEHGJIJ@AAS_TraceBoundingBox?3?5stack?5over@ 004d19f8     botlib:be_aas_sample.obj
 0002:00015a20       __real@3f7fbe77            004d1a20     botlib:be_aas_sample.obj
 0002:00015a24       ??_C@_0CA@MKOIMAGJ@AAS_TraceAreas?3?5stack?5overflow?6?$AA@ 004d1a24     botlib:be_aas_sample.obj
 0002:00015a44       ??_C@_0CA@CLALHCAJ@AAS_LinkEntity?3?5stack?5overflow?6?$AA@ 004d1a44     botlib:be_aas_sample.obj
 0002:00015a64       ??_C@_0CA@PMAJPFFP@AAS_LinkEntity?3?5aas?5not?5loaded?6?$AA@ 004d1a64     botlib:be_aas_sample.obj
 0002:00015a84       ??_C@_0CH@FGLCKOMK@AAS_AreaInfo?3?5areanum?5?$CFd?5out?5of?5@ 004d1a84     botlib:be_aas_sample.obj
 0002:00015aac       ??_C@_0DF@LNJENCAM@GeneticParentsAndChildSelection?3@ 004d1aac     botlib:be_ai_gen.obj
 0002:00015ae4       ??_C@_0DA@GJMCOLIK@GeneticParentsAndChildSelection?3@ 004d1ae4     botlib:be_ai_gen.obj
 0002:00015b14       ??_C@_01EPMOAMKG@$?$AA@    004d1b14     botlib:l_script.obj
 0002:00015b18       ??_C@_01IPJKGB@?$CD?$AA@   004d1b18     botlib:l_script.obj
 0002:00015b1c       ??_C@_01OGPIMHDM@?$DP?$AA@ 004d1b1c     botlib:l_script.obj
 0002:00015b20       ??_C@_01PJKLJHI@?$HO?$AA@  004d1b20     botlib:l_script.obj
 0002:00015b24       ??_C@_01JKBOJNNK@?$FO?$AA@ 004d1b24     botlib:l_script.obj
 0002:00015b28       ??_C@_01MIFGBAGJ@?$CL?$AA@ 004d1b28     botlib:l_script.obj
 0002:00015b2c       ??_C@_01FGNFDNOH@?$CF?$AA@ 004d1b2c     botlib:l_script.obj
 0002:00015b30       ??_C@_01NBENCBCI@?$CK?$AA@ 004d1b30     botlib:l_script.obj
 0002:00015b34       ??_C@_02FNAGIBCP@?4?$CK?$AA@ 004d1b34     botlib:l_script.obj
 0002:00015b38       ??_C@_02HBOOOICD@?9?$DO?$AA@ 004d1b38     botlib:l_script.obj
 0002:00015b3c       ??_C@_02FODMEDOG@?$DM?$DM?$AA@ 004d1b3c     botlib:l_script.obj
 0002:00015b40       ??_C@_02GPIOPFAK@?$DO?$DO?$AA@ 004d1b40     botlib:l_script.obj
 0002:00015b44       ??_C@_02MHEGNOJ@?$FO?$DN?$AA@ 004d1b44     botlib:l_script.obj
 0002:00015b48       ??_C@_02DHLNPPGH@?$HM?$DN?$AA@ 004d1b48     botlib:l_script.obj
 0002:00015b4c       ??_C@_02FGJGFEAB@?$CG?$DN?$AA@ 004d1b4c     botlib:l_script.obj
 0002:00015b50       ??_C@_02BAABKJLB@?9?9?$AA@ 004d1b50     botlib:l_script.obj
 0002:00015b54       ??_C@_02ECNGHCIF@?$CL?$CL?$AA@ 004d1b54     botlib:l_script.obj
 0002:00015b58       ??_C@_02FKMDLLOA@?9?$DN?$AA@ 004d1b58     botlib:l_script.obj
 0002:00015b5c       ??_C@_02FOEOMHFC@?$CL?$DN?$AA@ 004d1b5c     botlib:l_script.obj
 0002:00015b60       ??_C@_02FENAOKFI@?$CF?$DN?$AA@ 004d1b60     botlib:l_script.obj
 0002:00015b64       ??_C@_02FJEHGPIO@?1?$DN?$AA@ 004d1b64     botlib:l_script.obj
 0002:00015b68       ??_C@_02FPIMKNGF@?$CK?$DN?$AA@ 004d1b68     botlib:l_script.obj
 0002:00015b6c       ??_C@_02FDNJECIE@?$CB?$DN?$AA@ 004d1b6c     botlib:l_script.obj
 0002:00015b70       ??_C@_02EGOFBIJA@?$DN?$DN?$AA@ 004d1b70     botlib:l_script.obj
 0002:00015b74       ??_C@_02EHCHHCKH@?$DM?$DN?$AA@ 004d1b74     botlib:l_script.obj
 0002:00015b78       ??_C@_02EEKDKGMJ@?$DO?$DN?$AA@ 004d1b78     botlib:l_script.obj
 0002:00015b7c       ??_C@_02NONPIBCD@?$HM?$HM?$AA@ 004d1b7c     botlib:l_script.obj
 0002:00015b80       ??_C@_02PPKAJPJL@?$CG?$CG?$AA@ 004d1b80     botlib:l_script.obj
 0002:00015b84       ??_C@_03CDNPDDLA@?$DM?$DM?$DN?$AA@ 004d1b84     botlib:l_script.obj
 0002:00015b88       ??_C@_03IKFCCPFF@?$DO?$DO?$DN?$AA@ 004d1b88     botlib:l_script.obj
 0002:00015b8c       ??_C@_0BD@CDGAFDMK@unkown?5punctuation?$AA@ 004d1b8c     botlib:l_script.obj
 0002:00015ba0       ??_C@_0CE@DDEEFDJP@too?5large?5value?5in?5escape?5charac@ 004d1ba0     botlib:l_script.obj
 0002:00015bc4       ??_C@_0BE@LNBHEDIG@unknown?5escape?5char?$AA@ 004d1bc4     botlib:l_script.obj
 0002:00015bd8       ??_C@_0BJ@FPJNGGBK@newline?5inside?5string?5?$CFs?$AA@ 004d1bd8     botlib:l_script.obj
 0002:00015bf4       ??_C@_0BH@PEPCDKK@missing?5trailing?5quote?$AA@ 004d1bf4     botlib:l_script.obj
 0002:00015c0c       ??_C@_0CC@MBLDNBAM@string?5longer?5than?5MAX_TOKEN?5?$DN?5?$CF@ 004d1c0c     botlib:l_script.obj
 0002:00015c30       ??_C@_0CA@MNDCIFOG@name?5longer?5than?5MAX_TOKEN?5?$DN?5?$CFd?$AA@ 004d1c30     botlib:l_script.obj
 0002:00015c50       __real@41f0000000000000    004d1c50     botlib:l_script.obj
 0002:00015c58       ??_C@_0CC@HHKGPIHJ@number?5longer?5than?5MAX_TOKEN?5?$DN?5?$CF@ 004d1c58     botlib:l_script.obj
 0002:00015c7c       ??_C@_0CJ@GOJFKF@binary?5number?5longer?5than?5MAX_TO@ 004d1c7c     botlib:l_script.obj
 0002:00015ca8       ??_C@_0CO@IEAAEMOC@hexadecimal?5number?5longer?5than?5M@ 004d1ca8     botlib:l_script.obj
 0002:00015cd8       ??_C@_0CI@KHNHEENA@too?5many?5characters?5in?5literal?0?5@ 004d1cd8     botlib:l_script.obj
 0002:00015d00       ??_C@_0BO@LNDMFPAB@end?5of?5file?5before?5trailing?5?8?$AA@ 004d1d00     botlib:l_script.obj
 0002:00015d20       ??_C@_0CL@IOHHDOB@primitive?5token?5longer?5than?5MAX_@ 004d1d20     botlib:l_script.obj
 0002:00015d4c       ??_C@_0BB@HHMOOKCN@can?8t?5read?5token?$AA@ 004d1d4c     botlib:l_script.obj
 0002:00015d60       ??_C@_0BP@BHDDOFIL@BUG?3?5wrong?5punctuation?5subtype?$AA@ 004d1d60     botlib:l_script.obj
 0002:00015d80       ??_C@_0CA@NFDKBKI@expected?5float?5value?0?5found?5?$CFs?6?$AA@ 004d1d80     botlib:l_script.obj
 0002:00015da0       __real@bff0000000000000    004d1da0     botlib:l_script.obj
 0002:00015da8       ??_C@_0CC@CKEDEGB@expected?5integer?5value?0?5found?5?$CFs@ 004d1da8     botlib:l_script.obj
 0002:00015dcc       ??_C@_05GFOLEBJA@?$CFs?1?$CFs?$AA@ 004d1dcc     botlib:l_script.obj
 0002:00015dd4       ??_C@_0BP@CBDFEHDO@value?5?$CFd?5out?5of?5range?5?$FL?$CFd?0?5?$CFd?$FN?$AA@ 004d1dd4     botlib:l_struct.obj
 0002:00015df4       ??_C@_0BP@LFCOICHJ@value?5?$CFd?5out?5of?5range?5?$FL?$CFf?0?5?$CFf?$FN?$AA@ 004d1df4     botlib:l_struct.obj
 0002:00015e14       ??_C@_0BM@MDDDOOGF@float?5out?5of?5range?5?$FL?$CFf?0?5?$CFf?$FN?$AA@ 004d1e14     botlib:l_struct.obj
 0002:00015e30       ??_C@_0BB@EFFDGMEA@unexpected?5float?$AA@ 004d1e30     botlib:l_struct.obj
 0002:00015e44       ??_C@_0BK@IFJFBCJ@expected?5number?0?5found?5?$CFs?$AA@ 004d1e44     botlib:l_struct.obj
 0002:00015e60       ??_C@_0BK@KDOFCJEJ@unexpected?5punctuation?5?$CFs?$AA@ 004d1e60     botlib:l_struct.obj
 0002:00015e7c       ??_C@_0CC@POKHHIP@expected?5unsigned?5value?0?5found?5?$CF@ 004d1e7c     botlib:l_struct.obj
 0002:00015ea0       ??_C@_0BL@DCLIMJHG@expected?5a?5comma?0?5found?5?$CFs?$AA@ 004d1ea0     botlib:l_struct.obj
 0002:00015ebc       ??_C@_0BO@KOGKDPOB@BUG?3?5no?5sub?5structure?5defined?$AA@ 004d1ebc     botlib:l_struct.obj
 0002:00015edc       ??_C@_0BL@GLPBJIMC@unknown?5structure?5field?5?$CFs?$AA@ 004d1edc     botlib:l_struct.obj
 0002:00015ef8       ??_C@_01GPOEFGEJ@?7?$AA@   004d1ef8     botlib:l_struct.obj
 0002:00015efc       ??_C@_03LFNJCDHL@?$HN?$AN?6?$AA@ 004d1efc     botlib:l_struct.obj
 0002:00015f00       ??_C@_03MOCCBCKP@?$CFs?7?$AA@ 004d1f00     botlib:l_struct.obj
 0002:00015f04       ??_C@_03JALCHMKH@?$HL?$AN?6?$AA@ 004d1f04     botlib:l_struct.obj
 0002:00015f08       ??_C@_0BI@DBJMMGKJ@can?8t?5seek?5to?5aas?5lump?6?$AA@ 004d1f08     botlib:be_aas_file.obj
 0002:00015f20       ??_C@_0CA@GEEFHEDJ@AAS?5file?5not?5sequentially?5read?6?$AA@ 004d1f20     botlib:be_aas_file.obj
 0002:00015f40       ??_C@_0BM@NDIFACPH@aas?5file?5?$CFs?5is?5out?5of?5date?6?$AA@ 004d1f40     botlib:be_aas_file.obj
 0002:00015f5c       ??_C@_0CD@IPFFEFDG@aas?5file?5?$CFs?5is?5version?5?$CFi?0?5not?5?$CF@ 004d1f5c     botlib:be_aas_file.obj
 0002:00015f80       ??_C@_0BH@HDNIDKDF@?$CFs?5is?5not?5an?5AAS?5file?6?$AA@ 004d1f80     botlib:be_aas_file.obj
 0002:00015f98       ??_C@_0P@MNCIOHOD@can?8t?5open?5?$CFs?6?$AA@ 004d1f98     botlib:be_aas_file.obj
 0002:00015fa8       ??_C@_0BD@DAIGMAGG@trying?5to?5load?5?$CFs?6?$AA@ 004d1fa8     botlib:be_aas_file.obj
 0002:00015fbc       ??_C@_0BC@CBHACCGB@error?5opening?5?$CFs?6?$AA@ 004d1fbc     botlib:be_aas_file.obj
 0002:00015fd0       ??_C@_0M@JKCPKPL@writing?5?$CFs?6?$AA@ 004d1fd0     botlib:be_aas_file.obj
 0002:00015fdc       ??_C@_0BF@OFBIEKCH@AAS?5data?5optimized?4?6?$AA@ 004d1fdc     botlib:be_aas_optimize.obj
 0002:00015ff4       ??_C@_0DG@OCGFOOPH@portal?5area?5?$CFd?5is?5seperating?5mor@ 004d1ff4     botlib:be_aas_cluster.obj
 0002:0001602c       ??_C@_0BI@KOKCMCHN@AAS_MAX_PORTALINDEXSIZE?$AA@ 004d202c     botlib:be_aas_cluster.obj
 0002:00016044       ??_C@_0BF@NHJNBHCO@no?5portal?5of?5area?5?$CFd?$AA@ 004d2044     botlib:be_aas_cluster.obj
 0002:0001605c       ??_C@_0CO@OFKPJKFO@AAS_FloodClusterAreas_r?3?5areanum@ 004d205c     botlib:be_aas_cluster.obj
 0002:0001608c       ??_C@_0CL@KPDIAOMF@cluster?5?$CFd?5touched?5cluster?5?$CFd?5at@ 004d208c     botlib:be_aas_cluster.obj
 0002:000160b8       ??_C@_0BB@KELFLMDE@AAS_MAX_CLUSTERS?$AA@ 004d20b8     botlib:be_aas_cluster.obj
 0002:000160cc       ??_C@_0BA@ILOODELG@AAS_MAX_PORTALS?$AA@ 004d20cc     botlib:be_aas_cluster.obj
 0002:000160dc       ??_C@_0BA@DKADLPCK@MAX_PORTALAREAS?$AA@ 004d20dc     botlib:be_aas_cluster.obj
 0002:000160ec       ??_C@_0BG@IDPPIMFG@possible?5portal?3?5?$CFd?$AN?6?$AA@ 004d20ec     botlib:be_aas_cluster.obj
 0002:00016104       ??_C@_0BM@COFAHJCM@?$AN?$CF6d?5possible?5portal?5areas?6?$AA@ 004d2104     botlib:be_aas_cluster.obj
 0002:00016120       ??_C@_0CF@HNGHLOBA@portal?5area?5?$CFd?5has?5no?5back?5clust@ 004d2120     botlib:be_aas_cluster.obj
 0002:00016148       ??_C@_0CG@PPPPLOAP@portal?5area?5?$CFd?5has?5no?5front?5clus@ 004d2148     botlib:be_aas_cluster.obj
 0002:00016170       ??_C@_0BJ@EOFLMLFD@?$CF6d?5forced?5portal?5areas?6?$AA@ 004d2170     botlib:be_aas_cluster.obj
 0002:0001618c       ??_C@_0CC@ECEDAPMJ@area?5?$CFd?5is?5a?5forced?5portal?5area?$AN@ 004d218c     botlib:be_aas_cluster.obj
 0002:000161b0       ??_C@_0DB@NFDNPBEJ@?$CF6i?5AAS?5memory?1CPU?5usage?5?$CIthe?5lo@ 004d21b0     botlib:be_aas_cluster.obj
 0002:000161e4       ??_C@_0BO@NNGLPCLI@?$CF6i?5total?5reachability?5areas?6?$AA@ 004d21e4     botlib:be_aas_cluster.obj
 0002:00016204       ??_C@_0CG@PPPOPFBK@cluster?5?$CFd?5has?5?$CFd?5reachability?5a@ 004d2204     botlib:be_aas_cluster.obj
 0002:0001622c       ??_C@_0BG@IEMHKDCK@?$CF6d?5clusters?5created?6?$AA@ 004d222c     botlib:be_aas_cluster.obj
 0002:00016244       ??_C@_0BF@HJCLOJDI@?$CF6d?5portals?5created?6?$AA@ 004d2244     botlib:be_aas_cluster.obj
 0002:0001625c       ??_C@_0BF@LLJPMAL@portal?5?$CFd?3?5area?5?$CFd?$AN?6?$AA@ 004d225c     botlib:be_aas_cluster.obj
 0002:00016274       ??_C@_04HHNGKENO@?$AN?$CF6d?$AA@ 004d2274     botlib:be_aas_cluster.obj
 0002:0001627c       ??_C@_0BK@CDJHMKCM@?$AN?$CF6d?5removed?5portal?5areas?$AA@ 004d227c     botlib:be_aas_cluster.obj
 0002:00016298       ??_C@_0BA@BADKHCEE@forceclustering?$AA@ 004d2298     botlib:be_aas_cluster.obj
 0002:000162a8       ??_C@_0BJ@MGMOCNCM@edgenum?5?$CFd?5out?5of?5range?6?$AA@ 004d22a8     botlib:be_aas_debug.obj
 0002:000162c4       ??_C@_0BJ@BLFMMBJE@facenum?5?$CFd?5out?5of?5range?6?$AA@ 004d22c4     botlib:be_aas_debug.obj
 0002:000162e0       ??_C@_0BO@EKJMENEL@area?5?$CFd?5out?5of?5range?5?$FL0?0?5?$CFd?$FN?6?$AA@ 004d22e0     botlib:be_aas_debug.obj
 0002:00016300       __real@3ff8000000000000    004d2300     botlib:be_aas_debug.obj
 0002:000163b0       ??_C@_0P@MIGLKIOC@CorExitProcess?$AA@ 004d23b0     LIBC:crt0dat.obj
 0002:000163c0       ??_C@_0M@MBOPBNBK@mscoree?4dll?$AA@ 004d23c0     LIBC:crt0dat.obj
 0002:000163dc       ??_C@_05KLBDPFGC@e?$CL000?$AA@ 004d23dc     LIBC:cvt.obj
 0002:000163e8       __real@4150017ec0000000    004d23e8     LIBC:testfdiv.obj
 0002:000163f0       __real@4147ffff80000000    004d23f0     LIBC:testfdiv.obj
 0002:000163f8       ??_C@_0BK@NHEOCAHP@IsProcessorFeaturePresent?$AA@ 004d23f8     LIBC:testfdiv.obj
 0002:00016414       ??_C@_08CPNIBGIE@KERNEL32?$AA@ 004d2414     LIBC:testfdiv.obj
 0002:00016488       ??_C@_04MLLJIGOK@atan?$AA@ 004d2488     LIBC:libm_error.obj
 0002:00016490       ??_C@_04GFPJNGEK@ceil?$AA@ 004d2490     LIBC:libm_error.obj
 0002:00016498       ??_C@_05PBJFFIGL@floor?$AA@ 004d2498     LIBC:libm_error.obj
 0002:000164a0       ??_C@_04EHEDPDJG@modf?$AA@ 004d24a0     LIBC:libm_error.obj
 0002:000164a8       ??_C@_04HPAFEEIN@exp2?$AA@ 004d24a8     LIBC:libm_error.obj
 0002:000164b0       ??_C@_05EOHGHCHD@exp10?$AA@ 004d24b0     LIBC:libm_error.obj
 0002:000164b8       ??_C@_04KGLCPMCP@log2?$AA@ 004d24b8     LIBC:libm_error.obj
 0002:000164c0       ??_C@_03JGHBODFD@pow?$AA@  004d24c0     LIBC:libm_error.obj
 0002:000164c4       ??_C@_05HGHHAHAP@log10?$AA@ 004d24c4     LIBC:libm_error.obj
 0002:000164cc       ??_C@_03KHJOGHMM@exp?$AA@  004d24cc     LIBC:libm_error.obj
 0002:000164dc       ??_C@_0N@FFJGBINN@AuthenticAMD?$AA@ 004d24dc     LIBC:cpu_disp.obj
 0002:000164ec       ??_C@_13NOLLCAOD@?$AA?$AA?$AA?$AA@ 004d24ec     LIBC:a_map.obj
 0002:00016518       ___newctype                004d2518     LIBC:ctype.obj
 0002:00016818       __wctype                   004d2818     LIBC:ctype.obj
 0002:00016a20       ___lookuptable             004d2a20     LIBC:output.obj
 0002:00016a7c       ??_C@_1O@CEDCILHN@?$AA?$CI?$AAn?$AAu?$AAl?$AAl?$AA?$CJ?$AA?$AA@ 004d2a7c     LIBC:output.obj
 0002:00016a8c       ??_C@_06OJHGLDPL@?$CInull?$CJ?$AA@ 004d2a8c     LIBC:output.obj
 0002:00016aa4       ___dnames                  004d2aa4     LIBC:timeset.obj
 0002:00016abc       ___mnames                  004d2abc     LIBC:timeset.obj
 0002:00016ae4       ??_C@_02CLFPBFFP@TZ?$AA@   004d2ae4     LIBC:tzset.obj
 0002:00016af8       __DEFAULT_CW_in_mem        004d2af8     LIBC:common.obj
 0002:00016afa       __pi_by_2_to_61            004d2afa     LIBC:common.obj
 0002:00016b74       ??_C@_0P@GGKDKEEG@runtime?5error?5?$AA@ 004d2b74     LIBC:crt0msg.obj
 0002:00016b84       ??_C@_0O@MJNIPGOH@TLOSS?5error?$AN?6?$AA@ 004d2b84     LIBC:crt0msg.obj
 0002:00016b94       ??_C@_0N@BONNPDHF@SING?5error?$AN?6?$AA@ 004d2b94     LIBC:crt0msg.obj
 0002:00016ba4       ??_C@_0P@MBDAJNE@DOMAIN?5error?$AN?6?$AA@ 004d2ba4     LIBC:crt0msg.obj
 0002:00016bb8       ??_C@_0KC@BDDGGBEJ@R6029?$AN?6?9?5This?5application?5cannot@ 004d2bb8     LIBC:crt0msg.obj
 0002:00016c5c       ??_C@_0CF@KJDAIALP@R6028?$AN?6?9?5unable?5to?5initialize?5he@ 004d2c5c     LIBC:crt0msg.obj
 0002:00016c84       ??_C@_0DF@GAKBPDFP@R6027?$AN?6?9?5not?5enough?5space?5for?5lo@ 004d2c84     LIBC:crt0msg.obj
 0002:00016cbc       ??_C@_0DF@IBLNNAIG@R6026?$AN?6?9?5not?5enough?5space?5for?5st@ 004d2cbc     LIBC:crt0msg.obj
 0002:00016cf4       ??_C@_0CG@IOHKGFNJ@R6025?$AN?6?9?5pure?5virtual?5function?5c@ 004d2cf4     LIBC:crt0msg.obj
 0002:00016d1c       ??_C@_0DF@JIJJFJDC@R6024?$AN?6?9?5not?5enough?5space?5for?5_o@ 004d2d1c     LIBC:crt0msg.obj
 0002:00016d54       ??_C@_0CJ@EGEJHFME@R6019?$AN?6?9?5unable?5to?5open?5console?5@ 004d2d54     LIBC:crt0msg.obj
 0002:00016d80       ??_C@_0CB@GNHNIELH@R6018?$AN?6?9?5unexpected?5heap?5error?$AN?6@ 004d2d80     LIBC:crt0msg.obj
 0002:00016da4       ??_C@_0CN@FOLDKNG@R6017?$AN?6?9?5unexpected?5multithread?5@ 004d2da4     LIBC:crt0msg.obj
 0002:00016dd4       ??_C@_0CM@FAHFJNHO@R6016?$AN?6?9?5not?5enough?5space?5for?5th@ 004d2dd4     LIBC:crt0msg.obj
 0002:00016e00       ??_C@_0JG@LBKMGKLD@?$AN?6This?5application?5has?5requested@ 004d2e00     LIBC:crt0msg.obj
 0002:00016e98       ??_C@_0CM@FLCNIPKK@R6009?$AN?6?9?5not?5enough?5space?5for?5en@ 004d2e98     LIBC:crt0msg.obj
 0002:00016ec4       ??_C@_0CK@KMMJOAPP@R6008?$AN?6?9?5not?5enough?5space?5for?5ar@ 004d2ec4     LIBC:crt0msg.obj
 0002:00016ef0       ??_C@_0CF@HOHMHDEK@R6002?$AN?6?9?5floating?5point?5not?5load@ 004d2ef0     LIBC:crt0msg.obj
 0002:00016f18       ??_C@_0CF@GOGNBNAK@Microsoft?5Visual?5C?$CL?$CL?5Runtime?5Lib@ 004d2f18     LIBC:crt0msg.obj
 0002:00016f40       ??_C@_02PHMGELLB@?6?6?$AA@ 004d2f40     LIBC:crt0msg.obj
 0002:00016f44       ??_C@_0BK@OFGJDLJJ@Runtime?5Error?$CB?6?6Program?3?5?$AA@ 004d2f44     LIBC:crt0msg.obj
 0002:00016f60       ??_C@_0BH@DNAGHKFM@?$DMprogram?5name?5unknown?$DO?$AA@ 004d2f60     LIBC:crt0msg.obj
 0002:0001a8bc       ??_C@_0L@KDOEJCKC@_nextafter?$AA@ 004d68bc     LIBC:fpexcept.obj
 0002:0001a8c8       ??_C@_05JGDBENOH@_logb?$AA@ 004d68c8     LIBC:fpexcept.obj
 0002:0001a8d0       ??_C@_03ONILCKOB@_yn?$AA@  004d68d0     LIBC:fpexcept.obj
 0002:0001a8d4       ??_C@_03NAKIGLHK@_y1?$AA@  004d68d4     LIBC:fpexcept.obj
 0002:0001a8d8       ??_C@_03MJLDFKDL@_y0?$AA@  004d68d8     LIBC:fpexcept.obj
 0002:0001a8dc       ??_C@_05GKKHEGJL@frexp?$AA@ 004d68dc     LIBC:fpexcept.obj
 0002:0001a8e4       ??_C@_04KEPJIHGP@fmod?$AA@ 004d68e4     LIBC:fpexcept.obj
 0002:0001a8ec       ??_C@_06MEIMCGCF@_hypot?$AA@ 004d68ec     LIBC:fpexcept.obj
 0002:0001a8f4       ??_C@_05KBKMEMPO@_cabs?$AA@ 004d68f4     LIBC:fpexcept.obj
 0002:0001a8fc       ??_C@_05CEJMAHNP@ldexp?$AA@ 004d68fc     LIBC:fpexcept.obj
 0002:0001a904       ??_C@_04ODHECPBC@fabs?$AA@ 004d6904     LIBC:fpexcept.obj
 0002:0001a90c       ??_C@_03IIINPABG@tan?$AA@  004d690c     LIBC:fpexcept.obj
 0002:0001a910       ??_C@_03LALBNOCG@cos?$AA@  004d6910     LIBC:fpexcept.obj
 0002:0001a914       ??_C@_04EIAKFFMI@sqrt?$AA@ 004d6914     LIBC:fpexcept.obj
 0002:0001a91c       ??_C@_05KNGEOGJB@atan2?$AA@ 004d691c     LIBC:fpexcept.obj
 0002:0001a924       ??_C@_04PDIFKINK@acos?$AA@ 004d6924     LIBC:fpexcept.obj
 0002:0001a92c       ??_C@_04FIHNOPOL@asin?$AA@ 004d692c     LIBC:fpexcept.obj
 0002:0001a934       ??_C@_04FJHINJAO@tanh?$AA@ 004d6934     LIBC:fpexcept.obj
 0002:0001a93c       ??_C@_04HPJJNFIM@cosh?$AA@ 004d693c     LIBC:fpexcept.obj
 0002:0001a944       ??_C@_04COOMCNPB@sinh?$AA@ 004d6944     LIBC:fpexcept.obj
 0002:0001a978       ??_C@_09KLGCKDOD@Program?3?5?$AA@ 004d6978     LIBC:secfail.obj
 0002:0001a988       ??_C@_0KA@JEHFIFGP@A?5buffer?5overrun?5has?5been?5detect@ 004d6988     LIBC:secfail.obj
 0002:0001aa28       ??_C@_0BJ@MDEKIEOJ@Buffer?5overrun?5detected?$CB?$AA@ 004d6a28     LIBC:secfail.obj
 0002:0001aa48       ??_C@_0LB@BPLHHLFD@A?5security?5error?5of?5unknown?5caus@ 004d6a48     LIBC:secfail.obj
 0002:0001aafc       ??_C@_0CD@GMKACBEK@Unknown?5security?5failure?5detecte@ 004d6afc     LIBC:secfail.obj
 0002:0001ab2c       ??_C@_0BI@DFKBFLJE@GetProcessWindowStation?$AA@ 004d6b2c     LIBC:crtmbox.obj
 0002:0001ab44       ??_C@_0BK@CIDNPOGP@GetUserObjectInformationA?$AA@ 004d6b44     LIBC:crtmbox.obj
 0002:0001ab60       ??_C@_0BD@HHGDFDBJ@GetLastActivePopup?$AA@ 004d6b60     LIBC:crtmbox.obj
 0002:0001ab74       ??_C@_0BA@HNOPNCHB@GetActiveWindow?$AA@ 004d6b74     LIBC:crtmbox.obj
 0002:0001ab84       ??_C@_0M@CHKKJDAI@MessageBoxA?$AA@ 004d6b84     LIBC:crtmbox.obj
 0002:0001ab90       ??_C@_0L@GMPLCCII@user32?4dll?$AA@ 004d6b90     LIBC:crtmbox.obj
 0002:0001ab9c       ??_C@_06IMKFLFPG@1?$CDQNAN?$AA@ 004d6b9c     LIBC:x10fout.obj
 0002:0001aba4       ??_C@_05DNEBIAHO@1?$CDINF?$AA@ 004d6ba4     LIBC:x10fout.obj
 0002:0001abac       ??_C@_05PHHOCPM@1?$CDIND?$AA@ 004d6bac     LIBC:x10fout.obj
 0002:0001abb4       ??_C@_06PGGFOGJG@1?$CDSNAN?$AA@ 004d6bb4     LIBC:x10fout.obj
 0002:0001abd8       __load_config_used         004d6bd8     LIBC:loadcfg.obj
 0002:0001ac70       ___safe_se_handler_table   004d6c70     <linker-defined>
 0002:0001ac78       ___rtc_iaa                 004d6c78     LIBC:initsect.obj
 0002:0001ac7c       ___rtc_izz                 004d6c7c     LIBC:initsect.obj
 0002:0001ac80       ___rtc_taa                 004d6c80     LIBC:initsect.obj
 0002:0001ac84       ___rtc_tzz                 004d6c84     LIBC:initsect.obj
 0002:0001ac88       __IMPORT_DESCRIPTOR_WINMM  004d6c88     winmm:WINMM.dll
 0002:0001ac9c       __IMPORT_DESCRIPTOR_WSOCK32 004d6c9c     wsock32:WSOCK32.dll
 0002:0001acb0       __IMPORT_DESCRIPTOR_KERNEL32 004d6cb0     kernel32:KERNEL32.dll
 0002:0001acc4       __IMPORT_DESCRIPTOR_USER32 004d6cc4     user32:USER32.dll
 0002:0001acd8       __IMPORT_DESCRIPTOR_GDI32  004d6cd8     gdi32:GDI32.dll
 0002:0001acec       __IMPORT_DESCRIPTOR_ADVAPI32 004d6cec     advapi32:ADVAPI32.dll
 0002:0001ad00       __IMPORT_DESCRIPTOR_ole32  004d6d00     ole32:ole32.dll
 0002:0001ad14       __NULL_IMPORT_DESCRIPTOR   004d6d14     winmm:WINMM.dll
 0003:00000000       ___xc_a                    004d8000     LIBC:crt0init.obj
 0003:00000008       ___xc_z                    004d8008     LIBC:crt0init.obj
 0003:0000000c       ___xi_a                    004d800c     LIBC:crt0init.obj
 0003:00000024       ___xi_z                    004d8024     LIBC:crt0init.obj
 0003:00000028       ___xp_a                    004d8028     LIBC:crt0init.obj
 0003:00000030       ___xp_z                    004d8030     LIBC:crt0init.obj
 0003:00000034       ___xt_a                    004d8034     LIBC:crt0init.obj
 0003:00000038       ___xt_z                    004d8038     LIBC:crt0init.obj
 0003:00000048       _g_console_field_width     004d8048     cl_console.obj
 0003:0000004c       _console_color             004d804c     cl_console.obj
 0003:00000060       _keynames                  004d8060     cl_keys.obj
 0003:000003c0       _svc_strings               004d83c0     cl_parse.obj
 0003:000007c0       _demo_protocols            004d87c0     common.obj
 0003:000007d0       _emptystring               004d87d0     common.obj
 0003:000007e8       _numberstring              004d87e8     common.obj
 0003:000008d8       _cl_cdkey                  004d88d8     common.obj
 0003:000009d8       _kbitmask                  004d89d8     msg.obj
 0003:00000a58       _entityStateFields         004d8a58     msg.obj
 0003:00000cc0       _playerStateFields         004d8cc0     msg.obj
 0003:00000f00       _msg_hData                 004d8f00     msg.obj
 0003:00001308       _axisDefault               004d9308     q_math.obj
 0003:0000132c       _colorBlack                004d932c     q_math.obj
 0003:0000133c       _colorRed                  004d933c     q_math.obj
 0003:0000134c       _colorGreen                004d934c     q_math.obj
 0003:0000135c       _colorBlue                 004d935c     q_math.obj
 0003:0000136c       _colorYellow               004d936c     q_math.obj
 0003:0000137c       _colorMagenta              004d937c     q_math.obj
 0003:0000138c       _colorCyan                 004d938c     q_math.obj
 0003:0000139c       _colorWhite                004d939c     q_math.obj
 0003:000013ac       _colorLtGrey               004d93ac     q_math.obj
 0003:000013bc       _colorMdGrey               004d93bc     q_math.obj
 0003:000013cc       _colorDkGrey               004d93cc     q_math.obj
 0003:000013e0       _g_color_table             004d93e0     q_math.obj
 0003:00001460       _bytedirs                  004d9460     q_math.obj
 0003:000030d8       _joyDirectionKeys          004db0d8     win_input.obj
 0003:000031a0       _r_vidModes                004db1a0     renderer:tr_init.obj
 0003:000032b0       _entitySurface             004db2b0     renderer:tr_main.obj
 0003:000032b8       _gl_filter_min             004db2b8     renderer:tr_image.obj
 0003:000032bc       _gl_filter_max             004db2bc     renderer:tr_image.obj
 0003:000032c0       _modes                     004db2c0     renderer:tr_image.obj
 0003:00003308       _mipBlendColors            004db308     renderer:tr_image.obj
 0003:000033b0       _infoParms                 004db3b0     renderer:tr_shader.obj
 0003:00003644       _rb_surfaceTable           004db644     renderer:tr_surface.obj
 0003:000037a0       _edgeVerts                 004db7a0     renderer:tr_shade_calc.obj
 0003:000037d0       _lightOrigin               004db7d0     renderer:tr_shade_calc.obj
 0003:000037e0       _iteminfo_fields           004db7e0     botlib:be_ai_goal.obj
 0003:000038dc       _iteminfo_struct           004db8dc     botlib:be_ai_goal.obj
 0003:00003d28       _directives                004dbd28     botlib:l_precomp.obj
 0003:00003dc8       _dollardirectives          004dbdc8     botlib:l_precomp.obj
 0003:00003e98       _default_punctuations      004dbe98     botlib:l_script.obj
 0003:00004114       _nofaceflood               004dc114     botlib:be_aas_cluster.obj
 0003:00004118       _crctable                  004dc118     botlib:l_crc.obj
 0003:0000431c       __fltused                  004dc31c     LIBC:fpinit.obj
 0003:00004320       __ldused                   004dc320     LIBC:fpinit.obj
 0003:00004324       __FPinit                   004dc324     LIBC:fpinit.obj
 0003:00004328       __FPmtinit                 004dc328     LIBC:fpinit.obj
 0003:0000432c       __FPmtterm                 004dc32c     LIBC:fpinit.obj
 0003:00004350       __aexit_rtn                004dc350     LIBC:wincrt0.obj
 0003:00004354       ___app_type                004dc354     LIBC:wincrt0.obj
 0003:00004360       __half                     004dc360     LIBC:pow.obj
 0003:00004370       __cfltcvt_tab              004dc370     LIBC:cmiscdat.obj
 0003:00004390       __pmatherr                 004dc390     LIBC:libm_error.obj
 0003:000043a0       ___lc_clike                004dc3a0     LIBC:nlsdata2.obj
 0003:000043a4       __pctype                   004dc3a4     LIBC:ctype.obj
 0003:000043a8       __pwctype                  004dc3a8     LIBC:ctype.obj
 0003:000043ac       ___mb_cur_max              004dc3ac     LIBC:nlsdata1.obj
 0003:000043b0       ___decimal_point           004dc3b0     LIBC:nlsdata1.obj
 0003:000043b4       ___decimal_point_length    004dc3b4     LIBC:nlsdata1.obj
 0003:000043c0       ___nullstring              004dc3c0     LIBC:output.obj
 0003:000043c4       ___wnullstring             004dc3c4     LIBC:output.obj
 0003:000043c8       __iob                      004dc3c8     LIBC:_file.obj
 0003:00004648       __timezone                 004dc648     LIBC:timeset.obj
 0003:0000464c       __daylight                 004dc64c     LIBC:timeset.obj
 0003:00004650       __dstbias                  004dc650     LIBC:timeset.obj
 0003:000046d8       __tzname                   004dc6d8     LIBC:timeset.obj
 0003:00004700       __indefinite               004dc700     LIBC:87disp.obj
 0003:0000470a       __piby2                    004dc70a     LIBC:87disp.obj
 0003:0000471c       __cpower                   004dc71c     LIBC:87disp.obj
 0003:00004730       __NLG_Destination          004dc730     LIBC:exsup.obj
 0003:00004740       __amblksiz                 004dc740     LIBC:heapinit.obj
 0003:00004748       ___badioinfo               004dc748     LIBC:ioinit.obj
 0003:000048c0       ___security_cookie         004dc8c0     LIBC:seccook.obj
 0003:00004960       __XcptActTab               004dc960     LIBC:winxfltr.obj
 0003:000049d8       __First_FPE_Indx           004dc9d8     LIBC:winxfltr.obj
 0003:000049dc       __Num_FPE                  004dc9dc     LIBC:winxfltr.obj
 0003:000049e0       __XcptActTabCount          004dc9e0     LIBC:winxfltr.obj
 0003:000049e4       __fpecode                  004dc9e4     LIBC:winxfltr.obj
 0003:000049f0       __infinity                 004dc9f0     LIBC:87tran.obj
 0003:000049fa       __minfinity                004dc9fa     LIBC:87tran.obj
 0003:00004a04       __logemax                  004dca04     LIBC:87tran.obj
 0003:00004a34       __OP_EXPjmptab             004dca34     LIBC:87tran.obj
 0003:00004b80       __matherr_flag             004dcb80     LIBC:matherr.obj
 0003:00004c70       __d_inf                    004dcc70     LIBC:util.obj
 0003:00004c78       __d_ind                    004dcc78     LIBC:util.obj
 0003:00004c80       __d_max                    004dcc80     LIBC:util.obj
 0003:00004c88       __d_min                    004dcc88     LIBC:util.obj
 0003:00004c90       __d_mzero                  004dcc90     LIBC:util.obj
 0003:00004cb0       __lpdays                   004dccb0     LIBC:days.obj
 0003:00004ce4       __days                     004dcce4     LIBC:days.obj
 0003:00004e80       __pow10pos                 004dce80     LIBC:constpow.obj
 0003:00004fe0       __pow10neg                 004dcfe0     LIBC:constpow.obj
 0003:003027e4       _newsize                   007da7e4     cl_net_chan.obj
 0003:003f048c       _oldsize                   008c848c     msg.obj
 0003:003f050c       _vec3_origin               008c850c     q_math.obj
 0003:004149d4       _s_numSfx                  008ec9d4     snd_dma.obj
 0003:00414a04       _sfxScratchBuffer          008eca04     snd_mem.obj
 0003:00414a08       _sfxScratchPointer         008eca08     snd_mem.obj
 0003:00414a0c       _sfxScratchIndex           008eca0c     snd_mem.obj
 0003:0041ce9c       _gvm                       008f4e9c     sv_main.obj
 0003:0041d2c0       _currentVM                 008f52c0     vm.obj
 0003:0041d2c4       _lastVM                    008f52c4     vm.obj
 0003:0041dc78       _fh                        008f5c78     win_main.obj
 0003:00488448       _botlibsetup               00960448     botlib:be_interface.obj
 0003:0048844c       _consolemessageheap        0096044c     botlib:be_ai_chat.obj
 0003:00488450       _freeconsolemessages       00960450     botlib:be_ai_chat.obj
 0003:00488454       _matchtemplates            00960454     botlib:be_ai_chat.obj
 0003:00488458       _synonyms                  00960458     botlib:be_ai_chat.obj
 0003:0048845c       _randomstrings             0096045c     botlib:be_ai_chat.obj
 0003:00488460       _replychats                00960460     botlib:be_ai_chat.obj
 0003:00488464       _itemconfig                00960464     botlib:be_ai_goal.obj
 0003:00488468       _levelitemheap             00960468     botlib:be_ai_goal.obj
 0003:0048846c       _freelevelitems            0096046c     botlib:be_ai_goal.obj
 0003:00488470       _levelitems                00960470     botlib:be_ai_goal.obj
 0003:00488474       _numlevelitems             00960474     botlib:be_ai_goal.obj
 0003:00488478       _maplocations              00960478     botlib:be_ai_goal.obj
 0003:0048847c       _campspots                 0096047c     botlib:be_ai_goal.obj
 0003:00488480       _g_gametype                00960480     botlib:be_ai_goal.obj
 0003:00488484       _droppedweight             00960484     botlib:be_ai_goal.obj
 0003:004909e8       ___fastflag                009689e8     LIBC:fpinit.obj
 0003:004909ec       __adjust_fdiv              009689ec     LIBC:fpinit.obj
 0003:00490a0c       _errno                     00968a0c     LIBC:crt0dat.obj
 0003:00490a10       __doserrno                 00968a10     LIBC:crt0dat.obj
 0003:00490a14       __umaskval                 00968a14     LIBC:crt0dat.obj
 0003:00490a18       __osplatform               00968a18     LIBC:crt0dat.obj
 0003:00490a1c       __osver                    00968a1c     LIBC:crt0dat.obj
 0003:00490a20       __winver                   00968a20     LIBC:crt0dat.obj
 0003:00490a24       __winmajor                 00968a24     LIBC:crt0dat.obj
 0003:00490a28       __winminor                 00968a28     LIBC:crt0dat.obj
 0003:00490a2c       ___argc                    00968a2c     LIBC:crt0dat.obj
 0003:00490a30       ___argv                    00968a30     LIBC:crt0dat.obj
 0003:00490a34       ___wargv                   00968a34     LIBC:crt0dat.obj
 0003:00490a38       __environ                  00968a38     LIBC:crt0dat.obj
 0003:00490a3c       ___initenv                 00968a3c     LIBC:crt0dat.obj
 0003:00490a40       __wenviron                 00968a40     LIBC:crt0dat.obj
 0003:00490a44       ___winitenv                00968a44     LIBC:crt0dat.obj
 0003:00490a48       __pgmptr                   00968a48     LIBC:crt0dat.obj
 0003:00490a4c       __wpgmptr                  00968a4c     LIBC:crt0dat.obj
 0003:00490a50       __exitflag                 00968a50     LIBC:crt0dat.obj
 0003:00490a54       __C_Termination_Done       00968a54     LIBC:crt0dat.obj
 0003:00490a58       __C_Exit_Done              00968a58     LIBC:crt0dat.obj
 0003:00490a60       __aenvptr                  00968a60     LIBC:wincrt0.obj
 0003:00490a64       __wenvptr                  00968a64     LIBC:wincrt0.obj
 0003:00490a68       ___error_mode              00968a68     LIBC:wincrt0.obj
 0003:00490a8c       ___lc_handle               00968a8c     LIBC:nlsdata2.obj
 0003:00490aa4       ___lc_codepage             00968aa4     LIBC:nlsdata2.obj
 0003:00490aa8       ___lc_collate_cp           00968aa8     LIBC:nlsdata2.obj
 0003:00490aac       __stdbuf                   00968aac     LIBC:_sftbuf.obj
 0003:00490ab4       __cflush                   00968ab4     LIBC:_file.obj
 0003:00490b94       ?_pnhHeap@@3P6AHI@ZA       00968b94     LIBC:handler.obj
 0003:00490b98       __newmode                  00968b98     LIBC:_newmode.obj
 0003:00490bb8       __adbgmsg                  00968bb8     LIBC:crt0msg.obj
 0003:00490bbc       __pxcptinfoptrs            00968bbc     LIBC:winxfltr.obj
 0003:00490d04       __commode                  00968d04     LIBC:ncommode.obj
 0003:00490d6c       __fmode                    00968d6c     LIBC:txtmode.obj
 0003:00490d74       _r_fullscreen              00968d74     <common>
 0003:00490d80       _g_wv                      00968d80     <common>
 0003:00490e30       _vid_ypos                  00968e30     <common>
 0003:00490e34       _vid_xpos                  00968e34     <common>
 0003:00490e38       _pDirectSoundCreate        00968e38     <common>
 0003:00490e3c       _sys_timeBase              00968e3c     <common>
 0003:00490e40       _recvfromCount             00968e40     <common>
 0003:00490e44       _totalMsec                 00968e44     <common>
 0003:00490e48       _eventHead                 00968e48     <common>
 0003:00490e60       _eventQue                  00968e60     <common>
 0003:00492660       _countMsec                 0096a660     <common>
 0003:00492664       _eventTail                 0096a664     <common>
 0003:00492680       _sys_packetReceived        0096a680     <common>
 0003:00496680       _in_midi                   0096e680     <common>
 0003:00496684       _in_mouse                  0096e684     <common>
 0003:00496688       _in_midichannel            0096e688     <common>
 0003:0049668c       _in_joystick               0096e68c     <common>
 0003:00496690       _in_debugJoystick          0096e690     <common>
 0003:00496694       _in_joyBallScale           0096e694     <common>
 0003:00496698       _pDirectInputCreate        0096e698     <common>
 0003:0049669c       _joy_threshold             0096e69c     <common>
 0003:004966a0       _in_mididevice             0096e6a0     <common>
 0003:004966a4       _in_logitechbug            0096e6a4     <common>
 0003:004966a8       _in_midiport               0096e6a8     <common>
 0003:004966ac       _in_appactive              0096e6ac     <common>
 0003:004966c0       _vmTable                   0096e6c0     <common>
 0003:00496924       _vm_debugLevel             0096e924     <common>
 0003:00496940       _sv_worldSectors           0096e940     <common>
 0003:00496e40       _sv_numworldSectors        0096ee40     <common>
 0003:00496e44       _sv_maxPing                0096ee44     <common>
 0003:00496e60       _sv                        0096ee60     <common>
 0003:004e32a0       _sv_pure                   009bb2a0     <common>
 0003:004e32a4       _sv_rconPassword           009bb2a4     <common>
 0003:004e32c0       _svs                       009bb2c0     <common>
 0003:004ed320       _sv_master                 009c5320     <common>
 0003:004ed334       _sv_privateClients         009c5334     <common>
 0003:004ed338       _sv_maxclients             009c5338     <common>
 0003:004ed33c       _sv_hostname               009c533c     <common>
 0003:004ed340       _sv_showloss               009c5340     <common>
 0003:004ed344       _sv_reconnectlimit         009c5344     <common>
 0003:004ed348       _sv_floodProtect           009c5348     <common>
 0003:004ed34c       _sv_allowDownload          009c534c     <common>
 0003:004ed350       _sv_killserver             009c5350     <common>
 0003:004ed354       _sv_gametype               009c5354     <common>
 0003:004ed358       _sv_mapname                009c5358     <common>
 0003:004ed35c       _sv_maxRate                009c535c     <common>
 0003:004ed360       _sv_minPing                009c5360     <common>
 0003:004ed364       _sv_zombietime             009c5364     <common>
 0003:004ed368       _sv_privatePassword        009c5368     <common>
 0003:004ed36c       _sv_mapChecksum            009c536c     <common>
 0003:004ed370       _sv_timeout                009c5370     <common>
 0003:004ed374       _sv_padPackets             009c5374     <common>
 0003:004ed378       _sv_lanForceRate           009c5378     <common>
 0003:004ed37c       _sv_fps                    009c537c     <common>
 0003:004ed380       _sv_strictAuth             009c5380     <common>
 0003:004ed384       _sv_serverid               009c5384     <common>
 0003:004ed388       _botlib_export             009c5388     <common>
 0003:004ed38c       _bot_enable                009c538c     <common>
 0003:004ed390       _bot_maxdebugpolys         009c5390     <common>
 0003:004ed3a0       _mulawToShort              009c53a0     <common>
 0003:004ed5a0       _snd_p                     009c55a0     <common>
 0003:004ed5a4       _snd_linear_count          009c55a4     <common>
 0003:004ed5a8       _snd_out                   009c55a8     <common>
 0003:004ed5ac       _s_rawend                  009c55ac     <common>
 0003:004ed5b0       _s_musicVolume             009c55b0     <common>
 0003:004ed5b4       _s_volume                  009c55b4     <common>
 0003:004ed5b8       _s_separation              009c55b8     <common>
 0003:004ed5c0       _s_rawsamples              009c55c0     <common>
 0003:0050d5e0       _s_knownSfx                009e55e0     <common>
 0003:0056d600       _s_channels                00a45600     <common>
 0003:0056ec80       _loop_channels             00a46c80     <common>
 0003:00570300       _s_soundtime               00a48300     <common>
 0003:00570304       _s_mixahead                00a48304     <common>
 0003:00570308       _s_paintedtime             00a48308     <common>
 0003:0057030c       _numLoopChannels           00a4830c     <common>
 0003:00570310       _s_testsound               00a48310     <common>
 0003:00570314       _s_doppler                 00a48314     <common>
 0003:00570318       _s_khz                     00a48318     <common>
 0003:0057031c       _s_show                    00a4831c     <common>
 0003:00570320       _s_mixPreStep              00a48320     <common>
 0003:00570340       _dma                       00a48340     <common>
 0003:00570358       _showpackets               00a48358     <common>
 0003:0057035c       _qport                     00a4835c     <common>
 0003:00570360       _loopbacks                 00a48360     <common>
 0003:0057b2f0       _showdrop                  00a532f0     <common>
 0003:0057b2f4       _overflows                 00a532f4     <common>
 0003:0057b300       _pcount                    00a53300     <common>
 0003:0057b700       _lastValidBase             00a53700     <common>
 0003:0057b800       _lastValidGame             00a53800     <common>
 0003:0057b900       _cvar_vars                 00a53900     <common>
 0003:0057b904       _cvar_cheats               00a53904     <common>
 0003:0057b908       _cvar_modifiedFlags        00a53908     <common>
 0003:0057b920       _cvar_indexes              00a53920     <common>
 0003:00586920       _cvar_numIndexes           00a5e920     <common>
 0003:00586924       _com_blood                 00a5e924     <common>
 0003:00586928       _com_developer             00a5e928     <common>
 0003:0058692c       _com_cameraMode            00a5e92c     <common>
 0003:00586930       _com_viewlog               00a5e930     <common>
 0003:00586934       _com_fixedtime             00a5e934     <common>
 0003:00586938       _com_logfile               00a5e938     <common>
 0003:0058693c       _com_journalDataFile       00a5e93c     <common>
 0003:00586940       _cl_paused                 00a5e940     <common>
 0003:00586944       _com_journalFile           00a5e944     <common>
 0003:00586948       _com_timescale             00a5e948     <common>
 0003:0058694c       _time_backend              00a5e94c     <common>
 0003:00586950       _com_timedemo              00a5e950     <common>
 0003:00586954       _com_buildScript           00a5e954     <common>
 0003:00586958       _com_dedicated             00a5e958     <common>
 0003:0058695c       _com_sv_running            00a5e95c     <common>
 0003:00586960       _abortframe                00a5e960     <common>
 0003:005869a0       _com_consoleLines          00a5e9a0     <common>
 0003:00586a20       _debuglogfile              00a5ea20     <common>
 0003:00586a24       _com_version               00a5ea24     <common>
 0003:00586a40       _com_argv                  00a5ea40     <common>
 0003:00586b0c       _mainzone                  00a5eb0c     <common>
 0003:00586b20       _com_errorMessage          00a5eb20     <common>
 0003:00587b20       _com_numConsoleLines       00a5fb20     <common>
 0003:00587b24       _com_speeds                00a5fb24     <common>
 0003:00587b28       _sv_paused                 00a5fb28     <common>
 0003:00587b2c       _time_game                 00a5fb2c     <common>
 0003:00587b30       _smallzone                 00a5fb30     <common>
 0003:00587b34       _time_frontend             00a5fb34     <common>
 0003:00587b38       _com_journal               00a5fb38     <common>
 0003:00587b3c       _com_dropsim               00a5fb3c     <common>
 0003:00587b40       _com_showtrace             00a5fb40     <common>
 0003:00587b44       _com_frameMsec             00a5fb44     <common>
 0003:00587b48       _com_cl_running            00a5fb48     <common>
 0003:00587b4c       _com_argc                  00a5fb4c     <common>
 0003:00587b50       _com_maxfps                00a5fb50     <common>
 0003:00587b54       _com_frameTime             00a5fb54     <common>
 0003:00587b58       _com_introPlayed           00a5fb58     <common>
 0003:00587b5c       _com_fullyInitialized      00a5fb5c     <common>
 0003:00587b60       _com_errorEntered          00a5fb60     <common>
 0003:00587b64       _com_frameNumber           00a5fb64     <common>
 0003:00587b68       _cmd_wait                  00a5fb68     <common>
 0003:00587b80       _cmd_text_buf              00a5fb80     <common>
 0003:0058bb80       _cmd_text                  00a63b80     <common>
 0003:0058bb8c       _c_active_windings         00a63b8c     <common>
 0003:0058bb90       _c_removed                 00a63b90     <common>
 0003:0058bb94       _c_peak_windings           00a63b94     <common>
 0003:0058bb98       _c_winding_allocs          00a63b98     <common>
 0003:0058bb9c       _c_winding_points          00a63b9c     <common>
 0003:0058bba0       _c_totalPatchBlocks        00a63ba0     <common>
 0003:0058bba4       _c_totalPatchSurfaces      00a63ba4     <common>
 0003:0058bba8       _c_totalPatchEdges         00a63ba8     <common>
 0003:0058bbac       _cm_noAreas                00a63bac     <common>
 0003:0058bbb0       _cm_noCurves               00a63bb0     <common>
 0003:0058bbb4       _c_traces                  00a63bb4     <common>
 0003:0058bbc0       _box_model                 00a63bc0     <common>
 0003:0058bc00       _cm                        00a63c00     <common>
 0003:0058bcbc       _c_brush_traces            00a63cbc     <common>
 0003:0058bcc0       _box_brush                 00a63cc0     <common>
 0003:0058bcc4       _cmod_base                 00a63cc4     <common>
 0003:0058bcc8       _cm_playerCurveClip        00a63cc8     <common>
 0003:0058bccc       _c_pointcontents           00a63ccc     <common>
 0003:0058bcd0       _c_patch_traces            00a63cd0     <common>
 0003:0058bcd4       _box_planes                00a63cd4     <common>
 0003:0058bcd8       _uivm                      00a63cd8     <common>
 0003:0058bcdc       _cl_debuggraph             00a63cdc     <common>
 0003:0058bce0       _cl_graphscale             00a63ce0     <common>
 0003:0058bce4       _cl_graphshift             00a63ce4     <common>
 0003:0058bce8       _cl_timegraph              00a63ce8     <common>
 0003:0058bcec       _cl_graphheight            00a63cec     <common>
 0003:0058bcf0       _scr_initialized           00a63cf0     <common>
 0003:0058bcf4       _cl_connectedToPureServer  00a63cf4     <common>
 0003:0058bcf8       _cl_conXOffset             00a63cf8     <common>
 0003:0058bcfc       _cl_allowDownload          00a63cfc     <common>
 0003:0058bd00       _cl_showSend               00a63d00     <common>
 0003:0058bd04       _rconAddress               00a63d04     <common>
 0003:0058bd08       _cl_avidemo                00a63d08     <common>
 0003:0058bd20       _re                        00a63d20     <common>
 0003:0058bd94       _cl_nodelta                00a63d94     <common>
 0003:0058bd98       _cl_trn                    00a63d98     <common>
 0003:0058bda0       _cl                        00a63da0     <common>
 0003:006319e8       _cl_sensitivity            00b099e8     <common>
 0003:006319ec       _cl_forceavidemo           00b099ec     <common>
 0003:006319f0       _cl_timeout                00b099f0     <common>
 0003:006319f4       _m_yaw                     00b099f4     <common>
 0003:006319f8       _m_pitch                   00b099f8     <common>
 0003:006319fc       _cl_activeAction           00b099fc     <common>
 0003:00631a00       _cl_shownet                00b09a00     <common>
 0003:00631a04       _serverStatusCount         00b09a04     <common>
 0003:00631a20       _cls                       00b09a20     <common>
 0003:006e1400       _cl_pinglist               00bb9400     <common>
 0003:006e9780       _cl_showMouseRate          00bc1780     <common>
 0003:006e9784       _m_forward                 00bc1784     <common>
 0003:006e9788       _cl_packetdup              00bc1788     <common>
 0003:006e978c       _cl_mouseAccel             00bc178c     <common>
 0003:006e97a0       _clc                       00bc17a0     <common>
 0003:0071229c       _cl_maxpackets             00bea29c     <common>
 0003:007122a0       _cl_motd                   00bea2a0     <common>
 0003:007122a4       _cl_timedemo               00bea2a4     <common>
 0003:007122a8       _cl_motdString             00bea2a8     <common>
 0003:007122ac       _cl_freezeDemo             00bea2ac     <common>
 0003:007122b0       _cl_showTimeDelta          00bea2b0     <common>
 0003:007122c0       _cl_serverStatusList       00bea2c0     <common>
 0003:00732540       _cl_timeNudge              00c0a540     <common>
 0003:00732544       _cl_inGameVideo            00c0a544     <common>
 0003:00732548       _cl_noprint                00c0a548     <common>
 0003:0073254c       _m_side                    00c0a54c     <common>
 0003:00732550       _cl_serverStatusResendTime 00c0a550     <common>
 0003:00732554       _m_filter                  00c0a554     <common>
 0003:00732558       _cl_debugMove              00c0a558     <common>
 0003:0073255c       _cgvm                      00c0a55c     <common>
 0003:00732560       _cl_freelook               00c0a560     <common>
 0003:00732564       _rcon_client_password      00c0a564     <common>
 0003:00732568       _historyLine               00c0a568     <common>
 0003:0073256c       _key_overstrikeMode        00c0a56c     <common>
 0003:00732570       _nextHistoryLine           00c0a570     <common>
 0003:00732580       _g_consoleField            00c0a580     <common>
 0003:0073268c       _anykeydown                00c0a68c     <common>
 0003:00732690       _chat_playerNum            00c0a690     <common>
 0003:007326a0       _keys                      00c0a6a0     <common>
 0003:007332a0       _chat_team                 00c0b2a0     <common>
 0003:007332c0       _chatField                 00c0b2c0     <common>
 0003:007333e0       _historyEditLines          00c0b3e0     <common>
 0003:00735560       _in_up                     00c0d560     <common>
 0003:00735580       _in_forward                00c0d580     <common>
 0003:007355a0       _in_buttons                00c0d5a0     <common>
 0003:00735720       _in_right                  00c0d720     <common>
 0003:00735738       _cl_yawspeed               00c0d738     <common>
 0003:00735740       _in_lookdown               00c0d740     <common>
 0003:00735760       _in_left                   00c0d760     <common>
 0003:00735780       _in_moveleft               00c0d780     <common>
 0003:00735798       _cl_upspeed                00c0d798     <common>
 0003:0073579c       _cl_sidespeed              00c0d79c     <common>
 0003:007357a0       _old_com_frameTime         00c0d7a0     <common>
 0003:007357c0       _in_down                   00c0d7c0     <common>
 0003:007357e0       _in_strafe                 00c0d7e0     <common>
 0003:007357f8       _frame_msec                00c0d7f8     <common>
 0003:007357fc       _in_mlooking               00c0d7fc     <common>
 0003:00735800       _in_speed                  00c0d800     <common>
 0003:00735818       _cl_pitchspeed             00c0d818     <common>
 0003:00735820       _in_lookup                 00c0d820     <common>
 0003:00735838       _cl_run                    00c0d838     <common>
 0003:0073583c       _cl_forwardspeed           00c0d83c     <common>
 0003:00735840       _in_moveright              00c0d840     <common>
 0003:00735858       _cl_anglespeedkey          00c0d858     <common>
 0003:00735860       _in_back                   00c0d860     <common>
 0003:00735878       _con_notifytime            00c0d878     <common>
 0003:00735880       _con                       00c0d880     <common>
 0003:007458c8       _con_conspeed              00c1d8c8     <common>
 0003:007458cc       _r_activeFlares            00c1d8cc     <common>
 0003:007458e0       _r_flareStructs            00c1d8e0     <common>
 0003:007476e0       _r_inactiveFlares          00c1f6e0     <common>
 0003:00747700       _tess                      00c1f700     <common>
 0003:00760d64       _r_numentities             00c38d64     <common>
 0003:00760d68       _r_numdlights              00c38d68     <common>
 0003:00760d6c       _r_firstSceneDlight        00c38d6c     <common>
 0003:00760d70       _r_numpolyverts            00c38d70     <common>
 0003:00760d74       _r_firstScenePoly          00c38d74     <common>
 0003:00760d78       _r_firstSceneDrawSurf      00c38d78     <common>
 0003:00760d7c       _r_firstSceneEntity        00c38d7c     <common>
 0003:00760d80       _r_numpolys                00c38d80     <common>
 0003:00760d84       _c_gridVerts               00c38d84     <common>
 0003:00760d88       _c_subdivisions            00c38d88     <common>
 0003:00760d8c       _glimpRenderThread         00c38d8c     <common>
 0003:00760d90       _renderThreadHandle        00c38d90     <common>
 0003:00760d94       _renderActiveEvent         00c38d94     <common>
 0003:00760d98       _r_maskMinidriver          00c38d98     <common>
 0003:00760d9c       _renderCommandsEvent       00c38d9c     <common>
 0003:00760da0       _r_allowSoftwareGL         00c38da0     <common>
 0003:00760dc0       _glw_state                 00c38dc0     <common>
 0003:00760dec       _renderThreadId            00c38dec     <common>
 0003:00760df0       _renderCompletedEvent      00c38df0     <common>
 0003:00760df4       _loadmodel                 00c38df4     <common>
 0003:00760df8       _backEndData               00c38df8     <common>
 0003:00760e00       _backEnd                   00c38e00     <common>
 0003:0076130c       _renderCommandList         00c3930c     <common>
 0003:00761310       _c_blockedOnMain           00c39310     <common>
 0003:00761314       _renderThreadActive        00c39314     <common>
 0003:00761318       _c_blockedOnRender         00c39318     <common>
 0003:0076131c       _qglLoadIdentity           00c3931c     <common>
 0003:00761320       _qglEvalCoord2f            00c39320     <common>
 0003:00761324       _qglGetPointerv            00c39324     <common>
 0003:00761328       _qglGetError               00c39328     <common>
 0003:0076132c       _qglTexCoord4d             00c3932c     <common>
 0003:00761330       _qglDepthFunc              00c39330     <common>
 0003:00761334       _qglLighti                 00c39334     <common>
 0003:00761338       _qglCopyTexSubImage1D      00c39338     <common>
 0003:0076133c       _qglVertex3s               00c3933c     <common>
 0003:00761340       _qglLightModelf            00c39340     <common>
 0003:00761344       _qglInitNames              00c39344     <common>
 0003:00761348       _qwglUseFontBitmaps        00c39348     <common>
 0003:0076134c       _qglShadeModel             00c3934c     <common>
 0003:00761350       _qglGetMaterialiv          00c39350     <common>
 0003:00761354       _qglTexCoord3iv            00c39354     <common>
 0003:00761358       _qglMapGrid1d              00c39358     <common>
 0003:0076135c       _qglListBase               00c3935c     <common>
 0003:00761360       _qglNormal3d               00c39360     <common>
 0003:00761364       _qglRasterPos4dv           00c39364     <common>
 0003:00761368       _qglGetMapiv               00c39368     <common>
 0003:0076136c       _qglVertex3i               00c3936c     <common>
 0003:00761370       _qglTexCoord4iv            00c39370     <common>
 0003:00761374       _qglEvalCoord1d            00c39374     <common>
 0003:00761378       _qglMaterialfv             00c39378     <common>
 0003:0076137c       _qglEnableClientState      00c3937c     <common>
 0003:00761380       _qglEdgeFlagv              00c39380     <common>
 0003:00761384       _qglMaterialiv             00c39384     <common>
 0003:00761388       _qglNormal3bv              00c39388     <common>
 0003:0076138c       _qglDisableClientState     00c3938c     <common>
 0003:00761390       _qwglSwapBuffers           00c39390     <common>
 0003:00761394       _qglRectd                  00c39394     <common>
 0003:00761398       _qglColor4bv               00c39398     <common>
 0003:0076139c       _qwglUseFontOutlines       00c3939c     <common>
 0003:007613a0       _qglGetTexEnviv            00c393a0     <common>
 0003:007613a4       _qglTexCoord3d             00c393a4     <common>
 0003:007613a8       _qglVertex3f               00c393a8     <common>
 0003:007613ac       _qglEndList                00c393ac     <common>
 0003:007613b0       _qglTexCoordPointer        00c393b0     <common>
 0003:007613b4       _qglTexCoord3i             00c393b4     <common>
 0003:007613b8       _qglTexEnvf                00c393b8     <common>
 0003:007613bc       _qglFogiv                  00c393bc     <common>
 0003:007613c0       _qglRasterPos3f            00c393c0     <common>
 0003:007613c4       _qglMap2f                  00c393c4     <common>
 0003:007613c8       _qglTexCoord4dv            00c393c8     <common>
 0003:007613cc       _qglDisable                00c393cc     <common>
 0003:007613d0       _qglColor4uiv              00c393d0     <common>
 0003:007613d4       _qglRasterPos2d            00c393d4     <common>
 0003:007613d8       _qglFogfv                  00c393d8     <common>
 0003:007613dc       _qwglSwapLayerBuffers      00c393dc     <common>
 0003:007613e0       _qwglShareLists            00c393e0     <common>
 0003:007613e4       _qglTexEnvfv               00c393e4     <common>
 0003:007613e8       _qglPrioritizeTextures     00c393e8     <common>
 0003:007613ec       _qglLoadName               00c393ec     <common>
 0003:007613f0       _qglColor3ub               00c393f0     <common>
 0003:007613f4       _qglTexSubImage1D          00c393f4     <common>
 0003:007613f8       _qglColor4ub               00c393f8     <common>
 0003:007613fc       _qglRecti                  00c393fc     <common>
 0003:00761400       _qglTexParameteriv         00c39400     <common>
 0003:00761404       _qglTexCoord3dv            00c39404     <common>
 0003:00761408       _dllGetString              00c39408     <common>
 0003:0076140c       _qglColor3d                00c3940c     <common>
 0003:00761410       _qglLineStipple            00c39410     <common>
 0003:00761414       _qglGetTexParameterfv      00c39414     <common>
 0003:00761418       _qglGetPixelMapfv          00c39418     <common>
 0003:0076141c       _qglNormal3iv              00c3941c     <common>
 0003:00761420       _qglTexCoord1iv            00c39420     <common>
 0003:00761424       _qglTexCoord4f             00c39424     <common>
 0003:00761428       _qglTexCoord1f             00c39428     <common>
 0003:0076142c       _qglOrtho                  00c3942c     <common>
 0003:00761430       _qglVertex3fv              00c39430     <common>
 0003:00761434       _qglRasterPos2f            00c39434     <common>
 0003:00761438       _qglColor4b                00c39438     <common>
 0003:0076143c       _qglPixelStoref            00c3943c     <common>
 0003:00761440       _qglBlendFunc              00c39440     <common>
 0003:00761444       _qglRasterPos3sv           00c39444     <common>
 0003:00761448       _qglIndexsv                00c39448     <common>
 0003:0076144c       _qwglCopyContext           00c3944c     <common>
 0003:00761450       _qglSelectBuffer           00c39450     <common>
 0003:00761454       _qglPixelTransferf         00c39454     <common>
 0003:00761458       _qglVertex2s               00c39458     <common>
 0003:0076145c       _qwglDescribePixelFormat   00c3945c     <common>
 0003:00761460       _qglTexGend                00c39460     <common>
 0003:00761464       _qglNormal3dv              00c39464     <common>
 0003:00761468       _qglVertex3dv              00c39468     <common>
 0003:0076146c       _qglGetBooleanv            00c3946c     <common>
 0003:00761470       _qglRasterPos2dv           00c39470     <common>
 0003:00761474       _qglVertex2dv              00c39474     <common>
 0003:00761478       _qwglCreateLayerContext    00c39478     <common>
 0003:0076147c       _qglClipPlane              00c3947c     <common>
 0003:00761480       _qglPixelZoom              00c39480     <common>
 0003:00761484       _qglTexCoord4fv            00c39484     <common>
 0003:00761488       _qglGetString              00c39488     <common>
 0003:0076148c       _qglRasterPos2fv           00c3948c     <common>
 0003:00761490       _qglRasterPos3d            00c39490     <common>
 0003:00761494       _qwglChoosePixelFormat     00c39494     <common>
 0003:00761498       _qglColor4i                00c39498     <common>
 0003:0076149c       _qglIndexs                 00c3949c     <common>
 0003:007614a0       _qglLightModelfv           00c394a0     <common>
 0003:007614a4       _qglColor3iv               00c394a4     <common>
 0003:007614a8       _qglPushClientAttrib       00c394a8     <common>
 0003:007614ac       _qglTexCoord1sv            00c394ac     <common>
 0003:007614b0       _qglRotated                00c394b0     <common>
 0003:007614b4       _qwglGetCurrentContext     00c394b4     <common>
 0003:007614b8       _qglScaled                 00c394b8     <common>
 0003:007614bc       _qglColor3s                00c394bc     <common>
 0003:007614c0       _qglRectsv                 00c394c0     <common>
 0003:007614c4       _qglPixelStorei            00c394c4     <common>
 0003:007614c8       _qglRasterPos3iv           00c394c8     <common>
 0003:007614cc       _qglFogi                   00c394cc     <common>
 0003:007614d0       _qglCallLists              00c394d0     <common>
 0003:007614d4       _qglTexCoord3s             00c394d4     <common>
 0003:007614d8       _qglGenLists               00c394d8     <common>
 0003:007614dc       _qglMap1f                  00c394dc     <common>
 0003:007614e0       _qglVertex4sv              00c394e0     <common>
 0003:007614e4       _qglTexImage2D             00c394e4     <common>
 0003:007614e8       _qglGetMapfv               00c394e8     <common>
 0003:007614ec       _qglEdgeFlagPointer        00c394ec     <common>
 0003:007614f0       _qglGetDoublev             00c394f0     <common>
 0003:007614f4       _qglClearIndex             00c394f4     <common>
 0003:007614f8       _qglColorMaterial          00c394f8     <common>
 0003:007614fc       _qglLoadMatrixf            00c394fc     <common>
 0003:00761500       _qglPixelMapuiv            00c39500     <common>
 0003:00761504       _qglLightModeliv           00c39504     <common>
 0003:00761508       _qglGetTexGeniv            00c39508     <common>
 0003:0076150c       _qglRectf                  00c3950c     <common>
 0003:00761510       _qglTexCoord2f             00c39510     <common>
 0003:00761514       _qglGetIntegerv            00c39514     <common>
 0003:00761518       _qglVertex2d               00c39518     <common>
 0003:0076151c       _qglGetMapdv               00c3951c     <common>
 0003:00761520       _qglIsTexture              00c39520     <common>
 0003:00761524       _qglGetPixelMapusv         00c39524     <common>
 0003:00761528       _qglDepthMask              00c39528     <common>
 0003:0076152c       _qglMatrixMode             00c3952c     <common>
 0003:00761530       _qglPolygonMode            00c39530     <common>
 0003:00761534       _qglTexCoord4s             00c39534     <common>
 0003:00761538       _qglPushMatrix             00c39538     <common>
 0003:0076153c       _qwglGetProcAddress        00c3953c     <common>
 0003:00761540       _qglVertex2i               00c39540     <common>
 0003:00761544       _qglRasterPos3s            00c39544     <common>
 0003:00761548       _qglNormal3f               00c39548     <common>
 0003:0076154c       _qglIndexPointer           00c3954c     <common>
 0003:00761550       _qglAreTexturesResident    00c39550     <common>
 0003:00761554       _qglIndexfv                00c39554     <common>
 0003:00761558       _qglColorMask              00c39558     <common>
 0003:0076155c       _qglIndexd                 00c3955c     <common>
 0003:00761560       _qglGetLightfv             00c39560     <common>
 0003:00761564       _qglColor4usv              00c39564     <common>
 0003:00761568       _qglRasterPos4s            00c39568     <common>
 0003:0076156c       _qglLogicOp                00c3956c     <common>
 0003:00761570       _qglPushName               00c39570     <common>
 0003:00761574       _qglTexSubImage2D          00c39574     <common>
 0003:00761578       _qglEvalCoord2dv           00c39578     <common>
 0003:0076157c       _qglRectiv                 00c3957c     <common>
 0003:00761580       _qglStencilFunc            00c39580     <common>
 0003:00761584       _qglPopAttrib              00c39584     <common>
 0003:00761588       _qglTexCoord2fv            00c39588     <common>
 0003:0076158c       _qglRasterPos4i            00c3958c     <common>
 0003:00761590       _qglColor3b                00c39590     <common>
 0003:00761594       _qglPixelMapfv             00c39594     <common>
 0003:00761598       _qglColor4ubv              00c39598     <common>
 0003:0076159c       _dllIsList                 00c3959c     <common>
 0003:007615a0       _qglFlush                  00c395a0     <common>
 0003:007615a4       _qglColor3ui               00c395a4     <common>
 0003:007615a8       _qglEnd                    00c395a8     <common>
 0003:007615ac       _qglColor3dv               00c395ac     <common>
 0003:007615b0       _qglTranslated             00c395b0     <common>
 0003:007615b4       _qglNewList                00c395b4     <common>
 0003:007615b8       _qglGetTexLevelParameteriv 00c395b8     <common>
 0003:007615bc       _qglTexGenfv               00c395bc     <common>
 0003:007615c0       _qglReadPixels             00c395c0     <common>
 0003:007615c4       _qglGenTextures            00c395c4     <common>
 0003:007615c8       _qglRasterPos2sv           00c395c8     <common>
 0003:007615cc       _qglTexCoord1d             00c395cc     <common>
 0003:007615d0       _qglAccum                  00c395d0     <common>
 0003:007615d4       _qglColor4ui               00c395d4     <common>
 0003:007615d8       _qglScalef                 00c395d8     <common>
 0003:007615dc       _qglRasterPos4iv           00c395dc     <common>
 0003:007615e0       _qglIndexubv               00c395e0     <common>
 0003:007615e4       _qglEnable                 00c395e4     <common>
 0003:007615e8       _qglVertex3sv              00c395e8     <common>
 0003:007615ec       _qglRasterPos2i            00c395ec     <common>
 0003:007615f0       _qglTexGenf                00c395f0     <common>
 0003:007615f4       _qglNormal3b               00c395f4     <common>
 0003:007615f8       _qglIndexf                 00c395f8     <common>
 0003:007615fc       _qglPushAttrib             00c395fc     <common>
 0003:00761600       _qglTexCoord2d             00c39600     <common>
 0003:00761604       _qglLightiv                00c39604     <common>
 0003:00761608       _qglPassThrough            00c39608     <common>
 0003:0076160c       _qglCopyPixels             00c3960c     <common>
 0003:00761610       _qglMap2d                  00c39610     <common>
 0003:00761614       _qglIndexi                 00c39614     <common>
 0003:00761618       _qglColor3sv               00c39618     <common>
 0003:0076161c       _qglVertex4i               00c3961c     <common>
 0003:00761620       _qglDrawArrays             00c39620     <common>
 0003:00761624       _qglEvalMesh1              00c39624     <common>
 0003:00761628       _qglColor3usv              00c39628     <common>
 0003:0076162c       _qglNormalPointer          00c3962c     <common>
 0003:00761630       _qglRasterPos3dv           00c39630     <common>
 0003:00761634       _qglColor3f                00c39634     <common>
 0003:00761638       _qglLoadMatrixd            00c39638     <common>
 0003:0076163c       _qglEvalPoint1             00c3963c     <common>
 0003:00761640       _qglReadBuffer             00c39640     <common>
 0003:00761644       _qglBindTexture            00c39644     <common>
 0003:00761648       _dllRenderMode             00c39648     <common>
 0003:0076164c       _qglEvalCoord1dv           00c3964c     <common>
 0003:00761650       _qglTexCoord2iv            00c39650     <common>
 0003:00761654       _qglPolygonOffset          00c39654     <common>
 0003:00761658       _qglRasterPos4fv           00c39658     <common>
 0003:0076165c       _qglTexCoord1dv            00c3965c     <common>
 0003:00761660       _qglIndexub                00c39660     <common>
 0003:00761664       _qglArrayElement           00c39664     <common>
 0003:00761668       _qglVertex4dv              00c39668     <common>
 0003:0076166c       _qglColor3fv               00c3966c     <common>
 0003:00761670       _qglNormal3i               00c39670     <common>
 0003:00761674       _qglMultMatrixd            00c39674     <common>
 0003:00761678       _qglDrawElements           00c39678     <common>
 0003:0076167c       _qglTexEnvi                00c3967c     <common>
 0003:00761680       _qglVertex2f               00c39680     <common>
 0003:00761684       _qglColor4d                00c39684     <common>
 0003:00761688       _qglEvalPoint2             00c39688     <common>
 0003:0076168c       _qglGetTexLevelParameterfv 00c3968c     <common>
 0003:00761690       _qglHint                   00c39690     <common>
 0003:00761694       _qglPopName                00c39694     <common>
 0003:00761698       _dllGetError               00c39698     <common>
 0003:0076169c       _qglVertex2iv              00c3969c     <common>
 0003:007616a0       _qglRectfv                 00c396a0     <common>
 0003:007616a4       _qwglGetCurrentDC          00c396a4     <common>
 0003:007616a8       _qglColor4dv               00c396a8     <common>
 0003:007616ac       _qglColor3bv               00c396ac     <common>
 0003:007616b0       _qglLightfv                00c396b0     <common>
 0003:007616b4       _qglIndexiv                00c396b4     <common>
 0003:007616b8       _qglTexCoord4sv            00c396b8     <common>
 0003:007616bc       _qglPixelTransferi         00c396bc     <common>
 0003:007616c0       _qglAlphaFunc              00c396c0     <common>
 0003:007616c4       _qglScissor                00c396c4     <common>
 0003:007616c8       _qglRotatef                00c396c8     <common>
 0003:007616cc       _qglTranslatef             00c396cc     <common>
 0003:007616d0       _qwglGetLayerPaletteEntries 00c396d0     <common>
 0003:007616d4       _qglTexCoord2dv            00c396d4     <common>
 0003:007616d8       _qglTexImage1D             00c396d8     <common>
 0003:007616dc       _qglColor4iv               00c396dc     <common>
 0003:007616e0       _qglGetTexParameteriv      00c396e0     <common>
 0003:007616e4       _qglDrawBuffer             00c396e4     <common>
 0003:007616e8       _qglCullFace               00c396e8     <common>
 0003:007616ec       _qglRasterPos4d            00c396ec     <common>
 0003:007616f0       _qglVertex4iv              00c396f0     <common>
 0003:007616f4       _qglVertex2sv              00c396f4     <common>
 0003:007616f8       _qglCopyTexImage1D         00c396f8     <common>
 0003:007616fc       _qwglDescribeLayerPlane    00c396fc     <common>
 0003:00761700       _qglTexParameterfv         00c39700     <common>
 0003:00761704       _qglRenderMode             00c39704     <common>
 0003:00761708       _qglRasterPos4f            00c39708     <common>
 0003:0076170c       _qglPopClientAttrib        00c3970c     <common>
 0003:00761710       _qwglDeleteContext         00c39710     <common>
 0003:00761714       _qglFinish                 00c39714     <common>
 0003:00761718       _qglGetTexEnvfv            00c39718     <common>
 0003:0076171c       _qglEvalCoord1f            00c3971c     <common>
 0003:00761720       _qglBegin                  00c39720     <common>
 0003:00761724       _qglDeleteLists            00c39724     <common>
 0003:00761728       _qglFeedbackBuffer         00c39728     <common>
 0003:0076172c       _qglRasterPos3fv           00c3972c     <common>
 0003:00761730       _qwglSetPixelFormat        00c39730     <common>
 0003:00761734       _qglEvalCoord1fv           00c39734     <common>
 0003:00761738       _qglClear                  00c39738     <common>
 0003:0076173c       _qglPointSize              00c3973c     <common>
 0003:00761740       _qglDepthRange             00c39740     <common>
 0003:00761744       _qglPopMatrix              00c39744     <common>
 0003:00761748       _qglMapGrid2f              00c39748     <common>
 0003:0076174c       _qglGetTexGendv            00c3974c     <common>
 0003:00761750       _qglGetTexImage            00c39750     <common>
 0003:00761754       _qglVertex2fv              00c39754     <common>
 0003:00761758       _qglVertex3d               00c39758     <common>
 0003:0076175c       _qglNormal3fv              00c3975c     <common>
 0003:00761760       _qglTexCoord3sv            00c39760     <common>
 0003:00761764       _qglColor3ubv              00c39764     <common>
 0003:00761768       _qglEvalCoord2fv           00c39768     <common>
 0003:0076176c       _qglDrawPixels             00c3976c     <common>
 0003:00761770       _qwglGetPixelFormat        00c39770     <common>
 0003:00761774       _qglGetPixelMapuiv         00c39774     <common>
 0003:00761778       _qglColor3uiv              00c39778     <common>
 0003:0076177c       _qglStencilOp              00c3977c     <common>
 0003:00761780       _qglColorPointer           00c39780     <common>
 0003:00761784       _qglGetLightiv             00c39784     <common>
 0003:00761788       _qglFrontFace              00c39788     <common>
 0003:0076178c       _dllGenLists               00c3978c     <common>
 0003:00761790       _qglMaterialf              00c39790     <common>
 0003:00761794       _qwglSetLayerPaletteEntries 00c39794     <common>
 0003:00761798       _qglClearAccum             00c39798     <common>
 0003:0076179c       _qglColor3us               00c3979c     <common>
 0003:007617a0       _qglEvalMesh2              00c397a0     <common>
 0003:007617a4       _qwglRealizeLayerPalette   00c397a4     <common>
 0003:007617a8       _qglColor3i                00c397a8     <common>
 0003:007617ac       _qglViewport               00c397ac     <common>
 0003:007617b0       _qglVertex3iv              00c397b0     <common>
 0003:007617b4       _qglGetTexGenfv            00c397b4     <common>
 0003:007617b8       _qglIndexMask              00c397b8     <common>
 0003:007617bc       _qglVertex4d               00c397bc     <common>
 0003:007617c0       _qwglSwapIntervalEXT       00c397c0     <common>
 0003:007617c4       _qglEdgeFlag               00c397c4     <common>
 0003:007617c8       _qglRasterPos2iv           00c397c8     <common>
 0003:007617cc       _qglTexEnviv               00c397cc     <common>
 0003:007617d0       _qglVertexPointer          00c397d0     <common>
 0003:007617d4       _qglDeleteTextures         00c397d4     <common>
 0003:007617d8       _qglCopyTexImage2D         00c397d8     <common>
 0003:007617dc       _qglClearColor             00c397dc     <common>
 0003:007617e0       _qglFrustum                00c397e0     <common>
 0003:007617e4       _qglColor4sv               00c397e4     <common>
 0003:007617e8       _dllIsTexture              00c397e8     <common>
 0003:007617ec       _qglLightf                 00c397ec     <common>
 0003:007617f0       _qglBitmap                 00c397f0     <common>
 0003:007617f4       _qglColor4s                00c397f4     <common>
 0003:007617f8       _qglIsEnabled              00c397f8     <common>
 0003:007617fc       _qglGetMaterialfv          00c397fc     <common>
 0003:00761800       _qglColor4f                00c39800     <common>
 0003:00761804       _qglTexCoord2sv            00c39804     <common>
 0003:00761808       _qglMapGrid2d              00c39808     <common>
 0003:0076180c       _qglRectdv                 00c3980c     <common>
 0003:00761810       _qglFogf                   00c39810     <common>
 0003:00761814       _qglGetClipPlane           00c39814     <common>
 0003:00761818       _qglTexGendv               00c39818     <common>
 0003:0076181c       _qglRasterPos2s            00c3981c     <common>
 0003:00761820       _qglInterleavedArrays      00c39820     <common>
 0003:00761824       _qglTexCoord4i             00c39824     <common>
 0003:00761828       _qglTexCoord1i             00c39828     <common>
 0003:0076182c       _qglStencilMask            00c3982c     <common>
 0003:00761830       _qglTexGeniv               00c39830     <common>
 0003:00761834       _qglTexGeni                00c39834     <common>
 0003:00761838       _qglVertex4f               00c39838     <common>
 0003:0076183c       _qglTexCoord2s             00c3983c     <common>
 0003:00761840       _qglTexCoord3f             00c39840     <common>
 0003:00761844       _qglEvalCoord2d            00c39844     <common>
 0003:00761848       _qglMapGrid1f              00c39848     <common>
 0003:0076184c       _qglTexCoord2i             00c3984c     <common>
 0003:00761850       _qglPixelMapusv            00c39850     <common>
 0003:00761854       _qwglGetDeviceGammaRamp3DFX 00c39854     <common>
 0003:00761858       _qglTexCoord1fv            00c39858     <common>
 0003:0076185c       _qwglCreateContext         00c3985c     <common>
 0003:00761860       _qglPolygonStipple         00c39860     <common>
 0003:00761864       _qglCallList               00c39864     <common>
 0003:00761868       _qglClearDepth             00c39868     <common>
 0003:0076186c       _qglColor4us               00c3986c     <common>
 0003:00761870       _qglTexParameteri          00c39870     <common>
 0003:00761874       _qglGetFloatv              00c39874     <common>
 0003:00761878       _dllIsEnabled              00c39878     <common>
 0003:0076187c       _qglIndexdv                00c3987c     <common>
 0003:00761880       _qglVertex4fv              00c39880     <common>
 0003:00761884       _qglTexParameterf          00c39884     <common>
 0003:00761888       _qglRasterPos3i            00c39888     <common>
 0003:0076188c       _qglLightModeli            00c3988c     <common>
 0003:00761890       _qglRects                  00c39890     <common>
 0003:00761894       _qwglMakeCurrent           00c39894     <common>
 0003:00761898       _qglMultMatrixf            00c39898     <common>
 0003:0076189c       _qglMap1d                  00c3989c     <common>
 0003:007618a0       _qglLineWidth              00c398a0     <common>
 0003:007618a4       _qglMateriali              00c398a4     <common>
 0003:007618a8       _qglClearStencil           00c398a8     <common>
 0003:007618ac       _qglNormal3s               00c398ac     <common>
 0003:007618b0       _dllAreTexturesResident    00c398b0     <common>
 0003:007618b4       _qwglSetDeviceGammaRamp3DFX 00c398b4     <common>
 0003:007618b8       _qglTexCoord1s             00c398b8     <common>
 0003:007618bc       _qglRasterPos4sv           00c398bc     <common>
 0003:007618c0       _qglTexCoord3fv            00c398c0     <common>
 0003:007618c4       _qglIsList                 00c398c4     <common>
 0003:007618c8       _qglColor4fv               00c398c8     <common>
 0003:007618cc       _qglVertex4s               00c398cc     <common>
 0003:007618d0       _qglNormal3sv              00c398d0     <common>
 0003:007618d4       _qglGetPolygonStipple      00c398d4     <common>
 0003:007618d8       _qglCopyTexSubImage2D      00c398d8     <common>
 0003:007618e0       _tr                        00c398e0     <common>
 0003:0078b700       _ri                        00c63700     <common>
 0003:0078b768       _r_nocurves                00c63768     <common>
 0003:0078b76c       _r_verbose                 00c6376c     <common>
 0003:0078b770       _r_picmip                  00c63770     <common>
 0003:0078b774       _r_showImages              00c63774     <common>
 0003:0078b778       _r_norefresh               00c63778     <common>
 0003:0078b77c       _r_colorbits               00c6377c     <common>
 0003:0078b780       _r_flares                  00c63780     <common>
 0003:0078b784       _r_lightmap                00c63784     <common>
 0003:0078b788       _r_intensity               00c63788     <common>
 0003:0078b78c       _r_ext_multitexture        00c6378c     <common>
 0003:0078b790       _r_colorMipLevels          00c63790     <common>
 0003:0078b794       _r_drawentities            00c63794     <common>
 0003:0078b798       _r_shadows                 00c63798     <common>
 0003:0078b79c       _r_printShaders            00c6379c     <common>
 0003:0078b7a0       _r_showtris                00c637a0     <common>
 0003:0078b7a4       _r_measureOverdraw         00c637a4     <common>
 0003:0078b7a8       _r_allowExtensions         00c637a8     <common>
 0003:0078b7ac       _r_gamma                   00c637ac     <common>
 0003:0078b7b0       _r_portalOnly              00c637b0     <common>
 0003:0078b7b4       _r_textureMode             00c637b4     <common>
 0003:0078b7b8       _r_dlightBacks             00c637b8     <common>
 0003:0078b7bc       _r_maxpolyverts            00c637bc     <common>
 0003:0078b7c0       _r_lodbias                 00c637c0     <common>
 0003:0078b7c4       _r_lodCurveError           00c637c4     <common>
 0003:0078b7c8       _r_stencilbits             00c637c8     <common>
 0003:0078b7cc       _r_customwidth             00c637cc     <common>
 0003:0078b7d0       _qglClientActiveTextureARB 00c637d0     <common>
 0003:0078b7d4       _r_ignore                  00c637d4     <common>
 0003:0078b7d8       _r_flareSize               00c637d8     <common>
 0003:0078b7dc       _r_maxpolys                00c637dc     <common>
 0003:0078b7e0       _r_drawSun                 00c637e0     <common>
 0003:0078b7e4       _qglActiveTextureARB       00c637e4     <common>
 0003:0078b7e8       _r_nobind                  00c637e8     <common>
 0003:0078b7ec       _r_mode                    00c637ec     <common>
 0003:0078b7f0       _qglUnlockArraysEXT        00c637f0     <common>
 0003:0078b7f4       _r_debugLight              00c637f4     <common>
 0003:0078b7f8       _r_railSegmentLength       00c637f8     <common>
 0003:0078b7fc       _r_offsetFactor            00c637fc     <common>
 0003:0078b800       _r_lodscale                00c63800     <common>
 0003:0078b804       _r_drawworld               00c63804     <common>
 0003:0078b808       _r_railCoreWidth           00c63808     <common>
 0003:0078b80c       _r_customaspect            00c6380c     <common>
 0003:0078b810       _r_glDriver                00c63810     <common>
 0003:0078b814       _r_showcluster             00c63814     <common>
 0003:0078b818       _qglLockArraysEXT          00c63818     <common>
 0003:0078b81c       _r_stereo                  00c6381c     <common>
 0003:0078b820       _r_facePlaneCull           00c63820     <common>
 0003:0078b824       _r_fullbright              00c63824     <common>
 0003:0078b828       _r_uiFullScreen            00c63828     <common>
 0003:0078b82c       _r_drawBuffer              00c6382c     <common>
 0003:0078b830       _r_clear                   00c63830     <common>
 0003:0078b834       _qglMultiTexCoord2fARB     00c63834     <common>
 0003:0078b838       _r_nocull                  00c63838     <common>
 0003:0078b83c       _max_polyverts             00c6383c     <common>
 0003:0078b840       _max_polys                 00c63840     <common>
 0003:0078b844       _r_lockpvs                 00c63844     <common>
 0003:0078b848       _r_noportals               00c63848     <common>
 0003:0078b84c       _r_mapOverBrightBits       00c6384c     <common>
 0003:0078b850       _r_vertexLight             00c63850     <common>
 0003:0078b854       _r_offsetUnits             00c63854     <common>
 0003:0078b858       _r_railWidth               00c63858     <common>
 0003:0078b85c       _r_flareFade               00c6385c     <common>
 0003:0078b860       _r_novis                   00c63860     <common>
 0003:0078b864       _r_dynamiclight            00c63864     <common>
 0003:0078b868       _r_ignoreFastPath          00c63868     <common>
 0003:0078b86c       _r_ext_compressed_textures 00c6386c     <common>
 0003:0078b870       _r_skipBackEnd             00c63870     <common>
 0003:0078b874       _r_overBrightBits          00c63874     <common>
 0003:0078b878       _r_fastsky                 00c63878     <common>
 0003:0078b87c       _r_saveFontData            00c6387c     <common>
 0003:0078b880       _r_singleShader            00c63880     <common>
 0003:0078b884       _r_ext_gamma_control       00c63884     <common>
 0003:0078b8a0       _glState                   00c638a0     <common>
 0003:0078b8c0       _r_debugSort               00c638c0     <common>
 0003:0078b8c4       _r_ignoreGLErrors          00c638c4     <common>
 0003:0078b8c8       _r_showSmp                 00c638c8     <common>
 0003:0078b8cc       _r_shownormals             00c638cc     <common>
 0003:0078b8d0       _r_inGameVideo             00c638d0     <common>
 0003:0078b8d4       _r_primitives              00c638d4     <common>
 0003:0078b8d8       _r_finish                  00c638d8     <common>
 0003:0078b8dc       _r_showsky                 00c638dc     <common>
 0003:0078b8e0       _r_texturebits             00c638e0     <common>
 0003:0078b8e4       _r_roundImagesDown         00c638e4     <common>
 0003:0078b8e8       _r_speeds                  00c638e8     <common>
 0003:0078b8ec       _r_customheight            00c638ec     <common>
 0003:0078b8f0       _r_ignorehwgamma           00c638f0     <common>
 0003:0078b8f4       _r_swapInterval            00c638f4     <common>
 0003:0078b8f8       _r_logFile                 00c638f8     <common>
 0003:0078b8fc       _r_ambientScale            00c638fc     <common>
 0003:0078b900       _r_displayRefresh          00c63900     <common>
 0003:0078b904       _r_smp                     00c63904     <common>
 0003:0078b908       _r_simpleMipMaps           00c63908     <common>
 0003:0078b90c       _r_subdivisions            00c6390c     <common>
 0003:0078b920       _glConfig                  00c63920     <common>
 0003:0078e564       _r_znear                   00c66564     <common>
 0003:0078e568       _r_debugSurface            00c66568     <common>
 0003:0078e56c       _r_ext_texture_env_add     00c6656c     <common>
 0003:0078e570       _r_depthbits               00c66570     <common>
 0003:0078e574       _r_directedScale           00c66574     <common>
 0003:0078e578       _r_ext_compiled_vertex_array 00c66578     <common>
 0003:0078e57c       _r_detailTextures          00c6657c     <common>
 0003:0078e580       _numdebuglines             00c66580     <common>
 0003:0078e5a0       _debuglines                00c665a0     <common>
 0003:0078f5a0       _debuglinevisible          00c675a0     <common>
 0003:007905a0       _basefolder                00c685a0     <common>
 0003:007905e0       _allocatedmemory           00c685e0     <common>
 0003:007905e4       _numblocks                 00c685e4     <common>
 0003:007905e8       _totalmemorysize           00c685e8     <common>
 0003:007905ec       _numaaslinks               00c685ec     <common>
 0003:00790600       _bspworld                  00c68600     <common>
 0003:00792610       _calcgrapplereach          00c6a610     <common>
 0003:00792614       _reach_equalfloor          00c6a614     <common>
 0003:00792618       _reach_bfgjump             00c6a618     <common>
 0003:0079261c       _numlreachabilities        00c6a61c     <common>
 0003:00792620       _reach_elevator            00c6a620     <common>
 0003:00792624       _reach_swim                00c6a624     <common>
 0003:00792628       _reach_rocketjump          00c6a628     <common>
 0003:0079262c       _reach_funcbob             00c6a62c     <common>
 0003:00792630       _reachabilityheap          00c6a630     <common>
 0003:00792634       _reach_waterjump           00c6a634     <common>
 0003:00792638       _reach_walkoffledge        00c6a638     <common>
 0003:0079263c       _areareachability          00c6a63c     <common>
 0003:00792640       _reach_jumppad             00c6a640     <common>
 0003:00792644       _reach_rampjump            00c6a644     <common>
 0003:00792648       _reach_step                00c6a648     <common>
 0003:0079264c       _reach_doublejump          00c6a64c     <common>
 0003:00792650       _reach_strafejump          00c6a650     <common>
 0003:00792654       _reach_jump                00c6a654     <common>
 0003:00792658       _reach_ladder              00c6a658     <common>
 0003:0079265c       _reach_barrier             00c6a65c     <common>
 0003:00792660       _reach_walk                00c6a660     <common>
 0003:00792664       _reach_grapple             00c6a664     <common>
 0003:00792668       _nextreachability          00c6a668     <common>
 0003:0079266c       _reach_teleport            00c6a66c     <common>
 0003:00792670       _numareacacheupdates       00c6a670     <common>
 0003:00792674       _max_routingcachesize      00c6a674     <common>
 0003:00792678       _routingcachesize          00c6a678     <common>
 0003:0079267c       _numportalcacheupdates     00c6a67c     <common>
 0003:00792680       _midrangeareas             00c6a680     <common>
 0003:00792684       _numclusterareas           00c6a684     <common>
 0003:00792688       _clusterareas              00c6a688     <common>
 0003:007926a0       _aassettings               00c6a6a0     <common>
 0003:00792740       _weightFileList            00c6a740     <common>
 0003:00792940       _botcharacters             00c6a940     <common>
 0003:00792a60       _sourceFiles               00c6aa60     <common>
 0003:00792b60       _globaldefines             00c6ab60     <common>
 0003:00792b64       _numtokens                 00c6ab64     <common>
 0003:00792b68       _libvarlist                00c6ab68     <common>
 0003:00792b6c       _saveroutingcache          00c6ab6c     <common>
 0003:00792b80       _aasworld                  00c6ab80     <common>
 0003:00793d64       _botinputs                 00c6bd64     <common>
 0003:00793d80       _botgoalstates             00c6bd80     <common>
 0003:00793ea0       _botchatstates             00c6bea0     <common>
 0003:00793fc0       _ichatdata                 00c6bfc0     <common>
 0003:007940c0       _weapindex_bfg10k          00c6c0c0     <common>
 0003:007940e0       _modeltypes                00c6c0e0     <common>
 0003:007944e0       _weapindex_rocketlauncher  00c6c4e0     <common>
 0003:007944e4       _cmd_grappleoff            00c6c4e4     <common>
 0003:007944e8       _sv_gravity                00c6c4e8     <common>
 0003:007944ec       _sv_maxstep                00c6c4ec     <common>
 0003:007944f0       _cmd_grappleon             00c6c4f0     <common>
 0003:007944f4       _entitytypemissile         00c6c4f4     <common>
 0003:007944f8       _weapindex_grapple         00c6c4f8     <common>
 0003:007944fc       _offhandgrapple            00c6c4fc     <common>
 0003:00794500       _botmovestates             00c6c500     <common>
 0003:00794604       _sv_maxbarrier             00c6c604     <common>
 0003:00794620       _botimport                 00c6c620     <common>
 0003:00794680       _be_botlib_export          00c6c680     <common>
 0003:007948a0       _botlibglobals             00c6c8a0     <common>
 0003:007948b0       _bot_developer             00c6c8b0     <common>
 0003:007948b4       ___mblcid                  00c6c8b4     <common>
 0003:007948b8       ___ismbcodepage            00c6c8b8     <common>
 0003:007948c0       __mbctype                  00c6c8c0     <common>
 0003:007949c4       ___mbcodepage              00c6c9c4     <common>
 0003:007949d0       ___mbulinfo                00c6c9d0     <common>
 0003:007949e0       __mbcasemap                00c6c9e0     <common>
 0003:00794ae0       __nhandle                  00c6cae0     <common>
 0003:00794b00       ___pioinfo                 00c6cb00     <common>
 0003:00794c00       ___sbh_initialized         00c6cc00     <common>
 0003:00794c04       ___sbh_pHeaderDefer        00c6cc04     <common>
 0003:00794c08       ___sbh_cntHeaderList       00c6cc08     <common>
 0003:00794c0c       ___sbh_pHeaderList         00c6cc0c     <common>
 0003:00794c10       ___sbh_threshold           00c6cc10     <common>
 0003:00794c14       ___sbh_pHeaderScan         00c6cc14     <common>
 0003:00794c18       ___sbh_sizeHeaderList      00c6cc18     <common>
 0003:00794c1c       ___sbh_indGroupDefer       00c6cc1c     <common>
 0003:00794c20       __crtheap                  00c6cc20     <common>
 0003:00794c24       ___active_heap             00c6cc24     <common>
 0003:00794c28       ___piob                    00c6cc28     <common>
 0003:00794c40       __bufin                    00c6cc40     <common>
 0003:00795c40       __nstream                  00c6dc40     <common>
 0003:00795c44       ___use_sse2_mathfcns       00c6dc44     <common>
 0003:00795c48       ___sse2_available          00c6dc48     <common>
 0003:00795c4c       __acmdln                   00c6dc4c     <common>
 0003:00795c50       ___env_initialized         00c6dc50     <common>
 0003:00795c54       ___onexitend               00c6dc54     <common>
 0003:00795c58       ___onexitbegin             00c6dc58     <common>
 0003:00795c5c       ___mbctype_initialized     00c6dc5c     <common>
 0003:00795c60       __setjmpexused             00c6dc60     <common>

 entry point at        0001:000ad0d6

 Static symbols

 0001:00000770       _FloatAsInt                00401770 f   cl_cgame.obj
 0001:000019e0       _CIN_HandleForVideo        004029e0 f   cl_cin.obj
 0001:00001a10       _RllSetupTable             00402a10 f   cl_cin.obj
 0001:00001c70       _move8_32                  00402c70 f   cl_cin.obj
 0001:00001d50       _move4_32                  00402d50 f   cl_cin.obj
 0001:00001d90       _blit8_32                  00402d90 f   cl_cin.obj
 0001:00001e90       _blit4_32                  00402e90 f   cl_cin.obj
 0001:00001ee0       _blit2_32                  00402ee0 f   cl_cin.obj
 0001:00001ef0       _blitVQQuad32fs            00402ef0 f   cl_cin.obj
 0001:00002170       _ROQ_GenYUVTables          00403170 f   cl_cin.obj
 0001:00002210       _yuv_to_rgb                00403210 f   cl_cin.obj
 0001:00002290       _yuv_to_rgb24              00403290 f   cl_cin.obj
 0001:00002310       _decodeCodeBook            00403310 f   cl_cin.obj
 0001:000031b0       _recurseQuad               004041b0 f   cl_cin.obj
 0001:000032b0       _setupQuad                 004042b0 f   cl_cin.obj
 0001:000033c0       _readQuadInfo              004043c0 f   cl_cin.obj
 0001:00003510       _RoQPrepMcomp              00404510 f   cl_cin.obj
 0001:000035c0       _initRoQ                   004045c0 f   cl_cin.obj
 0001:00003600       _RoQ_init                  00404600 f   cl_cin.obj
 0001:000036d0       _RoQShutdown               004046d0 f   cl_cin.obj
 0001:00003d30       _RoQReset                  00404d30 f   cl_cin.obj
 0001:00003df0       _RoQInterrupt              00404df0 f   cl_cin.obj
 0001:00008310       _BigShort                  00409310 f   cl_main.obj
 0001:00008780       _CL_WalkDemoExt            00409780 f   cl_main.obj
 0001:0000a330       _CL_SetServerInfo          0040b330 f   cl_main.obj
 0001:0000a440       _CL_SetServerInfoByAddress 0040b440 f   cl_main.obj
 0001:0000cfd0       _CL_Netchan_Encode         0040dfd0 f   cl_net_chan.obj
 0001:0000d090       _CL_Netchan_Decode         0040e090 f   cl_net_chan.obj
 0001:0000e020       _SCR_DrawChar              0040f020 f   cl_scrn.obj
 0001:0000e420       _SCR_Strlen                0040f420 f   cl_scrn.obj
 0001:0000ea30       _GetClientState            0040fa30 f   cl_ui.obj
 0001:0000ec30       _LAN_ResetPings            0040fc30 f   cl_ui.obj
 0001:0000ec90       _LAN_AddServer             0040fc90 f   cl_ui.obj
 0001:0000ee00       _LAN_RemoveServer          0040fe00 f   cl_ui.obj
 0001:0000ef20       _LAN_GetServerCount        0040ff20 f   cl_ui.obj
 0001:0000ef60       _LAN_GetServerAddressString 0040ff60 f   cl_ui.obj
 0001:0000f020       _LAN_GetServerInfo         00410020 f   cl_ui.obj
 0001:0000f290       _LAN_GetServerPing         00410290 f   cl_ui.obj
 0001:0000f320       _LAN_GetServerPtr          00410320 f   cl_ui.obj
 0001:0000f3a0       _LAN_CompareServers        004103a0 f   cl_ui.obj
 0001:0000f450       _LAN_GetPingQueueCount     00410450 f   cl_ui.obj
 0001:0000f460       _LAN_ClearPing             00410460 f   cl_ui.obj
 0001:0000f470       _LAN_GetPing               00410470 f   cl_ui.obj
 0001:0000f490       _LAN_GetPingInfo           00410490 f   cl_ui.obj
 0001:0000f4a0       _LAN_MarkServerVisible     004104a0 f   cl_ui.obj
 0001:0000f580       _LAN_ServerIsVisible       00410580 f   cl_ui.obj
 0001:0000f620       _CL_GetGlconfig            00410620 f   cl_ui.obj
 0001:0000f640       _GetClipboardData          00410640 f   cl_ui.obj
 0001:0000f670       _Key_KeynumToStringBuf     00410670 f   cl_ui.obj
 0001:0000f690       _Key_GetBindingBuf         00410690 f   cl_ui.obj
 0001:0000f6e0       _GetConfigString           004106e0 f   cl_ui.obj
 0001:0000f720       _FloatAsInt                00410720 f   cl_ui.obj
 0001:0000f7c0       _CLUI_GetCDKey             004107c0 f   cl_ui.obj
 0001:0000f830       _CLUI_SetCDKey             00410830 f   cl_ui.obj
 0001:000118e0       _CM_SignbitsForNormal      004128e0 f   cm_patch.obj
 0001:00011920       _VectorLength              00412920 f   cm_patch.obj
 0001:00011950       _CM_NeedsSubdivision       00412950 f   cm_patch.obj
 0001:00011a20       _CM_Subdivide              00412a20 f   cm_patch.obj
 0001:00011ab0       _CM_TransposeGrid          00412ab0 f   cm_patch.obj
 0001:00011c10       _CrossProduct              00412c10 f   cm_patch.obj
 0001:00011c40       _CM_SetGridWrapWidth       00412c40 f   cm_patch.obj
 0001:00011ce0       _CM_SubdivideGridColumns   00412ce0 f   cm_patch.obj
 0001:00012010       _CM_ComparePoints          00413010 f   cm_patch.obj
 0001:00012080       _CM_RemoveDegenerateColumns 00413080 f   cm_patch.obj
 0001:00012410       _CM_PointOnPlaneSide       00413410 f   cm_patch.obj
 0001:00012470       _CM_GridPlane              00413470 f   cm_patch.obj
 0001:000124b0       _CM_SetBorderInward        004134b0 f   cm_patch.obj
 0001:00012900       _CM_ValidateFacet          00413900 f   cm_patch.obj
 0001:00014360       _CM_PlaneFromPoints        00415360 f   cm_patch.obj
 0001:00014400       _CM_FindPlane              00415400 f   cm_patch.obj
 0001:000145c0       _CM_EdgePlaneNum           004155c0 f   cm_patch.obj
 0001:000147c0       _CM_PatchCollideFromGrid   004157c0 f   cm_patch.obj
 0001:00015510       _VectorLength              00416510 f   cm_polylib.obj
 0001:00015690       _CrossProduct              00416690 f   cm_polylib.obj
 0001:00017630       _VectorLengthSquared       00418630 f   cm_trace.obj
 0001:000176d0       _VectorInverse             004186d0 f   cm_trace.obj
 0001:0001b950       _Hunk_SwapBanks            0041c950 f   common.obj
 0001:0001bb40       _Com_Crash_f               0041cb40 f   common.obj
 0001:0001bb50       _Com_WriteCDKey            0041cb50 f   common.obj
 0001:0001c0b0       _FindMatches               0041d0b0 f   common.obj
 0001:0001c140       _PrintMatches              0041d140 f   common.obj
 0001:0001c180       _keyConcatArgs             0041d180 f   common.obj
 0001:0001c250       _ConcatRemaining           0041d250 f   common.obj
 0001:0001d130       _Com_Error_f               0041e130 f   common.obj
 0001:0001d160       _Com_Freeze_f              0041e160 f   common.obj
 0001:0001dfa0       _generateHashValue         0041efa0 f   cvar.obj
 0001:0001dfe0       _Cvar_ValidateString       0041efe0 f   cvar.obj
 0001:0001e020       _Cvar_FindVar              0041f020 f   cvar.obj
 0001:0001efe0       _FS_HashFileName           0041ffe0 f   files.obj
 0001:0001f040       _FS_HandleForFile          00420040 f   files.obj
 0001:0001f080       _FS_FileForHandle          00420080 f   files.obj
 0001:0001f140       _FS_ReplaceSeparators      00420140 f   files.obj
 0001:0001f210       _FS_CreatePath             00420210 f   files.obj
 0001:0001f280       _FS_CopyFile               00420280 f   files.obj
 0001:0001f390       _FS_Remove                 00420390 f   files.obj
 0001:000207c0       _FS_LoadZipFile            004217c0 f   files.obj
 0001:00020af0       _FS_ReturnPath             00421af0 f   files.obj
 0001:00020b40       _FS_AddFileToList          00421b40 f   files.obj
 0001:00020f40       _Sys_CountFileList         00421f40 f   files.obj
 0001:00020f60       _Sys_ConcatenateFileLists  00421f60 f   files.obj
 0001:000217c0       _paksort                   004227c0 f   files.obj
 0001:000217e0       _FS_AddGameDirectory       004227e0 f   files.obj
 0001:00021ca0       _FS_ReorderPurePaks        00422ca0 f   files.obj
 0001:00021d10       _FS_Startup                00422d10 f   files.obj
 0001:00022c10       _FS_SetRestrictions        00423c10 f   files.obj
 0001:00023090       _add_bit                   00424090 f   huffman.obj
 0001:000230d0       _get_bit                   004240d0 f   huffman.obj
 0001:00023100       _get_ppnode                00424100 f   huffman.obj
 0001:00023130       _free_ppnode               00424130 f   huffman.obj
 0001:00023140       _swap                      00424140 f   huffman.obj
 0001:00023190       _swaplist                  00424190 f   huffman.obj
 0001:000231f0       _increment                 004241f0 f   huffman.obj
 0001:00023550       _send                      00424550 f   huffman.obj
 0001:00023c50       _Encode                    00424c50 f   md4.obj
 0001:00023c90       _Decode                    00424c90 f   md4.obj
 0001:00023cd0       _MD4Transform              00424cd0 f   md4.obj
 0001:000269b0       _BigShort                  004279b0 f   net_chan.obj
 0001:00027640       _VectorLength              00428640 f   q_math.obj
 0001:00027930       _CrossProduct              00428930 f   q_math.obj
 0001:00028de0       _SkipWhitespace            00429de0 f   q_shared.obj
 0001:0002a3b0       _VectorLengthSquared       0042b3b0 f   snd_dma.obj
 0001:0002a3d0       _DistanceSquared           0042b3d0 f   snd_dma.obj
 0001:0002a4f0       _S_HashSFXName             0042b4f0 f   snd_dma.obj
 0001:0002a540       _S_FindName                0042b540 f   snd_dma.obj
 0001:0002c590       _GetLittleShort            0042d590 f   snd_mem.obj
 0001:0002c5b0       _GetLittleLong             0042d5b0 f   snd_mem.obj
 0001:0002c5e0       _FindNextChunk             0042d5e0 f   snd_mem.obj
 0001:0002c660       _FindChunk                 0042d660 f   snd_mem.obj
 0001:0002c670       _GetWavinfo                0042d670 f   snd_mem.obj
 0001:0002c8a0       _ResampleSfx               0042d8a0 f   snd_mem.obj
 0001:0002c960       _ResampleSfxRaw            0042d960 f   snd_mem.obj
 0001:0002cda0       _S_PaintChannelFrom16      0042dda0 f   snd_mix.obj
 0001:0002e520       _CrossProduct              0042f520 f   sv_bot.obj
 0001:0002f020       _SV_GetPlayerByName        00430020 f   sv_ccmds.obj
 0001:0002f0f0       _BigShort                  004300f0 f   sv_ccmds.obj
 0001:0002f100       _SV_GetPlayerByNum         00430100 f   sv_ccmds.obj
 0001:0002f1c0       _SV_Map_f                  004301c0 f   sv_ccmds.obj
 0001:0002f310       _SV_MapRestart_f           00430310 f   sv_ccmds.obj
 0001:0002f590       _SV_Kick_f                 00430590 f   sv_ccmds.obj
 0001:0002f6f0       _SV_Ban_f                  004306f0 f   sv_ccmds.obj
 0001:0002f870       _SV_BanNum_f               00430870 f   sv_ccmds.obj
 0001:0002f9f0       _SV_KickNum_f              004309f0 f   sv_ccmds.obj
 0001:0002fa70       _SV_Status_f               00430a70 f   sv_ccmds.obj
 0001:0002fc80       _SV_ConSay_f               00430c80 f   sv_ccmds.obj
 0001:0002fd50       _SV_Serverinfo_f           00430d50 f   sv_ccmds.obj
 0001:0002fd70       _SV_Systeminfo_f           00430d70 f   sv_ccmds.obj
 0001:0002fd90       _SV_DumpUser_f             00430d90 f   sv_ccmds.obj
 0001:0002fdf0       _SV_KillServer_f           00430df0 f   sv_ccmds.obj
 0001:0002ff40       _BigShort                  00430f40 f   sv_client.obj
 0001:00030480       _SV_CloseDownload          00431480 f   sv_client.obj
 0001:00030a60       _SV_ResetPureClient_f      00431a60 f   sv_client.obj
 0001:00030cd0       _SV_UpdateUserinfo_f       00431cd0 f   sv_client.obj
 0001:00031510       _SV_Disconnect_f           00432510 f   sv_client.obj
 0001:00031530       _SV_VerifyPaks_f           00432530 f   sv_client.obj
 0001:000317b0       _SV_ClientCommand          004327b0 f   sv_client.obj
 0001:000318b0       _SV_UserMove               004328b0 f   sv_client.obj
 0001:00032a40       _FloatAsInt                00433a40 f   sv_game.obj
 0001:00034990       _SV_InitGameVM             00435990 f   sv_game.obj
 0001:00035cb0       _BigShort                  00436cb0 f   sv_main.obj
 0001:00036ec0       _SV_Netchan_Encode         00437ec0 f   sv_net_chan.obj
 0001:00036f60       _SV_Netchan_Decode         00437f60 f   sv_net_chan.obj
 0001:000371b0       _SV_EmitPacketEntities     004381b0 f   sv_snapshot.obj
 0001:000372d0       _VectorLengthSquared       004382d0 f   sv_snapshot.obj
 0001:000372f0       _SV_WriteSnapshotToClient  004382f0 f   sv_snapshot.obj
 0001:000374b0       _SV_QsortEntityNumbers     004384b0 f   sv_snapshot.obj
 0001:000374f0       _SV_AddEntToSnapshot       004384f0 f   sv_snapshot.obj
 0001:00037520       _SV_AddEntitiesVisibleFromPoint 00438520 f   sv_snapshot.obj
 0001:00037800       _SV_BuildClientSnapshot    00438800 f   sv_snapshot.obj
 0001:000379e0       _SV_RateMsec               004389e0 f   sv_snapshot.obj
 0001:000389d0       _unzlocal_getShort         004399d0 f   unzip.obj
 0001:00038a00       _unzlocal_getLong          00439a00 f   unzip.obj
 0001:00038a20       _strcmpcasenosensitive_internal 00439a20 f   unzip.obj
 0001:00038df0       _unzlocal_DosDateToTmuDate 00439df0 f   unzip.obj
 0001:00038e40       _unzlocal_GetCurrentFileInfoInternal 00439e40 f   unzip.obj
 0001:000394a0       _unzlocal_CheckCurrentFileCoherencyHeader 0043a4a0 f   unzip.obj
 0001:000397b0       _inflate_flush             0043a7b0 f   unzip.obj
 0001:000398b0       _huft_build                0043a8b0 f   unzip.obj
 0001:00039da0       _inflate_trees_bits        0043ada0 f   unzip.obj
 0001:00039e40       _inflate_trees_dynamic     0043ae40 f   unzip.obj
 0001:00039fc0       _inflate_trees_fixed       0043afc0 f   unzip.obj
 0001:00039ff0       _inflate_fast              0043aff0 f   unzip.obj
 0001:0003a360       _inflate_codes_new         0043b360 f   unzip.obj
 0001:0003a3a0       _inflate_codes             0043b3a0 f   unzip.obj
 0001:0003aa90       _inflate_codes_free        0043ba90 f   unzip.obj
 0001:0003aaa0       _adler32                   0043baa0 f   unzip.obj
 0001:0003abd0       _zcalloc                   0043bbd0 f   unzip.obj
 0001:0003abf0       _zcfree                    0043bbf0 f   unzip.obj
 0001:0003ac00       _inflate_blocks_reset      0043bc00 f   unzip.obj
 0001:0003ac70       _inflate_blocks_new        0043bc70 f   unzip.obj
 0001:0003ad00       _inflate_blocks            0043bd00 f   unzip.obj
 0001:0003b860       _inflate_blocks_free       0043c860 f   unzip.obj
 0001:0003b8e0       _inflateReset              0043c8e0 f   unzip.obj
 0001:0003b920       _inflateEnd                0043c920 f   unzip.obj
 0001:0003b970       _inflateInit2_             0043c970 f   unzip.obj
 0001:0003ba70       _inflate                   0043ca70 f   unzip.obj
 0001:0003c790       _VM_ProfileSort            0043d790 f   vm.obj
 0001:0003d780       _Constant4                 0043e780 f   vm_x86.obj
 0001:0003d7c0       _Constant1                 0043e7c0 f   vm_x86.obj
 0001:0003d7e0       _Emit1                     0043e7e0 f   vm_x86.obj
 0001:0003d810       _Emit4                     0043e810 f   vm_x86.obj
 0001:0003d850       _Hex                       0043e850 f   vm_x86.obj
 0001:0003d890       _EmitString                0043e890 f   vm_x86.obj
 0001:0003d950       _EmitCommand               0043e950 f   vm_x86.obj
 0001:0003d990       _EmitAddEDI4               0043e990 f   vm_x86.obj
 0001:0003da10       _EmitMovEAXEDI             0043ea10 f   vm_x86.obj
 0001:0003fc50       _MIDI_NoteOff              00440c50 f   win_input.obj
 0001:0003fc80       _MIDI_NoteOn               00440c80 f   win_input.obj
 0001:0003fce0       _MidiInProc@20             00440ce0 f   win_input.obj
 0001:0003fd50       _MidiInfo_f                00440d50 f   win_input.obj
 0001:0003fe80       _IN_StartupMIDI            00440e80 f   win_input.obj
 0001:0003ff50       _IN_ShutdownMIDI           00440f50 f   win_input.obj
 0001:00040900       _strgtr                    00441900 f   win_main.obj
 0001:00042a30       _NET_GetCvars              00443a30 f   win_net.obj
 0001:00042da0       _CPUID                     00443da0 f   win_shared.obj
 0001:00042de0       _IsPentium                 00443de0 f   win_shared.obj
 0001:00042e20       _Is3DNOW                   00443e20 f   win_shared.obj
 0001:00042ed0       _IsKNI                     00443ed0 f   win_shared.obj
 0001:00042f00       _IsMMX                     00443f00 f   win_shared.obj
 0001:00043010       _DSoundError               00444010 f   win_snd.obj
 0001:00043a80       _ConWndProc@16             00444a80 f   win_syscon.obj
 0001:000441c0       _WIN_DisableAltTab         004451c0 f   win_wndproc.obj
 0001:00044220       _WIN_EnableAltTab          00445220 f   win_wndproc.obj
 0001:00044280       _VID_AppActivate           00445280 f   win_wndproc.obj
 0001:000442d0       _MapKey                    004452d0 f   win_wndproc.obj
 0001:00044bb0       _AssertCvarRange           00445bb0 f   renderer:tr_init.obj
 0001:00044ef0       _R_ModeList_f              00445ef0 f   renderer:tr_init.obj
 0001:00045930       _GfxInfo_f                 00446930 f   renderer:tr_init.obj
 0001:00046890       _InitOpenGL                00447890 f   renderer:tr_init.obj
 0001:000471b0       _VectorLength              004481b0 f   renderer:tr_main.obj
 0001:000471e0       _VectorLengthSquared       004481e0 f   renderer:tr_main.obj
 0001:00047200       _CrossProduct              00448200 f   renderer:tr_main.obj
 0001:000479a0       _SetFarClip                004489a0 f   renderer:tr_main.obj
 0001:00048760       _IsMirror                  00449760 f   renderer:tr_main.obj
 0001:00048910       _shortsort                 00449910 f   renderer:tr_main.obj
 0001:00048ea0       _SurfIsOffscreen           00449ea0 f   renderer:tr_main.obj
 0001:00049460       _BooleanToString           0044a460 f   renderer:win_qgl.obj
 0001:00049480       _FuncToString              0044a480 f   renderer:win_qgl.obj
 0001:000494f0       _PrimToString              0044a4f0 f   renderer:win_qgl.obj
 0001:00049730       _CapToString               0044a730 f   renderer:win_qgl.obj
 0001:00049880       _TypeToString              0044a880 f   renderer:win_qgl.obj
 0001:00049900       _logAccum@8                0044a900 f   renderer:win_qgl.obj
 0001:00049920       _logAlphaFunc@8            0044a920 f   renderer:win_qgl.obj
 0001:00049960       _logAreTexturesResident@12 0044a960 f   renderer:win_qgl.obj
 0001:00049980       _logArrayElement@4         0044a980 f   renderer:win_qgl.obj
 0001:000499a0       _logBegin@4                0044a9a0 f   renderer:win_qgl.obj
 0001:000499d0       _logBindTexture@8          0044a9d0 f   renderer:win_qgl.obj
 0001:00049a00       _logBitmap@28              0044aa00 f   renderer:win_qgl.obj
 0001:00049a20       _BlendToName               0044aa20 f   renderer:win_qgl.obj
 0001:00049b30       _logBlendFunc@8            0044ab30 f   renderer:win_qgl.obj
 0001:00049ba0       _logCallList@4             0044aba0 f   renderer:win_qgl.obj
 0001:00049bd0       _logCallLists@12           0044abd0 f   renderer:win_qgl.obj
 0001:00049bf0       _logClear@4                0044abf0 f   renderer:win_qgl.obj
 0001:00049ca0       _logClearAccum@16          0044aca0 f   renderer:win_qgl.obj
 0001:00049cc0       _logClearColor@16          0044acc0 f   renderer:win_qgl.obj
 0001:00049ce0       _logClearDepth@8           0044ace0 f   renderer:win_qgl.obj
 0001:00049d10       _logClearIndex@4           0044ad10 f   renderer:win_qgl.obj
 0001:00049d30       _logClearStencil@4         0044ad30 f   renderer:win_qgl.obj
 0001:00049d60       _logClipPlane@8            0044ad60 f   renderer:win_qgl.obj
 0001:00049d80       _logColor3b@12             0044ad80 f   renderer:win_qgl.obj
 0001:00049da0       _logColor3bv@4             0044ada0 f   renderer:win_qgl.obj
 0001:00049dc0       _logColor3d@24             0044adc0 f   renderer:win_qgl.obj
 0001:00049e00       _logColor3dv@4             0044ae00 f   renderer:win_qgl.obj
 0001:00049e20       _logColor3f@12             0044ae20 f   renderer:win_qgl.obj
 0001:00049e40       _logColor3fv@4             0044ae40 f   renderer:win_qgl.obj
 0001:00049e60       _logColor3i@12             0044ae60 f   renderer:win_qgl.obj
 0001:00049e80       _logColor3iv@4             0044ae80 f   renderer:win_qgl.obj
 0001:00049ea0       _logColor3s@12             0044aea0 f   renderer:win_qgl.obj
 0001:00049ec0       _logColor3sv@4             0044aec0 f   renderer:win_qgl.obj
 0001:00049ee0       _logColor3ub@12            0044aee0 f   renderer:win_qgl.obj
 0001:00049f00       _logColor3ubv@4            0044af00 f   renderer:win_qgl.obj
 0001:00049f20       _logColor3ui@12            0044af20 f   renderer:win_qgl.obj
 0001:00049f40       _logColor3uiv@4            0044af40 f   renderer:win_qgl.obj
 0001:00049f60       _logColor3us@12            0044af60 f   renderer:win_qgl.obj
 0001:00049f80       _logColor3usv@4            0044af80 f   renderer:win_qgl.obj
 0001:00049fa0       _logColor4b@16             0044afa0 f   renderer:win_qgl.obj
 0001:00049fc0       _logColor4bv@4             0044afc0 f   renderer:win_qgl.obj
 0001:00049fe0       _logColor4d@32             0044afe0 f   renderer:win_qgl.obj
 0001:0004a020       _logColor4dv@4             0044b020 f   renderer:win_qgl.obj
 0001:0004a040       _logColor4f@16             0044b040 f   renderer:win_qgl.obj
 0001:0004a080       _logColor4fv@4             0044b080 f   renderer:win_qgl.obj
 0001:0004a0c0       _logColor4i@16             0044b0c0 f   renderer:win_qgl.obj
 0001:0004a0e0       _logColor4iv@4             0044b0e0 f   renderer:win_qgl.obj
 0001:0004a100       _logColor4s@16             0044b100 f   renderer:win_qgl.obj
 0001:0004a120       _logColor4sv@4             0044b120 f   renderer:win_qgl.obj
 0001:0004a140       _logColor4ub@16            0044b140 f   renderer:win_qgl.obj
 0001:0004a160       _logColor4ubv@4            0044b160 f   renderer:win_qgl.obj
 0001:0004a180       _logColor4ui@16            0044b180 f   renderer:win_qgl.obj
 0001:0004a1a0       _logColor4uiv@4            0044b1a0 f   renderer:win_qgl.obj
 0001:0004a1c0       _logColor4us@16            0044b1c0 f   renderer:win_qgl.obj
 0001:0004a1e0       _logColor4usv@4            0044b1e0 f   renderer:win_qgl.obj
 0001:0004a200       _logColorMask@16           0044b200 f   renderer:win_qgl.obj
 0001:0004a220       _logColorMaterial@8        0044b220 f   renderer:win_qgl.obj
 0001:0004a240       _logColorPointer@16        0044b240 f   renderer:win_qgl.obj
 0001:0004a280       _logCopyPixels@20          0044b280 f   renderer:win_qgl.obj
 0001:0004a2a0       _logCopyTexImage1D@28      0044b2a0 f   renderer:win_qgl.obj
 0001:0004a2c0       _logCopyTexImage2D@32      0044b2c0 f   renderer:win_qgl.obj
 0001:0004a2e0       _logCopyTexSubImage1D@24   0044b2e0 f   renderer:win_qgl.obj
 0001:0004a300       _logCopyTexSubImage2D@32   0044b300 f   renderer:win_qgl.obj
 0001:0004a320       _logCullFace@4             0044b320 f   renderer:win_qgl.obj
 0001:0004a360       _logDeleteLists@8          0044b360 f   renderer:win_qgl.obj
 0001:0004a380       _logDeleteTextures@8       0044b380 f   renderer:win_qgl.obj
 0001:0004a3a0       _logDepthFunc@4            0044b3a0 f   renderer:win_qgl.obj
 0001:0004a3d0       _logDepthMask@4            0044b3d0 f   renderer:win_qgl.obj
 0001:0004a410       _logDepthRange@16          0044b410 f   renderer:win_qgl.obj
 0001:0004a450       _logDisable@4              0044b450 f   renderer:win_qgl.obj
 0001:0004a480       _logDisableClientState@4   0044b480 f   renderer:win_qgl.obj
 0001:0004a4b0       _logDrawArrays@12          0044b4b0 f   renderer:win_qgl.obj
 0001:0004a4d0       _logDrawBuffer@4           0044b4d0 f   renderer:win_qgl.obj
 0001:0004a4f0       _logDrawElements@16        0044b4f0 f   renderer:win_qgl.obj
 0001:0004a540       _logDrawPixels@20          0044b540 f   renderer:win_qgl.obj
 0001:0004a560       _logEdgeFlag@4             0044b560 f   renderer:win_qgl.obj
 0001:0004a580       _logEdgeFlagPointer@8      0044b580 f   renderer:win_qgl.obj
 0001:0004a5a0       _logEdgeFlagv@4            0044b5a0 f   renderer:win_qgl.obj
 0001:0004a5c0       _logEnable@4               0044b5c0 f   renderer:win_qgl.obj
 0001:0004a5f0       _logEnableClientState@4    0044b5f0 f   renderer:win_qgl.obj
 0001:0004a620       _logEnd@0                  0044b620 f   renderer:win_qgl.obj
 0001:0004a640       _logEndList@0              0044b640 f   renderer:win_qgl.obj
 0001:0004a660       _logEvalCoord1d@8          0044b660 f   renderer:win_qgl.obj
 0001:0004a680       _logEvalCoord1dv@4         0044b680 f   renderer:win_qgl.obj
 0001:0004a6a0       _logEvalCoord1f@4          0044b6a0 f   renderer:win_qgl.obj
 0001:0004a6c0       _logEvalCoord1fv@4         0044b6c0 f   renderer:win_qgl.obj
 0001:0004a6e0       _logEvalCoord2d@16         0044b6e0 f   renderer:win_qgl.obj
 0001:0004a710       _logEvalCoord2dv@4         0044b710 f   renderer:win_qgl.obj
 0001:0004a730       _logEvalCoord2f@8          0044b730 f   renderer:win_qgl.obj
 0001:0004a750       _logEvalCoord2fv@4         0044b750 f   renderer:win_qgl.obj
 0001:0004a770       _logEvalMesh1@12           0044b770 f   renderer:win_qgl.obj
 0001:0004a790       _logEvalMesh2@20           0044b790 f   renderer:win_qgl.obj
 0001:0004a7b0       _logEvalPoint1@4           0044b7b0 f   renderer:win_qgl.obj
 0001:0004a7d0       _logEvalPoint2@8           0044b7d0 f   renderer:win_qgl.obj
 0001:0004a7f0       _logFeedbackBuffer@12      0044b7f0 f   renderer:win_qgl.obj
 0001:0004a810       _logFinish@0               0044b810 f   renderer:win_qgl.obj
 0001:0004a830       _logFlush@0                0044b830 f   renderer:win_qgl.obj
 0001:0004a850       _logFogf@8                 0044b850 f   renderer:win_qgl.obj
 0001:0004a870       _logFogfv@8                0044b870 f   renderer:win_qgl.obj
 0001:0004a890       _logFogi@8                 0044b890 f   renderer:win_qgl.obj
 0001:0004a8b0       _logFogiv@8                0044b8b0 f   renderer:win_qgl.obj
 0001:0004a8d0       _logFrontFace@4            0044b8d0 f   renderer:win_qgl.obj
 0001:0004a8f0       _logFrustum@48             0044b8f0 f   renderer:win_qgl.obj
 0001:0004a940       _logGenLists@4             0044b940 f   renderer:win_qgl.obj
 0001:0004a960       _logGenTextures@8          0044b960 f   renderer:win_qgl.obj
 0001:0004a980       _logGetBooleanv@8          0044b980 f   renderer:win_qgl.obj
 0001:0004a9a0       _logGetClipPlane@8         0044b9a0 f   renderer:win_qgl.obj
 0001:0004a9c0       _logGetDoublev@8           0044b9c0 f   renderer:win_qgl.obj
 0001:0004a9e0       _logGetError@0             0044b9e0 f   renderer:win_qgl.obj
 0001:0004aa00       _logGetFloatv@8            0044ba00 f   renderer:win_qgl.obj
 0001:0004aa20       _logGetIntegerv@8          0044ba20 f   renderer:win_qgl.obj
 0001:0004aa40       _logGetLightfv@12          0044ba40 f   renderer:win_qgl.obj
 0001:0004aa60       _logGetLightiv@12          0044ba60 f   renderer:win_qgl.obj
 0001:0004aa80       _logGetMapdv@12            0044ba80 f   renderer:win_qgl.obj
 0001:0004aaa0       _logGetMapfv@12            0044baa0 f   renderer:win_qgl.obj
 0001:0004aac0       _logGetMapiv@12            0044bac0 f   renderer:win_qgl.obj
 0001:0004aae0       _logGetMaterialfv@12       0044bae0 f   renderer:win_qgl.obj
 0001:0004ab00       _logGetMaterialiv@12       0044bb00 f   renderer:win_qgl.obj
 0001:0004ab20       _logGetPixelMapfv@8        0044bb20 f   renderer:win_qgl.obj
 0001:0004ab40       _logGetPixelMapuiv@8       0044bb40 f   renderer:win_qgl.obj
 0001:0004ab60       _logGetPixelMapusv@8       0044bb60 f   renderer:win_qgl.obj
 0001:0004ab80       _logGetPointerv@8          0044bb80 f   renderer:win_qgl.obj
 0001:0004aba0       _logGetPolygonStipple@4    0044bba0 f   renderer:win_qgl.obj
 0001:0004abc0       _logGetString@4            0044bbc0 f   renderer:win_qgl.obj
 0001:0004abe0       _logGetTexEnvfv@12         0044bbe0 f   renderer:win_qgl.obj
 0001:0004ac00       _logGetTexEnviv@12         0044bc00 f   renderer:win_qgl.obj
 0001:0004ac20       _logGetTexGendv@12         0044bc20 f   renderer:win_qgl.obj
 0001:0004ac40       _logGetTexGenfv@12         0044bc40 f   renderer:win_qgl.obj
 0001:0004ac60       _logGetTexGeniv@12         0044bc60 f   renderer:win_qgl.obj
 0001:0004ac80       _logGetTexImage@20         0044bc80 f   renderer:win_qgl.obj
 0001:0004aca0       _logGetTexLevelParameterfv@16 0044bca0 f   renderer:win_qgl.obj
 0001:0004acc0       _logGetTexLevelParameteriv@16 0044bcc0 f   renderer:win_qgl.obj
 0001:0004ace0       _logGetTexParameterfv@12   0044bce0 f   renderer:win_qgl.obj
 0001:0004ad00       _logGetTexParameteriv@12   0044bd00 f   renderer:win_qgl.obj
 0001:0004ad20       _logHint@8                 0044bd20 f   renderer:win_qgl.obj
 0001:0004ad50       _logIndexMask@4            0044bd50 f   renderer:win_qgl.obj
 0001:0004ad70       _logIndexPointer@12        0044bd70 f   renderer:win_qgl.obj
 0001:0004ad90       _logIndexd@8               0044bd90 f   renderer:win_qgl.obj
 0001:0004adb0       _logIndexdv@4              0044bdb0 f   renderer:win_qgl.obj
 0001:0004add0       _logIndexf@4               0044bdd0 f   renderer:win_qgl.obj
 0001:0004adf0       _logIndexfv@4              0044bdf0 f   renderer:win_qgl.obj
 0001:0004ae10       _logIndexi@4               0044be10 f   renderer:win_qgl.obj
 0001:0004ae30       _logIndexiv@4              0044be30 f   renderer:win_qgl.obj
 0001:0004ae50       _logIndexs@4               0044be50 f   renderer:win_qgl.obj
 0001:0004ae70       _logIndexsv@4              0044be70 f   renderer:win_qgl.obj
 0001:0004ae90       _logIndexub@4              0044be90 f   renderer:win_qgl.obj
 0001:0004aeb0       _logIndexubv@4             0044beb0 f   renderer:win_qgl.obj
 0001:0004aed0       _logInitNames@0            0044bed0 f   renderer:win_qgl.obj
 0001:0004aef0       _logInterleavedArrays@12   0044bef0 f   renderer:win_qgl.obj
 0001:0004af10       _logIsEnabled@4            0044bf10 f   renderer:win_qgl.obj
 0001:0004af30       _logIsList@4               0044bf30 f   renderer:win_qgl.obj
 0001:0004af50       _logIsTexture@4            0044bf50 f   renderer:win_qgl.obj
 0001:0004af70       _logLightModelf@8          0044bf70 f   renderer:win_qgl.obj
 0001:0004af90       _logLightModelfv@8         0044bf90 f   renderer:win_qgl.obj
 0001:0004afb0       _logLightModeli@8          0044bfb0 f   renderer:win_qgl.obj
 0001:0004afd0       _logLightModeliv@8         0044bfd0 f   renderer:win_qgl.obj
 0001:0004aff0       _logLightf@12              0044bff0 f   renderer:win_qgl.obj
 0001:0004b010       _logLightfv@12             0044c010 f   renderer:win_qgl.obj
 0001:0004b030       _logLighti@12              0044c030 f   renderer:win_qgl.obj
 0001:0004b050       _logLightiv@12             0044c050 f   renderer:win_qgl.obj
 0001:0004b070       _logLineStipple@8          0044c070 f   renderer:win_qgl.obj
 0001:0004b090       _logLineWidth@4            0044c090 f   renderer:win_qgl.obj
 0001:0004b0b0       _logListBase@4             0044c0b0 f   renderer:win_qgl.obj
 0001:0004b0d0       _logLoadIdentity@0         0044c0d0 f   renderer:win_qgl.obj
 0001:0004b0f0       _logLoadMatrixd@4          0044c0f0 f   renderer:win_qgl.obj
 0001:0004b110       _logLoadMatrixf@4          0044c110 f   renderer:win_qgl.obj
 0001:0004b130       _logLoadName@4             0044c130 f   renderer:win_qgl.obj
 0001:0004b150       _logLogicOp@4              0044c150 f   renderer:win_qgl.obj
 0001:0004b170       _logMap1d@32               0044c170 f   renderer:win_qgl.obj
 0001:0004b1c0       _logMap1f@24               0044c1c0 f   renderer:win_qgl.obj
 0001:0004b1e0       _logMap2d@56               0044c1e0 f   renderer:win_qgl.obj
 0001:0004b240       _logMap2f@40               0044c240 f   renderer:win_qgl.obj
 0001:0004b260       _logMapGrid1d@20           0044c260 f   renderer:win_qgl.obj
 0001:0004b290       _logMapGrid1f@12           0044c290 f   renderer:win_qgl.obj
 0001:0004b2b0       _logMapGrid2d@40           0044c2b0 f   renderer:win_qgl.obj
 0001:0004b300       _logMapGrid2f@24           0044c300 f   renderer:win_qgl.obj
 0001:0004b320       _logMaterialf@12           0044c320 f   renderer:win_qgl.obj
 0001:0004b340       _logMaterialfv@12          0044c340 f   renderer:win_qgl.obj
 0001:0004b360       _logMateriali@12           0044c360 f   renderer:win_qgl.obj
 0001:0004b380       _logMaterialiv@12          0044c380 f   renderer:win_qgl.obj
 0001:0004b3a0       _logMatrixMode@4           0044c3a0 f   renderer:win_qgl.obj
 0001:0004b3c0       _logMultMatrixd@4          0044c3c0 f   renderer:win_qgl.obj
 0001:0004b3e0       _logMultMatrixf@4          0044c3e0 f   renderer:win_qgl.obj
 0001:0004b400       _logNewList@8              0044c400 f   renderer:win_qgl.obj
 0001:0004b420       _logNormal3b@12            0044c420 f   renderer:win_qgl.obj
 0001:0004b440       _logNormal3bv@4            0044c440 f   renderer:win_qgl.obj
 0001:0004b460       _logNormal3d@24            0044c460 f   renderer:win_qgl.obj
 0001:0004b4a0       _logNormal3dv@4            0044c4a0 f   renderer:win_qgl.obj
 0001:0004b4c0       _logNormal3f@12            0044c4c0 f   renderer:win_qgl.obj
 0001:0004b4e0       _logNormal3fv@4            0044c4e0 f   renderer:win_qgl.obj
 0001:0004b500       _logNormal3i@12            0044c500 f   renderer:win_qgl.obj
 0001:0004b520       _logNormal3iv@4            0044c520 f   renderer:win_qgl.obj
 0001:0004b540       _logNormal3s@12            0044c540 f   renderer:win_qgl.obj
 0001:0004b560       _logNormal3sv@4            0044c560 f   renderer:win_qgl.obj
 0001:0004b580       _logNormalPointer@12       0044c580 f   renderer:win_qgl.obj
 0001:0004b5a0       _logOrtho@48               0044c5a0 f   renderer:win_qgl.obj
 0001:0004b5f0       _logPassThrough@4          0044c5f0 f   renderer:win_qgl.obj
 0001:0004b610       _logPixelMapfv@12          0044c610 f   renderer:win_qgl.obj
 0001:0004b630       _logPixelMapuiv@12         0044c630 f   renderer:win_qgl.obj
 0001:0004b650       _logPixelMapusv@12         0044c650 f   renderer:win_qgl.obj
 0001:0004b670       _logPixelStoref@8          0044c670 f   renderer:win_qgl.obj
 0001:0004b690       _logPixelStorei@8          0044c690 f   renderer:win_qgl.obj
 0001:0004b6b0       _logPixelTransferf@8       0044c6b0 f   renderer:win_qgl.obj
 0001:0004b6d0       _logPixelTransferi@8       0044c6d0 f   renderer:win_qgl.obj
 0001:0004b6f0       _logPixelZoom@8            0044c6f0 f   renderer:win_qgl.obj
 0001:0004b710       _logPointSize@4            0044c710 f   renderer:win_qgl.obj
 0001:0004b730       _logPolygonMode@8          0044c730 f   renderer:win_qgl.obj
 0001:0004b760       _logPolygonOffset@8        0044c760 f   renderer:win_qgl.obj
 0001:0004b780       _logPolygonStipple@4       0044c780 f   renderer:win_qgl.obj
 0001:0004b7a0       _logPopAttrib@0            0044c7a0 f   renderer:win_qgl.obj
 0001:0004b7c0       _logPopClientAttrib@0      0044c7c0 f   renderer:win_qgl.obj
 0001:0004b7e0       _logPopMatrix@0            0044c7e0 f   renderer:win_qgl.obj
 0001:0004b800       _logPopName@0              0044c800 f   renderer:win_qgl.obj
 0001:0004b820       _logPrioritizeTextures@12  0044c820 f   renderer:win_qgl.obj
 0001:0004b840       _logPushAttrib@4           0044c840 f   renderer:win_qgl.obj
 0001:0004b860       _logPushClientAttrib@4     0044c860 f   renderer:win_qgl.obj
 0001:0004b880       _logPushMatrix@0           0044c880 f   renderer:win_qgl.obj
 0001:0004b8a0       _logPushName@4             0044c8a0 f   renderer:win_qgl.obj
 0001:0004b8c0       _logRasterPos2d@16         0044c8c0 f   renderer:win_qgl.obj
 0001:0004b8f0       _logRasterPos2dv@4         0044c8f0 f   renderer:win_qgl.obj
 0001:0004b910       _logRasterPos2f@8          0044c910 f   renderer:win_qgl.obj
 0001:0004b930       _logRasterPos2fv@4         0044c930 f   renderer:win_qgl.obj
 0001:0004b950       _logRasterPos2i@8          0044c950 f   renderer:win_qgl.obj
 0001:0004b970       _logRasterPos2iv@4         0044c970 f   renderer:win_qgl.obj
 0001:0004b990       _logRasterPos2s@8          0044c990 f   renderer:win_qgl.obj
 0001:0004b9b0       _logRasterPos2sv@4         0044c9b0 f   renderer:win_qgl.obj
 0001:0004b9d0       _logRasterPos3d@24         0044c9d0 f   renderer:win_qgl.obj
 0001:0004ba10       _logRasterPos3dv@4         0044ca10 f   renderer:win_qgl.obj
 0001:0004ba30       _logRasterPos3f@12         0044ca30 f   renderer:win_qgl.obj
 0001:0004ba50       _logRasterPos3fv@4         0044ca50 f   renderer:win_qgl.obj
 0001:0004ba70       _logRasterPos3i@12         0044ca70 f   renderer:win_qgl.obj
 0001:0004ba90       _logRasterPos3iv@4         0044ca90 f   renderer:win_qgl.obj
 0001:0004bab0       _logRasterPos3s@12         0044cab0 f   renderer:win_qgl.obj
 0001:0004bad0       _logRasterPos3sv@4         0044cad0 f   renderer:win_qgl.obj
 0001:0004baf0       _logRasterPos4d@32         0044caf0 f   renderer:win_qgl.obj
 0001:0004bb30       _logRasterPos4dv@4         0044cb30 f   renderer:win_qgl.obj
 0001:0004bb50       _logRasterPos4f@16         0044cb50 f   renderer:win_qgl.obj
 0001:0004bb70       _logRasterPos4fv@4         0044cb70 f   renderer:win_qgl.obj
 0001:0004bb90       _logRasterPos4i@16         0044cb90 f   renderer:win_qgl.obj
 0001:0004bbb0       _logRasterPos4iv@4         0044cbb0 f   renderer:win_qgl.obj
 0001:0004bbd0       _logRasterPos4s@16         0044cbd0 f   renderer:win_qgl.obj
 0001:0004bbf0       _logRasterPos4sv@4         0044cbf0 f   renderer:win_qgl.obj
 0001:0004bc10       _logReadBuffer@4           0044cc10 f   renderer:win_qgl.obj
 0001:0004bc30       _logReadPixels@28          0044cc30 f   renderer:win_qgl.obj
 0001:0004bc50       _logRectd@32               0044cc50 f   renderer:win_qgl.obj
 0001:0004bc90       _logRectdv@8               0044cc90 f   renderer:win_qgl.obj
 0001:0004bcb0       _logRectf@16               0044ccb0 f   renderer:win_qgl.obj
 0001:0004bcd0       _logRectfv@8               0044ccd0 f   renderer:win_qgl.obj
 0001:0004bcf0       _logRecti@16               0044ccf0 f   renderer:win_qgl.obj
 0001:0004bd10       _logRectiv@8               0044cd10 f   renderer:win_qgl.obj
 0001:0004bd30       _logRects@16               0044cd30 f   renderer:win_qgl.obj
 0001:0004bd50       _logRectsv@8               0044cd50 f   renderer:win_qgl.obj
 0001:0004bd70       _logRenderMode@4           0044cd70 f   renderer:win_qgl.obj
 0001:0004bd90       _logRotated@32             0044cd90 f   renderer:win_qgl.obj
 0001:0004bdd0       _logRotatef@16             0044cdd0 f   renderer:win_qgl.obj
 0001:0004bdf0       _logScaled@24              0044cdf0 f   renderer:win_qgl.obj
 0001:0004be30       _logScalef@12              0044ce30 f   renderer:win_qgl.obj
 0001:0004be50       _logScissor@16             0044ce50 f   renderer:win_qgl.obj
 0001:0004be90       _logSelectBuffer@8         0044ce90 f   renderer:win_qgl.obj
 0001:0004beb0       _logShadeModel@4           0044ceb0 f   renderer:win_qgl.obj
 0001:0004bed0       _logStencilFunc@12         0044ced0 f   renderer:win_qgl.obj
 0001:0004bef0       _logStencilMask@4          0044cef0 f   renderer:win_qgl.obj
 0001:0004bf10       _logStencilOp@12           0044cf10 f   renderer:win_qgl.obj
 0001:0004bf30       _logTexCoord1d@8           0044cf30 f   renderer:win_qgl.obj
 0001:0004bf50       _logTexCoord1dv@4          0044cf50 f   renderer:win_qgl.obj
 0001:0004bf70       _logTexCoord1f@4           0044cf70 f   renderer:win_qgl.obj
 0001:0004bf90       _logTexCoord1fv@4          0044cf90 f   renderer:win_qgl.obj
 0001:0004bfb0       _logTexCoord1i@4           0044cfb0 f   renderer:win_qgl.obj
 0001:0004bfd0       _logTexCoord1iv@4          0044cfd0 f   renderer:win_qgl.obj
 0001:0004bff0       _logTexCoord1s@4           0044cff0 f   renderer:win_qgl.obj
 0001:0004c010       _logTexCoord1sv@4          0044d010 f   renderer:win_qgl.obj
 0001:0004c030       _logTexCoord2d@16          0044d030 f   renderer:win_qgl.obj
 0001:0004c060       _logTexCoord2dv@4          0044d060 f   renderer:win_qgl.obj
 0001:0004c080       _logTexCoord2f@8           0044d080 f   renderer:win_qgl.obj
 0001:0004c0a0       _logTexCoord2fv@4          0044d0a0 f   renderer:win_qgl.obj
 0001:0004c0c0       _logTexCoord2i@8           0044d0c0 f   renderer:win_qgl.obj
 0001:0004c0e0       _logTexCoord2iv@4          0044d0e0 f   renderer:win_qgl.obj
 0001:0004c100       _logTexCoord2s@8           0044d100 f   renderer:win_qgl.obj
 0001:0004c120       _logTexCoord2sv@4          0044d120 f   renderer:win_qgl.obj
 0001:0004c140       _logTexCoord3d@24          0044d140 f   renderer:win_qgl.obj
 0001:0004c180       _logTexCoord3dv@4          0044d180 f   renderer:win_qgl.obj
 0001:0004c1a0       _logTexCoord3f@12          0044d1a0 f   renderer:win_qgl.obj
 0001:0004c1c0       _logTexCoord3fv@4          0044d1c0 f   renderer:win_qgl.obj
 0001:0004c1e0       _logTexCoord3i@12          0044d1e0 f   renderer:win_qgl.obj
 0001:0004c200       _logTexCoord3iv@4          0044d200 f   renderer:win_qgl.obj
 0001:0004c220       _logTexCoord3s@12          0044d220 f   renderer:win_qgl.obj
 0001:0004c240       _logTexCoord3sv@4          0044d240 f   renderer:win_qgl.obj
 0001:0004c260       _logTexCoord4d@32          0044d260 f   renderer:win_qgl.obj
 0001:0004c2a0       _logTexCoord4dv@4          0044d2a0 f   renderer:win_qgl.obj
 0001:0004c2c0       _logTexCoord4f@16          0044d2c0 f   renderer:win_qgl.obj
 0001:0004c2e0       _logTexCoord4fv@4          0044d2e0 f   renderer:win_qgl.obj
 0001:0004c300       _logTexCoord4i@16          0044d300 f   renderer:win_qgl.obj
 0001:0004c320       _logTexCoord4iv@4          0044d320 f   renderer:win_qgl.obj
 0001:0004c340       _logTexCoord4s@16          0044d340 f   renderer:win_qgl.obj
 0001:0004c360       _logTexCoord4sv@4          0044d360 f   renderer:win_qgl.obj
 0001:0004c380       _logTexCoordPointer@16     0044d380 f   renderer:win_qgl.obj
 0001:0004c3c0       _logTexEnvf@12             0044d3c0 f   renderer:win_qgl.obj
 0001:0004c400       _logTexEnvfv@12            0044d400 f   renderer:win_qgl.obj
 0001:0004c420       _logTexEnvi@12             0044d420 f   renderer:win_qgl.obj
 0001:0004c460       _logTexEnviv@12            0044d460 f   renderer:win_qgl.obj
 0001:0004c480       _logTexGend@16             0044d480 f   renderer:win_qgl.obj
 0001:0004c4b0       _logTexGendv@12            0044d4b0 f   renderer:win_qgl.obj
 0001:0004c4d0       _logTexGenf@12             0044d4d0 f   renderer:win_qgl.obj
 0001:0004c4f0       _logTexGenfv@12            0044d4f0 f   renderer:win_qgl.obj
 0001:0004c510       _logTexGeni@12             0044d510 f   renderer:win_qgl.obj
 0001:0004c530       _logTexGeniv@12            0044d530 f   renderer:win_qgl.obj
 0001:0004c550       _logTexImage1D@32          0044d550 f   renderer:win_qgl.obj
 0001:0004c570       _logTexImage2D@36          0044d570 f   renderer:win_qgl.obj
 0001:0004c590       _logTexParameterf@12       0044d590 f   renderer:win_qgl.obj
 0001:0004c5d0       _logTexParameterfv@12      0044d5d0 f   renderer:win_qgl.obj
 0001:0004c5f0       _logTexParameteri@12       0044d5f0 f   renderer:win_qgl.obj
 0001:0004c630       _logTexParameteriv@12      0044d630 f   renderer:win_qgl.obj
 0001:0004c650       _logTexSubImage1D@28       0044d650 f   renderer:win_qgl.obj
 0001:0004c670       _logTexSubImage2D@36       0044d670 f   renderer:win_qgl.obj
 0001:0004c690       _logTranslated@24          0044d690 f   renderer:win_qgl.obj
 0001:0004c6d0       _logTranslatef@12          0044d6d0 f   renderer:win_qgl.obj
 0001:0004c6f0       _logVertex2d@16            0044d6f0 f   renderer:win_qgl.obj
 0001:0004c720       _logVertex2dv@4            0044d720 f   renderer:win_qgl.obj
 0001:0004c740       _logVertex2f@8             0044d740 f   renderer:win_qgl.obj
 0001:0004c760       _logVertex2fv@4            0044d760 f   renderer:win_qgl.obj
 0001:0004c780       _logVertex2i@8             0044d780 f   renderer:win_qgl.obj
 0001:0004c7a0       _logVertex2iv@4            0044d7a0 f   renderer:win_qgl.obj
 0001:0004c7c0       _logVertex2s@8             0044d7c0 f   renderer:win_qgl.obj
 0001:0004c7e0       _logVertex2sv@4            0044d7e0 f   renderer:win_qgl.obj
 0001:0004c800       _logVertex3d@24            0044d800 f   renderer:win_qgl.obj
 0001:0004c840       _logVertex3dv@4            0044d840 f   renderer:win_qgl.obj
 0001:0004c860       _logVertex3f@12            0044d860 f   renderer:win_qgl.obj
 0001:0004c880       _logVertex3fv@4            0044d880 f   renderer:win_qgl.obj
 0001:0004c8a0       _logVertex3i@12            0044d8a0 f   renderer:win_qgl.obj
 0001:0004c8c0       _logVertex3iv@4            0044d8c0 f   renderer:win_qgl.obj
 0001:0004c8e0       _logVertex3s@12            0044d8e0 f   renderer:win_qgl.obj
 0001:0004c900       _logVertex3sv@4            0044d900 f   renderer:win_qgl.obj
 0001:0004c920       _logVertex4d@32            0044d920 f   renderer:win_qgl.obj
 0001:0004c960       _logVertex4dv@4            0044d960 f   renderer:win_qgl.obj
 0001:0004c980       _logVertex4f@16            0044d980 f   renderer:win_qgl.obj
 0001:0004c9a0       _logVertex4fv@4            0044d9a0 f   renderer:win_qgl.obj
 0001:0004c9c0       _logVertex4i@16            0044d9c0 f   renderer:win_qgl.obj
 0001:0004c9e0       _logVertex4iv@4            0044d9e0 f   renderer:win_qgl.obj
 0001:0004ca00       _logVertex4s@16            0044da00 f   renderer:win_qgl.obj
 0001:0004ca20       _logVertex4sv@4            0044da20 f   renderer:win_qgl.obj
 0001:0004ca40       _logVertexPointer@16       0044da40 f   renderer:win_qgl.obj
 0001:0004ca80       _logViewport@16            0044da80 f   renderer:win_qgl.obj
 0001:0004d360       _GlideIsValid              0044e360 f   renderer:win_qgl.obj
 0001:000512b0       _generateHashValue         004522b0 f   renderer:tr_image.obj
 0001:000515e0       _ResampleTexture           004525e0 f   renderer:tr_image.obj
 0001:000518e0       _R_MipMap2                 004528e0 f   renderer:tr_image.obj
 0001:00051bb0       _R_MipMap                  00452bb0 f   renderer:tr_image.obj
 0001:00051d80       _R_BlendOverTexture        00452d80 f   renderer:tr_image.obj
 0001:00051df0       _Upload32                  00452df0 f   renderer:tr_image.obj
 0001:000523c0       _LoadBMP                   004533c0 f   renderer:tr_image.obj
 0001:000526e0       _LoadPCX                   004536e0 f   renderer:tr_image.obj
 0001:000528e0       _LoadPCX32                 004538e0 f   renderer:tr_image.obj
 0001:00052980       _LoadTGA                   00453980 f   renderer:tr_image.obj
 0001:00052de0       _LoadJPG                   00453de0 f   renderer:tr_image.obj
 0001:000535f0       _R_CreateDlightImage       004545f0 f   renderer:tr_image.obj
 0001:00053790       _R_CreateFogImage          00454790 f   renderer:tr_image.obj
 0001:000538b0       _R_CreateDefaultImage      004548b0 f   renderer:tr_image.obj
 0001:00053d00       _CommaParse                00454d00 f   renderer:tr_image.obj
 0001:00055060       _RB_Hyperspace             00456060 f   renderer:tr_backend.obj
 0001:000550b0       _SetViewportAndScissor     004560b0 f   renderer:tr_backend.obj
 0001:00056210       _R_LoadMD3                 00457210 f   renderer:tr_model.obj
 0001:00056450       _R_LoadMD4                 00457450 f   renderer:tr_model.obj
 0001:000567c0       _R_GetTag                  004577c0 f   renderer:tr_model.obj
 0001:00056d70       _generateHashValue         00457d70 f   renderer:tr_shader.obj
 0001:00056dd0       _ParseVector               00457dd0 f   renderer:tr_shader.obj
 0001:00056e90       _NameToAFunc               00457e90 f   renderer:tr_shader.obj
 0001:00056f00       _NameToSrcBlendMode        00457f00 f   renderer:tr_shader.obj
 0001:00057000       _NameToDstBlendMode        00458000 f   renderer:tr_shader.obj
 0001:000570e0       _NameToGenFunc             004580e0 f   renderer:tr_shader.obj
 0001:00057190       _ParseWaveForm             00458190 f   renderer:tr_shader.obj
 0001:00057230       _ParseTexMod               00458230 f   renderer:tr_shader.obj
 0001:00057660       _ParseStage                00458660 f   renderer:tr_shader.obj
 0001:00058270       _ParseDeform               00459270 f   renderer:tr_shader.obj
 0001:00058570       _ParseSkyParms             00459570 f   renderer:tr_shader.obj
 0001:00058850       _ParseSurfaceParm          00459850 f   renderer:tr_shader.obj
 0001:000588c0       _ParseShader               004598c0 f   renderer:tr_shader.obj
 0001:00058de0       _ComputeStageIteratorFunc  00459de0 f   renderer:tr_shader.obj
 0001:00058eb0       _CollapseMultitexture      00459eb0 f   renderer:tr_shader.obj
 0001:00059080       _FixRenderCommandList      0045a080 f   renderer:tr_shader.obj
 0001:00059170       _SortNewShader             0045a170 f   renderer:tr_shader.obj
 0001:00059290       _GeneratePermanentShader   0045a290 f   renderer:tr_shader.obj
 0001:00059440       _VertexLightingCollapse    0045a440 f   renderer:tr_shader.obj
 0001:000596b0       _FinishShader              0045a6b0 f   renderer:tr_shader.obj
 0001:00059920       _FindShaderInShaderText    0045a920 f   renderer:tr_shader.obj
 0001:0005a1e0       _ScanAndLoadShaderFiles    0045b1e0 f   renderer:tr_shader.obj
 0001:0005a500       _CreateInternalShaders     0045b500 f   renderer:tr_shader.obj
 0001:0005a5a0       _CreateExternalShaders     0045b5a0 f   renderer:tr_shader.obj
 0001:0005a7f0       _GLW_ChoosePFD             0045b7f0 f   renderer:win_glimp.obj
 0001:0005aac0       _GLW_CreatePFD             0045bac0 f   renderer:win_glimp.obj
 0001:0005aba0       _GLW_MakeContext           0045bba0 f   renderer:win_glimp.obj
 0001:0005ad10       _GLW_InitDriver            0045bd10 f   renderer:win_glimp.obj
 0001:0005aef0       _GLW_CreateWindow          0045bef0 f   renderer:win_glimp.obj
 0001:0005b1b0       _PrintCDSError             0045c1b0 f   renderer:win_glimp.obj
 0001:0005b260       _GLW_SetMode               0045c260 f   renderer:win_glimp.obj
 0001:0005b6a0       _GLW_InitExtensions        0045c6a0 f   renderer:win_glimp.obj
 0001:0005b9b0       _GLW_CheckOSVersion        0045c9b0 f   renderer:win_glimp.obj
 0001:0005be20       _GLW_StartDriverAndSetMode 0045ce20 f   renderer:win_glimp.obj
 0001:0005be70       _GLW_LoadOpenGL            0045ce70 f   renderer:win_glimp.obj
 0001:0005bfb0       _GLW_StartOpenGL           0045cfb0 f   renderer:win_glimp.obj
 0001:0005c8e0       _R_CullTriSurf             0045d8e0 f   renderer:tr_world.obj
 0001:0005c900       _R_CullGrid                0045d900 f   renderer:tr_world.obj
 0001:0005c9a0       _R_CullSurface             0045d9a0 f   renderer:tr_world.obj
 0001:0005ca50       _R_DlightFace              0045da50 f   renderer:tr_world.obj
 0001:0005cc70       _R_DlightGrid              0045dc70 f   renderer:tr_world.obj
 0001:0005cf50       _R_DlightTrisurf           0045df50 f   renderer:tr_world.obj
 0001:0005cf60       _R_DlightSurface           0045df60 f   renderer:tr_world.obj
 0001:0005cfb0       _R_AddWorldSurface         0045dfb0 f   renderer:tr_world.obj
 0001:0005d0c0       _R_RecursiveWorldNode      0045e0c0 f   renderer:tr_world.obj
 0001:0005d3c0       _R_PointInLeaf             0045e3c0 f   renderer:tr_world.obj
 0001:0005d430       _R_ClusterPVS              0045e430 f   renderer:tr_world.obj
 0001:0005d4c0       _R_MarkLeaves              0045e4c0 f   renderer:tr_world.obj
 0001:0005d6c0       _HSVtoRGB                  0045e6c0 f   renderer:tr_bsp.obj
 0001:0005d7c0       _VectorLength              0045e7c0 f   renderer:tr_bsp.obj
 0001:0005d7f0       _R_ColorShiftLightingBytes 0045e7f0 f   renderer:tr_bsp.obj
 0001:0005d890       _R_LoadLightmaps           0045e890 f   renderer:tr_bsp.obj
 0001:0005dad0       _R_LoadVisibility          0045ead0 f   renderer:tr_bsp.obj
 0001:0005db60       _ShaderForShaderNum        0045eb60 f   renderer:tr_bsp.obj
 0001:0005dbe0       _ParseFace                 0045ebe0 f   renderer:tr_bsp.obj
 0001:0005de00       _ParseMesh                 0045ee00 f   renderer:tr_bsp.obj
 0001:0005e060       _ParseTriSurf              0045f060 f   renderer:tr_bsp.obj
 0001:0005e2c0       _ParseFlare                0045f2c0 f   renderer:tr_bsp.obj
 0001:0005fcf0       _R_LoadSurfaces            00460cf0 f   renderer:tr_bsp.obj
 0001:0005feb0       _R_LoadSubmodels           00460eb0 f   renderer:tr_bsp.obj
 0001:0005ff80       _R_SetParent               00460f80 f   renderer:tr_bsp.obj
 0001:0005ffb0       _R_LoadNodesAndLeafs       00460fb0 f   renderer:tr_bsp.obj
 0001:00060190       _R_LoadShaders             00461190 f   renderer:tr_bsp.obj
 0001:00060210       _R_LoadMarksurfaces        00461210 f   renderer:tr_bsp.obj
 0001:00060290       _R_LoadPlanes              00461290 f   renderer:tr_bsp.obj
 0001:000603a0       _R_LoadFogs                004613a0 f   renderer:tr_bsp.obj
 0001:000618c0       _VectorLength              004628c0 f   renderer:tr_light.obj
 0001:000619f0       _R_SetupEntityLightingGrid 004629f0 f   renderer:tr_light.obj
 0001:00061dd0       _LogLight                  00462dd0 f   renderer:tr_light.obj
 0001:000622d0       _R_ChopPolyBehindPlane     004632d0 f   renderer:tr_marks.obj
 0001:000624f0       _VectorNormalizeFast       004634f0 f   renderer:tr_marks.obj
 0001:00062530       _VectorInverse             00463530 f   renderer:tr_marks.obj
 0001:00062690       _CrossProduct              00463690 f   renderer:tr_marks.obj
 0001:00063230       _GetNoiseValue             00464230 f   renderer:tr_noise.obj
 0001:00063590       _R_ArrayElementDiscrete@4  00464590 f   renderer:tr_shade.obj
 0001:00063620       _R_DrawStripElements       00464620 f   renderer:tr_shade.obj
 0001:00063770       _VectorLength              00464770 f   renderer:tr_shade.obj
 0001:000637a0       _R_DrawElements            004647a0 f   renderer:tr_shade.obj
 0001:00063810       _R_BindAnimatedImage       00464810 f   renderer:tr_shade.obj
 0001:00063880       _DrawTris                  00464880 f   renderer:tr_shade.obj
 0001:00063960       _DrawNormals               00464960 f   renderer:tr_shade.obj
 0001:00063af0       _DrawMultitextured         00464af0 f   renderer:tr_shade.obj
 0001:00063be0       _ProjectDlightTexture      00464be0 f   renderer:tr_shade.obj
 0001:00063fc0       _RB_FogPass                00464fc0 f   renderer:tr_shade.obj
 0001:00064120       _ComputeColors             00465120 f   renderer:tr_shade.obj
 0001:00064700       _ComputeTexCoords          00465700 f   renderer:tr_shade.obj
 0001:00064930       _RB_IterateStagesGeneric   00465930 f   renderer:tr_shade.obj
 0001:00065470       _ProjectRadius             00466470 f   renderer:tr_mesh.obj
 0001:00065560       _R_CullModel               00466560 f   renderer:tr_mesh.obj
 0001:00065ed0       _VectorNormalizeFast       00466ed0 f   renderer:tr_surface.obj
 0001:00065f10       _CrossProduct              00466f10 f   renderer:tr_surface.obj
 0001:00065f70       _RB_SurfaceSprite          00466f70 f   renderer:tr_surface.obj
 0001:00066590       _DoRailCore                00467590 f   renderer:tr_surface.obj
 0001:000668f0       _DoRailDiscs               004678f0 f   renderer:tr_surface.obj
 0001:000671b0       _VectorArrayNormalize      004681b0 f   renderer:tr_surface.obj
 0001:00067210       _LerpMeshVertexes          00468210 f   renderer:tr_surface.obj
 0001:00067b00       _LodErrorForVolume         00468b00 f   renderer:tr_surface.obj
 0001:00068530       _default_decompress_parms  00469530 f   renderer:jdapimin.obj
 0001:00068950       _output_pass_setup         00469950 f   renderer:jdapistd.obj
 0001:00068ba0       _init_source               00469ba0 f   renderer:jdatasrc.obj
 0001:00068bb0       _fill_input_buffer         00469bb0 f   renderer:jdatasrc.obj
 0001:00068bf0       _skip_input_data           00469bf0 f   renderer:jdatasrc.obj
 0001:00068c60       _term_source               00469c60 f   renderer:jdatasrc.obj
 0001:00068ce0       _error_exit                00469ce0 f   renderer:jerror.obj
 0001:00068d20       _output_message            00469d20 f   renderer:jerror.obj
 0001:00068d50       _emit_message              00469d50 f   renderer:jerror.obj
 0001:00068d90       _format_message            00469d90 f   renderer:jerror.obj
 0001:00068e40       _reset_error_mgr           00469e40 f   renderer:jerror.obj
 0001:000694e0       _add_huff_table            0046a4e0 f   renderer:jcparam.obj
 0001:00069540       _std_huff_tables           0046a540 f   renderer:jcparam.obj
 0001:000699b0       _fill_a_scan               0046a9b0 f   renderer:jcparam.obj
 0001:000699e0       _fill_scans                0046a9e0 f   renderer:jcparam.obj
 0001:00069a10       _fill_dc_scans             0046aa10 f   renderer:jcparam.obj
 0001:0006a500       _VectorNormalizeFast       0046b500 f   renderer:tr_flares.obj
 0001:0006aff0       _CrossProduct              0046bff0 f   renderer:tr_shadows.obj
 0001:0006b600       _AddSkyPolygon             0046c600 f   renderer:tr_sky.obj
 0001:0006b890       _ClipSkyPolygon            0046c890 f   renderer:tr_sky.obj
 0001:0006bbd0       _CrossProduct              0046cbd0 f   renderer:tr_sky.obj
 0001:0006bc00       _ClearSkyBox               0046cc00 f   renderer:tr_sky.obj
 0001:0006be10       _MakeSkyVec                0046ce10 f   renderer:tr_sky.obj
 0001:0006bf60       _DrawSkySide               0046cf60 f   renderer:tr_sky.obj
 0001:0006c040       _DrawSkyBox                0046d040 f   renderer:tr_sky.obj
 0001:0006c310       _FillCloudySkySide         0046d310 f   renderer:tr_sky.obj
 0001:0006c530       _FillCloudBox              0046d530 f   renderer:tr_sky.obj
 0001:0006cfe0       _LerpDrawVert              0046dfe0 f   renderer:tr_curve.obj
 0001:0006d090       _VectorLength              0046e090 f   renderer:tr_curve.obj
 0001:0006d0c0       _VectorLengthSquared       0046e0c0 f   renderer:tr_curve.obj
 0001:0006d0e0       _Transpose                 0046e0e0 f   renderer:tr_curve.obj
 0001:0006d230       _CrossProduct              0046e230 f   renderer:tr_curve.obj
 0001:0006d260       _MakeMeshNormals           0046e260 f   renderer:tr_curve.obj
 0001:0006d910       _InvertCtrl                0046e910 f   renderer:tr_curve.obj
 0001:0006d9b0       _InvertErrorTable          0046e9b0 f   renderer:tr_curve.obj
 0001:0006da90       _PutPointsOnCurve          0046ea90 f   renderer:tr_curve.obj
 0001:0006e8d0       _TableForFunc              0046f8d0 f   renderer:tr_shade_calc.obj
 0001:0006e930       _VectorLength              0046f930 f   renderer:tr_shade_calc.obj
 0001:0006e960       _VectorNormalizeFast       0046f960 f   renderer:tr_shade_calc.obj
 0001:0006e9a0       _CrossProduct              0046f9a0 f   renderer:tr_shade_calc.obj
 0001:0006ef40       _GlobalVectorToLocal       0046ff40 f   renderer:tr_shade_calc.obj
 0001:0006efb0       _AutospriteDeform          0046ffb0 f   renderer:tr_shade_calc.obj
 0001:0006f240       _Autosprite2Deform         00470240 f   renderer:tr_shade_calc.obj
 0001:00070230       _EvalWaveForm              00471230 f   renderer:tr_shade_calc.obj
 0001:00070270       _EvalWaveFormClamped       00471270 f   renderer:tr_shade_calc.obj
 0001:000709b0       _initial_setup             004719b0 f   renderer:jdinput.obj
 0001:00070ba0       _per_scan_setup            00471ba0 f   renderer:jdinput.obj
 0001:00070d40       _latch_quant_tables        00471d40 f   renderer:jdinput.obj
 0001:00070df0       _start_input_pass          00471df0 f   renderer:jdinput.obj
 0001:00070e30       _consume_markers           00471e30 f   renderer:jdinput.obj
 0001:00070ef0       _reset_input_controller    00471ef0 f   renderer:jdinput.obj
 0001:00070f30       _finish_input_pass         00471f30 f   renderer:jdinput.obj
 0001:00070fa0       _get_soi                   00471fa0 f   renderer:jdmarker.obj
 0001:00071040       _get_sof                   00472040 f   renderer:jdmarker.obj
 0001:00071350       _get_sos                   00472350 f   renderer:jdmarker.obj
 0001:00071640       _get_app0                  00472640 f   renderer:jdmarker.obj
 0001:000718b0       _get_app14                 004728b0 f   renderer:jdmarker.obj
 0001:00071a40       _get_dac                   00472a40 f   renderer:jdmarker.obj
 0001:00071ba0       _get_dht                   00472ba0 f   renderer:jdmarker.obj
 0001:00071ea0       _get_dqt                   00472ea0 f   renderer:jdmarker.obj
 0001:000720e0       _get_dri                   004730e0 f   renderer:jdmarker.obj
 0001:000721c0       _skip_variable             004731c0 f   renderer:jdmarker.obj
 0001:00072260       _next_marker               00473260 f   renderer:jdmarker.obj
 0001:00072360       _first_marker              00473360 f   renderer:jdmarker.obj
 0001:00072400       _read_markers              00473400 f   renderer:jdmarker.obj
 0001:00072790       _read_restart_marker       00473790 f   renderer:jdmarker.obj
 0001:00072920       _reset_marker_reader       00473920 f   renderer:jdmarker.obj
 0001:00072a10       _out_of_memory             00473a10 f   renderer:jmemmgr.obj
 0001:00072a30       _alloc_small               00473a30 f   renderer:jmemmgr.obj
 0001:00072b80       _alloc_large               00473b80 f   renderer:jmemmgr.obj
 0001:00072c40       _alloc_sarray              00473c40 f   renderer:jmemmgr.obj
 0001:00072cf0       _alloc_barray              00473cf0 f   renderer:jmemmgr.obj
 0001:00072da0       _request_virt_sarray       00473da0 f   renderer:jmemmgr.obj
 0001:00072e10       _request_virt_barray       00473e10 f   renderer:jmemmgr.obj
 0001:00072e80       _realize_virt_arrays       00473e80 f   renderer:jmemmgr.obj
 0001:00073020       _do_sarray_io              00474020 f   renderer:jmemmgr.obj
 0001:000730c0       _do_barray_io              004740c0 f   renderer:jmemmgr.obj
 0001:00073160       _access_virt_sarray        00474160 f   renderer:jmemmgr.obj
 0001:000732a0       _access_virt_barray        004742a0 f   renderer:jmemmgr.obj
 0001:000733f0       _free_pool                 004743f0 f   renderer:jmemmgr.obj
 0001:00073500       _self_destruct             00474500 f   renderer:jmemmgr.obj
 0001:000736f0       _use_merged_upsample       004746f0 f   renderer:jdmaster.obj
 0001:00073790       _prepare_range_limit_table 00474790 f   renderer:jdmaster.obj
 0001:00073810       _master_selection          00474810 f   renderer:jdmaster.obj
 0001:00073990       _prepare_for_output_pass   00474990 f   renderer:jdmaster.obj
 0001:00073ad0       _finish_output_pass        00474ad0 f   renderer:jdmaster.obj
 0001:00073b30       _emit_byte                 00474b30 f   renderer:jcmarker.obj
 0001:00073b70       _emit_marker               00474b70 f   renderer:jcmarker.obj
 0001:00073be0       _emit_2bytes               00474be0 f   renderer:jcmarker.obj
 0001:00073c50       _emit_dqt                  00474c50 f   renderer:jcmarker.obj
 0001:00073dc0       _emit_dht                  00474dc0 f   renderer:jcmarker.obj
 0001:00073f20       _emit_dac                  00474f20 f   renderer:jcmarker.obj
 0001:00073f30       _emit_dri                  00474f30 f   renderer:jcmarker.obj
 0001:00073f60       _emit_sof                  00474f60 f   renderer:jcmarker.obj
 0001:000740e0       _emit_sos                  004750e0 f   renderer:jcmarker.obj
 0001:000742c0       _emit_jfif_app0            004752c0 f   renderer:jcmarker.obj
 0001:000744d0       _emit_adobe_app14          004754d0 f   renderer:jcmarker.obj
 0001:00074640       _write_any_marker          00475640 f   renderer:jcmarker.obj
 0001:000746b0       _write_file_header         004756b0 f   renderer:jcmarker.obj
 0001:000746f0       _write_frame_header        004756f0 f   renderer:jcmarker.obj
 0001:000747d0       _write_scan_header         004757d0 f   renderer:jcmarker.obj
 0001:000748b0       _write_file_trailer        004758b0 f   renderer:jcmarker.obj
 0001:000748d0       _write_tables_only         004758d0 f   renderer:jcmarker.obj
 0001:00074a20       _process_data_simple_main  00475a20 f   renderer:jcmainct.obj
 0001:00074ad0       _start_pass_main           00475ad0 f   renderer:jcmainct.obj
 0001:00074bb0       _start_iMCU_row            00475bb0 f   renderer:jccoefct.obj
 0001:00074c00       _compress_data             00475c00 f   renderer:jccoefct.obj
 0001:00074ec0       _compress_output           00475ec0 f   renderer:jccoefct.obj
 0001:000750d0       _compress_first_pass       004760d0 f   renderer:jccoefct.obj
 0001:000752f0       _start_pass_coef           004762f0 f   renderer:jccoefct.obj
 0001:00075600       _dump_buffer               00476600 f   renderer:jchuff.obj
 0001:00075630       _emit_bits                 00476630 f   renderer:jchuff.obj
 0001:00075720       _flush_bits                00476720 f   renderer:jchuff.obj
 0001:00075750       _encode_one_block          00476750 f   renderer:jchuff.obj
 0001:000758a0       _emit_restart              004768a0 f   renderer:jchuff.obj
 0001:00075970       _encode_mcu_huff           00476970 f   renderer:jchuff.obj
 0001:00075af0       _finish_pass_huff          00476af0 f   renderer:jchuff.obj
 0001:00075bc0       _htest_one_block           00476bc0 f   renderer:jchuff.obj
 0001:00075c70       _encode_mcu_gather         00476c70 f   renderer:jchuff.obj
 0001:00075fa0       _finish_pass_gather        00476fa0 f   renderer:jchuff.obj
 0001:00076090       _start_pass_huff           00477090 f   renderer:jchuff.obj
 0001:00076290       _dump_buffer               00477290 f   renderer:jcphuff.obj
 0001:000762d0       _emit_bits                 004772d0 f   renderer:jcphuff.obj
 0001:00076410       _flush_bits                00477410 f   renderer:jcphuff.obj
 0001:00076430       _emit_symbol               00477430 f   renderer:jcphuff.obj
 0001:00076470       _emit_buffered_bits        00477470 f   renderer:jcphuff.obj
 0001:000764a0       _emit_eobrun               004774a0 f   renderer:jcphuff.obj
 0001:00076520       _emit_restart              00477520 f   renderer:jcphuff.obj
 0001:00076630       _encode_mcu_DC_first       00477630 f   renderer:jcphuff.obj
 0001:00076790       _encode_mcu_AC_first       00477790 f   renderer:jcphuff.obj
 0001:00076970       _encode_mcu_DC_refine      00477970 f   renderer:jcphuff.obj
 0001:00076a40       _encode_mcu_AC_refine      00477a40 f   renderer:jcphuff.obj
 0001:00076cd0       _finish_pass_phuff         00477cd0 f   renderer:jcphuff.obj
 0001:00076d20       _finish_pass_gather_phuff  00477d20 f   renderer:jcphuff.obj
 0001:00076e00       _start_pass_phuff          00477e00 f   renderer:jcphuff.obj
 0001:00077000       _start_pass_fdctmgr        00478000 f   renderer:jcdctmgr.obj
 0001:00077220       _forward_DCT_float         00478220 f   renderer:jcdctmgr.obj
 0001:00077980       _start_pass_prep           00478980 f   renderer:jcprepct.obj
 0001:000779d0       _expand_bottom_edge        004789d0 f   renderer:jcprepct.obj
 0001:00077a00       _pre_process_data          00478a00 f   renderer:jcprepct.obj
 0001:00077c10       _pre_process_context       00478c10 f   renderer:jcprepct.obj
 0001:00077ef0       _create_context_buffer     00478ef0 f   renderer:jcprepct.obj
 0001:000780f0       _start_pass_downsample     004790f0 f   renderer:jcsample.obj
 0001:00078100       _expand_right_edge         00479100 f   renderer:jcsample.obj
 0001:00078160       _sep_downsample            00479160 f   renderer:jcsample.obj
 0001:000781f0       _int_downsample            004791f0 f   renderer:jcsample.obj
 0001:00078320       _fullsize_downsample       00479320 f   renderer:jcsample.obj
 0001:00078370       _h2v1_downsample           00479370 f   renderer:jcsample.obj
 0001:00078410       _h2v2_downsample           00479410 f   renderer:jcsample.obj
 0001:000784f0       _h2v2_smooth_downsample    004794f0 f   renderer:jcsample.obj
 0001:00078780       _fullsize_smooth_downsample 00479780 f   renderer:jcsample.obj
 0001:00078a80       _rgb_ycc_start             00479a80 f   renderer:jccolor.obj
 0001:00078b60       _rgb_ycc_convert           00479b60 f   renderer:jccolor.obj
 0001:00078c80       _rgb_gray_convert          00479c80 f   renderer:jccolor.obj
 0001:00078d30       _cmyk_ycck_convert         00479d30 f   renderer:jccolor.obj
 0001:00078e90       _grayscale_convert         00479e90 f   renderer:jccolor.obj
 0001:00078f00       _null_convert              00479f00 f   renderer:jccolor.obj
 0001:00078f90       _null_method               00479f90 f   renderer:jccolor.obj
 0001:000791e0       _initial_setup             0047a1e0 f   renderer:jcmaster.obj
 0001:000793b0       _validate_script           0047a3b0 f   renderer:jcmaster.obj
 0001:00079780       _select_scan_parameters    0047a780 f   renderer:jcmaster.obj
 0001:00079870       _per_scan_setup            0047a870 f   renderer:jcmaster.obj
 0001:00079a40       _prepare_for_pass          0047aa40 f   renderer:jcmaster.obj
 0001:00079bd0       _pass_startup              0047abd0 f   renderer:jcmaster.obj
 0001:00079c00       _finish_pass_master        0047ac00 f   renderer:jcmaster.obj
 0001:00079e90       _alloc_funny_pointers      0047ae90 f   renderer:jdmainct.obj
 0001:00079f40       _make_funny_pointers       0047af40 f   renderer:jdmainct.obj
 0001:0007a090       _set_wraparound_pointers   0047b090 f   renderer:jdmainct.obj
 0001:0007a170       _set_bottom_pointers       0047b170 f   renderer:jdmainct.obj
 0001:0007a210       _process_data_simple_main  0047b210 f   renderer:jdmainct.obj
 0001:0007a280       _process_data_context_main 0047b280 f   renderer:jdmainct.obj
 0001:0007a3c0       _start_pass_main           0047b3c0 f   renderer:jdmainct.obj
 0001:0007a500       _start_iMCU_row            0047b500 f   renderer:jdcoefct.obj
 0001:0007a550       _start_input_pass          0047b550 f   renderer:jdcoefct.obj
 0001:0007a570       _start_output_pass         0047b570 f   renderer:jdcoefct.obj
 0001:0007a580       _decompress_onepass        0047b580 f   renderer:jdcoefct.obj
 0001:0007a820       _dummy_consume_data        0047b820 f   renderer:jdcoefct.obj
 0001:0007acd0       _process_restart           0047bcd0 f   renderer:jdhuff.obj
 0001:0007ad50       _decode_mcu                0047bd50 f   renderer:jdhuff.obj
 0001:0007b190       _start_pass_huff_decoder   0047c190 f   renderer:jdhuff.obj
 0001:0007b330       _start_pass                0047c330 f   renderer:jddctmgr.obj
 0001:0007b5d0       _post_process_1pass        0047c5d0 f   renderer:jdpostct.obj
 0001:0007b650       _start_pass_dpost          0047c650 f   renderer:jdpostct.obj
 0001:0007b740       _start_pass_upsample       0047c740 f   renderer:jdsample.obj
 0001:0007b760       _sep_upsample              0047c760 f   renderer:jdsample.obj
 0001:0007b840       _fullsize_upsample         0047c840 f   renderer:jdsample.obj
 0001:0007b850       _noop_upsample             0047c850 f   renderer:jdsample.obj
 0001:0007b860       _int_upsample              0047c860 f   renderer:jdsample.obj
 0001:0007b960       _h2v1_upsample             0047c960 f   renderer:jdsample.obj
 0001:0007b9c0       _h2v2_upsample             0047c9c0 f   renderer:jdsample.obj
 0001:0007ba40       _h2v1_fancy_upsample       0047ca40 f   renderer:jdsample.obj
 0001:0007bb00       _h2v2_fancy_upsample       0047cb00 f   renderer:jdsample.obj
 0001:0007be20       _build_ycc_rgb_table       0047ce20 f   renderer:jdcolor.obj
 0001:0007bef0       _ycc_rgb_convert           0047cef0 f   renderer:jdcolor.obj
 0001:0007c010       _null_convert              0047d010 f   renderer:jdcolor.obj
 0001:0007c090       _grayscale_convert         0047d090 f   renderer:jdcolor.obj
 0001:0007c0c0       _ycck_cmyk_convert         0047d0c0 f   renderer:jdcolor.obj
 0001:0007c210       _start_pass_dcolor         0047d210 f   renderer:jdcolor.obj
 0001:0007dcd0       _Init_AAS_Export           0047ecd0 f   botlib:be_interface.obj
 0001:0007dd70       _Init_EA_Export            0047ed70 f   botlib:be_interface.obj
 0001:0007de20       _Init_AI_Export            0047ee20 f   botlib:be_interface.obj
 0001:0007e3a0       _VectorLength              0047f3a0 f   botlib:be_ai_move.obj
 0001:0007e3d0       _VectorLengthSquared       0047f3d0 f   botlib:be_ai_move.obj
 0001:00088d70       _VectorLength              00489d70 f   botlib:be_ai_goal.obj
 0001:00093010       _VectorCompare             00494010 f   botlib:be_aas_entity.obj
 0001:00093050       _VectorLength              00494050 f   botlib:be_aas_entity.obj
 0001:00093c40       _VectorCompare             00494c40 f   botlib:be_aas_move.obj
 0001:00093c80       _VectorLength              00494c80 f   botlib:be_aas_move.obj
 0001:00095900       _VectorLength              00496900 f   botlib:be_aas_routealt.obj
 0001:00095ff0       _VectorLength              00496ff0 f   botlib:be_aas_route.obj
 0001:00098c70       _VectorLength              00499c70 f   botlib:be_aas_reach.obj
 0001:00098fe0       _VectorInverse             00499fe0 f   botlib:be_aas_reach.obj
 0001:00099000       _CrossProduct              0049a000 f   botlib:be_aas_reach.obj
 0001:000a2d90       _VectorLength              004a3d90 f   botlib:be_aas_sample.obj
 0001:000a2f20       _VectorInverse             004a3f20 f   botlib:be_aas_sample.obj
 0001:000a2f40       _CrossProduct              004a3f40 f   botlib:be_aas_sample.obj
 0001:000a9910       _CrossProduct              004aa910 f   botlib:be_aas_debug.obj
 0001:000ab6e0       _$$$00001                  004ac6e0 f   LIBC:strchr.obj
 0001:000ab86b       _store_dt                  004ac86b f   LIBC:asctime.obj
 0001:000abc9c       $$$00001                   004acc9c f   LIBC:longjmp.obj
 0001:000abd15       $$$00003                   004acd15 f   LIBC:longjmp.obj
 0001:000abedf       $$$00002                   004acedf f   LIBC:setjmp3.obj
 0001:000ac59b       _flsall                    004ad59b f   LIBC:fflush.obj
 0001:000ac620       _swap                      004ad620 f   LIBC:qsort.obj
 0001:000ac640       _shortsort                 004ad640 f   LIBC:qsort.obj
 0001:000aca5a       __initterm                 004ada5a f   LIBC:crt0dat.obj
 0001:000aca72       __initterm_e               004ada72 f   LIBC:crt0dat.obj
 0001:000acafa       _doexit                    004adafa f   LIBC:crt0dat.obj
 0001:000ad05c       _fast_error_exit           004ae05c f   LIBC:wincrt0.obj
 0001:000ad080       _check_managed_app         004ae080 f   LIBC:wincrt0.obj
 0001:000ad2ff       _$$$00002                  004ae2ff f   LIBC:pow.obj
 0001:000ad803       __shift                    004ae803 f   LIBC:cvt.obj
 0001:000ad911       __cftoe_g                  004ae911 f   LIBC:cvt.obj
 0001:000ada15       __cftof_g                  004aea15 f   LIBC:cvt.obj
 0001:000adf00       _has_osfxsr_set            004aef00 f   LIBC:cpu_disp.obj
 0001:000ae228       _strncnt                   004af228 f   LIBC:a_map.obj
 0001:000ae911       _write_char                004af911 f   LIBC:output.obj
 0001:000ae944       _write_multi_char          004af944 f   LIBC:output.obj
 0001:000ae968       _write_string              004af968 f   LIBC:output.obj
 0001:000ae99f       _get_int_arg               004af99f f   LIBC:output.obj
 0001:000ae9a8       _get_int64_arg             004af9a8 f   LIBC:output.obj
 0001:000ae9b4       _get_short_arg             004af9b4 f   LIBC:output.obj
 0001:000af33c       __hextodec                 004b033c f   LIBC:input.obj
 0001:000af36e       __inc                      004b036e f   LIBC:input.obj
 0001:000af384       __un_inc                   004b0384 f   LIBC:input.obj
 0001:000af391       __whiteout                 004b0391 f   LIBC:input.obj
 0001:000b0468       _cvtdate                   004b1468 f   LIBC:tzset.obj
 0001:000b09b3       _$$$00003                  004b19b3 f   LIBC:87disp.obj
 0001:000b0c7c       $$$00001                   004b1c7c f   LIBC:exsup.obj
 0001:000b0c9c       $$$00003                   004b1c9c f   LIBC:exsup.obj
 0001:000b0c9c       __unwind_handler           004b1c9c f   LIBC:exsup.obj
 0001:000b0cbe       $$$00005                   004b1cbe f   LIBC:exsup.obj
 0001:000b0d26       $$$00007                   004b1d26 f   LIBC:exsup.obj
 0001:000b0d6a       $$$00011                   004b1d6a f   LIBC:exsup.obj
 0001:000b3158       _report_failure            004b4158 f   LIBC:secchk.obj
 0001:000b347f       _xcptlookup                004b447f f   LIBC:winxfltr.obj
 0001:000b3766       _parse_cmdline             004b4766 f   LIBC:stdargv.obj
 0001:000b3bed       $$$00003                   004b4bed f   LIBC:exsup3.obj
 0001:000b4740       _$$$00001                  004b5740 f   LIBC:87tran.obj
 0001:000b4b17       _wfindenv                  004b5b17 f   LIBC:wsetenv.obj
 0001:000b4b68       _copy_environ              004b5b68 f   LIBC:wsetenv.obj
 0001:000b4e95       _findenv                   004b5e95 f   LIBC:setenv.obj
 0001:000b4ee2       _copy_environ              004b5ee2 f   LIBC:setenv.obj
 0001:000b5754       __abstract_cw              004b6754 f   LIBC:ieee87.obj
 0001:000b57e6       __hw_cw                    004b67e6 f   LIBC:ieee87.obj
 0001:000b5874       __abstract_sw              004b6874 f   LIBC:ieee87.obj
 0001:000b5ad0       _getSystemCP               004b6ad0 f   LIBC:mbctype.obj
 0001:000b5b16       _CPtoLCID                  004b6b16 f   LIBC:mbctype.obj
 0001:000b5b45       _setSBCS                   004b6b45 f   LIBC:mbctype.obj
 0001:000b5b6e       _setSBUpLow                004b6b6e f   LIBC:mbctype.obj
 0001:000b6400       __get_fname                004b7400 f   LIBC:fpexcept.obj
 0001:000b6c54       _strncnt                   004b7c54 f   LIBC:a_cmp.obj
 0001:000b83a6       _x_ismbbtype               004b93a6 f   LIBC:ismbbyte.obj
 0001:000ba5e3       _wcsncnt                   004bb5e3 f   LIBC:w_cmp.obj
